 orf_marker

 Timestamp is 5c762284 (Wed Feb 27 12:39:16 2019)

 Preferred load address is 10000000

 Start         Length     Name                   Class
 0001:00000000 00003c24H .text$di                CODE
 0001:00003c30 0001b83eH .text$mn                CODE
 0001:0001f470 00004734H .text$x                 CODE
 0001:00023bb0 00000e6aH .text$yd                CODE
 0002:00000000 00001070H .idata$5                DATA
 0002:00001070 00000004H .CRT$XCA                DATA
 0002:00001074 00000338H .CRT$XCU                DATA
 0002:000013ac 00000004H .CRT$XCZ                DATA
 0002:000013b0 00000004H .CRT$XIA                DATA
 0002:000013b4 00000004H .CRT$XIAA               DATA
 0002:000013b8 00000004H .CRT$XIC                DATA
 0002:000013bc 00000004H .CRT$XIZ                DATA
 0002:000013c0 00004698H .rdata                  DATA
 0002:00005a58 00000070H .rdata$debug            DATA
 0002:00005ac8 00001f10H .rdata$r                DATA
 0002:000079e0 000003b8H .rdata$sxdata           DATA
 0002:00007d98 00000004H .rtc$IAA                DATA
 0002:00007d9c 00000004H .rtc$IZZ                DATA
 0002:00007da0 00000004H .rtc$TAA                DATA
 0002:00007da4 00000004H .rtc$TZZ                DATA
 0002:00007da8 00005164H .xdata$x                DATA
 0002:0000cf10 00000053H .edata                  DATA
 0002:0000cf64 0000012cH .idata$2                DATA
 0002:0000d090 00000014H .idata$3                DATA
 0002:0000d0a4 00001070H .idata$4                DATA
 0002:0000e114 0000d006H .idata$6                DATA
 0003:00000000 00000304H .data                   DATA
 0003:00000308 00000d64H .data$r                 DATA
 0003:00001070 0000071cH .bss                    DATA
 0004:00000000 00000058H .rsrc$01                DATA
 0004:00000060 00000180H .rsrc$02                DATA

  Address         Publics by Value              Rva+Base       Lib:Object

 0000:00000000       ___guard_fids_count        00000000     <absolute>
 0000:00000000       ___guard_flags             00000000     <absolute>
 0000:00000000       ___guard_fids_table        00000000     <absolute>
 0000:00000000       __except_list              00000000     <absolute>
 0000:000000ee       ___safe_se_handler_count   000000ee     <absolute>
 0000:00009876       __ldused                   00009876     <absolute>
 0000:00009876       __fltused                  00009876     <absolute>
 0000:00000000       ___ImageBase               10000000     <linker-defined>
 0001:00003c30       ??$_Allocate@D@std@@YAPADIPAD@Z 10004c30 f i ORFDialog.obj
 0001:00003c60       ??$_Move@AAPAUData@QListData@@@std@@YA$$QAPAUData@QListData@@AAPAU12@@Z 10004c60 f i ORFDialog.obj
 0001:00003c70       ??$acquireMemoryFence@H@?$QGenericAtomicOps@U?$QAtomicOpsBySize@$03@@@@SAXABH@Z 10004c70 f i ORFDialog.obj
 0001:00003c80       ??$addressof@D@std@@YAPADAAD@Z 10004c80 f i ORFDialog.obj
 0001:00003c90       ??$atomic@H@?$QAtomicOpsBySize@$03@@CAPAJPAH@Z 10004c90 f i ORFDialog.obj
 0001:00003ca0       ??$construct@PADAAPAD@?$_Wrap_alloc@V?$allocator@D@std@@@std@@QAEXPAPADAAPAD@Z 10004ca0 f i ORFDialog.obj
 0001:00003cc0       ??$construct@PADAAPAD@?$allocator@D@std@@QAEXPAPADAAPAD@Z 10004cc0 f i ORFDialog.obj
 0001:00003ce0       ??$construct@PADAAPAD@?$allocator_traits@V?$allocator@D@std@@@std@@SAXAAV?$allocator@D@1@PAPADAAPAD@Z 10004ce0 f i ORFDialog.obj
 0001:00003d00       ??$deref@H@?$QAtomicOpsBySize@$03@@SA_NAAH@Z 10004d00 f i ORFDialog.obj
 0001:00003d20       ??$destroy@PAD@?$_Wrap_alloc@V?$allocator@D@std@@@std@@QAEXPAPAD@Z 10004d20 f i ORFDialog.obj
 0001:00003d30       ??$destroy@PAD@?$allocator@D@std@@QAEXPAPAD@Z 10004d30 f i ORFDialog.obj
 0001:00003d40       ??$destroy@PAD@?$allocator_traits@V?$allocator@D@std@@@std@@SAXAAV?$allocator@D@1@PAPAD@Z 10004d40 f i ORFDialog.obj
 0001:00003d50       ??$forward@AAPAD@std@@YAAAPADAAPAD@Z 10004d50 f i ORFDialog.obj
 0001:00003d60       ??$load@H@?$QGenericAtomicOps@U?$QAtomicOpsBySize@$03@@@@SAHABH@Z 10004d60 f i ORFDialog.obj
 0001:00003d70       ??$loadAcquire@H@?$QGenericAtomicOps@U?$QAtomicOpsBySize@$03@@@@SAHABH@Z 10004d70 f i ORFDialog.obj
 0001:00003d80       ??$orderedMemoryFence@H@?$QGenericAtomicOps@U?$QAtomicOpsBySize@$03@@@@SAXABH@Z 10004d80 f i ORFDialog.obj
 0001:00003d90       ??$qMapLessThanKey@W4DNATranslationRole@U2@@@@YA_NABW4DNATranslationRole@U2@@0@Z 10004d90 f i ORFDialog.obj
 0001:00003db0       ??$qMetaTypeId@PAVQAction@@@@YAHXZ 10004db0 f i ORFDialog.obj
 0001:00003dc0       ??$qRegisterMetaType@PAVQAction@@@@YAHPBDPAPAVQAction@@W4DefinedType@?$MetaTypeDefinedHelper@PAVQAction@@$00@QtPrivate@@@Z 10004dc0 f i ORFDialog.obj
 0001:00003e80       ??$qRegisterNormalizedMetaType@PAVQAction@@@@YAHABVQByteArray@@PAPAVQAction@@W4DefinedType@?$MetaTypeDefinedHelper@PAVQAction@@$00@QtPrivate@@@Z 10004e80 f i ORFDialog.obj
 0001:00003ee0       ??$qSwap@PAUData@QListData@@@@YAXAAPAUData@QListData@@0@Z 10004ee0 f i ORFDialog.obj
 0001:00003f00       ??$qVariantFromValue@PAVQAction@@@@YA?AVQVariant@@ABQAVQAction@@@Z 10004f00 f i ORFDialog.obj
 0001:00003f30       ??$qobject_cast@PAVAutoAnnotationsUpdateTask@U2@@@@YAPAVAutoAnnotationsUpdateTask@U2@@PAVQObject@@@Z 10004f30 f i ORFDialog.obj
 0001:00003f50       ??$qobject_cast@PAVQAction@@@@YAPAVQAction@@PAVQObject@@@Z 10004f50 f i ORFDialog.obj
 0001:00003f70       ??$qvariant_cast@PAVQAction@@@@YAPAVQAction@@ABVQVariant@@@Z 10004f70 f i ORFDialog.obj
 0001:00003f80       ??$ref@H@?$QAtomicOpsBySize@$03@@SA_NAAH@Z 10004f80 f i ORFDialog.obj
 0001:00003fa0       ??$releaseMemoryFence@H@?$QGenericAtomicOps@U?$QAtomicOpsBySize@$03@@@@SAXABH@Z 10004fa0 f i ORFDialog.obj
 0001:00003fb0       ??$storeRelease@HH@?$QGenericAtomicOps@U?$QAtomicOpsBySize@$03@@@@SAXAAHH@Z 10004fb0 f i ORFDialog.obj
 0001:00003fc0       ??$swap@PAUData@QListData@@@std@@YAXAAPAUData@QListData@@0@Z 10004fc0 f i ORFDialog.obj
 0001:00003fe0       ??$value@PAVQAction@@@QVariant@@QBEPAVQAction@@XZ 10004fe0 f i ORFDialog.obj
 0001:00003ff0       ??0?$AbstractId@H@U2@@IAE@ABH@Z 10004ff0 f i ORFDialog.obj
 0001:00004010       ??0?$QFlags@W4AlignmentFlag@Qt@@@@QAE@PQPrivate@0@H@Z 10005010 f i ORFDialog.obj
 0001:00004020       ??0?$QFlags@W4StandardButton@QDialogButtonBox@@@@QAE@VQFlag@@@Z 10005020 f i ORFDialog.obj
 0001:00004030       ??0?$QFlags@W4StandardButton@QDialogButtonBox@@@@QAE@W4StandardButton@QDialogButtonBox@@@Z 10005030 f i ORFDialog.obj
 0001:00004040       ??0?$QFlags@W4StandardButton@QMessageBox@@@@QAE@W4StandardButton@QMessageBox@@@Z 10005040 f i ORFDialog.obj
 0001:00004050       ??0?$QFlags@W4TypeFlag@QMetaType@@@@QAE@VQFlag@@@Z 10005050 f i ORFDialog.obj
 0001:00004060       ??0?$QFlags@W4WindowType@Qt@@@@QAE@PQPrivate@0@H@Z 10005060 f i ORFDialog.obj
 0001:00004070       ??0?$QForeachContainer@$$CBV?$QList@PAVTask@U2@@@@@@QAE@ABV?$QList@PAVTask@U2@@@@@Z 10005070 f i ORFDialog.obj
 0001:000040b0       ??0?$QForeachContainer@V?$QList@PAVQAction@@@@@@QAE@ABV?$QList@PAVQAction@@@@@Z 100050b0 f i ORFDialog.obj
 0001:000040f0       ??0?$QForeachContainer@V?$QList@VORFFindResult@U2@@@@@@QAE@ABV?$QList@VORFFindResult@U2@@@@@Z 100050f0 f i ORFDialog.obj
 0001:00004130       ??0?$QList@PAVQAction@@@@QAE@ABV0@@Z 10005130 f i ORFDialog.obj
 0001:000041f0       ??0?$QList@PAVTask@U2@@@@QAE@ABV0@@Z 100051f0 f i ORFDialog.obj
 0001:000042b0       ??0?$QList@URegionPreset@U2@@@@QAE@XZ 100052b0 f i ORFDialog.obj
 0001:000042c0       ??0?$QList@UTriplet@U2@@@@QAE@ABV0@@Z 100052c0 f i ORFDialog.obj
 0001:00004380       ??0?$QList@UTriplet@U2@@@@QAE@XZ 10005380 f i ORFDialog.obj
 0001:00004390       ??0?$QList@VORFFindResult@U2@@@@QAE@ABV0@@Z 10005390 f i ORFDialog.obj
 0001:00004450       ??0?$QMap@W4DNATranslationRole@U2@@V?$QList@UTriplet@U2@@@@@@QAE@ABV0@@Z 10005450 f i ORFDialog.obj
 0001:000044c0       ??0?$_String_alloc@$0A@U?$_String_base_types@DV?$allocator@D@std@@@std@@@std@@QAE@ABV?$allocator@D@1@@Z 100054c0 f i ORFDialog.obj
 0001:000044e0       ??0?$_String_val@U?$_Simple_types@D@std@@@std@@QAE@XZ 100054e0 f i ORFDialog.obj
 0001:00004500       ??0?$_Wrap_alloc@V?$allocator@D@std@@@std@@QAE@XZ 10005500 f i ORFDialog.obj
 0001:00004510       ??0?$allocator@D@std@@QAE@XZ 10005510 f i ORFDialog.obj
 0001:00004520       ??0?$basic_string@DU?$char_traits@D@std@@V?$allocator@D@2@@std@@QAE@PBD@Z 10005520 f i ORFDialog.obj
 0001:00004580       ??0AbstractInt32Id@U2@@IAE@H@Z 10005580 f i ORFDialog.obj
 0001:000045a0       ??0ORFDialog@U2@@QAE@PAVADVSequenceObjectContext@1@@Z 100055a0 f   ORFDialog.obj
 0001:00004a70       ??0ORFListItem@U2@@QAE@ABVORFFindResult@1@@Z 10005a70 f   ORFDialog.obj
 0001:00004e30       ??0QFlag@@QAE@H@Z          10005e30 f i ORFDialog.obj
 0001:00004e40       ??0QLatin1Char@@QAE@D@Z    10005e40 f i ORFDialog.obj
 0001:00004e50       ??0ServiceType@U2@@QAE@H@Z 10005e50 f i ORFDialog.obj
 0001:00004e70       ??0_Generic_error_category@std@@QAE@XZ 10005e70 f i ORFDialog.obj
 0001:00004e80       ??0_Ignore@std@@QAE@XZ     10005e80 f i ORFDialog.obj
 0001:00004e90       ??0_Iostream_error_category@std@@QAE@XZ 10005e90 f i ORFDialog.obj
 0001:00004ea0       ??0_System_error_category@std@@QAE@XZ 10005ea0 f i ORFDialog.obj
 0001:00004eb0       ??0const_iterator@?$QList@PAVQAction@@@@QAE@PAUNode@1@@Z 10005eb0 f i ORFDialog.obj
 0001:00004ec0       ??0const_iterator@?$QList@PAVTask@U2@@@@QAE@PAUNode@1@@Z 10005ec0 f i ORFDialog.obj
 0001:00004ed0       ??0const_iterator@?$QList@VORFFindResult@U2@@@@QAE@PAUNode@1@@Z 10005ed0 f i ORFDialog.obj
 0001:00004ee0       ??0error_category@std@@QAE@XZ 10005ee0 f i ORFDialog.obj
 0001:00004ef0       ??0error_condition@std@@QAE@HABVerror_category@1@@Z 10005ef0 f i ORFDialog.obj
 0001:00004f10       ??0iterator@?$QMap@W4DNATranslationRole@U2@@V?$QList@UTriplet@U2@@@@@@QAE@PAU?$QMapNode@W4DNATranslationRole@U2@@V?$QList@UTriplet@U2@@@@@@@Z 10005f10 f i ORFDialog.obj
 0001:00004f20       ??1?$AbstractId@H@U2@@MAE@XZ 10005f20 f i ORFDialog.obj
 0001:00004f30       ??1?$QForeachContainer@$$CBV?$QList@PAVTask@U2@@@@@@QAE@XZ 10005f30 f i ORFDialog.obj
 0001:00004f60       ??1?$QForeachContainer@V?$QList@PAVQAction@@@@@@QAE@XZ 10005f60 f i ORFDialog.obj
 0001:00004f90       ??1?$QForeachContainer@V?$QList@VORFFindResult@U2@@@@@@QAE@XZ 10005f90 f i ORFDialog.obj
 0001:00004fa0       ??1?$QList@PAVQAction@@@@QAE@XZ 10005fa0 f i ORFDialog.obj
 0001:00004fd0       ??1?$QList@PAVTask@U2@@@@QAE@XZ 10005fd0 f i ORFDialog.obj
 0001:00005000       ??1?$QList@URegionPreset@U2@@@@QAE@XZ 10006000 f i ORFDialog.obj
 0001:00005030       ??1?$QList@UTriplet@U2@@@@QAE@XZ 10006030 f i ORFDialog.obj
 0001:00005090       ??1?$QList@VORFFindResult@U2@@@@QAE@XZ 10006090 f i ORFDialog.obj
 0001:000050f0       ??1?$QMap@W4DNATranslationRole@U2@@V?$QList@UTriplet@U2@@@@@@QAE@XZ 100060f0 f i ORFDialog.obj
 0001:00005150       ??1?$basic_string@DU?$char_traits@D@std@@V?$allocator@D@2@@std@@QAE@XZ 10006150 f i ORFDialog.obj
 0001:00005180       ??1AbstractInt32Id@U2@@UAE@XZ 10006180 f i ORFDialog.obj
 0001:00005190       ??1ORFDialog@U2@@UAE@XZ    10006190 f i ORFDialog.obj
 0001:000051a0       ??1ORFListItem@U2@@UAE@XZ  100061a0 f i ORFDialog.obj
 0001:000051b0       ??1RegionPreset@U2@@QAE@XZ 100061b0 f i ORFDialog.obj
 0001:000051c0       ??1ServiceType@U2@@UAE@XZ  100061c0 f i ORFDialog.obj
 0001:000051d0       ??1_Generic_error_category@std@@UAE@XZ 100061d0 f i ORFDialog.obj
 0001:000051e0       ??1_Iostream_error_category@std@@UAE@XZ 100061e0 f i ORFDialog.obj
 0001:000051f0       ??1_System_error_category@std@@UAE@XZ 100061f0 f i ORFDialog.obj
 0001:00005200       ??1error_category@std@@UAE@XZ 10006200 f i ORFDialog.obj
 0001:00005210       ??2@YAPAXIPAX@Z            10006210 f i ORFDialog.obj
 0001:00005220       ??3@YAXPAX0@Z              10006220 f i ORFDialog.obj
 0001:00005230       ??4?$QList@UTriplet@U2@@@@QAEAAV0@ABV0@@Z 10006230 f i ORFDialog.obj
 0001:00005270       ??8error_category@std@@QBE_NABV01@@Z 10006270 f i ORFDialog.obj
 0001:00005280       ??8error_condition@std@@QBE_NABV01@@Z 10006280 f i ORFDialog.obj
 0001:000052a0       ??9const_iterator@?$QList@PAVQAction@@@@QBE_NABV01@@Z 100062a0 f i ORFDialog.obj
 0001:000052c0       ??9const_iterator@?$QList@PAVTask@U2@@@@QBE_NABV01@@Z 100062c0 f i ORFDialog.obj
 0001:000052e0       ??9const_iterator@?$QList@VORFFindResult@U2@@@@QBE_NABV01@@Z 100062e0 f i ORFDialog.obj
 0001:00005300       ??A?$QList@UTriplet@U2@@@@QBEABUTriplet@U2@@H@Z 10006300 f i ORFDialog.obj
 0001:00005320       ??A?$QMap@W4DNATranslationRole@U2@@V?$QList@UTriplet@U2@@@@@@QAEAAV?$QList@UTriplet@U2@@@@ABW4DNATranslationRole@U2@@@Z 10006320 f i ORFDialog.obj
 0001:000053f0       ??B?$QFlags@W4TypeFlag@QMetaType@@@@QBEHXZ 100063f0 f i ORFDialog.obj
 0001:00005400       ??BQFlag@@QBEHXZ           10006400 f i ORFDialog.obj
 0001:00005410       ??C?$QSharedDataPointer@VAnnotationData@U2@@@@QAEPAVAnnotationData@U2@@XZ 10006410 f i ORFDialog.obj
 0001:00005430       ??Dconst_iterator@?$QList@PAVQAction@@@@QBEABQAVQAction@@XZ 10006430 f i ORFDialog.obj
 0001:00005440       ??Dconst_iterator@?$QList@PAVTask@U2@@@@QBEABQAVTask@U2@@XZ 10006440 f i ORFDialog.obj
 0001:00005450       ??Dconst_iterator@?$QList@VORFFindResult@U2@@@@QBEABVORFFindResult@U2@@XZ 10006450 f i ORFDialog.obj
 0001:00005460       ??Diterator@?$QMap@W4DNATranslationRole@U2@@V?$QList@UTriplet@U2@@@@@@QBEAAV?$QList@UTriplet@U2@@@@XZ 10006460 f i ORFDialog.obj
 0001:00005470       ??Econst_iterator@?$QList@PAVQAction@@@@QAEAAV01@XZ 10006470 f i ORFDialog.obj
 0001:00005480       ??Econst_iterator@?$QList@PAVTask@U2@@@@QAEAAV01@XZ 10006480 f i ORFDialog.obj
 0001:00005490       ??Econst_iterator@?$QList@VORFFindResult@U2@@@@QAEAAV01@XZ 10006490 f i ORFDialog.obj
 0001:000054a0       ??H@YA?BVQString@@ABV0@0@Z 100064a0 f i ORFDialog.obj
 0001:00005510       ??H@YA?BVQString@@ABV0@PBD@Z 10006510 f i ORFDialog.obj
 0001:000055b0       ??H@YA?BVQString@@PBDABV0@@Z 100065b0 f i ORFDialog.obj
 0001:00005620       ??I?$QFlags@W4TypeFlag@QMetaType@@@@QBE?AV0@W4TypeFlag@QMetaType@@@Z 10006620 f i ORFDialog.obj
 0001:00005640       ??MORFListItem@U2@@UBE_NABVQTreeWidgetItem@@@Z 10006640 f   ORFDialog.obj
 0001:00005c70       ??U?$QFlags@W4StandardButton@QDialogButtonBox@@@@QBE?AV0@W4StandardButton@QDialogButtonBox@@@Z 10006c70 f i ORFDialog.obj
 0001:00005c90       ??U@YA?AV?$QFlags@W4StandardButton@QDialogButtonBox@@@@W4StandardButton@QDialogButtonBox@@0@Z 10006c90 f i ORFDialog.obj
 0001:00005ca0       ??_5?$QFlags@W4TypeFlag@QMetaType@@@@QAEAAV0@W4TypeFlag@QMetaType@@@Z 10006ca0 f i ORFDialog.obj
 0001:00005cae       ??_EORFDialog@U2@@W7AEPAXI@Z 10006cae f i ORFDialog.obj
 0001:00005cb6       ??_EORFFindTask@U2@@WJA@AEPAXI@Z 10006cb6 f i ORFDialog.obj
 0001:00005cc1       ??_EQCheckBox@@W7AEPAXI@Z  10006cc1 f i ORFDialog.obj
 0001:00005cc9       ??_EQComboBox@@W7AEPAXI@Z  10006cc9 f i ORFDialog.obj
 0001:00005cd1       ??_EQDialogButtonBox@@W7AEPAXI@Z 10006cd1 f i ORFDialog.obj
 0001:00005cd9       ??_EQGridLayout@@W7AEPAXI@Z 10006cd9 f i ORFDialog.obj
 0001:00005ce1       ??_EQGroupBox@@W7AEPAXI@Z  10006ce1 f i ORFDialog.obj
 0001:00005ce9       ??_EQHBoxLayout@@W7AEPAXI@Z 10006ce9 f i ORFDialog.obj
 0001:00005cf1       ??_EQLabel@@W7AEPAXI@Z     10006cf1 f i ORFDialog.obj
 0001:00005cf9       ??_EQPushButton@@W7AEPAXI@Z 10006cf9 f i ORFDialog.obj
 0001:00005d01       ??_EQRadioButton@@W7AEPAXI@Z 10006d01 f i ORFDialog.obj
 0001:00005d09       ??_EQSpinBox@@W7AEPAXI@Z   10006d09 f i ORFDialog.obj
 0001:00005d11       ??_EQTabWidget@@W7AEPAXI@Z 10006d11 f i ORFDialog.obj
 0001:00005d19       ??_EQTextEdit@@W7AEPAXI@Z  10006d19 f i ORFDialog.obj
 0001:00005d21       ??_EQTreeWidget@@W7AEPAXI@Z 10006d21 f i ORFDialog.obj
 0001:00005d29       ??_EQVBoxLayout@@W7AEPAXI@Z 10006d29 f i ORFDialog.obj
 0001:00005d31       ??_EQWidget@@W7AEPAXI@Z    10006d31 f i ORFDialog.obj
 0001:00005d39       ??_ERegionSelector@U2@@W7AEPAXI@Z 10006d39 f i ORFDialog.obj
 0001:00005d50       ??_E?$AbstractId@H@U2@@MAEPAXI@Z 10006d50 f i ORFDialog.obj
 0001:00005d50       ??_G?$AbstractId@H@U2@@MAEPAXI@Z 10006d50 f i ORFDialog.obj
 0001:00005d80       ??_G?$QList@UTriplet@U2@@@@QAEPAXI@Z 10006d80 f i ORFDialog.obj
 0001:00005db0       ??_GAbstractInt32Id@U2@@UAEPAXI@Z 10006db0 f i ORFDialog.obj
 0001:00005db0       ??_EAbstractInt32Id@U2@@UAEPAXI@Z 10006db0 f i ORFDialog.obj
 0001:00005de0       ??_GAnnotationData@U2@@QAEPAXI@Z 10006de0 f i ORFDialog.obj
 0001:00005e10       ??_GCreateAnnotationWidgetController@U2@@UAEPAXI@Z 10006e10 f i ORFDialog.obj
 0001:00005e10       ??_ECreateAnnotationWidgetController@U2@@UAEPAXI@Z 10006e10 f i ORFDialog.obj
 0001:00005e40       ??_GHelpButton@U2@@UAEPAXI@Z 10006e40 f i ORFDialog.obj
 0001:00005e40       ??_EHelpButton@U2@@UAEPAXI@Z 10006e40 f i ORFDialog.obj
 0001:00005e70       ??_EORFDialog@U2@@UAEPAXI@Z 10006e70 f i ORFDialog.obj
 0001:00005e70       ??_GORFDialog@U2@@UAEPAXI@Z 10006e70 f i ORFDialog.obj
 0001:00005ea0       ??_GORFFindTask@U2@@UAEPAXI@Z 10006ea0 f i ORFDialog.obj
 0001:00005ea0       ??_EORFFindTask@U2@@UAEPAXI@Z 10006ea0 f i ORFDialog.obj
 0001:00005ed0       ??_EORFListItem@U2@@UAEPAXI@Z 10006ed0 f i ORFDialog.obj
 0001:00005ed0       ??_GORFListItem@U2@@UAEPAXI@Z 10006ed0 f i ORFDialog.obj
 0001:00005f00       ??_EQCheckBox@@UAEPAXI@Z   10006f00 f i ORFDialog.obj
 0001:00005f00       ??_GQCheckBox@@UAEPAXI@Z   10006f00 f i ORFDialog.obj
 0001:00005f30       ??_EQComboBox@@UAEPAXI@Z   10006f30 f i ORFDialog.obj
 0001:00005f30       ??_GQComboBox@@UAEPAXI@Z   10006f30 f i ORFDialog.obj
 0001:00005f60       ??_GQDialogButtonBox@@UAEPAXI@Z 10006f60 f i ORFDialog.obj
 0001:00005f60       ??_EQDialogButtonBox@@UAEPAXI@Z 10006f60 f i ORFDialog.obj
 0001:00005f90       ??_EQGridLayout@@UAEPAXI@Z 10006f90 f i ORFDialog.obj
 0001:00005f90       ??_GQGridLayout@@UAEPAXI@Z 10006f90 f i ORFDialog.obj
 0001:00005fc0       ??_EQGroupBox@@UAEPAXI@Z   10006fc0 f i ORFDialog.obj
 0001:00005fc0       ??_GQGroupBox@@UAEPAXI@Z   10006fc0 f i ORFDialog.obj
 0001:00005ff0       ??_GQHBoxLayout@@UAEPAXI@Z 10006ff0 f i ORFDialog.obj
 0001:00005ff0       ??_EQHBoxLayout@@UAEPAXI@Z 10006ff0 f i ORFDialog.obj
 0001:00006020       ??_EQLabel@@UAEPAXI@Z      10007020 f i ORFDialog.obj
 0001:00006020       ??_GQLabel@@UAEPAXI@Z      10007020 f i ORFDialog.obj
 0001:00006050       ??_GQPushButton@@UAEPAXI@Z 10007050 f i ORFDialog.obj
 0001:00006050       ??_EQPushButton@@UAEPAXI@Z 10007050 f i ORFDialog.obj
 0001:00006080       ??_EQRadioButton@@UAEPAXI@Z 10007080 f i ORFDialog.obj
 0001:00006080       ??_GQRadioButton@@UAEPAXI@Z 10007080 f i ORFDialog.obj
 0001:000060b0       ??_EQSpacerItem@@UAEPAXI@Z 100070b0 f i ORFDialog.obj
 0001:000060b0       ??_GQSpacerItem@@UAEPAXI@Z 100070b0 f i ORFDialog.obj
 0001:000060e0       ??_GQSpinBox@@UAEPAXI@Z    100070e0 f i ORFDialog.obj
 0001:000060e0       ??_EQSpinBox@@UAEPAXI@Z    100070e0 f i ORFDialog.obj
 0001:00006110       ??_GQTabWidget@@UAEPAXI@Z  10007110 f i ORFDialog.obj
 0001:00006110       ??_EQTabWidget@@UAEPAXI@Z  10007110 f i ORFDialog.obj
 0001:00006140       ??_EQTextEdit@@UAEPAXI@Z   10007140 f i ORFDialog.obj
 0001:00006140       ??_GQTextEdit@@UAEPAXI@Z   10007140 f i ORFDialog.obj
 0001:00006170       ??_GQTimer@@UAEPAXI@Z      10007170 f i ORFDialog.obj
 0001:00006170       ??_EQTimer@@UAEPAXI@Z      10007170 f i ORFDialog.obj
 0001:000061a0       ??_GQTreeWidget@@UAEPAXI@Z 100071a0 f i ORFDialog.obj
 0001:000061a0       ??_EQTreeWidget@@UAEPAXI@Z 100071a0 f i ORFDialog.obj
 0001:000061d0       ??_EQVBoxLayout@@UAEPAXI@Z 100071d0 f i ORFDialog.obj
 0001:000061d0       ??_GQVBoxLayout@@UAEPAXI@Z 100071d0 f i ORFDialog.obj
 0001:00006200       ??_EQWidget@@UAEPAXI@Z     10007200 f i ORFDialog.obj
 0001:00006200       ??_GQWidget@@UAEPAXI@Z     10007200 f i ORFDialog.obj
 0001:00006230       ??_GRegionPreset@U2@@QAEPAXI@Z 10007230 f i ORFDialog.obj
 0001:00006260       ??_GRegionSelector@U2@@UAEPAXI@Z 10007260 f i ORFDialog.obj
 0001:00006260       ??_ERegionSelector@U2@@UAEPAXI@Z 10007260 f i ORFDialog.obj
 0001:00006290       ??_GServiceType@U2@@UAEPAXI@Z 10007290 f i ORFDialog.obj
 0001:00006290       ??_EServiceType@U2@@UAEPAXI@Z 10007290 f i ORFDialog.obj
 0001:000062c0       ??_G_Generic_error_category@std@@UAEPAXI@Z 100072c0 f i ORFDialog.obj
 0001:000062c0       ??_E_Generic_error_category@std@@UAEPAXI@Z 100072c0 f i ORFDialog.obj
 0001:000062f0       ??_G_Iostream_error_category@std@@UAEPAXI@Z 100072f0 f i ORFDialog.obj
 0001:000062f0       ??_E_Iostream_error_category@std@@UAEPAXI@Z 100072f0 f i ORFDialog.obj
 0001:00006320       ??_E_System_error_category@std@@UAEPAXI@Z 10007320 f i ORFDialog.obj
 0001:00006320       ??_G_System_error_category@std@@UAEPAXI@Z 10007320 f i ORFDialog.obj
 0001:00006350       ??_Eerror_category@std@@UAEPAXI@Z 10007350 f i ORFDialog.obj
 0001:00006350       ??_Gerror_category@std@@UAEPAXI@Z 10007350 f i ORFDialog.obj
 0001:00006380       ?Construct@?$QMetaTypeFunctionHelper@PAVQAction@@$00@QtMetaTypePrivate@@SAPAXPAXPBX@Z 10007380 f i ORFDialog.obj
 0001:000063b0       ?Create@?$QMetaTypeFunctionHelper@PAVQAction@@$00@QtMetaTypePrivate@@SAPAXPBX@Z 100073b0 f i ORFDialog.obj
 0001:000063f0       ?Delete@?$QMetaTypeFunctionHelper@PAVQAction@@$00@QtMetaTypePrivate@@SAXPAX@Z 100073f0 f i ORFDialog.obj
 0001:00006400       ?Destruct@?$QMetaTypeFunctionHelper@PAVQAction@@$00@QtMetaTypePrivate@@SAXPAX@Z 10007400 f i ORFDialog.obj
 0001:00006410       ?_Copy@?$basic_string@DU?$char_traits@D@std@@V?$allocator@D@2@@std@@QAEXII@Z 10007410 f i ORFDialog.obj
 0001:00006560       ?_Eos@?$basic_string@DU?$char_traits@D@std@@V?$allocator@D@2@@std@@QAEXI@Z 10007560 f i ORFDialog.obj
 0001:00006590       ?_Getal@?$_String_alloc@$0A@U?$_String_base_types@DV?$allocator@D@std@@@std@@@std@@QBE?AU?$_Wrap_alloc@V?$allocator@D@std@@@2@XZ 10007590 f i ORFDialog.obj
 0001:000065a0       ?_Grow@?$basic_string@DU?$char_traits@D@std@@V?$allocator@D@2@@std@@QAE_NI_N@Z 100075a0 f i ORFDialog.obj
 0001:00006650       ?_Inside@?$basic_string@DU?$char_traits@D@std@@V?$allocator@D@2@@std@@QAE_NPBD@Z 10007650 f i ORFDialog.obj
 0001:00006690       ?_Myptr@?$_String_val@U?$_Simple_types@D@std@@@std@@QAEPADXZ 10007690 f i ORFDialog.obj
 0001:000066a0       ?_Myptr@?$_String_val@U?$_Simple_types@D@std@@@std@@QBEPBDXZ 100076a0 f i ORFDialog.obj
 0001:000066b0       ?_Tidy@?$basic_string@DU?$char_traits@D@std@@V?$allocator@D@2@@std@@QAEX_NI@Z 100076b0 f i ORFDialog.obj
 0001:00006700       ?_Xlen@?$basic_string@DU?$char_traits@D@std@@V?$allocator@D@2@@std@@QBEXXZ 10007700 f i ORFDialog.obj
 0001:00006710       ?_Xran@?$basic_string@DU?$char_traits@D@std@@V?$allocator@D@2@@std@@QBEXXZ 10007710 f i ORFDialog.obj
 0001:00006720       ?accept@ORFDialog@U2@@UAEXXZ 10007720 f   ORFDialog.obj
 0001:00006a10       ?allocate@?$_Wrap_alloc@V?$allocator@D@std@@@std@@QAEPADI@Z 10007a10 f i ORFDialog.obj
 0001:00006a40       ?allocate@?$allocator@D@std@@QAEPADI@Z 10007a40 f i ORFDialog.obj
 0001:00006a70       ?assign@?$basic_string@DU?$char_traits@D@std@@V?$allocator@D@2@@std@@QAEAAV12@ABV12@II@Z 10007a70 f i ORFDialog.obj
 0001:00006b90       ?assign@?$basic_string@DU?$char_traits@D@std@@V?$allocator@D@2@@std@@QAEAAV12@PBD@Z 10007b90 f i ORFDialog.obj
 0001:00006bd0       ?assign@?$basic_string@DU?$char_traits@D@std@@V?$allocator@D@2@@std@@QAEAAV12@PBDI@Z 10007bd0 f i ORFDialog.obj
 0001:00006cd0       ?assign@?$char_traits@D@std@@SAXAADABD@Z 10007cd0 f i ORFDialog.obj
 0001:00006ce0       ?begin@?$QList@PAVQAction@@@@QBE?AVconst_iterator@1@XZ 10007ce0 f i ORFDialog.obj
 0001:00006d00       ?begin@?$QList@PAVTask@U2@@@@QBE?AVconst_iterator@1@XZ 10007d00 f i ORFDialog.obj
 0001:00006d20       ?begin@?$QList@VORFFindResult@U2@@@@QBE?AVconst_iterator@1@XZ 10007d20 f i ORFDialog.obj
 0001:00006d40       ?category@error_code@std@@QBEABVerror_category@2@XZ 10007d40 f i ORFDialog.obj
 0001:00006d50       ?category@error_condition@std@@QBEABVerror_category@2@XZ 10007d50 f i ORFDialog.obj
 0001:00006d60       ?clone@?$QSharedDataPointer@VAnnotationData@U2@@@@IAEPAVAnnotationData@U2@@XZ 10007d60 f i ORFDialog.obj
 0001:00006dd0       ?connectGUI@ORFDialog@U2@@AAEXXZ 10007dd0 f   ORFDialog.obj
 0001:00006e60       ?copy@?$QMapNode@W4DNATranslationRole@U2@@V?$QList@UTriplet@U2@@@@@@QBEPAU1@PAU?$QMapData@W4DNATranslationRole@U2@@V?$QList@UTriplet@U2@@@@@@@Z 10007e60 f i ORFDialog.obj
 0001:00006ef0       ?copy@?$char_traits@D@std@@SAPADPADPBDI@Z 10007ef0 f i ORFDialog.obj
 0001:00006f10       ?create@?$QMapData@W4DNATranslationRole@U2@@V?$QList@UTriplet@U2@@@@@@SAPAU1@XZ 10007f10 f i ORFDialog.obj
 0001:00006f20       ?createAnnotationWidget@ORFDialog@U2@@AAEXXZ 10007f20 f   ORFDialog.obj
 0001:000070b0       ?createNode@?$QMapData@W4DNATranslationRole@U2@@V?$QList@UTriplet@U2@@@@@@QAEPAU?$QMapNode@W4DNATranslationRole@U2@@V?$QList@UTriplet@U2@@@@@@ABW4DNATranslationRole@U2@@ABV?$QList@UTriplet@U2@@@@PAU2@_N@Z 100080b0 f i ORFDialog.obj
 0001:00007150       ?data_ptr@?$QStaticStringData@$04@@QBEPAU?$QTypedArrayData@G@@XZ 10008150 f i ORFDialog.obj
 0001:00007160       ?data_ptr@?$QStaticStringData@$05@@QBEPAU?$QTypedArrayData@G@@XZ 10008160 f i ORFDialog.obj
 0001:00007170       ?data_ptr@?$QStaticStringData@$07@@QBEPAU?$QTypedArrayData@G@@XZ 10008170 f i ORFDialog.obj
 0001:00007180       ?data_ptr@?$QStaticStringData@$08@@QBEPAU?$QTypedArrayData@G@@XZ 10008180 f i ORFDialog.obj
 0001:00007190       ?data_ptr@?$QStaticStringData@$09@@QBEPAU?$QTypedArrayData@G@@XZ 10008190 f i ORFDialog.obj
 0001:000071a0       ?data_ptr@?$QStaticStringData@$0BA@@@QBEPAU?$QTypedArrayData@G@@XZ 100081a0 f i ORFDialog.obj
 0001:000071b0       ?data_ptr@?$QStaticStringData@$0BB@@@QBEPAU?$QTypedArrayData@G@@XZ 100081b0 f i ORFDialog.obj
 0001:000071c0       ?data_ptr@?$QStaticStringData@$0BC@@@QBEPAU?$QTypedArrayData@G@@XZ 100081c0 f i ORFDialog.obj
 0001:000071d0       ?data_ptr@?$QStaticStringData@$0BD@@@QBEPAU?$QTypedArrayData@G@@XZ 100081d0 f i ORFDialog.obj
 0001:000071e0       ?data_ptr@?$QStaticStringData@$0L@@@QBEPAU?$QTypedArrayData@G@@XZ 100081e0 f i ORFDialog.obj
 0001:000071f0       ?data_ptr@?$QStaticStringData@$0M@@@QBEPAU?$QTypedArrayData@G@@XZ 100081f0 f i ORFDialog.obj
 0001:00007200       ?data_ptr@?$QStaticStringData@$0N@@@QBEPAU?$QTypedArrayData@G@@XZ 10008200 f i ORFDialog.obj
 0001:00007210       ?data_ptr@?$QStaticStringData@$0O@@@QBEPAU?$QTypedArrayData@G@@XZ 10008210 f i ORFDialog.obj
 0001:00007220       ?dealloc@?$QList@PAVQAction@@@@AAEXPAUData@QListData@@@Z 10008220 f i ORFDialog.obj
 0001:00007240       ?dealloc@?$QList@PAVTask@U2@@@@AAEXPAUData@QListData@@@Z 10008240 f i ORFDialog.obj
 0001:00007260       ?dealloc@?$QList@URegionPreset@U2@@@@AAEXPAUData@QListData@@@Z 10008260 f i ORFDialog.obj
 0001:000072c0       ?dealloc@?$QList@UTriplet@U2@@@@AAEXPAUData@QListData@@@Z 100082c0 f i ORFDialog.obj
 0001:00007310       ?dealloc@?$QList@VORFFindResult@U2@@@@AAEXPAUData@QListData@@@Z 10008310 f i ORFDialog.obj
 0001:00007360       ?deallocate@?$_Wrap_alloc@V?$allocator@D@std@@@std@@QAEXPADI@Z 10008360 f i ORFDialog.obj
 0001:00007380       ?deallocate@?$allocator@D@std@@QAEXPADI@Z 10008380 f i ORFDialog.obj
 0001:000073a0       ?default_error_condition@_System_error_category@std@@UBE?AVerror_condition@2@H@Z 100083a0 f i ORFDialog.obj
 0001:000073e0       ?default_error_condition@error_category@std@@UBE?AVerror_condition@2@H@Z 100083e0 f i ORFDialog.obj
 0001:00007400       ?deref@?$QBasicAtomicInteger@H@@QAE_NXZ 10008400 f i ORFDialog.obj
 0001:00007410       ?deref@RefCount@QtPrivate@@QAE_NXZ 10008410 f i ORFDialog.obj
 0001:00007430       ?destroy@?$QMapData@W4DNATranslationRole@U2@@V?$QList@UTriplet@U2@@@@@@QAEXXZ 10008430 f i ORFDialog.obj
 0001:00007480       ?destroySubTree@?$QMapNode@W4DNATranslationRole@U2@@V?$QList@UTriplet@U2@@@@@@QAEXXZ 10008480 f i ORFDialog.obj
 0001:000074a0       ?detach@?$QMap@W4DNATranslationRole@U2@@V?$QList@UTriplet@U2@@@@@@QAEXXZ 100084a0 f i ORFDialog.obj
 0001:000074c0       ?detach@?$QSharedDataPointer@VAnnotationData@U2@@@@QAEXXZ 100084c0 f i ORFDialog.obj
 0001:000074d0       ?detach_helper@?$QMap@W4DNATranslationRole@U2@@V?$QList@UTriplet@U2@@@@@@AAEXXZ 100084d0 f i ORFDialog.obj
 0001:00007580       ?detach_helper@?$QSharedDataPointer@VAnnotationData@U2@@@@AAEXXZ 10008580 f i ORFDialog.obj
 0001:00007620       ?empty@?$QList@VORFFindResult@U2@@@@QBE_NXZ 10008620 f i ORFDialog.obj
 0001:00007630       ?end@?$QList@PAVQAction@@@@QBE?AVconst_iterator@1@XZ 10008630 f i ORFDialog.obj
 0001:00007650       ?end@?$QList@PAVTask@U2@@@@QBE?AVconst_iterator@1@XZ 10008650 f i ORFDialog.obj
 0001:00007670       ?end@?$QList@VORFFindResult@U2@@@@QBE?AVconst_iterator@1@XZ 10008670 f i ORFDialog.obj
 0001:00007690       ?end@?$QMapData@W4DNATranslationRole@U2@@V?$QList@UTriplet@U2@@@@@@QAEPAU?$QMapNode@W4DNATranslationRole@U2@@V?$QList@UTriplet@U2@@@@@@XZ 10008690 f i ORFDialog.obj
 0001:000076a0       ?equivalent@error_category@std@@UBE_NABVerror_code@2@H@Z 100086a0 f i ORFDialog.obj
 0001:000076c0       ?equivalent@error_category@std@@UBE_NHABVerror_condition@2@@Z 100086c0 f i ORFDialog.obj
 0001:00007700       ?erase@?$basic_string@DU?$char_traits@D@std@@V?$allocator@D@2@@std@@QAEAAV12@I@Z 10008700 f i ORFDialog.obj
 0001:00007740       ?erase@?$basic_string@DU?$char_traits@D@std@@V?$allocator@D@2@@std@@QAEAAV12@II@Z 10008740 f i ORFDialog.obj
 0001:000077e0       ?eventFilter@ORFDialog@U2@@MAE_NPAVQObject@@PAVQEvent@@@Z 100087e0 f   ORFDialog.obj
 0001:00007830       ?findNode@?$QMapData@W4DNATranslationRole@U2@@V?$QList@UTriplet@U2@@@@@@QBEPAU?$QMapNode@W4DNATranslationRole@U2@@V?$QList@UTriplet@U2@@@@@@ABW4DNATranslationRole@U2@@@Z 10008830 f i ORFDialog.obj
 0001:00007870       ?findStartedAAUpdateTask@ORFDialog@U2@@AAEXXZ 10008870 f   ORFDialog.obj
 0001:00007b40       ?generic_category@std@@YAABVerror_category@1@XZ 10008b40 f i ORFDialog.obj
 0001:00007b50       ?getAlgStrand@ORFDialog@U2@@ABE?AW4ORFAlgorithmStrand@2@XZ 10008b50 f   ORFDialog.obj
 0001:00007b80       ?getCodons@DNATranslation3to1Impl@U2@@QBE?AV?$QMap@W4DNATranslationRole@U2@@V?$QList@UTriplet@U2@@@@@@XZ 10008b80 f i ORFDialog.obj
 0001:00007bb0       ?getCompleteSearchRegion@ORFDialog@U2@@ABE?AVU2Region@2@PA_N@Z 10008bb0 f   ORFDialog.obj
 0001:00007c10       ?getSettings@ORFDialog@U2@@AAEXAAVORFAlgorithmSettings@2@@Z 10008c10 f   ORFDialog.obj
 0001:00007e80       ?importResults@ORFDialog@U2@@AAEXXZ 10008e80 f   ORFDialog.obj
 0001:00007fd0       ?initSettings@ORFDialog@U2@@AAEXXZ 10008fd0 f   ORFDialog.obj
 0001:000080c0       ?insert@?$QMap@W4DNATranslationRole@U2@@V?$QList@UTriplet@U2@@@@@@QAE?AViterator@1@ABW4DNATranslationRole@U2@@ABV?$QList@UTriplet@U2@@@@@Z 100090c0 f i ORFDialog.obj
 0001:00008170       ?invoke@?$ObjectInvoker@U?$QVariantValueHelper@PAVQAction@@@QtPrivate@@ABVQVariant@@PAVQAction@@@QtPrivate@@SAPAVQAction@@ABVQVariant@@@Z 10009170 f i ORFDialog.obj
 0001:00008180       ?isEmpty@?$QList@VORFFindResult@U2@@@@QBE_NXZ 10009180 f i ORFDialog.obj
 0001:00008190       ?isShared@RefCount@QtPrivate@@QBE_NXZ 10009190 f i ORFDialog.obj
 0001:000081b0       ?isValid@AbstractInt32Id@U2@@UBE_NXZ 100091b0 f i ORFDialog.obj
 0001:000081c0       ?leftNode@?$QMapNode@W4DNATranslationRole@U2@@V?$QList@UTriplet@U2@@@@@@QBEPAU1@XZ 100091c0 f i ORFDialog.obj
 0001:000081d0       ?length@?$char_traits@D@std@@SAIPBD@Z 100091d0 f i ORFDialog.obj
 0001:000081f0       ?load@?$QBasicAtomicInteger@H@@QBEHXZ 100091f0 f i ORFDialog.obj
 0001:00008200       ?loadAcquire@?$QBasicAtomicInteger@H@@QBEHXZ 10009200 f i ORFDialog.obj
 0001:00008210       ?lowerBound@?$QMapNode@W4DNATranslationRole@U2@@V?$QList@UTriplet@U2@@@@@@QAEPAU1@ABW4DNATranslationRole@U2@@@Z 10009210 f i ORFDialog.obj
 0001:00008240       ?max_size@?$_Wrap_alloc@V?$allocator@D@std@@@std@@QBEIXZ 10009240 f i ORFDialog.obj
 0001:00008250       ?max_size@?$allocator@D@std@@QBEIXZ 10009250 f i ORFDialog.obj
 0001:00008260       ?max_size@?$allocator_traits@V?$allocator@D@std@@@std@@SAIABV?$allocator@D@2@@Z 10009260 f i ORFDialog.obj
 0001:00008270       ?max_size@?$basic_string@DU?$char_traits@D@std@@V?$allocator@D@2@@std@@QBEIXZ 10009270 f i ORFDialog.obj
 0001:00008280       ?message@_Generic_error_category@std@@UBE?AV?$basic_string@DU?$char_traits@D@std@@V?$allocator@D@2@@2@H@Z 10009280 f i ORFDialog.obj
 0001:00008300       ?message@_Iostream_error_category@std@@UBE?AV?$basic_string@DU?$char_traits@D@std@@V?$allocator@D@2@@2@H@Z 10009300 f i ORFDialog.obj
 0001:00008350       ?message@_System_error_category@std@@UBE?AV?$basic_string@DU?$char_traits@D@std@@V?$allocator@D@2@@2@H@Z 10009350 f i ORFDialog.obj
 0001:000083d0       ?metaType@?$QVariantValueHelper@PAVQAction@@@QtPrivate@@SAPAVQAction@@ABVQVariant@@@Z 100093d0 f i ORFDialog.obj
 0001:00008420       ?move@?$char_traits@D@std@@SAPADPADPBDI@Z 10009420 f i ORFDialog.obj
 0001:00008440       ?name@_Generic_error_category@std@@UBEPBDXZ 10009440 f i ORFDialog.obj
 0001:00008450       ?name@_Iostream_error_category@std@@UBEPBDXZ 10009450 f i ORFDialog.obj
 0001:00008460       ?name@_System_error_category@std@@UBEPBDXZ 10009460 f i ORFDialog.obj
 0001:00008470       ?node_copy@?$QList@PAVQAction@@@@AAEXPAUNode@1@00@Z 10009470 f i ORFDialog.obj
 0001:000084a0       ?node_copy@?$QList@PAVTask@U2@@@@AAEXPAUNode@1@00@Z 100094a0 f i ORFDialog.obj
 0001:000084d0       ?node_copy@?$QList@UTriplet@U2@@@@AAEXPAUNode@1@00@Z 100094d0 f i ORFDialog.obj
 0001:00008580       ?node_copy@?$QList@VORFFindResult@U2@@@@AAEXPAUNode@1@00@Z 10009580 f i ORFDialog.obj
 0001:00008640       ?node_destruct@?$QList@PAVQAction@@@@AAEXPAUNode@1@0@Z 10009640 f i ORFDialog.obj
 0001:00008650       ?node_destruct@?$QList@PAVTask@U2@@@@AAEXPAUNode@1@0@Z 10009650 f i ORFDialog.obj
 0001:00008660       ?node_destruct@?$QList@URegionPreset@U2@@@@AAEXPAUNode@1@0@Z 10009660 f i ORFDialog.obj
 0001:000086a0       ?node_destruct@?$QList@UTriplet@U2@@@@AAEXPAUNode@1@0@Z 100096a0 f i ORFDialog.obj
 0001:000086d0       ?node_destruct@?$QList@VORFFindResult@U2@@@@AAEXPAUNode@1@0@Z 100096d0 f i ORFDialog.obj
 0001:00008700       ?object@?$QVariantValueHelper@PAVQAction@@@QtPrivate@@SAPAVQAction@@ABVQVariant@@@Z 10009700 f i ORFDialog.obj
 0001:00008790       ?qt_metatype_id@?$QMetaTypeId2@PAVQAction@@@@SAHXZ 10009790 f i ORFDialog.obj
 0001:000087a0       ?qt_metatype_id@?$QMetaTypeId@PAVQAction@@@@SAHXZ 100097a0 f i ORFDialog.obj
 0001:00008850       ?qt_metatype_id@?$QMetaTypeIdHelper@PAVQAction@@$00@QtPrivate@@SAHXZ 10009850 f i ORFDialog.obj
 0001:00008860       ?qt_noop@@YAXXZ            10009860 f i ORFDialog.obj
 0001:00008870       ?ref@?$QBasicAtomicInteger@H@@QAE_NXZ 10009870 f i ORFDialog.obj
 0001:00008890       ?ref@RefCount@QtPrivate@@QAE_NXZ 10009890 f i ORFDialog.obj
 0001:000088b0       ?registerConverter@?$AssociativeContainerConverterHelper@PAVQAction@@$0A@@QtPrivate@@SA_NH@Z 100098b0 f i ORFDialog.obj
 0001:000088c0       ?registerConverter@?$IsPair@PAVQAction@@@QtPrivate@@SA_NH@Z 100098c0 f i ORFDialog.obj
 0001:000088d0       ?registerConverter@?$MetaTypeSmartPointerHelper@PAVQAction@@X@QtPrivate@@SA_NH@Z 100098d0 f i ORFDialog.obj
 0001:000088e0       ?registerConverter@?$SequentialContainerConverterHelper@PAVQAction@@$0A@@QtPrivate@@SA_NH@Z 100098e0 f i ORFDialog.obj
 0001:000088f0       ?reject@ORFDialog@U2@@UAEXXZ 100098f0 f   ORFDialog.obj
 0001:00008910       ?retranslateUi@Ui_ORFDialogBase@@QAEXPAVQDialog@@@Z 10009910 f i ORFDialog.obj
 0001:000094b0       ?rightNode@?$QMapNode@W4DNATranslationRole@U2@@V?$QList@UTriplet@U2@@@@@@QBEPAU1@XZ 1000a4b0 f i ORFDialog.obj
 0001:000094c0       ?root@?$QMapData@W4DNATranslationRole@U2@@V?$QList@UTriplet@U2@@@@@@QBEPAU?$QMapNode@W4DNATranslationRole@U2@@V?$QList@UTriplet@U2@@@@@@XZ 1000a4c0 f i ORFDialog.obj
 0001:000094d0       ?runTask@ORFDialog@U2@@AAEXXZ 1000a4d0 f   ORFDialog.obj
 0001:00009660       ?setupUi@Ui_ORFDialogBase@@QAEXPAVQDialog@@@Z 1000a660 f i ORFDialog.obj
 0001:0000ae60       ?size@?$QList@UTriplet@U2@@@@QBEHXZ 1000be60 f i ORFDialog.obj
 0001:0000ae70       ?size@?$basic_string@DU?$char_traits@D@std@@V?$allocator@D@2@@std@@QBEIXZ 1000be70 f i ORFDialog.obj
 0001:0000ae80       ?sl_onClearList@ORFDialog@U2@@AAEXXZ 1000be80 f   ORFDialog.obj
 0001:0000aea0       ?sl_onFindAll@ORFDialog@U2@@AAEXXZ 1000bea0 f   ORFDialog.obj
 0001:0000af70       ?sl_onResultActivated@ORFDialog@U2@@AAEXPAVQTreeWidgetItem@@H@Z 1000bf70 f   ORFDialog.obj
 0001:0000af90       ?sl_onTaskFinished@ORFDialog@U2@@AAEXPAVTask@2@@Z 1000bf90 f   ORFDialog.obj
 0001:0000aff0       ?sl_onTimer@ORFDialog@U2@@AAEXXZ 1000bff0 f   ORFDialog.obj
 0001:0000b000       ?sl_translationChanged@ORFDialog@U2@@AAEXXZ 1000c000 f   ORFDialog.obj
 0001:0000b600       ?storeRelease@?$QBasicAtomicInteger@H@@QAEXH@Z 1000c600 f i ORFDialog.obj
 0001:0000b610       ?swap@?$QList@UTriplet@U2@@@@QAEXAAV1@@Z 1000c610 f i ORFDialog.obj
 0001:0000b630       ?system_category@std@@YAABVerror_category@1@XZ 1000c630 f i ORFDialog.obj
 0001:0000b640       ?t@Node@?$QList@PAVQAction@@@@QAEAAPAVQAction@@XZ 1000c640 f i ORFDialog.obj
 0001:0000b650       ?t@Node@?$QList@PAVTask@U2@@@@QAEAAPAVTask@U2@@XZ 1000c650 f i ORFDialog.obj
 0001:0000b660       ?t@Node@?$QList@UTriplet@U2@@@@QAEAAUTriplet@U2@@XZ 1000c660 f i ORFDialog.obj
 0001:0000b670       ?t@Node@?$QList@VORFFindResult@U2@@@@QAEAAVORFFindResult@U2@@XZ 1000c670 f i ORFDialog.obj
 0001:0000b680       ?tr@ORFDialog@U2@@SA?AVQString@@PBD0H@Z 1000c680 f i ORFDialog.obj
 0001:0000b750       ?updateState@ORFDialog@U2@@AAEXXZ 1000c750 f   ORFDialog.obj
 0001:0000b810       ?updateStatus@ORFDialog@U2@@AAEXXZ 1000c810 f   ORFDialog.obj
 0001:0000b960       ?value@?$MetaObjectForType@PAVQAction@@$00@QtPrivate@@SAPBUQMetaObject@@XZ 1000c960 f i ORFDialog.obj
 0001:0000b970       ?value@error_code@std@@QBEHXZ 1000c970 f i ORFDialog.obj
 0001:0000b980       ?value@error_condition@std@@QBEHXZ 1000c980 f i ORFDialog.obj
 0001:0000b990       _hypot                     1000c990 f i ORFDialog.obj
 0001:0000b9c0       ??$?0VORFDialog@U2@@@?$QWeakPointer@VQObject@@@@AAE@PAVORFDialog@U2@@_N@Z 1000c9c0 f i ORFMarkerPlugin.obj
 0001:0000ba00       ??$qDeleteAll@V?$QList@PAVXMLTestFactory@U2@@@@@@YAXABV?$QList@PAVXMLTestFactory@U2@@@@@Z 1000ca00 f i ORFMarkerPlugin.obj
 0001:0000ba40       ??$qDeleteAll@Vconst_iterator@?$QList@PAVXMLTestFactory@U2@@@@@@YAXVconst_iterator@?$QList@PAVXMLTestFactory@U2@@@@0@Z 1000ca40 f i ORFMarkerPlugin.obj
 0001:0000ba70       ??$qobject_cast@PAVAnnotatedDNAView@U2@@@@YAPAVAnnotatedDNAView@U2@@PAVQObject@@@Z 1000ca70 f i ORFMarkerPlugin.obj
 0001:0000ba90       ??$qobject_cast@PAVGObjectViewAction@U2@@@@YAPAVGObjectViewAction@U2@@PAVQObject@@@Z 1000ca90 f i ORFMarkerPlugin.obj
 0001:0000bab0       ??$qobject_cast@PAVXMLTestFormat@U2@@@@YAPAVXMLTestFormat@U2@@PAVQObject@@@Z 1000cab0 f i ORFMarkerPlugin.obj
 0001:0000bad0       ??0?$GAutoDeleteList@VXMLTestFactory@U2@@@U2@@QAE@PAVQObject@@@Z 1000cad0 f i ORFMarkerPlugin.obj
 0001:0000bb00       ??0?$QFlags@W4ADVGlobalActionFlag@U2@@@@QAE@VQFlag@@@Z 1000cb00 f i ORFMarkerPlugin.obj
 0001:0000bb10       ??0?$QFlags@W4ADVGlobalActionFlag@U2@@@@QAE@W4ADVGlobalActionFlag@U2@@@Z 1000cb10 f i ORFMarkerPlugin.obj
 0001:0000bb20       ??0?$QFlags@W4TaskFlag@U2@@@@QAE@VQFlag@@@Z 1000cb20 f i ORFMarkerPlugin.obj
 0001:0000bb30       ??0?$QFlags@W4TaskFlag@U2@@@@QAE@W4TaskFlag@U2@@@Z 1000cb30 f i ORFMarkerPlugin.obj
 0001:0000bb40       ??0?$QForeachContainer@V?$QList@PAVXMLTestFactory@U2@@@@@@QAE@ABV?$QList@PAVXMLTestFactory@U2@@@@@Z 1000cb40 f i ORFMarkerPlugin.obj
 0001:0000bb80       ??0?$QList@PAVXMLTestFactory@U2@@@@QAE@$$QAV0@@Z 1000cb80 f i ORFMarkerPlugin.obj
 0001:0000bba0       ??0?$QList@PAVXMLTestFactory@U2@@@@QAE@ABV0@@Z 1000cba0 f i ORFMarkerPlugin.obj
 0001:0000bc60       ??0?$QList@PAVXMLTestFactory@U2@@@@QAE@XZ 1000cc60 f i ORFMarkerPlugin.obj
 0001:0000bc70       ??0?$QObjectScopedPointer@VORFDialog@U2@@@U2@@QAE@PAVORFDialog@1@@Z 1000cc70 f i ORFMarkerPlugin.obj
 0001:0000bcb0       ??0?$QPointer@VORFDialog@U2@@@@QAE@PAVORFDialog@U2@@@Z 1000ccb0 f i ORFMarkerPlugin.obj
 0001:0000bcf0       ??0?$QVector@VU2Region@U2@@@@QAE@XZ 1000ccf0 f i ORFMarkerPlugin.obj
 0001:0000bd00       ??0GObjectViewFactoryId@U2@@QAE@PBD@Z 1000cd00 f i ORFMarkerPlugin.obj
 0001:0000bd40       ??0GTest_ORFMarkerTask@U2@@QAE@PAVXMLTestFormat@1@ABVQString@@PAVGTest@1@PBVGTestEnvironment@1@ABV?$QList@PAVGTest@U2@@@@ABVQDomElement@@@Z 1000cd40 f i ORFMarkerPlugin.obj
 0001:0000be50       ??0GTest_ORFMarkerTaskFactory@GTest_ORFMarkerTask@U2@@QAE@XZ 1000ce50 f i ORFMarkerPlugin.obj
 0001:0000bed0       ??0ORFMarkerPlugin@U2@@QAE@XZ 1000ced0 f   ORFMarkerPlugin.obj
 0001:0000c170       ??0ORFViewContext@U2@@QAE@PAVQObject@@@Z 1000d170 f   ORFMarkerPlugin.obj
 0001:0000c200       ??0const_iterator@?$QList@PAVXMLTestFactory@U2@@@@QAE@PAUNode@1@@Z 1000d200 f i ORFMarkerPlugin.obj
 0001:0000c210       ??1?$GAutoDeleteList@VXMLTestFactory@U2@@@U2@@UAE@XZ 1000d210 f i ORFMarkerPlugin.obj
 0001:0000c2d0       ??1?$QForeachContainer@V?$QList@PAVXMLTestFactory@U2@@@@@@QAE@XZ 1000d2d0 f i ORFMarkerPlugin.obj
 0001:0000c300       ??1?$QList@PAVXMLTestFactory@U2@@@@QAE@XZ 1000d300 f i ORFMarkerPlugin.obj
 0001:0000c330       ??1?$QObjectScopedPointer@VORFDialog@U2@@@U2@@QAE@XZ 1000d330 f i ORFMarkerPlugin.obj
 0001:0000c3b0       ??1?$QPointer@VORFDialog@U2@@@@QAE@XZ 1000d3b0 f i ORFMarkerPlugin.obj
 0001:0000c3d0       ??1?$QVector@VU2Region@U2@@@@QAE@XZ 1000d3d0 f i ORFMarkerPlugin.obj
 0001:0000c410       ??1?$QWeakPointer@VQObject@@@@QAE@XZ 1000d410 f i ORFMarkerPlugin.obj
 0001:0000c430       ??1ExternalRefCountData@QtSharedPointer@@QAE@XZ 1000d430 f i ORFMarkerPlugin.obj
 0001:0000c440       ??1GObjectViewFactoryId@U2@@QAE@XZ 1000d440 f i ORFMarkerPlugin.obj
 0001:0000c450       ??1GTest_ORFMarkerTask@U2@@UAE@XZ 1000d450 f i ORFMarkerPlugin.obj
 0001:0000c510       ??1GTest_ORFMarkerTaskFactory@GTest_ORFMarkerTask@U2@@UAE@XZ 1000d510 f i ORFMarkerPlugin.obj
 0001:0000c520       ??1ORFMarkerPlugin@U2@@UAE@XZ 1000d520 f   ORFMarkerPlugin.obj
 0001:0000c530       ??1ORFViewContext@U2@@UAE@XZ 1000d530 f i ORFMarkerPlugin.obj
 0001:0000c540       ??3ExternalRefCountData@QtSharedPointer@@SAXPAX@Z 1000d540 f i ORFMarkerPlugin.obj
 0001:0000c550       ??4?$QList@PAVXMLTestFactory@U2@@@@QAEAAV0@$$QAV0@@Z 1000d550 f i ORFMarkerPlugin.obj
 0001:0000c570       ??9const_iterator@?$QList@PAVXMLTestFactory@U2@@@@QBE_NABV01@@Z 1000d570 f i ORFMarkerPlugin.obj
 0001:0000c590       ??C?$QObjectScopedPointer@VORFDialog@U2@@@U2@@QBEPAVORFDialog@1@XZ 1000d590 f i ORFMarkerPlugin.obj
 0001:0000c5b0       ??C?$QPointer@VORFDialog@U2@@@@QBEPAVORFDialog@U2@@XZ 1000d5b0 f i ORFMarkerPlugin.obj
 0001:0000c5d0       ??Dconst_iterator@?$QList@PAVXMLTestFactory@U2@@@@QBEABQAVXMLTestFactory@U2@@XZ 1000d5d0 f i ORFMarkerPlugin.obj
 0001:0000c5e0       ??Econst_iterator@?$QList@PAVXMLTestFactory@U2@@@@QAEAAV01@XZ 1000d5e0 f i ORFMarkerPlugin.obj
 0001:0000c5f0       ??U?$QFlags@W4ADVGlobalActionFlag@U2@@@@QBE?AV0@W4ADVGlobalActionFlag@U2@@@Z 1000d5f0 f i ORFMarkerPlugin.obj
 0001:0000c610       ??U?$QFlags@W4TaskFlag@U2@@@@QBE?AV0@W4TaskFlag@U2@@@Z 1000d610 f i ORFMarkerPlugin.obj
 0001:0000c621       ??_EORFViewContext@U2@@W7AEPAXI@Z 1000d621 f i ORFMarkerPlugin.obj
 0001:0000c630       ??_E?$GAutoDeleteList@VXMLTestFactory@U2@@@U2@@UAEPAXI@Z 1000d630 f i ORFMarkerPlugin.obj
 0001:0000c630       ??_G?$GAutoDeleteList@VXMLTestFactory@U2@@@U2@@UAEPAXI@Z 1000d630 f i ORFMarkerPlugin.obj
 0001:0000c660       ??_EADVGlobalAction@U2@@UAEPAXI@Z 1000d660 f i ORFMarkerPlugin.obj
 0001:0000c660       ??_GADVGlobalAction@U2@@UAEPAXI@Z 1000d660 f i ORFMarkerPlugin.obj
 0001:0000c690       ??_GExternalRefCountData@QtSharedPointer@@QAEPAXI@Z 1000d690 f i ORFMarkerPlugin.obj
 0001:0000c6b0       ??_EGTest_ORFMarkerTask@U2@@UAEPAXI@Z 1000d6b0 f i ORFMarkerPlugin.obj
 0001:0000c6b0       ??_GGTest_ORFMarkerTask@U2@@UAEPAXI@Z 1000d6b0 f i ORFMarkerPlugin.obj
 0001:0000c6e0       ??_GGTest_ORFMarkerTaskFactory@GTest_ORFMarkerTask@U2@@UAEPAXI@Z 1000d6e0 f i ORFMarkerPlugin.obj
 0001:0000c6e0       ??_EGTest_ORFMarkerTaskFactory@GTest_ORFMarkerTask@U2@@UAEPAXI@Z 1000d6e0 f i ORFMarkerPlugin.obj
 0001:0000c710       ??_EORFMarkerPlugin@U2@@UAEPAXI@Z 1000d710 f i ORFMarkerPlugin.obj
 0001:0000c710       ??_GORFMarkerPlugin@U2@@UAEPAXI@Z 1000d710 f i ORFMarkerPlugin.obj
 0001:0000c740       ??_EORFViewContext@U2@@UAEPAXI@Z 1000d740 f i ORFMarkerPlugin.obj
 0001:0000c740       ??_GORFViewContext@U2@@UAEPAXI@Z 1000d740 f i ORFMarkerPlugin.obj
 0001:0000c770       ?append@?$QList@PAVXMLTestFactory@U2@@@@QAEXABQAVXMLTestFactory@U2@@@Z 1000d770 f i ORFMarkerPlugin.obj
 0001:0000c800       ?begin@?$QList@PAVXMLTestFactory@U2@@@@QBE?AVconst_iterator@1@XZ 1000d800 f i ORFMarkerPlugin.obj
 0001:0000c820       ?begin@?$QTypedArrayData@VU2Region@U2@@@@QAEPAVU2Region@U2@@PAV23@@Z 1000d820 f i ORFMarkerPlugin.obj
 0001:0000c830       ?createFactory@GTest_ORFMarkerTask@U2@@SAPAVXMLTestFactory@2@XZ 1000d830 f i ORFMarkerPlugin.obj
 0001:0000c8d0       ?createTest@GTest_ORFMarkerTaskFactory@GTest_ORFMarkerTask@U2@@UAEPAVGTest@3@PAVXMLTestFormat@3@ABVQString@@PAV43@PBVGTestEnvironment@3@ABV?$QList@PAVGTest@U2@@@@ABVQDomElement@@@Z 1000d8d0 f i ORFMarkerPlugin.obj
 0001:0000c950       ?createTestFactories@ORFMarkerTests@U2@@SA?AV?$QList@PAVXMLTestFactory@U2@@@@XZ 1000d950 f   ORFMarkerPlugin.obj
 0001:0000c9c0       ?data@?$QPointer@VORFDialog@U2@@@@QBEPAVORFDialog@U2@@XZ 1000d9c0 f i ORFMarkerPlugin.obj
 0001:0000c9e0       ?data@?$QTypedArrayData@VU2Region@U2@@@@QAEPAVU2Region@U2@@XZ 1000d9e0 f i ORFMarkerPlugin.obj
 0001:0000c9f0       ?data@?$QWeakPointer@VQObject@@@@QBEPAVQObject@@XZ 1000d9f0 f i ORFMarkerPlugin.obj
 0001:0000ca10       ?dealloc@?$QList@PAVXMLTestFactory@U2@@@@AAEXPAUData@QListData@@@Z 1000da10 f i ORFMarkerPlugin.obj
 0001:0000ca30       ?deallocate@?$QTypedArrayData@VU2Region@U2@@@@SAXPAUQArrayData@@@Z 1000da30 f i ORFMarkerPlugin.obj
 0001:0000ca50       ?destruct@?$QVector@VU2Region@U2@@@@AAEXPAVU2Region@U2@@0@Z 1000da50 f i ORFMarkerPlugin.obj
 0001:0000ca60       ?detach_helper_grow@?$QList@PAVXMLTestFactory@U2@@@@AAEPAUNode@1@HH@Z 1000da60 f i ORFMarkerPlugin.obj
 0001:0000cb70       ?end@?$QList@PAVXMLTestFactory@U2@@@@QBE?AVconst_iterator@1@XZ 1000db70 f i ORFMarkerPlugin.obj
 0001:0000cb90       ?end@?$QTypedArrayData@VU2Region@U2@@@@QAEPAVU2Region@U2@@PAV23@@Z 1000db90 f i ORFMarkerPlugin.obj
 0001:0000cbb0       ?freeData@?$QVector@VU2Region@U2@@@@AAEXPAU?$QTypedArrayData@VU2Region@U2@@@@@Z 1000dbb0 f i ORFMarkerPlugin.obj
 0001:0000cbe0       ?initViewContext@ORFViewContext@U2@@MAEXPAVGObjectView@2@@Z 1000dbe0 f   ORFMarkerPlugin.obj
 0001:0000cd80       ?node_construct@?$QList@PAVXMLTestFactory@U2@@@@AAEXPAUNode@1@ABQAVXMLTestFactory@U2@@@Z 1000dd80 f i ORFMarkerPlugin.obj
 0001:0000cda0       ?node_copy@?$QList@PAVXMLTestFactory@U2@@@@AAEXPAUNode@1@00@Z 1000dda0 f i ORFMarkerPlugin.obj
 0001:0000cdd0       ?node_destruct@?$QList@PAVXMLTestFactory@U2@@@@AAEXPAUNode@1@0@Z 1000ddd0 f i ORFMarkerPlugin.obj
 0001:0000cde0       ?node_destruct@?$QList@PAVXMLTestFactory@U2@@@@AAEXPAUNode@1@@Z 1000dde0 f i ORFMarkerPlugin.obj
 0001:0000cdf0       ?sharedNull@?$QTypedArrayData@VU2Region@U2@@@@SAPAU1@XZ 1000ddf0 f i ORFMarkerPlugin.obj
 0001:0000ce00       ?sl_showDialog@ORFViewContext@U2@@IAEXXZ 1000de00 f   ORFMarkerPlugin.obj
 0001:0000cf10       ?t@Node@?$QList@PAVXMLTestFactory@U2@@@@QAEAAPAVXMLTestFactory@U2@@XZ 1000df10 f i ORFMarkerPlugin.obj
 0001:0000cf20       ?tr@ORFMarkerPlugin@U2@@SA?AVQString@@PBD0H@Z 1000df20 f i ORFMarkerPlugin.obj
 0001:0000cf50       ?tr@ORFViewContext@U2@@SA?AVQString@@PBD0H@Z 1000df50 f i ORFMarkerPlugin.obj
 0001:0000cf80       _ugene_plugin_init         1000df80 f   ORFMarkerPlugin.obj
 0001:0000cfa0       ??$?0VAnnotationTableObject@U2@@@?$QWeakPointer@VQObject@@@@AAE@PAVAnnotationTableObject@U2@@_N@Z 1000dfa0 f i ORFMarkerTask.obj
 0001:0000cfe0       ??$fromValue@VU2Region@U2@@@QVariant@@SA?AV0@ABVU2Region@U2@@@Z 1000dfe0 f i ORFMarkerTask.obj
 0001:0000d000       ??$qMetaTypeId@VU2Region@U2@@@@YAHXZ 1000e000 f i ORFMarkerTask.obj
 0001:0000d010       ??$qRegisterMetaType@VU2Region@U2@@@@YAHPBDPAVU2Region@U2@@W4DefinedType@?$MetaTypeDefinedHelper@VU2Region@U2@@$00@QtPrivate@@@Z 1000e010 f i ORFMarkerTask.obj
 0001:0000d0d0       ??$qRegisterNormalizedMetaType@VU2Region@U2@@@@YAHABVQByteArray@@PAVU2Region@U2@@W4DefinedType@?$MetaTypeDefinedHelper@VU2Region@U2@@$00@QtPrivate@@@Z 1000e0d0 f i ORFMarkerTask.obj
 0001:0000d130       ??$qVariantFromValue@VU2Region@U2@@@@YA?AVQVariant@@ABVU2Region@U2@@@Z 1000e130 f i ORFMarkerTask.obj
 0001:0000d160       ??$qvariant_cast@VU2Region@U2@@@@YA?AVU2Region@U2@@ABVQVariant@@@Z 1000e160 f i ORFMarkerTask.obj
 0001:0000d180       ??$value@VU2Region@U2@@@QVariant@@QBE?AVU2Region@U2@@XZ 1000e180 f i ORFMarkerTask.obj
 0001:0000d1a0       ??0?$QForeachContainer@$$CBV?$QList@VORFFindResult@U2@@@@@@QAE@ABV?$QList@VORFFindResult@U2@@@@@Z 1000e1a0 f i ORFMarkerTask.obj
 0001:0000d1e0       ??0?$QList@PAVTask@U2@@@@QAE@XZ 1000e1e0 f i ORFMarkerTask.obj
 0001:0000d1f0       ??0?$QList@V?$QSharedDataPointer@VAnnotationData@U2@@@@@@QAE@XZ 1000e1f0 f i ORFMarkerTask.obj
 0001:0000d200       ??0?$QPointer@VAnnotationTableObject@U2@@@@QAE@PAVAnnotationTableObject@U2@@@Z 1000e200 f i ORFMarkerTask.obj
 0001:0000d240       ??0?$QSharedDataPointer@VAnnotationData@U2@@@@QAE@ABV0@@Z 1000e240 f i ORFMarkerTask.obj
 0001:0000d260       ??0FindORFsToAnnotationsTask@U2@@QAE@PAVAnnotationTableObject@1@ABVU2EntityRef@1@ABVORFAlgorithmSettings@1@ABVQString@@3@Z 1000e260 f   ORFMarkerTask.obj
 0001:0000d420       ??0ORFAutoAnnotationsUpdater@U2@@QAE@XZ 1000e420 f   ORFMarkerTask.obj
 0001:0000d4a0       ??1?$QForeachContainer@$$CBV?$QList@VORFFindResult@U2@@@@@@QAE@XZ 1000e4a0 f i ORFMarkerTask.obj
 0001:0000d4b0       ??1?$QList@V?$QSharedDataPointer@VAnnotationData@U2@@@@@@QAE@XZ 1000e4b0 f i ORFMarkerTask.obj
 0001:0000d500       ??1?$QPointer@VAnnotationTableObject@U2@@@@QAE@XZ 1000e500 f i ORFMarkerTask.obj
 0001:0000d520       ??1?$QSharedDataPointer@VAnnotationData@U2@@@@QAE@XZ 1000e520 f i ORFMarkerTask.obj
 0001:0000d550       ??1FindORFsToAnnotationsTask@U2@@UAE@XZ 1000e550 f i ORFMarkerTask.obj
 0001:0000d600       ??1ORFAutoAnnotationsUpdater@U2@@UAE@XZ 1000e600 f i ORFMarkerTask.obj
 0001:0000d610       ??6?$QList@PAVTask@U2@@@@QAEAAV0@ABQAVTask@U2@@@Z 1000e610 f i ORFMarkerTask.obj
 0001:0000d630       ??6?$QList@V?$QSharedDataPointer@VAnnotationData@U2@@@@@@QAEAAV0@ABV?$QSharedDataPointer@VAnnotationData@U2@@@@@Z 1000e630 f i ORFMarkerTask.obj
 0001:0000d650       ??B?$QPointer@VAnnotationTableObject@U2@@@@QBEPAVAnnotationTableObject@U2@@XZ 1000e650 f i ORFMarkerTask.obj
 0001:0000d670       ??_G?$QSharedDataPointer@VAnnotationData@U2@@@@QAEPAXI@Z 1000e670 f i ORFMarkerTask.obj
 0001:0000d6c0       ??_ECreateAnnotationsTask@U2@@UAEPAXI@Z 1000e6c0 f i ORFMarkerTask.obj
 0001:0000d6c0       ??_GCreateAnnotationsTask@U2@@UAEPAXI@Z 1000e6c0 f i ORFMarkerTask.obj
 0001:0000d6f0       ??_EFindORFsToAnnotationsTask@U2@@UAEPAXI@Z 1000e6f0 f i ORFMarkerTask.obj
 0001:0000d6f0       ??_GFindORFsToAnnotationsTask@U2@@UAEPAXI@Z 1000e6f0 f i ORFMarkerTask.obj
 0001:0000d720       ??_EORFAutoAnnotationsUpdater@U2@@UAEPAXI@Z 1000e720 f i ORFMarkerTask.obj
 0001:0000d720       ??_GORFAutoAnnotationsUpdater@U2@@UAEPAXI@Z 1000e720 f i ORFMarkerTask.obj
 0001:0000d750       ?Construct@?$QMetaTypeFunctionHelper@VU2Region@U2@@$00@QtMetaTypePrivate@@SAPAXPAXPBX@Z 1000e750 f i ORFMarkerTask.obj
 0001:0000d790       ?Create@?$QMetaTypeFunctionHelper@VU2Region@U2@@$00@QtMetaTypePrivate@@SAPAXPBX@Z 1000e790 f i ORFMarkerTask.obj
 0001:0000d7e0       ?Delete@?$QMetaTypeFunctionHelper@VU2Region@U2@@$00@QtMetaTypePrivate@@SAXPAX@Z 1000e7e0 f i ORFMarkerTask.obj
 0001:0000d7f0       ?Destruct@?$QMetaTypeFunctionHelper@VU2Region@U2@@$00@QtMetaTypePrivate@@SAXPAX@Z 1000e7f0 f i ORFMarkerTask.obj
 0001:0000d800       ?append@?$QList@PAVTask@U2@@@@QAEXABQAVTask@U2@@@Z 1000e800 f i ORFMarkerTask.obj
 0001:0000d890       ?append@?$QList@V?$QSharedDataPointer@VAnnotationData@U2@@@@@@QAEXABV?$QSharedDataPointer@VAnnotationData@U2@@@@@Z 1000e890 f i ORFMarkerTask.obj
 0001:0000d960       ?checkConstraints@ORFAutoAnnotationsUpdater@U2@@UAE_NABUAutoAnnotationConstraints@2@@Z 1000e960 f   ORFMarkerTask.obj
 0001:0000d980       ?createAutoAnnotationsUpdateTask@ORFAutoAnnotationsUpdater@U2@@UAEPAVTask@2@PBVAutoAnnotationObject@2@@Z 1000e980 f   ORFMarkerTask.obj
 0001:0000db80       ?data@?$QPointer@VAnnotationTableObject@U2@@@@QBEPAVAnnotationTableObject@U2@@XZ 1000eb80 f i ORFMarkerTask.obj
 0001:0000dba0       ?dealloc@?$QList@V?$QSharedDataPointer@VAnnotationData@U2@@@@@@AAEXPAUData@QListData@@@Z 1000eba0 f i ORFMarkerTask.obj
 0001:0000dbd0       ?detach_helper_grow@?$QList@PAVTask@U2@@@@AAEPAUNode@1@HH@Z 1000ebd0 f i ORFMarkerTask.obj
 0001:0000dce0       ?detach_helper_grow@?$QList@V?$QSharedDataPointer@VAnnotationData@U2@@@@@@AAEPAUNode@1@HH@Z 1000ece0 f i ORFMarkerTask.obj
 0001:0000de50       ?invoke@?$MetaTypeInvoker@U?$QVariantValueHelper@VU2Region@U2@@@QtPrivate@@ABVQVariant@@VU2Region@U2@@@QtPrivate@@SA?AVU2Region@U2@@ABVQVariant@@@Z 1000ee50 f i ORFMarkerTask.obj
 0001:0000de70       ?metaType@?$QVariantValueHelper@VU2Region@U2@@@QtPrivate@@SA?AVU2Region@U2@@ABVQVariant@@@Z 1000ee70 f i ORFMarkerTask.obj
 0001:0000df00       ?node_construct@?$QList@PAVTask@U2@@@@AAEXPAUNode@1@ABQAVTask@U2@@@Z 1000ef00 f i ORFMarkerTask.obj
 0001:0000df20       ?node_construct@?$QList@V?$QSharedDataPointer@VAnnotationData@U2@@@@@@AAEXPAUNode@1@ABV?$QSharedDataPointer@VAnnotationData@U2@@@@@Z 1000ef20 f i ORFMarkerTask.obj
 0001:0000df50       ?node_copy@?$QList@V?$QSharedDataPointer@VAnnotationData@U2@@@@@@AAEXPAUNode@1@00@Z 1000ef50 f i ORFMarkerTask.obj
 0001:0000df90       ?node_destruct@?$QList@PAVTask@U2@@@@AAEXPAUNode@1@@Z 1000ef90 f i ORFMarkerTask.obj
 0001:0000dfa0       ?node_destruct@?$QList@V?$QSharedDataPointer@VAnnotationData@U2@@@@@@AAEXPAUNode@1@0@Z 1000efa0 f i ORFMarkerTask.obj
 0001:0000dff0       ?node_destruct@?$QList@V?$QSharedDataPointer@VAnnotationData@U2@@@@@@AAEXPAUNode@1@@Z 1000eff0 f i ORFMarkerTask.obj
 0001:0000e030       ?onSubTaskFinished@FindORFsToAnnotationsTask@U2@@UAE?AV?$QList@PAVTask@U2@@@@PAVTask@2@@Z 1000f030 f   ORFMarkerTask.obj
 0001:0000e420       ?qt_metatype_id@?$QMetaTypeId2@VU2Region@U2@@@@SAHXZ 1000f420 f i ORFMarkerTask.obj
 0001:0000e430       ?qt_metatype_id@?$QMetaTypeId@VU2Region@U2@@@@SAHXZ 1000f430 f i ORFMarkerTask.obj
 0001:0000e4d0       ?qt_metatype_id@?$QMetaTypeIdHelper@VU2Region@U2@@$00@QtPrivate@@SAHXZ 1000f4d0 f i ORFMarkerTask.obj
 0001:0000e4e0       ?read@ORFSettingsKeys@U2@@SAXAAVORFAlgorithmSettings@2@PBVSettings@2@@Z 1000f4e0 f   ORFMarkerTask.obj
 0001:0000e8e0       ?registerConverter@?$AssociativeContainerConverterHelper@VU2Region@U2@@$0A@@QtPrivate@@SA_NH@Z 1000f8e0 f i ORFMarkerTask.obj
 0001:0000e8f0       ?registerConverter@?$IsPair@VU2Region@U2@@@QtPrivate@@SA_NH@Z 1000f8f0 f i ORFMarkerTask.obj
 0001:0000e900       ?registerConverter@?$MetaTypeSmartPointerHelper@VU2Region@U2@@X@QtPrivate@@SA_NH@Z 1000f900 f i ORFMarkerTask.obj
 0001:0000e910       ?registerConverter@?$SequentialContainerConverterHelper@VU2Region@U2@@$0A@@QtPrivate@@SA_NH@Z 1000f910 f i ORFMarkerTask.obj
 0001:0000e920       ?save@ORFSettingsKeys@U2@@SAXABVORFAlgorithmSettings@2@PAVSettings@2@@Z 1000f920 f   ORFMarkerTask.obj
 0001:0000ebd0       ?tr@FindORFsToAnnotationsTask@U2@@SA?AVQString@@PBD0H@Z 1000fbd0 f i ORFMarkerTask.obj
 0001:0000ec00       ?tr@ORFAutoAnnotationsUpdater@U2@@SA?AVQString@@PBD0H@Z 1000fc00 f i ORFMarkerTask.obj
 0001:0000ec30       ?value@?$MetaObjectForType@VU2Region@U2@@$0A@@QtPrivate@@SAPBUQMetaObject@@XZ 1000fc30 f i ORFMarkerTask.obj
 0001:0000ec40       ??$_Move@AAVU2Region@U2@@@std@@YA$$QAVU2Region@U2@@AAV12@@Z 1000fc40 f i ORFMarkerTests.obj
 0001:0000ec50       ??$getContext@VU2SequenceObject@U2@@@GTest@U2@@SAPAVU2SequenceObject@1@PBV01@ABVQString@@@Z 1000fc50 f i ORFMarkerTests.obj
 0001:0000ec70       ??$qSort@V?$QVector@VU2Region@U2@@@@@@YAXAAV?$QVector@VU2Region@U2@@@@@Z 1000fc70 f i ORFMarkerTests.obj
 0001:0000ecc0       ??$qSortHelper@PAVU2Region@U2@@V12@@QAlgorithmsPrivate@@YAXPAVU2Region@U2@@0ABV12@@Z 1000fcc0 f i ORFMarkerTests.obj
 0001:0000ece0       ??$qSortHelper@PAVU2Region@U2@@V12@V?$qLess@VU2Region@U2@@@@@QAlgorithmsPrivate@@YAXPAVU2Region@U2@@0ABV12@V?$qLess@VU2Region@U2@@@@@Z 1000fce0 f i ORFMarkerTests.obj
 0001:0000ee90       ??$qSwap@VU2Region@U2@@@@YAXAAVU2Region@U2@@0@Z 1000fe90 f i ORFMarkerTests.obj
 0001:0000eeb0       ??$qobject_cast@PAVU2SequenceObject@U2@@@@YAPAVU2SequenceObject@U2@@PAVQObject@@@Z 1000feb0 f i ORFMarkerTests.obj
 0001:0000eed0       ??$swap@VU2Region@U2@@@std@@YAXAAVU2Region@U2@@0@Z 1000fed0 f i ORFMarkerTests.obj
 0001:0000eef0       ??0?$QFlags@W4AllocationOption@QArrayData@@@@QAE@W4AllocationOption@QArrayData@@@Z 1000fef0 f i ORFMarkerTests.obj
 0001:0000ef00       ??0?$QForeachContainer@VQStringList@@@@QAE@ABVQStringList@@@Z 1000ff00 f i ORFMarkerTests.obj
 0001:0000ef40       ??0?$QList@VQString@@@@QAE@ABV0@@Z 1000ff40 f i ORFMarkerTests.obj
 0001:0000f000       ??0QStringList@@QAE@ABV0@@Z 10010000 f i ORFMarkerTests.obj
 0001:0000f020       ??0Translator@U2@@QAE@PBVU2SequenceObject@1@ABVQString@@@Z 10010020 f   ORFMarkerTests.obj
 0001:0000f0d0       ??0const_iterator@?$QList@VQString@@@@QAE@PAUNode@1@@Z 100100d0 f i ORFMarkerTests.obj
 0001:0000f0e0       ??0iterator@?$QList@VQString@@@@QAE@PAUNode@1@@Z 100100e0 f i ORFMarkerTests.obj
 0001:0000f0f0       ??1?$QForeachContainer@VQStringList@@@@QAE@XZ 100100f0 f i ORFMarkerTests.obj
 0001:0000f100       ??1?$QList@VQString@@@@QAE@XZ 10010100 f i ORFMarkerTests.obj
 0001:0000f160       ??1QStringList@@QAE@XZ     10010160 f i ORFMarkerTests.obj
 0001:0000f170       ??8?$QVector@VU2Region@U2@@@@QBE_NABV0@@Z 10010170 f i ORFMarkerTests.obj
 0001:0000f210       ??9?$QVector@VU2Region@U2@@@@QBE_NABV0@@Z 10010210 f i ORFMarkerTests.obj
 0001:0000f230       ??9const_iterator@?$QList@VQString@@@@QBE_NABV01@@Z 10010230 f i ORFMarkerTests.obj
 0001:0000f250       ??Dconst_iterator@?$QList@VQString@@@@QBEABVQString@@XZ 10010250 f i ORFMarkerTests.obj
 0001:0000f260       ??Diterator@?$QList@VQString@@@@QBEAAVQString@@XZ 10010260 f i ORFMarkerTests.obj
 0001:0000f270       ??Econst_iterator@?$QList@VQString@@@@QAEAAV01@XZ 10010270 f i ORFMarkerTests.obj
 0001:0000f280       ??Fiterator@?$QList@VQString@@@@QAEAAV01@XZ 10010280 f i ORFMarkerTests.obj
 0001:0000f290       ??R?$qLess@VU2Region@U2@@@@QBE_NABVU2Region@U2@@0@Z 10010290 f i ORFMarkerTests.obj
 0001:0000f2c0       ??_GQString@@QAEPAXI@Z     100102c0 f i ORFMarkerTests.obj
 0001:0000f2f0       ?allocate@?$QTypedArrayData@VU2Region@U2@@@@SAPAU1@IV?$QFlags@W4AllocationOption@QArrayData@@@@@Z 100102f0 f i ORFMarkerTests.obj
 0001:0000f310       ?append@?$QVector@VU2Region@U2@@@@QAEXABVU2Region@U2@@@Z 10010310 f i ORFMarkerTests.obj
 0001:0000f390       ?begin@?$QList@VQString@@@@QAE?AViterator@1@XZ 10010390 f i ORFMarkerTests.obj
 0001:0000f3d0       ?begin@?$QList@VQString@@@@QBE?AVconst_iterator@1@XZ 100103d0 f i ORFMarkerTests.obj
 0001:0000f3f0       ?begin@?$QVector@VU2Region@U2@@@@QAEPAVU2Region@U2@@XZ 100103f0 f i ORFMarkerTests.obj
 0001:0000f450       ?dealloc@?$QList@VQString@@@@AAEXPAUData@QListData@@@Z 10010450 f i ORFMarkerTests.obj
 0001:0000f490       ?defaultConstruct@?$QVector@VU2Region@U2@@@@AAEXPAVU2Region@U2@@0@Z 10010490 f i ORFMarkerTests.obj
 0001:0000f4b0       ?detach@?$QList@VQString@@@@QAEXXZ 100104b0 f i ORFMarkerTests.obj
 0001:0000f4d0       ?detach@?$QVector@VU2Region@U2@@@@QAEXXZ 100104d0 f i ORFMarkerTests.obj
 0001:0000f520       ?detach_helper@?$QList@VQString@@@@AAEXH@Z 10010520 f i ORFMarkerTests.obj
 0001:0000f610       ?detach_helper@?$QList@VQString@@@@AAEXXZ 10010610 f i ORFMarkerTests.obj
 0001:0000f620       ?empty@?$QVector@VU2Region@U2@@@@QBE_NXZ 10010620 f i ORFMarkerTests.obj
 0001:0000f630       ?end@?$QList@VQString@@@@QAE?AViterator@1@XZ 10010630 f i ORFMarkerTests.obj
 0001:0000f670       ?end@?$QList@VQString@@@@QBE?AVconst_iterator@1@XZ 10010670 f i ORFMarkerTests.obj
 0001:0000f690       ?end@?$QVector@VU2Region@U2@@@@QAEPAVU2Region@U2@@XZ 10010690 f i ORFMarkerTests.obj
 0001:0000f710       ?first@?$QList@VQString@@@@QAEAAVQString@@XZ 10010710 f i ORFMarkerTests.obj
 0001:0000f740       ?getAminoTranslation@Translator@U2@@QBEPAVDNATranslation@2@XZ 10010740 f i ORFMarkerTests.obj
 0001:0000f750       ?getComplTranslation@Translator@U2@@QBEPAVDNATranslation@2@XZ 10010750 f i ORFMarkerTests.obj
 0001:0000f760       ?init@GTest_ORFMarkerTask@U2@@QAEXPAVXMLTestFormat@2@ABVQDomElement@@@Z 10010760 f   ORFMarkerTests.obj
 0001:000103d0       ?isDetached@?$QVector@VU2Region@U2@@@@QBE_NXZ 100113d0 f i ORFMarkerTests.obj
 0001:00010400       ?last@?$QList@VQString@@@@QAEAAVQString@@XZ 10011400 f i ORFMarkerTests.obj
 0001:00010430       ?node_copy@?$QList@VQString@@@@AAEXPAUNode@1@00@Z 10011430 f i ORFMarkerTests.obj
 0001:000104d0       ?node_destruct@?$QList@VQString@@@@AAEXPAUNode@1@0@Z 100114d0 f i ORFMarkerTests.obj
 0001:00010500       ?prepare@GTest_ORFMarkerTask@U2@@UAEXXZ 10011500 f   ORFMarkerTests.obj
 0001:00010680       ?reallocData@?$QVector@VU2Region@U2@@@@AAEXHHV?$QFlags@W4AllocationOption@QArrayData@@@@@Z 10011680 f i ORFMarkerTests.obj
 0001:000108c0       ?report@GTest_ORFMarkerTask@U2@@UAE?AW4ReportResult@Task@2@XZ 100118c0 f   ORFMarkerTests.obj
 0001:00010da0       ?size@?$QList@VQString@@@@QBEHXZ 10011da0 f i ORFMarkerTests.obj
 0001:00010db0       ?size@?$QVector@VU2Region@U2@@@@QBEHXZ 10011db0 f i ORFMarkerTests.obj
 0001:00010dc0       ?t@Node@?$QList@VQString@@@@QAEAAVQString@@XZ 10011dc0 f i ORFMarkerTests.obj
 0001:00010dd0       ?unsharableEmpty@?$QTypedArrayData@VU2Region@U2@@@@SAPAU1@XZ 10011dd0 f i ORFMarkerTests.obj
 0001:00010df0       ??$_Move@AAPAU?$QTypedArrayData@VU2Qualifier@U2@@@@@std@@YA$$QAPAU?$QTypedArrayData@VU2Qualifier@U2@@@@AAPAU1@@Z 10011df0 f i ORFQuery.obj
 0001:00010e00       ??$getAttributeValueWithoutScript@H@Attribute@U2@@QBEHXZ 10011e00 f i ORFQuery.obj
 0001:00010e40       ??$getAttributeValueWithoutScript@VQString@@@Attribute@U2@@QBE?AVQString@@XZ 10011e40 f i ORFQuery.obj
 0001:00010e60       ??$qMapLessThanKey@VQString@@@@YA_NABVQString@@0@Z 10011e60 f i ORFQuery.obj
 0001:00010e70       ??$qMetaTypeId@H@@YAHXZ    10011e70 f i ORFQuery.obj
 0001:00010e80       ??$qMetaTypeId@VQString@@@@YAHXZ 10011e80 f i ORFQuery.obj
 0001:00010e90       ??$qSwap@PAU?$QTypedArrayData@VU2Qualifier@U2@@@@@@YAXAAPAU?$QTypedArrayData@VU2Qualifier@U2@@@@0@Z 10011e90 f i ORFQuery.obj
 0001:00010eb0       ??$qvariant_cast@H@@YAHABVQVariant@@@Z 10011eb0 f i ORFQuery.obj
 0001:00010ef0       ??$qvariant_cast@VQString@@@@YA?AVQString@@ABVQVariant@@@Z 10011ef0 f i ORFQuery.obj
 0001:00010f10       ??$swap@PAU?$QTypedArrayData@VU2Qualifier@U2@@@@@std@@YAXAAPAU?$QTypedArrayData@VU2Qualifier@U2@@@@0@Z 10011f10 f i ORFQuery.obj
 0001:00010f30       ??$value@H@QVariant@@QBEHXZ 10011f30 f i ORFQuery.obj
 0001:00010f70       ??$value@VQString@@@QVariant@@QBE?AVQString@@XZ 10011f70 f i ORFQuery.obj
 0001:00010f90       ??0?$QForeachContainer@$$CBV?$QVector@VU2Region@U2@@@@@@QAE@ABV?$QVector@VU2Region@U2@@@@@Z 10011f90 f i ORFQuery.obj
 0001:00011010       ??0?$QForeachContainer@V?$QList@PAVDNATranslation@U2@@@@@@QAE@ABV?$QList@PAVDNATranslation@U2@@@@@Z 10012010 f i ORFQuery.obj
 0001:00011050       ??0?$QForeachContainer@V?$QList@PAVORFFindTask@U2@@@@@@QAE@ABV?$QList@PAVORFFindTask@U2@@@@@Z 10012050 f i ORFQuery.obj
 0001:00011090       ??0?$QForeachContainer@V?$QList@V?$QSharedDataPointer@VAnnotationData@U2@@@@@@@@QAE@ABV?$QList@V?$QSharedDataPointer@VAnnotationData@U2@@@@@@@Z 10012090 f i ORFQuery.obj
 0001:000110d0       ??0?$QList@PAVDNATranslation@U2@@@@QAE@ABV0@@Z 100120d0 f i ORFQuery.obj
 0001:00011190       ??0?$QList@PAVORFFindTask@U2@@@@QAE@ABV0@@Z 10012190 f i ORFQuery.obj
 0001:00011250       ??0?$QList@PAVORFFindTask@U2@@@@QAE@XZ 10012250 f i ORFQuery.obj
 0001:00011260       ??0?$QList@V?$QSharedDataPointer@VAnnotationData@U2@@@@@@QAE@ABV0@@Z 10012260 f i ORFQuery.obj
 0001:00011320       ??0?$QList@VORFFindResult@U2@@@@QAE@XZ 10012320 f i ORFQuery.obj
 0001:00011330       ??0?$QMap@VQString@@PAVPropertyDelegate@U2@@@@QAE@XZ 10012330 f i ORFQuery.obj
 0001:00011340       ??0?$QMap@VQString@@VQVariant@@@@QAE@XZ 10012340 f i ORFQuery.obj
 0001:00011350       ??0?$QSharedDataPointer@VQDResultUnitData@U2@@@@QAE@PAVQDResultUnitData@U2@@@Z 10012350 f i ORFQuery.obj
 0001:00011370       ??0?$QVector@VU2Qualifier@U2@@@@QAE@ABV0@@Z 10012370 f i ORFQuery.obj
 0001:00011430       ??0?$QVector@VU2Region@U2@@@@QAE@ABV0@@Z 10012430 f i ORFQuery.obj
 0001:000114f0       ??0QDORFActor@U2@@QAE@PBVQDActorPrototype@1@@Z 100124f0 f   ORFQuery.obj
 0001:00011640       ??0QDORFActorPrototype@U2@@QAE@XZ 10012640 f   ORFQuery.obj
 0001:000123e0       ??0const_iterator@?$QList@PAVDNATranslation@U2@@@@QAE@PAUNode@1@@Z 100133e0 f i ORFQuery.obj
 0001:000123f0       ??0const_iterator@?$QList@PAVORFFindTask@U2@@@@QAE@PAUNode@1@@Z 100133f0 f i ORFQuery.obj
 0001:00012400       ??0const_iterator@?$QList@V?$QSharedDataPointer@VAnnotationData@U2@@@@@@QAE@PAUNode@1@@Z 10013400 f i ORFQuery.obj
 0001:00012410       ??0iterator@?$QMap@VQString@@PAVPropertyDelegate@U2@@@@QAE@PAU?$QMapNode@VQString@@PAVPropertyDelegate@U2@@@@@Z 10013410 f i ORFQuery.obj
 0001:00012420       ??0iterator@?$QMap@VQString@@PAVQDSchemeUnit@U2@@@@QAE@PAU?$QMapNode@VQString@@PAVQDSchemeUnit@U2@@@@@Z 10013420 f i ORFQuery.obj
 0001:00012430       ??0iterator@?$QMap@VQString@@VQVariant@@@@QAE@PAU?$QMapNode@VQString@@VQVariant@@@@@Z 10013430 f i ORFQuery.obj
 0001:00012440       ??1?$QExplicitlySharedDataPointer@VDataType@U2@@@@QAE@XZ 10013440 f i ORFQuery.obj
 0001:00012460       ??1?$QForeachContainer@$$CBV?$QVector@VU2Region@U2@@@@@@QAE@XZ 10013460 f i ORFQuery.obj
 0001:000124a0       ??1?$QForeachContainer@V?$QList@PAVDNATranslation@U2@@@@@@QAE@XZ 100134a0 f i ORFQuery.obj
 0001:000124d0       ??1?$QForeachContainer@V?$QList@PAVORFFindTask@U2@@@@@@QAE@XZ 100134d0 f i ORFQuery.obj
 0001:00012500       ??1?$QForeachContainer@V?$QList@V?$QSharedDataPointer@VAnnotationData@U2@@@@@@@@QAE@XZ 10013500 f i ORFQuery.obj
 0001:00012550       ??1?$QList@PAVDNATranslation@U2@@@@QAE@XZ 10013550 f i ORFQuery.obj
 0001:00012580       ??1?$QList@PAVORFFindTask@U2@@@@QAE@XZ 10013580 f i ORFQuery.obj
 0001:000125b0       ??1?$QMap@VQString@@PAVAttribute@U2@@@@QAE@XZ 100135b0 f i ORFQuery.obj
 0001:00012620       ??1?$QMap@VQString@@PAVPropertyDelegate@U2@@@@QAE@XZ 10013620 f i ORFQuery.obj
 0001:00012690       ??1?$QMap@VQString@@VQVariant@@@@QAE@XZ 10013690 f i ORFQuery.obj
 0001:000126e0       ??1?$QSharedDataPointer@VQDResultUnitData@U2@@@@QAE@XZ 100136e0 f i ORFQuery.obj
 0001:00012710       ??1?$QVector@VU2Qualifier@U2@@@@QAE@XZ 10013710 f i ORFQuery.obj
 0001:00012780       ??1QDORFActor@U2@@UAE@XZ   10013780 f i ORFQuery.obj
 0001:00012800       ??1QDORFActorPrototype@U2@@UAE@XZ 10013800 f i ORFQuery.obj
 0001:00012810       ??4?$QList@PAVORFFindTask@U2@@@@QAEAAV0@$$QAV0@@Z 10013810 f i ORFQuery.obj
 0001:00012830       ??4?$QList@VORFFindResult@U2@@@@QAEAAV0@ABV0@@Z 10013830 f i ORFQuery.obj
 0001:00012870       ??4?$QVector@VU2Qualifier@U2@@@@QAEAAV0@ABV0@@Z 10013870 f i ORFQuery.obj
 0001:000128b0       ??6?$QList@PAVAttribute@U2@@@@QAEAAV0@ABQAVAttribute@U2@@@Z 100138b0 f i ORFQuery.obj
 0001:000128d0       ??6?$QList@VORFFindResult@U2@@@@QAEAAV0@ABV0@@Z 100138d0 f i ORFQuery.obj
 0001:000128f0       ??9const_iterator@?$QList@PAVDNATranslation@U2@@@@QBE_NABV01@@Z 100138f0 f i ORFQuery.obj
 0001:00012910       ??9const_iterator@?$QList@PAVORFFindTask@U2@@@@QBE_NABV01@@Z 10013910 f i ORFQuery.obj
 0001:00012930       ??9const_iterator@?$QList@V?$QSharedDataPointer@VAnnotationData@U2@@@@@@QBE_NABV01@@Z 10013930 f i ORFQuery.obj
 0001:00012950       ??A?$QMap@VQString@@PAVPropertyDelegate@U2@@@@QAEAAPAVPropertyDelegate@U2@@ABVQString@@@Z 10013950 f i ORFQuery.obj
 0001:000129d0       ??A?$QMap@VQString@@PAVQDSchemeUnit@U2@@@@QAEAAPAVQDSchemeUnit@U2@@ABVQString@@@Z 100139d0 f i ORFQuery.obj
 0001:00012a50       ??A?$QMap@VQString@@VQVariant@@@@QAEAAVQVariant@@ABVQString@@@Z 10013a50 f i ORFQuery.obj
 0001:00012b20       ??A?$QVector@VU2Region@U2@@@@QBEABVU2Region@U2@@H@Z 10013b20 f i ORFQuery.obj
 0001:00012b40       ??C?$QSharedDataPointer@VAnnotationData@U2@@@@QBEPBVAnnotationData@U2@@XZ 10013b40 f i ORFQuery.obj
 0001:00012b50       ??C?$QSharedDataPointer@VQDResultUnitData@U2@@@@QAEPAVQDResultUnitData@U2@@XZ 10013b50 f i ORFQuery.obj
 0001:00012b70       ??Dconst_iterator@?$QList@PAVDNATranslation@U2@@@@QBEABQAVDNATranslation@U2@@XZ 10013b70 f i ORFQuery.obj
 0001:00012b80       ??Dconst_iterator@?$QList@PAVORFFindTask@U2@@@@QBEABQAVORFFindTask@U2@@XZ 10013b80 f i ORFQuery.obj
 0001:00012b90       ??Dconst_iterator@?$QList@V?$QSharedDataPointer@VAnnotationData@U2@@@@@@QBEABV?$QSharedDataPointer@VAnnotationData@U2@@@@XZ 10013b90 f i ORFQuery.obj
 0001:00012ba0       ??Diterator@?$QMap@VQString@@PAVPropertyDelegate@U2@@@@QBEAAPAVPropertyDelegate@U2@@XZ 10013ba0 f i ORFQuery.obj
 0001:00012bb0       ??Diterator@?$QMap@VQString@@PAVQDSchemeUnit@U2@@@@QBEAAPAVQDSchemeUnit@U2@@XZ 10013bb0 f i ORFQuery.obj
 0001:00012bc0       ??Diterator@?$QMap@VQString@@VQVariant@@@@QBEAAVQVariant@@XZ 10013bc0 f i ORFQuery.obj
 0001:00012bd0       ??Econst_iterator@?$QList@PAVDNATranslation@U2@@@@QAEAAV01@XZ 10013bd0 f i ORFQuery.obj
 0001:00012be0       ??Econst_iterator@?$QList@PAVORFFindTask@U2@@@@QAEAAV01@XZ 10013be0 f i ORFQuery.obj
 0001:00012bf0       ??Econst_iterator@?$QList@V?$QSharedDataPointer@VAnnotationData@U2@@@@@@QAEAAV01@XZ 10013bf0 f i ORFQuery.obj
 0001:00012c00       ??Y?$QList@VORFFindResult@U2@@@@QAEAAV0@ABV0@@Z 10013c00 f i ORFQuery.obj
 0001:00012d00       ??_GAttribute@U2@@UAEPAXI@Z 10013d00 f i ORFQuery.obj
 0001:00012d00       ??_EAttribute@U2@@UAEPAXI@Z 10013d00 f i ORFQuery.obj
 0001:00012d30       ??_EComboBoxDelegate@U2@@UAEPAXI@Z 10013d30 f i ORFQuery.obj
 0001:00012d30       ??_GComboBoxDelegate@U2@@UAEPAXI@Z 10013d30 f i ORFQuery.obj
 0001:00012d60       ??_GDelegateEditor@U2@@UAEPAXI@Z 10013d60 f i ORFQuery.obj
 0001:00012d60       ??_EDelegateEditor@U2@@UAEPAXI@Z 10013d60 f i ORFQuery.obj
 0001:00012d90       ??_EFailTask@U2@@UAEPAXI@Z 10013d90 f i ORFQuery.obj
 0001:00012d90       ??_GFailTask@U2@@UAEPAXI@Z 10013d90 f i ORFQuery.obj
 0001:00012dc0       ??_GQDORFActor@U2@@UAEPAXI@Z 10013dc0 f i ORFQuery.obj
 0001:00012dc0       ??_EQDORFActor@U2@@UAEPAXI@Z 10013dc0 f i ORFQuery.obj
 0001:00012e50       ??_EQDORFActorPrototype@U2@@UAEPAXI@Z 10013e50 f i ORFQuery.obj
 0001:00012e50       ??_GQDORFActorPrototype@U2@@UAEPAXI@Z 10013e50 f i ORFQuery.obj
 0001:00012e80       ??_GQDResultUnitData@U2@@QAEPAXI@Z 10013e80 f i ORFQuery.obj
 0001:00012eb0       ??_GQVariant@@QAEPAXI@Z    10013eb0 f i ORFQuery.obj
 0001:00012ee0       ??_ESpinBoxDelegate@U2@@UAEPAXI@Z 10013ee0 f i ORFQuery.obj
 0001:00012ee0       ??_GSpinBoxDelegate@U2@@UAEPAXI@Z 10013ee0 f i ORFQuery.obj
 0001:00012f10       ??_GTask@U2@@UAEPAXI@Z     10013f10 f i ORFQuery.obj
 0001:00012f10       ??_ETask@U2@@UAEPAXI@Z     10013f10 f i ORFQuery.obj
 0001:00012f40       ??_ETaskSignalMapper@U2@@UAEPAXI@Z 10013f40 f i ORFQuery.obj
 0001:00012f40       ??_GTaskSignalMapper@U2@@UAEPAXI@Z 10013f40 f i ORFQuery.obj
 0001:00012f70       ??_GU2Qualifier@U2@@QAEPAXI@Z 10013f70 f i ORFQuery.obj
 0001:00012fa0       ?allocate@?$QTypedArrayData@VU2Qualifier@U2@@@@SAPAU1@IV?$QFlags@W4AllocationOption@QArrayData@@@@@Z 10013fa0 f i ORFQuery.obj
 0001:00012fc0       ?append@?$QList@PAVAttribute@U2@@@@QAEXABQAVAttribute@U2@@@Z 10013fc0 f i ORFQuery.obj
 0001:00013050       ?append@?$QList@PAVORFFindTask@U2@@@@QAEXABQAVORFFindTask@U2@@@Z 10014050 f i ORFQuery.obj
 0001:000130e0       ?begin@?$QList@PAVDNATranslation@U2@@@@QBE?AVconst_iterator@1@XZ 100140e0 f i ORFQuery.obj
 0001:00013100       ?begin@?$QList@PAVORFFindTask@U2@@@@QBE?AVconst_iterator@1@XZ 10014100 f i ORFQuery.obj
 0001:00013120       ?begin@?$QList@V?$QSharedDataPointer@VAnnotationData@U2@@@@@@QBE?AVconst_iterator@1@XZ 10014120 f i ORFQuery.obj
 0001:00013140       ?begin@?$QTypedArrayData@VU2Qualifier@U2@@@@QAEPAVU2Qualifier@U2@@PAV23@@Z 10014140 f i ORFQuery.obj
 0001:00013150       ?begin@?$QVector@VU2Region@U2@@@@QBEPBVU2Region@U2@@XZ 10014150 f i ORFQuery.obj
 0001:00013160       ?clear@?$QList@PAVORFFindTask@U2@@@@QAEXXZ 10014160 f i ORFQuery.obj
 0001:00013190       ?clone@?$QSharedDataPointer@VQDResultUnitData@U2@@@@IAEPAVQDResultUnitData@U2@@XZ 10014190 f i ORFQuery.obj
 0001:00013200       ?constBegin@?$QTypedArrayData@VU2Region@U2@@@@QBEPBVU2Region@U2@@PBV23@@Z 10014200 f i ORFQuery.obj
 0001:00013210       ?constEnd@?$QTypedArrayData@VU2Region@U2@@@@QBEPBVU2Region@U2@@PBV23@@Z 10014210 f i ORFQuery.obj
 0001:00013230       ?copy@?$QMapNode@VQString@@PAVPropertyDelegate@U2@@@@QBEPAU1@PAU?$QMapData@VQString@@PAVPropertyDelegate@U2@@@@@Z 10014230 f i ORFQuery.obj
 0001:000132c0       ?copy@?$QMapNode@VQString@@PAVQDSchemeUnit@U2@@@@QBEPAU1@PAU?$QMapData@VQString@@PAVQDSchemeUnit@U2@@@@@Z 100142c0 f i ORFQuery.obj
 0001:00013350       ?copy@?$QMapNode@VQString@@VQVariant@@@@QBEPAU1@PAU?$QMapData@VQString@@VQVariant@@@@@Z 10014350 f i ORFQuery.obj
 0001:000133e0       ?copyConstruct@?$QVector@VU2Qualifier@U2@@@@AAEXPBVU2Qualifier@U2@@0PAV23@@Z 100143e0 f i ORFQuery.obj
 0001:00013460       ?copyConstruct@?$QVector@VU2Region@U2@@@@AAEXPBVU2Region@U2@@0PAV23@@Z 10014460 f i ORFQuery.obj
 0001:00013480       ?create@?$QMapData@VQString@@PAVPropertyDelegate@U2@@@@SAPAU1@XZ 10014480 f i ORFQuery.obj
 0001:00013490       ?create@?$QMapData@VQString@@PAVQDSchemeUnit@U2@@@@SAPAU1@XZ 10014490 f i ORFQuery.obj
 0001:000134a0       ?create@?$QMapData@VQString@@VQVariant@@@@SAPAU1@XZ 100144a0 f i ORFQuery.obj
 0001:000134b0       ?createInstance@QDORFActorPrototype@U2@@UBEPAVQDActor@2@XZ 100144b0 f i ORFQuery.obj
 0001:00013520       ?createNode@?$QMapData@VQString@@PAVPropertyDelegate@U2@@@@QAEPAU?$QMapNode@VQString@@PAVPropertyDelegate@U2@@@@ABVQString@@ABQAVPropertyDelegate@U2@@PAU2@_N@Z 10014520 f i ORFQuery.obj
 0001:000135c0       ?createNode@?$QMapData@VQString@@PAVQDSchemeUnit@U2@@@@QAEPAU?$QMapNode@VQString@@PAVQDSchemeUnit@U2@@@@ABVQString@@ABQAVQDSchemeUnit@U2@@PAU2@_N@Z 100145c0 f i ORFQuery.obj
 0001:00013660       ?createNode@?$QMapData@VQString@@VQVariant@@@@QAEPAU?$QMapNode@VQString@@VQVariant@@@@ABVQString@@ABVQVariant@@PAU2@_N@Z 10014660 f i ORFQuery.obj
 0001:00013720       ?data@?$QTypedArrayData@VU2Qualifier@U2@@@@QAEPAVU2Qualifier@U2@@XZ 10014720 f i ORFQuery.obj
 0001:00013730       ?data@?$QTypedArrayData@VU2Region@U2@@@@QBEPBVU2Region@U2@@XZ 10014730 f i ORFQuery.obj
 0001:00013740       ?dealloc@?$QList@PAVAttribute@U2@@@@AAEXPAUData@QListData@@@Z 10014740 f i ORFQuery.obj
 0001:00013760       ?dealloc@?$QList@PAVDNATranslation@U2@@@@AAEXPAUData@QListData@@@Z 10014760 f i ORFQuery.obj
 0001:00013780       ?dealloc@?$QList@PAVORFFindTask@U2@@@@AAEXPAUData@QListData@@@Z 10014780 f i ORFQuery.obj
 0001:000137a0       ?deallocate@?$QTypedArrayData@VU2Qualifier@U2@@@@SAXPAUQArrayData@@@Z 100147a0 f i ORFQuery.obj
 0001:000137c0       ?defaultColor@QDORFActor@U2@@UBE?AVQColor@@XZ 100147c0 f i ORFQuery.obj
 0001:000137f0       ?destroy@?$QMapData@VQString@@PAVAttribute@U2@@@@QAEXXZ 100147f0 f i ORFQuery.obj
 0001:00013840       ?destroy@?$QMapData@VQString@@PAVPropertyDelegate@U2@@@@QAEXXZ 10014840 f i ORFQuery.obj
 0001:00013890       ?destroy@?$QMapData@VQString@@PAVQDSchemeUnit@U2@@@@QAEXXZ 10014890 f i ORFQuery.obj
 0001:000138e0       ?destroy@?$QMapData@VQString@@VQVariant@@@@QAEXXZ 100148e0 f i ORFQuery.obj
 0001:00013910       ?destroySubTree@?$QMapNode@VQString@@PAVAttribute@U2@@@@QAEXXZ 10014910 f i ORFQuery.obj
 0001:00013940       ?destroySubTree@?$QMapNode@VQString@@PAVPropertyDelegate@U2@@@@QAEXXZ 10014940 f i ORFQuery.obj
 0001:00013970       ?destroySubTree@?$QMapNode@VQString@@PAVQDSchemeUnit@U2@@@@QAEXXZ 10014970 f i ORFQuery.obj
 0001:000139a0       ?destroySubTree@?$QMapNode@VQString@@VQVariant@@@@QAEXXZ 100149a0 f i ORFQuery.obj
 0001:000139e0       ?destruct@?$QVector@VU2Qualifier@U2@@@@AAEXPAVU2Qualifier@U2@@0@Z 100149e0 f i ORFQuery.obj
 0001:00013a10       ?detach@?$QMap@VQString@@PAVPropertyDelegate@U2@@@@QAEXXZ 10014a10 f i ORFQuery.obj
 0001:00013a30       ?detach@?$QMap@VQString@@PAVQDSchemeUnit@U2@@@@QAEXXZ 10014a30 f i ORFQuery.obj
 0001:00013a50       ?detach@?$QMap@VQString@@VQVariant@@@@QAEXXZ 10014a50 f i ORFQuery.obj
 0001:00013a70       ?detach@?$QSharedDataPointer@VQDResultUnitData@U2@@@@QAEXXZ 10014a70 f i ORFQuery.obj
 0001:00013a80       ?detach_helper@?$QMap@VQString@@PAVPropertyDelegate@U2@@@@AAEXXZ 10014a80 f i ORFQuery.obj
 0001:00013b30       ?detach_helper@?$QMap@VQString@@PAVQDSchemeUnit@U2@@@@AAEXXZ 10014b30 f i ORFQuery.obj
 0001:00013be0       ?detach_helper@?$QMap@VQString@@VQVariant@@@@AAEXXZ 10014be0 f i ORFQuery.obj
 0001:00013c60       ?detach_helper@?$QSharedDataPointer@VQDResultUnitData@U2@@@@AAEXXZ 10014c60 f i ORFQuery.obj
 0001:00013d00       ?detach_helper_grow@?$QList@PAVAttribute@U2@@@@AAEPAUNode@1@HH@Z 10014d00 f i ORFQuery.obj
 0001:00013e10       ?detach_helper_grow@?$QList@PAVORFFindTask@U2@@@@AAEPAUNode@1@HH@Z 10014e10 f i ORFQuery.obj
 0001:00013f20       ?detach_helper_grow@?$QList@VORFFindResult@U2@@@@AAEPAUNode@1@HH@Z 10014f20 f i ORFQuery.obj
 0001:000140a0       ?end@?$QList@PAVDNATranslation@U2@@@@QBE?AVconst_iterator@1@XZ 100150a0 f i ORFQuery.obj
 0001:000140c0       ?end@?$QList@PAVORFFindTask@U2@@@@QBE?AVconst_iterator@1@XZ 100150c0 f i ORFQuery.obj
 0001:000140e0       ?end@?$QList@V?$QSharedDataPointer@VAnnotationData@U2@@@@@@QBE?AVconst_iterator@1@XZ 100150e0 f i ORFQuery.obj
 0001:00014100       ?end@?$QMapData@VQString@@PAVPropertyDelegate@U2@@@@QAEPAU?$QMapNode@VQString@@PAVPropertyDelegate@U2@@@@XZ 10015100 f i ORFQuery.obj
 0001:00014110       ?end@?$QMapData@VQString@@PAVQDSchemeUnit@U2@@@@QAEPAU?$QMapNode@VQString@@PAVQDSchemeUnit@U2@@@@XZ 10015110 f i ORFQuery.obj
 0001:00014120       ?end@?$QMapData@VQString@@VQVariant@@@@QAEPAU?$QMapNode@VQString@@VQVariant@@@@XZ 10015120 f i ORFQuery.obj
 0001:00014130       ?end@?$QTypedArrayData@VU2Qualifier@U2@@@@QAEPAVU2Qualifier@U2@@PAV23@@Z 10015130 f i ORFQuery.obj
 0001:00014150       ?end@?$QVector@VU2Region@U2@@@@QBEPBVU2Region@U2@@XZ 10015150 f i ORFQuery.obj
 0001:00014170       ?findNode@?$QMapData@VQString@@PAVAttribute@U2@@@@QBEPAU?$QMapNode@VQString@@PAVAttribute@U2@@@@ABVQString@@@Z 10015170 f i ORFQuery.obj
 0001:000141b0       ?findNode@?$QMapData@VQString@@PAVPropertyDelegate@U2@@@@QBEPAU?$QMapNode@VQString@@PAVPropertyDelegate@U2@@@@ABVQString@@@Z 100151b0 f i ORFQuery.obj
 0001:000141f0       ?findNode@?$QMapData@VQString@@PAVQDSchemeUnit@U2@@@@QBEPAU?$QMapNode@VQString@@PAVQDSchemeUnit@U2@@@@ABVQString@@@Z 100151f0 f i ORFQuery.obj
 0001:00014230       ?findNode@?$QMapData@VQString@@VQVariant@@@@QBEPAU?$QMapNode@VQString@@VQVariant@@@@ABVQString@@@Z 10015230 f i ORFQuery.obj
 0001:00014270       ?freeData@?$QVector@VU2Qualifier@U2@@@@AAEXPAU?$QTypedArrayData@VU2Qualifier@U2@@@@@Z 10015270 f i ORFQuery.obj
 0001:000142c0       ?getAlgorithmTask@QDORFActor@U2@@UAEPAVTask@2@ABV?$QVector@VU2Region@U2@@@@@Z 100152c0 f   ORFQuery.obj
 0001:00014870       ?getIcon@QDORFActorPrototype@U2@@UBE?AVQIcon@@XZ 10015870 f i ORFQuery.obj
 0001:000148f0       ?getMaxResultLen@QDORFActor@U2@@UBEHXZ 100158f0 f   ORFQuery.obj
 0001:00014940       ?getMinResultLen@QDORFActor@U2@@UBEHXZ 10015940 f   ORFQuery.obj
 0001:00014990       ?getText@QDORFActor@U2@@UBE?AVQString@@XZ 10015990 f   ORFQuery.obj
 0001:00015000       ?insert@?$QMap@VQString@@PAVPropertyDelegate@U2@@@@QAE?AViterator@1@ABVQString@@ABQAVPropertyDelegate@U2@@@Z 10016000 f i ORFQuery.obj
 0001:000150c0       ?insert@?$QMap@VQString@@PAVQDSchemeUnit@U2@@@@QAE?AViterator@1@ABVQString@@ABQAVQDSchemeUnit@U2@@@Z 100160c0 f i ORFQuery.obj
 0001:00015180       ?insert@?$QMap@VQString@@VQVariant@@@@QAE?AViterator@1@ABVQString@@ABVQVariant@@@Z 10016180 f i ORFQuery.obj
 0001:00015240       ?invoke@?$MetaTypeInvoker@U?$QVariantValueHelper@H@QtPrivate@@ABVQVariant@@H@QtPrivate@@SAHABVQVariant@@@Z 10016240 f i ORFQuery.obj
 0001:00015280       ?invoke@?$MetaTypeInvoker@U?$QVariantValueHelper@VQString@@@QtPrivate@@ABVQVariant@@VQString@@@QtPrivate@@SA?AVQString@@ABVQVariant@@@Z 10016280 f i ORFQuery.obj
 0001:000152a0       ?leftNode@?$QMapNode@VQString@@PAVAttribute@U2@@@@QBEPAU1@XZ 100162a0 f i ORFQuery.obj
 0001:000152b0       ?leftNode@?$QMapNode@VQString@@PAVPropertyDelegate@U2@@@@QBEPAU1@XZ 100162b0 f i ORFQuery.obj
 0001:000152c0       ?leftNode@?$QMapNode@VQString@@PAVQDSchemeUnit@U2@@@@QBEPAU1@XZ 100162c0 f i ORFQuery.obj
 0001:000152d0       ?leftNode@?$QMapNode@VQString@@VQVariant@@@@QBEPAU1@XZ 100162d0 f i ORFQuery.obj
 0001:000152e0       ?lowerBound@?$QMapNode@VQString@@PAVAttribute@U2@@@@QAEPAU1@ABVQString@@@Z 100162e0 f i ORFQuery.obj
 0001:00015320       ?lowerBound@?$QMapNode@VQString@@PAVPropertyDelegate@U2@@@@QAEPAU1@ABVQString@@@Z 10016320 f i ORFQuery.obj
 0001:00015360       ?lowerBound@?$QMapNode@VQString@@PAVQDSchemeUnit@U2@@@@QAEPAU1@ABVQString@@@Z 10016360 f i ORFQuery.obj
 0001:000153a0       ?lowerBound@?$QMapNode@VQString@@VQVariant@@@@QAEPAU1@ABVQString@@@Z 100163a0 f i ORFQuery.obj
 0001:000153e0       ?metaType@?$QVariantValueHelper@H@QtPrivate@@SAHABVQVariant@@@Z 100163e0 f i ORFQuery.obj
 0001:00015420       ?metaType@?$QVariantValueHelper@VQString@@@QtPrivate@@SA?AVQString@@ABVQVariant@@@Z 10016420 f i ORFQuery.obj
 0001:000154e0       ?node_construct@?$QList@PAVAttribute@U2@@@@AAEXPAUNode@1@ABQAVAttribute@U2@@@Z 100164e0 f i ORFQuery.obj
 0001:00015500       ?node_construct@?$QList@PAVORFFindTask@U2@@@@AAEXPAUNode@1@ABQAVORFFindTask@U2@@@Z 10016500 f i ORFQuery.obj
 0001:00015520       ?node_copy@?$QList@PAVAttribute@U2@@@@AAEXPAUNode@1@00@Z 10016520 f i ORFQuery.obj
 0001:00015550       ?node_copy@?$QList@PAVDNATranslation@U2@@@@AAEXPAUNode@1@00@Z 10016550 f i ORFQuery.obj
 0001:00015580       ?node_copy@?$QList@PAVORFFindTask@U2@@@@AAEXPAUNode@1@00@Z 10016580 f i ORFQuery.obj
 0001:000155b0       ?node_destruct@?$QList@PAVAttribute@U2@@@@AAEXPAUNode@1@0@Z 100165b0 f i ORFQuery.obj
 0001:000155c0       ?node_destruct@?$QList@PAVAttribute@U2@@@@AAEXPAUNode@1@@Z 100165c0 f i ORFQuery.obj
 0001:000155d0       ?node_destruct@?$QList@PAVDNATranslation@U2@@@@AAEXPAUNode@1@0@Z 100165d0 f i ORFQuery.obj
 0001:000155e0       ?node_destruct@?$QList@PAVORFFindTask@U2@@@@AAEXPAUNode@1@0@Z 100165e0 f i ORFQuery.obj
 0001:000155f0       ?node_destruct@?$QList@PAVORFFindTask@U2@@@@AAEXPAUNode@1@@Z 100165f0 f i ORFQuery.obj
 0001:00015600       ?qt_metatype_id@?$QMetaTypeId2@H@@SAHXZ 10016600 f i ORFQuery.obj
 0001:00015610       ?qt_metatype_id@?$QMetaTypeId2@VQString@@@@SAHXZ 10016610 f i ORFQuery.obj
 0001:00015620       ?rightNode@?$QMapNode@VQString@@PAVAttribute@U2@@@@QBEPAU1@XZ 10016620 f i ORFQuery.obj
 0001:00015630       ?rightNode@?$QMapNode@VQString@@PAVPropertyDelegate@U2@@@@QBEPAU1@XZ 10016630 f i ORFQuery.obj
 0001:00015640       ?rightNode@?$QMapNode@VQString@@PAVQDSchemeUnit@U2@@@@QBEPAU1@XZ 10016640 f i ORFQuery.obj
 0001:00015650       ?rightNode@?$QMapNode@VQString@@VQVariant@@@@QBEPAU1@XZ 10016650 f i ORFQuery.obj
 0001:00015660       ?root@?$QMapData@VQString@@PAVAttribute@U2@@@@QBEPAU?$QMapNode@VQString@@PAVAttribute@U2@@@@XZ 10016660 f i ORFQuery.obj
 0001:00015670       ?root@?$QMapData@VQString@@PAVPropertyDelegate@U2@@@@QBEPAU?$QMapNode@VQString@@PAVPropertyDelegate@U2@@@@XZ 10016670 f i ORFQuery.obj
 0001:00015680       ?root@?$QMapData@VQString@@PAVQDSchemeUnit@U2@@@@QBEPAU?$QMapNode@VQString@@PAVQDSchemeUnit@U2@@@@XZ 10016680 f i ORFQuery.obj
 0001:00015690       ?root@?$QMapData@VQString@@VQVariant@@@@QBEPAU?$QMapNode@VQString@@VQVariant@@@@XZ 10016690 f i ORFQuery.obj
 0001:000156a0       ?size@?$QList@VORFFindResult@U2@@@@QBEHXZ 100166a0 f i ORFQuery.obj
 0001:000156b0       ?sl_onAlgorithmTaskFinished@QDORFActor@U2@@AAEXPAVTask@2@@Z 100166b0 f   ORFQuery.obj
 0001:00015dd0       ?swap@?$QList@VORFFindResult@U2@@@@QAEXAAV1@@Z 10016dd0 f i ORFQuery.obj
 0001:00015df0       ?swap@?$QVector@VU2Qualifier@U2@@@@QAEXAAV1@@Z 10016df0 f i ORFQuery.obj
 0001:00015e10       ?t@Node@?$QList@PAVDNATranslation@U2@@@@QAEAAPAVDNATranslation@U2@@XZ 10016e10 f i ORFQuery.obj
 0001:00015e20       ?t@Node@?$QList@PAVORFFindTask@U2@@@@QAEAAPAVORFFindTask@U2@@XZ 10016e20 f i ORFQuery.obj
 0001:00015e30       ?t@Node@?$QList@V?$QSharedDataPointer@VAnnotationData@U2@@@@@@QAEAAV?$QSharedDataPointer@VAnnotationData@U2@@@@XZ 10016e30 f i ORFQuery.obj
 0001:00015e40       ?tr@QDORFActor@U2@@SA?AVQString@@PBD0H@Z 10016e40 f i ORFQuery.obj
 0001:00015e70       ?value@?$QMap@VQString@@PAVAttribute@U2@@@@QBEQAVAttribute@U2@@ABVQString@@ABQAV23@@Z 10016e70 f i ORFQuery.obj
 0001:00015ec0       ?value@?$QMap@VQString@@PAVQDSchemeUnit@U2@@@@QBEQAVQDSchemeUnit@U2@@ABVQString@@ABQAV23@@Z 10016ec0 f i ORFQuery.obj
 0001:00015f10       ??$?0VQString@@V0@@?$QPair@VQString@@VQVariant@@@@QAE@$$QAU?$QPair@VQString@@V1@@@@Z 10016f10 f i ORFWorker.obj
 0001:00015f70       ??$_Move@AAPAVDataType@U2@@@std@@YA$$QAPAVDataType@U2@@AAPAV12@@Z 10016f70 f i ORFWorker.obj
 0001:00015f80       ??$getAttributeValue@H@Attribute@U2@@QBEHPAVWorkflowContext@Workflow@1@@Z 10016f80 f i ORFWorker.obj
 0001:00016350       ??$getAttributeValue@VQString@@@Attribute@U2@@QBE?AVQString@@PAVWorkflowContext@Workflow@1@@Z 10017350 f i ORFWorker.obj
 0001:000166e0       ??$getAttributeValue@_N@Attribute@U2@@QBE_NPAVWorkflowContext@Workflow@1@@Z 100176e0 f i ORFWorker.obj
 0001:00016720       ??$getAttributeValueWithoutScript@_N@Attribute@U2@@QBE_NXZ 10017720 f i ORFWorker.obj
 0001:00016760       ??$qMakePair@VQString@@V1@@@YA?AU?$QPair@VQString@@V1@@@ABVQString@@0@Z 10017760 f i ORFWorker.obj
 0001:000167c0       ??$qMapLessThanKey@VDescriptor@U2@@@@YA_NABVDescriptor@U2@@0@Z 100177c0 f i ORFWorker.obj
 0001:000167e0       ??$qMetaTypeId@V?$QSharedDataPointer@VDbiDataHandler@Workflow@U2@@@@@@YAHXZ 100177e0 f i ORFWorker.obj
 0001:000167f0       ??$qMetaTypeId@_N@@YAHXZ   100177f0 f i ORFWorker.obj
 0001:00016800       ??$qRegisterMetaType@V?$QSharedDataPointer@VDbiDataHandler@Workflow@U2@@@@@@YAHPBDPAV?$QSharedDataPointer@VDbiDataHandler@Workflow@U2@@@@W4DefinedType@?$MetaTypeDefinedHelper@V?$QSharedDataPointer@VDbiDataHandler@Workflow@U2@@@@$00@QtPrivate@@@Z 10017800 f i ORFWorker.obj
 0001:000168c0       ??$qRegisterNormalizedMetaType@V?$QSharedDataPointer@VDbiDataHandler@Workflow@U2@@@@@@YAHABVQByteArray@@PAV?$QSharedDataPointer@VDbiDataHandler@Workflow@U2@@@@W4DefinedType@?$MetaTypeDefinedHelper@V?$QSharedDataPointer@VDbiDataHandler@Workflow@U2@@@@$00@QtPrivate@@@Z 100178c0 f i ORFWorker.obj
 0001:00016920       ??$qSwap@PAVDataType@U2@@@@YAXAAPAVDataType@U2@@0@Z 10017920 f i ORFWorker.obj
 0001:00016940       ??$qVariantFromValue@V?$QSharedDataPointer@VDbiDataHandler@Workflow@U2@@@@@@YA?AVQVariant@@ABV?$QSharedDataPointer@VDbiDataHandler@Workflow@U2@@@@@Z 10017940 f i ORFWorker.obj
 0001:00016970       ??$qobject_cast@PAVIntegralBusPort@Workflow@U2@@@@YAPAVIntegralBusPort@Workflow@U2@@PAVQObject@@@Z 10017970 f i ORFWorker.obj
 0001:00016990       ??$qobject_cast@PAVORFFindTask@U2@@@@YAPAVORFFindTask@U2@@PAVQObject@@@Z 10017990 f i ORFWorker.obj
 0001:000169b0       ??$qvariant_cast@V?$QSharedDataPointer@VDbiDataHandler@Workflow@U2@@@@@@YA?AV?$QSharedDataPointer@VDbiDataHandler@Workflow@U2@@@@ABVQVariant@@@Z 100179b0 f i ORFWorker.obj
 0001:000169d0       ??$qvariant_cast@_N@@YA_NABVQVariant@@@Z 100179d0 f i ORFWorker.obj
 0001:00016a10       ??$swap@PAVDataType@U2@@@std@@YAXAAPAVDataType@U2@@0@Z 10017a10 f i ORFWorker.obj
 0001:00016a30       ??$value@V?$QSharedDataPointer@VDbiDataHandler@Workflow@U2@@@@@QVariant@@QBE?AV?$QSharedDataPointer@VDbiDataHandler@Workflow@U2@@@@XZ 10017a30 f i ORFWorker.obj
 0001:00016a50       ??$value@_N@QVariant@@QBE_NXZ 10017a50 f i ORFWorker.obj
 0001:00016a90       ??0?$PrompterBase@VORFPrompter@LocalWorkflow@U2@@@U2@@QAE@PAVActor@Workflow@1@_N@Z 10017a90 f i ORFWorker.obj
 0001:00016ac0       ??0?$QExplicitlySharedDataPointer@VDataType@U2@@@@QAE@ABV0@@Z 10017ac0 f i ORFWorker.obj
 0001:00016ae0       ??0?$QExplicitlySharedDataPointer@VDataType@U2@@@@QAE@PAVDataType@U2@@@Z 10017ae0 f i ORFWorker.obj
 0001:00016b00       ??0?$QExplicitlySharedDataPointer@VDataType@U2@@@@QAE@XZ 10017b00 f i ORFWorker.obj
 0001:00016b10       ??0?$QForeachContainer@V?$QList@PAVPort@Workflow@U2@@@@@@QAE@ABV?$QList@PAVPort@Workflow@U2@@@@@Z 10017b10 f i ORFWorker.obj
 0001:00016b50       ??0?$QForeachContainer@V?$QList@VDescriptor@U2@@@@@@QAE@ABV?$QList@VDescriptor@U2@@@@@Z 10017b50 f i ORFWorker.obj
 0001:00016b90       ??0?$QList@PAVAttribute@U2@@@@QAE@XZ 10017b90 f i ORFWorker.obj
 0001:00016ba0       ??0?$QList@PAVPort@Workflow@U2@@@@QAE@ABV0@@Z 10017ba0 f i ORFWorker.obj
 0001:00016c60       ??0?$QList@PAVPortDescriptor@Workflow@U2@@@@QAE@XZ 10017c60 f i ORFWorker.obj
 0001:00016c70       ??0?$QList@U?$QPair@VQString@@VQVariant@@@@@@QAE@XZ 10017c70 f i ORFWorker.obj
 0001:00016c80       ??0?$QList@VDescriptor@U2@@@@QAE@$$QAV0@@Z 10017c80 f i ORFWorker.obj
 0001:00016ca0       ??0?$QList@VDescriptor@U2@@@@QAE@ABV0@@Z 10017ca0 f i ORFWorker.obj
 0001:00016d60       ??0?$QList@VDescriptor@U2@@@@QAE@XZ 10017d60 f i ORFWorker.obj
 0001:00016d70       ??0?$QMap@VDescriptor@U2@@V?$QExplicitlySharedDataPointer@VDataType@U2@@@@@@QAE@XZ 10017d70 f i ORFWorker.obj
 0001:00016d80       ??0?$QMap@VQString@@VQScriptValue@@@@QAE@XZ 10017d80 f i ORFWorker.obj
 0001:00016d90       ??0?$QPair@VQString@@V1@@@QAE@ABVQString@@0@Z 10017d90 f i ORFWorker.obj
 0001:00016df0       ??0?$QPair@VQString@@VQVariant@@@@QAE@ABU0@@Z 10017df0 f i ORFWorker.obj
 0001:00016e50       ??0?$QScopedPointer@VU2SequenceObject@U2@@U?$QScopedPointerDeleter@VU2SequenceObject@U2@@@@@@QAE@PAVU2SequenceObject@U2@@@Z 10017e50 f i ORFWorker.obj
 0001:00016e60       ??0?$QSharedDataPointer@VDbiDataHandler@Workflow@U2@@@@QAE@$$QAV0@@Z 10017e60 f i ORFWorker.obj
 0001:00016e80       ??0?$QSharedDataPointer@VDbiDataHandler@Workflow@U2@@@@QAE@ABV0@@Z 10017e80 f i ORFWorker.obj
 0001:00016ea0       ??0?$QSharedDataPointer@VDbiDataHandler@Workflow@U2@@@@QAE@XZ 10017ea0 f i ORFWorker.obj
 0001:00016eb0       ??0ORFPrompter@LocalWorkflow@U2@@QAE@PAVActor@Workflow@2@@Z 10017eb0 f i ORFWorker.obj
 0001:00016ee0       ??0ORFWorker@LocalWorkflow@U2@@QAE@PAVActor@Workflow@2@@Z 10017ee0 f   ORFWorker.obj
 0001:00016fc0       ??0ORFWorkerFactory@LocalWorkflow@U2@@QAE@XZ 10017fc0 f i ORFWorker.obj
 0001:00016fe0       ??0const_iterator@?$QList@PAVPort@Workflow@U2@@@@QAE@PAUNode@1@@Z 10017fe0 f i ORFWorker.obj
 0001:00016ff0       ??0const_iterator@?$QList@VDescriptor@U2@@@@QAE@PAUNode@1@@Z 10017ff0 f i ORFWorker.obj
 0001:00017000       ??0const_iterator@?$QMap@VDescriptor@U2@@VQVariant@@@@QAE@PBU?$QMapNode@VDescriptor@U2@@VQVariant@@@@@Z 10018000 f i ORFWorker.obj
 0001:00017010       ??0iterator@?$QMap@VDescriptor@U2@@V?$QExplicitlySharedDataPointer@VDataType@U2@@@@@@QAE@PAU?$QMapNode@VDescriptor@U2@@V?$QExplicitlySharedDataPointer@VDataType@U2@@@@@@@Z 10018010 f i ORFWorker.obj
 0001:00017020       ??0iterator@?$QMap@VQString@@VQScriptValue@@@@QAE@PAU?$QMapNode@VQString@@VQScriptValue@@@@@Z 10018020 f i ORFWorker.obj
 0001:00017030       ??1?$PrompterBase@VORFPrompter@LocalWorkflow@U2@@@U2@@UAE@XZ 10018030 f i ORFWorker.obj
 0001:00017040       ??1?$QForeachContainer@V?$QList@PAVPort@Workflow@U2@@@@@@QAE@XZ 10018040 f i ORFWorker.obj
 0001:00017070       ??1?$QForeachContainer@V?$QList@VDescriptor@U2@@@@@@QAE@XZ 10018070 f i ORFWorker.obj
 0001:000170a0       ??1?$QList@PAVAttribute@U2@@@@QAE@XZ 100180a0 f i ORFWorker.obj
 0001:000170d0       ??1?$QList@PAVPort@Workflow@U2@@@@QAE@XZ 100180d0 f i ORFWorker.obj
 0001:00017100       ??1?$QList@PAVPortDescriptor@Workflow@U2@@@@QAE@XZ 10018100 f i ORFWorker.obj
 0001:00017130       ??1?$QList@U?$QPair@VQString@@VQVariant@@@@@@QAE@XZ 10018130 f i ORFWorker.obj
 0001:00017180       ??1?$QList@VDescriptor@U2@@@@QAE@XZ 10018180 f i ORFWorker.obj
 0001:000171b0       ??1?$QMap@VDescriptor@U2@@V?$QExplicitlySharedDataPointer@VDataType@U2@@@@@@QAE@XZ 100181b0 f i ORFWorker.obj
 0001:00017200       ??1?$QMap@VQString@@VQScriptValue@@@@QAE@XZ 10018200 f i ORFWorker.obj
 0001:00017250       ??1?$QPair@VQString@@V1@@@QAE@XZ 10018250 f i ORFWorker.obj
 0001:000172b0       ??1?$QPair@VQString@@VQVariant@@@@QAE@XZ 100182b0 f i ORFWorker.obj
 0001:00017310       ??1?$QScopedPointer@VU2SequenceObject@U2@@U?$QScopedPointerDeleter@VU2SequenceObject@U2@@@@@@QAE@XZ 10018310 f i ORFWorker.obj
 0001:00017320       ??1?$QSharedDataPointer@VDbiDataHandler@Workflow@U2@@@@QAE@XZ 10018320 f i ORFWorker.obj
 0001:00017340       ??1ORFPrompter@LocalWorkflow@U2@@UAE@XZ 10018340 f i ORFWorker.obj
 0001:00017350       ??1ORFWorker@LocalWorkflow@U2@@UAE@XZ 10018350 f i ORFWorker.obj
 0001:000173c0       ??1ORFWorkerFactory@LocalWorkflow@U2@@UAE@XZ 100183c0 f i ORFWorker.obj
 0001:000173d0       ??4?$QExplicitlySharedDataPointer@VDataType@U2@@@@QAEAAV0@$$QAV0@@Z 100183d0 f i ORFWorker.obj
 0001:000173f0       ??4?$QExplicitlySharedDataPointer@VDataType@U2@@@@QAEAAV0@ABV0@@Z 100183f0 f i ORFWorker.obj
 0001:00017440       ??6?$QList@PAVPortDescriptor@Workflow@U2@@@@QAEAAV0@ABQAVPortDescriptor@Workflow@U2@@@Z 10018440 f i ORFWorker.obj
 0001:00017460       ??8const_iterator@?$QMap@VDescriptor@U2@@VQVariant@@@@QBE_NABV01@@Z 10018460 f i ORFWorker.obj
 0001:00017480       ??9const_iterator@?$QList@PAVPort@Workflow@U2@@@@QBE_NABV01@@Z 10018480 f i ORFWorker.obj
 0001:000174a0       ??9const_iterator@?$QList@VDescriptor@U2@@@@QBE_NABV01@@Z 100184a0 f i ORFWorker.obj
 0001:000174c0       ??9const_iterator@?$QMap@VDescriptor@U2@@VQVariant@@@@QBE_NABV01@@Z 100184c0 f i ORFWorker.obj
 0001:000174e0       ??A?$QMap@VDescriptor@U2@@V?$QExplicitlySharedDataPointer@VDataType@U2@@@@@@QAEAAV?$QExplicitlySharedDataPointer@VDataType@U2@@@@ABVDescriptor@U2@@@Z 100184e0 f i ORFWorker.obj
 0001:000175a0       ??A?$QMap@VQString@@VQScriptValue@@@@QAEAAVQScriptValue@@ABVQString@@@Z 100185a0 f i ORFWorker.obj
 0001:00017670       ??C?$QScopedPointer@VU2SequenceObject@U2@@U?$QScopedPointerDeleter@VU2SequenceObject@U2@@@@@@QBEPAVU2SequenceObject@U2@@XZ 10018670 f i ORFWorker.obj
 0001:00017680       ??Dconst_iterator@?$QList@PAVPort@Workflow@U2@@@@QBEABQAVPort@Workflow@U2@@XZ 10018680 f i ORFWorker.obj
 0001:00017690       ??Dconst_iterator@?$QList@VDescriptor@U2@@@@QBEABVDescriptor@U2@@XZ 10018690 f i ORFWorker.obj
 0001:000176a0       ??Diterator@?$QMap@VDescriptor@U2@@V?$QExplicitlySharedDataPointer@VDataType@U2@@@@@@QBEAAV?$QExplicitlySharedDataPointer@VDataType@U2@@@@XZ 100186a0 f i ORFWorker.obj
 0001:000176b0       ??Diterator@?$QMap@VQString@@VQScriptValue@@@@QBEAAVQScriptValue@@XZ 100186b0 f i ORFWorker.obj
 0001:000176c0       ??Econst_iterator@?$QList@PAVPort@Workflow@U2@@@@QAEAAV01@XZ 100186c0 f i ORFWorker.obj
 0001:000176d0       ??Econst_iterator@?$QList@VDescriptor@U2@@@@QAEAAV01@XZ 100186d0 f i ORFWorker.obj
 0001:000176e0       ??Econst_iterator@?$QMap@VDescriptor@U2@@VQVariant@@@@QAEAAV01@XZ 100186e0 f i ORFWorker.obj
 0001:000176f1       ??_E?$PrompterBase@VORFPrompter@LocalWorkflow@U2@@@U2@@WM@AEPAXI@Z 100186f1 f i ORFWorker.obj
 0001:000176f9       ??_EORFPrompter@LocalWorkflow@U2@@WM@AEPAXI@Z 100186f9 f i ORFWorker.obj
 0001:00017701       ??_EORFWorker@LocalWorkflow@U2@@W7AEPAXI@Z 10018701 f i ORFWorker.obj
 0001:00017709       ??_EORFWorker@LocalWorkflow@U2@@WBA@AEPAXI@Z 10018709 f i ORFWorker.obj
 0001:00017711       ??_EORFWorkerFactory@LocalWorkflow@U2@@W7AEPAXI@Z 10018711 f i ORFWorker.obj
 0001:00017720       ??_E?$PrompterBase@VORFPrompter@LocalWorkflow@U2@@@U2@@UAEPAXI@Z 10018720 f i ORFWorker.obj
 0001:00017720       ??_G?$PrompterBase@VORFPrompter@LocalWorkflow@U2@@@U2@@UAEPAXI@Z 10018720 f i ORFWorker.obj
 0001:00017750       ??_G?$QExplicitlySharedDataPointer@VDataType@U2@@@@QAEPAXI@Z 10018750 f i ORFWorker.obj
 0001:00017790       ??_G?$QPair@VQString@@VQVariant@@@@QAEPAXI@Z 10018790 f i ORFWorker.obj
 0001:00017800       ??_G?$QSharedDataPointer@VDbiDataHandler@Workflow@U2@@@@QAEPAXI@Z 10018800 f i ORFWorker.obj
 0001:00017840       ??_EDescriptor@U2@@UAEPAXI@Z 10018840 f i ORFWorker.obj
 0001:00017840       ??_GDescriptor@U2@@UAEPAXI@Z 10018840 f i ORFWorker.obj
 0001:00017870       ??_GIntegralBusActorPrototype@Workflow@U2@@UAEPAXI@Z 10018870 f i ORFWorker.obj
 0001:00017870       ??_EIntegralBusActorPrototype@Workflow@U2@@UAEPAXI@Z 10018870 f i ORFWorker.obj
 0001:000178a0       ??_GMapDataType@U2@@UAEPAXI@Z 100188a0 f i ORFWorker.obj
 0001:000178a0       ??_EMapDataType@U2@@UAEPAXI@Z 100188a0 f i ORFWorker.obj
 0001:000178d0       ??_GORFPrompter@LocalWorkflow@U2@@UAEPAXI@Z 100188d0 f i ORFWorker.obj
 0001:000178d0       ??_EORFPrompter@LocalWorkflow@U2@@UAEPAXI@Z 100188d0 f i ORFWorker.obj
 0001:00017900       ??_EORFWorker@LocalWorkflow@U2@@UAEPAXI@Z 10018900 f i ORFWorker.obj
 0001:00017900       ??_GORFWorker@LocalWorkflow@U2@@UAEPAXI@Z 10018900 f i ORFWorker.obj
 0001:00017980       ??_EORFWorkerFactory@LocalWorkflow@U2@@UAEPAXI@Z 10018980 f i ORFWorker.obj
 0001:00017980       ??_GORFWorkerFactory@LocalWorkflow@U2@@UAEPAXI@Z 10018980 f i ORFWorker.obj
 0001:000179b0       ??_EPortDescriptor@Workflow@U2@@UAEPAXI@Z 100189b0 f i ORFWorker.obj
 0001:000179b0       ??_GPortDescriptor@Workflow@U2@@UAEPAXI@Z 100189b0 f i ORFWorker.obj
 0001:000179e0       ??_GQScriptValue@@QAEPAXI@Z 100189e0 f i ORFWorker.obj
 0001:00017a10       ?Construct@?$QMetaTypeFunctionHelper@V?$QSharedDataPointer@VDbiDataHandler@Workflow@U2@@@@$00@QtMetaTypePrivate@@SAPAXPAXPBX@Z 10018a10 f i ORFWorker.obj
 0001:00017a60       ?Create@?$QMetaTypeFunctionHelper@V?$QSharedDataPointer@VDbiDataHandler@Workflow@U2@@@@$00@QtMetaTypePrivate@@SAPAXPBX@Z 10018a60 f i ORFWorker.obj
 0001:00017ab0       ?Delete@?$QMetaTypeFunctionHelper@V?$QSharedDataPointer@VDbiDataHandler@Workflow@U2@@@@$00@QtMetaTypePrivate@@SAXPAX@Z 10018ab0 f i ORFWorker.obj
 0001:00017af0       ?Destruct@?$QMetaTypeFunctionHelper@V?$QSharedDataPointer@VDbiDataHandler@Workflow@U2@@@@$00@QtMetaTypePrivate@@SAXPAX@Z 10018af0 f i ORFWorker.obj
 0001:00017b20       ?append@?$QList@PAVPortDescriptor@Workflow@U2@@@@QAEXABQAVPortDescriptor@Workflow@U2@@@Z 10018b20 f i ORFWorker.obj
 0001:00017bb0       ?append@?$QList@U?$QPair@VQString@@VQVariant@@@@@@QAEXABU?$QPair@VQString@@VQVariant@@@@@Z 10018bb0 f i ORFWorker.obj
 0001:00017c40       ?append@?$QList@VDescriptor@U2@@@@QAEXABVDescriptor@U2@@@Z 10018c40 f i ORFWorker.obj
 0001:00017d30       ?begin@?$QList@PAVPort@Workflow@U2@@@@QBE?AVconst_iterator@1@XZ 10018d30 f i ORFWorker.obj
 0001:00017d50       ?begin@?$QList@VDescriptor@U2@@@@QBE?AVconst_iterator@1@XZ 10018d50 f i ORFWorker.obj
 0001:00017d70       ?begin@?$QMap@VDescriptor@U2@@VQVariant@@@@QBE?AVconst_iterator@1@XZ 10018d70 f i ORFWorker.obj
 0001:00017d90       ?begin@?$QMapData@VDescriptor@U2@@VQVariant@@@@QAEPAU?$QMapNode@VDescriptor@U2@@VQVariant@@@@XZ 10018d90 f i ORFWorker.obj
 0001:00017da0       ?cleanup@?$QScopedPointerDeleter@VU2SequenceObject@U2@@@@SAXPAVU2SequenceObject@U2@@@Z 10018da0 f i ORFWorker.obj
 0001:00017dc0       ?cleanup@ORFWorker@LocalWorkflow@U2@@UAEXXZ 10018dc0 f   ORFWorker.obj
 0001:00017dd0       ?composeRichDoc@ORFPrompter@LocalWorkflow@U2@@MAE?AVQString@@XZ 10018dd0 f   ORFWorker.obj
 0001:000186e0       ?copy@?$QMapNode@VDescriptor@U2@@V?$QExplicitlySharedDataPointer@VDataType@U2@@@@@@QBEPAU1@PAU?$QMapData@VDescriptor@U2@@V?$QExplicitlySharedDataPointer@VDataType@U2@@@@@@@Z 100196e0 f i ORFWorker.obj
 0001:00018770       ?copy@?$QMapNode@VQString@@VQScriptValue@@@@QBEPAU1@PAU?$QMapData@VQString@@VQScriptValue@@@@@Z 10019770 f i ORFWorker.obj
 0001:00018800       ?create@?$QMapData@VDescriptor@U2@@V?$QExplicitlySharedDataPointer@VDataType@U2@@@@@@SAPAU1@XZ 10019800 f i ORFWorker.obj
 0001:00018810       ?create@?$QMapData@VQString@@VQScriptValue@@@@SAPAU1@XZ 10019810 f i ORFWorker.obj
 0001:00018820       ?createDescription@?$PrompterBase@VORFPrompter@LocalWorkflow@U2@@@U2@@UAEPAVActorDocument@Workflow@2@PAVActor@42@@Z 10019820 f i ORFWorker.obj
 0001:00018ac0       ?createNode@?$QMapData@VDescriptor@U2@@V?$QExplicitlySharedDataPointer@VDataType@U2@@@@@@QAEPAU?$QMapNode@VDescriptor@U2@@V?$QExplicitlySharedDataPointer@VDataType@U2@@@@@@ABVDescriptor@U2@@ABV?$QExplicitlySharedDataPointer@VDataType@U2@@@@PAU2@_N@Z 10019ac0 f i ORFWorker.obj
 0001:00018b80       ?createNode@?$QMapData@VQString@@VQScriptValue@@@@QAEPAU?$QMapNode@VQString@@VQScriptValue@@@@ABVQString@@ABVQScriptValue@@PAU2@_N@Z 10019b80 f i ORFWorker.obj
 0001:00018c40       ?createWorker@ORFWorkerFactory@LocalWorkflow@U2@@UAEPAVWorker@Workflow@3@PAVActor@53@@Z 10019c40 f i ORFWorker.obj
 0001:00018cb0       ?dealloc@?$QList@PAVPort@Workflow@U2@@@@AAEXPAUData@QListData@@@Z 10019cb0 f i ORFWorker.obj
 0001:00018cd0       ?dealloc@?$QList@PAVPortDescriptor@Workflow@U2@@@@AAEXPAUData@QListData@@@Z 10019cd0 f i ORFWorker.obj
 0001:00018cf0       ?dealloc@?$QList@U?$QPair@VQString@@VQVariant@@@@@@AAEXPAUData@QListData@@@Z 10019cf0 f i ORFWorker.obj
 0001:00018d20       ?dealloc@?$QList@VDescriptor@U2@@@@AAEXPAUData@QListData@@@Z 10019d20 f i ORFWorker.obj
 0001:00018d70       ?destroy@?$QMapData@VDescriptor@U2@@V?$QExplicitlySharedDataPointer@VDataType@U2@@@@@@QAEXXZ 10019d70 f i ORFWorker.obj
 0001:00018da0       ?destroy@?$QMapData@VQString@@VQScriptValue@@@@QAEXXZ 10019da0 f i ORFWorker.obj
 0001:00018dd0       ?destroySubTree@?$QMapNode@VDescriptor@U2@@V?$QExplicitlySharedDataPointer@VDataType@U2@@@@@@QAEXXZ 10019dd0 f i ORFWorker.obj
 0001:00018e20       ?destroySubTree@?$QMapNode@VQString@@VQScriptValue@@@@QAEXXZ 10019e20 f i ORFWorker.obj
 0001:00018e60       ?detach@?$QMap@VDescriptor@U2@@V?$QExplicitlySharedDataPointer@VDataType@U2@@@@@@QAEXXZ 10019e60 f i ORFWorker.obj
 0001:00018e80       ?detach@?$QMap@VQString@@VQScriptValue@@@@QAEXXZ 10019e80 f i ORFWorker.obj
 0001:00018ea0       ?detach_helper@?$QList@VDescriptor@U2@@@@AAEXH@Z 10019ea0 f i ORFWorker.obj
 0001:00018f70       ?detach_helper@?$QMap@VDescriptor@U2@@V?$QExplicitlySharedDataPointer@VDataType@U2@@@@@@AAEXXZ 10019f70 f i ORFWorker.obj
 0001:00018ff0       ?detach_helper@?$QMap@VQString@@VQScriptValue@@@@AAEXXZ 10019ff0 f i ORFWorker.obj
 0001:00019070       ?detach_helper_grow@?$QList@PAVPortDescriptor@Workflow@U2@@@@AAEPAUNode@1@HH@Z 1001a070 f i ORFWorker.obj
 0001:00019180       ?detach_helper_grow@?$QList@U?$QPair@VQString@@VQVariant@@@@@@AAEPAUNode@1@HH@Z 1001a180 f i ORFWorker.obj
 0001:000192f0       ?detach_helper_grow@?$QList@VDescriptor@U2@@@@AAEPAUNode@1@HH@Z 1001a2f0 f i ORFWorker.obj
 0001:00019440       ?end@?$QList@PAVPort@Workflow@U2@@@@QBE?AVconst_iterator@1@XZ 1001a440 f i ORFWorker.obj
 0001:00019460       ?end@?$QList@VDescriptor@U2@@@@QBE?AVconst_iterator@1@XZ 1001a460 f i ORFWorker.obj
 0001:00019480       ?end@?$QMap@VDescriptor@U2@@VQVariant@@@@QBE?AVconst_iterator@1@XZ 1001a480 f i ORFWorker.obj
 0001:000194a0       ?end@?$QMapData@VDescriptor@U2@@V?$QExplicitlySharedDataPointer@VDataType@U2@@@@@@QAEPAU?$QMapNode@VDescriptor@U2@@V?$QExplicitlySharedDataPointer@VDataType@U2@@@@@@XZ 1001a4a0 f i ORFWorker.obj
 0001:000194b0       ?end@?$QMapData@VDescriptor@U2@@VQVariant@@@@QAEPAU?$QMapNode@VDescriptor@U2@@VQVariant@@@@XZ 1001a4b0 f i ORFWorker.obj
 0001:000194c0       ?end@?$QMapData@VQString@@VQScriptValue@@@@QAEPAU?$QMapNode@VQString@@VQScriptValue@@@@XZ 1001a4c0 f i ORFWorker.obj
 0001:000194d0       ?findNode@?$QMapData@VDescriptor@U2@@V?$QExplicitlySharedDataPointer@VDataType@U2@@@@@@QBEPAU?$QMapNode@VDescriptor@U2@@V?$QExplicitlySharedDataPointer@VDataType@U2@@@@@@ABVDescriptor@U2@@@Z 1001a4d0 f i ORFWorker.obj
 0001:00019510       ?findNode@?$QMapData@VDescriptor@U2@@VQVariant@@@@QBEPAU?$QMapNode@VDescriptor@U2@@VQVariant@@@@ABVDescriptor@U2@@@Z 1001a510 f i ORFWorker.obj
 0001:00019550       ?findNode@?$QMapData@VQString@@PAVIntegralBus@Workflow@U2@@@@QBEPAU?$QMapNode@VQString@@PAVIntegralBus@Workflow@U2@@@@ABVQString@@@Z 1001a550 f i ORFWorker.obj
 0001:00019590       ?findNode@?$QMapData@VQString@@VQScriptValue@@@@QBEPAU?$QMapNode@VQString@@VQScriptValue@@@@ABVQString@@@Z 1001a590 f i ORFWorker.obj
 0001:00019700       ?init@ORFWorker@LocalWorkflow@U2@@UAEXXZ 1001a700 f   ORFWorker.obj
 0001:00019800       ?init@ORFWorkerFactory@LocalWorkflow@U2@@SAXXZ 1001a800 f   ORFWorker.obj
 0001:0001ae90       ?insert@?$QMap@VDescriptor@U2@@V?$QExplicitlySharedDataPointer@VDataType@U2@@@@@@QAE?AViterator@1@ABVDescriptor@U2@@ABV?$QExplicitlySharedDataPointer@VDataType@U2@@@@@Z 1001be90 f i ORFWorker.obj
 0001:0001af90       ?insert@?$QMap@VQString@@VQScriptValue@@@@QAE?AViterator@1@ABVQString@@ABVQScriptValue@@@Z 1001bf90 f i ORFWorker.obj
 0001:0001b050       ?invoke@?$MetaTypeInvoker@U?$QVariantValueHelper@V?$QSharedDataPointer@VDbiDataHandler@Workflow@U2@@@@@QtPrivate@@ABVQVariant@@V?$QSharedDataPointer@VDbiDataHandler@Workflow@U2@@@@@QtPrivate@@SA?AV?$QSharedDataPointer@VDbiDataHandler@Workflow@U2@@@@ABVQVariant@@@Z 1001c050 f i ORFWorker.obj
 0001:0001b070       ?invoke@?$MetaTypeInvoker@U?$QVariantValueHelper@_N@QtPrivate@@ABVQVariant@@_N@QtPrivate@@SA_NABVQVariant@@@Z 1001c070 f i ORFWorker.obj
 0001:0001b0b0       ?isNull@?$QScopedPointer@VU2SequenceObject@U2@@U?$QScopedPointerDeleter@VU2SequenceObject@U2@@@@@@QBE_NXZ 1001c0b0 f i ORFWorker.obj
 0001:0001b0c0       ?key@const_iterator@?$QMap@VDescriptor@U2@@VQVariant@@@@QBEABVDescriptor@U2@@XZ 1001c0c0 f i ORFWorker.obj
 0001:0001b0d0       ?leftNode@?$QMapNode@VDescriptor@U2@@V?$QExplicitlySharedDataPointer@VDataType@U2@@@@@@QBEPAU1@XZ 1001c0d0 f i ORFWorker.obj
 0001:0001b0e0       ?leftNode@?$QMapNode@VDescriptor@U2@@VQVariant@@@@QBEPAU1@XZ 1001c0e0 f i ORFWorker.obj
 0001:0001b0f0       ?leftNode@?$QMapNode@VQString@@PAVIntegralBus@Workflow@U2@@@@QBEPAU1@XZ 1001c0f0 f i ORFWorker.obj
 0001:0001b100       ?leftNode@?$QMapNode@VQString@@VQScriptValue@@@@QBEPAU1@XZ 1001c100 f i ORFWorker.obj
 0001:0001b110       ?lowerBound@?$QMapNode@VDescriptor@U2@@V?$QExplicitlySharedDataPointer@VDataType@U2@@@@@@QAEPAU1@ABVDescriptor@U2@@@Z 1001c110 f i ORFWorker.obj
 0001:0001b150       ?lowerBound@?$QMapNode@VDescriptor@U2@@VQVariant@@@@QAEPAU1@ABVDescriptor@U2@@@Z 1001c150 f i ORFWorker.obj
 0001:0001b190       ?lowerBound@?$QMapNode@VQString@@PAVIntegralBus@Workflow@U2@@@@QAEPAU1@ABVQString@@@Z 1001c190 f i ORFWorker.obj
 0001:0001b1d0       ?lowerBound@?$QMapNode@VQString@@VQScriptValue@@@@QAEPAU1@ABVQString@@@Z 1001c1d0 f i ORFWorker.obj
 0001:0001b210       ?metaType@?$QVariantValueHelper@V?$QSharedDataPointer@VDbiDataHandler@Workflow@U2@@@@@QtPrivate@@SA?AV?$QSharedDataPointer@VDbiDataHandler@Workflow@U2@@@@ABVQVariant@@@Z 1001c210 f i ORFWorker.obj
 0001:0001b310       ?metaType@?$QVariantValueHelper@_N@QtPrivate@@SA_NABVQVariant@@@Z 1001c310 f i ORFWorker.obj
 0001:0001b350       ?nextNode@?$QMapNode@VDescriptor@U2@@VQVariant@@@@QBEPBU1@XZ 1001c350 f i ORFWorker.obj
 0001:0001b360       ?node_construct@?$QList@PAVPortDescriptor@Workflow@U2@@@@AAEXPAUNode@1@ABQAVPortDescriptor@Workflow@U2@@@Z 1001c360 f i ORFWorker.obj
 0001:0001b380       ?node_construct@?$QList@U?$QPair@VQString@@VQVariant@@@@@@AAEXPAUNode@1@ABU?$QPair@VQString@@VQVariant@@@@@Z 1001c380 f i ORFWorker.obj
 0001:0001b410       ?node_construct@?$QList@VDescriptor@U2@@@@AAEXPAUNode@1@ABVDescriptor@U2@@@Z 1001c410 f i ORFWorker.obj
 0001:0001b4a0       ?node_copy@?$QList@PAVPort@Workflow@U2@@@@AAEXPAUNode@1@00@Z 1001c4a0 f i ORFWorker.obj
 0001:0001b4d0       ?node_copy@?$QList@PAVPortDescriptor@Workflow@U2@@@@AAEXPAUNode@1@00@Z 1001c4d0 f i ORFWorker.obj
 0001:0001b500       ?node_copy@?$QList@U?$QPair@VQString@@VQVariant@@@@@@AAEXPAUNode@1@00@Z 1001c500 f i ORFWorker.obj
 0001:0001b600       ?node_copy@?$QList@VDescriptor@U2@@@@AAEXPAUNode@1@00@Z 1001c600 f i ORFWorker.obj
 0001:0001b6d0       ?node_destruct@?$QList@PAVPort@Workflow@U2@@@@AAEXPAUNode@1@0@Z 1001c6d0 f i ORFWorker.obj
 0001:0001b6e0       ?node_destruct@?$QList@PAVPortDescriptor@Workflow@U2@@@@AAEXPAUNode@1@0@Z 1001c6e0 f i ORFWorker.obj
 0001:0001b6f0       ?node_destruct@?$QList@PAVPortDescriptor@Workflow@U2@@@@AAEXPAUNode@1@@Z 1001c6f0 f i ORFWorker.obj
 0001:0001b700       ?node_destruct@?$QList@U?$QPair@VQString@@VQVariant@@@@@@AAEXPAUNode@1@0@Z 1001c700 f i ORFWorker.obj
 0001:0001b780       ?node_destruct@?$QList@U?$QPair@VQString@@VQVariant@@@@@@AAEXPAUNode@1@@Z 1001c780 f i ORFWorker.obj
 0001:0001b7f0       ?node_destruct@?$QList@VDescriptor@U2@@@@AAEXPAUNode@1@0@Z 1001c7f0 f i ORFWorker.obj
 0001:0001b820       ?node_destruct@?$QList@VDescriptor@U2@@@@AAEXPAUNode@1@@Z 1001c820 f i ORFWorker.obj
 0001:0001b840       ?qt_metatype_id@?$QMetaTypeId2@V?$QSharedDataPointer@VDbiDataHandler@Workflow@U2@@@@@@SAHXZ 1001c840 f i ORFWorker.obj
 0001:0001b850       ?qt_metatype_id@?$QMetaTypeId2@_N@@SAHXZ 1001c850 f i ORFWorker.obj
 0001:0001b860       ?qt_metatype_id@?$QMetaTypeId@V?$QSharedDataPointer@VDbiDataHandler@Workflow@U2@@@@@@SAHXZ 1001c860 f i ORFWorker.obj
 0001:0001b900       ?qt_metatype_id@?$QMetaTypeIdHelper@V?$QSharedDataPointer@VDbiDataHandler@Workflow@U2@@@@$00@QtPrivate@@SAHXZ 1001c900 f i ORFWorker.obj
 0001:0001b910       ?registerConverter@?$AssociativeContainerConverterHelper@V?$QSharedDataPointer@VDbiDataHandler@Workflow@U2@@@@$0A@@QtPrivate@@SA_NH@Z 1001c910 f i ORFWorker.obj
 0001:0001b920       ?registerConverter@?$IsPair@V?$QSharedDataPointer@VDbiDataHandler@Workflow@U2@@@@@QtPrivate@@SA_NH@Z 1001c920 f i ORFWorker.obj
 0001:0001b930       ?registerConverter@?$MetaTypeSmartPointerHelper@V?$QSharedDataPointer@VDbiDataHandler@Workflow@U2@@@@X@QtPrivate@@SA_NH@Z 1001c930 f i ORFWorker.obj
 0001:0001b940       ?registerConverter@?$SequentialContainerConverterHelper@V?$QSharedDataPointer@VDbiDataHandler@Workflow@U2@@@@$0A@@QtPrivate@@SA_NH@Z 1001c940 f i ORFWorker.obj
 0001:0001b950       ?reserve@?$QList@VDescriptor@U2@@@@QAEXH@Z 1001c950 f i ORFWorker.obj
 0001:0001b980       ?rightNode@?$QMapNode@VDescriptor@U2@@V?$QExplicitlySharedDataPointer@VDataType@U2@@@@@@QBEPAU1@XZ 1001c980 f i ORFWorker.obj
 0001:0001b990       ?rightNode@?$QMapNode@VDescriptor@U2@@VQVariant@@@@QBEPAU1@XZ 1001c990 f i ORFWorker.obj
 0001:0001b9a0       ?rightNode@?$QMapNode@VQString@@PAVIntegralBus@Workflow@U2@@@@QBEPAU1@XZ 1001c9a0 f i ORFWorker.obj
 0001:0001b9b0       ?rightNode@?$QMapNode@VQString@@VQScriptValue@@@@QBEPAU1@XZ 1001c9b0 f i ORFWorker.obj
 0001:0001b9c0       ?root@?$QMapData@VDescriptor@U2@@V?$QExplicitlySharedDataPointer@VDataType@U2@@@@@@QBEPAU?$QMapNode@VDescriptor@U2@@V?$QExplicitlySharedDataPointer@VDataType@U2@@@@@@XZ 1001c9c0 f i ORFWorker.obj
 0001:0001b9d0       ?root@?$QMapData@VDescriptor@U2@@VQVariant@@@@QBEPAU?$QMapNode@VDescriptor@U2@@VQVariant@@@@XZ 1001c9d0 f i ORFWorker.obj
 0001:0001b9e0       ?root@?$QMapData@VQString@@PAVIntegralBus@Workflow@U2@@@@QBEPAU?$QMapNode@VQString@@PAVIntegralBus@Workflow@U2@@@@XZ 1001c9e0 f i ORFWorker.obj
 0001:0001b9f0       ?root@?$QMapData@VQString@@VQScriptValue@@@@QBEPAU?$QMapNode@VQString@@VQScriptValue@@@@XZ 1001c9f0 f i ORFWorker.obj
 0001:0001ba00       ?size@?$QMap@VDescriptor@U2@@VQVariant@@@@QBEHXZ 1001ca00 f i ORFWorker.obj
 0001:0001ba10       ?sl_taskFinished@ORFWorker@LocalWorkflow@U2@@AAEXXZ 1001ca10 f   ORFWorker.obj
 0001:0001bbf0       ?t@Node@?$QList@PAVPort@Workflow@U2@@@@QAEAAPAVPort@Workflow@U2@@XZ 1001cbf0 f i ORFWorker.obj
 0001:0001bc00       ?t@Node@?$QList@VDescriptor@U2@@@@QAEAAVDescriptor@U2@@XZ 1001cc00 f i ORFWorker.obj
 0001:0001bc10       ?tick@ORFWorker@LocalWorkflow@U2@@UAEPAVTask@3@XZ 1001cc10 f   ORFWorker.obj
 0001:0001c2f0       ?tr@ORFPrompter@LocalWorkflow@U2@@SA?AVQString@@PBD0H@Z 1001d2f0 f i ORFWorker.obj
 0001:0001c320       ?tr@ORFWorker@LocalWorkflow@U2@@SA?AVQString@@PBD0H@Z 1001d320 f i ORFWorker.obj
 0001:0001c350       ?uniqueKeys@?$QMap@VDescriptor@U2@@VQVariant@@@@QBE?AV?$QList@VDescriptor@U2@@@@XZ 1001d350 f i ORFWorker.obj
 0001:0001c450       ?value@?$MetaObjectForType@V?$QSharedDataPointer@VDbiDataHandler@Workflow@U2@@@@$0A@@QtPrivate@@SAPBUQMetaObject@@XZ 1001d450 f i ORFWorker.obj
 0001:0001c460       ?value@?$QMap@VDescriptor@U2@@VQVariant@@@@QBE?BVQVariant@@ABVDescriptor@U2@@ABV2@@Z 1001d460 f i ORFWorker.obj
 0001:0001c4c0       ?value@?$QMap@VQString@@PAVIntegralBus@Workflow@U2@@@@QBEQAVIntegralBus@Workflow@U2@@ABVQString@@ABQAV234@@Z 1001d4c0 f i ORFWorker.obj
 0001:0001c510       ?value@?$QMap@VQString@@VQVariant@@@@QBE?BVQVariant@@ABVQString@@ABV2@@Z 1001d510 f i ORFWorker.obj
 0001:0001c580       ??$qMetaTypeId@PAVTask@U2@@@@YAHXZ 1001d580 f i moc_ORFDialog.obj
 0001:0001c590       ??$qRegisterMetaType@PAVTask@U2@@@@YAHXZ 1001d590 f i moc_ORFDialog.obj
 0001:0001c5a0       ??$qRegisterNormalizedMetaType@PAVTask@U2@@@@YAHABVQByteArray@@PAPAVTask@U2@@W4DefinedType@?$MetaTypeDefinedHelper@PAVTask@U2@@$00@QtPrivate@@@Z 1001d5a0 f i moc_ORFDialog.obj
 0001:0001c600       ??C?$QScopedPointer@VQObjectData@@U?$QScopedPointerDeleter@VQObjectData@@@@@@QBEPAVQObjectData@@XZ 1001d600 f i moc_ORFDialog.obj
 0001:0001c610       ?Construct@?$QMetaTypeFunctionHelper@PAVTask@U2@@$00@QtMetaTypePrivate@@SAPAXPAXPBX@Z 1001d610 f i moc_ORFDialog.obj
 0001:0001c640       ?Create@?$QMetaTypeFunctionHelper@PAVTask@U2@@$00@QtMetaTypePrivate@@SAPAXPBX@Z 1001d640 f i moc_ORFDialog.obj
 0001:0001c680       ?Delete@?$QMetaTypeFunctionHelper@PAVTask@U2@@$00@QtMetaTypePrivate@@SAXPAX@Z 1001d680 f i moc_ORFDialog.obj
 0001:0001c690       ?Destruct@?$QMetaTypeFunctionHelper@PAVTask@U2@@$00@QtMetaTypePrivate@@SAXPAX@Z 1001d690 f i moc_ORFDialog.obj
 0001:0001c6a0       ?metaObject@ORFDialog@U2@@UBEPBUQMetaObject@@XZ 1001d6a0 f   moc_ORFDialog.obj
 0001:0001c6c0       ?qt_metacall@ORFDialog@U2@@UAEHW4Call@QMetaObject@@HPAPAX@Z 1001d6c0 f   moc_ORFDialog.obj
 0001:0001c720       ?qt_metacast@ORFDialog@U2@@UAEPAXPBD@Z 1001d720 f   moc_ORFDialog.obj
 0001:0001c7c0       ?qt_metatype_id@?$QMetaTypeId2@PAVTask@U2@@@@SAHXZ 1001d7c0 f i moc_ORFDialog.obj
 0001:0001c7d0       ?qt_metatype_id@?$QMetaTypeIdHelper@PAVTask@U2@@$00@QtPrivate@@SAHXZ 1001d7d0 f i moc_ORFDialog.obj
 0001:0001c7e0       ?qt_metatype_id@?$QMetaTypeIdQObject@PAVTask@U2@@$00@@SAHXZ 1001d7e0 f i moc_ORFDialog.obj
 0001:0001c8c0       ?qt_static_metacall@ORFDialog@U2@@CAXPAVQObject@@W4Call@QMetaObject@@HPAPAX@Z 1001d8c0 f   moc_ORFDialog.obj
 0001:0001c9a0       ?registerConverter@?$AssociativeContainerConverterHelper@PAVTask@U2@@$0A@@QtPrivate@@SA_NH@Z 1001d9a0 f i moc_ORFDialog.obj
 0001:0001c9b0       ?registerConverter@?$IsPair@PAVTask@U2@@@QtPrivate@@SA_NH@Z 1001d9b0 f i moc_ORFDialog.obj
 0001:0001c9c0       ?registerConverter@?$MetaTypeSmartPointerHelper@PAVTask@U2@@X@QtPrivate@@SA_NH@Z 1001d9c0 f i moc_ORFDialog.obj
 0001:0001c9d0       ?registerConverter@?$SequentialContainerConverterHelper@PAVTask@U2@@$0A@@QtPrivate@@SA_NH@Z 1001d9d0 f i moc_ORFDialog.obj
 0001:0001c9e0       ?value@?$MetaObjectForType@PAVTask@U2@@$00@QtPrivate@@SAPBUQMetaObject@@XZ 1001d9e0 f i moc_ORFDialog.obj
 0001:0001c9f0       ?metaObject@ORFMarkerPlugin@U2@@UBEPBUQMetaObject@@XZ 1001d9f0 f   moc_ORFMarkerPlugin.obj
 0001:0001ca10       ?metaObject@ORFViewContext@U2@@UBEPBUQMetaObject@@XZ 1001da10 f   moc_ORFMarkerPlugin.obj
 0001:0001ca30       ?qt_metacall@ORFMarkerPlugin@U2@@UAEHW4Call@QMetaObject@@HPAPAX@Z 1001da30 f   moc_ORFMarkerPlugin.obj
 0001:0001ca40       ?qt_metacall@ORFViewContext@U2@@UAEHW4Call@QMetaObject@@HPAPAX@Z 1001da40 f   moc_ORFMarkerPlugin.obj
 0001:0001caa0       ?qt_metacast@ORFMarkerPlugin@U2@@UAEPAXPBD@Z 1001daa0 f   moc_ORFMarkerPlugin.obj
 0001:0001cb00       ?qt_metacast@ORFViewContext@U2@@UAEPAXPBD@Z 1001db00 f   moc_ORFMarkerPlugin.obj
 0001:0001cb60       ?qt_static_metacall@ORFMarkerPlugin@U2@@CAXPAVQObject@@W4Call@QMetaObject@@HPAPAX@Z 1001db60 f   moc_ORFMarkerPlugin.obj
 0001:0001cb70       ?qt_static_metacall@ORFViewContext@U2@@CAXPAVQObject@@W4Call@QMetaObject@@HPAPAX@Z 1001db70 f   moc_ORFMarkerPlugin.obj
 0001:0001cb90       ?metaObject@FindORFsToAnnotationsTask@U2@@UBEPBUQMetaObject@@XZ 1001db90 f   moc_ORFMarkerTask.obj
 0001:0001cbb0       ?metaObject@ORFAutoAnnotationsUpdater@U2@@UBEPBUQMetaObject@@XZ 1001dbb0 f   moc_ORFMarkerTask.obj
 0001:0001cbd0       ?qt_metacall@FindORFsToAnnotationsTask@U2@@UAEHW4Call@QMetaObject@@HPAPAX@Z 1001dbd0 f   moc_ORFMarkerTask.obj
 0001:0001cbe0       ?qt_metacall@ORFAutoAnnotationsUpdater@U2@@UAEHW4Call@QMetaObject@@HPAPAX@Z 1001dbe0 f   moc_ORFMarkerTask.obj
 0001:0001cbf0       ?qt_metacast@FindORFsToAnnotationsTask@U2@@UAEPAXPBD@Z 1001dbf0 f   moc_ORFMarkerTask.obj
 0001:0001cc50       ?qt_metacast@ORFAutoAnnotationsUpdater@U2@@UAEPAXPBD@Z 1001dc50 f   moc_ORFMarkerTask.obj
 0001:0001ccb0       ?qt_static_metacall@FindORFsToAnnotationsTask@U2@@CAXPAVQObject@@W4Call@QMetaObject@@HPAPAX@Z 1001dcb0 f   moc_ORFMarkerTask.obj
 0001:0001ccc0       ?qt_static_metacall@ORFAutoAnnotationsUpdater@U2@@CAXPAVQObject@@W4Call@QMetaObject@@HPAPAX@Z 1001dcc0 f   moc_ORFMarkerTask.obj
 0001:0001ccd0       ?metaObject@GTest_ORFMarkerTask@U2@@UBEPBUQMetaObject@@XZ 1001dcd0 f   moc_ORFMarkerTests.obj
 0001:0001ccf0       ?qt_metacall@GTest_ORFMarkerTask@U2@@UAEHW4Call@QMetaObject@@HPAPAX@Z 1001dcf0 f   moc_ORFMarkerTests.obj
 0001:0001cd00       ?qt_metacast@GTest_ORFMarkerTask@U2@@UAEPAXPBD@Z 1001dd00 f   moc_ORFMarkerTests.obj
 0001:0001cd60       ?qt_static_metacall@GTest_ORFMarkerTask@U2@@CAXPAVQObject@@W4Call@QMetaObject@@HPAPAX@Z 1001dd60 f   moc_ORFMarkerTests.obj
 0001:0001cd70       ?metaObject@QDORFActor@U2@@UBEPBUQMetaObject@@XZ 1001dd70 f   moc_ORFQuery.obj
 0001:0001cd90       ?qt_metacall@QDORFActor@U2@@UAEHW4Call@QMetaObject@@HPAPAX@Z 1001dd90 f   moc_ORFQuery.obj
 0001:0001cdf0       ?qt_metacast@QDORFActor@U2@@UAEPAXPBD@Z 1001ddf0 f   moc_ORFQuery.obj
 0001:0001ce50       ?qt_static_metacall@QDORFActor@U2@@CAXPAVQObject@@W4Call@QMetaObject@@HPAPAX@Z 1001de50 f   moc_ORFQuery.obj
 0001:0001ceb0       ?metaObject@ORFPrompter@LocalWorkflow@U2@@UBEPBUQMetaObject@@XZ 1001deb0 f   moc_ORFWorker.obj
 0001:0001ced0       ?metaObject@ORFWorker@LocalWorkflow@U2@@UBEPBUQMetaObject@@XZ 1001ded0 f   moc_ORFWorker.obj
 0001:0001cef0       ?qt_metacall@ORFPrompter@LocalWorkflow@U2@@UAEHW4Call@QMetaObject@@HPAPAX@Z 1001def0 f   moc_ORFWorker.obj
 0001:0001cf00       ?qt_metacall@ORFWorker@LocalWorkflow@U2@@UAEHW4Call@QMetaObject@@HPAPAX@Z 1001df00 f   moc_ORFWorker.obj
 0001:0001cf60       ?qt_metacast@ORFPrompter@LocalWorkflow@U2@@UAEPAXPBD@Z 1001df60 f   moc_ORFWorker.obj
 0001:0001cfc0       ?qt_metacast@ORFWorker@LocalWorkflow@U2@@UAEPAXPBD@Z 1001dfc0 f   moc_ORFWorker.obj
 0001:0001d020       ?qt_static_metacall@ORFPrompter@LocalWorkflow@U2@@CAXPAVQObject@@W4Call@QMetaObject@@HPAPAX@Z 1001e020 f   moc_ORFWorker.obj
 0001:0001d030       ?qt_static_metacall@ORFWorker@LocalWorkflow@U2@@CAXPAVQObject@@W4Call@QMetaObject@@HPAPAX@Z 1001e030 f   moc_ORFWorker.obj
 0001:0001d050       ??0initializer@?A0xaf06a44c@@QAE@XZ 1001e050 f i qrc_orf_marker.obj
 0001:0001d070       ??1initializer@?A0xaf06a44c@@QAE@XZ 1001e070 f i qrc_orf_marker.obj
 0001:0001d090       ?qCleanupResources_orf_marker@@YAHXZ 1001e090 f   qrc_orf_marker.obj
 0001:0001d0b0       ?qInitResources_orf_marker@@YAHXZ 1001e0b0 f   qrc_orf_marker.obj
 0001:0001d0d0       ?intersect@U2Region@U2@@QBE?AV12@ABV12@@Z 1001e0d0 f   U2Core:U2Core.dll
 0001:0001d0d6       ?setRegion@LRegionsSelection@U2@@QAEXABVU2Region@2@@Z 1001e0d6 f   U2Core:U2Core.dll
 0001:0001d0dc       ??0Logger@U2@@QAE@ABVQString@@@Z 1001e0dc f   U2Core:U2Core.dll
 0001:0001d0e2       ??1Logger@U2@@UAE@XZ       1001e0e2 f   U2Core:U2Core.dll
 0001:0001d0e8       ?error@Logger@U2@@QAEXABVQString@@@Z 1001e0e8 f   U2Core:U2Core.dll
 0001:0001d0ee       ?getTaskName@Task@U2@@QBE?AVQString@@XZ 1001e0ee f   U2Core:U2Core.dll
 0001:0001d0f4       ?cancel@Task@U2@@QAEXXZ    1001e0f4 f   U2Core:U2Core.dll
 0001:0001d0fa       ??8U2EntityRef@U2@@QBE_NABV01@@Z 1001e0fa f   U2Core:U2Core.dll
 0001:0001d100       ??0GObjectReference@U2@@QAE@PBVGObject@1@_N@Z 1001e100 f   U2Core:U2Core.dll
 0001:0001d106       ??1GObjectReference@U2@@QAE@XZ 1001e106 f   U2Core:U2Core.dll
 0001:0001d10c       ??4GObjectReference@U2@@QAEAAV01@ABV01@@Z 1001e10c f   U2Core:U2Core.dll
 0001:0001d112       ?getSequenceLength@U2SequenceObject@U2@@QBE_JXZ 1001e112 f   U2Core:U2Core.dll
 0001:0001d118       ?isCircular@U2SequenceObject@U2@@QBE_NXZ 1001e118 f   U2Core:U2Core.dll
 0001:0001d11e       ??1AnnotationData@U2@@QAE@XZ 1001e11e f   U2Core:U2Core.dll
 0001:0001d124       ??0AnnotationData@U2@@QAE@ABV01@@Z 1001e124 f   U2Core:U2Core.dll
 0001:0001d12a       ?getSettings@AppContext@U2@@SAPAVSettings@2@XZ 1001e12a f   U2Core:U2Core.dll
 0001:0001d130       ?getTaskScheduler@AppContext@U2@@SAPAVTaskScheduler@2@XZ 1001e130 f   U2Core:U2Core.dll
 0001:0001d136       ?warningTitle@L10N@U2@@SA?AVQString@@XZ 1001e136 f   U2Core:U2Core.dll
 0001:0001d13c       ?getSequenceObject@AutoAnnotationsUpdateTask@U2@@QBEPAVU2SequenceObject@2@XZ 1001e13c f   U2Core:U2Core.dll
 0001:0001d142       ?cleanup@Task@U2@@UAEXXZ   1001e142 f   U2Core:U2Core.dll
 0001:0001d148       ?generateReport@Task@U2@@UBE?AVQString@@XZ 1001e148 f   U2Core:U2Core.dll
 0001:0001d14e       ?getNumParallelSubtasks@Task@U2@@UBEHXZ 1001e14e f   U2Core:U2Core.dll
 0001:0001d154       ?getParentTask@Task@U2@@UBEPAV12@XZ 1001e154 f   U2Core:U2Core.dll
 0001:0001d15a       ?getSubtaskWithErrors@Task@U2@@UBEPAV12@XZ 1001e15a f   U2Core:U2Core.dll
 0001:0001d160       ?getTaskId@Task@U2@@UBE_JXZ 1001e160 f   U2Core:U2Core.dll
 0001:0001d166       ?getTopLevelParentTask@Task@U2@@UAEPAV12@XZ 1001e166 f   U2Core:U2Core.dll
 0001:0001d16c       ?getWarnings@Task@U2@@UBE?AVQStringList@@XZ 1001e16c f   U2Core:U2Core.dll
 0001:0001d172       ?hasSubtasksWithErrors@Task@U2@@UBE_NXZ 1001e172 f   U2Core:U2Core.dll
 0001:0001d178       ?hasWarning@Task@U2@@UBE_NXZ 1001e178 f   U2Core:U2Core.dll
 0001:0001d17e       ?isNotificationReport@Task@U2@@UBE_NXZ 1001e17e f   U2Core:U2Core.dll
 0001:0001d184       ?isReportingEnabled@Task@U2@@UBE_NXZ 1001e184 f   U2Core:U2Core.dll
 0001:0001d18a       ?isReportingSupported@Task@U2@@UBE_NXZ 1001e18a f   U2Core:U2Core.dll
 0001:0001d190       ?isTopLevelTask@Task@U2@@UBE_NXZ 1001e190 f   U2Core:U2Core.dll
 0001:0001d196       ?onSubTaskFinished@Task@U2@@MAE?AV?$QList@PAVTask@U2@@@@PAV12@@Z 1001e196 f   U2Core:U2Core.dll
 0001:0001d19c       ?prepare@Task@U2@@UAEXXZ   1001e19c f   U2Core:U2Core.dll
 0001:0001d1a2       ?propagateSubtaskError@Task@U2@@UAE_NXZ 1001e1a2 f   U2Core:U2Core.dll
 0001:0001d1a8       ?report@Task@U2@@UAE?AW4ReportResult@12@XZ 1001e1a8 f   U2Core:U2Core.dll
 0001:0001d1ae       ?setCollectChildrensWarningsFlag@Task@U2@@UAEX_N@Z 1001e1ae f   U2Core:U2Core.dll
 0001:0001d1b4       ?setNoAutoDelete@Task@U2@@UAEX_N@Z 1001e1b4 f   U2Core:U2Core.dll
 0001:0001d1ba       ?setNotificationReport@Task@U2@@UAEX_N@Z 1001e1ba f   U2Core:U2Core.dll
 0001:0001d1c0       ?setReportingEnabled@Task@U2@@UAEX_N@Z 1001e1c0 f   U2Core:U2Core.dll
 0001:0001d1c6       ?setReportingSupported@Task@U2@@UAEX_N@Z 1001e1c6 f   U2Core:U2Core.dll
 0001:0001d1cc       ?getMainWindow@AppContext@U2@@SAPAVMainWindow@2@XZ 1001e1cc f   U2Core:U2Core.dll
 0001:0001d1d2       ?getTestFramework@AppContext@U2@@SAPAVTestFramework@2@XZ 1001e1d2 f   U2Core:U2Core.dll
 0001:0001d1d8       ?getAutoAnnotationsSupport@AppContext@U2@@SAPAVAutoAnnotationsSupport@2@XZ 1001e1d8 f   U2Core:U2Core.dll
 0001:0001d1de       ?getQDActorProtoRegistry@AppContext@U2@@SAPAVQDActorPrototypeRegistry@2@XZ 1001e1de f   U2Core:U2Core.dll
 0001:0001d1e4       ?registerAutoAnnotationsUpdater@AutoAnnotationsSupport@U2@@QAEXPAVAutoAnnotationsUpdater@2@@Z 1001e1e4 f   U2Core:U2Core.dll
 0001:0001d1ea       ??0Plugin@U2@@QAE@ABVQString@@0_NW4PluginState@1@@Z 1001e1ea f   U2Core:U2Core.dll
 0001:0001d1f0       ??1Plugin@U2@@UAE@XZ       1001e1f0 f   U2Core:U2Core.dll
 0001:0001d1f6       ?run@Task@U2@@UAEXXZ       1001e1f6 f   U2Core:U2Core.dll
 0001:0001d1fc       ??1U2EntityRef@U2@@QAE@XZ  1001e1fc f   U2Core:U2Core.dll
 0001:0001d202       ??0U2EntityRef@U2@@QAE@ABV01@@Z 1001e202 f   U2Core:U2Core.dll
 0001:0001d208       ?getDNATranslationRegistry@AppContext@U2@@SAPAVDNATranslationRegistry@2@XZ 1001e208 f   U2Core:U2Core.dll
 0001:0001d20e       ??0Task@U2@@QAE@ABVQString@@V?$QFlags@W4TaskFlag@U2@@@@@Z 1001e20e f   U2Core:U2Core.dll
 0001:0001d214       ?addSubTask@Task@U2@@QAEXPAV12@@Z 1001e214 f   U2Core:U2Core.dll
 0001:0001d21a       ?setError@Task@U2@@QAEXABVQString@@@Z 1001e21a f   U2Core:U2Core.dll
 0001:0001d220       ??1Task@U2@@UAE@XZ         1001e220 f   U2Core:U2Core.dll
 0001:0001d226       ??0CreateAnnotationsTask@U2@@QAE@PAVAnnotationTableObject@1@ABV?$QList@V?$QSharedDataPointer@VAnnotationData@U2@@@@@@ABVQString@@@Z 1001e226 f   U2Core:U2Core.dll
 0001:0001d22c       ??1CreateAnnotationsTask@U2@@UAE@XZ 1001e22c f   U2Core:U2Core.dll
 0001:0001d232       ?lookupTranslation@DNATranslationRegistry@U2@@QAEPAVDNATranslation@2@ABVQString@@@Z 1001e232 f   U2Core:U2Core.dll
 0001:0001d238       ?findComplementTT@GObjectUtils@U2@@SAPAVDNATranslation@2@PBVDNAAlphabet@2@@Z 1001e238 f   U2Core:U2Core.dll
 0001:0001d23e       ?addDescriptionQualifier@U1AnnotationUtils@U2@@SAXAAV?$QList@V?$QSharedDataPointer@VAnnotationData@U2@@@@@@ABVQString@@@Z 1001e23e f   U2Core:U2Core.dll
 0001:0001d244       ?getSequenceRef@U2SequenceObject@U2@@QBE?AVU2EntityRef@2@XZ 1001e244 f   U2Core:U2Core.dll
 0001:0001d24a       ?getAlphabet@U2SequenceObject@U2@@QBEPBVDNAAlphabet@2@XZ 1001e24a f   U2Core:U2Core.dll
 0001:0001d250       ?getAminoTT@AutoAnnotationObject@U2@@QBEPAVDNATranslation@2@XZ 1001e250 f   U2Core:U2Core.dll
 0001:0001d256       ??0AutoAnnotationsUpdater@U2@@QAE@ABVQString@@0_N1@Z 1001e256 f   U2Core:U2Core.dll
 0001:0001d25c       ??1AutoAnnotationsUpdater@U2@@UAE@XZ 1001e25c f   U2Core:U2Core.dll
 0001:0001d262       ?metaObject@CreateAnnotationsTask@U2@@UBEPBUQMetaObject@@XZ 1001e262 f   U2Core:U2Core.dll
 0001:0001d268       ?qt_metacall@CreateAnnotationsTask@U2@@UAEHW4Call@QMetaObject@@HPAPAX@Z 1001e268 f   U2Core:U2Core.dll
 0001:0001d26e       ?qt_metacast@CreateAnnotationsTask@U2@@UAEPAXPBD@Z 1001e26e f   U2Core:U2Core.dll
 0001:0001d274       ?report@CreateAnnotationsTask@U2@@UAE?AW4ReportResult@Task@2@XZ 1001e274 f   U2Core:U2Core.dll
 0001:0001d27a       ?run@CreateAnnotationsTask@U2@@UAEXXZ 1001e27a f   U2Core:U2Core.dll
 0001:0001d280       ?lookupTranslation@DNATranslationRegistry@U2@@QAEPAVDNATranslation@2@PBVDNAAlphabet@2@W4DNATranslationType@2@ABVQString@@@Z 1001e280 f   U2Core:U2Core.dll
 0001:0001d286       ?lookupComplementTranslation@DNATranslationRegistry@U2@@QAEPAVDNATranslation@2@PBVDNAAlphabet@2@@Z 1001e286 f   U2Core:U2Core.dll
 0001:0001d28c       ??CU2Location@U2@@QBEPBVU2LocationData@1@XZ 1001e28c f   U2Core:U2Core.dll
 0001:0001d292       ??1U2Qualifier@U2@@QAE@XZ  1001e292 f   U2Core:U2Core.dll
 0001:0001d298       ??0U2Qualifier@U2@@QAE@ABV01@@Z 1001e298 f   U2Core:U2Core.dll
 0001:0001d29e       ?getStrand@AnnotationData@U2@@QBE?AVU2Strand@2@XZ 1001e29e f   U2Core:U2Core.dll
 0001:0001d2a4       ?getDNAAlphabetRegistry@AppContext@U2@@SAPAVDNAAlphabetRegistry@2@XZ 1001e2a4 f   U2Core:U2Core.dll
 0001:0001d2aa       ?lookupTranslation@DNATranslationRegistry@U2@@QAE?AV?$QList@PAVDNATranslation@U2@@@@PBVDNAAlphabet@2@W4DNATranslationType@2@@Z 1001e2aa f   U2Core:U2Core.dll
 0001:0001d2b0       ?NUCL_DNA_DEFAULT@BaseDNAAlphabetIds@U2@@SA?BVQString@@XZ 1001e2b0 f   U2Core:U2Core.dll
 0001:0001d2b6       ??0TaskSignalMapper@U2@@QAE@PAVTask@1@@Z 1001e2b6 f   U2Core:U2Core.dll
 0001:0001d2bc       ??0FailTask@U2@@QAE@ABVQString@@@Z 1001e2bc f   U2Core:U2Core.dll
 0001:0001d2c2       ??1FailTask@U2@@UAE@XZ     1001e2c2 f   U2Core:U2Core.dll
 0001:0001d2c8       ?suffixBp@L10N@U2@@SA?AVQString@@XZ 1001e2c8 f   U2Core:U2Core.dll
 0001:0001d2ce       ?metaObject@FailTask@U2@@UBEPBUQMetaObject@@XZ 1001e2ce f   U2Core:U2Core.dll
 0001:0001d2d4       ?metaObject@Task@U2@@UBEPBUQMetaObject@@XZ 1001e2d4 f   U2Core:U2Core.dll
 0001:0001d2da       ?metaObject@TaskSignalMapper@U2@@UBEPBUQMetaObject@@XZ 1001e2da f   U2Core:U2Core.dll
 0001:0001d2e0       ?qt_metacall@FailTask@U2@@UAEHW4Call@QMetaObject@@HPAPAX@Z 1001e2e0 f   U2Core:U2Core.dll
 0001:0001d2e6       ?qt_metacall@Task@U2@@UAEHW4Call@QMetaObject@@HPAPAX@Z 1001e2e6 f   U2Core:U2Core.dll
 0001:0001d2ec       ?qt_metacall@TaskSignalMapper@U2@@UAEHW4Call@QMetaObject@@HPAPAX@Z 1001e2ec f   U2Core:U2Core.dll
 0001:0001d2f2       ?qt_metacast@FailTask@U2@@UAEPAXPBD@Z 1001e2f2 f   U2Core:U2Core.dll
 0001:0001d2f8       ?qt_metacast@Task@U2@@UAEPAXPBD@Z 1001e2f8 f   U2Core:U2Core.dll
 0001:0001d2fe       ?qt_metacast@TaskSignalMapper@U2@@UAEPAXPBD@Z 1001e2fe f   U2Core:U2Core.dll
 0001:0001d304       ?info@Logger@U2@@QAEXABVQString@@@Z 1001e304 f   U2Core:U2Core.dll
 0001:0001d30a       ??0TaskStateInfo@U2@@QAE@XZ 1001e30a f   U2Core:U2Core.dll
 0001:0001d310       ?getError@TaskStateInfo@U2@@UBE?AVQString@@XZ 1001e310 f   U2Core:U2Core.dll
 0001:0001d316       ?setError@TaskStateInfo@U2@@UAEXABVQString@@@Z 1001e316 f   U2Core:U2Core.dll
 0001:0001d31c       ??1TaskStateInfo@U2@@UAE@XZ 1001e31c f   U2Core:U2Core.dll
 0001:0001d322       ?hasError@Task@U2@@QBE_NXZ 1001e322 f   U2Core:U2Core.dll
 0001:0001d328       ?runScript@ScriptTask@U2@@SA?AVQScriptValue@@PAVQScriptEngine@@ABV?$QMap@VQString@@VQScriptValue@@@@ABVQString@@AAVTaskStateInfo@2@@Z 1001e328 f   U2Core:U2Core.dll
 0001:0001d32e       ?getSequenceName@U2SequenceObject@U2@@QBE?AVQString@@XZ 1001e32e f   U2Core:U2Core.dll
 0001:0001d334       ?qt_metacast@Plugin@U2@@UAEPAXPBD@Z 1001e334 f   U2Core:U2Core.dll
 0001:0001d33a       ?qt_metacall@Plugin@U2@@UAEHW4Call@QMetaObject@@HPAPAX@Z 1001e33a f   U2Core:U2Core.dll
 0001:0001d340       ?qt_metacast@AutoAnnotationsUpdater@U2@@UAEPAXPBD@Z 1001e340 f   U2Core:U2Core.dll
 0001:0001d346       ?qt_metacall@AutoAnnotationsUpdater@U2@@UAEHW4Call@QMetaObject@@HPAPAX@Z 1001e346 f   U2Core:U2Core.dll
 0001:0001d34c       ??0ORFFindTask@U2@@QAE@ABVORFAlgorithmSettings@1@ABVU2EntityRef@1@@Z 1001e34c f   U2Algorithm:U2Algorithm.dll
 0001:0001d352       ?popResults@ORFFindTask@U2@@QAE?AV?$QList@VORFFindResult@U2@@@@XZ 1001e352 f   U2Algorithm:U2Algorithm.dll
 0001:0001d358       ??1ORFFindTask@U2@@UAE@XZ  1001e358 f   U2Algorithm:U2Algorithm.dll
 0001:0001d35e       ?metaObject@ORFFindTask@U2@@UBEPBUQMetaObject@@XZ 1001e35e f   U2Algorithm:U2Algorithm.dll
 0001:0001d364       ?onResult@ORFFindTask@U2@@UAEXABVORFFindResult@2@AAVU2OpStatus@2@@Z 1001e364 f   U2Algorithm:U2Algorithm.dll
 0001:0001d36a       ?qt_metacall@ORFFindTask@U2@@UAEHW4Call@QMetaObject@@HPAPAX@Z 1001e36a f   U2Algorithm:U2Algorithm.dll
 0001:0001d370       ?qt_metacast@ORFFindTask@U2@@UAEPAXPBD@Z 1001e370 f   U2Algorithm:U2Algorithm.dll
 0001:0001d376       ?run@ORFFindTask@U2@@UAEXXZ 1001e376 f   U2Algorithm:U2Algorithm.dll
 0001:0001d37c       ?toAnnotation@ORFFindResult@U2@@QBE?AV?$QSharedDataPointer@VAnnotationData@U2@@@@ABVQString@@@Z 1001e37c f   U2Algorithm:U2Algorithm.dll
 0001:0001d382       ?getStrandStringId@ORFAlgorithmSettings@U2@@SA?AVQString@@W4ORFAlgorithmStrand@2@@Z 1001e382 f   U2Algorithm:U2Algorithm.dll
 0001:0001d388       ?getStrandByStringId@ORFAlgorithmSettings@U2@@SA?AW4ORFAlgorithmStrand@2@ABVQString@@@Z 1001e388 f   U2Algorithm:U2Algorithm.dll
 0001:0001d38e       ?toTable@ORFFindResult@U2@@SA?AV?$QList@V?$QSharedDataPointer@VAnnotationData@U2@@@@@@ABV?$QList@VORFFindResult@U2@@@@ABVQString@@@Z 1001e38e f   U2Algorithm:U2Algorithm.dll
 0001:0001d394       ??0RegionSelector@U2@@QAE@PAVQWidget@@_J_NPAVDNASequenceSelection@1@2V?$QList@URegionPreset@U2@@@@@Z 1001e394 f   U2Gui:U2Gui.dll
 0001:0001d39a       ?getRegion@RegionSelector@U2@@QBE?AVU2Region@2@PA_N@Z 1001e39a f   U2Gui:U2Gui.dll
 0001:0001d3a0       ?isWholeSequenceSelected@RegionSelector@U2@@QBE_NXZ 1001e3a0 f   U2Gui:U2Gui.dll
 0001:0001d3a6       ?setWholeRegionSelected@RegionSelector@U2@@QAEXXZ 1001e3a6 f   U2Gui:U2Gui.dll
 0001:0001d3ac       ?showErrorMessage@RegionSelector@U2@@QAEXXZ 1001e3ac f   U2Gui:U2Gui.dll
 0001:0001d3b2       ?getWidget@GObjectView@U2@@QAEPAVQWidget@@XZ 1001e3b2 f   U2Gui:U2Gui.dll
 0001:0001d3b8       ??0CreateAnnotationModel@U2@@QAE@XZ 1001e3b8 f   U2Gui:U2Gui.dll
 0001:0001d3be       ?getAnnotationObject@CreateAnnotationModel@U2@@QBEPAVAnnotationTableObject@2@XZ 1001e3be f   U2Gui:U2Gui.dll
 0001:0001d3c4       ??1CreateAnnotationModel@U2@@QAE@XZ 1001e3c4 f   U2Gui:U2Gui.dll
 0001:0001d3ca       ??0CreateAnnotationWidgetController@U2@@QAE@ABVCreateAnnotationModel@1@PAVQObject@@W4AnnotationWidgetMode@01@@Z 1001e3ca f   U2Gui:U2Gui.dll
 0001:0001d3d0       ?validate@CreateAnnotationWidgetController@U2@@QAE?AVQString@@XZ 1001e3d0 f   U2Gui:U2Gui.dll
 0001:0001d3d6       ?prepareAnnotationObject@CreateAnnotationWidgetController@U2@@QAE_NXZ 1001e3d6 f   U2Gui:U2Gui.dll
 0001:0001d3dc       ?useAutoAnnotationModel@CreateAnnotationWidgetController@U2@@QBE_NXZ 1001e3dc f   U2Gui:U2Gui.dll
 0001:0001d3e2       ?getWidget@CreateAnnotationWidgetController@U2@@QBEPAVQWidget@@XZ 1001e3e2 f   U2Gui:U2Gui.dll
 0001:0001d3e8       ??1CreateAnnotationWidgetController@U2@@UAE@XZ 1001e3e8 f   U2Gui:U2Gui.dll
 0001:0001d3ee       ??0HelpButton@U2@@QAE@PAVQObject@@PAVQDialogButtonBox@@ABVQString@@@Z 1001e3ee f   U2Gui:U2Gui.dll
 0001:0001d3f4       ??1HelpButton@U2@@UAE@XZ   1001e3f4 f   U2Gui:U2Gui.dll
 0001:0001d3fa       ?metaObject@CreateAnnotationWidgetController@U2@@UBEPBUQMetaObject@@XZ 1001e3fa f   U2Gui:U2Gui.dll
 0001:0001d400       ?metaObject@HelpButton@U2@@UBEPBUQMetaObject@@XZ 1001e400 f   U2Gui:U2Gui.dll
 0001:0001d406       ?metaObject@RegionSelector@U2@@UBEPBUQMetaObject@@XZ 1001e406 f   U2Gui:U2Gui.dll
 0001:0001d40c       ?qt_metacall@CreateAnnotationWidgetController@U2@@UAEHW4Call@QMetaObject@@HPAPAX@Z 1001e40c f   U2Gui:U2Gui.dll
 0001:0001d412       ?qt_metacall@HelpButton@U2@@UAEHW4Call@QMetaObject@@HPAPAX@Z 1001e412 f   U2Gui:U2Gui.dll
 0001:0001d418       ?qt_metacall@RegionSelector@U2@@UAEHW4Call@QMetaObject@@HPAPAX@Z 1001e418 f   U2Gui:U2Gui.dll
 0001:0001d41e       ?qt_metacast@CreateAnnotationWidgetController@U2@@UAEPAXPBD@Z 1001e41e f   U2Gui:U2Gui.dll
 0001:0001d424       ?qt_metacast@HelpButton@U2@@UAEPAXPBD@Z 1001e424 f   U2Gui:U2Gui.dll
 0001:0001d42a       ?qt_metacast@RegionSelector@U2@@UAEPAXPBD@Z 1001e42a f   U2Gui:U2Gui.dll
 0001:0001d430       ?sl_buttonClicked@HelpButton@U2@@MAEXXZ 1001e430 f   U2Gui:U2Gui.dll
 0001:0001d436       ?getObjectView@GObjectViewAction@U2@@QBEPAVGObjectView@2@XZ 1001e436 f   U2Gui:U2Gui.dll
 0001:0001d43c       ??0GObjectViewWindowContext@U2@@QAE@PAVQObject@@ABVGObjectViewFactoryId@1@@Z 1001e43c f   U2Gui:U2Gui.dll
 0001:0001d442       ??1GObjectViewWindowContext@U2@@UAE@XZ 1001e442 f   U2Gui:U2Gui.dll
 0001:0001d448       ?buildMenu@GObjectViewWindowContext@U2@@MAEXPAVGObjectView@2@PAVQMenu@@@Z 1001e448 f   U2Gui:U2Gui.dll
 0001:0001d44e       ?canHandle@GObjectViewObjectHandler@U2@@UAE_NPAVGObjectView@2@PAVGObject@2@@Z 1001e44e f   U2Gui:U2Gui.dll
 0001:0001d454       ?disconnectView@GObjectViewWindowContext@U2@@MAEXPAVGObjectView@2@@Z 1001e454 f   U2Gui:U2Gui.dll
 0001:0001d45a       ?init@GObjectViewWindowContext@U2@@UAEXXZ 1001e45a f   U2Gui:U2Gui.dll
 0001:0001d460       ?onObjectAdded@GObjectViewObjectHandler@U2@@UAEXPAVGObjectView@2@PAVGObject@2@@Z 1001e460 f   U2Gui:U2Gui.dll
 0001:0001d466       ?onObjectRemoved@GObjectViewWindowContext@U2@@UAEXPAVGObjectView@2@PAVGObject@2@@Z 1001e466 f   U2Gui:U2Gui.dll
 0001:0001d46c       ?sl_buildContextMenu@GObjectViewWindowContext@U2@@MAEXPAVGObjectView@2@PAVQMenu@@@Z 1001e46c f   U2Gui:U2Gui.dll
 0001:0001d472       ?sl_buildStaticMenu@GObjectViewWindowContext@U2@@MAEXPAVGObjectView@2@PAVQMenu@@@Z 1001e472 f   U2Gui:U2Gui.dll
 0001:0001d478       ?sl_windowAdded@GObjectViewWindowContext@U2@@MAEXPAVMWMDIWindow@2@@Z 1001e478 f   U2Gui:U2Gui.dll
 0001:0001d47e       ?sl_windowClosing@GObjectViewWindowContext@U2@@MAEXPAVMWMDIWindow@2@@Z 1001e47e f   U2Gui:U2Gui.dll
 0001:0001d484       ?qt_metacast@GObjectViewWindowContext@U2@@UAEPAXPBD@Z 1001e484 f   U2Gui:U2Gui.dll
 0001:0001d48a       ?qt_metacall@GObjectViewWindowContext@U2@@UAEHW4Call@QMetaObject@@HPAPAX@Z 1001e48a f   U2Gui:U2Gui.dll
 0001:0001d490       ?triggerAutoAnnotationsUpdate@AutoAnnotationUtils@U2@@SAXPAVADVSequenceObjectContext@2@ABVQString@@@Z 1001e490 f   U2View:U2View.dll
 0001:0001d496       ?getSequenceLength@SequenceObjectContext@U2@@QBE_JXZ 1001e496 f   U2View:U2View.dll
 0001:0001d49c       ?createGeneticCodeMenu@SequenceObjectContext@U2@@QAEPAVQMenu@@XZ 1001e49c f   U2View:U2View.dll
 0001:0001d4a2       ?tryAddObject@AnnotatedDNAView@U2@@QAE?AVQString@@PAVGObject@2@@Z 1001e4a2 f   U2View:U2View.dll
 0001:0001d4a8       ??0ADVGlobalAction@U2@@QAE@PAVAnnotatedDNAView@1@ABVQIcon@@ABVQString@@HV?$QFlags@W4ADVGlobalActionFlag@U2@@@@@Z 1001e4a8 f   U2View:U2View.dll
 0001:0001d4ae       ?addAlphabetFilter@ADVGlobalAction@U2@@QAEXW4DNAAlphabetType@@@Z 1001e4ae f   U2View:U2View.dll
 0001:0001d4b4       ??1ADVGlobalAction@U2@@UAE@XZ 1001e4b4 f   U2View:U2View.dll
 0001:0001d4ba       ?getSequenceInFocus@AnnotatedDNAView@U2@@QBEPAVADVSequenceObjectContext@2@XZ 1001e4ba f   U2View:U2View.dll
 0001:0001d4c0       ?metaObject@ADVGlobalAction@U2@@UBEPBUQMetaObject@@XZ 1001e4c0 f   U2View:U2View.dll
 0001:0001d4c6       ?qt_metacall@ADVGlobalAction@U2@@UAEHW4Call@QMetaObject@@HPAPAX@Z 1001e4c6 f   U2View:U2View.dll
 0001:0001d4cc       ?qt_metacast@ADVGlobalAction@U2@@UAEPAXPBD@Z 1001e4cc f   U2View:U2View.dll
 0001:0001d4d2       ?findFormat@GTestFormatRegistry@U2@@QAEPAVGTestFormat@2@ABVQString@@@Z 1001e4d2 f   U2Test:U2Test.dll
 0001:0001d4d8       ??0XMLTestFactory@U2@@QAE@ABVQString@@@Z 1001e4d8 f   U2Test:U2Test.dll
 0001:0001d4de       ??1XMLTestFactory@U2@@UAE@XZ 1001e4de f   U2Test:U2Test.dll
 0001:0001d4e4       ??0XmlTest@U2@@QAE@ABVQString@@PAVGTest@1@PBVGTestEnvironment@1@V?$QFlags@W4TaskFlag@U2@@@@ABV?$QList@PAVGTest@U2@@@@@Z 1001e4e4 f   U2Test:U2Test.dll
 0001:0001d4ea       ??1XmlTest@U2@@UAE@XZ      1001e4ea f   U2Test:U2Test.dll
 0001:0001d4f0       ?getContext@GTest@U2@@QBEPAVQObject@@ABVQString@@@Z 1001e4f0 f   U2Test:U2Test.dll
 0001:0001d4f6       ?failMissingValue@GTest@U2@@IAEXABVQString@@@Z 1001e4f6 f   U2Test:U2Test.dll
 0001:0001d4fc       ?qt_metacast@GTest@U2@@UAEPAXPBD@Z 1001e4fc f   U2Test:U2Test.dll
 0001:0001d502       ?qt_metacall@GTest@U2@@UAEHW4Call@QMetaObject@@HPAPAX@Z 1001e502 f   U2Test:U2Test.dll
 0001:0001d508       ?registerProto@QDActorPrototypeRegistry@U2@@QAEXPAVQDActorPrototype@2@@Z 1001e508 f   U2Lang:U2Lang.dll
 0001:0001d50e       ??0Descriptor@U2@@QAE@ABVQString@@00@Z 1001e50e f   U2Lang:U2Lang.dll
 0001:0001d514       ??1Descriptor@U2@@UAE@XZ   1001e514 f   U2Lang:U2Lang.dll
 0001:0001d51a       ?setId@Descriptor@U2@@QAEXABVQString@@@Z 1001e51a f   U2Lang:U2Lang.dll
 0001:0001d520       ?setDisplayName@Descriptor@U2@@QAEXABVQString@@@Z 1001e520 f   U2Lang:U2Lang.dll
 0001:0001d526       ?setDocumentation@Descriptor@U2@@QAEXABVQString@@@Z 1001e526 f   U2Lang:U2Lang.dll
 0001:0001d52c       ??0Attribute@U2@@QAE@ABVDescriptor@1@V?$QExplicitlySharedDataPointer@VDataType@U2@@@@_NABVQVariant@@@Z 1001e52c f   U2Lang:U2Lang.dll
 0001:0001d532       ??1Attribute@U2@@UAE@XZ    1001e532 f   U2Lang:U2Lang.dll
 0001:0001d538       ?si_modified@QDParameters@U2@@QAEXXZ 1001e538 f   U2Lang:U2Lang.dll
 0001:0001d53e       ??0QDResultUnitData@U2@@QAE@XZ 1001e53e f   U2Lang:U2Lang.dll
 0001:0001d544       ??1QDResultUnitData@U2@@QAE@XZ 1001e544 f   U2Lang:U2Lang.dll
 0001:0001d54a       ??0QDResultUnitData@U2@@QAE@ABV01@@Z 1001e54a f   U2Lang:U2Lang.dll
 0001:0001d550       ?buildGroupFromSingleResult@QDResultGroup@U2@@SAXABV?$QSharedDataPointer@VQDResultUnitData@U2@@@@AAV?$QList@PAVQDResultGroup@U2@@@@@Z 1001e550 f   U2Lang:U2Lang.dll
 0001:0001d556       ??0QDActorPrototype@U2@@QAE@XZ 1001e556 f   U2Lang:U2Lang.dll
 0001:0001d55c       ??1QDActorPrototype@U2@@UAE@XZ 1001e55c f   U2Lang:U2Lang.dll
 0001:0001d562       ??0QDActor@U2@@QAE@PBVQDActorPrototype@1@@Z 1001e562 f   U2Lang:U2Lang.dll
 0001:0001d568       ??1QDActor@U2@@UAE@XZ      1001e568 f   U2Lang:U2Lang.dll
 0001:0001d56e       ?getStrandToRun@QDActor@U2@@IBE?AW4QDStrandOption@2@XZ 1001e56e f   U2Lang:U2Lang.dll
 0001:0001d574       ??0QDSchemeUnit@U2@@QAE@PAVQDActor@1@@Z 1001e574 f   U2Lang:U2Lang.dll
 0001:0001d57a       ?getEntityRef@QDScheme@U2@@QBE?AVU2EntityRef@2@XZ 1001e57a f   U2Lang:U2Lang.dll
 0001:0001d580       ?STRING_TYPE@BaseTypes@U2@@SA?AV?$QExplicitlySharedDataPointer@VDataType@U2@@@@XZ 1001e580 f   U2Lang:U2Lang.dll
 0001:0001d586       ?BOOL_TYPE@BaseTypes@U2@@SA?AV?$QExplicitlySharedDataPointer@VDataType@U2@@@@XZ 1001e586 f   U2Lang:U2Lang.dll
 0001:0001d58c       ?NUM_TYPE@BaseTypes@U2@@SA?AV?$QExplicitlySharedDataPointer@VDataType@U2@@@@XZ 1001e58c f   U2Lang:U2Lang.dll
 0001:0001d592       ?clone@Attribute@U2@@UAEPAV12@XZ 1001e592 f   U2Lang:U2Lang.dll
 0001:0001d598       ?getAttributePureValue@Attribute@U2@@UBEABVQVariant@@XZ 1001e598 f   U2Lang:U2Lang.dll
 0001:0001d59e       ?getDefaultPureValue@Attribute@U2@@UBEABVQVariant@@XZ 1001e59e f   U2Lang:U2Lang.dll
 0001:0001d5a4       ?getGroup@Attribute@U2@@UAE?AW4AttributeGroup@2@XZ 1001e5a4 f   U2Lang:U2Lang.dll
 0001:0001d5aa       ?getWidget@ConfigurationEditor@U2@@UAEPAVQWidget@@XZ 1001e5aa f   U2Lang:U2Lang.dll
 0001:0001d5b0       ?hasStrand@QDActor@U2@@UBE_NXZ 1001e5b0 f   U2Lang:U2Lang.dll
 0001:0001d5b6       ?isDefaultValue@Attribute@U2@@UBE_NXZ 1001e5b6 f   U2Lang:U2Lang.dll
 0001:0001d5bc       ?isEmpty@Attribute@U2@@UBE_NXZ 1001e5bc f   U2Lang:U2Lang.dll
 0001:0001d5c2       ?isEmpty@ConfigurationEditor@U2@@UBE_NXZ 1001e5c2 f   U2Lang:U2Lang.dll
 0001:0001d5c8       ?loadConfiguration@QDActor@U2@@UAEXABV?$QList@U?$QPair@VQString@@V1@@@@@@Z 1001e5c8 f   U2Lang:U2Lang.dll
 0001:0001d5ce       ?saveConfiguration@QDActor@U2@@UBE?AV?$QList@U?$QPair@VQString@@V1@@@@@XZ 1001e5ce f   U2Lang:U2Lang.dll
 0001:0001d5d4       ?setAttributeValue@Attribute@U2@@UAEXABVQVariant@@@Z 1001e5d4 f   U2Lang:U2Lang.dll
 0001:0001d5da       ?type@PropertyDelegate@U2@@UBE?AW4Type@12@XZ 1001e5da f   U2Lang:U2Lang.dll
 0001:0001d5e0       ?update@PropertyDelegate@U2@@UAEXXZ 1001e5e0 f   U2Lang:U2Lang.dll
 0001:0001d5e6       ?updateActorIds@Attribute@U2@@UAEXABV?$QMap@VQString@@V1@@@@Z 1001e5e6 f   U2Lang:U2Lang.dll
 0001:0001d5ec       ?updateEditor@QDActor@U2@@UAEXXZ 1001e5ec f   U2Lang:U2Lang.dll
 0001:0001d5f2       ?validate@Attribute@U2@@UAE_NAAV?$QList@VWorkflowNotification@U2@@@@@Z 1001e5f2 f   U2Lang:U2Lang.dll
 0001:0001d5f8       ??0Descriptor@U2@@QAE@PBD@Z 1001e5f8 f   U2Lang:U2Lang.dll
 0001:0001d5fe       ?getId@Descriptor@U2@@QBE?AVQString@@XZ 1001e5fe f   U2Lang:U2Lang.dll
 0001:0001d604       ??0Descriptor@U2@@QAE@ABV01@@Z 1001e604 f   U2Lang:U2Lang.dll
 0001:0001d60a       ?setIconPath@VisualDescriptor@U2@@QAEXABVQString@@@Z 1001e60a f   U2Lang:U2Lang.dll
 0001:0001d610       ??0MapDataType@U2@@QAE@ABVDescriptor@1@ABV?$QMap@VDescriptor@U2@@V?$QExplicitlySharedDataPointer@VDataType@U2@@@@@@@Z 1001e610 f   U2Lang:U2Lang.dll
 0001:0001d616       ??1MapDataType@U2@@UAE@XZ  1001e616 f   U2Lang:U2Lang.dll
 0001:0001d61c       ?initEngine@WorkflowScriptLibrary@U2@@SAXPAVWorkflowScriptEngine@2@@Z 1001e61c f   U2Lang:U2Lang.dll
 0001:0001d622       ?getSequenceObject@StorageUtils@Workflow@U2@@SAPAVU2SequenceObject@3@PAVDbiDataStorage@23@ABV?$QSharedDataPointer@VDbiDataHandler@Workflow@U2@@@@@Z 1001e622 f   U2Lang:U2Lang.dll
 0001:0001d628       ?getDataStorage@WorkflowContext@Workflow@U2@@QAEPAVDbiDataStorage@23@XZ 1001e628 f   U2Lang:U2Lang.dll
 0001:0001d62e       ??0WorkflowScriptEngine@U2@@QAE@PAVWorkflowContext@Workflow@1@@Z 1001e62e f   U2Lang:U2Lang.dll
 0001:0001d634       ??1WorkflowScriptEngine@U2@@UAE@XZ 1001e634 f   U2Lang:U2Lang.dll
 0001:0001d63a       ?isEmpty@AttributeScript@U2@@QBE_NXZ 1001e63a f   U2Lang:U2Lang.dll
 0001:0001d640       ?getScriptText@AttributeScript@U2@@QBEABVQString@@XZ 1001e640 f   U2Lang:U2Lang.dll
 0001:0001d646       ?getScriptVars@AttributeScript@U2@@QBEABV?$QMap@VDescriptor@U2@@VQVariant@@@@XZ 1001e646 f   U2Lang:U2Lang.dll
 0001:0001d64c       ?getLabel@Actor@Workflow@U2@@QBE?AVQString@@XZ 1001e64c f   U2Lang:U2Lang.dll
 0001:0001d652       ?getPort@Actor@Workflow@U2@@QBEPAVPort@23@ABVQString@@@Z 1001e652 f   U2Lang:U2Lang.dll
 0001:0001d658       ?getInputPorts@Actor@Workflow@U2@@QBE?AV?$QList@PAVPort@Workflow@U2@@@@XZ 1001e658 f   U2Lang:U2Lang.dll
 0001:0001d65e       ?getOutputPorts@Actor@Workflow@U2@@QBE?AV?$QList@PAVPort@Workflow@U2@@@@XZ 1001e65e f   U2Lang:U2Lang.dll
 0001:0001d664       ??0PortDescriptor@Workflow@U2@@QAE@ABVDescriptor@2@V?$QExplicitlySharedDataPointer@VDataType@U2@@@@_N2I@Z 1001e664 f   U2Lang:U2Lang.dll
 0001:0001d66a       ??1PortDescriptor@Workflow@U2@@UAE@XZ 1001e66a f   U2Lang:U2Lang.dll
 0001:0001d670       ??0ActorPrototype@Workflow@U2@@QAE@ABVDescriptor@2@ABV?$QList@PAVPortDescriptor@Workflow@U2@@@@ABV?$QList@PAVAttribute@U2@@@@@Z 1001e670 f   U2Lang:U2Lang.dll
 0001:0001d676       ??1ActorPrototype@Workflow@U2@@UAE@XZ 1001e676 f   U2Lang:U2Lang.dll
 0001:0001d67c       ?setEditor@ActorPrototype@Workflow@U2@@QAEXPAVConfigurationEditor@3@@Z 1001e67c f   U2Lang:U2Lang.dll
 0001:0001d682       ?setPrompter@ActorPrototype@Workflow@U2@@QAEXPAVPrompter@23@@Z 1001e682 f   U2Lang:U2Lang.dll
 0001:0001d688       ?getProducer@IntegralBusPort@Workflow@U2@@QAEPAVActor@23@ABVQString@@@Z 1001e688 f   U2Lang:U2Lang.dll
 0001:0001d68e       ??0Message@Workflow@U2@@QAE@V?$QExplicitlySharedDataPointer@VDataType@U2@@@@ABVQVariant@@H@Z 1001e68e f   U2Lang:U2Lang.dll
 0001:0001d694       ?getData@Message@Workflow@U2@@QBE?AVQVariant@@XZ 1001e694 f   U2Lang:U2Lang.dll
 0001:0001d69a       ?isEmpty@Message@Workflow@U2@@QBE_NXZ 1001e69a f   U2Lang:U2Lang.dll
 0001:0001d6a0       ?getEmptyMapMessage@Message@Workflow@U2@@SA?AV123@XZ 1001e6a0 f   U2Lang:U2Lang.dll
 0001:0001d6a6       ??1Message@Workflow@U2@@QAE@XZ 1001e6a6 f   U2Lang:U2Lang.dll
 0001:0001d6ac       ??0DomainFactory@Workflow@U2@@QAE@ABVQString@@@Z 1001e6ac f   U2Lang:U2Lang.dll
 0001:0001d6b2       ??1DomainFactory@Workflow@U2@@UAE@XZ 1001e6b2 f   U2Lang:U2Lang.dll
 0001:0001d6b8       ??0BaseWorker@LocalWorkflow@U2@@QAE@PAVActor@Workflow@2@_N@Z 1001e6b8 f   U2Lang:U2Lang.dll
 0001:0001d6be       ??1BaseWorker@LocalWorkflow@U2@@UAE@XZ 1001e6be f   U2Lang:U2Lang.dll
 0001:0001d6c4       ??0PrompterBaseImpl@U2@@QAE@PAVActor@Workflow@1@@Z 1001e6c4 f   U2Lang:U2Lang.dll
 0001:0001d6ca       ?getRequiredParam@PrompterBaseImpl@U2@@QAE?AVQString@@ABV3@@Z 1001e6ca f   U2Lang:U2Lang.dll
 0001:0001d6d0       ?getParameter@PrompterBaseImpl@U2@@QAE?AVQVariant@@ABVQString@@@Z 1001e6d0 f   U2Lang:U2Lang.dll
 0001:0001d6d6       ?getHyperlink@PrompterBaseImpl@U2@@SA?AVQString@@ABV3@0@Z 1001e6d6 f   U2Lang:U2Lang.dll
 0001:0001d6dc       ?getHyperlink@PrompterBaseImpl@U2@@SA?AVQString@@ABV3@H@Z 1001e6dc f   U2Lang:U2Lang.dll
 0001:0001d6e2       ??1PrompterBaseImpl@U2@@UAE@XZ 1001e6e2 f   U2Lang:U2Lang.dll
 0001:0001d6e8       ?getInstance@WorkflowEnv@Workflow@U2@@KAPAV123@XZ 1001e6e8 f   U2Lang:U2Lang.dll
 0001:0001d6ee       ?registerProto@ActorPrototypeRegistry@Workflow@U2@@QAEXABVDescriptor@3@PAVActorPrototype@23@@Z 1001e6ee f   U2Lang:U2Lang.dll
 0001:0001d6f4       ?DNA_SEQUENCE_TYPE@BaseTypes@U2@@SA?AV?$QExplicitlySharedDataPointer@VDataType@U2@@@@XZ 1001e6f4 f   U2Lang:U2Lang.dll
 0001:0001d6fa       ?ANNOTATION_TABLE_TYPE@BaseTypes@U2@@SA?AV?$QExplicitlySharedDataPointer@VDataType@U2@@@@XZ 1001e6fa f   U2Lang:U2Lang.dll
 0001:0001d700       ?DNA_SEQUENCE_SLOT@BaseSlots@Workflow@U2@@SA?BVDescriptor@3@XZ 1001e700 f   U2Lang:U2Lang.dll
 0001:0001d706       ?ANNOTATION_TABLE_SLOT@BaseSlots@Workflow@U2@@SA?BVDescriptor@3@XZ 1001e706 f   U2Lang:U2Lang.dll
 0001:0001d70c       ?IN_SEQ_PORT_ID@BasePorts@Workflow@U2@@SA?BVQString@@XZ 1001e70c f   U2Lang:U2Lang.dll
 0001:0001d712       ?OUT_ANNOTATIONS_PORT_ID@BasePorts@Workflow@U2@@SA?BVQString@@XZ 1001e712 f   U2Lang:U2Lang.dll
 0001:0001d718       ?CATEGORY_BASIC@BaseActorCategories@Workflow@U2@@SA?BVDescriptor@3@XZ 1001e718 f   U2Lang:U2Lang.dll
 0001:0001d71e       ?STRAND_ATTRIBUTE@BaseAttributes@Workflow@U2@@SA?BVDescriptor@3@XZ 1001e71e f   U2Lang:U2Lang.dll
 0001:0001d724       ?STRAND_BOTH@BaseAttributes@Workflow@U2@@SA?BVQString@@XZ 1001e724 f   U2Lang:U2Lang.dll
 0001:0001d72a       ?STRAND_DIRECT@BaseAttributes@Workflow@U2@@SA?BVQString@@XZ 1001e72a f   U2Lang:U2Lang.dll
 0001:0001d730       ?STRAND_COMPLEMENTARY@BaseAttributes@Workflow@U2@@SA?BVQString@@XZ 1001e730 f   U2Lang:U2Lang.dll
 0001:0001d736       ?STRAND_ATTRIBUTE_VALUES_MAP@BaseAttributes@Workflow@U2@@SA?BV?$QMap@VQString@@VQVariant@@@@XZ 1001e736 f   U2Lang:U2Lang.dll
 0001:0001d73c       ?addCommunication@BaseWorker@LocalWorkflow@U2@@UAE_NABVQString@@PAVCommunicationChannel@Workflow@3@@Z 1001e73c f   U2Lang:U2Lang.dll
 0001:0001d742       ?canTaskBeCanceled@BaseWorker@LocalWorkflow@U2@@MBE_NPAVTask@3@@Z 1001e742 f   U2Lang:U2Lang.dll
 0001:0001d748       ?createConnection@DomainFactory@Workflow@U2@@UAEPAVCommunicationChannel@23@PAVLink@23@@Z 1001e748 f   U2Lang:U2Lang.dll
 0001:0001d74e       ?createInstance@ActorPrototype@Workflow@U2@@UAEPAVActor@23@ABVQString@@PAVAttributeScript@3@ABV?$QMap@VQString@@VQVariant@@@@@Z 1001e74e f   U2Lang:U2Lang.dll
 0001:0001d754       ?createPort@IntegralBusActorPrototype@Workflow@U2@@UAEPAVPort@23@ABVPortDescriptor@23@PAVActor@23@@Z 1001e754 f   U2Lang:U2Lang.dll
 0001:0001d75a       ?createScheduler@DomainFactory@Workflow@U2@@UAEPAVScheduler@23@PAVSchema@23@@Z 1001e75a f   U2Lang:U2Lang.dll
 0001:0001d760       ?destroy@DomainFactory@Workflow@U2@@UAEXPAVScheduler@23@PAVSchema@23@@Z 1001e760 f   U2Lang:U2Lang.dll
 0001:0001d766       ?getActorId@BaseWorker@LocalWorkflow@U2@@UBE?AVQString@@XZ 1001e766 f   U2Lang:U2Lang.dll
 0001:0001d76c       ?getAllDescriptors@MapDataType@U2@@UBE?AV?$QList@VDescriptor@U2@@@@XZ 1001e76c f   U2Lang:U2Lang.dll
 0001:0001d772       ?getAllEntries@?$IdRegistry@VDomainFactory@Workflow@U2@@@U2@@UBE?AV?$QList@PAVDomainFactory@Workflow@U2@@@@XZ 1001e772 f   U2Lang:U2Lang.dll
 0001:0001d778       ?getAllIds@?$IdRegistry@VDomainFactory@Workflow@U2@@@U2@@UBE?AV?$QList@VQString@@@@XZ 1001e778 f   U2Lang:U2Lang.dll
 0001:0001d77e       ?getById@?$IdRegistry@VDomainFactory@Workflow@U2@@@U2@@UAEPAVDomainFactory@Workflow@2@ABVQString@@@Z 1001e77e f   U2Lang:U2Lang.dll
 0001:0001d784       ?getCommunication@BaseWorker@LocalWorkflow@U2@@UAEPAVCommunicationChannel@Workflow@3@ABVQString@@@Z 1001e784 f   U2Lang:U2Lang.dll
 0001:0001d78a       ?getDatatypeByDescriptor@MapDataType@U2@@UBE?AV?$QExplicitlySharedDataPointer@VDataType@U2@@@@ABVDescriptor@2@@Z 1001e78a f   U2Lang:U2Lang.dll
 0001:0001d790       ?getDatatypesMap@MapDataType@U2@@UBE?AV?$QMap@VDescriptor@U2@@V?$QExplicitlySharedDataPointer@VDataType@U2@@@@@@XZ 1001e790 f   U2Lang:U2Lang.dll
 0001:0001d796       ?getMessageAndSetupScriptValues@BaseWorker@LocalWorkflow@U2@@UAE?AVMessage@Workflow@3@PAVCommunicationChannel@53@@Z 1001e796 f   U2Lang:U2Lang.dll
 0001:0001d79c       ?getOutputFiles@BaseWorker@LocalWorkflow@U2@@UAE?AVQStringList@@XZ 1001e79c f   U2Lang:U2Lang.dll
 0001:0001d7a2       ?getType@PortDescriptor@Workflow@U2@@UBE?AV?$QExplicitlySharedDataPointer@VDataType@U2@@@@XZ 1001e7a2 f   U2Lang:U2Lang.dll
 0001:0001d7a8       ?isAcceptableDrop@ActorPrototype@Workflow@U2@@UBE_NPBVQMimeData@@PAV?$QMap@VQString@@VQVariant@@@@@Z 1001e7a8 f   U2Lang:U2Lang.dll
 0001:0001d7ae       ?isDone@BaseWorker@LocalWorkflow@U2@@UBE_NXZ 1001e7ae f   U2Lang:U2Lang.dll
 0001:0001d7b4       ?isReady@BaseWorker@LocalWorkflow@U2@@UBE_NXZ 1001e7b4 f   U2Lang:U2Lang.dll
 0001:0001d7ba       ?kind@MapDataType@U2@@UBE?AW4Kind@DataType@2@XZ 1001e7ba f   U2Lang:U2Lang.dll
 0001:0001d7c0       ?metaObject@PrompterBaseImpl@U2@@UBEPBUQMetaObject@@XZ 1001e7c0 f   U2Lang:U2Lang.dll
 0001:0001d7c6       ?qt_metacall@PrompterBaseImpl@U2@@UAEHW4Call@QMetaObject@@HPAPAX@Z 1001e7c6 f   U2Lang:U2Lang.dll
 0001:0001d7cc       ?qt_metacast@PrompterBaseImpl@U2@@UAEPAXPBD@Z 1001e7cc f   U2Lang:U2Lang.dll
 0001:0001d7d2       ?registerEntry@?$IdRegistry@VDomainFactory@Workflow@U2@@@U2@@UAE_NPAVDomainFactory@Workflow@2@@Z 1001e7d2 f   U2Lang:U2Lang.dll
 0001:0001d7d8       ?setDone@BaseWorker@LocalWorkflow@U2@@UAEXXZ 1001e7d8 f   U2Lang:U2Lang.dll
 0001:0001d7de       ?setVisibleSlot@PortDescriptor@Workflow@U2@@UAEXABVQString@@_N@Z 1001e7de f   U2Lang:U2Lang.dll
 0001:0001d7e4       ?sl_actorModified@PrompterBaseImpl@U2@@MAEXXZ 1001e7e4 f   U2Lang:U2Lang.dll
 0001:0001d7ea       ?unregisterEntry@?$IdRegistry@VDomainFactory@Workflow@U2@@@U2@@UAEPAVDomainFactory@Workflow@2@ABVQString@@@Z 1001e7ea f   U2Lang:U2Lang.dll
 0001:0001d7f0       ?update@PrompterBaseImpl@U2@@UAEXABV?$QMap@VQString@@VQVariant@@@@@Z 1001e7f0 f   U2Lang:U2Lang.dll
 0001:0001d7f6       ?qt_metacast@QDActor@U2@@UAEPAXPBD@Z 1001e7f6 f   U2Lang:U2Lang.dll
 0001:0001d7fc       ?qt_metacall@QDActor@U2@@UAEHW4Call@QMetaObject@@HPAPAX@Z 1001e7fc f   U2Lang:U2Lang.dll
 0001:0001d802       ?qt_metacast@BaseWorker@LocalWorkflow@U2@@UAEPAXPBD@Z 1001e802 f   U2Lang:U2Lang.dll
 0001:0001d808       ?qt_metacall@BaseWorker@LocalWorkflow@U2@@UAEHW4Call@QMetaObject@@HPAPAX@Z 1001e808 f   U2Lang:U2Lang.dll
 0001:0001d80e       ??0DelegateEditor@U2@@QAE@ABV?$QMap@VQString@@PAVPropertyDelegate@U2@@@@@Z 1001e80e f   U2Designer:U2Designer.dll
 0001:0001d814       ??1DelegateEditor@U2@@UAE@XZ 1001e814 f   U2Designer:U2Designer.dll
 0001:0001d81a       ??0SpinBoxDelegate@U2@@QAE@ABV?$QMap@VQString@@VQVariant@@@@PAVQObject@@@Z 1001e81a f   U2Designer:U2Designer.dll
 0001:0001d820       ??1SpinBoxDelegate@U2@@UAE@XZ 1001e820 f   U2Designer:U2Designer.dll
 0001:0001d826       ??0ComboBoxDelegate@U2@@QAE@ABV?$QMap@VQString@@VQVariant@@@@PAVQObject@@@Z 1001e826 f   U2Designer:U2Designer.dll
 0001:0001d82c       ??1ComboBoxDelegate@U2@@UAE@XZ 1001e82c f   U2Designer:U2Designer.dll
 0001:0001d832       ?addDelegate@DelegateEditor@U2@@UAEXPAVPropertyDelegate@2@ABVQString@@@Z 1001e832 f   U2Designer:U2Designer.dll
 0001:0001d838       ?clone@ComboBoxDelegate@U2@@UAEPAVPropertyDelegate@2@XZ 1001e838 f   U2Designer:U2Designer.dll
 0001:0001d83e       ?clone@DelegateEditor@U2@@UAEPAVConfigurationEditor@2@XZ 1001e83e f   U2Designer:U2Designer.dll
 0001:0001d844       ?clone@SpinBoxDelegate@U2@@UAEPAVPropertyDelegate@2@XZ 1001e844 f   U2Designer:U2Designer.dll
 0001:0001d84a       ?commit@DelegateEditor@U2@@UAEXXZ 1001e84a f   U2Designer:U2Designer.dll
 0001:0001d850       ?createEditor@ComboBoxDelegate@U2@@UBEPAVQWidget@@PAV3@ABVQStyleOptionViewItem@@ABVQModelIndex@@@Z 1001e850 f   U2Designer:U2Designer.dll
 0001:0001d856       ?createEditor@SpinBoxDelegate@U2@@UBEPAVQWidget@@PAV3@ABVQStyleOptionViewItem@@ABVQModelIndex@@@Z 1001e856 f   U2Designer:U2Designer.dll
 0001:0001d85c       ?createWizardWidget@ComboBoxDelegate@U2@@UBEPAVPropertyWidget@2@AAVU2OpStatus@2@PAVQWidget@@@Z 1001e85c f   U2Designer:U2Designer.dll
 0001:0001d862       ?createWizardWidget@SpinBoxDelegate@U2@@UBEPAVPropertyWidget@2@AAVU2OpStatus@2@PAVQWidget@@@Z 1001e862 f   U2Designer:U2Designer.dll
 0001:0001d868       ?getDelegate@DelegateEditor@U2@@UAEPAVPropertyDelegate@2@ABVQString@@@Z 1001e868 f   U2Designer:U2Designer.dll
 0001:0001d86e       ?getDisplayValue@ComboBoxDelegate@U2@@UBE?AVQVariant@@ABV3@@Z 1001e86e f   U2Designer:U2Designer.dll
 0001:0001d874       ?getDisplayValue@SpinBoxDelegate@U2@@UBE?AVQVariant@@ABV3@@Z 1001e874 f   U2Designer:U2Designer.dll
 0001:0001d87a       ?getItems@ComboBoxDelegate@U2@@UBEXAAV?$QMap@VQString@@VQVariant@@@@@Z 1001e87a f   U2Designer:U2Designer.dll
 0001:0001d880       ?getItems@SpinBoxDelegate@U2@@UBEXAAV?$QMap@VQString@@VQVariant@@@@@Z 1001e880 f   U2Designer:U2Designer.dll
 0001:0001d886       ?metaObject@ComboBoxDelegate@U2@@UBEPBUQMetaObject@@XZ 1001e886 f   U2Designer:U2Designer.dll
 0001:0001d88c       ?metaObject@DelegateEditor@U2@@UBEPBUQMetaObject@@XZ 1001e88c f   U2Designer:U2Designer.dll
 0001:0001d892       ?metaObject@SpinBoxDelegate@U2@@UBEPBUQMetaObject@@XZ 1001e892 f   U2Designer:U2Designer.dll
 0001:0001d898       ?qt_metacall@ComboBoxDelegate@U2@@UAEHW4Call@QMetaObject@@HPAPAX@Z 1001e898 f   U2Designer:U2Designer.dll
 0001:0001d89e       ?qt_metacall@DelegateEditor@U2@@UAEHW4Call@QMetaObject@@HPAPAX@Z 1001e89e f   U2Designer:U2Designer.dll
 0001:0001d8a4       ?qt_metacall@SpinBoxDelegate@U2@@UAEHW4Call@QMetaObject@@HPAPAX@Z 1001e8a4 f   U2Designer:U2Designer.dll
 0001:0001d8aa       ?qt_metacast@ComboBoxDelegate@U2@@UAEPAXPBD@Z 1001e8aa f   U2Designer:U2Designer.dll
 0001:0001d8b0       ?qt_metacast@DelegateEditor@U2@@UAEPAXPBD@Z 1001e8b0 f   U2Designer:U2Designer.dll
 0001:0001d8b6       ?qt_metacast@SpinBoxDelegate@U2@@UAEPAXPBD@Z 1001e8b6 f   U2Designer:U2Designer.dll
 0001:0001d8bc       ?removeDelegate@DelegateEditor@U2@@UAEPAVPropertyDelegate@2@ABVQString@@@Z 1001e8bc f   U2Designer:U2Designer.dll
 0001:0001d8c2       ?setEditorData@ComboBoxDelegate@U2@@UBEXPAVQWidget@@ABVQModelIndex@@@Z 1001e8c2 f   U2Designer:U2Designer.dll
 0001:0001d8c8       ?setEditorData@SpinBoxDelegate@U2@@UBEXPAVQWidget@@ABVQModelIndex@@@Z 1001e8c8 f   U2Designer:U2Designer.dll
 0001:0001d8ce       ?setModelData@ComboBoxDelegate@U2@@UBEXPAVQWidget@@PAVQAbstractItemModel@@ABVQModelIndex@@@Z 1001e8ce f   U2Designer:U2Designer.dll
 0001:0001d8d4       ?setModelData@SpinBoxDelegate@U2@@UBEXPAVQWidget@@PAVQAbstractItemModel@@ABVQModelIndex@@@Z 1001e8d4 f   U2Designer:U2Designer.dll
 0001:0001d8da       ?updateDelegate@DelegateEditor@U2@@UAEXABVQString@@@Z 1001e8da f   U2Designer:U2Designer.dll
 0001:0001d8e0       ?updateDelegates@DelegateEditor@U2@@UAEXXZ 1001e8e0 f   U2Designer:U2Designer.dll
 0001:0001d8e6       ??0ComboBoxDelegate@U2@@QAE@ABV?$QList@U?$QPair@VQString@@VQVariant@@@@@@PAVQObject@@@Z 1001e8e6 f   U2Designer:U2Designer.dll
 0001:0001d8ec       ??0QSizePolicy@@QAE@W4Policy@0@0W4ControlType@0@@Z 1001e8ec f   Qt5Widgets:Qt5Widgets.dll
 0001:0001d8f2       ?setHorizontalStretch@QSizePolicy@@QAEXH@Z 1001e8f2 f   Qt5Widgets:Qt5Widgets.dll
 0001:0001d8f8       ?setVerticalStretch@QSizePolicy@@QAEXH@Z 1001e8f8 f   Qt5Widgets:Qt5Widgets.dll
 0001:0001d8fe       ??0QWidget@@QAE@PAV0@V?$QFlags@W4WindowType@Qt@@@@@Z 1001e8fe f   Qt5Widgets:Qt5Widgets.dll
 0001:0001d904       ??1QWidget@@UAE@XZ         1001e904 f   Qt5Widgets:Qt5Widgets.dll
 0001:0001d90a       ?setEnabled@QWidget@@QAEX_N@Z 1001e90a f   Qt5Widgets:Qt5Widgets.dll
 0001:0001d910       ?setDisabled@QWidget@@QAEX_N@Z 1001e910 f   Qt5Widgets:Qt5Widgets.dll
 0001:0001d916       ?setMinimumSize@QWidget@@QAEXHH@Z 1001e916 f   Qt5Widgets:Qt5Widgets.dll
 0001:0001d91c       ?setMaximumSize@QWidget@@QAEXHH@Z 1001e91c f   Qt5Widgets:Qt5Widgets.dll
 0001:0001d922       ?setWindowTitle@QWidget@@QAEXABVQString@@@Z 1001e922 f   Qt5Widgets:Qt5Widgets.dll
 0001:0001d928       ?setToolTip@QWidget@@QAEXABVQString@@@Z 1001e928 f   Qt5Widgets:Qt5Widgets.dll
 0001:0001d92e       ?setWhatsThis@QWidget@@QAEXABVQString@@@Z 1001e92e f   Qt5Widgets:Qt5Widgets.dll
 0001:0001d934       ?setFocus@QWidget@@QAEXW4FocusReason@Qt@@@Z 1001e934 f   Qt5Widgets:Qt5Widgets.dll
 0001:0001d93a       ?resize@QWidget@@QAEXABVQSize@@@Z 1001e93a f   Qt5Widgets:Qt5Widgets.dll
 0001:0001d940       ?sizePolicy@QWidget@@QBE?AVQSizePolicy@@XZ 1001e940 f   Qt5Widgets:Qt5Widgets.dll
 0001:0001d946       ?setSizePolicy@QWidget@@QAEXVQSizePolicy@@@Z 1001e946 f   Qt5Widgets:Qt5Widgets.dll
 0001:0001d94c       ?setLayout@QWidget@@QAEXPAVQLayout@@@Z 1001e94c f   Qt5Widgets:Qt5Widgets.dll
 0001:0001d952       ?actions@QWidget@@QBE?AV?$QList@PAVQAction@@@@XZ 1001e952 f   Qt5Widgets:Qt5Widgets.dll
 0001:0001d958       ?setAttribute@QWidget@@QAEXW4WidgetAttribute@Qt@@_N@Z 1001e958 f   Qt5Widgets:Qt5Widgets.dll
 0001:0001d95e       ?text@QAction@@QBE?AVQString@@XZ 1001e95e f   Qt5Widgets:Qt5Widgets.dll
 0001:0001d964       ?isChecked@QAction@@QBE_NXZ 1001e964 f   Qt5Widgets:Qt5Widgets.dll
 0001:0001d96a       ?activate@QAction@@QAEXW4ActionEvent@1@@Z 1001e96a f   Qt5Widgets:Qt5Widgets.dll
 0001:0001d970       ?setText@QAbstractButton@@QAEXABVQString@@@Z 1001e970 f   Qt5Widgets:Qt5Widgets.dll
 0001:0001d976       ?setShortcut@QAbstractButton@@QAEXABVQKeySequence@@@Z 1001e976 f   Qt5Widgets:Qt5Widgets.dll
 0001:0001d97c       ?isChecked@QAbstractButton@@QBE_NXZ 1001e97c f   Qt5Widgets:Qt5Widgets.dll
 0001:0001d982       ?setChecked@QAbstractButton@@QAEX_N@Z 1001e982 f   Qt5Widgets:Qt5Widgets.dll
 0001:0001d988       ??0QCheckBox@@QAE@PAVQWidget@@@Z 1001e988 f   Qt5Widgets:Qt5Widgets.dll
 0001:0001d98e       ??1QCheckBox@@UAE@XZ       1001e98e f   Qt5Widgets:Qt5Widgets.dll
 0001:0001d994       ??0QTabWidget@@QAE@PAVQWidget@@@Z 1001e994 f   Qt5Widgets:Qt5Widgets.dll
 0001:0001d99a       ??1QTabWidget@@UAE@XZ      1001e99a f   Qt5Widgets:Qt5Widgets.dll
 0001:0001d9a0       ?addTab@QTabWidget@@QAEHPAVQWidget@@ABVQString@@@Z 1001e9a0 f   Qt5Widgets:Qt5Widgets.dll
 0001:0001d9a6       ?setTabText@QTabWidget@@QAEXHABVQString@@@Z 1001e9a6 f   Qt5Widgets:Qt5Widgets.dll
 0001:0001d9ac       ?indexOf@QTabWidget@@QBEHPAVQWidget@@@Z 1001e9ac f   Qt5Widgets:Qt5Widgets.dll
 0001:0001d9b2       ?setCurrentIndex@QTabWidget@@QAEXH@Z 1001e9b2 f   Qt5Widgets:Qt5Widgets.dll
 0001:0001d9b8       ??0QComboBox@@QAE@PAVQWidget@@@Z 1001e9b8 f   Qt5Widgets:Qt5Widgets.dll
 0001:0001d9be       ??1QComboBox@@UAE@XZ       1001e9be f   Qt5Widgets:Qt5Widgets.dll
 0001:0001d9c4       ?count@QComboBox@@QBEHXZ   1001e9c4 f   Qt5Widgets:Qt5Widgets.dll
 0001:0001d9ca       ?currentIndex@QComboBox@@QBEHXZ 1001e9ca f   Qt5Widgets:Qt5Widgets.dll
 0001:0001d9d0       ?itemData@QComboBox@@QBE?AVQVariant@@HH@Z 1001e9d0 f   Qt5Widgets:Qt5Widgets.dll
 0001:0001d9d6       ?insertItem@QComboBox@@QAEXHABVQIcon@@ABVQString@@ABVQVariant@@@Z 1001e9d6 f   Qt5Widgets:Qt5Widgets.dll
 0001:0001d9dc       ?setCurrentIndex@QComboBox@@QAEXH@Z 1001e9dc f   Qt5Widgets:Qt5Widgets.dll
 0001:0001d9e2       ??0QDialog@@QAE@PAVQWidget@@V?$QFlags@W4WindowType@Qt@@@@@Z 1001e9e2 f   Qt5Widgets:Qt5Widgets.dll
 0001:0001d9e8       ??1QDialog@@UAE@XZ         1001e9e8 f   Qt5Widgets:Qt5Widgets.dll
 0001:0001d9ee       ?setSizeGripEnabled@QDialog@@QAEX_N@Z 1001e9ee f   Qt5Widgets:Qt5Widgets.dll
 0001:0001d9f4       ?accept@QDialog@@UAEXXZ    1001e9f4 f   Qt5Widgets:Qt5Widgets.dll
 0001:0001d9fa       ?reject@QDialog@@UAEXXZ    1001e9fa f   Qt5Widgets:Qt5Widgets.dll
 0001:0001da00       ??0QDialogButtonBox@@QAE@PAVQWidget@@@Z 1001ea00 f   Qt5Widgets:Qt5Widgets.dll
 0001:0001da06       ??1QDialogButtonBox@@UAE@XZ 1001ea06 f   Qt5Widgets:Qt5Widgets.dll
 0001:0001da0c       ?setStandardButtons@QDialogButtonBox@@QAEXV?$QFlags@W4StandardButton@QDialogButtonBox@@@@@Z 1001ea0c f   Qt5Widgets:Qt5Widgets.dll
 0001:0001da12       ?button@QDialogButtonBox@@QBEPAVQPushButton@@W4StandardButton@1@@Z 1001ea12 f   Qt5Widgets:Qt5Widgets.dll
 0001:0001da18       ??0QSpacerItem@@QAE@HHW4Policy@QSizePolicy@@0@Z 1001ea18 f   Qt5Widgets:Qt5Widgets.dll
 0001:0001da1e       ??1QSpacerItem@@UAE@XZ     1001ea1e f   Qt5Widgets:Qt5Widgets.dll
 0001:0001da24       ?setMargin@QLayout@@QAEXH@Z 1001ea24 f   Qt5Widgets:Qt5Widgets.dll
 0001:0001da2a       ?setContentsMargins@QLayout@@QAEXHHHH@Z 1001ea2a f   Qt5Widgets:Qt5Widgets.dll
 0001:0001da30       ?setSizeConstraint@QLayout@@QAEXW4SizeConstraint@1@@Z 1001ea30 f   Qt5Widgets:Qt5Widgets.dll
 0001:0001da36       ?addWidget@QBoxLayout@@QAEXPAVQWidget@@HV?$QFlags@W4AlignmentFlag@Qt@@@@@Z 1001ea36 f   Qt5Widgets:Qt5Widgets.dll
 0001:0001da3c       ?addLayout@QBoxLayout@@QAEXPAVQLayout@@H@Z 1001ea3c f   Qt5Widgets:Qt5Widgets.dll
 0001:0001da42       ?setSpacing@QBoxLayout@@QAEXH@Z 1001ea42 f   Qt5Widgets:Qt5Widgets.dll
 0001:0001da48       ??0QHBoxLayout@@QAE@XZ     1001ea48 f   Qt5Widgets:Qt5Widgets.dll
 0001:0001da4e       ??1QHBoxLayout@@UAE@XZ     1001ea4e f   Qt5Widgets:Qt5Widgets.dll
 0001:0001da54       ??0QVBoxLayout@@QAE@XZ     1001ea54 f   Qt5Widgets:Qt5Widgets.dll
 0001:0001da5a       ??0QVBoxLayout@@QAE@PAVQWidget@@@Z 1001ea5a f   Qt5Widgets:Qt5Widgets.dll
 0001:0001da60       ??1QVBoxLayout@@UAE@XZ     1001ea60 f   Qt5Widgets:Qt5Widgets.dll
 0001:0001da66       ??0QGridLayout@@QAE@XZ     1001ea66 f   Qt5Widgets:Qt5Widgets.dll
 0001:0001da6c       ??1QGridLayout@@UAE@XZ     1001ea6c f   Qt5Widgets:Qt5Widgets.dll
 0001:0001da72       ?setSpacing@QGridLayout@@QAEXH@Z 1001ea72 f   Qt5Widgets:Qt5Widgets.dll
 0001:0001da78       ?addWidget@QGridLayout@@QAEXPAVQWidget@@HHHHV?$QFlags@W4AlignmentFlag@Qt@@@@@Z 1001ea78 f   Qt5Widgets:Qt5Widgets.dll
 0001:0001da7e       ?addLayout@QGridLayout@@QAEXPAVQLayout@@HHHHV?$QFlags@W4AlignmentFlag@Qt@@@@@Z 1001ea7e f   Qt5Widgets:Qt5Widgets.dll
 0001:0001da84       ??0QGroupBox@@QAE@PAVQWidget@@@Z 1001ea84 f   Qt5Widgets:Qt5Widgets.dll
 0001:0001da8a       ??1QGroupBox@@UAE@XZ       1001ea8a f   Qt5Widgets:Qt5Widgets.dll
 0001:0001da90       ?setTitle@QGroupBox@@QAEXABVQString@@@Z 1001ea90 f   Qt5Widgets:Qt5Widgets.dll
 0001:0001da96       ?setDefaultSectionSize@QHeaderView@@QAEXH@Z 1001ea96 f   Qt5Widgets:Qt5Widgets.dll
 0001:0001da9c       ?setMinimumSectionSize@QHeaderView@@QAEXH@Z 1001ea9c f   Qt5Widgets:Qt5Widgets.dll
 0001:0001daa2       ??0QLabel@@QAE@PAVQWidget@@V?$QFlags@W4WindowType@Qt@@@@@Z 1001eaa2 f   Qt5Widgets:Qt5Widgets.dll
 0001:0001daa8       ??1QLabel@@UAE@XZ          1001eaa8 f   Qt5Widgets:Qt5Widgets.dll
 0001:0001daae       ?setText@QLabel@@QAEXABVQString@@@Z 1001eaae f   Qt5Widgets:Qt5Widgets.dll
 0001:0001dab4       ??0QPushButton@@QAE@PAVQWidget@@@Z 1001eab4 f   Qt5Widgets:Qt5Widgets.dll
 0001:0001daba       ??1QPushButton@@UAE@XZ     1001eaba f   Qt5Widgets:Qt5Widgets.dll
 0001:0001dac0       ?setDefault@QPushButton@@QAEX_N@Z 1001eac0 f   Qt5Widgets:Qt5Widgets.dll
 0001:0001dac6       ?setFlat@QPushButton@@QAEX_N@Z 1001eac6 f   Qt5Widgets:Qt5Widgets.dll
 0001:0001dacc       ??0QRadioButton@@QAE@PAVQWidget@@@Z 1001eacc f   Qt5Widgets:Qt5Widgets.dll
 0001:0001dad2       ??1QRadioButton@@UAE@XZ    1001ead2 f   Qt5Widgets:Qt5Widgets.dll
 0001:0001dad8       ??0QSpinBox@@QAE@PAVQWidget@@@Z 1001ead8 f   Qt5Widgets:Qt5Widgets.dll
 0001:0001dade       ??1QSpinBox@@UAE@XZ        1001eade f   Qt5Widgets:Qt5Widgets.dll
 0001:0001dae4       ?value@QSpinBox@@QBEHXZ    1001eae4 f   Qt5Widgets:Qt5Widgets.dll
 0001:0001daea       ?setSuffix@QSpinBox@@QAEXABVQString@@@Z 1001eaea f   Qt5Widgets:Qt5Widgets.dll
 0001:0001daf0       ?setSingleStep@QSpinBox@@QAEXH@Z 1001eaf0 f   Qt5Widgets:Qt5Widgets.dll
 0001:0001daf6       ?setMinimum@QSpinBox@@QAEXH@Z 1001eaf6 f   Qt5Widgets:Qt5Widgets.dll
 0001:0001dafc       ?setMaximum@QSpinBox@@QAEXH@Z 1001eafc f   Qt5Widgets:Qt5Widgets.dll
 0001:0001db02       ?setValue@QSpinBox@@QAEXH@Z 1001eb02 f   Qt5Widgets:Qt5Widgets.dll
 0001:0001db08       ??0QTextEdit@@QAE@PAVQWidget@@@Z 1001eb08 f   Qt5Widgets:Qt5Widgets.dll
 0001:0001db0e       ??1QTextEdit@@UAE@XZ       1001eb0e f   Qt5Widgets:Qt5Widgets.dll
 0001:0001db14       ?setReadOnly@QTextEdit@@QAEX_N@Z 1001eb14 f   Qt5Widgets:Qt5Widgets.dll
 0001:0001db1a       ?setText@QTextEdit@@QAEXABVQString@@@Z 1001eb1a f   Qt5Widgets:Qt5Widgets.dll
 0001:0001db20       ?clear@QTextEdit@@QAEXXZ   1001eb20 f   Qt5Widgets:Qt5Widgets.dll
 0001:0001db26       ?header@QTreeView@@QBEPAVQHeaderView@@XZ 1001eb26 f   Qt5Widgets:Qt5Widgets.dll
 0001:0001db2c       ?setRootIsDecorated@QTreeView@@QAEX_N@Z 1001eb2c f   Qt5Widgets:Qt5Widgets.dll
 0001:0001db32       ?setSortingEnabled@QTreeView@@QAEX_N@Z 1001eb32 f   Qt5Widgets:Qt5Widgets.dll
 0001:0001db38       ?sortByColumn@QTreeView@@QAEXH@Z 1001eb38 f   Qt5Widgets:Qt5Widgets.dll
 0001:0001db3e       ??0QTreeWidgetItem@@QAE@H@Z 1001eb3e f   Qt5Widgets:Qt5Widgets.dll
 0001:0001db44       ??1QTreeWidgetItem@@UAE@XZ 1001eb44 f   Qt5Widgets:Qt5Widgets.dll
 0001:0001db4a       ?text@QTreeWidgetItem@@QBE?AVQString@@H@Z 1001eb4a f   Qt5Widgets:Qt5Widgets.dll
 0001:0001db50       ?setText@QTreeWidgetItem@@QAEXHABVQString@@@Z 1001eb50 f   Qt5Widgets:Qt5Widgets.dll
 0001:0001db56       ??0QTreeWidget@@QAE@PAVQWidget@@@Z 1001eb56 f   Qt5Widgets:Qt5Widgets.dll
 0001:0001db5c       ??1QTreeWidget@@UAE@XZ     1001eb5c f   Qt5Widgets:Qt5Widgets.dll
 0001:0001db62       ?topLevelItemCount@QTreeWidget@@QBEHXZ 1001eb62 f   Qt5Widgets:Qt5Widgets.dll
 0001:0001db68       ?addTopLevelItem@QTreeWidget@@QAEXPAVQTreeWidgetItem@@@Z 1001eb68 f   Qt5Widgets:Qt5Widgets.dll
 0001:0001db6e       ?headerItem@QTreeWidget@@QBEPAVQTreeWidgetItem@@XZ 1001eb6e f   Qt5Widgets:Qt5Widgets.dll
 0001:0001db74       ?currentItem@QTreeWidget@@QBEPAVQTreeWidgetItem@@XZ 1001eb74 f   Qt5Widgets:Qt5Widgets.dll
 0001:0001db7a       ?sortColumn@QTreeWidget@@QBEHXZ 1001eb7a f   Qt5Widgets:Qt5Widgets.dll
 0001:0001db80       ?clear@QTreeWidget@@QAEXXZ 1001eb80 f   Qt5Widgets:Qt5Widgets.dll
 0001:0001db86       ?warning@QMessageBox@@SA?AW4StandardButton@1@PAVQWidget@@ABVQString@@1V?$QFlags@W4StandardButton@QMessageBox@@@@W421@@Z 1001eb86 f   Qt5Widgets:Qt5Widgets.dll
 0001:0001db8c       ?warning@QMessageBox@@SAHPAVQWidget@@ABVQString@@1HHH@Z 1001eb8c f   Qt5Widgets:Qt5Widgets.dll
 0001:0001db92       ?actionEvent@QWidget@@MAEXPAVQActionEvent@@@Z 1001eb92 f   Qt5Widgets:Qt5Widgets.dll
 0001:0001db98       ?addItem@QBoxLayout@@UAEXPAVQLayoutItem@@@Z 1001eb98 f   Qt5Widgets:Qt5Widgets.dll
 0001:0001db9e       ?addItem@QGridLayout@@MAEXPAVQLayoutItem@@@Z 1001eb9e f   Qt5Widgets:Qt5Widgets.dll
 0001:0001dba4       ?canInsertFromMimeData@QTextEdit@@MBE_NPBVQMimeData@@@Z 1001eba4 f   Qt5Widgets:Qt5Widgets.dll
 0001:0001dbaa       ?changeEvent@QAbstractButton@@MAEXPAVQEvent@@@Z 1001ebaa f   Qt5Widgets:Qt5Widgets.dll
 0001:0001dbb0       ?changeEvent@QAbstractSpinBox@@MAEXPAVQEvent@@@Z 1001ebb0 f   Qt5Widgets:Qt5Widgets.dll
 0001:0001dbb6       ?changeEvent@QComboBox@@MAEXPAVQEvent@@@Z 1001ebb6 f   Qt5Widgets:Qt5Widgets.dll
 0001:0001dbbc       ?changeEvent@QDialogButtonBox@@MAEXPAVQEvent@@@Z 1001ebbc f   Qt5Widgets:Qt5Widgets.dll
 0001:0001dbc2       ?changeEvent@QFrame@@MAEXPAVQEvent@@@Z 1001ebc2 f   Qt5Widgets:Qt5Widgets.dll
 0001:0001dbc8       ?changeEvent@QGroupBox@@MAEXPAVQEvent@@@Z 1001ebc8 f   Qt5Widgets:Qt5Widgets.dll
 0001:0001dbce       ?changeEvent@QLabel@@MAEXPAVQEvent@@@Z 1001ebce f   Qt5Widgets:Qt5Widgets.dll
 0001:0001dbd4       ?changeEvent@QTabWidget@@MAEXPAVQEvent@@@Z 1001ebd4 f   Qt5Widgets:Qt5Widgets.dll
 0001:0001dbda       ?changeEvent@QTextEdit@@MAEXPAVQEvent@@@Z 1001ebda f   Qt5Widgets:Qt5Widgets.dll
 0001:0001dbe0       ?changeEvent@QWidget@@MAEXPAVQEvent@@@Z 1001ebe0 f   Qt5Widgets:Qt5Widgets.dll
 0001:0001dbe6       ?checkStateSet@QAbstractButton@@MAEXXZ 1001ebe6 f   Qt5Widgets:Qt5Widgets.dll
 0001:0001dbec       ?checkStateSet@QCheckBox@@MAEXXZ 1001ebec f   Qt5Widgets:Qt5Widgets.dll
 0001:0001dbf2       ?childEvent@QGroupBox@@MAEXPAVQChildEvent@@@Z 1001ebf2 f   Qt5Widgets:Qt5Widgets.dll
 0001:0001dbf8       ?childEvent@QLayout@@MAEXPAVQChildEvent@@@Z 1001ebf8 f   Qt5Widgets:Qt5Widgets.dll
 0001:0001dbfe       ?clear@QAbstractSpinBox@@UAEXXZ 1001ebfe f   Qt5Widgets:Qt5Widgets.dll
 0001:0001dc04       ?clone@QTreeWidgetItem@@UBEPAV1@XZ 1001ec04 f   Qt5Widgets:Qt5Widgets.dll
 0001:0001dc0a       ?closeEditor@QAbstractItemView@@MAEXPAVQWidget@@W4EndEditHint@QAbstractItemDelegate@@@Z 1001ec0a f   Qt5Widgets:Qt5Widgets.dll
 0001:0001dc10       ?closeEvent@QAbstractSpinBox@@MAEXPAVQCloseEvent@@@Z 1001ec10 f   Qt5Widgets:Qt5Widgets.dll
 0001:0001dc16       ?closeEvent@QDialog@@MAEXPAVQCloseEvent@@@Z 1001ec16 f   Qt5Widgets:Qt5Widgets.dll
 0001:0001dc1c       ?closeEvent@QWidget@@MAEXPAVQCloseEvent@@@Z 1001ec1c f   Qt5Widgets:Qt5Widgets.dll
 0001:0001dc22       ?commitData@QAbstractItemView@@MAEXPAVQWidget@@@Z 1001ec22 f   Qt5Widgets:Qt5Widgets.dll
 0001:0001dc28       ?contextMenuEvent@QAbstractScrollArea@@MAEXPAVQContextMenuEvent@@@Z 1001ec28 f   Qt5Widgets:Qt5Widgets.dll
 0001:0001dc2e       ?contextMenuEvent@QAbstractSpinBox@@MAEXPAVQContextMenuEvent@@@Z 1001ec2e f   Qt5Widgets:Qt5Widgets.dll
 0001:0001dc34       ?contextMenuEvent@QComboBox@@MAEXPAVQContextMenuEvent@@@Z 1001ec34 f   Qt5Widgets:Qt5Widgets.dll
 0001:0001dc3a       ?contextMenuEvent@QDialog@@MAEXPAVQContextMenuEvent@@@Z 1001ec3a f   Qt5Widgets:Qt5Widgets.dll
 0001:0001dc40       ?contextMenuEvent@QLabel@@MAEXPAVQContextMenuEvent@@@Z 1001ec40 f   Qt5Widgets:Qt5Widgets.dll
 0001:0001dc46       ?contextMenuEvent@QTextEdit@@MAEXPAVQContextMenuEvent@@@Z 1001ec46 f   Qt5Widgets:Qt5Widgets.dll
 0001:0001dc4c       ?contextMenuEvent@QWidget@@MAEXPAVQContextMenuEvent@@@Z 1001ec4c f   Qt5Widgets:Qt5Widgets.dll
 0001:0001dc52       ?controlTypes@QLayout@@UBE?AV?$QFlags@W4ControlType@QSizePolicy@@@@XZ 1001ec52 f   Qt5Widgets:Qt5Widgets.dll
 0001:0001dc58       ?controlTypes@QLayoutItem@@UBE?AV?$QFlags@W4ControlType@QSizePolicy@@@@XZ 1001ec58 f   Qt5Widgets:Qt5Widgets.dll
 0001:0001dc5e       ?count@QBoxLayout@@UBEHXZ  1001ec5e f   Qt5Widgets:Qt5Widgets.dll
 0001:0001dc64       ?count@QGridLayout@@UBEHXZ 1001ec64 f   Qt5Widgets:Qt5Widgets.dll
 0001:0001dc6a       ?createMimeDataFromSelection@QTextEdit@@MBEPAVQMimeData@@XZ 1001ec6a f   Qt5Widgets:Qt5Widgets.dll
 0001:0001dc70       ?currentChanged@QTreeView@@MAEXABVQModelIndex@@0@Z 1001ec70 f   Qt5Widgets:Qt5Widgets.dll
 0001:0001dc76       ?data@QTreeWidgetItem@@UBE?AVQVariant@@HH@Z 1001ec76 f   Qt5Widgets:Qt5Widgets.dll
 0001:0001dc7c       ?dataChanged@QTreeView@@UAEXABVQModelIndex@@0ABV?$QVector@H@@@Z 1001ec7c f   Qt5Widgets:Qt5Widgets.dll
 0001:0001dc82       ?devType@QWidget@@UBEHXZ   1001ec82 f   Qt5Widgets:Qt5Widgets.dll
 0001:0001dc88       ?doItemsLayout@QTreeView@@UAEXXZ 1001ec88 f   Qt5Widgets:Qt5Widgets.dll
 0001:0001dc8e       ?doSetTextCursor@QTextEdit@@MAEXABVQTextCursor@@@Z 1001ec8e f   Qt5Widgets:Qt5Widgets.dll
 0001:0001dc94       ?done@QDialog@@UAEXH@Z     1001ec94 f   Qt5Widgets:Qt5Widgets.dll
 0001:0001dc9a       ?dragEnterEvent@QAbstractItemView@@MAEXPAVQDragEnterEvent@@@Z 1001ec9a f   Qt5Widgets:Qt5Widgets.dll
 0001:0001dca0       ?dragEnterEvent@QTextEdit@@MAEXPAVQDragEnterEvent@@@Z 1001eca0 f   Qt5Widgets:Qt5Widgets.dll
 0001:0001dca6       ?dragEnterEvent@QWidget@@MAEXPAVQDragEnterEvent@@@Z 1001eca6 f   Qt5Widgets:Qt5Widgets.dll
 0001:0001dcac       ?dragLeaveEvent@QAbstractItemView@@MAEXPAVQDragLeaveEvent@@@Z 1001ecac f   Qt5Widgets:Qt5Widgets.dll
 0001:0001dcb2       ?dragLeaveEvent@QTextEdit@@MAEXPAVQDragLeaveEvent@@@Z 1001ecb2 f   Qt5Widgets:Qt5Widgets.dll
 0001:0001dcb8       ?dragLeaveEvent@QWidget@@MAEXPAVQDragLeaveEvent@@@Z 1001ecb8 f   Qt5Widgets:Qt5Widgets.dll
 0001:0001dcbe       ?dragMoveEvent@QTextEdit@@MAEXPAVQDragMoveEvent@@@Z 1001ecbe f   Qt5Widgets:Qt5Widgets.dll
 0001:0001dcc4       ?dragMoveEvent@QTreeView@@MAEXPAVQDragMoveEvent@@@Z 1001ecc4 f   Qt5Widgets:Qt5Widgets.dll
 0001:0001dcca       ?dragMoveEvent@QWidget@@MAEXPAVQDragMoveEvent@@@Z 1001ecca f   Qt5Widgets:Qt5Widgets.dll
 0001:0001dcd0       ?drawBranches@QTreeView@@MBEXPAVQPainter@@ABVQRect@@ABVQModelIndex@@@Z 1001ecd0 f   Qt5Widgets:Qt5Widgets.dll
 0001:0001dcd6       ?drawRow@QTreeView@@MBEXPAVQPainter@@ABVQStyleOptionViewItem@@ABVQModelIndex@@@Z 1001ecd6 f   Qt5Widgets:Qt5Widgets.dll
 0001:0001dcdc       ?dropEvent@QTextEdit@@MAEXPAVQDropEvent@@@Z 1001ecdc f   Qt5Widgets:Qt5Widgets.dll
 0001:0001dce2       ?dropEvent@QTreeWidget@@MAEXPAVQDropEvent@@@Z 1001ece2 f   Qt5Widgets:Qt5Widgets.dll
 0001:0001dce8       ?dropEvent@QWidget@@MAEXPAVQDropEvent@@@Z 1001ece8 f   Qt5Widgets:Qt5Widgets.dll
 0001:0001dcee       ?dropMimeData@QTreeWidget@@MAE_NPAVQTreeWidgetItem@@HPBVQMimeData@@W4DropAction@Qt@@@Z 1001ecee f   Qt5Widgets:Qt5Widgets.dll
 0001:0001dcf4       ?edit@QAbstractItemView@@MAE_NABVQModelIndex@@W4EditTrigger@1@PAVQEvent@@@Z 1001ecf4 f   Qt5Widgets:Qt5Widgets.dll
 0001:0001dcfa       ?editorDestroyed@QAbstractItemView@@MAEXPAVQObject@@@Z 1001ecfa f   Qt5Widgets:Qt5Widgets.dll
 0001:0001dd00       ?enterEvent@QWidget@@MAEXPAVQEvent@@@Z 1001ed00 f   Qt5Widgets:Qt5Widgets.dll
 0001:0001dd06       ?event@QCheckBox@@MAE_NPAVQEvent@@@Z 1001ed06 f   Qt5Widgets:Qt5Widgets.dll
 0001:0001dd0c       ?event@QComboBox@@UAE_NPAVQEvent@@@Z 1001ed0c f   Qt5Widgets:Qt5Widgets.dll
 0001:0001dd12       ?event@QDialogButtonBox@@MAE_NPAVQEvent@@@Z 1001ed12 f   Qt5Widgets:Qt5Widgets.dll
 0001:0001dd18       ?event@QGroupBox@@MAE_NPAVQEvent@@@Z 1001ed18 f   Qt5Widgets:Qt5Widgets.dll
 0001:0001dd1e       ?event@QLabel@@MAE_NPAVQEvent@@@Z 1001ed1e f   Qt5Widgets:Qt5Widgets.dll
 0001:0001dd24       ?event@QPushButton@@MAE_NPAVQEvent@@@Z 1001ed24 f   Qt5Widgets:Qt5Widgets.dll
 0001:0001dd2a       ?event@QRadioButton@@MAE_NPAVQEvent@@@Z 1001ed2a f   Qt5Widgets:Qt5Widgets.dll
 0001:0001dd30       ?event@QSpinBox@@MAE_NPAVQEvent@@@Z 1001ed30 f   Qt5Widgets:Qt5Widgets.dll
 0001:0001dd36       ?event@QTabWidget@@MAE_NPAVQEvent@@@Z 1001ed36 f   Qt5Widgets:Qt5Widgets.dll
 0001:0001dd3c       ?event@QTextEdit@@MAE_NPAVQEvent@@@Z 1001ed3c f   Qt5Widgets:Qt5Widgets.dll
 0001:0001dd42       ?event@QTreeWidget@@MAE_NPAVQEvent@@@Z 1001ed42 f   Qt5Widgets:Qt5Widgets.dll
 0001:0001dd48       ?event@QWidget@@MAE_NPAVQEvent@@@Z 1001ed48 f   Qt5Widgets:Qt5Widgets.dll
 0001:0001dd4e       ?eventFilter@QAbstractScrollArea@@MAE_NPAVQObject@@PAVQEvent@@@Z 1001ed4e f   Qt5Widgets:Qt5Widgets.dll
 0001:0001dd54       ?exec@QDialog@@UAEHXZ      1001ed54 f   Qt5Widgets:Qt5Widgets.dll
 0001:0001dd5a       ?expandingDirections@QBoxLayout@@UBE?AV?$QFlags@W4Orientation@Qt@@@@XZ 1001ed5a f   Qt5Widgets:Qt5Widgets.dll
 0001:0001dd60       ?expandingDirections@QGridLayout@@UBE?AV?$QFlags@W4Orientation@Qt@@@@XZ 1001ed60 f   Qt5Widgets:Qt5Widgets.dll
 0001:0001dd66       ?expandingDirections@QSpacerItem@@UBE?AV?$QFlags@W4Orientation@Qt@@@@XZ 1001ed66 f   Qt5Widgets:Qt5Widgets.dll
 0001:0001dd6c       ?fixup@QSpinBox@@MBEXAAVQString@@@Z 1001ed6c f   Qt5Widgets:Qt5Widgets.dll
 0001:0001dd72       ?focusInEvent@QAbstractButton@@MAEXPAVQFocusEvent@@@Z 1001ed72 f   Qt5Widgets:Qt5Widgets.dll
 0001:0001dd78       ?focusInEvent@QAbstractItemView@@MAEXPAVQFocusEvent@@@Z 1001ed78 f   Qt5Widgets:Qt5Widgets.dll
 0001:0001dd7e       ?focusInEvent@QAbstractSpinBox@@MAEXPAVQFocusEvent@@@Z 1001ed7e f   Qt5Widgets:Qt5Widgets.dll
 0001:0001dd84       ?focusInEvent@QComboBox@@MAEXPAVQFocusEvent@@@Z 1001ed84 f   Qt5Widgets:Qt5Widgets.dll
 0001:0001dd8a       ?focusInEvent@QGroupBox@@MAEXPAVQFocusEvent@@@Z 1001ed8a f   Qt5Widgets:Qt5Widgets.dll
 0001:0001dd90       ?focusInEvent@QLabel@@MAEXPAVQFocusEvent@@@Z 1001ed90 f   Qt5Widgets:Qt5Widgets.dll
 0001:0001dd96       ?focusInEvent@QPushButton@@MAEXPAVQFocusEvent@@@Z 1001ed96 f   Qt5Widgets:Qt5Widgets.dll
 0001:0001dd9c       ?focusInEvent@QTextEdit@@MAEXPAVQFocusEvent@@@Z 1001ed9c f   Qt5Widgets:Qt5Widgets.dll
 0001:0001dda2       ?focusInEvent@QWidget@@MAEXPAVQFocusEvent@@@Z 1001eda2 f   Qt5Widgets:Qt5Widgets.dll
 0001:0001dda8       ?focusNextPrevChild@QAbstractItemView@@MAE_N_N@Z 1001eda8 f   Qt5Widgets:Qt5Widgets.dll
 0001:0001ddae       ?focusNextPrevChild@QLabel@@MAE_N_N@Z 1001edae f   Qt5Widgets:Qt5Widgets.dll
 0001:0001ddb4       ?focusNextPrevChild@QTextEdit@@MAE_N_N@Z 1001edb4 f   Qt5Widgets:Qt5Widgets.dll
 0001:0001ddba       ?focusNextPrevChild@QWidget@@MAE_N_N@Z 1001edba f   Qt5Widgets:Qt5Widgets.dll
 0001:0001ddc0       ?focusOutEvent@QAbstractButton@@MAEXPAVQFocusEvent@@@Z 1001edc0 f   Qt5Widgets:Qt5Widgets.dll
 0001:0001ddc6       ?focusOutEvent@QAbstractItemView@@MAEXPAVQFocusEvent@@@Z 1001edc6 f   Qt5Widgets:Qt5Widgets.dll
 0001:0001ddcc       ?focusOutEvent@QAbstractSpinBox@@MAEXPAVQFocusEvent@@@Z 1001edcc f   Qt5Widgets:Qt5Widgets.dll
 0001:0001ddd2       ?focusOutEvent@QComboBox@@MAEXPAVQFocusEvent@@@Z 1001edd2 f   Qt5Widgets:Qt5Widgets.dll
 0001:0001ddd8       ?focusOutEvent@QLabel@@MAEXPAVQFocusEvent@@@Z 1001edd8 f   Qt5Widgets:Qt5Widgets.dll
 0001:0001ddde       ?focusOutEvent@QPushButton@@MAEXPAVQFocusEvent@@@Z 1001edde f   Qt5Widgets:Qt5Widgets.dll
 0001:0001dde4       ?focusOutEvent@QTextEdit@@MAEXPAVQFocusEvent@@@Z 1001ede4 f   Qt5Widgets:Qt5Widgets.dll
 0001:0001ddea       ?focusOutEvent@QWidget@@MAEXPAVQFocusEvent@@@Z 1001edea f   Qt5Widgets:Qt5Widgets.dll
 0001:0001ddf0       ?geometry@QLayout@@UBE?AVQRect@@XZ 1001edf0 f   Qt5Widgets:Qt5Widgets.dll
 0001:0001ddf6       ?geometry@QSpacerItem@@UBE?AVQRect@@XZ 1001edf6 f   Qt5Widgets:Qt5Widgets.dll
 0001:0001ddfc       ?hasHeightForWidth@QBoxLayout@@UBE_NXZ 1001edfc f   Qt5Widgets:Qt5Widgets.dll
 0001:0001de02       ?hasHeightForWidth@QGridLayout@@UBE_NXZ 1001ee02 f   Qt5Widgets:Qt5Widgets.dll
 0001:0001de08       ?hasHeightForWidth@QLayoutItem@@UBE_NXZ 1001ee08 f   Qt5Widgets:Qt5Widgets.dll
 0001:0001de0e       ?hasHeightForWidth@QTabWidget@@UBE_NXZ 1001ee0e f   Qt5Widgets:Qt5Widgets.dll
 0001:0001de14       ?hasHeightForWidth@QWidget@@UBE_NXZ 1001ee14 f   Qt5Widgets:Qt5Widgets.dll
 0001:0001de1a       ?heightForWidth@QBoxLayout@@UBEHH@Z 1001ee1a f   Qt5Widgets:Qt5Widgets.dll
 0001:0001de20       ?heightForWidth@QGridLayout@@UBEHH@Z 1001ee20 f   Qt5Widgets:Qt5Widgets.dll
 0001:0001de26       ?heightForWidth@QLabel@@UBEHH@Z 1001ee26 f   Qt5Widgets:Qt5Widgets.dll
 0001:0001de2c       ?heightForWidth@QLayoutItem@@UBEHH@Z 1001ee2c f   Qt5Widgets:Qt5Widgets.dll
 0001:0001de32       ?heightForWidth@QTabWidget@@UBEHH@Z 1001ee32 f   Qt5Widgets:Qt5Widgets.dll
 0001:0001de38       ?heightForWidth@QWidget@@UBEHH@Z 1001ee38 f   Qt5Widgets:Qt5Widgets.dll
 0001:0001de3e       ?hideEvent@QAbstractSpinBox@@MAEXPAVQHideEvent@@@Z 1001ee3e f   Qt5Widgets:Qt5Widgets.dll
 0001:0001de44       ?hideEvent@QComboBox@@MAEXPAVQHideEvent@@@Z 1001ee44 f   Qt5Widgets:Qt5Widgets.dll
 0001:0001de4a       ?hideEvent@QWidget@@MAEXPAVQHideEvent@@@Z 1001ee4a f   Qt5Widgets:Qt5Widgets.dll
 0001:0001de50       ?hidePopup@QComboBox@@UAEXXZ 1001ee50 f   Qt5Widgets:Qt5Widgets.dll
 0001:0001de56       ?hitButton@QAbstractButton@@MBE_NABVQPoint@@@Z 1001ee56 f   Qt5Widgets:Qt5Widgets.dll
 0001:0001de5c       ?hitButton@QCheckBox@@MBE_NABVQPoint@@@Z 1001ee5c f   Qt5Widgets:Qt5Widgets.dll
 0001:0001de62       ?hitButton@QRadioButton@@MBE_NABVQPoint@@@Z 1001ee62 f   Qt5Widgets:Qt5Widgets.dll
 0001:0001de68       ?horizontalOffset@QTreeView@@MBEHXZ 1001ee68 f   Qt5Widgets:Qt5Widgets.dll
 0001:0001de6e       ?horizontalScrollbarAction@QTreeView@@MAEXH@Z 1001ee6e f   Qt5Widgets:Qt5Widgets.dll
 0001:0001de74       ?horizontalScrollbarValueChanged@QAbstractItemView@@MAEXH@Z 1001ee74 f   Qt5Widgets:Qt5Widgets.dll
 0001:0001de7a       ?indexAt@QTreeView@@UBE?AVQModelIndex@@ABVQPoint@@@Z 1001ee7a f   Qt5Widgets:Qt5Widgets.dll
 0001:0001de80       ?indexOf@QLayout@@UBEHPAVQWidget@@@Z 1001ee80 f   Qt5Widgets:Qt5Widgets.dll
 0001:0001de86       ?initPainter@QWidget@@MBEXPAVQPainter@@@Z 1001ee86 f   Qt5Widgets:Qt5Widgets.dll
 0001:0001de8c       ?inputMethodEvent@QAbstractItemView@@MAEXPAVQInputMethodEvent@@@Z 1001ee8c f   Qt5Widgets:Qt5Widgets.dll
 0001:0001de92       ?inputMethodEvent@QComboBox@@MAEXPAVQInputMethodEvent@@@Z 1001ee92 f   Qt5Widgets:Qt5Widgets.dll
 0001:0001de98       ?inputMethodEvent@QTextEdit@@MAEXPAVQInputMethodEvent@@@Z 1001ee98 f   Qt5Widgets:Qt5Widgets.dll
 0001:0001de9e       ?inputMethodEvent@QWidget@@MAEXPAVQInputMethodEvent@@@Z 1001ee9e f   Qt5Widgets:Qt5Widgets.dll
 0001:0001dea4       ?inputMethodQuery@QAbstractItemView@@UBE?AVQVariant@@W4InputMethodQuery@Qt@@@Z 1001eea4 f   Qt5Widgets:Qt5Widgets.dll
 0001:0001deaa       ?inputMethodQuery@QAbstractSpinBox@@UBE?AVQVariant@@W4InputMethodQuery@Qt@@@Z 1001eeaa f   Qt5Widgets:Qt5Widgets.dll
 0001:0001deb0       ?inputMethodQuery@QComboBox@@UBE?AVQVariant@@W4InputMethodQuery@Qt@@@Z 1001eeb0 f   Qt5Widgets:Qt5Widgets.dll
 0001:0001deb6       ?inputMethodQuery@QTextEdit@@UBE?AVQVariant@@W4InputMethodQuery@Qt@@@Z 1001eeb6 f   Qt5Widgets:Qt5Widgets.dll
 0001:0001debc       ?inputMethodQuery@QWidget@@UBE?AVQVariant@@W4InputMethodQuery@Qt@@@Z 1001eebc f   Qt5Widgets:Qt5Widgets.dll
 0001:0001dec2       ?insertFromMimeData@QTextEdit@@MAEXPBVQMimeData@@@Z 1001eec2 f   Qt5Widgets:Qt5Widgets.dll
 0001:0001dec8       ?invalidate@QBoxLayout@@UAEXXZ 1001eec8 f   Qt5Widgets:Qt5Widgets.dll
 0001:0001dece       ?invalidate@QGridLayout@@UAEXXZ 1001eece f   Qt5Widgets:Qt5Widgets.dll
 0001:0001ded4       ?invalidate@QLayoutItem@@UAEXXZ 1001eed4 f   Qt5Widgets:Qt5Widgets.dll
 0001:0001deda       ?isEmpty@QLayout@@UBE_NXZ  1001eeda f   Qt5Widgets:Qt5Widgets.dll
 0001:0001dee0       ?isEmpty@QSpacerItem@@UBE_NXZ 1001eee0 f   Qt5Widgets:Qt5Widgets.dll
 0001:0001dee6       ?isIndexHidden@QTreeView@@MBE_NABVQModelIndex@@@Z 1001eee6 f   Qt5Widgets:Qt5Widgets.dll
 0001:0001deec       ?itemAt@QBoxLayout@@UBEPAVQLayoutItem@@H@Z 1001eeec f   Qt5Widgets:Qt5Widgets.dll
 0001:0001def2       ?itemAt@QGridLayout@@UBEPAVQLayoutItem@@H@Z 1001eef2 f   Qt5Widgets:Qt5Widgets.dll
 0001:0001def8       ?keyPressEvent@QAbstractButton@@MAEXPAVQKeyEvent@@@Z 1001eef8 f   Qt5Widgets:Qt5Widgets.dll
 0001:0001defe       ?keyPressEvent@QAbstractSpinBox@@MAEXPAVQKeyEvent@@@Z 1001eefe f   Qt5Widgets:Qt5Widgets.dll
 0001:0001df04       ?keyPressEvent@QComboBox@@MAEXPAVQKeyEvent@@@Z 1001ef04 f   Qt5Widgets:Qt5Widgets.dll
 0001:0001df0a       ?keyPressEvent@QDialog@@MAEXPAVQKeyEvent@@@Z 1001ef0a f   Qt5Widgets:Qt5Widgets.dll
 0001:0001df10       ?keyPressEvent@QLabel@@MAEXPAVQKeyEvent@@@Z 1001ef10 f   Qt5Widgets:Qt5Widgets.dll
 0001:0001df16       ?keyPressEvent@QPushButton@@MAEXPAVQKeyEvent@@@Z 1001ef16 f   Qt5Widgets:Qt5Widgets.dll
 0001:0001df1c       ?keyPressEvent@QTabWidget@@MAEXPAVQKeyEvent@@@Z 1001ef1c f   Qt5Widgets:Qt5Widgets.dll
 0001:0001df22       ?keyPressEvent@QTextEdit@@MAEXPAVQKeyEvent@@@Z 1001ef22 f   Qt5Widgets:Qt5Widgets.dll
 0001:0001df28       ?keyPressEvent@QTreeView@@MAEXPAVQKeyEvent@@@Z 1001ef28 f   Qt5Widgets:Qt5Widgets.dll
 0001:0001df2e       ?keyPressEvent@QWidget@@MAEXPAVQKeyEvent@@@Z 1001ef2e f   Qt5Widgets:Qt5Widgets.dll
 0001:0001df34       ?keyReleaseEvent@QAbstractButton@@MAEXPAVQKeyEvent@@@Z 1001ef34 f   Qt5Widgets:Qt5Widgets.dll
 0001:0001df3a       ?keyReleaseEvent@QAbstractSpinBox@@MAEXPAVQKeyEvent@@@Z 1001ef3a f   Qt5Widgets:Qt5Widgets.dll
 0001:0001df40       ?keyReleaseEvent@QComboBox@@MAEXPAVQKeyEvent@@@Z 1001ef40 f   Qt5Widgets:Qt5Widgets.dll
 0001:0001df46       ?keyReleaseEvent@QTextEdit@@MAEXPAVQKeyEvent@@@Z 1001ef46 f   Qt5Widgets:Qt5Widgets.dll
 0001:0001df4c       ?keyReleaseEvent@QWidget@@MAEXPAVQKeyEvent@@@Z 1001ef4c f   Qt5Widgets:Qt5Widgets.dll
 0001:0001df52       ?keyboardSearch@QTreeView@@UAEXABVQString@@@Z 1001ef52 f   Qt5Widgets:Qt5Widgets.dll
 0001:0001df58       ?layout@QLayout@@UAEPAV1@XZ 1001ef58 f   Qt5Widgets:Qt5Widgets.dll
 0001:0001df5e       ?layout@QLayoutItem@@UAEPAVQLayout@@XZ 1001ef5e f   Qt5Widgets:Qt5Widgets.dll
 0001:0001df64       ?leaveEvent@QWidget@@MAEXPAVQEvent@@@Z 1001ef64 f   Qt5Widgets:Qt5Widgets.dll
 0001:0001df6a       ?loadResource@QTextEdit@@UAE?AVQVariant@@HABVQUrl@@@Z 1001ef6a f   Qt5Widgets:Qt5Widgets.dll
 0001:0001df70       ?maximumSize@QBoxLayout@@UBE?AVQSize@@XZ 1001ef70 f   Qt5Widgets:Qt5Widgets.dll
 0001:0001df76       ?maximumSize@QGridLayout@@UBE?AVQSize@@XZ 1001ef76 f   Qt5Widgets:Qt5Widgets.dll
 0001:0001df7c       ?maximumSize@QSpacerItem@@UBE?AVQSize@@XZ 1001ef7c f   Qt5Widgets:Qt5Widgets.dll
 0001:0001df82       ?metaObject@QCheckBox@@UBEPBUQMetaObject@@XZ 1001ef82 f   Qt5Widgets:Qt5Widgets.dll
 0001:0001df88       ?metaObject@QComboBox@@UBEPBUQMetaObject@@XZ 1001ef88 f   Qt5Widgets:Qt5Widgets.dll
 0001:0001df8e       ?metaObject@QDialogButtonBox@@UBEPBUQMetaObject@@XZ 1001ef8e f   Qt5Widgets:Qt5Widgets.dll
 0001:0001df94       ?metaObject@QGridLayout@@UBEPBUQMetaObject@@XZ 1001ef94 f   Qt5Widgets:Qt5Widgets.dll
 0001:0001df9a       ?metaObject@QGroupBox@@UBEPBUQMetaObject@@XZ 1001ef9a f   Qt5Widgets:Qt5Widgets.dll
 0001:0001dfa0       ?metaObject@QHBoxLayout@@UBEPBUQMetaObject@@XZ 1001efa0 f   Qt5Widgets:Qt5Widgets.dll
 0001:0001dfa6       ?metaObject@QLabel@@UBEPBUQMetaObject@@XZ 1001efa6 f   Qt5Widgets:Qt5Widgets.dll
 0001:0001dfac       ?metaObject@QPushButton@@UBEPBUQMetaObject@@XZ 1001efac f   Qt5Widgets:Qt5Widgets.dll
 0001:0001dfb2       ?metaObject@QRadioButton@@UBEPBUQMetaObject@@XZ 1001efb2 f   Qt5Widgets:Qt5Widgets.dll
 0001:0001dfb8       ?metaObject@QSpinBox@@UBEPBUQMetaObject@@XZ 1001efb8 f   Qt5Widgets:Qt5Widgets.dll
 0001:0001dfbe       ?metaObject@QTabWidget@@UBEPBUQMetaObject@@XZ 1001efbe f   Qt5Widgets:Qt5Widgets.dll
 0001:0001dfc4       ?metaObject@QTextEdit@@UBEPBUQMetaObject@@XZ 1001efc4 f   Qt5Widgets:Qt5Widgets.dll
 0001:0001dfca       ?metaObject@QTreeWidget@@UBEPBUQMetaObject@@XZ 1001efca f   Qt5Widgets:Qt5Widgets.dll
 0001:0001dfd0       ?metaObject@QVBoxLayout@@UBEPBUQMetaObject@@XZ 1001efd0 f   Qt5Widgets:Qt5Widgets.dll
 0001:0001dfd6       ?metaObject@QWidget@@UBEPBUQMetaObject@@XZ 1001efd6 f   Qt5Widgets:Qt5Widgets.dll
 0001:0001dfdc       ?metric@QWidget@@MBEHW4PaintDeviceMetric@QPaintDevice@@@Z 1001efdc f   Qt5Widgets:Qt5Widgets.dll
 0001:0001dfe2       ?mimeData@QTreeWidget@@MBEPAVQMimeData@@V?$QList@PAVQTreeWidgetItem@@@@@Z 1001efe2 f   Qt5Widgets:Qt5Widgets.dll
 0001:0001dfe8       ?mimeTypes@QTreeWidget@@MBE?AVQStringList@@XZ 1001efe8 f   Qt5Widgets:Qt5Widgets.dll
 0001:0001dfee       ?minimumHeightForWidth@QBoxLayout@@UBEHH@Z 1001efee f   Qt5Widgets:Qt5Widgets.dll
 0001:0001dff4       ?minimumHeightForWidth@QGridLayout@@UBEHH@Z 1001eff4 f   Qt5Widgets:Qt5Widgets.dll
 0001:0001dffa       ?minimumHeightForWidth@QLayoutItem@@UBEHH@Z 1001effa f   Qt5Widgets:Qt5Widgets.dll
 0001:0001e000       ?minimumSize@QBoxLayout@@UBE?AVQSize@@XZ 1001f000 f   Qt5Widgets:Qt5Widgets.dll
 0001:0001e006       ?minimumSize@QGridLayout@@UBE?AVQSize@@XZ 1001f006 f   Qt5Widgets:Qt5Widgets.dll
 0001:0001e00c       ?minimumSize@QSpacerItem@@UBE?AVQSize@@XZ 1001f00c f   Qt5Widgets:Qt5Widgets.dll
 0001:0001e012       ?minimumSizeHint@QAbstractScrollArea@@UBE?AVQSize@@XZ 1001f012 f   Qt5Widgets:Qt5Widgets.dll
 0001:0001e018       ?minimumSizeHint@QAbstractSpinBox@@UBE?AVQSize@@XZ 1001f018 f   Qt5Widgets:Qt5Widgets.dll
 0001:0001e01e       ?minimumSizeHint@QCheckBox@@UBE?AVQSize@@XZ 1001f01e f   Qt5Widgets:Qt5Widgets.dll
 0001:0001e024       ?minimumSizeHint@QComboBox@@UBE?AVQSize@@XZ 1001f024 f   Qt5Widgets:Qt5Widgets.dll
 0001:0001e02a       ?minimumSizeHint@QDialog@@UBE?AVQSize@@XZ 1001f02a f   Qt5Widgets:Qt5Widgets.dll
 0001:0001e030       ?minimumSizeHint@QGroupBox@@UBE?AVQSize@@XZ 1001f030 f   Qt5Widgets:Qt5Widgets.dll
 0001:0001e036       ?minimumSizeHint@QLabel@@UBE?AVQSize@@XZ 1001f036 f   Qt5Widgets:Qt5Widgets.dll
 0001:0001e03c       ?minimumSizeHint@QPushButton@@UBE?AVQSize@@XZ 1001f03c f   Qt5Widgets:Qt5Widgets.dll
 0001:0001e042       ?minimumSizeHint@QRadioButton@@UBE?AVQSize@@XZ 1001f042 f   Qt5Widgets:Qt5Widgets.dll
 0001:0001e048       ?minimumSizeHint@QTabWidget@@UBE?AVQSize@@XZ 1001f048 f   Qt5Widgets:Qt5Widgets.dll
 0001:0001e04e       ?minimumSizeHint@QWidget@@UBE?AVQSize@@XZ 1001f04e f   Qt5Widgets:Qt5Widgets.dll
 0001:0001e054       ?mouseDoubleClickEvent@QTextEdit@@MAEXPAVQMouseEvent@@@Z 1001f054 f   Qt5Widgets:Qt5Widgets.dll
 0001:0001e05a       ?mouseDoubleClickEvent@QTreeView@@MAEXPAVQMouseEvent@@@Z 1001f05a f   Qt5Widgets:Qt5Widgets.dll
 0001:0001e060       ?mouseDoubleClickEvent@QWidget@@MAEXPAVQMouseEvent@@@Z 1001f060 f   Qt5Widgets:Qt5Widgets.dll
 0001:0001e066       ?mouseMoveEvent@QAbstractButton@@MAEXPAVQMouseEvent@@@Z 1001f066 f   Qt5Widgets:Qt5Widgets.dll
 0001:0001e06c       ?mouseMoveEvent@QAbstractSpinBox@@MAEXPAVQMouseEvent@@@Z 1001f06c f   Qt5Widgets:Qt5Widgets.dll
 0001:0001e072       ?mouseMoveEvent@QCheckBox@@MAEXPAVQMouseEvent@@@Z 1001f072 f   Qt5Widgets:Qt5Widgets.dll
 0001:0001e078       ?mouseMoveEvent@QGroupBox@@MAEXPAVQMouseEvent@@@Z 1001f078 f   Qt5Widgets:Qt5Widgets.dll
 0001:0001e07e       ?mouseMoveEvent@QLabel@@MAEXPAVQMouseEvent@@@Z 1001f07e f   Qt5Widgets:Qt5Widgets.dll
 0001:0001e084       ?mouseMoveEvent@QRadioButton@@MAEXPAVQMouseEvent@@@Z 1001f084 f   Qt5Widgets:Qt5Widgets.dll
 0001:0001e08a       ?mouseMoveEvent@QTextEdit@@MAEXPAVQMouseEvent@@@Z 1001f08a f   Qt5Widgets:Qt5Widgets.dll
 0001:0001e090       ?mouseMoveEvent@QTreeView@@MAEXPAVQMouseEvent@@@Z 1001f090 f   Qt5Widgets:Qt5Widgets.dll
 0001:0001e096       ?mouseMoveEvent@QWidget@@MAEXPAVQMouseEvent@@@Z 1001f096 f   Qt5Widgets:Qt5Widgets.dll
 0001:0001e09c       ?mousePressEvent@QAbstractButton@@MAEXPAVQMouseEvent@@@Z 1001f09c f   Qt5Widgets:Qt5Widgets.dll
 0001:0001e0a2       ?mousePressEvent@QAbstractSpinBox@@MAEXPAVQMouseEvent@@@Z 1001f0a2 f   Qt5Widgets:Qt5Widgets.dll
 0001:0001e0a8       ?mousePressEvent@QComboBox@@MAEXPAVQMouseEvent@@@Z 1001f0a8 f   Qt5Widgets:Qt5Widgets.dll
 0001:0001e0ae       ?mousePressEvent@QGroupBox@@MAEXPAVQMouseEvent@@@Z 1001f0ae f   Qt5Widgets:Qt5Widgets.dll
 0001:0001e0b4       ?mousePressEvent@QLabel@@MAEXPAVQMouseEvent@@@Z 1001f0b4 f   Qt5Widgets:Qt5Widgets.dll
 0001:0001e0ba       ?mousePressEvent@QTextEdit@@MAEXPAVQMouseEvent@@@Z 1001f0ba f   Qt5Widgets:Qt5Widgets.dll
 0001:0001e0c0       ?mousePressEvent@QTreeView@@MAEXPAVQMouseEvent@@@Z 1001f0c0 f   Qt5Widgets:Qt5Widgets.dll
 0001:0001e0c6       ?mousePressEvent@QWidget@@MAEXPAVQMouseEvent@@@Z 1001f0c6 f   Qt5Widgets:Qt5Widgets.dll
 0001:0001e0cc       ?mouseReleaseEvent@QAbstractButton@@MAEXPAVQMouseEvent@@@Z 1001f0cc f   Qt5Widgets:Qt5Widgets.dll
 0001:0001e0d2       ?mouseReleaseEvent@QAbstractSpinBox@@MAEXPAVQMouseEvent@@@Z 1001f0d2 f   Qt5Widgets:Qt5Widgets.dll
 0001:0001e0d8       ?mouseReleaseEvent@QComboBox@@MAEXPAVQMouseEvent@@@Z 1001f0d8 f   Qt5Widgets:Qt5Widgets.dll
 0001:0001e0de       ?mouseReleaseEvent@QGroupBox@@MAEXPAVQMouseEvent@@@Z 1001f0de f   Qt5Widgets:Qt5Widgets.dll
 0001:0001e0e4       ?mouseReleaseEvent@QLabel@@MAEXPAVQMouseEvent@@@Z 1001f0e4 f   Qt5Widgets:Qt5Widgets.dll
 0001:0001e0ea       ?mouseReleaseEvent@QTextEdit@@MAEXPAVQMouseEvent@@@Z 1001f0ea f   Qt5Widgets:Qt5Widgets.dll
 0001:0001e0f0       ?mouseReleaseEvent@QTreeView@@MAEXPAVQMouseEvent@@@Z 1001f0f0 f   Qt5Widgets:Qt5Widgets.dll
 0001:0001e0f6       ?mouseReleaseEvent@QWidget@@MAEXPAVQMouseEvent@@@Z 1001f0f6 f   Qt5Widgets:Qt5Widgets.dll
 0001:0001e0fc       ?moveCursor@QTreeView@@MAE?AVQModelIndex@@W4CursorAction@QAbstractItemView@@V?$QFlags@W4KeyboardModifier@Qt@@@@@Z 1001f0fc f   Qt5Widgets:Qt5Widgets.dll
 0001:0001e102       ?moveEvent@QWidget@@MAEXPAVQMoveEvent@@@Z 1001f102 f   Qt5Widgets:Qt5Widgets.dll
 0001:0001e108       ?nativeEvent@QWidget@@MAE_NABVQByteArray@@PAXPAJ@Z 1001f108 f   Qt5Widgets:Qt5Widgets.dll
 0001:0001e10e       ?nextCheckState@QAbstractButton@@MAEXXZ 1001f10e f   Qt5Widgets:Qt5Widgets.dll
 0001:0001e114       ?nextCheckState@QCheckBox@@MAEXXZ 1001f114 f   Qt5Widgets:Qt5Widgets.dll
 0001:0001e11a       ?open@QDialog@@UAEXXZ      1001f11a f   Qt5Widgets:Qt5Widgets.dll
 0001:0001e120       ?paintEngine@QWidget@@UBEPAVQPaintEngine@@XZ 1001f120 f   Qt5Widgets:Qt5Widgets.dll
 0001:0001e126       ?paintEvent@QAbstractSpinBox@@MAEXPAVQPaintEvent@@@Z 1001f126 f   Qt5Widgets:Qt5Widgets.dll
 0001:0001e12c       ?paintEvent@QCheckBox@@MAEXPAVQPaintEvent@@@Z 1001f12c f   Qt5Widgets:Qt5Widgets.dll
 0001:0001e132       ?paintEvent@QComboBox@@MAEXPAVQPaintEvent@@@Z 1001f132 f   Qt5Widgets:Qt5Widgets.dll
 0001:0001e138       ?paintEvent@QGroupBox@@MAEXPAVQPaintEvent@@@Z 1001f138 f   Qt5Widgets:Qt5Widgets.dll
 0001:0001e13e       ?paintEvent@QLabel@@MAEXPAVQPaintEvent@@@Z 1001f13e f   Qt5Widgets:Qt5Widgets.dll
 0001:0001e144       ?paintEvent@QPushButton@@MAEXPAVQPaintEvent@@@Z 1001f144 f   Qt5Widgets:Qt5Widgets.dll
 0001:0001e14a       ?paintEvent@QRadioButton@@MAEXPAVQPaintEvent@@@Z 1001f14a f   Qt5Widgets:Qt5Widgets.dll
 0001:0001e150       ?paintEvent@QTabWidget@@MAEXPAVQPaintEvent@@@Z 1001f150 f   Qt5Widgets:Qt5Widgets.dll
 0001:0001e156       ?paintEvent@QTextEdit@@MAEXPAVQPaintEvent@@@Z 1001f156 f   Qt5Widgets:Qt5Widgets.dll
 0001:0001e15c       ?paintEvent@QTreeView@@MAEXPAVQPaintEvent@@@Z 1001f15c f   Qt5Widgets:Qt5Widgets.dll
 0001:0001e162       ?paintEvent@QWidget@@MAEXPAVQPaintEvent@@@Z 1001f162 f   Qt5Widgets:Qt5Widgets.dll
 0001:0001e168       ?qt_metacall@QCheckBox@@UAEHW4Call@QMetaObject@@HPAPAX@Z 1001f168 f   Qt5Widgets:Qt5Widgets.dll
 0001:0001e16e       ?qt_metacall@QComboBox@@UAEHW4Call@QMetaObject@@HPAPAX@Z 1001f16e f   Qt5Widgets:Qt5Widgets.dll
 0001:0001e174       ?qt_metacall@QDialogButtonBox@@UAEHW4Call@QMetaObject@@HPAPAX@Z 1001f174 f   Qt5Widgets:Qt5Widgets.dll
 0001:0001e17a       ?qt_metacall@QGridLayout@@UAEHW4Call@QMetaObject@@HPAPAX@Z 1001f17a f   Qt5Widgets:Qt5Widgets.dll
 0001:0001e180       ?qt_metacall@QGroupBox@@UAEHW4Call@QMetaObject@@HPAPAX@Z 1001f180 f   Qt5Widgets:Qt5Widgets.dll
 0001:0001e186       ?qt_metacall@QHBoxLayout@@UAEHW4Call@QMetaObject@@HPAPAX@Z 1001f186 f   Qt5Widgets:Qt5Widgets.dll
 0001:0001e18c       ?qt_metacall@QLabel@@UAEHW4Call@QMetaObject@@HPAPAX@Z 1001f18c f   Qt5Widgets:Qt5Widgets.dll
 0001:0001e192       ?qt_metacall@QPushButton@@UAEHW4Call@QMetaObject@@HPAPAX@Z 1001f192 f   Qt5Widgets:Qt5Widgets.dll
 0001:0001e198       ?qt_metacall@QRadioButton@@UAEHW4Call@QMetaObject@@HPAPAX@Z 1001f198 f   Qt5Widgets:Qt5Widgets.dll
 0001:0001e19e       ?qt_metacall@QSpinBox@@UAEHW4Call@QMetaObject@@HPAPAX@Z 1001f19e f   Qt5Widgets:Qt5Widgets.dll
 0001:0001e1a4       ?qt_metacall@QTabWidget@@UAEHW4Call@QMetaObject@@HPAPAX@Z 1001f1a4 f   Qt5Widgets:Qt5Widgets.dll
 0001:0001e1aa       ?qt_metacall@QTextEdit@@UAEHW4Call@QMetaObject@@HPAPAX@Z 1001f1aa f   Qt5Widgets:Qt5Widgets.dll
 0001:0001e1b0       ?qt_metacall@QTreeWidget@@UAEHW4Call@QMetaObject@@HPAPAX@Z 1001f1b0 f   Qt5Widgets:Qt5Widgets.dll
 0001:0001e1b6       ?qt_metacall@QVBoxLayout@@UAEHW4Call@QMetaObject@@HPAPAX@Z 1001f1b6 f   Qt5Widgets:Qt5Widgets.dll
 0001:0001e1bc       ?qt_metacall@QWidget@@UAEHW4Call@QMetaObject@@HPAPAX@Z 1001f1bc f   Qt5Widgets:Qt5Widgets.dll
 0001:0001e1c2       ?qt_metacast@QCheckBox@@UAEPAXPBD@Z 1001f1c2 f   Qt5Widgets:Qt5Widgets.dll
 0001:0001e1c8       ?qt_metacast@QComboBox@@UAEPAXPBD@Z 1001f1c8 f   Qt5Widgets:Qt5Widgets.dll
 0001:0001e1ce       ?qt_metacast@QDialogButtonBox@@UAEPAXPBD@Z 1001f1ce f   Qt5Widgets:Qt5Widgets.dll
 0001:0001e1d4       ?qt_metacast@QGridLayout@@UAEPAXPBD@Z 1001f1d4 f   Qt5Widgets:Qt5Widgets.dll
 0001:0001e1da       ?qt_metacast@QGroupBox@@UAEPAXPBD@Z 1001f1da f   Qt5Widgets:Qt5Widgets.dll
 0001:0001e1e0       ?qt_metacast@QHBoxLayout@@UAEPAXPBD@Z 1001f1e0 f   Qt5Widgets:Qt5Widgets.dll
 0001:0001e1e6       ?qt_metacast@QLabel@@UAEPAXPBD@Z 1001f1e6 f   Qt5Widgets:Qt5Widgets.dll
 0001:0001e1ec       ?qt_metacast@QPushButton@@UAEPAXPBD@Z 1001f1ec f   Qt5Widgets:Qt5Widgets.dll
 0001:0001e1f2       ?qt_metacast@QRadioButton@@UAEPAXPBD@Z 1001f1f2 f   Qt5Widgets:Qt5Widgets.dll
 0001:0001e1f8       ?qt_metacast@QSpinBox@@UAEPAXPBD@Z 1001f1f8 f   Qt5Widgets:Qt5Widgets.dll
 0001:0001e1fe       ?qt_metacast@QTabWidget@@UAEPAXPBD@Z 1001f1fe f   Qt5Widgets:Qt5Widgets.dll
 0001:0001e204       ?qt_metacast@QTextEdit@@UAEPAXPBD@Z 1001f204 f   Qt5Widgets:Qt5Widgets.dll
 0001:0001e20a       ?qt_metacast@QTreeWidget@@UAEPAXPBD@Z 1001f20a f   Qt5Widgets:Qt5Widgets.dll
 0001:0001e210       ?qt_metacast@QVBoxLayout@@UAEPAXPBD@Z 1001f210 f   Qt5Widgets:Qt5Widgets.dll
 0001:0001e216       ?qt_metacast@QWidget@@UAEPAXPBD@Z 1001f216 f   Qt5Widgets:Qt5Widgets.dll
 0001:0001e21c       ?read@QTreeWidgetItem@@UAEXAAVQDataStream@@@Z 1001f21c f   Qt5Widgets:Qt5Widgets.dll
 0001:0001e222       ?redirected@QWidget@@MBEPAVQPaintDevice@@PAVQPoint@@@Z 1001f222 f   Qt5Widgets:Qt5Widgets.dll
 0001:0001e228       ?reset@QTreeView@@UAEXXZ   1001f228 f   Qt5Widgets:Qt5Widgets.dll
 0001:0001e22e       ?resizeEvent@QAbstractItemView@@MAEXPAVQResizeEvent@@@Z 1001f22e f   Qt5Widgets:Qt5Widgets.dll
 0001:0001e234       ?resizeEvent@QAbstractSpinBox@@MAEXPAVQResizeEvent@@@Z 1001f234 f   Qt5Widgets:Qt5Widgets.dll
 0001:0001e23a       ?resizeEvent@QComboBox@@MAEXPAVQResizeEvent@@@Z 1001f23a f   Qt5Widgets:Qt5Widgets.dll
 0001:0001e240       ?resizeEvent@QDialog@@MAEXPAVQResizeEvent@@@Z 1001f240 f   Qt5Widgets:Qt5Widgets.dll
 0001:0001e246       ?resizeEvent@QGroupBox@@MAEXPAVQResizeEvent@@@Z 1001f246 f   Qt5Widgets:Qt5Widgets.dll
 0001:0001e24c       ?resizeEvent@QTabWidget@@MAEXPAVQResizeEvent@@@Z 1001f24c f   Qt5Widgets:Qt5Widgets.dll
 0001:0001e252       ?resizeEvent@QTextEdit@@MAEXPAVQResizeEvent@@@Z 1001f252 f   Qt5Widgets:Qt5Widgets.dll
 0001:0001e258       ?resizeEvent@QWidget@@MAEXPAVQResizeEvent@@@Z 1001f258 f   Qt5Widgets:Qt5Widgets.dll
 0001:0001e25e       ?rowsAboutToBeRemoved@QTreeView@@MAEXABVQModelIndex@@HH@Z 1001f25e f   Qt5Widgets:Qt5Widgets.dll
 0001:0001e264       ?rowsInserted@QTreeView@@MAEXABVQModelIndex@@HH@Z 1001f264 f   Qt5Widgets:Qt5Widgets.dll
 0001:0001e26a       ?scrollContentsBy@QTextEdit@@MAEXHH@Z 1001f26a f   Qt5Widgets:Qt5Widgets.dll
 0001:0001e270       ?scrollContentsBy@QTreeView@@MAEXHH@Z 1001f270 f   Qt5Widgets:Qt5Widgets.dll
 0001:0001e276       ?scrollTo@QTreeView@@UAEXABVQModelIndex@@W4ScrollHint@QAbstractItemView@@@Z 1001f276 f   Qt5Widgets:Qt5Widgets.dll
 0001:0001e27c       ?selectAll@QTreeView@@UAEXXZ 1001f27c f   Qt5Widgets:Qt5Widgets.dll
 0001:0001e282       ?selectedIndexes@QTreeView@@MBE?AV?$QList@VQModelIndex@@@@XZ 1001f282 f   Qt5Widgets:Qt5Widgets.dll
 0001:0001e288       ?selectionChanged@QTreeView@@MAEXABVQItemSelection@@0@Z 1001f288 f   Qt5Widgets:Qt5Widgets.dll
 0001:0001e28e       ?selectionCommand@QAbstractItemView@@MBE?AV?$QFlags@W4SelectionFlag@QItemSelectionModel@@@@ABVQModelIndex@@PBVQEvent@@@Z 1001f28e f   Qt5Widgets:Qt5Widgets.dll
 0001:0001e294       ?setData@QTreeWidgetItem@@UAEXHHABVQVariant@@@Z 1001f294 f   Qt5Widgets:Qt5Widgets.dll
 0001:0001e29a       ?setGeometry@QBoxLayout@@UAEXABVQRect@@@Z 1001f29a f   Qt5Widgets:Qt5Widgets.dll
 0001:0001e2a0       ?setGeometry@QGridLayout@@UAEXABVQRect@@@Z 1001f2a0 f   Qt5Widgets:Qt5Widgets.dll
 0001:0001e2a6       ?setGeometry@QSpacerItem@@UAEXABVQRect@@@Z 1001f2a6 f   Qt5Widgets:Qt5Widgets.dll
 0001:0001e2ac       ?setModel@QTreeWidget@@EAEXPAVQAbstractItemModel@@@Z 1001f2ac f   Qt5Widgets:Qt5Widgets.dll
 0001:0001e2b2       ?setRootIndex@QTreeView@@UAEXABVQModelIndex@@@Z 1001f2b2 f   Qt5Widgets:Qt5Widgets.dll
 0001:0001e2b8       ?setSelection@QTreeView@@MAEXABVQRect@@V?$QFlags@W4SelectionFlag@QItemSelectionModel@@@@@Z 1001f2b8 f   Qt5Widgets:Qt5Widgets.dll
 0001:0001e2be       ?setSelectionModel@QTreeWidget@@UAEXPAVQItemSelectionModel@@@Z 1001f2be f   Qt5Widgets:Qt5Widgets.dll
 0001:0001e2c4       ?setVisible@QDialog@@UAEX_N@Z 1001f2c4 f   Qt5Widgets:Qt5Widgets.dll
 0001:0001e2ca       ?setVisible@QWidget@@UAEX_N@Z 1001f2ca f   Qt5Widgets:Qt5Widgets.dll
 0001:0001e2d0       ?setupViewport@QAbstractScrollArea@@UAEXPAVQWidget@@@Z 1001f2d0 f   Qt5Widgets:Qt5Widgets.dll
 0001:0001e2d6       ?sharedPainter@QWidget@@MBEPAVQPainter@@XZ 1001f2d6 f   Qt5Widgets:Qt5Widgets.dll
 0001:0001e2dc       ?showEvent@QAbstractSpinBox@@MAEXPAVQShowEvent@@@Z 1001f2dc f   Qt5Widgets:Qt5Widgets.dll
 0001:0001e2e2       ?showEvent@QComboBox@@MAEXPAVQShowEvent@@@Z 1001f2e2 f   Qt5Widgets:Qt5Widgets.dll
 0001:0001e2e8       ?showEvent@QDialog@@MAEXPAVQShowEvent@@@Z 1001f2e8 f   Qt5Widgets:Qt5Widgets.dll
 0001:0001e2ee       ?showEvent@QTabWidget@@MAEXPAVQShowEvent@@@Z 1001f2ee f   Qt5Widgets:Qt5Widgets.dll
 0001:0001e2f4       ?showEvent@QTextEdit@@MAEXPAVQShowEvent@@@Z 1001f2f4 f   Qt5Widgets:Qt5Widgets.dll
 0001:0001e2fa       ?showEvent@QWidget@@MAEXPAVQShowEvent@@@Z 1001f2fa f   Qt5Widgets:Qt5Widgets.dll
 0001:0001e300       ?showPopup@QComboBox@@UAEXXZ 1001f300 f   Qt5Widgets:Qt5Widgets.dll
 0001:0001e306       ?sizeHint@QAbstractScrollArea@@UBE?AVQSize@@XZ 1001f306 f   Qt5Widgets:Qt5Widgets.dll
 0001:0001e30c       ?sizeHint@QAbstractSpinBox@@UBE?AVQSize@@XZ 1001f30c f   Qt5Widgets:Qt5Widgets.dll
 0001:0001e312       ?sizeHint@QBoxLayout@@UBE?AVQSize@@XZ 1001f312 f   Qt5Widgets:Qt5Widgets.dll
 0001:0001e318       ?sizeHint@QCheckBox@@UBE?AVQSize@@XZ 1001f318 f   Qt5Widgets:Qt5Widgets.dll
 0001:0001e31e       ?sizeHint@QComboBox@@UBE?AVQSize@@XZ 1001f31e f   Qt5Widgets:Qt5Widgets.dll
 0001:0001e324       ?sizeHint@QDialog@@UBE?AVQSize@@XZ 1001f324 f   Qt5Widgets:Qt5Widgets.dll
 0001:0001e32a       ?sizeHint@QGridLayout@@UBE?AVQSize@@XZ 1001f32a f   Qt5Widgets:Qt5Widgets.dll
 0001:0001e330       ?sizeHint@QLabel@@UBE?AVQSize@@XZ 1001f330 f   Qt5Widgets:Qt5Widgets.dll
 0001:0001e336       ?sizeHint@QPushButton@@UBE?AVQSize@@XZ 1001f336 f   Qt5Widgets:Qt5Widgets.dll
 0001:0001e33c       ?sizeHint@QRadioButton@@UBE?AVQSize@@XZ 1001f33c f   Qt5Widgets:Qt5Widgets.dll
 0001:0001e342       ?sizeHint@QSpacerItem@@UBE?AVQSize@@XZ 1001f342 f   Qt5Widgets:Qt5Widgets.dll
 0001:0001e348       ?sizeHint@QTabWidget@@UBE?AVQSize@@XZ 1001f348 f   Qt5Widgets:Qt5Widgets.dll
 0001:0001e34e       ?sizeHint@QWidget@@UBE?AVQSize@@XZ 1001f34e f   Qt5Widgets:Qt5Widgets.dll
 0001:0001e354       ?sizeHintForColumn@QTreeView@@MBEHH@Z 1001f354 f   Qt5Widgets:Qt5Widgets.dll
 0001:0001e35a       ?sizeHintForRow@QAbstractItemView@@UBEHH@Z 1001f35a f   Qt5Widgets:Qt5Widgets.dll
 0001:0001e360       ?spacerItem@QLayoutItem@@UAEPAVQSpacerItem@@XZ 1001f360 f   Qt5Widgets:Qt5Widgets.dll
 0001:0001e366       ?spacerItem@QSpacerItem@@UAEPAV1@XZ 1001f366 f   Qt5Widgets:Qt5Widgets.dll
 0001:0001e36c       ?startDrag@QAbstractItemView@@MAEXV?$QFlags@W4DropAction@Qt@@@@@Z 1001f36c f   Qt5Widgets:Qt5Widgets.dll
 0001:0001e372       ?stepBy@QAbstractSpinBox@@UAEXH@Z 1001f372 f   Qt5Widgets:Qt5Widgets.dll
 0001:0001e378       ?stepEnabled@QAbstractSpinBox@@MBE?AV?$QFlags@W4StepEnabledFlag@QAbstractSpinBox@@@@XZ 1001f378 f   Qt5Widgets:Qt5Widgets.dll
 0001:0001e37e       ?supportedDropActions@QTreeWidget@@MBE?AV?$QFlags@W4DropAction@Qt@@@@XZ 1001f37e f   Qt5Widgets:Qt5Widgets.dll
 0001:0001e384       ?tabInserted@QTabWidget@@MAEXH@Z 1001f384 f   Qt5Widgets:Qt5Widgets.dll
 0001:0001e38a       ?tabRemoved@QTabWidget@@MAEXH@Z 1001f38a f   Qt5Widgets:Qt5Widgets.dll
 0001:0001e390       ?tabletEvent@QWidget@@MAEXPAVQTabletEvent@@@Z 1001f390 f   Qt5Widgets:Qt5Widgets.dll
 0001:0001e396       ?takeAt@QBoxLayout@@UAEPAVQLayoutItem@@H@Z 1001f396 f   Qt5Widgets:Qt5Widgets.dll
 0001:0001e39c       ?takeAt@QGridLayout@@UAEPAVQLayoutItem@@H@Z 1001f39c f   Qt5Widgets:Qt5Widgets.dll
 0001:0001e3a2       ?textFromValue@QSpinBox@@MBE?AVQString@@H@Z 1001f3a2 f   Qt5Widgets:Qt5Widgets.dll
 0001:0001e3a8       ?timerEvent@QAbstractButton@@MAEXPAVQTimerEvent@@@Z 1001f3a8 f   Qt5Widgets:Qt5Widgets.dll
 0001:0001e3ae       ?timerEvent@QAbstractSpinBox@@MAEXPAVQTimerEvent@@@Z 1001f3ae f   Qt5Widgets:Qt5Widgets.dll
 0001:0001e3b4       ?timerEvent@QTextEdit@@MAEXPAVQTimerEvent@@@Z 1001f3b4 f   Qt5Widgets:Qt5Widgets.dll
 0001:0001e3ba       ?timerEvent@QTreeView@@MAEXPAVQTimerEvent@@@Z 1001f3ba f   Qt5Widgets:Qt5Widgets.dll
 0001:0001e3c0       ?updateEditorData@QAbstractItemView@@MAEXXZ 1001f3c0 f   Qt5Widgets:Qt5Widgets.dll
 0001:0001e3c6       ?updateEditorGeometries@QAbstractItemView@@MAEXXZ 1001f3c6 f   Qt5Widgets:Qt5Widgets.dll
 0001:0001e3cc       ?updateGeometries@QTreeView@@MAEXXZ 1001f3cc f   Qt5Widgets:Qt5Widgets.dll
 0001:0001e3d2       ?validate@QSpinBox@@MBE?AW4State@QValidator@@AAVQString@@AAH@Z 1001f3d2 f   Qt5Widgets:Qt5Widgets.dll
 0001:0001e3d8       ?valueFromText@QSpinBox@@MBEHABVQString@@@Z 1001f3d8 f   Qt5Widgets:Qt5Widgets.dll
 0001:0001e3de       ?verticalOffset@QTreeView@@MBEHXZ 1001f3de f   Qt5Widgets:Qt5Widgets.dll
 0001:0001e3e4       ?verticalScrollbarAction@QAbstractItemView@@MAEXH@Z 1001f3e4 f   Qt5Widgets:Qt5Widgets.dll
 0001:0001e3ea       ?verticalScrollbarValueChanged@QAbstractItemView@@MAEXH@Z 1001f3ea f   Qt5Widgets:Qt5Widgets.dll
 0001:0001e3f0       ?viewOptions@QAbstractItemView@@MBE?AVQStyleOptionViewItem@@XZ 1001f3f0 f   Qt5Widgets:Qt5Widgets.dll
 0001:0001e3f6       ?viewportEvent@QAbstractScrollArea@@MAE_NPAVQEvent@@@Z 1001f3f6 f   Qt5Widgets:Qt5Widgets.dll
 0001:0001e3fc       ?viewportEvent@QTreeView@@MAE_NPAVQEvent@@@Z 1001f3fc f   Qt5Widgets:Qt5Widgets.dll
 0001:0001e402       ?viewportSizeHint@QAbstractScrollArea@@MBE?AVQSize@@XZ 1001f402 f   Qt5Widgets:Qt5Widgets.dll
 0001:0001e408       ?viewportSizeHint@QTreeView@@MBE?AVQSize@@XZ 1001f408 f   Qt5Widgets:Qt5Widgets.dll
 0001:0001e40e       ?visualRect@QTreeView@@UBE?AVQRect@@ABVQModelIndex@@@Z 1001f40e f   Qt5Widgets:Qt5Widgets.dll
 0001:0001e414       ?visualRegionForSelection@QTreeView@@MBE?AVQRegion@@ABVQItemSelection@@@Z 1001f414 f   Qt5Widgets:Qt5Widgets.dll
 0001:0001e41a       ?wheelEvent@QAbstractScrollArea@@MAEXPAVQWheelEvent@@@Z 1001f41a f   Qt5Widgets:Qt5Widgets.dll
 0001:0001e420       ?wheelEvent@QAbstractSpinBox@@MAEXPAVQWheelEvent@@@Z 1001f420 f   Qt5Widgets:Qt5Widgets.dll
 0001:0001e426       ?wheelEvent@QComboBox@@MAEXPAVQWheelEvent@@@Z 1001f426 f   Qt5Widgets:Qt5Widgets.dll
 0001:0001e42c       ?wheelEvent@QTextEdit@@MAEXPAVQWheelEvent@@@Z 1001f42c f   Qt5Widgets:Qt5Widgets.dll
 0001:0001e432       ?wheelEvent@QWidget@@MAEXPAVQWheelEvent@@@Z 1001f432 f   Qt5Widgets:Qt5Widgets.dll
 0001:0001e438       ?widget@QLayoutItem@@UAEPAVQWidget@@XZ 1001f438 f   Qt5Widgets:Qt5Widgets.dll
 0001:0001e43e       ?write@QTreeWidgetItem@@UBEXAAVQDataStream@@@Z 1001f43e f   Qt5Widgets:Qt5Widgets.dll
 0001:0001e444       ?event@QAction@@MAE_NPAVQEvent@@@Z 1001f444 f   Qt5Widgets:Qt5Widgets.dll
 0001:0001e44a       ?destroyEditor@QAbstractItemDelegate@@UBEXPAVQWidget@@ABVQModelIndex@@@Z 1001f44a f   Qt5Widgets:Qt5Widgets.dll
 0001:0001e450       ?drawCheck@QItemDelegate@@MBEXPAVQPainter@@ABVQStyleOptionViewItem@@ABVQRect@@W4CheckState@Qt@@@Z 1001f450 f   Qt5Widgets:Qt5Widgets.dll
 0001:0001e456       ?drawDecoration@QItemDelegate@@MBEXPAVQPainter@@ABVQStyleOptionViewItem@@ABVQRect@@ABVQPixmap@@@Z 1001f456 f   Qt5Widgets:Qt5Widgets.dll
 0001:0001e45c       ?drawDisplay@QItemDelegate@@MBEXPAVQPainter@@ABVQStyleOptionViewItem@@ABVQRect@@ABVQString@@@Z 1001f45c f   Qt5Widgets:Qt5Widgets.dll
 0001:0001e462       ?drawFocus@QItemDelegate@@MBEXPAVQPainter@@ABVQStyleOptionViewItem@@ABVQRect@@@Z 1001f462 f   Qt5Widgets:Qt5Widgets.dll
 0001:0001e468       ?editorEvent@QItemDelegate@@MAE_NPAVQEvent@@PAVQAbstractItemModel@@ABVQStyleOptionViewItem@@ABVQModelIndex@@@Z 1001f468 f   Qt5Widgets:Qt5Widgets.dll
 0001:0001e46e       ?eventFilter@QItemDelegate@@MAE_NPAVQObject@@PAVQEvent@@@Z 1001f46e f   Qt5Widgets:Qt5Widgets.dll
 0001:0001e474       ?helpEvent@QAbstractItemDelegate@@UAE_NPAVQHelpEvent@@PAVQAbstractItemView@@ABVQStyleOptionViewItem@@ABVQModelIndex@@@Z 1001f474 f   Qt5Widgets:Qt5Widgets.dll
 0001:0001e47a       ?paint@QItemDelegate@@UBEXPAVQPainter@@ABVQStyleOptionViewItem@@ABVQModelIndex@@@Z 1001f47a f   Qt5Widgets:Qt5Widgets.dll
 0001:0001e480       ?paintingRoles@QAbstractItemDelegate@@UBE?AV?$QVector@H@@XZ 1001f480 f   Qt5Widgets:Qt5Widgets.dll
 0001:0001e486       ?sizeHint@QItemDelegate@@UBE?AVQSize@@ABVQStyleOptionViewItem@@ABVQModelIndex@@@Z 1001f486 f   Qt5Widgets:Qt5Widgets.dll
 0001:0001e48c       ?updateEditorGeometry@QItemDelegate@@UBEXPAVQWidget@@ABVQStyleOptionViewItem@@ABVQModelIndex@@@Z 1001f48c f   Qt5Widgets:Qt5Widgets.dll
 0001:0001e492       ?qt_metacast@QDialog@@UAEPAXPBD@Z 1001f492 f   Qt5Widgets:Qt5Widgets.dll
 0001:0001e498       ?qt_metacall@QDialog@@UAEHW4Call@QMetaObject@@HPAPAX@Z 1001f498 f   Qt5Widgets:Qt5Widgets.dll
 0001:0001e49e       ??0QKeySequence@@QAE@ABVQString@@W4SequenceFormat@0@@Z 1001f49e f   Qt5Gui:Qt5Gui.dll
 0001:0001e4a4       ??1QKeySequence@@QAE@XZ    1001f4a4 f   Qt5Gui:Qt5Gui.dll
 0001:0001e4aa       ??0QIcon@@QAE@XZ           1001f4aa f   Qt5Gui:Qt5Gui.dll
 0001:0001e4b0       ??1QIcon@@QAE@XZ           1001f4b0 f   Qt5Gui:Qt5Gui.dll
 0001:0001e4b6       ??0QIcon@@QAE@ABVQString@@@Z 1001f4b6 f   Qt5Gui:Qt5Gui.dll
 0001:0001e4bc       ?setRgb@QColor@@QAEXHHHH@Z 1001f4bc f   Qt5Gui:Qt5Gui.dll
 0001:0001e4c2       ?clear@QTextDocument@@UAEXXZ 1001f4c2 f   Qt5Gui:Qt5Gui.dll
 0001:0001e4c8       ?createObject@QTextDocument@@MAEPAVQTextObject@@ABVQTextFormat@@@Z 1001f4c8 f   Qt5Gui:Qt5Gui.dll
 0001:0001e4ce       ?loadResource@QTextDocument@@MAE?AVQVariant@@HABVQUrl@@@Z 1001f4ce f   Qt5Gui:Qt5Gui.dll
 0001:0001e4d4       ??0QScriptValue@@QAE@XZ    1001f4d4 f   Qt5Script:Qt5Script.dll
 0001:0001e4da       ??1QScriptValue@@QAE@XZ    1001f4da f   Qt5Script:Qt5Script.dll
 0001:0001e4e0       ??0QScriptValue@@QAE@ABV0@@Z 1001f4e0 f   Qt5Script:Qt5Script.dll
 0001:0001e4e6       ??4QScriptValue@@QAEAAV0@ABV0@@Z 1001f4e6 f   Qt5Script:Qt5Script.dll
 0001:0001e4ec       ?isNumber@QScriptValue@@QBE_NXZ 1001f4ec f   Qt5Script:Qt5Script.dll
 0001:0001e4f2       ?isString@QScriptValue@@QBE_NXZ 1001f4f2 f   Qt5Script:Qt5Script.dll
 0001:0001e4f8       ?toString@QScriptValue@@QBE?AVQString@@XZ 1001f4f8 f   Qt5Script:Qt5Script.dll
 0001:0001e4fe       ?toInt32@QScriptValue@@QBEHXZ 1001f4fe f   Qt5Script:Qt5Script.dll
 0001:0001e504       ??1QScriptEngine@@UAE@XZ   1001f504 f   Qt5Script:Qt5Script.dll
 0001:0001e50a       ?newVariant@QScriptEngine@@QAE?AVQScriptValue@@ABVQVariant@@@Z 1001f50a f   Qt5Script:Qt5Script.dll
 0001:0001e510       ?attribute@QDomElement@@QBE?AVQString@@ABV2@0@Z 1001f510 f   Qt5Xml:Qt5Xml.dll
 0001:0001e516       ??1QByteArray@@QAE@XZ      1001f516 f   Qt5Core:Qt5Core.dll
 0001:0001e51c       ?detach@QListData@@QAEPAUData@1@H@Z 1001f51c f   Qt5Core:Qt5Core.dll
 0001:0001e522       ?dispose@QListData@@SAXPAUData@1@@Z 1001f522 f   Qt5Core:Qt5Core.dll
 0001:0001e528       ?cast@QMetaObject@@QBEPAVQObject@@PAV2@@Z 1001f528 f   Qt5Core:Qt5Core.dll
 0001:0001e52e       ?tr@QMetaObject@@QBE?AVQString@@PBD0H@Z 1001f52e f   Qt5Core:Qt5Core.dll
 0001:0001e534       ?normalizedType@QMetaObject@@SA?AVQByteArray@@PBD@Z 1001f534 f   Qt5Core:Qt5Core.dll
 0001:0001e53a       ?connectSlotsByName@QMetaObject@@SAXPAVQObject@@@Z 1001f53a f   Qt5Core:Qt5Core.dll
 0001:0001e540       ??1Connection@QMetaObject@@QAE@XZ 1001f540 f   Qt5Core:Qt5Core.dll
 0001:0001e546       ?registerNormalizedType@QMetaType@@SAHABVQByteArray@@P6AXPAX@ZP6APAXPBX@Z2P6APAX13@ZHV?$QFlags@W4TypeFlag@QMetaType@@@@PBUQMetaObject@@@Z 1001f546 f   Qt5Core:Qt5Core.dll
 0001:0001e54c       ?registerNormalizedTypedef@QMetaType@@SAHABVQByteArray@@H@Z 1001f54c f   Qt5Core:Qt5Core.dll
 0001:0001e552       ?typeFlags@QMetaType@@SA?AV?$QFlags@W4TypeFlag@QMetaType@@@@H@Z 1001f552 f   Qt5Core:Qt5Core.dll
 0001:0001e558       ?freeNodeAndRebalance@QMapDataBase@@QAEXPAUQMapNodeBase@@@Z 1001f558 f   Qt5Core:Qt5Core.dll
 0001:0001e55e       ?recalcMostLeftNode@QMapDataBase@@QAEXXZ 1001f55e f   Qt5Core:Qt5Core.dll
 0001:0001e564       ?createNode@QMapDataBase@@QAEPAUQMapNodeBase@@HHPAU2@_N@Z 1001f564 f   Qt5Core:Qt5Core.dll
 0001:0001e56a       ?freeTree@QMapDataBase@@QAEXPAUQMapNodeBase@@H@Z 1001f56a f   Qt5Core:Qt5Core.dll
 0001:0001e570       ?createData@QMapDataBase@@SAPAU1@XZ 1001f570 f   Qt5Core:Qt5Core.dll
 0001:0001e576       ?freeData@QMapDataBase@@SAXPAU1@@Z 1001f576 f   Qt5Core:Qt5Core.dll
 0001:0001e57c       ??0QChar@@QAE@UQLatin1Char@@@Z 1001f57c f   Qt5Core:Qt5Core.dll
 0001:0001e582       ??0QString@@QAE@XZ         1001f582 f   Qt5Core:Qt5Core.dll
 0001:0001e588       ??0QString@@QAE@ABV0@@Z    1001f588 f   Qt5Core:Qt5Core.dll
 0001:0001e58e       ??1QString@@QAE@XZ         1001f58e f   Qt5Core:Qt5Core.dll
 0001:0001e594       ??4QString@@QAEAAV0@ABV0@@Z 1001f594 f   Qt5Core:Qt5Core.dll
 0001:0001e59a       ??4QString@@QAEAAV0@$$QAV0@@Z 1001f59a f   Qt5Core:Qt5Core.dll
 0001:0001e5a0       ?arg@QString@@QBE?AV1@_JHHVQChar@@@Z 1001f5a0 f   Qt5Core:Qt5Core.dll
 0001:0001e5a6       ?arg@QString@@QBE?AV1@HHHVQChar@@@Z 1001f5a6 f   Qt5Core:Qt5Core.dll
 0001:0001e5ac       ?arg@QString@@QBE?AV1@ABV1@HVQChar@@@Z 1001f5ac f   Qt5Core:Qt5Core.dll
 0001:0001e5b2       ?append@QString@@QAEAAV1@VQChar@@@Z 1001f5b2 f   Qt5Core:Qt5Core.dll
 0001:0001e5b8       ?append@QString@@QAEAAV1@ABV1@@Z 1001f5b8 f   Qt5Core:Qt5Core.dll
 0001:0001e5be       ?fromUtf8@QString@@SA?AV1@PBDH@Z 1001f5be f   Qt5Core:Qt5Core.dll
 0001:0001e5c4       ?number@QString@@SA?AV1@_JH@Z 1001f5c4 f   Qt5Core:Qt5Core.dll
 0001:0001e5ca       ??8@YA_NABVQString@@0@Z    1001f5ca f   Qt5Core:Qt5Core.dll
 0001:0001e5d0       ??M@YA_NABVQString@@0@Z    1001f5d0 f   Qt5Core:Qt5Core.dll
 0001:0001e5d6       ?fromAscii_helper@QString@@CAPAU?$QTypedArrayData@G@@PBDH@Z 1001f5d6 f   Qt5Core:Qt5Core.dll
 0001:0001e5dc       ?objectName@QObject@@QBE?AVQString@@XZ 1001f5dc f   Qt5Core:Qt5Core.dll
 0001:0001e5e2       ?setObjectName@QObject@@QAEXABVQString@@@Z 1001f5e2 f   Qt5Core:Qt5Core.dll
 0001:0001e5e8       ?installEventFilter@QObject@@QAEXPAV1@@Z 1001f5e8 f   Qt5Core:Qt5Core.dll
 0001:0001e5ee       ?connect@QObject@@SA?AVConnection@QMetaObject@@PBV1@PBD01W4ConnectionType@Qt@@@Z 1001f5ee f   Qt5Core:Qt5Core.dll
 0001:0001e5f4       ?connect@QObject@@QBE?AVConnection@QMetaObject@@PBV1@PBD1W4ConnectionType@Qt@@@Z 1001f5f4 f   Qt5Core:Qt5Core.dll
 0001:0001e5fa       ?sender@QObject@@IBEPAV1@XZ 1001f5fa f   Qt5Core:Qt5Core.dll
 0001:0001e600       ??1QVariant@@QAE@XZ        1001f600 f   Qt5Core:Qt5Core.dll
 0001:0001e606       ??0QVariant@@QAE@HPBXI@Z   1001f606 f   Qt5Core:Qt5Core.dll
 0001:0001e60c       ?userType@QVariant@@QBEHXZ 1001f60c f   Qt5Core:Qt5Core.dll
 0001:0001e612       ?constData@QVariant@@QBEPBXXZ 1001f612 f   Qt5Core:Qt5Core.dll
 0001:0001e618       ?convert@QVariant@@QBE_NHPAX@Z 1001f618 f   Qt5Core:Qt5Core.dll
 0001:0001e61e       ?translate@QCoreApplication@@SA?AVQString@@PBD00H@Z 1001f61e f   Qt5Core:Qt5Core.dll
 0001:0001e624       ??0QTimer@@QAE@PAVQObject@@@Z 1001f624 f   Qt5Core:Qt5Core.dll
 0001:0001e62a       ??1QTimer@@UAE@XZ          1001f62a f   Qt5Core:Qt5Core.dll
 0001:0001e630       ?start@QTimer@@QAEXH@Z     1001f630 f   Qt5Core:Qt5Core.dll
 0001:0001e636       ?stop@QTimer@@QAEXXZ       1001f636 f   Qt5Core:Qt5Core.dll
 0001:0001e63c       ?childEvent@QObject@@MAEXPAVQChildEvent@@@Z 1001f63c f   Qt5Core:Qt5Core.dll
 0001:0001e642       ?connectNotify@QObject@@MAEXABVQMetaMethod@@@Z 1001f642 f   Qt5Core:Qt5Core.dll
 0001:0001e648       ?customEvent@QObject@@MAEXPAVQEvent@@@Z 1001f648 f   Qt5Core:Qt5Core.dll
 0001:0001e64e       ?disconnectNotify@QObject@@MAEXABVQMetaMethod@@@Z 1001f64e f   Qt5Core:Qt5Core.dll
 0001:0001e654       ?event@QObject@@UAE_NPAVQEvent@@@Z 1001f654 f   Qt5Core:Qt5Core.dll
 0001:0001e65a       ?eventFilter@QObject@@UAE_NPAV1@PAVQEvent@@@Z 1001f65a f   Qt5Core:Qt5Core.dll
 0001:0001e660       ?metaObject@QTimer@@UBEPBUQMetaObject@@XZ 1001f660 f   Qt5Core:Qt5Core.dll
 0001:0001e666       ?qt_metacall@QTimer@@UAEHW4Call@QMetaObject@@HPAPAX@Z 1001f666 f   Qt5Core:Qt5Core.dll
 0001:0001e66c       ?qt_metacast@QTimer@@UAEPAXPBD@Z 1001f66c f   Qt5Core:Qt5Core.dll
 0001:0001e672       ?timerEvent@QObject@@MAEXPAVQTimerEvent@@@Z 1001f672 f   Qt5Core:Qt5Core.dll
 0001:0001e678       ?timerEvent@QTimer@@MAEXPAVQTimerEvent@@@Z 1001f678 f   Qt5Core:Qt5Core.dll
 0001:0001e67e       ?data@QArrayData@@QAEPAXXZ 1001f67e f   Qt5Core:Qt5Core.dll
 0001:0001e684       ?deallocate@QArrayData@@SAXPAU1@II@Z 1001f684 f   Qt5Core:Qt5Core.dll
 0001:0001e68a       ?detach_grow@QListData@@QAEPAUData@1@PAHH@Z 1001f68a f   Qt5Core:Qt5Core.dll
 0001:0001e690       ?append@QListData@@QAEPAPAXXZ 1001f690 f   Qt5Core:Qt5Core.dll
 0001:0001e696       ??0QObject@@QAE@PAV0@@Z    1001f696 f   Qt5Core:Qt5Core.dll
 0001:0001e69c       ??1QObject@@UAE@XZ         1001f69c f   Qt5Core:Qt5Core.dll
 0001:0001e6a2       ?getAndRef@ExternalRefCountData@QtSharedPointer@@SAPAU12@PBVQObject@@@Z 1001f6a2 f   Qt5Core:Qt5Core.dll
 0001:0001e6a8       ?metaObject@QObject@@UBEPBUQMetaObject@@XZ 1001f6a8 f   Qt5Core:Qt5Core.dll
 0001:0001e6ae       ?qt_metacall@QObject@@UAEHW4Call@QMetaObject@@HPAPAX@Z 1001f6ae f   Qt5Core:Qt5Core.dll
 0001:0001e6b4       ?qt_metacast@QObject@@UAEPAXPBD@Z 1001f6b4 f   Qt5Core:Qt5Core.dll
 0001:0001e6ba       ??0QVariant@@QAE@XZ        1001f6ba f   Qt5Core:Qt5Core.dll
 0001:0001e6c0       ??0QVariant@@QAE@H@Z       1001f6c0 f   Qt5Core:Qt5Core.dll
 0001:0001e6c6       ??0QVariant@@QAE@_N@Z      1001f6c6 f   Qt5Core:Qt5Core.dll
 0001:0001e6cc       ??0QVariant@@QAE@PBD@Z     1001f6cc f   Qt5Core:Qt5Core.dll
 0001:0001e6d2       ??0QVariant@@QAE@ABVQString@@@Z 1001f6d2 f   Qt5Core:Qt5Core.dll
 0001:0001e6d8       ?toInt@QVariant@@QBEHPA_N@Z 1001f6d8 f   Qt5Core:Qt5Core.dll
 0001:0001e6de       ?toBool@QVariant@@QBE_NXZ  1001f6de f   Qt5Core:Qt5Core.dll
 0001:0001e6e4       ?toString@QVariant@@QBE?AVQString@@XZ 1001f6e4 f   Qt5Core:Qt5Core.dll
 0001:0001e6ea       ?qBadAlloc@@YAXXZ          1001f6ea f   Qt5Core:Qt5Core.dll
 0001:0001e6f0       ?allocate@QArrayData@@SAPAU1@IIIV?$QFlags@W4AllocationOption@QArrayData@@@@@Z 1001f6f0 f   Qt5Core:Qt5Core.dll
 0001:0001e6f6       ??4QString@@QAEAAV0@VQChar@@@Z 1001f6f6 f   Qt5Core:Qt5Core.dll
 0001:0001e6fc       ?split@QString@@QBE?AVQStringList@@ABVQRegExp@@W4SplitBehavior@1@@Z 1001f6fc f   Qt5Core:Qt5Core.dll
 0001:0001e702       ?toInt@QString@@QBEHPA_NH@Z 1001f702 f   Qt5Core:Qt5Core.dll
 0001:0001e708       ??8QString@@QBE_NPBD@Z     1001f708 f   Qt5Core:Qt5Core.dll
 0001:0001e70e       ??0QRegExp@@QAE@ABVQString@@W4CaseSensitivity@Qt@@W4PatternSyntax@0@@Z 1001f70e f   Qt5Core:Qt5Core.dll
 0001:0001e714       ??1QRegExp@@QAE@XZ         1001f714 f   Qt5Core:Qt5Core.dll
 0001:0001e71a       ?data@QArrayData@@QBEPBXXZ 1001f71a f   Qt5Core:Qt5Core.dll
 0001:0001e720       ??0QString@@QAE@$$QAV0@@Z  1001f720 f   Qt5Core:Qt5Core.dll
 0001:0001e726       ?append@QListData@@QAEPAPAXABU1@@Z 1001f726 f   Qt5Core:Qt5Core.dll
 0001:0001e72c       ??0QVariant@@QAE@ABV0@@Z   1001f72c f   Qt5Core:Qt5Core.dll
 0001:0001e732       ??4QVariant@@QAEAAV0@ABV0@@Z 1001f732 f   Qt5Core:Qt5Core.dll
 0001:0001e738       ??4QVariant@@QAEAAV0@$$QAV0@@Z 1001f738 f   Qt5Core:Qt5Core.dll
 0001:0001e73e       ?startsWith@QString@@QBE_NABV1@W4CaseSensitivity@Qt@@@Z 1001f73e f   Qt5Core:Qt5Core.dll
 0001:0001e744       ?toLower@QString@@QBE?AV1@XZ 1001f744 f   Qt5Core:Qt5Core.dll
 0001:0001e74a       ??4QString@@QAEAAV0@PBD@Z  1001f74a f   Qt5Core:Qt5Core.dll
 0001:0001e750       ?realloc@QListData@@QAEXH@Z 1001f750 f   Qt5Core:Qt5Core.dll
 0001:0001e756       ?nextNode@QMapNodeBase@@QBEPBU1@XZ 1001f756 f   Qt5Core:Qt5Core.dll
 0001:0001e75c       ?toMap@QVariant@@QBE?AV?$QMap@VQString@@VQVariant@@@@XZ 1001f75c f   Qt5Core:Qt5Core.dll
 0001:0001e762       ??0QByteArray@@QAE@XZ      1001f762 f   Qt5Core:Qt5Core.dll
 0001:0001e768       ?reserve@QByteArray@@QAEXH@Z 1001f768 f   Qt5Core:Qt5Core.dll
 0001:0001e76e       ?append@QByteArray@@QAEAAV1@D@Z 1001f76e f   Qt5Core:Qt5Core.dll
 0001:0001e774       ?append@QByteArray@@QAEAAV1@PBD@Z 1001f774 f   Qt5Core:Qt5Core.dll
 0001:0001e77a       ?className@QMetaObject@@QBEPBDXZ 1001f77a f   Qt5Core:Qt5Core.dll
 0001:0001e780       ?dynamicMetaObject@QObjectData@@QBEPAUQMetaObject@@XZ 1001f780 f   Qt5Core:Qt5Core.dll
 0001:0001e786       ?qRegisterResourceData@@YA_NHPBE00@Z 1001f786 f   Qt5Core:Qt5Core.dll
 0001:0001e78c       ?qUnregisterResourceData@@YA_NHPBE00@Z 1001f78c f   Qt5Core:Qt5Core.dll
 0001:0001e792       ?_Xbad_alloc@std@@YAXXZ    1001f792 f   msvcprt:MSVCP120.dll
 0001:0001e798       ?_Xlength_error@std@@YAXPBD@Z 1001f798 f   msvcprt:MSVCP120.dll
 0001:0001e79e       ?_Xout_of_range@std@@YAXPBD@Z 1001f79e f   msvcprt:MSVCP120.dll
 0001:0001e7a4       ?_Syserror_map@std@@YAPBDH@Z 1001f7a4 f   msvcprt:MSVCP120.dll
 0001:0001e7aa       ?_Winerror_map@std@@YAPBDH@Z 1001f7aa f   msvcprt:MSVCP120.dll
 0001:0001e7b0       __purecall                 1001f7b0 f   MSVCRT:MSVCR120.dll
 0001:0001e7b6       ??2@YAPAXI@Z               1001f7b6 f   MSVCRT:MSVCR120.dll
 0001:0001e7bc       ??3@YAXPAX@Z               1001f7bc f   MSVCRT:MSVCR120.dll
 0001:0001e7c2       ___atonexitinit            1001f7c2 f   MSVCRT:atonexit.obj
 0001:0001e7fe       __onexit                   1001f7fe f   MSVCRT:atonexit.obj
 0001:0001e8a7       _atexit                    1001f8a7 f   MSVCRT:atonexit.obj
 0001:0001e8bc       _memmove                   1001f8bc f   MSVCRT:MSVCR120.dll
 0001:0001e8c2       __hypot                    1001f8c2 f   MSVCRT:MSVCR120.dll
 0001:0001e8c8       @__security_check_cookie@4 1001f8c8 f   MSVCRT:secchk.obj
 0001:0001e8d8       __CxxThrowException@8      1001f8d8 f   MSVCRT:MSVCR120.dll
 0001:0001e8de       ___CxxFrameHandler3        1001f8de f   MSVCRT:MSVCR120.dll
 0001:0001e8e4       _memcpy                    1001f8e4 f   MSVCRT:MSVCR120.dll
 0001:0001e8ea       ??0type_info@@AAE@ABV0@@Z  1001f8ea f   MSVCRT:ti_inst.obj
 0001:0001e8f5       ??4type_info@@AAEAAV0@ABV0@@Z 1001f8f5 f   MSVCRT:ti_inst.obj
 0001:0001e8fa       ??_Etype_info@@UAEPAXI@Z   1001f8fa f i MSVCRT:ti_inst.obj
 0001:0001e950       _memset                    1001f950 f   MSVCRT:MSVCR120.dll
 0001:0001e9a2       _NtCurrentTeb              1001f9a2 f i MSVCRT:crtdll.obj
 0001:0001e9a9       __CRT_INIT@12              1001f9a9 f   MSVCRT:crtdll.obj
 0001:0001eba0       __DllMainCRTStartup@12     1001fba0 f   MSVCRT:crtdll.obj
 0001:0001ecf6       __lock                     1001fcf6 f   MSVCRT:MSVCR120.dll
 0001:0001ecfc       __unlock                   1001fcfc f   MSVCRT:MSVCR120.dll
 0001:0001ed02       __calloc_crt               1001fd02 f   MSVCRT:MSVCR120.dll
 0001:0001ed08       ___dllonexit               1001fd08 f   MSVCRT:MSVCR120.dll
 0001:0001ed10       __SEH_prolog4              1001fd10 f   MSVCRT:sehprolg4.obj
 0001:0001ed55       __SEH_epilog4              1001fd55 f   MSVCRT:sehprolg4.obj
 0001:0001ed69       __except_handler4          1001fd69 f   MSVCRT:chandler4gs.obj
 0001:0001ed8c       ___raise_securityfailure   1001fd8c f   MSVCRT:gs_report.obj
 0001:0001edc9       ___report_gsfailure        1001fdc9 f   MSVCRT:gs_report.obj
 0001:0001eec4       ___report_rangecheckfailure 1001fec4 f   MSVCRT:gs_report.obj
 0001:0001eed0       ___report_securityfailure  1001fed0 f   MSVCRT:gs_report.obj
 0001:0001efa0       ___report_securityfailureEx 1001ffa0 f   MSVCRT:gs_report.obj
 0001:0001f0b6       ??_M@YGXPAXIHP6EX0@Z@Z     100200b6 f   MSVCRT:ehvecdtr.obj
 0001:0001f13e       ?__ArrayUnwind@@YGXPAXIHP6EX0@Z@Z 1002013e f   MSVCRT:ehvecdtr.obj
 0001:0001f19c       ??1type_info@@UAE@XZ       1002019c f   MSVCRT:MSVCR120.dll
 0001:0001f1a2       ___CppXcptFilter           100201a2 f   MSVCRT:MSVCR120.dll
 0001:0001f1a8       __amsg_exit                100201a8 f   MSVCRT:MSVCR120.dll
 0001:0001f1b0       __FindPESection            100201b0 f   MSVCRT:pesect.obj
 0001:0001f200       __IsNonwritableInCurrentImage 10020200 f   MSVCRT:pesect.obj
 0001:0001f2c0       __ValidateImageBase        100202c0 f   MSVCRT:pesect.obj
 0001:0001f2f2       _free                      100202f2 f   MSVCRT:MSVCR120.dll
 0001:0001f2f8       ___security_init_cookie    100202f8 f   MSVCRT:gs_support.obj
 0001:0001f394       _DllMain@12                10020394 f   MSVCRT:dllmain.obj
 0001:0001f3b6       __malloc_crt               100203b6 f   MSVCRT:MSVCR120.dll
 0001:0001f3bc       __RTC_Initialize           100203bc f   MSVCRT:initsect.obj
 0001:0001f3dc       __RTC_Terminate            100203dc f   MSVCRT:initsect.obj
 0001:0001f3fc       __initterm                 100203fc f   MSVCRT:MSVCR120.dll
 0001:0001f402       __initterm_e               10020402 f   MSVCRT:MSVCR120.dll
 0001:0001f408       ___clean_type_info_names   10020408 f   MSVCRT:tncleanup.obj
 0001:0001f414       __except_handler4_common   10020414 f   MSVCRT:MSVCR120.dll
 0001:0001f41a       __crt_debugger_hook        1002041a f   MSVCRT:MSVCR120.dll
 0001:0001f420       ___crtUnhandledException   10020420 f   MSVCRT:MSVCR120.dll
 0001:0001f426       ___crtTerminateProcess     10020426 f   MSVCRT:MSVCR120.dll
 0001:0001f42c       ?terminate@@YAXXZ          1002042c f   MSVCRT:MSVCR120.dll
 0001:0001f432       ___clean_type_info_names_internal 10020432 f   MSVCRT:MSVCR120.dll
 0001:0001f438       _EncodePointer@4           10020438 f   kernel32:KERNEL32.dll
 0001:0001f43e       _DecodePointer@4           1002043e f   kernel32:KERNEL32.dll
 0001:0001f444       _IsDebuggerPresent@0       10020444 f   kernel32:KERNEL32.dll
 0001:0001f44a       _IsProcessorFeaturePresent@4 1002044a f   kernel32:KERNEL32.dll
 0001:0001f450       _QueryPerformanceCounter@4 10020450 f   kernel32:KERNEL32.dll
 0001:0001f456       _GetCurrentProcessId@0     10020456 f   kernel32:KERNEL32.dll
 0001:0001f45c       _GetCurrentThreadId@0      1002045c f   kernel32:KERNEL32.dll
 0001:0001f462       _GetSystemTimeAsFileTime@4 10020462 f   kernel32:KERNEL32.dll
 0001:0001f468       _DisableThreadLibraryCalls@4 10020468 f   kernel32:KERNEL32.dll
 0002:00000000       __imp__DisableThreadLibraryCalls@4 10026000     kernel32:KERNEL32.dll
 0002:00000004       __imp__GetSystemTimeAsFileTime@4 10026004     kernel32:KERNEL32.dll
 0002:00000008       __imp__GetCurrentThreadId@0 10026008     kernel32:KERNEL32.dll
 0002:0000000c       __imp__GetCurrentProcessId@0 1002600c     kernel32:KERNEL32.dll
 0002:00000010       __imp__QueryPerformanceCounter@4 10026010     kernel32:KERNEL32.dll
 0002:00000014       __imp__IsProcessorFeaturePresent@4 10026014     kernel32:KERNEL32.dll
 0002:00000018       __imp__IsDebuggerPresent@0 10026018     kernel32:KERNEL32.dll
 0002:0000001c       __imp__DecodePointer@4     1002601c     kernel32:KERNEL32.dll
 0002:00000020       __imp__EncodePointer@4     10026020     kernel32:KERNEL32.dll
 0002:00000024       \177KERNEL32_NULL_THUNK_DATA 10026024     kernel32:KERNEL32.dll
 0002:00000028       __imp_?_Xlength_error@std@@YAXPBD@Z 10026028     msvcprt:MSVCP120.dll
 0002:0000002c       __imp_?_Xout_of_range@std@@YAXPBD@Z 1002602c     msvcprt:MSVCP120.dll
 0002:00000030       __imp_?_Syserror_map@std@@YAPBDH@Z 10026030     msvcprt:MSVCP120.dll
 0002:00000034       __imp_?_Winerror_map@std@@YAPBDH@Z 10026034     msvcprt:MSVCP120.dll
 0002:00000038       __imp_?_Xbad_alloc@std@@YAXXZ 10026038     msvcprt:MSVCP120.dll
 0002:0000003c       \177MSVCP120_NULL_THUNK_DATA 1002603c     msvcprt:MSVCP120.dll
 0002:00000040       __imp___initterm_e         10026040     MSVCRT:MSVCR120.dll
 0002:00000044       __imp___initterm           10026044     MSVCRT:MSVCR120.dll
 0002:00000048       __imp___malloc_crt         10026048     MSVCRT:MSVCR120.dll
 0002:0000004c       __imp__free                1002604c     MSVCRT:MSVCR120.dll
 0002:00000050       __imp___amsg_exit          10026050     MSVCRT:MSVCR120.dll
 0002:00000054       __imp___except_handler4_common 10026054     MSVCRT:MSVCR120.dll
 0002:00000058       __imp_??1type_info@@UAE@XZ 10026058     MSVCRT:MSVCR120.dll
 0002:0000005c       __imp___onexit             1002605c     MSVCRT:MSVCR120.dll
 0002:00000060       __imp____dllonexit         10026060     MSVCRT:MSVCR120.dll
 0002:00000064       __imp___calloc_crt         10026064     MSVCRT:MSVCR120.dll
 0002:00000068       __imp___unlock             10026068     MSVCRT:MSVCR120.dll
 0002:0000006c       __imp___lock               1002606c     MSVCRT:MSVCR120.dll
 0002:00000070       __imp__memset              10026070     MSVCRT:MSVCR120.dll
 0002:00000074       __imp__memcpy              10026074     MSVCRT:MSVCR120.dll
 0002:00000078       __imp____CxxFrameHandler3  10026078     MSVCRT:MSVCR120.dll
 0002:0000007c       __imp___CxxThrowException@8 1002607c     MSVCRT:MSVCR120.dll
 0002:00000080       __imp___hypot              10026080     MSVCRT:MSVCR120.dll
 0002:00000084       __imp__memmove             10026084     MSVCRT:MSVCR120.dll
 0002:00000088       __imp_??3@YAXPAX@Z         10026088     MSVCRT:MSVCR120.dll
 0002:0000008c       __imp_??2@YAPAXI@Z         1002608c     MSVCRT:MSVCR120.dll
 0002:00000090       __imp___purecall           10026090     MSVCRT:MSVCR120.dll
 0002:00000094       __imp___crt_debugger_hook  10026094     MSVCRT:MSVCR120.dll
 0002:00000098       __imp____crtUnhandledException 10026098     MSVCRT:MSVCR120.dll
 0002:0000009c       __imp____crtTerminateProcess 1002609c     MSVCRT:MSVCR120.dll
 0002:000000a0       __imp_?terminate@@YAXXZ    100260a0     MSVCRT:MSVCR120.dll
 0002:000000a4       __imp____clean_type_info_names_internal 100260a4     MSVCRT:MSVCR120.dll
 0002:000000a8       __imp____CppXcptFilter     100260a8     MSVCRT:MSVCR120.dll
 0002:000000ac       \177MSVCR120_NULL_THUNK_DATA 100260ac     MSVCRT:MSVCR120.dll
 0002:000000b0       __imp_?qUnregisterResourceData@@YA_NHPBE00@Z 100260b0     Qt5Core:Qt5Core.dll
 0002:000000b4       __imp_?qRegisterResourceData@@YA_NHPBE00@Z 100260b4     Qt5Core:Qt5Core.dll
 0002:000000b8       __imp_?dynamicMetaObject@QObjectData@@QBEPAUQMetaObject@@XZ 100260b8     Qt5Core:Qt5Core.dll
 0002:000000bc       __imp_?className@QMetaObject@@QBEPBDXZ 100260bc     Qt5Core:Qt5Core.dll
 0002:000000c0       __imp_?append@QByteArray@@QAEAAV1@PBD@Z 100260c0     Qt5Core:Qt5Core.dll
 0002:000000c4       __imp_?append@QByteArray@@QAEAAV1@D@Z 100260c4     Qt5Core:Qt5Core.dll
 0002:000000c8       __imp_?reserve@QByteArray@@QAEXH@Z 100260c8     Qt5Core:Qt5Core.dll
 0002:000000cc       __imp_??0QByteArray@@QAE@XZ 100260cc     Qt5Core:Qt5Core.dll
 0002:000000d0       __imp_?toMap@QVariant@@QBE?AV?$QMap@VQString@@VQVariant@@@@XZ 100260d0     Qt5Core:Qt5Core.dll
 0002:000000d4       __imp_?nextNode@QMapNodeBase@@QBEPBU1@XZ 100260d4     Qt5Core:Qt5Core.dll
 0002:000000d8       __imp_?realloc@QListData@@QAEXH@Z 100260d8     Qt5Core:Qt5Core.dll
 0002:000000dc       __imp_??4QString@@QAEAAV0@PBD@Z 100260dc     Qt5Core:Qt5Core.dll
 0002:000000e0       __imp_?toLower@QString@@QBE?AV1@XZ 100260e0     Qt5Core:Qt5Core.dll
 0002:000000e4       __imp_?startsWith@QString@@QBE_NABV1@W4CaseSensitivity@Qt@@@Z 100260e4     Qt5Core:Qt5Core.dll
 0002:000000e8       __imp_?shared_null@QMapDataBase@@2U1@B 100260e8     Qt5Core:Qt5Core.dll
 0002:000000ec       __imp_??4QVariant@@QAEAAV0@$$QAV0@@Z 100260ec     Qt5Core:Qt5Core.dll
 0002:000000f0       __imp_??4QVariant@@QAEAAV0@ABV0@@Z 100260f0     Qt5Core:Qt5Core.dll
 0002:000000f4       __imp_??0QVariant@@QAE@ABV0@@Z 100260f4     Qt5Core:Qt5Core.dll
 0002:000000f8       __imp_?append@QListData@@QAEPAPAXABU1@@Z 100260f8     Qt5Core:Qt5Core.dll
 0002:000000fc       __imp_??0QString@@QAE@$$QAV0@@Z 100260fc     Qt5Core:Qt5Core.dll
 0002:00000100       __imp_?data@QArrayData@@QBEPBXXZ 10026100     Qt5Core:Qt5Core.dll
 0002:00000104       __imp_??1QRegExp@@QAE@XZ   10026104     Qt5Core:Qt5Core.dll
 0002:00000108       __imp_??0QRegExp@@QAE@ABVQString@@W4CaseSensitivity@Qt@@W4PatternSyntax@0@@Z 10026108     Qt5Core:Qt5Core.dll
 0002:0000010c       __imp_??8QString@@QBE_NPBD@Z 1002610c     Qt5Core:Qt5Core.dll
 0002:00000110       __imp_?toInt@QString@@QBEHPA_NH@Z 10026110     Qt5Core:Qt5Core.dll
 0002:00000114       __imp_?split@QString@@QBE?AVQStringList@@ABVQRegExp@@W4SplitBehavior@1@@Z 10026114     Qt5Core:Qt5Core.dll
 0002:00000118       __imp_??4QString@@QAEAAV0@VQChar@@@Z 10026118     Qt5Core:Qt5Core.dll
 0002:0000011c       __imp_?allocate@QArrayData@@SAPAU1@IIIV?$QFlags@W4AllocationOption@QArrayData@@@@@Z 1002611c     Qt5Core:Qt5Core.dll
 0002:00000120       __imp_?qBadAlloc@@YAXXZ    10026120     Qt5Core:Qt5Core.dll
 0002:00000124       __imp_?toString@QVariant@@QBE?AVQString@@XZ 10026124     Qt5Core:Qt5Core.dll
 0002:00000128       __imp_?toBool@QVariant@@QBE_NXZ 10026128     Qt5Core:Qt5Core.dll
 0002:0000012c       __imp_?toInt@QVariant@@QBEHPA_N@Z 1002612c     Qt5Core:Qt5Core.dll
 0002:00000130       __imp_??0QVariant@@QAE@ABVQString@@@Z 10026130     Qt5Core:Qt5Core.dll
 0002:00000134       __imp_??0QVariant@@QAE@PBD@Z 10026134     Qt5Core:Qt5Core.dll
 0002:00000138       __imp_??0QVariant@@QAE@_N@Z 10026138     Qt5Core:Qt5Core.dll
 0002:0000013c       __imp_??0QVariant@@QAE@H@Z 1002613c     Qt5Core:Qt5Core.dll
 0002:00000140       __imp_??0QVariant@@QAE@XZ  10026140     Qt5Core:Qt5Core.dll
 0002:00000144       __imp_?shared_null@QArrayData@@2QBU1@B 10026144     Qt5Core:Qt5Core.dll
 0002:00000148       __imp_?qt_metacast@QObject@@UAEPAXPBD@Z 10026148     Qt5Core:Qt5Core.dll
 0002:0000014c       __imp_?qt_metacall@QObject@@UAEHW4Call@QMetaObject@@HPAPAX@Z 1002614c     Qt5Core:Qt5Core.dll
 0002:00000150       __imp_?metaObject@QObject@@UBEPBUQMetaObject@@XZ 10026150     Qt5Core:Qt5Core.dll
 0002:00000154       __imp_?getAndRef@ExternalRefCountData@QtSharedPointer@@SAPAU12@PBVQObject@@@Z 10026154     Qt5Core:Qt5Core.dll
 0002:00000158       __imp_??1QObject@@UAE@XZ   10026158     Qt5Core:Qt5Core.dll
 0002:0000015c       __imp_??0QObject@@QAE@PAV0@@Z 1002615c     Qt5Core:Qt5Core.dll
 0002:00000160       __imp_?append@QListData@@QAEPAPAXXZ 10026160     Qt5Core:Qt5Core.dll
 0002:00000164       __imp_?detach_grow@QListData@@QAEPAUData@1@PAHH@Z 10026164     Qt5Core:Qt5Core.dll
 0002:00000168       __imp_?deallocate@QArrayData@@SAXPAU1@II@Z 10026168     Qt5Core:Qt5Core.dll
 0002:0000016c       __imp_?data@QArrayData@@QAEPAXXZ 1002616c     Qt5Core:Qt5Core.dll
 0002:00000170       __imp_?shared_null@QListData@@2UData@1@B 10026170     Qt5Core:Qt5Core.dll
 0002:00000174       __imp_?timerEvent@QTimer@@MAEXPAVQTimerEvent@@@Z 10026174     Qt5Core:Qt5Core.dll
 0002:00000178       __imp_?timerEvent@QObject@@MAEXPAVQTimerEvent@@@Z 10026178     Qt5Core:Qt5Core.dll
 0002:0000017c       __imp_?qt_metacast@QTimer@@UAEPAXPBD@Z 1002617c     Qt5Core:Qt5Core.dll
 0002:00000180       __imp_?qt_metacall@QTimer@@UAEHW4Call@QMetaObject@@HPAPAX@Z 10026180     Qt5Core:Qt5Core.dll
 0002:00000184       __imp_?metaObject@QTimer@@UBEPBUQMetaObject@@XZ 10026184     Qt5Core:Qt5Core.dll
 0002:00000188       __imp_?eventFilter@QObject@@UAE_NPAV1@PAVQEvent@@@Z 10026188     Qt5Core:Qt5Core.dll
 0002:0000018c       __imp_?event@QObject@@UAE_NPAVQEvent@@@Z 1002618c     Qt5Core:Qt5Core.dll
 0002:00000190       __imp_?disconnectNotify@QObject@@MAEXABVQMetaMethod@@@Z 10026190     Qt5Core:Qt5Core.dll
 0002:00000194       __imp_?customEvent@QObject@@MAEXPAVQEvent@@@Z 10026194     Qt5Core:Qt5Core.dll
 0002:00000198       __imp_?connectNotify@QObject@@MAEXABVQMetaMethod@@@Z 10026198     Qt5Core:Qt5Core.dll
 0002:0000019c       __imp_?childEvent@QObject@@MAEXPAVQChildEvent@@@Z 1002619c     Qt5Core:Qt5Core.dll
 0002:000001a0       __imp_?stop@QTimer@@QAEXXZ 100261a0     Qt5Core:Qt5Core.dll
 0002:000001a4       __imp_?start@QTimer@@QAEXH@Z 100261a4     Qt5Core:Qt5Core.dll
 0002:000001a8       __imp_??1QTimer@@UAE@XZ    100261a8     Qt5Core:Qt5Core.dll
 0002:000001ac       __imp_??0QTimer@@QAE@PAVQObject@@@Z 100261ac     Qt5Core:Qt5Core.dll
 0002:000001b0       __imp_?translate@QCoreApplication@@SA?AVQString@@PBD00H@Z 100261b0     Qt5Core:Qt5Core.dll
 0002:000001b4       __imp_?convert@QVariant@@QBE_NHPAX@Z 100261b4     Qt5Core:Qt5Core.dll
 0002:000001b8       __imp_?constData@QVariant@@QBEPBXXZ 100261b8     Qt5Core:Qt5Core.dll
 0002:000001bc       __imp_?userType@QVariant@@QBEHXZ 100261bc     Qt5Core:Qt5Core.dll
 0002:000001c0       __imp_??0QVariant@@QAE@HPBXI@Z 100261c0     Qt5Core:Qt5Core.dll
 0002:000001c4       __imp_??1QVariant@@QAE@XZ  100261c4     Qt5Core:Qt5Core.dll
 0002:000001c8       __imp_?sender@QObject@@IBEPAV1@XZ 100261c8     Qt5Core:Qt5Core.dll
 0002:000001cc       __imp_?connect@QObject@@QBE?AVConnection@QMetaObject@@PBV1@PBD1W4ConnectionType@Qt@@@Z 100261cc     Qt5Core:Qt5Core.dll
 0002:000001d0       __imp_?connect@QObject@@SA?AVConnection@QMetaObject@@PBV1@PBD01W4ConnectionType@Qt@@@Z 100261d0     Qt5Core:Qt5Core.dll
 0002:000001d4       __imp_?installEventFilter@QObject@@QAEXPAV1@@Z 100261d4     Qt5Core:Qt5Core.dll
 0002:000001d8       __imp_?setObjectName@QObject@@QAEXABVQString@@@Z 100261d8     Qt5Core:Qt5Core.dll
 0002:000001dc       __imp_?objectName@QObject@@QBE?AVQString@@XZ 100261dc     Qt5Core:Qt5Core.dll
 0002:000001e0       __imp_?fromAscii_helper@QString@@CAPAU?$QTypedArrayData@G@@PBDH@Z 100261e0     Qt5Core:Qt5Core.dll
 0002:000001e4       __imp_??M@YA_NABVQString@@0@Z 100261e4     Qt5Core:Qt5Core.dll
 0002:000001e8       __imp_??8@YA_NABVQString@@0@Z 100261e8     Qt5Core:Qt5Core.dll
 0002:000001ec       __imp_?number@QString@@SA?AV1@_JH@Z 100261ec     Qt5Core:Qt5Core.dll
 0002:000001f0       __imp_?fromUtf8@QString@@SA?AV1@PBDH@Z 100261f0     Qt5Core:Qt5Core.dll
 0002:000001f4       __imp_?append@QString@@QAEAAV1@ABV1@@Z 100261f4     Qt5Core:Qt5Core.dll
 0002:000001f8       __imp_?append@QString@@QAEAAV1@VQChar@@@Z 100261f8     Qt5Core:Qt5Core.dll
 0002:000001fc       __imp_?arg@QString@@QBE?AV1@ABV1@HVQChar@@@Z 100261fc     Qt5Core:Qt5Core.dll
 0002:00000200       __imp_?arg@QString@@QBE?AV1@HHHVQChar@@@Z 10026200     Qt5Core:Qt5Core.dll
 0002:00000204       __imp_?arg@QString@@QBE?AV1@_JHHVQChar@@@Z 10026204     Qt5Core:Qt5Core.dll
 0002:00000208       __imp_??4QString@@QAEAAV0@$$QAV0@@Z 10026208     Qt5Core:Qt5Core.dll
 0002:0000020c       __imp_??4QString@@QAEAAV0@ABV0@@Z 1002620c     Qt5Core:Qt5Core.dll
 0002:00000210       __imp_??1QString@@QAE@XZ   10026210     Qt5Core:Qt5Core.dll
 0002:00000214       __imp_??0QString@@QAE@ABV0@@Z 10026214     Qt5Core:Qt5Core.dll
 0002:00000218       __imp_??0QString@@QAE@XZ   10026218     Qt5Core:Qt5Core.dll
 0002:0000021c       __imp_??0QChar@@QAE@UQLatin1Char@@@Z 1002621c     Qt5Core:Qt5Core.dll
 0002:00000220       __imp_?freeData@QMapDataBase@@SAXPAU1@@Z 10026220     Qt5Core:Qt5Core.dll
 0002:00000224       __imp_?createData@QMapDataBase@@SAPAU1@XZ 10026224     Qt5Core:Qt5Core.dll
 0002:00000228       __imp_?freeTree@QMapDataBase@@QAEXPAUQMapNodeBase@@H@Z 10026228     Qt5Core:Qt5Core.dll
 0002:0000022c       __imp_?createNode@QMapDataBase@@QAEPAUQMapNodeBase@@HHPAU2@_N@Z 1002622c     Qt5Core:Qt5Core.dll
 0002:00000230       __imp_?recalcMostLeftNode@QMapDataBase@@QAEXXZ 10026230     Qt5Core:Qt5Core.dll
 0002:00000234       __imp_?freeNodeAndRebalance@QMapDataBase@@QAEXPAUQMapNodeBase@@@Z 10026234     Qt5Core:Qt5Core.dll
 0002:00000238       __imp_?typeFlags@QMetaType@@SA?AV?$QFlags@W4TypeFlag@QMetaType@@@@H@Z 10026238     Qt5Core:Qt5Core.dll
 0002:0000023c       __imp_?registerNormalizedTypedef@QMetaType@@SAHABVQByteArray@@H@Z 1002623c     Qt5Core:Qt5Core.dll
 0002:00000240       __imp_?registerNormalizedType@QMetaType@@SAHABVQByteArray@@P6AXPAX@ZP6APAXPBX@Z2P6APAX13@ZHV?$QFlags@W4TypeFlag@QMetaType@@@@PBUQMetaObject@@@Z 10026240     Qt5Core:Qt5Core.dll
 0002:00000244       __imp_??1Connection@QMetaObject@@QAE@XZ 10026244     Qt5Core:Qt5Core.dll
 0002:00000248       __imp_?connectSlotsByName@QMetaObject@@SAXPAVQObject@@@Z 10026248     Qt5Core:Qt5Core.dll
 0002:0000024c       __imp_?normalizedType@QMetaObject@@SA?AVQByteArray@@PBD@Z 1002624c     Qt5Core:Qt5Core.dll
 0002:00000250       __imp_?tr@QMetaObject@@QBE?AVQString@@PBD0H@Z 10026250     Qt5Core:Qt5Core.dll
 0002:00000254       __imp_?cast@QMetaObject@@QBEPAVQObject@@PAV2@@Z 10026254     Qt5Core:Qt5Core.dll
 0002:00000258       __imp_?dispose@QListData@@SAXPAUData@1@@Z 10026258     Qt5Core:Qt5Core.dll
 0002:0000025c       __imp_?detach@QListData@@QAEPAUData@1@H@Z 1002625c     Qt5Core:Qt5Core.dll
 0002:00000260       __imp_??1QByteArray@@QAE@XZ 10026260     Qt5Core:Qt5Core.dll
 0002:00000264       \177Qt5Core_NULL_THUNK_DATA 10026264     Qt5Core:Qt5Core.dll
 0002:00000268       __imp_??0QKeySequence@@QAE@ABVQString@@W4SequenceFormat@0@@Z 10026268     Qt5Gui:Qt5Gui.dll
 0002:0000026c       __imp_??0QIcon@@QAE@XZ     1002626c     Qt5Gui:Qt5Gui.dll
 0002:00000270       __imp_??1QIcon@@QAE@XZ     10026270     Qt5Gui:Qt5Gui.dll
 0002:00000274       __imp_??0QIcon@@QAE@ABVQString@@@Z 10026274     Qt5Gui:Qt5Gui.dll
 0002:00000278       __imp_?setRgb@QColor@@QAEXHHHH@Z 10026278     Qt5Gui:Qt5Gui.dll
 0002:0000027c       __imp_?clear@QTextDocument@@UAEXXZ 1002627c     Qt5Gui:Qt5Gui.dll
 0002:00000280       __imp_?createObject@QTextDocument@@MAEPAVQTextObject@@ABVQTextFormat@@@Z 10026280     Qt5Gui:Qt5Gui.dll
 0002:00000284       __imp_?loadResource@QTextDocument@@MAE?AVQVariant@@HABVQUrl@@@Z 10026284     Qt5Gui:Qt5Gui.dll
 0002:00000288       __imp_??1QKeySequence@@QAE@XZ 10026288     Qt5Gui:Qt5Gui.dll
 0002:0000028c       \177Qt5Gui_NULL_THUNK_DATA 1002628c     Qt5Gui:Qt5Gui.dll
 0002:00000290       __imp_??1QScriptValue@@QAE@XZ 10026290     Qt5Script:Qt5Script.dll
 0002:00000294       __imp_??0QScriptValue@@QAE@ABV0@@Z 10026294     Qt5Script:Qt5Script.dll
 0002:00000298       __imp_??4QScriptValue@@QAEAAV0@ABV0@@Z 10026298     Qt5Script:Qt5Script.dll
 0002:0000029c       __imp_?isNumber@QScriptValue@@QBE_NXZ 1002629c     Qt5Script:Qt5Script.dll
 0002:000002a0       __imp_?isString@QScriptValue@@QBE_NXZ 100262a0     Qt5Script:Qt5Script.dll
 0002:000002a4       __imp_?toString@QScriptValue@@QBE?AVQString@@XZ 100262a4     Qt5Script:Qt5Script.dll
 0002:000002a8       __imp_?toInt32@QScriptValue@@QBEHXZ 100262a8     Qt5Script:Qt5Script.dll
 0002:000002ac       __imp_??1QScriptEngine@@UAE@XZ 100262ac     Qt5Script:Qt5Script.dll
 0002:000002b0       __imp_?newVariant@QScriptEngine@@QAE?AVQScriptValue@@ABVQVariant@@@Z 100262b0     Qt5Script:Qt5Script.dll
 0002:000002b4       __imp_??0QScriptValue@@QAE@XZ 100262b4     Qt5Script:Qt5Script.dll
 0002:000002b8       \177Qt5Script_NULL_THUNK_DATA 100262b8     Qt5Script:Qt5Script.dll
 0002:000002bc       __imp_?staticMetaObject@QDialog@@2UQMetaObject@@B 100262bc     Qt5Widgets:Qt5Widgets.dll
 0002:000002c0       __imp_?qt_metacall@QDialog@@UAEHW4Call@QMetaObject@@HPAPAX@Z 100262c0     Qt5Widgets:Qt5Widgets.dll
 0002:000002c4       __imp_?qt_metacast@QDialog@@UAEPAXPBD@Z 100262c4     Qt5Widgets:Qt5Widgets.dll
 0002:000002c8       __imp_?updateEditorGeometry@QItemDelegate@@UBEXPAVQWidget@@ABVQStyleOptionViewItem@@ABVQModelIndex@@@Z 100262c8     Qt5Widgets:Qt5Widgets.dll
 0002:000002cc       __imp_?sizeHint@QItemDelegate@@UBE?AVQSize@@ABVQStyleOptionViewItem@@ABVQModelIndex@@@Z 100262cc     Qt5Widgets:Qt5Widgets.dll
 0002:000002d0       __imp_?paintingRoles@QAbstractItemDelegate@@UBE?AV?$QVector@H@@XZ 100262d0     Qt5Widgets:Qt5Widgets.dll
 0002:000002d4       __imp_?paint@QItemDelegate@@UBEXPAVQPainter@@ABVQStyleOptionViewItem@@ABVQModelIndex@@@Z 100262d4     Qt5Widgets:Qt5Widgets.dll
 0002:000002d8       __imp_?helpEvent@QAbstractItemDelegate@@UAE_NPAVQHelpEvent@@PAVQAbstractItemView@@ABVQStyleOptionViewItem@@ABVQModelIndex@@@Z 100262d8     Qt5Widgets:Qt5Widgets.dll
 0002:000002dc       __imp_?eventFilter@QItemDelegate@@MAE_NPAVQObject@@PAVQEvent@@@Z 100262dc     Qt5Widgets:Qt5Widgets.dll
 0002:000002e0       __imp_?editorEvent@QItemDelegate@@MAE_NPAVQEvent@@PAVQAbstractItemModel@@ABVQStyleOptionViewItem@@ABVQModelIndex@@@Z 100262e0     Qt5Widgets:Qt5Widgets.dll
 0002:000002e4       __imp_?drawFocus@QItemDelegate@@MBEXPAVQPainter@@ABVQStyleOptionViewItem@@ABVQRect@@@Z 100262e4     Qt5Widgets:Qt5Widgets.dll
 0002:000002e8       __imp_?drawDisplay@QItemDelegate@@MBEXPAVQPainter@@ABVQStyleOptionViewItem@@ABVQRect@@ABVQString@@@Z 100262e8     Qt5Widgets:Qt5Widgets.dll
 0002:000002ec       __imp_?drawDecoration@QItemDelegate@@MBEXPAVQPainter@@ABVQStyleOptionViewItem@@ABVQRect@@ABVQPixmap@@@Z 100262ec     Qt5Widgets:Qt5Widgets.dll
 0002:000002f0       __imp_?drawCheck@QItemDelegate@@MBEXPAVQPainter@@ABVQStyleOptionViewItem@@ABVQRect@@W4CheckState@Qt@@@Z 100262f0     Qt5Widgets:Qt5Widgets.dll
 0002:000002f4       __imp_?destroyEditor@QAbstractItemDelegate@@UBEXPAVQWidget@@ABVQModelIndex@@@Z 100262f4     Qt5Widgets:Qt5Widgets.dll
 0002:000002f8       __imp_?event@QAction@@MAE_NPAVQEvent@@@Z 100262f8     Qt5Widgets:Qt5Widgets.dll
 0002:000002fc       __imp_?staticMetaObject@QAction@@2UQMetaObject@@B 100262fc     Qt5Widgets:Qt5Widgets.dll
 0002:00000300       __imp_?write@QTreeWidgetItem@@UBEXAAVQDataStream@@@Z 10026300     Qt5Widgets:Qt5Widgets.dll
 0002:00000304       __imp_?widget@QLayoutItem@@UAEPAVQWidget@@XZ 10026304     Qt5Widgets:Qt5Widgets.dll
 0002:00000308       __imp_?wheelEvent@QWidget@@MAEXPAVQWheelEvent@@@Z 10026308     Qt5Widgets:Qt5Widgets.dll
 0002:0000030c       __imp_?wheelEvent@QTextEdit@@MAEXPAVQWheelEvent@@@Z 1002630c     Qt5Widgets:Qt5Widgets.dll
 0002:00000310       __imp_?wheelEvent@QComboBox@@MAEXPAVQWheelEvent@@@Z 10026310     Qt5Widgets:Qt5Widgets.dll
 0002:00000314       __imp_?wheelEvent@QAbstractSpinBox@@MAEXPAVQWheelEvent@@@Z 10026314     Qt5Widgets:Qt5Widgets.dll
 0002:00000318       __imp_?wheelEvent@QAbstractScrollArea@@MAEXPAVQWheelEvent@@@Z 10026318     Qt5Widgets:Qt5Widgets.dll
 0002:0000031c       __imp_?visualRegionForSelection@QTreeView@@MBE?AVQRegion@@ABVQItemSelection@@@Z 1002631c     Qt5Widgets:Qt5Widgets.dll
 0002:00000320       __imp_?visualRect@QTreeView@@UBE?AVQRect@@ABVQModelIndex@@@Z 10026320     Qt5Widgets:Qt5Widgets.dll
 0002:00000324       __imp_?viewportSizeHint@QTreeView@@MBE?AVQSize@@XZ 10026324     Qt5Widgets:Qt5Widgets.dll
 0002:00000328       __imp_?viewportSizeHint@QAbstractScrollArea@@MBE?AVQSize@@XZ 10026328     Qt5Widgets:Qt5Widgets.dll
 0002:0000032c       __imp_?viewportEvent@QTreeView@@MAE_NPAVQEvent@@@Z 1002632c     Qt5Widgets:Qt5Widgets.dll
 0002:00000330       __imp_?viewportEvent@QAbstractScrollArea@@MAE_NPAVQEvent@@@Z 10026330     Qt5Widgets:Qt5Widgets.dll
 0002:00000334       __imp_?viewOptions@QAbstractItemView@@MBE?AVQStyleOptionViewItem@@XZ 10026334     Qt5Widgets:Qt5Widgets.dll
 0002:00000338       __imp_?verticalScrollbarValueChanged@QAbstractItemView@@MAEXH@Z 10026338     Qt5Widgets:Qt5Widgets.dll
 0002:0000033c       __imp_?verticalScrollbarAction@QAbstractItemView@@MAEXH@Z 1002633c     Qt5Widgets:Qt5Widgets.dll
 0002:00000340       __imp_?verticalOffset@QTreeView@@MBEHXZ 10026340     Qt5Widgets:Qt5Widgets.dll
 0002:00000344       __imp_?valueFromText@QSpinBox@@MBEHABVQString@@@Z 10026344     Qt5Widgets:Qt5Widgets.dll
 0002:00000348       __imp_?validate@QSpinBox@@MBE?AW4State@QValidator@@AAVQString@@AAH@Z 10026348     Qt5Widgets:Qt5Widgets.dll
 0002:0000034c       __imp_?updateGeometries@QTreeView@@MAEXXZ 1002634c     Qt5Widgets:Qt5Widgets.dll
 0002:00000350       __imp_?updateEditorGeometries@QAbstractItemView@@MAEXXZ 10026350     Qt5Widgets:Qt5Widgets.dll
 0002:00000354       __imp_?updateEditorData@QAbstractItemView@@MAEXXZ 10026354     Qt5Widgets:Qt5Widgets.dll
 0002:00000358       __imp_?timerEvent@QTreeView@@MAEXPAVQTimerEvent@@@Z 10026358     Qt5Widgets:Qt5Widgets.dll
 0002:0000035c       __imp_?timerEvent@QTextEdit@@MAEXPAVQTimerEvent@@@Z 1002635c     Qt5Widgets:Qt5Widgets.dll
 0002:00000360       __imp_?timerEvent@QAbstractSpinBox@@MAEXPAVQTimerEvent@@@Z 10026360     Qt5Widgets:Qt5Widgets.dll
 0002:00000364       __imp_?timerEvent@QAbstractButton@@MAEXPAVQTimerEvent@@@Z 10026364     Qt5Widgets:Qt5Widgets.dll
 0002:00000368       __imp_?textFromValue@QSpinBox@@MBE?AVQString@@H@Z 10026368     Qt5Widgets:Qt5Widgets.dll
 0002:0000036c       __imp_?takeAt@QGridLayout@@UAEPAVQLayoutItem@@H@Z 1002636c     Qt5Widgets:Qt5Widgets.dll
 0002:00000370       __imp_?takeAt@QBoxLayout@@UAEPAVQLayoutItem@@H@Z 10026370     Qt5Widgets:Qt5Widgets.dll
 0002:00000374       __imp_?tabletEvent@QWidget@@MAEXPAVQTabletEvent@@@Z 10026374     Qt5Widgets:Qt5Widgets.dll
 0002:00000378       __imp_?tabRemoved@QTabWidget@@MAEXH@Z 10026378     Qt5Widgets:Qt5Widgets.dll
 0002:0000037c       __imp_?tabInserted@QTabWidget@@MAEXH@Z 1002637c     Qt5Widgets:Qt5Widgets.dll
 0002:00000380       __imp_?supportedDropActions@QTreeWidget@@MBE?AV?$QFlags@W4DropAction@Qt@@@@XZ 10026380     Qt5Widgets:Qt5Widgets.dll
 0002:00000384       __imp_?stepEnabled@QAbstractSpinBox@@MBE?AV?$QFlags@W4StepEnabledFlag@QAbstractSpinBox@@@@XZ 10026384     Qt5Widgets:Qt5Widgets.dll
 0002:00000388       __imp_?stepBy@QAbstractSpinBox@@UAEXH@Z 10026388     Qt5Widgets:Qt5Widgets.dll
 0002:0000038c       __imp_?startDrag@QAbstractItemView@@MAEXV?$QFlags@W4DropAction@Qt@@@@@Z 1002638c     Qt5Widgets:Qt5Widgets.dll
 0002:00000390       __imp_?spacerItem@QSpacerItem@@UAEPAV1@XZ 10026390     Qt5Widgets:Qt5Widgets.dll
 0002:00000394       __imp_?spacerItem@QLayoutItem@@UAEPAVQSpacerItem@@XZ 10026394     Qt5Widgets:Qt5Widgets.dll
 0002:00000398       __imp_?sizeHintForRow@QAbstractItemView@@UBEHH@Z 10026398     Qt5Widgets:Qt5Widgets.dll
 0002:0000039c       __imp_?sizeHintForColumn@QTreeView@@MBEHH@Z 1002639c     Qt5Widgets:Qt5Widgets.dll
 0002:000003a0       __imp_?sizeHint@QWidget@@UBE?AVQSize@@XZ 100263a0     Qt5Widgets:Qt5Widgets.dll
 0002:000003a4       __imp_?sizeHint@QTabWidget@@UBE?AVQSize@@XZ 100263a4     Qt5Widgets:Qt5Widgets.dll
 0002:000003a8       __imp_?sizeHint@QSpacerItem@@UBE?AVQSize@@XZ 100263a8     Qt5Widgets:Qt5Widgets.dll
 0002:000003ac       __imp_?sizeHint@QRadioButton@@UBE?AVQSize@@XZ 100263ac     Qt5Widgets:Qt5Widgets.dll
 0002:000003b0       __imp_?sizeHint@QPushButton@@UBE?AVQSize@@XZ 100263b0     Qt5Widgets:Qt5Widgets.dll
 0002:000003b4       __imp_?sizeHint@QLabel@@UBE?AVQSize@@XZ 100263b4     Qt5Widgets:Qt5Widgets.dll
 0002:000003b8       __imp_?sizeHint@QGridLayout@@UBE?AVQSize@@XZ 100263b8     Qt5Widgets:Qt5Widgets.dll
 0002:000003bc       __imp_?sizeHint@QDialog@@UBE?AVQSize@@XZ 100263bc     Qt5Widgets:Qt5Widgets.dll
 0002:000003c0       __imp_?sizeHint@QComboBox@@UBE?AVQSize@@XZ 100263c0     Qt5Widgets:Qt5Widgets.dll
 0002:000003c4       __imp_?sizeHint@QCheckBox@@UBE?AVQSize@@XZ 100263c4     Qt5Widgets:Qt5Widgets.dll
 0002:000003c8       __imp_?sizeHint@QBoxLayout@@UBE?AVQSize@@XZ 100263c8     Qt5Widgets:Qt5Widgets.dll
 0002:000003cc       __imp_?sizeHint@QAbstractSpinBox@@UBE?AVQSize@@XZ 100263cc     Qt5Widgets:Qt5Widgets.dll
 0002:000003d0       __imp_?sizeHint@QAbstractScrollArea@@UBE?AVQSize@@XZ 100263d0     Qt5Widgets:Qt5Widgets.dll
 0002:000003d4       __imp_?showPopup@QComboBox@@UAEXXZ 100263d4     Qt5Widgets:Qt5Widgets.dll
 0002:000003d8       __imp_?showEvent@QWidget@@MAEXPAVQShowEvent@@@Z 100263d8     Qt5Widgets:Qt5Widgets.dll
 0002:000003dc       __imp_?showEvent@QTextEdit@@MAEXPAVQShowEvent@@@Z 100263dc     Qt5Widgets:Qt5Widgets.dll
 0002:000003e0       __imp_?showEvent@QTabWidget@@MAEXPAVQShowEvent@@@Z 100263e0     Qt5Widgets:Qt5Widgets.dll
 0002:000003e4       __imp_?showEvent@QDialog@@MAEXPAVQShowEvent@@@Z 100263e4     Qt5Widgets:Qt5Widgets.dll
 0002:000003e8       __imp_?showEvent@QComboBox@@MAEXPAVQShowEvent@@@Z 100263e8     Qt5Widgets:Qt5Widgets.dll
 0002:000003ec       __imp_?showEvent@QAbstractSpinBox@@MAEXPAVQShowEvent@@@Z 100263ec     Qt5Widgets:Qt5Widgets.dll
 0002:000003f0       __imp_?sharedPainter@QWidget@@MBEPAVQPainter@@XZ 100263f0     Qt5Widgets:Qt5Widgets.dll
 0002:000003f4       __imp_?setupViewport@QAbstractScrollArea@@UAEXPAVQWidget@@@Z 100263f4     Qt5Widgets:Qt5Widgets.dll
 0002:000003f8       __imp_?setVisible@QWidget@@UAEX_N@Z 100263f8     Qt5Widgets:Qt5Widgets.dll
 0002:000003fc       __imp_?setVisible@QDialog@@UAEX_N@Z 100263fc     Qt5Widgets:Qt5Widgets.dll
 0002:00000400       __imp_?setSelectionModel@QTreeWidget@@UAEXPAVQItemSelectionModel@@@Z 10026400     Qt5Widgets:Qt5Widgets.dll
 0002:00000404       __imp_?setSelection@QTreeView@@MAEXABVQRect@@V?$QFlags@W4SelectionFlag@QItemSelectionModel@@@@@Z 10026404     Qt5Widgets:Qt5Widgets.dll
 0002:00000408       __imp_?setRootIndex@QTreeView@@UAEXABVQModelIndex@@@Z 10026408     Qt5Widgets:Qt5Widgets.dll
 0002:0000040c       __imp_?setModel@QTreeWidget@@EAEXPAVQAbstractItemModel@@@Z 1002640c     Qt5Widgets:Qt5Widgets.dll
 0002:00000410       __imp_?setGeometry@QSpacerItem@@UAEXABVQRect@@@Z 10026410     Qt5Widgets:Qt5Widgets.dll
 0002:00000414       __imp_?setGeometry@QGridLayout@@UAEXABVQRect@@@Z 10026414     Qt5Widgets:Qt5Widgets.dll
 0002:00000418       __imp_?setGeometry@QBoxLayout@@UAEXABVQRect@@@Z 10026418     Qt5Widgets:Qt5Widgets.dll
 0002:0000041c       __imp_?setData@QTreeWidgetItem@@UAEXHHABVQVariant@@@Z 1002641c     Qt5Widgets:Qt5Widgets.dll
 0002:00000420       __imp_?selectionCommand@QAbstractItemView@@MBE?AV?$QFlags@W4SelectionFlag@QItemSelectionModel@@@@ABVQModelIndex@@PBVQEvent@@@Z 10026420     Qt5Widgets:Qt5Widgets.dll
 0002:00000424       __imp_?selectionChanged@QTreeView@@MAEXABVQItemSelection@@0@Z 10026424     Qt5Widgets:Qt5Widgets.dll
 0002:00000428       __imp_?selectedIndexes@QTreeView@@MBE?AV?$QList@VQModelIndex@@@@XZ 10026428     Qt5Widgets:Qt5Widgets.dll
 0002:0000042c       __imp_?selectAll@QTreeView@@UAEXXZ 1002642c     Qt5Widgets:Qt5Widgets.dll
 0002:00000430       __imp_?scrollTo@QTreeView@@UAEXABVQModelIndex@@W4ScrollHint@QAbstractItemView@@@Z 10026430     Qt5Widgets:Qt5Widgets.dll
 0002:00000434       __imp_?scrollContentsBy@QTreeView@@MAEXHH@Z 10026434     Qt5Widgets:Qt5Widgets.dll
 0002:00000438       __imp_?scrollContentsBy@QTextEdit@@MAEXHH@Z 10026438     Qt5Widgets:Qt5Widgets.dll
 0002:0000043c       __imp_?rowsInserted@QTreeView@@MAEXABVQModelIndex@@HH@Z 1002643c     Qt5Widgets:Qt5Widgets.dll
 0002:00000440       __imp_?rowsAboutToBeRemoved@QTreeView@@MAEXABVQModelIndex@@HH@Z 10026440     Qt5Widgets:Qt5Widgets.dll
 0002:00000444       __imp_?resizeEvent@QWidget@@MAEXPAVQResizeEvent@@@Z 10026444     Qt5Widgets:Qt5Widgets.dll
 0002:00000448       __imp_?resizeEvent@QTextEdit@@MAEXPAVQResizeEvent@@@Z 10026448     Qt5Widgets:Qt5Widgets.dll
 0002:0000044c       __imp_?resizeEvent@QTabWidget@@MAEXPAVQResizeEvent@@@Z 1002644c     Qt5Widgets:Qt5Widgets.dll
 0002:00000450       __imp_?resizeEvent@QGroupBox@@MAEXPAVQResizeEvent@@@Z 10026450     Qt5Widgets:Qt5Widgets.dll
 0002:00000454       __imp_?resizeEvent@QDialog@@MAEXPAVQResizeEvent@@@Z 10026454     Qt5Widgets:Qt5Widgets.dll
 0002:00000458       __imp_?resizeEvent@QComboBox@@MAEXPAVQResizeEvent@@@Z 10026458     Qt5Widgets:Qt5Widgets.dll
 0002:0000045c       __imp_?resizeEvent@QAbstractSpinBox@@MAEXPAVQResizeEvent@@@Z 1002645c     Qt5Widgets:Qt5Widgets.dll
 0002:00000460       __imp_?resizeEvent@QAbstractItemView@@MAEXPAVQResizeEvent@@@Z 10026460     Qt5Widgets:Qt5Widgets.dll
 0002:00000464       __imp_?reset@QTreeView@@UAEXXZ 10026464     Qt5Widgets:Qt5Widgets.dll
 0002:00000468       __imp_?redirected@QWidget@@MBEPAVQPaintDevice@@PAVQPoint@@@Z 10026468     Qt5Widgets:Qt5Widgets.dll
 0002:0000046c       __imp_?read@QTreeWidgetItem@@UAEXAAVQDataStream@@@Z 1002646c     Qt5Widgets:Qt5Widgets.dll
 0002:00000470       __imp_?qt_metacast@QWidget@@UAEPAXPBD@Z 10026470     Qt5Widgets:Qt5Widgets.dll
 0002:00000474       __imp_?qt_metacast@QVBoxLayout@@UAEPAXPBD@Z 10026474     Qt5Widgets:Qt5Widgets.dll
 0002:00000478       __imp_?qt_metacast@QTreeWidget@@UAEPAXPBD@Z 10026478     Qt5Widgets:Qt5Widgets.dll
 0002:0000047c       __imp_?qt_metacast@QTextEdit@@UAEPAXPBD@Z 1002647c     Qt5Widgets:Qt5Widgets.dll
 0002:00000480       __imp_?qt_metacast@QTabWidget@@UAEPAXPBD@Z 10026480     Qt5Widgets:Qt5Widgets.dll
 0002:00000484       __imp_?qt_metacast@QSpinBox@@UAEPAXPBD@Z 10026484     Qt5Widgets:Qt5Widgets.dll
 0002:00000488       __imp_?qt_metacast@QRadioButton@@UAEPAXPBD@Z 10026488     Qt5Widgets:Qt5Widgets.dll
 0002:0000048c       __imp_?qt_metacast@QPushButton@@UAEPAXPBD@Z 1002648c     Qt5Widgets:Qt5Widgets.dll
 0002:00000490       __imp_?qt_metacast@QLabel@@UAEPAXPBD@Z 10026490     Qt5Widgets:Qt5Widgets.dll
 0002:00000494       __imp_?qt_metacast@QHBoxLayout@@UAEPAXPBD@Z 10026494     Qt5Widgets:Qt5Widgets.dll
 0002:00000498       __imp_?qt_metacast@QGroupBox@@UAEPAXPBD@Z 10026498     Qt5Widgets:Qt5Widgets.dll
 0002:0000049c       __imp_?qt_metacast@QGridLayout@@UAEPAXPBD@Z 1002649c     Qt5Widgets:Qt5Widgets.dll
 0002:000004a0       __imp_?qt_metacast@QDialogButtonBox@@UAEPAXPBD@Z 100264a0     Qt5Widgets:Qt5Widgets.dll
 0002:000004a4       __imp_?qt_metacast@QComboBox@@UAEPAXPBD@Z 100264a4     Qt5Widgets:Qt5Widgets.dll
 0002:000004a8       __imp_?qt_metacast@QCheckBox@@UAEPAXPBD@Z 100264a8     Qt5Widgets:Qt5Widgets.dll
 0002:000004ac       __imp_?qt_metacall@QWidget@@UAEHW4Call@QMetaObject@@HPAPAX@Z 100264ac     Qt5Widgets:Qt5Widgets.dll
 0002:000004b0       __imp_?qt_metacall@QVBoxLayout@@UAEHW4Call@QMetaObject@@HPAPAX@Z 100264b0     Qt5Widgets:Qt5Widgets.dll
 0002:000004b4       __imp_?qt_metacall@QTreeWidget@@UAEHW4Call@QMetaObject@@HPAPAX@Z 100264b4     Qt5Widgets:Qt5Widgets.dll
 0002:000004b8       __imp_?qt_metacall@QTextEdit@@UAEHW4Call@QMetaObject@@HPAPAX@Z 100264b8     Qt5Widgets:Qt5Widgets.dll
 0002:000004bc       __imp_?qt_metacall@QTabWidget@@UAEHW4Call@QMetaObject@@HPAPAX@Z 100264bc     Qt5Widgets:Qt5Widgets.dll
 0002:000004c0       __imp_?qt_metacall@QSpinBox@@UAEHW4Call@QMetaObject@@HPAPAX@Z 100264c0     Qt5Widgets:Qt5Widgets.dll
 0002:000004c4       __imp_?qt_metacall@QRadioButton@@UAEHW4Call@QMetaObject@@HPAPAX@Z 100264c4     Qt5Widgets:Qt5Widgets.dll
 0002:000004c8       __imp_?qt_metacall@QPushButton@@UAEHW4Call@QMetaObject@@HPAPAX@Z 100264c8     Qt5Widgets:Qt5Widgets.dll
 0002:000004cc       __imp_?qt_metacall@QLabel@@UAEHW4Call@QMetaObject@@HPAPAX@Z 100264cc     Qt5Widgets:Qt5Widgets.dll
 0002:000004d0       __imp_?qt_metacall@QHBoxLayout@@UAEHW4Call@QMetaObject@@HPAPAX@Z 100264d0     Qt5Widgets:Qt5Widgets.dll
 0002:000004d4       __imp_?qt_metacall@QGroupBox@@UAEHW4Call@QMetaObject@@HPAPAX@Z 100264d4     Qt5Widgets:Qt5Widgets.dll
 0002:000004d8       __imp_?qt_metacall@QGridLayout@@UAEHW4Call@QMetaObject@@HPAPAX@Z 100264d8     Qt5Widgets:Qt5Widgets.dll
 0002:000004dc       __imp_?qt_metacall@QDialogButtonBox@@UAEHW4Call@QMetaObject@@HPAPAX@Z 100264dc     Qt5Widgets:Qt5Widgets.dll
 0002:000004e0       __imp_?qt_metacall@QComboBox@@UAEHW4Call@QMetaObject@@HPAPAX@Z 100264e0     Qt5Widgets:Qt5Widgets.dll
 0002:000004e4       __imp_?qt_metacall@QCheckBox@@UAEHW4Call@QMetaObject@@HPAPAX@Z 100264e4     Qt5Widgets:Qt5Widgets.dll
 0002:000004e8       __imp_?paintEvent@QWidget@@MAEXPAVQPaintEvent@@@Z 100264e8     Qt5Widgets:Qt5Widgets.dll
 0002:000004ec       __imp_?paintEvent@QTreeView@@MAEXPAVQPaintEvent@@@Z 100264ec     Qt5Widgets:Qt5Widgets.dll
 0002:000004f0       __imp_?paintEvent@QTextEdit@@MAEXPAVQPaintEvent@@@Z 100264f0     Qt5Widgets:Qt5Widgets.dll
 0002:000004f4       __imp_?paintEvent@QTabWidget@@MAEXPAVQPaintEvent@@@Z 100264f4     Qt5Widgets:Qt5Widgets.dll
 0002:000004f8       __imp_?paintEvent@QRadioButton@@MAEXPAVQPaintEvent@@@Z 100264f8     Qt5Widgets:Qt5Widgets.dll
 0002:000004fc       __imp_?paintEvent@QPushButton@@MAEXPAVQPaintEvent@@@Z 100264fc     Qt5Widgets:Qt5Widgets.dll
 0002:00000500       __imp_?paintEvent@QLabel@@MAEXPAVQPaintEvent@@@Z 10026500     Qt5Widgets:Qt5Widgets.dll
 0002:00000504       __imp_?paintEvent@QGroupBox@@MAEXPAVQPaintEvent@@@Z 10026504     Qt5Widgets:Qt5Widgets.dll
 0002:00000508       __imp_?paintEvent@QComboBox@@MAEXPAVQPaintEvent@@@Z 10026508     Qt5Widgets:Qt5Widgets.dll
 0002:0000050c       __imp_?paintEvent@QCheckBox@@MAEXPAVQPaintEvent@@@Z 1002650c     Qt5Widgets:Qt5Widgets.dll
 0002:00000510       __imp_?paintEvent@QAbstractSpinBox@@MAEXPAVQPaintEvent@@@Z 10026510     Qt5Widgets:Qt5Widgets.dll
 0002:00000514       __imp_?paintEngine@QWidget@@UBEPAVQPaintEngine@@XZ 10026514     Qt5Widgets:Qt5Widgets.dll
 0002:00000518       __imp_?open@QDialog@@UAEXXZ 10026518     Qt5Widgets:Qt5Widgets.dll
 0002:0000051c       __imp_?nextCheckState@QCheckBox@@MAEXXZ 1002651c     Qt5Widgets:Qt5Widgets.dll
 0002:00000520       __imp_?nextCheckState@QAbstractButton@@MAEXXZ 10026520     Qt5Widgets:Qt5Widgets.dll
 0002:00000524       __imp_?nativeEvent@QWidget@@MAE_NABVQByteArray@@PAXPAJ@Z 10026524     Qt5Widgets:Qt5Widgets.dll
 0002:00000528       __imp_?moveEvent@QWidget@@MAEXPAVQMoveEvent@@@Z 10026528     Qt5Widgets:Qt5Widgets.dll
 0002:0000052c       __imp_?moveCursor@QTreeView@@MAE?AVQModelIndex@@W4CursorAction@QAbstractItemView@@V?$QFlags@W4KeyboardModifier@Qt@@@@@Z 1002652c     Qt5Widgets:Qt5Widgets.dll
 0002:00000530       __imp_?mouseReleaseEvent@QWidget@@MAEXPAVQMouseEvent@@@Z 10026530     Qt5Widgets:Qt5Widgets.dll
 0002:00000534       __imp_?mouseReleaseEvent@QTreeView@@MAEXPAVQMouseEvent@@@Z 10026534     Qt5Widgets:Qt5Widgets.dll
 0002:00000538       __imp_?mouseReleaseEvent@QTextEdit@@MAEXPAVQMouseEvent@@@Z 10026538     Qt5Widgets:Qt5Widgets.dll
 0002:0000053c       __imp_?mouseReleaseEvent@QLabel@@MAEXPAVQMouseEvent@@@Z 1002653c     Qt5Widgets:Qt5Widgets.dll
 0002:00000540       __imp_?mouseReleaseEvent@QGroupBox@@MAEXPAVQMouseEvent@@@Z 10026540     Qt5Widgets:Qt5Widgets.dll
 0002:00000544       __imp_?mouseReleaseEvent@QComboBox@@MAEXPAVQMouseEvent@@@Z 10026544     Qt5Widgets:Qt5Widgets.dll
 0002:00000548       __imp_?mouseReleaseEvent@QAbstractSpinBox@@MAEXPAVQMouseEvent@@@Z 10026548     Qt5Widgets:Qt5Widgets.dll
 0002:0000054c       __imp_?mouseReleaseEvent@QAbstractButton@@MAEXPAVQMouseEvent@@@Z 1002654c     Qt5Widgets:Qt5Widgets.dll
 0002:00000550       __imp_?mousePressEvent@QWidget@@MAEXPAVQMouseEvent@@@Z 10026550     Qt5Widgets:Qt5Widgets.dll
 0002:00000554       __imp_?mousePressEvent@QTreeView@@MAEXPAVQMouseEvent@@@Z 10026554     Qt5Widgets:Qt5Widgets.dll
 0002:00000558       __imp_?mousePressEvent@QTextEdit@@MAEXPAVQMouseEvent@@@Z 10026558     Qt5Widgets:Qt5Widgets.dll
 0002:0000055c       __imp_?mousePressEvent@QLabel@@MAEXPAVQMouseEvent@@@Z 1002655c     Qt5Widgets:Qt5Widgets.dll
 0002:00000560       __imp_?mousePressEvent@QGroupBox@@MAEXPAVQMouseEvent@@@Z 10026560     Qt5Widgets:Qt5Widgets.dll
 0002:00000564       __imp_?mousePressEvent@QComboBox@@MAEXPAVQMouseEvent@@@Z 10026564     Qt5Widgets:Qt5Widgets.dll
 0002:00000568       __imp_?mousePressEvent@QAbstractSpinBox@@MAEXPAVQMouseEvent@@@Z 10026568     Qt5Widgets:Qt5Widgets.dll
 0002:0000056c       __imp_?mousePressEvent@QAbstractButton@@MAEXPAVQMouseEvent@@@Z 1002656c     Qt5Widgets:Qt5Widgets.dll
 0002:00000570       __imp_?mouseMoveEvent@QWidget@@MAEXPAVQMouseEvent@@@Z 10026570     Qt5Widgets:Qt5Widgets.dll
 0002:00000574       __imp_?mouseMoveEvent@QTreeView@@MAEXPAVQMouseEvent@@@Z 10026574     Qt5Widgets:Qt5Widgets.dll
 0002:00000578       __imp_?mouseMoveEvent@QTextEdit@@MAEXPAVQMouseEvent@@@Z 10026578     Qt5Widgets:Qt5Widgets.dll
 0002:0000057c       __imp_?mouseMoveEvent@QRadioButton@@MAEXPAVQMouseEvent@@@Z 1002657c     Qt5Widgets:Qt5Widgets.dll
 0002:00000580       __imp_?mouseMoveEvent@QLabel@@MAEXPAVQMouseEvent@@@Z 10026580     Qt5Widgets:Qt5Widgets.dll
 0002:00000584       __imp_?mouseMoveEvent@QGroupBox@@MAEXPAVQMouseEvent@@@Z 10026584     Qt5Widgets:Qt5Widgets.dll
 0002:00000588       __imp_?mouseMoveEvent@QCheckBox@@MAEXPAVQMouseEvent@@@Z 10026588     Qt5Widgets:Qt5Widgets.dll
 0002:0000058c       __imp_?mouseMoveEvent@QAbstractSpinBox@@MAEXPAVQMouseEvent@@@Z 1002658c     Qt5Widgets:Qt5Widgets.dll
 0002:00000590       __imp_?mouseMoveEvent@QAbstractButton@@MAEXPAVQMouseEvent@@@Z 10026590     Qt5Widgets:Qt5Widgets.dll
 0002:00000594       __imp_?mouseDoubleClickEvent@QWidget@@MAEXPAVQMouseEvent@@@Z 10026594     Qt5Widgets:Qt5Widgets.dll
 0002:00000598       __imp_?mouseDoubleClickEvent@QTreeView@@MAEXPAVQMouseEvent@@@Z 10026598     Qt5Widgets:Qt5Widgets.dll
 0002:0000059c       __imp_?mouseDoubleClickEvent@QTextEdit@@MAEXPAVQMouseEvent@@@Z 1002659c     Qt5Widgets:Qt5Widgets.dll
 0002:000005a0       __imp_?minimumSizeHint@QWidget@@UBE?AVQSize@@XZ 100265a0     Qt5Widgets:Qt5Widgets.dll
 0002:000005a4       __imp_?minimumSizeHint@QTabWidget@@UBE?AVQSize@@XZ 100265a4     Qt5Widgets:Qt5Widgets.dll
 0002:000005a8       __imp_?minimumSizeHint@QRadioButton@@UBE?AVQSize@@XZ 100265a8     Qt5Widgets:Qt5Widgets.dll
 0002:000005ac       __imp_?minimumSizeHint@QPushButton@@UBE?AVQSize@@XZ 100265ac     Qt5Widgets:Qt5Widgets.dll
 0002:000005b0       __imp_?minimumSizeHint@QLabel@@UBE?AVQSize@@XZ 100265b0     Qt5Widgets:Qt5Widgets.dll
 0002:000005b4       __imp_?minimumSizeHint@QGroupBox@@UBE?AVQSize@@XZ 100265b4     Qt5Widgets:Qt5Widgets.dll
 0002:000005b8       __imp_?minimumSizeHint@QDialog@@UBE?AVQSize@@XZ 100265b8     Qt5Widgets:Qt5Widgets.dll
 0002:000005bc       __imp_?minimumSizeHint@QComboBox@@UBE?AVQSize@@XZ 100265bc     Qt5Widgets:Qt5Widgets.dll
 0002:000005c0       __imp_?minimumSizeHint@QCheckBox@@UBE?AVQSize@@XZ 100265c0     Qt5Widgets:Qt5Widgets.dll
 0002:000005c4       __imp_?minimumSizeHint@QAbstractSpinBox@@UBE?AVQSize@@XZ 100265c4     Qt5Widgets:Qt5Widgets.dll
 0002:000005c8       __imp_?minimumSizeHint@QAbstractScrollArea@@UBE?AVQSize@@XZ 100265c8     Qt5Widgets:Qt5Widgets.dll
 0002:000005cc       __imp_?minimumSize@QSpacerItem@@UBE?AVQSize@@XZ 100265cc     Qt5Widgets:Qt5Widgets.dll
 0002:000005d0       __imp_??0QSizePolicy@@QAE@W4Policy@0@0W4ControlType@0@@Z 100265d0     Qt5Widgets:Qt5Widgets.dll
 0002:000005d4       __imp_?setHorizontalStretch@QSizePolicy@@QAEXH@Z 100265d4     Qt5Widgets:Qt5Widgets.dll
 0002:000005d8       __imp_?setVerticalStretch@QSizePolicy@@QAEXH@Z 100265d8     Qt5Widgets:Qt5Widgets.dll
 0002:000005dc       __imp_??0QWidget@@QAE@PAV0@V?$QFlags@W4WindowType@Qt@@@@@Z 100265dc     Qt5Widgets:Qt5Widgets.dll
 0002:000005e0       __imp_??1QWidget@@UAE@XZ   100265e0     Qt5Widgets:Qt5Widgets.dll
 0002:000005e4       __imp_?setEnabled@QWidget@@QAEX_N@Z 100265e4     Qt5Widgets:Qt5Widgets.dll
 0002:000005e8       __imp_?setDisabled@QWidget@@QAEX_N@Z 100265e8     Qt5Widgets:Qt5Widgets.dll
 0002:000005ec       __imp_?setMinimumSize@QWidget@@QAEXHH@Z 100265ec     Qt5Widgets:Qt5Widgets.dll
 0002:000005f0       __imp_?setMaximumSize@QWidget@@QAEXHH@Z 100265f0     Qt5Widgets:Qt5Widgets.dll
 0002:000005f4       __imp_?setWindowTitle@QWidget@@QAEXABVQString@@@Z 100265f4     Qt5Widgets:Qt5Widgets.dll
 0002:000005f8       __imp_?setToolTip@QWidget@@QAEXABVQString@@@Z 100265f8     Qt5Widgets:Qt5Widgets.dll
 0002:000005fc       __imp_?setWhatsThis@QWidget@@QAEXABVQString@@@Z 100265fc     Qt5Widgets:Qt5Widgets.dll
 0002:00000600       __imp_?setFocus@QWidget@@QAEXW4FocusReason@Qt@@@Z 10026600     Qt5Widgets:Qt5Widgets.dll
 0002:00000604       __imp_?resize@QWidget@@QAEXABVQSize@@@Z 10026604     Qt5Widgets:Qt5Widgets.dll
 0002:00000608       __imp_?sizePolicy@QWidget@@QBE?AVQSizePolicy@@XZ 10026608     Qt5Widgets:Qt5Widgets.dll
 0002:0000060c       __imp_?setSizePolicy@QWidget@@QAEXVQSizePolicy@@@Z 1002660c     Qt5Widgets:Qt5Widgets.dll
 0002:00000610       __imp_?setLayout@QWidget@@QAEXPAVQLayout@@@Z 10026610     Qt5Widgets:Qt5Widgets.dll
 0002:00000614       __imp_?actions@QWidget@@QBE?AV?$QList@PAVQAction@@@@XZ 10026614     Qt5Widgets:Qt5Widgets.dll
 0002:00000618       __imp_?setAttribute@QWidget@@QAEXW4WidgetAttribute@Qt@@_N@Z 10026618     Qt5Widgets:Qt5Widgets.dll
 0002:0000061c       __imp_?text@QAction@@QBE?AVQString@@XZ 1002661c     Qt5Widgets:Qt5Widgets.dll
 0002:00000620       __imp_?isChecked@QAction@@QBE_NXZ 10026620     Qt5Widgets:Qt5Widgets.dll
 0002:00000624       __imp_?activate@QAction@@QAEXW4ActionEvent@1@@Z 10026624     Qt5Widgets:Qt5Widgets.dll
 0002:00000628       __imp_?setText@QAbstractButton@@QAEXABVQString@@@Z 10026628     Qt5Widgets:Qt5Widgets.dll
 0002:0000062c       __imp_?setShortcut@QAbstractButton@@QAEXABVQKeySequence@@@Z 1002662c     Qt5Widgets:Qt5Widgets.dll
 0002:00000630       __imp_?isChecked@QAbstractButton@@QBE_NXZ 10026630     Qt5Widgets:Qt5Widgets.dll
 0002:00000634       __imp_?setChecked@QAbstractButton@@QAEX_N@Z 10026634     Qt5Widgets:Qt5Widgets.dll
 0002:00000638       __imp_??0QCheckBox@@QAE@PAVQWidget@@@Z 10026638     Qt5Widgets:Qt5Widgets.dll
 0002:0000063c       __imp_??1QCheckBox@@UAE@XZ 1002663c     Qt5Widgets:Qt5Widgets.dll
 0002:00000640       __imp_??0QTabWidget@@QAE@PAVQWidget@@@Z 10026640     Qt5Widgets:Qt5Widgets.dll
 0002:00000644       __imp_??1QTabWidget@@UAE@XZ 10026644     Qt5Widgets:Qt5Widgets.dll
 0002:00000648       __imp_?addTab@QTabWidget@@QAEHPAVQWidget@@ABVQString@@@Z 10026648     Qt5Widgets:Qt5Widgets.dll
 0002:0000064c       __imp_?setTabText@QTabWidget@@QAEXHABVQString@@@Z 1002664c     Qt5Widgets:Qt5Widgets.dll
 0002:00000650       __imp_?indexOf@QTabWidget@@QBEHPAVQWidget@@@Z 10026650     Qt5Widgets:Qt5Widgets.dll
 0002:00000654       __imp_?setCurrentIndex@QTabWidget@@QAEXH@Z 10026654     Qt5Widgets:Qt5Widgets.dll
 0002:00000658       __imp_??0QComboBox@@QAE@PAVQWidget@@@Z 10026658     Qt5Widgets:Qt5Widgets.dll
 0002:0000065c       __imp_??1QComboBox@@UAE@XZ 1002665c     Qt5Widgets:Qt5Widgets.dll
 0002:00000660       __imp_?count@QComboBox@@QBEHXZ 10026660     Qt5Widgets:Qt5Widgets.dll
 0002:00000664       __imp_?currentIndex@QComboBox@@QBEHXZ 10026664     Qt5Widgets:Qt5Widgets.dll
 0002:00000668       __imp_?itemData@QComboBox@@QBE?AVQVariant@@HH@Z 10026668     Qt5Widgets:Qt5Widgets.dll
 0002:0000066c       __imp_?insertItem@QComboBox@@QAEXHABVQIcon@@ABVQString@@ABVQVariant@@@Z 1002666c     Qt5Widgets:Qt5Widgets.dll
 0002:00000670       __imp_?setCurrentIndex@QComboBox@@QAEXH@Z 10026670     Qt5Widgets:Qt5Widgets.dll
 0002:00000674       __imp_??0QDialog@@QAE@PAVQWidget@@V?$QFlags@W4WindowType@Qt@@@@@Z 10026674     Qt5Widgets:Qt5Widgets.dll
 0002:00000678       __imp_??1QDialog@@UAE@XZ   10026678     Qt5Widgets:Qt5Widgets.dll
 0002:0000067c       __imp_?setSizeGripEnabled@QDialog@@QAEX_N@Z 1002667c     Qt5Widgets:Qt5Widgets.dll
 0002:00000680       __imp_?accept@QDialog@@UAEXXZ 10026680     Qt5Widgets:Qt5Widgets.dll
 0002:00000684       __imp_?reject@QDialog@@UAEXXZ 10026684     Qt5Widgets:Qt5Widgets.dll
 0002:00000688       __imp_??0QDialogButtonBox@@QAE@PAVQWidget@@@Z 10026688     Qt5Widgets:Qt5Widgets.dll
 0002:0000068c       __imp_??1QDialogButtonBox@@UAE@XZ 1002668c     Qt5Widgets:Qt5Widgets.dll
 0002:00000690       __imp_?setStandardButtons@QDialogButtonBox@@QAEXV?$QFlags@W4StandardButton@QDialogButtonBox@@@@@Z 10026690     Qt5Widgets:Qt5Widgets.dll
 0002:00000694       __imp_?button@QDialogButtonBox@@QBEPAVQPushButton@@W4StandardButton@1@@Z 10026694     Qt5Widgets:Qt5Widgets.dll
 0002:00000698       __imp_??0QSpacerItem@@QAE@HHW4Policy@QSizePolicy@@0@Z 10026698     Qt5Widgets:Qt5Widgets.dll
 0002:0000069c       __imp_??1QSpacerItem@@UAE@XZ 1002669c     Qt5Widgets:Qt5Widgets.dll
 0002:000006a0       __imp_?setMargin@QLayout@@QAEXH@Z 100266a0     Qt5Widgets:Qt5Widgets.dll
 0002:000006a4       __imp_?setContentsMargins@QLayout@@QAEXHHHH@Z 100266a4     Qt5Widgets:Qt5Widgets.dll
 0002:000006a8       __imp_?setSizeConstraint@QLayout@@QAEXW4SizeConstraint@1@@Z 100266a8     Qt5Widgets:Qt5Widgets.dll
 0002:000006ac       __imp_?addWidget@QBoxLayout@@QAEXPAVQWidget@@HV?$QFlags@W4AlignmentFlag@Qt@@@@@Z 100266ac     Qt5Widgets:Qt5Widgets.dll
 0002:000006b0       __imp_?addLayout@QBoxLayout@@QAEXPAVQLayout@@H@Z 100266b0     Qt5Widgets:Qt5Widgets.dll
 0002:000006b4       __imp_?setSpacing@QBoxLayout@@QAEXH@Z 100266b4     Qt5Widgets:Qt5Widgets.dll
 0002:000006b8       __imp_??0QHBoxLayout@@QAE@XZ 100266b8     Qt5Widgets:Qt5Widgets.dll
 0002:000006bc       __imp_??1QHBoxLayout@@UAE@XZ 100266bc     Qt5Widgets:Qt5Widgets.dll
 0002:000006c0       __imp_??0QVBoxLayout@@QAE@XZ 100266c0     Qt5Widgets:Qt5Widgets.dll
 0002:000006c4       __imp_??0QVBoxLayout@@QAE@PAVQWidget@@@Z 100266c4     Qt5Widgets:Qt5Widgets.dll
 0002:000006c8       __imp_??1QVBoxLayout@@UAE@XZ 100266c8     Qt5Widgets:Qt5Widgets.dll
 0002:000006cc       __imp_??0QGridLayout@@QAE@XZ 100266cc     Qt5Widgets:Qt5Widgets.dll
 0002:000006d0       __imp_??1QGridLayout@@UAE@XZ 100266d0     Qt5Widgets:Qt5Widgets.dll
 0002:000006d4       __imp_?setSpacing@QGridLayout@@QAEXH@Z 100266d4     Qt5Widgets:Qt5Widgets.dll
 0002:000006d8       __imp_?addWidget@QGridLayout@@QAEXPAVQWidget@@HHHHV?$QFlags@W4AlignmentFlag@Qt@@@@@Z 100266d8     Qt5Widgets:Qt5Widgets.dll
 0002:000006dc       __imp_?addLayout@QGridLayout@@QAEXPAVQLayout@@HHHHV?$QFlags@W4AlignmentFlag@Qt@@@@@Z 100266dc     Qt5Widgets:Qt5Widgets.dll
 0002:000006e0       __imp_??0QGroupBox@@QAE@PAVQWidget@@@Z 100266e0     Qt5Widgets:Qt5Widgets.dll
 0002:000006e4       __imp_??1QGroupBox@@UAE@XZ 100266e4     Qt5Widgets:Qt5Widgets.dll
 0002:000006e8       __imp_?setTitle@QGroupBox@@QAEXABVQString@@@Z 100266e8     Qt5Widgets:Qt5Widgets.dll
 0002:000006ec       __imp_?setDefaultSectionSize@QHeaderView@@QAEXH@Z 100266ec     Qt5Widgets:Qt5Widgets.dll
 0002:000006f0       __imp_?setMinimumSectionSize@QHeaderView@@QAEXH@Z 100266f0     Qt5Widgets:Qt5Widgets.dll
 0002:000006f4       __imp_??0QLabel@@QAE@PAVQWidget@@V?$QFlags@W4WindowType@Qt@@@@@Z 100266f4     Qt5Widgets:Qt5Widgets.dll
 0002:000006f8       __imp_??1QLabel@@UAE@XZ    100266f8     Qt5Widgets:Qt5Widgets.dll
 0002:000006fc       __imp_?setText@QLabel@@QAEXABVQString@@@Z 100266fc     Qt5Widgets:Qt5Widgets.dll
 0002:00000700       __imp_??0QPushButton@@QAE@PAVQWidget@@@Z 10026700     Qt5Widgets:Qt5Widgets.dll
 0002:00000704       __imp_??1QPushButton@@UAE@XZ 10026704     Qt5Widgets:Qt5Widgets.dll
 0002:00000708       __imp_?setDefault@QPushButton@@QAEX_N@Z 10026708     Qt5Widgets:Qt5Widgets.dll
 0002:0000070c       __imp_?setFlat@QPushButton@@QAEX_N@Z 1002670c     Qt5Widgets:Qt5Widgets.dll
 0002:00000710       __imp_??0QRadioButton@@QAE@PAVQWidget@@@Z 10026710     Qt5Widgets:Qt5Widgets.dll
 0002:00000714       __imp_??1QRadioButton@@UAE@XZ 10026714     Qt5Widgets:Qt5Widgets.dll
 0002:00000718       __imp_??0QSpinBox@@QAE@PAVQWidget@@@Z 10026718     Qt5Widgets:Qt5Widgets.dll
 0002:0000071c       __imp_??1QSpinBox@@UAE@XZ  1002671c     Qt5Widgets:Qt5Widgets.dll
 0002:00000720       __imp_?value@QSpinBox@@QBEHXZ 10026720     Qt5Widgets:Qt5Widgets.dll
 0002:00000724       __imp_?setSuffix@QSpinBox@@QAEXABVQString@@@Z 10026724     Qt5Widgets:Qt5Widgets.dll
 0002:00000728       __imp_?setSingleStep@QSpinBox@@QAEXH@Z 10026728     Qt5Widgets:Qt5Widgets.dll
 0002:0000072c       __imp_?setMinimum@QSpinBox@@QAEXH@Z 1002672c     Qt5Widgets:Qt5Widgets.dll
 0002:00000730       __imp_?setMaximum@QSpinBox@@QAEXH@Z 10026730     Qt5Widgets:Qt5Widgets.dll
 0002:00000734       __imp_?setValue@QSpinBox@@QAEXH@Z 10026734     Qt5Widgets:Qt5Widgets.dll
 0002:00000738       __imp_??0QTextEdit@@QAE@PAVQWidget@@@Z 10026738     Qt5Widgets:Qt5Widgets.dll
 0002:0000073c       __imp_??1QTextEdit@@UAE@XZ 1002673c     Qt5Widgets:Qt5Widgets.dll
 0002:00000740       __imp_?setReadOnly@QTextEdit@@QAEX_N@Z 10026740     Qt5Widgets:Qt5Widgets.dll
 0002:00000744       __imp_?setText@QTextEdit@@QAEXABVQString@@@Z 10026744     Qt5Widgets:Qt5Widgets.dll
 0002:00000748       __imp_?clear@QTextEdit@@QAEXXZ 10026748     Qt5Widgets:Qt5Widgets.dll
 0002:0000074c       __imp_?header@QTreeView@@QBEPAVQHeaderView@@XZ 1002674c     Qt5Widgets:Qt5Widgets.dll
 0002:00000750       __imp_?setRootIsDecorated@QTreeView@@QAEX_N@Z 10026750     Qt5Widgets:Qt5Widgets.dll
 0002:00000754       __imp_?setSortingEnabled@QTreeView@@QAEX_N@Z 10026754     Qt5Widgets:Qt5Widgets.dll
 0002:00000758       __imp_?sortByColumn@QTreeView@@QAEXH@Z 10026758     Qt5Widgets:Qt5Widgets.dll
 0002:0000075c       __imp_??0QTreeWidgetItem@@QAE@H@Z 1002675c     Qt5Widgets:Qt5Widgets.dll
 0002:00000760       __imp_??1QTreeWidgetItem@@UAE@XZ 10026760     Qt5Widgets:Qt5Widgets.dll
 0002:00000764       __imp_?text@QTreeWidgetItem@@QBE?AVQString@@H@Z 10026764     Qt5Widgets:Qt5Widgets.dll
 0002:00000768       __imp_?setText@QTreeWidgetItem@@QAEXHABVQString@@@Z 10026768     Qt5Widgets:Qt5Widgets.dll
 0002:0000076c       __imp_??0QTreeWidget@@QAE@PAVQWidget@@@Z 1002676c     Qt5Widgets:Qt5Widgets.dll
 0002:00000770       __imp_??1QTreeWidget@@UAE@XZ 10026770     Qt5Widgets:Qt5Widgets.dll
 0002:00000774       __imp_?topLevelItemCount@QTreeWidget@@QBEHXZ 10026774     Qt5Widgets:Qt5Widgets.dll
 0002:00000778       __imp_?addTopLevelItem@QTreeWidget@@QAEXPAVQTreeWidgetItem@@@Z 10026778     Qt5Widgets:Qt5Widgets.dll
 0002:0000077c       __imp_?headerItem@QTreeWidget@@QBEPAVQTreeWidgetItem@@XZ 1002677c     Qt5Widgets:Qt5Widgets.dll
 0002:00000780       __imp_?currentItem@QTreeWidget@@QBEPAVQTreeWidgetItem@@XZ 10026780     Qt5Widgets:Qt5Widgets.dll
 0002:00000784       __imp_?sortColumn@QTreeWidget@@QBEHXZ 10026784     Qt5Widgets:Qt5Widgets.dll
 0002:00000788       __imp_?clear@QTreeWidget@@QAEXXZ 10026788     Qt5Widgets:Qt5Widgets.dll
 0002:0000078c       __imp_?warning@QMessageBox@@SA?AW4StandardButton@1@PAVQWidget@@ABVQString@@1V?$QFlags@W4StandardButton@QMessageBox@@@@W421@@Z 1002678c     Qt5Widgets:Qt5Widgets.dll
 0002:00000790       __imp_?warning@QMessageBox@@SAHPAVQWidget@@ABVQString@@1HHH@Z 10026790     Qt5Widgets:Qt5Widgets.dll
 0002:00000794       __imp_?actionEvent@QWidget@@MAEXPAVQActionEvent@@@Z 10026794     Qt5Widgets:Qt5Widgets.dll
 0002:00000798       __imp_?addItem@QBoxLayout@@UAEXPAVQLayoutItem@@@Z 10026798     Qt5Widgets:Qt5Widgets.dll
 0002:0000079c       __imp_?addItem@QGridLayout@@MAEXPAVQLayoutItem@@@Z 1002679c     Qt5Widgets:Qt5Widgets.dll
 0002:000007a0       __imp_?canInsertFromMimeData@QTextEdit@@MBE_NPBVQMimeData@@@Z 100267a0     Qt5Widgets:Qt5Widgets.dll
 0002:000007a4       __imp_?changeEvent@QAbstractButton@@MAEXPAVQEvent@@@Z 100267a4     Qt5Widgets:Qt5Widgets.dll
 0002:000007a8       __imp_?changeEvent@QAbstractSpinBox@@MAEXPAVQEvent@@@Z 100267a8     Qt5Widgets:Qt5Widgets.dll
 0002:000007ac       __imp_?changeEvent@QComboBox@@MAEXPAVQEvent@@@Z 100267ac     Qt5Widgets:Qt5Widgets.dll
 0002:000007b0       __imp_?changeEvent@QDialogButtonBox@@MAEXPAVQEvent@@@Z 100267b0     Qt5Widgets:Qt5Widgets.dll
 0002:000007b4       __imp_?changeEvent@QFrame@@MAEXPAVQEvent@@@Z 100267b4     Qt5Widgets:Qt5Widgets.dll
 0002:000007b8       __imp_?changeEvent@QGroupBox@@MAEXPAVQEvent@@@Z 100267b8     Qt5Widgets:Qt5Widgets.dll
 0002:000007bc       __imp_?changeEvent@QLabel@@MAEXPAVQEvent@@@Z 100267bc     Qt5Widgets:Qt5Widgets.dll
 0002:000007c0       __imp_?changeEvent@QTabWidget@@MAEXPAVQEvent@@@Z 100267c0     Qt5Widgets:Qt5Widgets.dll
 0002:000007c4       __imp_?changeEvent@QTextEdit@@MAEXPAVQEvent@@@Z 100267c4     Qt5Widgets:Qt5Widgets.dll
 0002:000007c8       __imp_?changeEvent@QWidget@@MAEXPAVQEvent@@@Z 100267c8     Qt5Widgets:Qt5Widgets.dll
 0002:000007cc       __imp_?checkStateSet@QAbstractButton@@MAEXXZ 100267cc     Qt5Widgets:Qt5Widgets.dll
 0002:000007d0       __imp_?checkStateSet@QCheckBox@@MAEXXZ 100267d0     Qt5Widgets:Qt5Widgets.dll
 0002:000007d4       __imp_?childEvent@QGroupBox@@MAEXPAVQChildEvent@@@Z 100267d4     Qt5Widgets:Qt5Widgets.dll
 0002:000007d8       __imp_?childEvent@QLayout@@MAEXPAVQChildEvent@@@Z 100267d8     Qt5Widgets:Qt5Widgets.dll
 0002:000007dc       __imp_?clear@QAbstractSpinBox@@UAEXXZ 100267dc     Qt5Widgets:Qt5Widgets.dll
 0002:000007e0       __imp_?clone@QTreeWidgetItem@@UBEPAV1@XZ 100267e0     Qt5Widgets:Qt5Widgets.dll
 0002:000007e4       __imp_?closeEditor@QAbstractItemView@@MAEXPAVQWidget@@W4EndEditHint@QAbstractItemDelegate@@@Z 100267e4     Qt5Widgets:Qt5Widgets.dll
 0002:000007e8       __imp_?closeEvent@QAbstractSpinBox@@MAEXPAVQCloseEvent@@@Z 100267e8     Qt5Widgets:Qt5Widgets.dll
 0002:000007ec       __imp_?closeEvent@QDialog@@MAEXPAVQCloseEvent@@@Z 100267ec     Qt5Widgets:Qt5Widgets.dll
 0002:000007f0       __imp_?closeEvent@QWidget@@MAEXPAVQCloseEvent@@@Z 100267f0     Qt5Widgets:Qt5Widgets.dll
 0002:000007f4       __imp_?commitData@QAbstractItemView@@MAEXPAVQWidget@@@Z 100267f4     Qt5Widgets:Qt5Widgets.dll
 0002:000007f8       __imp_?contextMenuEvent@QAbstractScrollArea@@MAEXPAVQContextMenuEvent@@@Z 100267f8     Qt5Widgets:Qt5Widgets.dll
 0002:000007fc       __imp_?contextMenuEvent@QAbstractSpinBox@@MAEXPAVQContextMenuEvent@@@Z 100267fc     Qt5Widgets:Qt5Widgets.dll
 0002:00000800       __imp_?contextMenuEvent@QComboBox@@MAEXPAVQContextMenuEvent@@@Z 10026800     Qt5Widgets:Qt5Widgets.dll
 0002:00000804       __imp_?contextMenuEvent@QDialog@@MAEXPAVQContextMenuEvent@@@Z 10026804     Qt5Widgets:Qt5Widgets.dll
 0002:00000808       __imp_?contextMenuEvent@QLabel@@MAEXPAVQContextMenuEvent@@@Z 10026808     Qt5Widgets:Qt5Widgets.dll
 0002:0000080c       __imp_?contextMenuEvent@QTextEdit@@MAEXPAVQContextMenuEvent@@@Z 1002680c     Qt5Widgets:Qt5Widgets.dll
 0002:00000810       __imp_?contextMenuEvent@QWidget@@MAEXPAVQContextMenuEvent@@@Z 10026810     Qt5Widgets:Qt5Widgets.dll
 0002:00000814       __imp_?controlTypes@QLayout@@UBE?AV?$QFlags@W4ControlType@QSizePolicy@@@@XZ 10026814     Qt5Widgets:Qt5Widgets.dll
 0002:00000818       __imp_?controlTypes@QLayoutItem@@UBE?AV?$QFlags@W4ControlType@QSizePolicy@@@@XZ 10026818     Qt5Widgets:Qt5Widgets.dll
 0002:0000081c       __imp_?count@QBoxLayout@@UBEHXZ 1002681c     Qt5Widgets:Qt5Widgets.dll
 0002:00000820       __imp_?count@QGridLayout@@UBEHXZ 10026820     Qt5Widgets:Qt5Widgets.dll
 0002:00000824       __imp_?createMimeDataFromSelection@QTextEdit@@MBEPAVQMimeData@@XZ 10026824     Qt5Widgets:Qt5Widgets.dll
 0002:00000828       __imp_?currentChanged@QTreeView@@MAEXABVQModelIndex@@0@Z 10026828     Qt5Widgets:Qt5Widgets.dll
 0002:0000082c       __imp_?data@QTreeWidgetItem@@UBE?AVQVariant@@HH@Z 1002682c     Qt5Widgets:Qt5Widgets.dll
 0002:00000830       __imp_?dataChanged@QTreeView@@UAEXABVQModelIndex@@0ABV?$QVector@H@@@Z 10026830     Qt5Widgets:Qt5Widgets.dll
 0002:00000834       __imp_?devType@QWidget@@UBEHXZ 10026834     Qt5Widgets:Qt5Widgets.dll
 0002:00000838       __imp_?doItemsLayout@QTreeView@@UAEXXZ 10026838     Qt5Widgets:Qt5Widgets.dll
 0002:0000083c       __imp_?doSetTextCursor@QTextEdit@@MAEXABVQTextCursor@@@Z 1002683c     Qt5Widgets:Qt5Widgets.dll
 0002:00000840       __imp_?done@QDialog@@UAEXH@Z 10026840     Qt5Widgets:Qt5Widgets.dll
 0002:00000844       __imp_?dragEnterEvent@QAbstractItemView@@MAEXPAVQDragEnterEvent@@@Z 10026844     Qt5Widgets:Qt5Widgets.dll
 0002:00000848       __imp_?dragEnterEvent@QTextEdit@@MAEXPAVQDragEnterEvent@@@Z 10026848     Qt5Widgets:Qt5Widgets.dll
 0002:0000084c       __imp_?dragEnterEvent@QWidget@@MAEXPAVQDragEnterEvent@@@Z 1002684c     Qt5Widgets:Qt5Widgets.dll
 0002:00000850       __imp_?dragLeaveEvent@QAbstractItemView@@MAEXPAVQDragLeaveEvent@@@Z 10026850     Qt5Widgets:Qt5Widgets.dll
 0002:00000854       __imp_?dragLeaveEvent@QTextEdit@@MAEXPAVQDragLeaveEvent@@@Z 10026854     Qt5Widgets:Qt5Widgets.dll
 0002:00000858       __imp_?dragLeaveEvent@QWidget@@MAEXPAVQDragLeaveEvent@@@Z 10026858     Qt5Widgets:Qt5Widgets.dll
 0002:0000085c       __imp_?dragMoveEvent@QTextEdit@@MAEXPAVQDragMoveEvent@@@Z 1002685c     Qt5Widgets:Qt5Widgets.dll
 0002:00000860       __imp_?dragMoveEvent@QTreeView@@MAEXPAVQDragMoveEvent@@@Z 10026860     Qt5Widgets:Qt5Widgets.dll
 0002:00000864       __imp_?dragMoveEvent@QWidget@@MAEXPAVQDragMoveEvent@@@Z 10026864     Qt5Widgets:Qt5Widgets.dll
 0002:00000868       __imp_?drawBranches@QTreeView@@MBEXPAVQPainter@@ABVQRect@@ABVQModelIndex@@@Z 10026868     Qt5Widgets:Qt5Widgets.dll
 0002:0000086c       __imp_?drawRow@QTreeView@@MBEXPAVQPainter@@ABVQStyleOptionViewItem@@ABVQModelIndex@@@Z 1002686c     Qt5Widgets:Qt5Widgets.dll
 0002:00000870       __imp_?dropEvent@QTextEdit@@MAEXPAVQDropEvent@@@Z 10026870     Qt5Widgets:Qt5Widgets.dll
 0002:00000874       __imp_?dropEvent@QTreeWidget@@MAEXPAVQDropEvent@@@Z 10026874     Qt5Widgets:Qt5Widgets.dll
 0002:00000878       __imp_?dropEvent@QWidget@@MAEXPAVQDropEvent@@@Z 10026878     Qt5Widgets:Qt5Widgets.dll
 0002:0000087c       __imp_?dropMimeData@QTreeWidget@@MAE_NPAVQTreeWidgetItem@@HPBVQMimeData@@W4DropAction@Qt@@@Z 1002687c     Qt5Widgets:Qt5Widgets.dll
 0002:00000880       __imp_?edit@QAbstractItemView@@MAE_NABVQModelIndex@@W4EditTrigger@1@PAVQEvent@@@Z 10026880     Qt5Widgets:Qt5Widgets.dll
 0002:00000884       __imp_?editorDestroyed@QAbstractItemView@@MAEXPAVQObject@@@Z 10026884     Qt5Widgets:Qt5Widgets.dll
 0002:00000888       __imp_?enterEvent@QWidget@@MAEXPAVQEvent@@@Z 10026888     Qt5Widgets:Qt5Widgets.dll
 0002:0000088c       __imp_?event@QCheckBox@@MAE_NPAVQEvent@@@Z 1002688c     Qt5Widgets:Qt5Widgets.dll
 0002:00000890       __imp_?event@QComboBox@@UAE_NPAVQEvent@@@Z 10026890     Qt5Widgets:Qt5Widgets.dll
 0002:00000894       __imp_?event@QDialogButtonBox@@MAE_NPAVQEvent@@@Z 10026894     Qt5Widgets:Qt5Widgets.dll
 0002:00000898       __imp_?event@QGroupBox@@MAE_NPAVQEvent@@@Z 10026898     Qt5Widgets:Qt5Widgets.dll
 0002:0000089c       __imp_?event@QLabel@@MAE_NPAVQEvent@@@Z 1002689c     Qt5Widgets:Qt5Widgets.dll
 0002:000008a0       __imp_?event@QPushButton@@MAE_NPAVQEvent@@@Z 100268a0     Qt5Widgets:Qt5Widgets.dll
 0002:000008a4       __imp_?event@QRadioButton@@MAE_NPAVQEvent@@@Z 100268a4     Qt5Widgets:Qt5Widgets.dll
 0002:000008a8       __imp_?event@QSpinBox@@MAE_NPAVQEvent@@@Z 100268a8     Qt5Widgets:Qt5Widgets.dll
 0002:000008ac       __imp_?event@QTabWidget@@MAE_NPAVQEvent@@@Z 100268ac     Qt5Widgets:Qt5Widgets.dll
 0002:000008b0       __imp_?event@QTextEdit@@MAE_NPAVQEvent@@@Z 100268b0     Qt5Widgets:Qt5Widgets.dll
 0002:000008b4       __imp_?event@QTreeWidget@@MAE_NPAVQEvent@@@Z 100268b4     Qt5Widgets:Qt5Widgets.dll
 0002:000008b8       __imp_?event@QWidget@@MAE_NPAVQEvent@@@Z 100268b8     Qt5Widgets:Qt5Widgets.dll
 0002:000008bc       __imp_?eventFilter@QAbstractScrollArea@@MAE_NPAVQObject@@PAVQEvent@@@Z 100268bc     Qt5Widgets:Qt5Widgets.dll
 0002:000008c0       __imp_?exec@QDialog@@UAEHXZ 100268c0     Qt5Widgets:Qt5Widgets.dll
 0002:000008c4       __imp_?expandingDirections@QBoxLayout@@UBE?AV?$QFlags@W4Orientation@Qt@@@@XZ 100268c4     Qt5Widgets:Qt5Widgets.dll
 0002:000008c8       __imp_?expandingDirections@QGridLayout@@UBE?AV?$QFlags@W4Orientation@Qt@@@@XZ 100268c8     Qt5Widgets:Qt5Widgets.dll
 0002:000008cc       __imp_?expandingDirections@QSpacerItem@@UBE?AV?$QFlags@W4Orientation@Qt@@@@XZ 100268cc     Qt5Widgets:Qt5Widgets.dll
 0002:000008d0       __imp_?fixup@QSpinBox@@MBEXAAVQString@@@Z 100268d0     Qt5Widgets:Qt5Widgets.dll
 0002:000008d4       __imp_?focusInEvent@QAbstractButton@@MAEXPAVQFocusEvent@@@Z 100268d4     Qt5Widgets:Qt5Widgets.dll
 0002:000008d8       __imp_?focusInEvent@QAbstractItemView@@MAEXPAVQFocusEvent@@@Z 100268d8     Qt5Widgets:Qt5Widgets.dll
 0002:000008dc       __imp_?focusInEvent@QAbstractSpinBox@@MAEXPAVQFocusEvent@@@Z 100268dc     Qt5Widgets:Qt5Widgets.dll
 0002:000008e0       __imp_?focusInEvent@QComboBox@@MAEXPAVQFocusEvent@@@Z 100268e0     Qt5Widgets:Qt5Widgets.dll
 0002:000008e4       __imp_?focusInEvent@QGroupBox@@MAEXPAVQFocusEvent@@@Z 100268e4     Qt5Widgets:Qt5Widgets.dll
 0002:000008e8       __imp_?focusInEvent@QLabel@@MAEXPAVQFocusEvent@@@Z 100268e8     Qt5Widgets:Qt5Widgets.dll
 0002:000008ec       __imp_?focusInEvent@QPushButton@@MAEXPAVQFocusEvent@@@Z 100268ec     Qt5Widgets:Qt5Widgets.dll
 0002:000008f0       __imp_?focusInEvent@QTextEdit@@MAEXPAVQFocusEvent@@@Z 100268f0     Qt5Widgets:Qt5Widgets.dll
 0002:000008f4       __imp_?focusInEvent@QWidget@@MAEXPAVQFocusEvent@@@Z 100268f4     Qt5Widgets:Qt5Widgets.dll
 0002:000008f8       __imp_?focusNextPrevChild@QAbstractItemView@@MAE_N_N@Z 100268f8     Qt5Widgets:Qt5Widgets.dll
 0002:000008fc       __imp_?focusNextPrevChild@QLabel@@MAE_N_N@Z 100268fc     Qt5Widgets:Qt5Widgets.dll
 0002:00000900       __imp_?focusNextPrevChild@QTextEdit@@MAE_N_N@Z 10026900     Qt5Widgets:Qt5Widgets.dll
 0002:00000904       __imp_?focusNextPrevChild@QWidget@@MAE_N_N@Z 10026904     Qt5Widgets:Qt5Widgets.dll
 0002:00000908       __imp_?focusOutEvent@QAbstractButton@@MAEXPAVQFocusEvent@@@Z 10026908     Qt5Widgets:Qt5Widgets.dll
 0002:0000090c       __imp_?focusOutEvent@QAbstractItemView@@MAEXPAVQFocusEvent@@@Z 1002690c     Qt5Widgets:Qt5Widgets.dll
 0002:00000910       __imp_?focusOutEvent@QAbstractSpinBox@@MAEXPAVQFocusEvent@@@Z 10026910     Qt5Widgets:Qt5Widgets.dll
 0002:00000914       __imp_?focusOutEvent@QComboBox@@MAEXPAVQFocusEvent@@@Z 10026914     Qt5Widgets:Qt5Widgets.dll
 0002:00000918       __imp_?focusOutEvent@QLabel@@MAEXPAVQFocusEvent@@@Z 10026918     Qt5Widgets:Qt5Widgets.dll
 0002:0000091c       __imp_?focusOutEvent@QPushButton@@MAEXPAVQFocusEvent@@@Z 1002691c     Qt5Widgets:Qt5Widgets.dll
 0002:00000920       __imp_?focusOutEvent@QTextEdit@@MAEXPAVQFocusEvent@@@Z 10026920     Qt5Widgets:Qt5Widgets.dll
 0002:00000924       __imp_?focusOutEvent@QWidget@@MAEXPAVQFocusEvent@@@Z 10026924     Qt5Widgets:Qt5Widgets.dll
 0002:00000928       __imp_?geometry@QLayout@@UBE?AVQRect@@XZ 10026928     Qt5Widgets:Qt5Widgets.dll
 0002:0000092c       __imp_?geometry@QSpacerItem@@UBE?AVQRect@@XZ 1002692c     Qt5Widgets:Qt5Widgets.dll
 0002:00000930       __imp_?hasHeightForWidth@QBoxLayout@@UBE_NXZ 10026930     Qt5Widgets:Qt5Widgets.dll
 0002:00000934       __imp_?hasHeightForWidth@QGridLayout@@UBE_NXZ 10026934     Qt5Widgets:Qt5Widgets.dll
 0002:00000938       __imp_?hasHeightForWidth@QLayoutItem@@UBE_NXZ 10026938     Qt5Widgets:Qt5Widgets.dll
 0002:0000093c       __imp_?hasHeightForWidth@QTabWidget@@UBE_NXZ 1002693c     Qt5Widgets:Qt5Widgets.dll
 0002:00000940       __imp_?hasHeightForWidth@QWidget@@UBE_NXZ 10026940     Qt5Widgets:Qt5Widgets.dll
 0002:00000944       __imp_?heightForWidth@QBoxLayout@@UBEHH@Z 10026944     Qt5Widgets:Qt5Widgets.dll
 0002:00000948       __imp_?heightForWidth@QGridLayout@@UBEHH@Z 10026948     Qt5Widgets:Qt5Widgets.dll
 0002:0000094c       __imp_?heightForWidth@QLabel@@UBEHH@Z 1002694c     Qt5Widgets:Qt5Widgets.dll
 0002:00000950       __imp_?heightForWidth@QLayoutItem@@UBEHH@Z 10026950     Qt5Widgets:Qt5Widgets.dll
 0002:00000954       __imp_?heightForWidth@QTabWidget@@UBEHH@Z 10026954     Qt5Widgets:Qt5Widgets.dll
 0002:00000958       __imp_?heightForWidth@QWidget@@UBEHH@Z 10026958     Qt5Widgets:Qt5Widgets.dll
 0002:0000095c       __imp_?hideEvent@QAbstractSpinBox@@MAEXPAVQHideEvent@@@Z 1002695c     Qt5Widgets:Qt5Widgets.dll
 0002:00000960       __imp_?hideEvent@QComboBox@@MAEXPAVQHideEvent@@@Z 10026960     Qt5Widgets:Qt5Widgets.dll
 0002:00000964       __imp_?hideEvent@QWidget@@MAEXPAVQHideEvent@@@Z 10026964     Qt5Widgets:Qt5Widgets.dll
 0002:00000968       __imp_?hidePopup@QComboBox@@UAEXXZ 10026968     Qt5Widgets:Qt5Widgets.dll
 0002:0000096c       __imp_?hitButton@QAbstractButton@@MBE_NABVQPoint@@@Z 1002696c     Qt5Widgets:Qt5Widgets.dll
 0002:00000970       __imp_?hitButton@QCheckBox@@MBE_NABVQPoint@@@Z 10026970     Qt5Widgets:Qt5Widgets.dll
 0002:00000974       __imp_?hitButton@QRadioButton@@MBE_NABVQPoint@@@Z 10026974     Qt5Widgets:Qt5Widgets.dll
 0002:00000978       __imp_?horizontalOffset@QTreeView@@MBEHXZ 10026978     Qt5Widgets:Qt5Widgets.dll
 0002:0000097c       __imp_?horizontalScrollbarAction@QTreeView@@MAEXH@Z 1002697c     Qt5Widgets:Qt5Widgets.dll
 0002:00000980       __imp_?horizontalScrollbarValueChanged@QAbstractItemView@@MAEXH@Z 10026980     Qt5Widgets:Qt5Widgets.dll
 0002:00000984       __imp_?indexAt@QTreeView@@UBE?AVQModelIndex@@ABVQPoint@@@Z 10026984     Qt5Widgets:Qt5Widgets.dll
 0002:00000988       __imp_?indexOf@QLayout@@UBEHPAVQWidget@@@Z 10026988     Qt5Widgets:Qt5Widgets.dll
 0002:0000098c       __imp_?initPainter@QWidget@@MBEXPAVQPainter@@@Z 1002698c     Qt5Widgets:Qt5Widgets.dll
 0002:00000990       __imp_?inputMethodEvent@QAbstractItemView@@MAEXPAVQInputMethodEvent@@@Z 10026990     Qt5Widgets:Qt5Widgets.dll
 0002:00000994       __imp_?inputMethodEvent@QComboBox@@MAEXPAVQInputMethodEvent@@@Z 10026994     Qt5Widgets:Qt5Widgets.dll
 0002:00000998       __imp_?inputMethodEvent@QTextEdit@@MAEXPAVQInputMethodEvent@@@Z 10026998     Qt5Widgets:Qt5Widgets.dll
 0002:0000099c       __imp_?inputMethodEvent@QWidget@@MAEXPAVQInputMethodEvent@@@Z 1002699c     Qt5Widgets:Qt5Widgets.dll
 0002:000009a0       __imp_?inputMethodQuery@QAbstractItemView@@UBE?AVQVariant@@W4InputMethodQuery@Qt@@@Z 100269a0     Qt5Widgets:Qt5Widgets.dll
 0002:000009a4       __imp_?inputMethodQuery@QAbstractSpinBox@@UBE?AVQVariant@@W4InputMethodQuery@Qt@@@Z 100269a4     Qt5Widgets:Qt5Widgets.dll
 0002:000009a8       __imp_?inputMethodQuery@QComboBox@@UBE?AVQVariant@@W4InputMethodQuery@Qt@@@Z 100269a8     Qt5Widgets:Qt5Widgets.dll
 0002:000009ac       __imp_?inputMethodQuery@QTextEdit@@UBE?AVQVariant@@W4InputMethodQuery@Qt@@@Z 100269ac     Qt5Widgets:Qt5Widgets.dll
 0002:000009b0       __imp_?inputMethodQuery@QWidget@@UBE?AVQVariant@@W4InputMethodQuery@Qt@@@Z 100269b0     Qt5Widgets:Qt5Widgets.dll
 0002:000009b4       __imp_?insertFromMimeData@QTextEdit@@MAEXPBVQMimeData@@@Z 100269b4     Qt5Widgets:Qt5Widgets.dll
 0002:000009b8       __imp_?invalidate@QBoxLayout@@UAEXXZ 100269b8     Qt5Widgets:Qt5Widgets.dll
 0002:000009bc       __imp_?invalidate@QGridLayout@@UAEXXZ 100269bc     Qt5Widgets:Qt5Widgets.dll
 0002:000009c0       __imp_?invalidate@QLayoutItem@@UAEXXZ 100269c0     Qt5Widgets:Qt5Widgets.dll
 0002:000009c4       __imp_?isEmpty@QLayout@@UBE_NXZ 100269c4     Qt5Widgets:Qt5Widgets.dll
 0002:000009c8       __imp_?isEmpty@QSpacerItem@@UBE_NXZ 100269c8     Qt5Widgets:Qt5Widgets.dll
 0002:000009cc       __imp_?isIndexHidden@QTreeView@@MBE_NABVQModelIndex@@@Z 100269cc     Qt5Widgets:Qt5Widgets.dll
 0002:000009d0       __imp_?itemAt@QBoxLayout@@UBEPAVQLayoutItem@@H@Z 100269d0     Qt5Widgets:Qt5Widgets.dll
 0002:000009d4       __imp_?itemAt@QGridLayout@@UBEPAVQLayoutItem@@H@Z 100269d4     Qt5Widgets:Qt5Widgets.dll
 0002:000009d8       __imp_?keyPressEvent@QAbstractButton@@MAEXPAVQKeyEvent@@@Z 100269d8     Qt5Widgets:Qt5Widgets.dll
 0002:000009dc       __imp_?keyPressEvent@QAbstractSpinBox@@MAEXPAVQKeyEvent@@@Z 100269dc     Qt5Widgets:Qt5Widgets.dll
 0002:000009e0       __imp_?keyPressEvent@QComboBox@@MAEXPAVQKeyEvent@@@Z 100269e0     Qt5Widgets:Qt5Widgets.dll
 0002:000009e4       __imp_?keyPressEvent@QDialog@@MAEXPAVQKeyEvent@@@Z 100269e4     Qt5Widgets:Qt5Widgets.dll
 0002:000009e8       __imp_?keyPressEvent@QLabel@@MAEXPAVQKeyEvent@@@Z 100269e8     Qt5Widgets:Qt5Widgets.dll
 0002:000009ec       __imp_?keyPressEvent@QPushButton@@MAEXPAVQKeyEvent@@@Z 100269ec     Qt5Widgets:Qt5Widgets.dll
 0002:000009f0       __imp_?keyPressEvent@QTabWidget@@MAEXPAVQKeyEvent@@@Z 100269f0     Qt5Widgets:Qt5Widgets.dll
 0002:000009f4       __imp_?keyPressEvent@QTextEdit@@MAEXPAVQKeyEvent@@@Z 100269f4     Qt5Widgets:Qt5Widgets.dll
 0002:000009f8       __imp_?keyPressEvent@QTreeView@@MAEXPAVQKeyEvent@@@Z 100269f8     Qt5Widgets:Qt5Widgets.dll
 0002:000009fc       __imp_?keyPressEvent@QWidget@@MAEXPAVQKeyEvent@@@Z 100269fc     Qt5Widgets:Qt5Widgets.dll
 0002:00000a00       __imp_?keyReleaseEvent@QAbstractButton@@MAEXPAVQKeyEvent@@@Z 10026a00     Qt5Widgets:Qt5Widgets.dll
 0002:00000a04       __imp_?keyReleaseEvent@QAbstractSpinBox@@MAEXPAVQKeyEvent@@@Z 10026a04     Qt5Widgets:Qt5Widgets.dll
 0002:00000a08       __imp_?keyReleaseEvent@QComboBox@@MAEXPAVQKeyEvent@@@Z 10026a08     Qt5Widgets:Qt5Widgets.dll
 0002:00000a0c       __imp_?keyReleaseEvent@QTextEdit@@MAEXPAVQKeyEvent@@@Z 10026a0c     Qt5Widgets:Qt5Widgets.dll
 0002:00000a10       __imp_?keyReleaseEvent@QWidget@@MAEXPAVQKeyEvent@@@Z 10026a10     Qt5Widgets:Qt5Widgets.dll
 0002:00000a14       __imp_?keyboardSearch@QTreeView@@UAEXABVQString@@@Z 10026a14     Qt5Widgets:Qt5Widgets.dll
 0002:00000a18       __imp_?layout@QLayout@@UAEPAV1@XZ 10026a18     Qt5Widgets:Qt5Widgets.dll
 0002:00000a1c       __imp_?layout@QLayoutItem@@UAEPAVQLayout@@XZ 10026a1c     Qt5Widgets:Qt5Widgets.dll
 0002:00000a20       __imp_?leaveEvent@QWidget@@MAEXPAVQEvent@@@Z 10026a20     Qt5Widgets:Qt5Widgets.dll
 0002:00000a24       __imp_?loadResource@QTextEdit@@UAE?AVQVariant@@HABVQUrl@@@Z 10026a24     Qt5Widgets:Qt5Widgets.dll
 0002:00000a28       __imp_?maximumSize@QBoxLayout@@UBE?AVQSize@@XZ 10026a28     Qt5Widgets:Qt5Widgets.dll
 0002:00000a2c       __imp_?maximumSize@QGridLayout@@UBE?AVQSize@@XZ 10026a2c     Qt5Widgets:Qt5Widgets.dll
 0002:00000a30       __imp_?maximumSize@QSpacerItem@@UBE?AVQSize@@XZ 10026a30     Qt5Widgets:Qt5Widgets.dll
 0002:00000a34       __imp_?metaObject@QCheckBox@@UBEPBUQMetaObject@@XZ 10026a34     Qt5Widgets:Qt5Widgets.dll
 0002:00000a38       __imp_?metaObject@QComboBox@@UBEPBUQMetaObject@@XZ 10026a38     Qt5Widgets:Qt5Widgets.dll
 0002:00000a3c       __imp_?metaObject@QDialogButtonBox@@UBEPBUQMetaObject@@XZ 10026a3c     Qt5Widgets:Qt5Widgets.dll
 0002:00000a40       __imp_?metaObject@QGridLayout@@UBEPBUQMetaObject@@XZ 10026a40     Qt5Widgets:Qt5Widgets.dll
 0002:00000a44       __imp_?metaObject@QGroupBox@@UBEPBUQMetaObject@@XZ 10026a44     Qt5Widgets:Qt5Widgets.dll
 0002:00000a48       __imp_?metaObject@QHBoxLayout@@UBEPBUQMetaObject@@XZ 10026a48     Qt5Widgets:Qt5Widgets.dll
 0002:00000a4c       __imp_?metaObject@QLabel@@UBEPBUQMetaObject@@XZ 10026a4c     Qt5Widgets:Qt5Widgets.dll
 0002:00000a50       __imp_?metaObject@QPushButton@@UBEPBUQMetaObject@@XZ 10026a50     Qt5Widgets:Qt5Widgets.dll
 0002:00000a54       __imp_?metaObject@QRadioButton@@UBEPBUQMetaObject@@XZ 10026a54     Qt5Widgets:Qt5Widgets.dll
 0002:00000a58       __imp_?metaObject@QSpinBox@@UBEPBUQMetaObject@@XZ 10026a58     Qt5Widgets:Qt5Widgets.dll
 0002:00000a5c       __imp_?metaObject@QTabWidget@@UBEPBUQMetaObject@@XZ 10026a5c     Qt5Widgets:Qt5Widgets.dll
 0002:00000a60       __imp_?metaObject@QTextEdit@@UBEPBUQMetaObject@@XZ 10026a60     Qt5Widgets:Qt5Widgets.dll
 0002:00000a64       __imp_?metaObject@QTreeWidget@@UBEPBUQMetaObject@@XZ 10026a64     Qt5Widgets:Qt5Widgets.dll
 0002:00000a68       __imp_?metaObject@QVBoxLayout@@UBEPBUQMetaObject@@XZ 10026a68     Qt5Widgets:Qt5Widgets.dll
 0002:00000a6c       __imp_?metaObject@QWidget@@UBEPBUQMetaObject@@XZ 10026a6c     Qt5Widgets:Qt5Widgets.dll
 0002:00000a70       __imp_?metric@QWidget@@MBEHW4PaintDeviceMetric@QPaintDevice@@@Z 10026a70     Qt5Widgets:Qt5Widgets.dll
 0002:00000a74       __imp_?mimeData@QTreeWidget@@MBEPAVQMimeData@@V?$QList@PAVQTreeWidgetItem@@@@@Z 10026a74     Qt5Widgets:Qt5Widgets.dll
 0002:00000a78       __imp_?mimeTypes@QTreeWidget@@MBE?AVQStringList@@XZ 10026a78     Qt5Widgets:Qt5Widgets.dll
 0002:00000a7c       __imp_?minimumHeightForWidth@QBoxLayout@@UBEHH@Z 10026a7c     Qt5Widgets:Qt5Widgets.dll
 0002:00000a80       __imp_?minimumHeightForWidth@QGridLayout@@UBEHH@Z 10026a80     Qt5Widgets:Qt5Widgets.dll
 0002:00000a84       __imp_?minimumHeightForWidth@QLayoutItem@@UBEHH@Z 10026a84     Qt5Widgets:Qt5Widgets.dll
 0002:00000a88       __imp_?minimumSize@QBoxLayout@@UBE?AVQSize@@XZ 10026a88     Qt5Widgets:Qt5Widgets.dll
 0002:00000a8c       __imp_?minimumSize@QGridLayout@@UBE?AVQSize@@XZ 10026a8c     Qt5Widgets:Qt5Widgets.dll
 0002:00000a90       \177Qt5Widgets_NULL_THUNK_DATA 10026a90     Qt5Widgets:Qt5Widgets.dll
 0002:00000a94       __imp_?attribute@QDomElement@@QBE?AVQString@@ABV2@0@Z 10026a94     Qt5Xml:Qt5Xml.dll
 0002:00000a98       \177Qt5Xml_NULL_THUNK_DATA 10026a98     Qt5Xml:Qt5Xml.dll
 0002:00000a9c       __imp_?staticMetaObject@ORFFindTask@U2@@2UQMetaObject@@B 10026a9c     U2Algorithm:U2Algorithm.dll
 0002:00000aa0       __imp_?toTable@ORFFindResult@U2@@SA?AV?$QList@V?$QSharedDataPointer@VAnnotationData@U2@@@@@@ABV?$QList@VORFFindResult@U2@@@@ABVQString@@@Z 10026aa0     U2Algorithm:U2Algorithm.dll
 0002:00000aa4       __imp_?STRAND_BOTH@ORFAlgorithmSettings@U2@@2VQString@@B 10026aa4     U2Algorithm:U2Algorithm.dll
 0002:00000aa8       __imp_?getStrandByStringId@ORFAlgorithmSettings@U2@@SA?AW4ORFAlgorithmStrand@2@ABVQString@@@Z 10026aa8     U2Algorithm:U2Algorithm.dll
 0002:00000aac       __imp_?getStrandStringId@ORFAlgorithmSettings@U2@@SA?AVQString@@W4ORFAlgorithmStrand@2@@Z 10026aac     U2Algorithm:U2Algorithm.dll
 0002:00000ab0       __imp_?toAnnotation@ORFFindResult@U2@@QBE?AV?$QSharedDataPointer@VAnnotationData@U2@@@@ABVQString@@@Z 10026ab0     U2Algorithm:U2Algorithm.dll
 0002:00000ab4       __imp_?ANNOTATION_GROUP_NAME@ORFAlgorithmSettings@U2@@2VQString@@B 10026ab4     U2Algorithm:U2Algorithm.dll
 0002:00000ab8       __imp_?run@ORFFindTask@U2@@UAEXXZ 10026ab8     U2Algorithm:U2Algorithm.dll
 0002:00000abc       __imp_?qt_metacast@ORFFindTask@U2@@UAEPAXPBD@Z 10026abc     U2Algorithm:U2Algorithm.dll
 0002:00000ac0       __imp_?qt_metacall@ORFFindTask@U2@@UAEHW4Call@QMetaObject@@HPAPAX@Z 10026ac0     U2Algorithm:U2Algorithm.dll
 0002:00000ac4       __imp_?onResult@ORFFindTask@U2@@UAEXABVORFFindResult@2@AAVU2OpStatus@2@@Z 10026ac4     U2Algorithm:U2Algorithm.dll
 0002:00000ac8       __imp_?metaObject@ORFFindTask@U2@@UBEPBUQMetaObject@@XZ 10026ac8     U2Algorithm:U2Algorithm.dll
 0002:00000acc       __imp_??1ORFFindTask@U2@@UAE@XZ 10026acc     U2Algorithm:U2Algorithm.dll
 0002:00000ad0       __imp_?popResults@ORFFindTask@U2@@QAE?AV?$QList@VORFFindResult@U2@@@@XZ 10026ad0     U2Algorithm:U2Algorithm.dll
 0002:00000ad4       __imp_??0ORFFindTask@U2@@QAE@ABVORFAlgorithmSettings@1@ABVU2EntityRef@1@@Z 10026ad4     U2Algorithm:U2Algorithm.dll
 0002:00000ad8       \177U2Algorithm_NULL_THUNK_DATA 10026ad8     U2Algorithm:U2Algorithm.dll
 0002:00000adc       __imp_?staticMetaObject@AutoAnnotationsUpdater@U2@@2UQMetaObject@@B 10026adc     U2Core:U2Core.dll
 0002:00000ae0       __imp_?qt_metacall@AutoAnnotationsUpdater@U2@@UAEHW4Call@QMetaObject@@HPAPAX@Z 10026ae0     U2Core:U2Core.dll
 0002:00000ae4       __imp_?qt_metacast@AutoAnnotationsUpdater@U2@@UAEPAXPBD@Z 10026ae4     U2Core:U2Core.dll
 0002:00000ae8       __imp_?staticMetaObject@Plugin@U2@@2UQMetaObject@@B 10026ae8     U2Core:U2Core.dll
 0002:00000aec       __imp_?qt_metacall@Plugin@U2@@UAEHW4Call@QMetaObject@@HPAPAX@Z 10026aec     U2Core:U2Core.dll
 0002:00000af0       __imp_?qt_metacast@Plugin@U2@@UAEPAXPBD@Z 10026af0     U2Core:U2Core.dll
 0002:00000af4       __imp_?staticMetaObject@Task@U2@@2UQMetaObject@@B 10026af4     U2Core:U2Core.dll
 0002:00000af8       __imp_?getSequenceName@U2SequenceObject@U2@@QBE?AVQString@@XZ 10026af8     U2Core:U2Core.dll
 0002:00000afc       __imp_?runScript@ScriptTask@U2@@SA?AVQScriptValue@@PAVQScriptEngine@@ABV?$QMap@VQString@@VQScriptValue@@@@ABVQString@@AAVTaskStateInfo@2@@Z 10026afc     U2Core:U2Core.dll
 0002:00000b00       __imp_?hasError@Task@U2@@QBE_NXZ 10026b00     U2Core:U2Core.dll
 0002:00000b04       __imp_??1TaskStateInfo@U2@@UAE@XZ 10026b04     U2Core:U2Core.dll
 0002:00000b08       __imp_?setError@TaskStateInfo@U2@@UAEXABVQString@@@Z 10026b08     U2Core:U2Core.dll
 0002:00000b0c       __imp_?getError@TaskStateInfo@U2@@UBE?AVQString@@XZ 10026b0c     U2Core:U2Core.dll
 0002:00000b10       __imp_??0TaskStateInfo@U2@@QAE@XZ 10026b10     U2Core:U2Core.dll
 0002:00000b14       __imp_?info@Logger@U2@@QAEXABVQString@@@Z 10026b14     U2Core:U2Core.dll
 0002:00000b18       __imp_?qt_metacast@TaskSignalMapper@U2@@UAEPAXPBD@Z 10026b18     U2Core:U2Core.dll
 0002:00000b1c       __imp_?qt_metacast@Task@U2@@UAEPAXPBD@Z 10026b1c     U2Core:U2Core.dll
 0002:00000b20       __imp_?qt_metacast@FailTask@U2@@UAEPAXPBD@Z 10026b20     U2Core:U2Core.dll
 0002:00000b24       __imp_?qt_metacall@TaskSignalMapper@U2@@UAEHW4Call@QMetaObject@@HPAPAX@Z 10026b24     U2Core:U2Core.dll
 0002:00000b28       __imp_?setRegion@LRegionsSelection@U2@@QAEXABVU2Region@2@@Z 10026b28     U2Core:U2Core.dll
 0002:00000b2c       __imp_??0Logger@U2@@QAE@ABVQString@@@Z 10026b2c     U2Core:U2Core.dll
 0002:00000b30       __imp_??1Logger@U2@@UAE@XZ 10026b30     U2Core:U2Core.dll
 0002:00000b34       __imp_?error@Logger@U2@@QAEXABVQString@@@Z 10026b34     U2Core:U2Core.dll
 0002:00000b38       __imp_?getTaskName@Task@U2@@QBE?AVQString@@XZ 10026b38     U2Core:U2Core.dll
 0002:00000b3c       __imp_?cancel@Task@U2@@QAEXXZ 10026b3c     U2Core:U2Core.dll
 0002:00000b40       __imp_??8U2EntityRef@U2@@QBE_NABV01@@Z 10026b40     U2Core:U2Core.dll
 0002:00000b44       __imp_??0GObjectReference@U2@@QAE@PBVGObject@1@_N@Z 10026b44     U2Core:U2Core.dll
 0002:00000b48       __imp_??1GObjectReference@U2@@QAE@XZ 10026b48     U2Core:U2Core.dll
 0002:00000b4c       __imp_??4GObjectReference@U2@@QAEAAV01@ABV01@@Z 10026b4c     U2Core:U2Core.dll
 0002:00000b50       __imp_?getSequenceLength@U2SequenceObject@U2@@QBE_JXZ 10026b50     U2Core:U2Core.dll
 0002:00000b54       __imp_?isCircular@U2SequenceObject@U2@@QBE_NXZ 10026b54     U2Core:U2Core.dll
 0002:00000b58       __imp_??1AnnotationData@U2@@QAE@XZ 10026b58     U2Core:U2Core.dll
 0002:00000b5c       __imp_??0AnnotationData@U2@@QAE@ABV01@@Z 10026b5c     U2Core:U2Core.dll
 0002:00000b60       __imp_?getSettings@AppContext@U2@@SAPAVSettings@2@XZ 10026b60     U2Core:U2Core.dll
 0002:00000b64       __imp_?getTaskScheduler@AppContext@U2@@SAPAVTaskScheduler@2@XZ 10026b64     U2Core:U2Core.dll
 0002:00000b68       __imp_?warningTitle@L10N@U2@@SA?AVQString@@XZ 10026b68     U2Core:U2Core.dll
 0002:00000b6c       __imp_?getSequenceObject@AutoAnnotationsUpdateTask@U2@@QBEPAVU2SequenceObject@2@XZ 10026b6c     U2Core:U2Core.dll
 0002:00000b70       __imp_?cleanup@Task@U2@@UAEXXZ 10026b70     U2Core:U2Core.dll
 0002:00000b74       __imp_?generateReport@Task@U2@@UBE?AVQString@@XZ 10026b74     U2Core:U2Core.dll
 0002:00000b78       __imp_?getNumParallelSubtasks@Task@U2@@UBEHXZ 10026b78     U2Core:U2Core.dll
 0002:00000b7c       __imp_?getParentTask@Task@U2@@UBEPAV12@XZ 10026b7c     U2Core:U2Core.dll
 0002:00000b80       __imp_?getSubtaskWithErrors@Task@U2@@UBEPAV12@XZ 10026b80     U2Core:U2Core.dll
 0002:00000b84       __imp_?getTaskId@Task@U2@@UBE_JXZ 10026b84     U2Core:U2Core.dll
 0002:00000b88       __imp_?getTopLevelParentTask@Task@U2@@UAEPAV12@XZ 10026b88     U2Core:U2Core.dll
 0002:00000b8c       __imp_?getWarnings@Task@U2@@UBE?AVQStringList@@XZ 10026b8c     U2Core:U2Core.dll
 0002:00000b90       __imp_?hasSubtasksWithErrors@Task@U2@@UBE_NXZ 10026b90     U2Core:U2Core.dll
 0002:00000b94       __imp_?hasWarning@Task@U2@@UBE_NXZ 10026b94     U2Core:U2Core.dll
 0002:00000b98       __imp_?isNotificationReport@Task@U2@@UBE_NXZ 10026b98     U2Core:U2Core.dll
 0002:00000b9c       __imp_?isReportingEnabled@Task@U2@@UBE_NXZ 10026b9c     U2Core:U2Core.dll
 0002:00000ba0       __imp_?isReportingSupported@Task@U2@@UBE_NXZ 10026ba0     U2Core:U2Core.dll
 0002:00000ba4       __imp_?isTopLevelTask@Task@U2@@UBE_NXZ 10026ba4     U2Core:U2Core.dll
 0002:00000ba8       __imp_?onSubTaskFinished@Task@U2@@MAE?AV?$QList@PAVTask@U2@@@@PAV12@@Z 10026ba8     U2Core:U2Core.dll
 0002:00000bac       __imp_?prepare@Task@U2@@UAEXXZ 10026bac     U2Core:U2Core.dll
 0002:00000bb0       __imp_?propagateSubtaskError@Task@U2@@UAE_NXZ 10026bb0     U2Core:U2Core.dll
 0002:00000bb4       __imp_?report@Task@U2@@UAE?AW4ReportResult@12@XZ 10026bb4     U2Core:U2Core.dll
 0002:00000bb8       __imp_?setCollectChildrensWarningsFlag@Task@U2@@UAEX_N@Z 10026bb8     U2Core:U2Core.dll
 0002:00000bbc       __imp_?setNoAutoDelete@Task@U2@@UAEX_N@Z 10026bbc     U2Core:U2Core.dll
 0002:00000bc0       __imp_?setNotificationReport@Task@U2@@UAEX_N@Z 10026bc0     U2Core:U2Core.dll
 0002:00000bc4       __imp_?setReportingEnabled@Task@U2@@UAEX_N@Z 10026bc4     U2Core:U2Core.dll
 0002:00000bc8       __imp_?setReportingSupported@Task@U2@@UAEX_N@Z 10026bc8     U2Core:U2Core.dll
 0002:00000bcc       __imp_?staticMetaObject@AutoAnnotationsUpdateTask@U2@@2UQMetaObject@@B 10026bcc     U2Core:U2Core.dll
 0002:00000bd0       __imp_?NAME@AutoAnnotationsUpdateTask@U2@@2VQString@@B 10026bd0     U2Core:U2Core.dll
 0002:00000bd4       __imp_?getMainWindow@AppContext@U2@@SAPAVMainWindow@2@XZ 10026bd4     U2Core:U2Core.dll
 0002:00000bd8       __imp_?getTestFramework@AppContext@U2@@SAPAVTestFramework@2@XZ 10026bd8     U2Core:U2Core.dll
 0002:00000bdc       __imp_?getAutoAnnotationsSupport@AppContext@U2@@SAPAVAutoAnnotationsSupport@2@XZ 10026bdc     U2Core:U2Core.dll
 0002:00000be0       __imp_?getQDActorProtoRegistry@AppContext@U2@@SAPAVQDActorPrototypeRegistry@2@XZ 10026be0     U2Core:U2Core.dll
 0002:00000be4       __imp_?registerAutoAnnotationsUpdater@AutoAnnotationsSupport@U2@@QAEXPAVAutoAnnotationsUpdater@2@@Z 10026be4     U2Core:U2Core.dll
 0002:00000be8       __imp_??0Plugin@U2@@QAE@ABVQString@@0_NW4PluginState@1@@Z 10026be8     U2Core:U2Core.dll
 0002:00000bec       __imp_??1Plugin@U2@@UAE@XZ 10026bec     U2Core:U2Core.dll
 0002:00000bf0       __imp_?run@Task@U2@@UAEXXZ 10026bf0     U2Core:U2Core.dll
 0002:00000bf4       __imp_??1U2EntityRef@U2@@QAE@XZ 10026bf4     U2Core:U2Core.dll
 0002:00000bf8       __imp_??0U2EntityRef@U2@@QAE@ABV01@@Z 10026bf8     U2Core:U2Core.dll
 0002:00000bfc       __imp_?getDNATranslationRegistry@AppContext@U2@@SAPAVDNATranslationRegistry@2@XZ 10026bfc     U2Core:U2Core.dll
 0002:00000c00       __imp_??0Task@U2@@QAE@ABVQString@@V?$QFlags@W4TaskFlag@U2@@@@@Z 10026c00     U2Core:U2Core.dll
 0002:00000c04       __imp_?addSubTask@Task@U2@@QAEXPAV12@@Z 10026c04     U2Core:U2Core.dll
 0002:00000c08       __imp_?setError@Task@U2@@QAEXABVQString@@@Z 10026c08     U2Core:U2Core.dll
 0002:00000c0c       __imp_??1Task@U2@@UAE@XZ   10026c0c     U2Core:U2Core.dll
 0002:00000c10       __imp_??0CreateAnnotationsTask@U2@@QAE@PAVAnnotationTableObject@1@ABV?$QList@V?$QSharedDataPointer@VAnnotationData@U2@@@@@@ABVQString@@@Z 10026c10     U2Core:U2Core.dll
 0002:00000c14       __imp_??1CreateAnnotationsTask@U2@@UAE@XZ 10026c14     U2Core:U2Core.dll
 0002:00000c18       __imp_?lookupTranslation@DNATranslationRegistry@U2@@QAEPAVDNATranslation@2@ABVQString@@@Z 10026c18     U2Core:U2Core.dll
 0002:00000c1c       __imp_?findComplementTT@GObjectUtils@U2@@SAPAVDNATranslation@2@PBVDNAAlphabet@2@@Z 10026c1c     U2Core:U2Core.dll
 0002:00000c20       __imp_?addDescriptionQualifier@U1AnnotationUtils@U2@@SAXAAV?$QList@V?$QSharedDataPointer@VAnnotationData@U2@@@@@@ABVQString@@@Z 10026c20     U2Core:U2Core.dll
 0002:00000c24       __imp_?getSequenceRef@U2SequenceObject@U2@@QBE?AVU2EntityRef@2@XZ 10026c24     U2Core:U2Core.dll
 0002:00000c28       __imp_?getAlphabet@U2SequenceObject@U2@@QBEPBVDNAAlphabet@2@XZ 10026c28     U2Core:U2Core.dll
 0002:00000c2c       __imp_?getAminoTT@AutoAnnotationObject@U2@@QBEPAVDNATranslation@2@XZ 10026c2c     U2Core:U2Core.dll
 0002:00000c30       __imp_??0AutoAnnotationsUpdater@U2@@QAE@ABVQString@@0_N1@Z 10026c30     U2Core:U2Core.dll
 0002:00000c34       __imp_??1AutoAnnotationsUpdater@U2@@UAE@XZ 10026c34     U2Core:U2Core.dll
 0002:00000c38       __imp_?metaObject@CreateAnnotationsTask@U2@@UBEPBUQMetaObject@@XZ 10026c38     U2Core:U2Core.dll
 0002:00000c3c       __imp_?qt_metacall@CreateAnnotationsTask@U2@@UAEHW4Call@QMetaObject@@HPAPAX@Z 10026c3c     U2Core:U2Core.dll
 0002:00000c40       __imp_?qt_metacast@CreateAnnotationsTask@U2@@UAEPAXPBD@Z 10026c40     U2Core:U2Core.dll
 0002:00000c44       __imp_?report@CreateAnnotationsTask@U2@@UAE?AW4ReportResult@Task@2@XZ 10026c44     U2Core:U2Core.dll
 0002:00000c48       __imp_?run@CreateAnnotationsTask@U2@@UAEXXZ 10026c48     U2Core:U2Core.dll
 0002:00000c4c       __imp_?lookupTranslation@DNATranslationRegistry@U2@@QAEPAVDNATranslation@2@PBVDNAAlphabet@2@W4DNATranslationType@2@ABVQString@@@Z 10026c4c     U2Core:U2Core.dll
 0002:00000c50       __imp_?lookupComplementTranslation@DNATranslationRegistry@U2@@QAEPAVDNATranslation@2@PBVDNAAlphabet@2@@Z 10026c50     U2Core:U2Core.dll
 0002:00000c54       __imp_?staticMetaObject@U2SequenceObject@U2@@2UQMetaObject@@B 10026c54     U2Core:U2Core.dll
 0002:00000c58       __imp_??CU2Location@U2@@QBEPBVU2LocationData@1@XZ 10026c58     U2Core:U2Core.dll
 0002:00000c5c       __imp_??1U2Qualifier@U2@@QAE@XZ 10026c5c     U2Core:U2Core.dll
 0002:00000c60       __imp_??0U2Qualifier@U2@@QAE@ABV01@@Z 10026c60     U2Core:U2Core.dll
 0002:00000c64       __imp_?getStrand@AnnotationData@U2@@QBE?AVU2Strand@2@XZ 10026c64     U2Core:U2Core.dll
 0002:00000c68       __imp_?getDNAAlphabetRegistry@AppContext@U2@@SAPAVDNAAlphabetRegistry@2@XZ 10026c68     U2Core:U2Core.dll
 0002:00000c6c       __imp_?lookupTranslation@DNATranslationRegistry@U2@@QAE?AV?$QList@PAVDNATranslation@U2@@@@PBVDNAAlphabet@2@W4DNATranslationType@2@@Z 10026c6c     U2Core:U2Core.dll
 0002:00000c70       __imp_?NUCL_DNA_DEFAULT@BaseDNAAlphabetIds@U2@@SA?BVQString@@XZ 10026c70     U2Core:U2Core.dll
 0002:00000c74       __imp_??0TaskSignalMapper@U2@@QAE@PAVTask@1@@Z 10026c74     U2Core:U2Core.dll
 0002:00000c78       __imp_??0FailTask@U2@@QAE@ABVQString@@@Z 10026c78     U2Core:U2Core.dll
 0002:00000c7c       __imp_??1FailTask@U2@@UAE@XZ 10026c7c     U2Core:U2Core.dll
 0002:00000c80       __imp_?suffixBp@L10N@U2@@SA?AVQString@@XZ 10026c80     U2Core:U2Core.dll
 0002:00000c84       __imp_?metaObject@FailTask@U2@@UBEPBUQMetaObject@@XZ 10026c84     U2Core:U2Core.dll
 0002:00000c88       __imp_?metaObject@Task@U2@@UBEPBUQMetaObject@@XZ 10026c88     U2Core:U2Core.dll
 0002:00000c8c       __imp_?metaObject@TaskSignalMapper@U2@@UBEPBUQMetaObject@@XZ 10026c8c     U2Core:U2Core.dll
 0002:00000c90       __imp_?qt_metacall@FailTask@U2@@UAEHW4Call@QMetaObject@@HPAPAX@Z 10026c90     U2Core:U2Core.dll
 0002:00000c94       __imp_?qt_metacall@Task@U2@@UAEHW4Call@QMetaObject@@HPAPAX@Z 10026c94     U2Core:U2Core.dll
 0002:00000c98       __imp_?intersect@U2Region@U2@@QBE?AV12@ABV12@@Z 10026c98     U2Core:U2Core.dll
 0002:00000c9c       \177U2Core_NULL_THUNK_DATA 10026c9c     U2Core:U2Core.dll
 0002:00000ca0       __imp_??1DelegateEditor@U2@@UAE@XZ 10026ca0     U2Designer:U2Designer.dll
 0002:00000ca4       __imp_??0SpinBoxDelegate@U2@@QAE@ABV?$QMap@VQString@@VQVariant@@@@PAVQObject@@@Z 10026ca4     U2Designer:U2Designer.dll
 0002:00000ca8       __imp_??1SpinBoxDelegate@U2@@UAE@XZ 10026ca8     U2Designer:U2Designer.dll
 0002:00000cac       __imp_??0ComboBoxDelegate@U2@@QAE@ABV?$QMap@VQString@@VQVariant@@@@PAVQObject@@@Z 10026cac     U2Designer:U2Designer.dll
 0002:00000cb0       __imp_??1ComboBoxDelegate@U2@@UAE@XZ 10026cb0     U2Designer:U2Designer.dll
 0002:00000cb4       __imp_?addDelegate@DelegateEditor@U2@@UAEXPAVPropertyDelegate@2@ABVQString@@@Z 10026cb4     U2Designer:U2Designer.dll
 0002:00000cb8       __imp_?clone@ComboBoxDelegate@U2@@UAEPAVPropertyDelegate@2@XZ 10026cb8     U2Designer:U2Designer.dll
 0002:00000cbc       __imp_?clone@DelegateEditor@U2@@UAEPAVConfigurationEditor@2@XZ 10026cbc     U2Designer:U2Designer.dll
 0002:00000cc0       __imp_?clone@SpinBoxDelegate@U2@@UAEPAVPropertyDelegate@2@XZ 10026cc0     U2Designer:U2Designer.dll
 0002:00000cc4       __imp_?commit@DelegateEditor@U2@@UAEXXZ 10026cc4     U2Designer:U2Designer.dll
 0002:00000cc8       __imp_?createEditor@ComboBoxDelegate@U2@@UBEPAVQWidget@@PAV3@ABVQStyleOptionViewItem@@ABVQModelIndex@@@Z 10026cc8     U2Designer:U2Designer.dll
 0002:00000ccc       __imp_?createEditor@SpinBoxDelegate@U2@@UBEPAVQWidget@@PAV3@ABVQStyleOptionViewItem@@ABVQModelIndex@@@Z 10026ccc     U2Designer:U2Designer.dll
 0002:00000cd0       __imp_?createWizardWidget@ComboBoxDelegate@U2@@UBEPAVPropertyWidget@2@AAVU2OpStatus@2@PAVQWidget@@@Z 10026cd0     U2Designer:U2Designer.dll
 0002:00000cd4       __imp_?createWizardWidget@SpinBoxDelegate@U2@@UBEPAVPropertyWidget@2@AAVU2OpStatus@2@PAVQWidget@@@Z 10026cd4     U2Designer:U2Designer.dll
 0002:00000cd8       __imp_?getDelegate@DelegateEditor@U2@@UAEPAVPropertyDelegate@2@ABVQString@@@Z 10026cd8     U2Designer:U2Designer.dll
 0002:00000cdc       __imp_?getDisplayValue@ComboBoxDelegate@U2@@UBE?AVQVariant@@ABV3@@Z 10026cdc     U2Designer:U2Designer.dll
 0002:00000ce0       __imp_?getDisplayValue@SpinBoxDelegate@U2@@UBE?AVQVariant@@ABV3@@Z 10026ce0     U2Designer:U2Designer.dll
 0002:00000ce4       __imp_?getItems@ComboBoxDelegate@U2@@UBEXAAV?$QMap@VQString@@VQVariant@@@@@Z 10026ce4     U2Designer:U2Designer.dll
 0002:00000ce8       __imp_?getItems@SpinBoxDelegate@U2@@UBEXAAV?$QMap@VQString@@VQVariant@@@@@Z 10026ce8     U2Designer:U2Designer.dll
 0002:00000cec       __imp_?metaObject@ComboBoxDelegate@U2@@UBEPBUQMetaObject@@XZ 10026cec     U2Designer:U2Designer.dll
 0002:00000cf0       __imp_?metaObject@DelegateEditor@U2@@UBEPBUQMetaObject@@XZ 10026cf0     U2Designer:U2Designer.dll
 0002:00000cf4       __imp_?metaObject@SpinBoxDelegate@U2@@UBEPBUQMetaObject@@XZ 10026cf4     U2Designer:U2Designer.dll
 0002:00000cf8       __imp_?qt_metacall@ComboBoxDelegate@U2@@UAEHW4Call@QMetaObject@@HPAPAX@Z 10026cf8     U2Designer:U2Designer.dll
 0002:00000cfc       __imp_?qt_metacall@DelegateEditor@U2@@UAEHW4Call@QMetaObject@@HPAPAX@Z 10026cfc     U2Designer:U2Designer.dll
 0002:00000d00       __imp_?qt_metacall@SpinBoxDelegate@U2@@UAEHW4Call@QMetaObject@@HPAPAX@Z 10026d00     U2Designer:U2Designer.dll
 0002:00000d04       __imp_?qt_metacast@ComboBoxDelegate@U2@@UAEPAXPBD@Z 10026d04     U2Designer:U2Designer.dll
 0002:00000d08       __imp_?qt_metacast@DelegateEditor@U2@@UAEPAXPBD@Z 10026d08     U2Designer:U2Designer.dll
 0002:00000d0c       __imp_?qt_metacast@SpinBoxDelegate@U2@@UAEPAXPBD@Z 10026d0c     U2Designer:U2Designer.dll
 0002:00000d10       __imp_?removeDelegate@DelegateEditor@U2@@UAEPAVPropertyDelegate@2@ABVQString@@@Z 10026d10     U2Designer:U2Designer.dll
 0002:00000d14       __imp_?setEditorData@ComboBoxDelegate@U2@@UBEXPAVQWidget@@ABVQModelIndex@@@Z 10026d14     U2Designer:U2Designer.dll
 0002:00000d18       __imp_?setEditorData@SpinBoxDelegate@U2@@UBEXPAVQWidget@@ABVQModelIndex@@@Z 10026d18     U2Designer:U2Designer.dll
 0002:00000d1c       __imp_?setModelData@ComboBoxDelegate@U2@@UBEXPAVQWidget@@PAVQAbstractItemModel@@ABVQModelIndex@@@Z 10026d1c     U2Designer:U2Designer.dll
 0002:00000d20       __imp_?setModelData@SpinBoxDelegate@U2@@UBEXPAVQWidget@@PAVQAbstractItemModel@@ABVQModelIndex@@@Z 10026d20     U2Designer:U2Designer.dll
 0002:00000d24       __imp_?updateDelegate@DelegateEditor@U2@@UAEXABVQString@@@Z 10026d24     U2Designer:U2Designer.dll
 0002:00000d28       __imp_?updateDelegates@DelegateEditor@U2@@UAEXXZ 10026d28     U2Designer:U2Designer.dll
 0002:00000d2c       __imp_??0ComboBoxDelegate@U2@@QAE@ABV?$QList@U?$QPair@VQString@@VQVariant@@@@@@PAVQObject@@@Z 10026d2c     U2Designer:U2Designer.dll
 0002:00000d30       __imp_??0DelegateEditor@U2@@QAE@ABV?$QMap@VQString@@PAVPropertyDelegate@U2@@@@@Z 10026d30     U2Designer:U2Designer.dll
 0002:00000d34       \177U2Designer_NULL_THUNK_DATA 10026d34     U2Designer:U2Designer.dll
 0002:00000d38       __imp_?sl_buildContextMenu@GObjectViewWindowContext@U2@@MAEXPAVGObjectView@2@PAVQMenu@@@Z 10026d38     U2Gui:U2Gui.dll
 0002:00000d3c       __imp_?getRegion@RegionSelector@U2@@QBE?AVU2Region@2@PA_N@Z 10026d3c     U2Gui:U2Gui.dll
 0002:00000d40       __imp_?isWholeSequenceSelected@RegionSelector@U2@@QBE_NXZ 10026d40     U2Gui:U2Gui.dll
 0002:00000d44       __imp_?setWholeRegionSelected@RegionSelector@U2@@QAEXXZ 10026d44     U2Gui:U2Gui.dll
 0002:00000d48       __imp_?showErrorMessage@RegionSelector@U2@@QAEXXZ 10026d48     U2Gui:U2Gui.dll
 0002:00000d4c       __imp_?getWidget@GObjectView@U2@@QAEPAVQWidget@@XZ 10026d4c     U2Gui:U2Gui.dll
 0002:00000d50       __imp_??0CreateAnnotationModel@U2@@QAE@XZ 10026d50     U2Gui:U2Gui.dll
 0002:00000d54       __imp_?getAnnotationObject@CreateAnnotationModel@U2@@QBEPAVAnnotationTableObject@2@XZ 10026d54     U2Gui:U2Gui.dll
 0002:00000d58       __imp_??1CreateAnnotationModel@U2@@QAE@XZ 10026d58     U2Gui:U2Gui.dll
 0002:00000d5c       __imp_??0CreateAnnotationWidgetController@U2@@QAE@ABVCreateAnnotationModel@1@PAVQObject@@W4AnnotationWidgetMode@01@@Z 10026d5c     U2Gui:U2Gui.dll
 0002:00000d60       __imp_?validate@CreateAnnotationWidgetController@U2@@QAE?AVQString@@XZ 10026d60     U2Gui:U2Gui.dll
 0002:00000d64       __imp_?prepareAnnotationObject@CreateAnnotationWidgetController@U2@@QAE_NXZ 10026d64     U2Gui:U2Gui.dll
 0002:00000d68       __imp_?useAutoAnnotationModel@CreateAnnotationWidgetController@U2@@QBE_NXZ 10026d68     U2Gui:U2Gui.dll
 0002:00000d6c       __imp_?getWidget@CreateAnnotationWidgetController@U2@@QBEPAVQWidget@@XZ 10026d6c     U2Gui:U2Gui.dll
 0002:00000d70       __imp_??1CreateAnnotationWidgetController@U2@@UAE@XZ 10026d70     U2Gui:U2Gui.dll
 0002:00000d74       __imp_??0HelpButton@U2@@QAE@PAVQObject@@PAVQDialogButtonBox@@ABVQString@@@Z 10026d74     U2Gui:U2Gui.dll
 0002:00000d78       __imp_??1HelpButton@U2@@UAE@XZ 10026d78     U2Gui:U2Gui.dll
 0002:00000d7c       __imp_?metaObject@CreateAnnotationWidgetController@U2@@UBEPBUQMetaObject@@XZ 10026d7c     U2Gui:U2Gui.dll
 0002:00000d80       __imp_?metaObject@HelpButton@U2@@UBEPBUQMetaObject@@XZ 10026d80     U2Gui:U2Gui.dll
 0002:00000d84       __imp_?metaObject@RegionSelector@U2@@UBEPBUQMetaObject@@XZ 10026d84     U2Gui:U2Gui.dll
 0002:00000d88       __imp_?qt_metacall@CreateAnnotationWidgetController@U2@@UAEHW4Call@QMetaObject@@HPAPAX@Z 10026d88     U2Gui:U2Gui.dll
 0002:00000d8c       __imp_?qt_metacall@HelpButton@U2@@UAEHW4Call@QMetaObject@@HPAPAX@Z 10026d8c     U2Gui:U2Gui.dll
 0002:00000d90       __imp_?qt_metacall@RegionSelector@U2@@UAEHW4Call@QMetaObject@@HPAPAX@Z 10026d90     U2Gui:U2Gui.dll
 0002:00000d94       __imp_?qt_metacast@CreateAnnotationWidgetController@U2@@UAEPAXPBD@Z 10026d94     U2Gui:U2Gui.dll
 0002:00000d98       __imp_?qt_metacast@HelpButton@U2@@UAEPAXPBD@Z 10026d98     U2Gui:U2Gui.dll
 0002:00000d9c       __imp_?qt_metacast@RegionSelector@U2@@UAEPAXPBD@Z 10026d9c     U2Gui:U2Gui.dll
 0002:00000da0       __imp_?sl_buttonClicked@HelpButton@U2@@MAEXXZ 10026da0     U2Gui:U2Gui.dll
 0002:00000da4       __imp_?getObjectView@GObjectViewAction@U2@@QBEPAVGObjectView@2@XZ 10026da4     U2Gui:U2Gui.dll
 0002:00000da8       __imp_??0GObjectViewWindowContext@U2@@QAE@PAVQObject@@ABVGObjectViewFactoryId@1@@Z 10026da8     U2Gui:U2Gui.dll
 0002:00000dac       __imp_??1GObjectViewWindowContext@U2@@UAE@XZ 10026dac     U2Gui:U2Gui.dll
 0002:00000db0       __imp_?staticMetaObject@GObjectViewWindowContext@U2@@2UQMetaObject@@B 10026db0     U2Gui:U2Gui.dll
 0002:00000db4       __imp_?qt_metacall@GObjectViewWindowContext@U2@@UAEHW4Call@QMetaObject@@HPAPAX@Z 10026db4     U2Gui:U2Gui.dll
 0002:00000db8       __imp_?qt_metacast@GObjectViewWindowContext@U2@@UAEPAXPBD@Z 10026db8     U2Gui:U2Gui.dll
 0002:00000dbc       __imp_?staticMetaObject@GObjectViewAction@U2@@2UQMetaObject@@B 10026dbc     U2Gui:U2Gui.dll
 0002:00000dc0       __imp_?sl_windowClosing@GObjectViewWindowContext@U2@@MAEXPAVMWMDIWindow@2@@Z 10026dc0     U2Gui:U2Gui.dll
 0002:00000dc4       __imp_?sl_windowAdded@GObjectViewWindowContext@U2@@MAEXPAVMWMDIWindow@2@@Z 10026dc4     U2Gui:U2Gui.dll
 0002:00000dc8       __imp_?sl_buildStaticMenu@GObjectViewWindowContext@U2@@MAEXPAVGObjectView@2@PAVQMenu@@@Z 10026dc8     U2Gui:U2Gui.dll
 0002:00000dcc       __imp_??0RegionSelector@U2@@QAE@PAVQWidget@@_J_NPAVDNASequenceSelection@1@2V?$QList@URegionPreset@U2@@@@@Z 10026dcc     U2Gui:U2Gui.dll
 0002:00000dd0       __imp_?onObjectRemoved@GObjectViewWindowContext@U2@@UAEXPAVGObjectView@2@PAVGObject@2@@Z 10026dd0     U2Gui:U2Gui.dll
 0002:00000dd4       __imp_?onObjectAdded@GObjectViewObjectHandler@U2@@UAEXPAVGObjectView@2@PAVGObject@2@@Z 10026dd4     U2Gui:U2Gui.dll
 0002:00000dd8       __imp_?init@GObjectViewWindowContext@U2@@UAEXXZ 10026dd8     U2Gui:U2Gui.dll
 0002:00000ddc       __imp_?disconnectView@GObjectViewWindowContext@U2@@MAEXPAVGObjectView@2@@Z 10026ddc     U2Gui:U2Gui.dll
 0002:00000de0       __imp_?canHandle@GObjectViewObjectHandler@U2@@UAE_NPAVGObjectView@2@PAVGObject@2@@Z 10026de0     U2Gui:U2Gui.dll
 0002:00000de4       __imp_?buildMenu@GObjectViewWindowContext@U2@@MAEXPAVGObjectView@2@PAVQMenu@@@Z 10026de4     U2Gui:U2Gui.dll
 0002:00000de8       \177U2Gui_NULL_THUNK_DATA  10026de8     U2Gui:U2Gui.dll
 0002:00000dec       __imp_?getType@PortDescriptor@Workflow@U2@@UBE?AV?$QExplicitlySharedDataPointer@VDataType@U2@@@@XZ 10026dec     U2Lang:U2Lang.dll
 0002:00000df0       __imp_?isAcceptableDrop@ActorPrototype@Workflow@U2@@UBE_NPBVQMimeData@@PAV?$QMap@VQString@@VQVariant@@@@@Z 10026df0     U2Lang:U2Lang.dll
 0002:00000df4       __imp_?isDone@BaseWorker@LocalWorkflow@U2@@UBE_NXZ 10026df4     U2Lang:U2Lang.dll
 0002:00000df8       __imp_?isReady@BaseWorker@LocalWorkflow@U2@@UBE_NXZ 10026df8     U2Lang:U2Lang.dll
 0002:00000dfc       __imp_?kind@MapDataType@U2@@UBE?AW4Kind@DataType@2@XZ 10026dfc     U2Lang:U2Lang.dll
 0002:00000e00       __imp_??0Attribute@U2@@QAE@ABVDescriptor@1@V?$QExplicitlySharedDataPointer@VDataType@U2@@@@_NABVQVariant@@@Z 10026e00     U2Lang:U2Lang.dll
 0002:00000e04       __imp_??1Attribute@U2@@UAE@XZ 10026e04     U2Lang:U2Lang.dll
 0002:00000e08       __imp_?metaObject@PrompterBaseImpl@U2@@UBEPBUQMetaObject@@XZ 10026e08     U2Lang:U2Lang.dll
 0002:00000e0c       __imp_?qt_metacall@PrompterBaseImpl@U2@@UAEHW4Call@QMetaObject@@HPAPAX@Z 10026e0c     U2Lang:U2Lang.dll
 0002:00000e10       __imp_?qt_metacast@PrompterBaseImpl@U2@@UAEPAXPBD@Z 10026e10     U2Lang:U2Lang.dll
 0002:00000e14       __imp_?registerEntry@?$IdRegistry@VDomainFactory@Workflow@U2@@@U2@@UAE_NPAVDomainFactory@Workflow@2@@Z 10026e14     U2Lang:U2Lang.dll
 0002:00000e18       __imp_?setDone@BaseWorker@LocalWorkflow@U2@@UAEXXZ 10026e18     U2Lang:U2Lang.dll
 0002:00000e1c       __imp_?setVisibleSlot@PortDescriptor@Workflow@U2@@UAEXABVQString@@_N@Z 10026e1c     U2Lang:U2Lang.dll
 0002:00000e20       __imp_?setDocumentation@Descriptor@U2@@QAEXABVQString@@@Z 10026e20     U2Lang:U2Lang.dll
 0002:00000e24       __imp_?sl_actorModified@PrompterBaseImpl@U2@@MAEXXZ 10026e24     U2Lang:U2Lang.dll
 0002:00000e28       __imp_?unregisterEntry@?$IdRegistry@VDomainFactory@Workflow@U2@@@U2@@UAEPAVDomainFactory@Workflow@2@ABVQString@@@Z 10026e28     U2Lang:U2Lang.dll
 0002:00000e2c       __imp_?update@PrompterBaseImpl@U2@@UAEXABV?$QMap@VQString@@VQVariant@@@@@Z 10026e2c     U2Lang:U2Lang.dll
 0002:00000e30       __imp_?staticMetaObject@IntegralBusPort@Workflow@U2@@2UQMetaObject@@B 10026e30     U2Lang:U2Lang.dll
 0002:00000e34       __imp_?ID@LocalDomainFactory@LocalWorkflow@U2@@2VQString@@B 10026e34     U2Lang:U2Lang.dll
 0002:00000e38       __imp_?qt_metacast@QDActor@U2@@UAEPAXPBD@Z 10026e38     U2Lang:U2Lang.dll
 0002:00000e3c       __imp_?qt_metacall@QDActor@U2@@UAEHW4Call@QMetaObject@@HPAPAX@Z 10026e3c     U2Lang:U2Lang.dll
 0002:00000e40       __imp_?staticMetaObject@QDActor@U2@@2UQMetaObject@@B 10026e40     U2Lang:U2Lang.dll
 0002:00000e44       __imp_?qt_metacast@BaseWorker@LocalWorkflow@U2@@UAEPAXPBD@Z 10026e44     U2Lang:U2Lang.dll
 0002:00000e48       __imp_?qt_metacall@BaseWorker@LocalWorkflow@U2@@UAEHW4Call@QMetaObject@@HPAPAX@Z 10026e48     U2Lang:U2Lang.dll
 0002:00000e4c       __imp_?staticMetaObject@BaseWorker@LocalWorkflow@U2@@2UQMetaObject@@B 10026e4c     U2Lang:U2Lang.dll
 0002:00000e50       __imp_?staticMetaObject@PrompterBaseImpl@U2@@2UQMetaObject@@B 10026e50     U2Lang:U2Lang.dll
 0002:00000e54       __imp_?registerProto@QDActorPrototypeRegistry@U2@@QAEXPAVQDActorPrototype@2@@Z 10026e54     U2Lang:U2Lang.dll
 0002:00000e58       __imp_??0Descriptor@U2@@QAE@ABVQString@@00@Z 10026e58     U2Lang:U2Lang.dll
 0002:00000e5c       __imp_??1Descriptor@U2@@UAE@XZ 10026e5c     U2Lang:U2Lang.dll
 0002:00000e60       __imp_?setId@Descriptor@U2@@QAEXABVQString@@@Z 10026e60     U2Lang:U2Lang.dll
 0002:00000e64       __imp_?setDisplayName@Descriptor@U2@@QAEXABVQString@@@Z 10026e64     U2Lang:U2Lang.dll
 0002:00000e68       __imp_?si_modified@QDParameters@U2@@QAEXXZ 10026e68     U2Lang:U2Lang.dll
 0002:00000e6c       __imp_??0QDResultUnitData@U2@@QAE@XZ 10026e6c     U2Lang:U2Lang.dll
 0002:00000e70       __imp_??1QDResultUnitData@U2@@QAE@XZ 10026e70     U2Lang:U2Lang.dll
 0002:00000e74       __imp_??0QDResultUnitData@U2@@QAE@ABV01@@Z 10026e74     U2Lang:U2Lang.dll
 0002:00000e78       __imp_?buildGroupFromSingleResult@QDResultGroup@U2@@SAXABV?$QSharedDataPointer@VQDResultUnitData@U2@@@@AAV?$QList@PAVQDResultGroup@U2@@@@@Z 10026e78     U2Lang:U2Lang.dll
 0002:00000e7c       __imp_??0QDActorPrototype@U2@@QAE@XZ 10026e7c     U2Lang:U2Lang.dll
 0002:00000e80       __imp_??1QDActorPrototype@U2@@UAE@XZ 10026e80     U2Lang:U2Lang.dll
 0002:00000e84       __imp_??0QDActor@U2@@QAE@PBVQDActorPrototype@1@@Z 10026e84     U2Lang:U2Lang.dll
 0002:00000e88       __imp_??1QDActor@U2@@UAE@XZ 10026e88     U2Lang:U2Lang.dll
 0002:00000e8c       __imp_?getStrandToRun@QDActor@U2@@IBE?AW4QDStrandOption@2@XZ 10026e8c     U2Lang:U2Lang.dll
 0002:00000e90       __imp_??0QDSchemeUnit@U2@@QAE@PAVQDActor@1@@Z 10026e90     U2Lang:U2Lang.dll
 0002:00000e94       __imp_?getEntityRef@QDScheme@U2@@QBE?AVU2EntityRef@2@XZ 10026e94     U2Lang:U2Lang.dll
 0002:00000e98       __imp_?STRING_TYPE@BaseTypes@U2@@SA?AV?$QExplicitlySharedDataPointer@VDataType@U2@@@@XZ 10026e98     U2Lang:U2Lang.dll
 0002:00000e9c       __imp_?BOOL_TYPE@BaseTypes@U2@@SA?AV?$QExplicitlySharedDataPointer@VDataType@U2@@@@XZ 10026e9c     U2Lang:U2Lang.dll
 0002:00000ea0       __imp_?NUM_TYPE@BaseTypes@U2@@SA?AV?$QExplicitlySharedDataPointer@VDataType@U2@@@@XZ 10026ea0     U2Lang:U2Lang.dll
 0002:00000ea4       __imp_?clone@Attribute@U2@@UAEPAV12@XZ 10026ea4     U2Lang:U2Lang.dll
 0002:00000ea8       __imp_?getAttributePureValue@Attribute@U2@@UBEABVQVariant@@XZ 10026ea8     U2Lang:U2Lang.dll
 0002:00000eac       __imp_?getDefaultPureValue@Attribute@U2@@UBEABVQVariant@@XZ 10026eac     U2Lang:U2Lang.dll
 0002:00000eb0       __imp_?getGroup@Attribute@U2@@UAE?AW4AttributeGroup@2@XZ 10026eb0     U2Lang:U2Lang.dll
 0002:00000eb4       __imp_?getWidget@ConfigurationEditor@U2@@UAEPAVQWidget@@XZ 10026eb4     U2Lang:U2Lang.dll
 0002:00000eb8       __imp_?hasStrand@QDActor@U2@@UBE_NXZ 10026eb8     U2Lang:U2Lang.dll
 0002:00000ebc       __imp_?isDefaultValue@Attribute@U2@@UBE_NXZ 10026ebc     U2Lang:U2Lang.dll
 0002:00000ec0       __imp_?isEmpty@Attribute@U2@@UBE_NXZ 10026ec0     U2Lang:U2Lang.dll
 0002:00000ec4       __imp_?isEmpty@ConfigurationEditor@U2@@UBE_NXZ 10026ec4     U2Lang:U2Lang.dll
 0002:00000ec8       __imp_?loadConfiguration@QDActor@U2@@UAEXABV?$QList@U?$QPair@VQString@@V1@@@@@@Z 10026ec8     U2Lang:U2Lang.dll
 0002:00000ecc       __imp_?saveConfiguration@QDActor@U2@@UBE?AV?$QList@U?$QPair@VQString@@V1@@@@@XZ 10026ecc     U2Lang:U2Lang.dll
 0002:00000ed0       __imp_?setAttributeValue@Attribute@U2@@UAEXABVQVariant@@@Z 10026ed0     U2Lang:U2Lang.dll
 0002:00000ed4       __imp_?type@PropertyDelegate@U2@@UBE?AW4Type@12@XZ 10026ed4     U2Lang:U2Lang.dll
 0002:00000ed8       __imp_?update@PropertyDelegate@U2@@UAEXXZ 10026ed8     U2Lang:U2Lang.dll
 0002:00000edc       __imp_?updateActorIds@Attribute@U2@@UAEXABV?$QMap@VQString@@V1@@@@Z 10026edc     U2Lang:U2Lang.dll
 0002:00000ee0       __imp_?updateEditor@QDActor@U2@@UAEXXZ 10026ee0     U2Lang:U2Lang.dll
 0002:00000ee4       __imp_?validate@Attribute@U2@@UAE_NAAV?$QList@VWorkflowNotification@U2@@@@@Z 10026ee4     U2Lang:U2Lang.dll
 0002:00000ee8       __imp_?DEFAULT_MAX_RESULT_LENGTH@QDActor@U2@@2HB 10026ee8     U2Lang:U2Lang.dll
 0002:00000eec       __imp_??0Descriptor@U2@@QAE@PBD@Z 10026eec     U2Lang:U2Lang.dll
 0002:00000ef0       __imp_?getId@Descriptor@U2@@QBE?AVQString@@XZ 10026ef0     U2Lang:U2Lang.dll
 0002:00000ef4       __imp_??0Descriptor@U2@@QAE@ABV01@@Z 10026ef4     U2Lang:U2Lang.dll
 0002:00000ef8       __imp_?setIconPath@VisualDescriptor@U2@@QAEXABVQString@@@Z 10026ef8     U2Lang:U2Lang.dll
 0002:00000efc       __imp_??0MapDataType@U2@@QAE@ABVDescriptor@1@ABV?$QMap@VDescriptor@U2@@V?$QExplicitlySharedDataPointer@VDataType@U2@@@@@@@Z 10026efc     U2Lang:U2Lang.dll
 0002:00000f00       __imp_??1MapDataType@U2@@UAE@XZ 10026f00     U2Lang:U2Lang.dll
 0002:00000f04       __imp_?initEngine@WorkflowScriptLibrary@U2@@SAXPAVWorkflowScriptEngine@2@@Z 10026f04     U2Lang:U2Lang.dll
 0002:00000f08       __imp_?getSequenceObject@StorageUtils@Workflow@U2@@SAPAVU2SequenceObject@3@PAVDbiDataStorage@23@ABV?$QSharedDataPointer@VDbiDataHandler@Workflow@U2@@@@@Z 10026f08     U2Lang:U2Lang.dll
 0002:00000f0c       __imp_?getDataStorage@WorkflowContext@Workflow@U2@@QAEPAVDbiDataStorage@23@XZ 10026f0c     U2Lang:U2Lang.dll
 0002:00000f10       __imp_??0WorkflowScriptEngine@U2@@QAE@PAVWorkflowContext@Workflow@1@@Z 10026f10     U2Lang:U2Lang.dll
 0002:00000f14       __imp_??1WorkflowScriptEngine@U2@@UAE@XZ 10026f14     U2Lang:U2Lang.dll
 0002:00000f18       __imp_?isEmpty@AttributeScript@U2@@QBE_NXZ 10026f18     U2Lang:U2Lang.dll
 0002:00000f1c       __imp_?getScriptText@AttributeScript@U2@@QBEABVQString@@XZ 10026f1c     U2Lang:U2Lang.dll
 0002:00000f20       __imp_?getScriptVars@AttributeScript@U2@@QBEABV?$QMap@VDescriptor@U2@@VQVariant@@@@XZ 10026f20     U2Lang:U2Lang.dll
 0002:00000f24       __imp_?getLabel@Actor@Workflow@U2@@QBE?AVQString@@XZ 10026f24     U2Lang:U2Lang.dll
 0002:00000f28       __imp_?getPort@Actor@Workflow@U2@@QBEPAVPort@23@ABVQString@@@Z 10026f28     U2Lang:U2Lang.dll
 0002:00000f2c       __imp_?getInputPorts@Actor@Workflow@U2@@QBE?AV?$QList@PAVPort@Workflow@U2@@@@XZ 10026f2c     U2Lang:U2Lang.dll
 0002:00000f30       __imp_?getOutputPorts@Actor@Workflow@U2@@QBE?AV?$QList@PAVPort@Workflow@U2@@@@XZ 10026f30     U2Lang:U2Lang.dll
 0002:00000f34       __imp_??0PortDescriptor@Workflow@U2@@QAE@ABVDescriptor@2@V?$QExplicitlySharedDataPointer@VDataType@U2@@@@_N2I@Z 10026f34     U2Lang:U2Lang.dll
 0002:00000f38       __imp_??1PortDescriptor@Workflow@U2@@UAE@XZ 10026f38     U2Lang:U2Lang.dll
 0002:00000f3c       __imp_??0ActorPrototype@Workflow@U2@@QAE@ABVDescriptor@2@ABV?$QList@PAVPortDescriptor@Workflow@U2@@@@ABV?$QList@PAVAttribute@U2@@@@@Z 10026f3c     U2Lang:U2Lang.dll
 0002:00000f40       __imp_??1ActorPrototype@Workflow@U2@@UAE@XZ 10026f40     U2Lang:U2Lang.dll
 0002:00000f44       __imp_?setEditor@ActorPrototype@Workflow@U2@@QAEXPAVConfigurationEditor@3@@Z 10026f44     U2Lang:U2Lang.dll
 0002:00000f48       __imp_?setPrompter@ActorPrototype@Workflow@U2@@QAEXPAVPrompter@23@@Z 10026f48     U2Lang:U2Lang.dll
 0002:00000f4c       __imp_?getProducer@IntegralBusPort@Workflow@U2@@QAEPAVActor@23@ABVQString@@@Z 10026f4c     U2Lang:U2Lang.dll
 0002:00000f50       __imp_??0Message@Workflow@U2@@QAE@V?$QExplicitlySharedDataPointer@VDataType@U2@@@@ABVQVariant@@H@Z 10026f50     U2Lang:U2Lang.dll
 0002:00000f54       __imp_?getData@Message@Workflow@U2@@QBE?AVQVariant@@XZ 10026f54     U2Lang:U2Lang.dll
 0002:00000f58       __imp_?isEmpty@Message@Workflow@U2@@QBE_NXZ 10026f58     U2Lang:U2Lang.dll
 0002:00000f5c       __imp_?getEmptyMapMessage@Message@Workflow@U2@@SA?AV123@XZ 10026f5c     U2Lang:U2Lang.dll
 0002:00000f60       __imp_??1Message@Workflow@U2@@QAE@XZ 10026f60     U2Lang:U2Lang.dll
 0002:00000f64       __imp_??0DomainFactory@Workflow@U2@@QAE@ABVQString@@@Z 10026f64     U2Lang:U2Lang.dll
 0002:00000f68       __imp_??1DomainFactory@Workflow@U2@@UAE@XZ 10026f68     U2Lang:U2Lang.dll
 0002:00000f6c       __imp_??0BaseWorker@LocalWorkflow@U2@@QAE@PAVActor@Workflow@2@_N@Z 10026f6c     U2Lang:U2Lang.dll
 0002:00000f70       __imp_??1BaseWorker@LocalWorkflow@U2@@UAE@XZ 10026f70     U2Lang:U2Lang.dll
 0002:00000f74       __imp_??0PrompterBaseImpl@U2@@QAE@PAVActor@Workflow@1@@Z 10026f74     U2Lang:U2Lang.dll
 0002:00000f78       __imp_?getRequiredParam@PrompterBaseImpl@U2@@QAE?AVQString@@ABV3@@Z 10026f78     U2Lang:U2Lang.dll
 0002:00000f7c       __imp_?getParameter@PrompterBaseImpl@U2@@QAE?AVQVariant@@ABVQString@@@Z 10026f7c     U2Lang:U2Lang.dll
 0002:00000f80       __imp_?getHyperlink@PrompterBaseImpl@U2@@SA?AVQString@@ABV3@0@Z 10026f80     U2Lang:U2Lang.dll
 0002:00000f84       __imp_?getHyperlink@PrompterBaseImpl@U2@@SA?AVQString@@ABV3@H@Z 10026f84     U2Lang:U2Lang.dll
 0002:00000f88       __imp_??1PrompterBaseImpl@U2@@UAE@XZ 10026f88     U2Lang:U2Lang.dll
 0002:00000f8c       __imp_?getInstance@WorkflowEnv@Workflow@U2@@KAPAV123@XZ 10026f8c     U2Lang:U2Lang.dll
 0002:00000f90       __imp_?registerProto@ActorPrototypeRegistry@Workflow@U2@@QAEXABVDescriptor@3@PAVActorPrototype@23@@Z 10026f90     U2Lang:U2Lang.dll
 0002:00000f94       __imp_?DNA_SEQUENCE_TYPE@BaseTypes@U2@@SA?AV?$QExplicitlySharedDataPointer@VDataType@U2@@@@XZ 10026f94     U2Lang:U2Lang.dll
 0002:00000f98       __imp_?ANNOTATION_TABLE_TYPE@BaseTypes@U2@@SA?AV?$QExplicitlySharedDataPointer@VDataType@U2@@@@XZ 10026f98     U2Lang:U2Lang.dll
 0002:00000f9c       __imp_?DNA_SEQUENCE_SLOT@BaseSlots@Workflow@U2@@SA?BVDescriptor@3@XZ 10026f9c     U2Lang:U2Lang.dll
 0002:00000fa0       __imp_?ANNOTATION_TABLE_SLOT@BaseSlots@Workflow@U2@@SA?BVDescriptor@3@XZ 10026fa0     U2Lang:U2Lang.dll
 0002:00000fa4       __imp_?IN_SEQ_PORT_ID@BasePorts@Workflow@U2@@SA?BVQString@@XZ 10026fa4     U2Lang:U2Lang.dll
 0002:00000fa8       __imp_?OUT_ANNOTATIONS_PORT_ID@BasePorts@Workflow@U2@@SA?BVQString@@XZ 10026fa8     U2Lang:U2Lang.dll
 0002:00000fac       __imp_?CATEGORY_BASIC@BaseActorCategories@Workflow@U2@@SA?BVDescriptor@3@XZ 10026fac     U2Lang:U2Lang.dll
 0002:00000fb0       __imp_?STRAND_ATTRIBUTE@BaseAttributes@Workflow@U2@@SA?BVDescriptor@3@XZ 10026fb0     U2Lang:U2Lang.dll
 0002:00000fb4       __imp_?STRAND_BOTH@BaseAttributes@Workflow@U2@@SA?BVQString@@XZ 10026fb4     U2Lang:U2Lang.dll
 0002:00000fb8       __imp_?STRAND_DIRECT@BaseAttributes@Workflow@U2@@SA?BVQString@@XZ 10026fb8     U2Lang:U2Lang.dll
 0002:00000fbc       __imp_?STRAND_COMPLEMENTARY@BaseAttributes@Workflow@U2@@SA?BVQString@@XZ 10026fbc     U2Lang:U2Lang.dll
 0002:00000fc0       __imp_?STRAND_ATTRIBUTE_VALUES_MAP@BaseAttributes@Workflow@U2@@SA?BV?$QMap@VQString@@VQVariant@@@@XZ 10026fc0     U2Lang:U2Lang.dll
 0002:00000fc4       __imp_?addCommunication@BaseWorker@LocalWorkflow@U2@@UAE_NABVQString@@PAVCommunicationChannel@Workflow@3@@Z 10026fc4     U2Lang:U2Lang.dll
 0002:00000fc8       __imp_?canTaskBeCanceled@BaseWorker@LocalWorkflow@U2@@MBE_NPAVTask@3@@Z 10026fc8     U2Lang:U2Lang.dll
 0002:00000fcc       __imp_?createConnection@DomainFactory@Workflow@U2@@UAEPAVCommunicationChannel@23@PAVLink@23@@Z 10026fcc     U2Lang:U2Lang.dll
 0002:00000fd0       __imp_?createInstance@ActorPrototype@Workflow@U2@@UAEPAVActor@23@ABVQString@@PAVAttributeScript@3@ABV?$QMap@VQString@@VQVariant@@@@@Z 10026fd0     U2Lang:U2Lang.dll
 0002:00000fd4       __imp_?createPort@IntegralBusActorPrototype@Workflow@U2@@UAEPAVPort@23@ABVPortDescriptor@23@PAVActor@23@@Z 10026fd4     U2Lang:U2Lang.dll
 0002:00000fd8       __imp_?createScheduler@DomainFactory@Workflow@U2@@UAEPAVScheduler@23@PAVSchema@23@@Z 10026fd8     U2Lang:U2Lang.dll
 0002:00000fdc       __imp_?destroy@DomainFactory@Workflow@U2@@UAEXPAVScheduler@23@PAVSchema@23@@Z 10026fdc     U2Lang:U2Lang.dll
 0002:00000fe0       __imp_?getActorId@BaseWorker@LocalWorkflow@U2@@UBE?AVQString@@XZ 10026fe0     U2Lang:U2Lang.dll
 0002:00000fe4       __imp_?getAllDescriptors@MapDataType@U2@@UBE?AV?$QList@VDescriptor@U2@@@@XZ 10026fe4     U2Lang:U2Lang.dll
 0002:00000fe8       __imp_?getAllEntries@?$IdRegistry@VDomainFactory@Workflow@U2@@@U2@@UBE?AV?$QList@PAVDomainFactory@Workflow@U2@@@@XZ 10026fe8     U2Lang:U2Lang.dll
 0002:00000fec       __imp_?getAllIds@?$IdRegistry@VDomainFactory@Workflow@U2@@@U2@@UBE?AV?$QList@VQString@@@@XZ 10026fec     U2Lang:U2Lang.dll
 0002:00000ff0       __imp_?getById@?$IdRegistry@VDomainFactory@Workflow@U2@@@U2@@UAEPAVDomainFactory@Workflow@2@ABVQString@@@Z 10026ff0     U2Lang:U2Lang.dll
 0002:00000ff4       __imp_?getCommunication@BaseWorker@LocalWorkflow@U2@@UAEPAVCommunicationChannel@Workflow@3@ABVQString@@@Z 10026ff4     U2Lang:U2Lang.dll
 0002:00000ff8       __imp_?getDatatypeByDescriptor@MapDataType@U2@@UBE?AV?$QExplicitlySharedDataPointer@VDataType@U2@@@@ABVDescriptor@2@@Z 10026ff8     U2Lang:U2Lang.dll
 0002:00000ffc       __imp_?getDatatypesMap@MapDataType@U2@@UBE?AV?$QMap@VDescriptor@U2@@V?$QExplicitlySharedDataPointer@VDataType@U2@@@@@@XZ 10026ffc     U2Lang:U2Lang.dll
 0002:00001000       __imp_?getMessageAndSetupScriptValues@BaseWorker@LocalWorkflow@U2@@UAE?AVMessage@Workflow@3@PAVCommunicationChannel@53@@Z 10027000     U2Lang:U2Lang.dll
 0002:00001004       __imp_?getOutputFiles@BaseWorker@LocalWorkflow@U2@@UAE?AVQStringList@@XZ 10027004     U2Lang:U2Lang.dll
 0002:00001008       \177U2Lang_NULL_THUNK_DATA 10027008     U2Lang:U2Lang.dll
 0002:0000100c       __imp_?findFormat@GTestFormatRegistry@U2@@QAEPAVGTestFormat@2@ABVQString@@@Z 1002700c     U2Test:U2Test.dll
 0002:00001010       __imp_?staticMetaObject@GTest@U2@@2UQMetaObject@@B 10027010     U2Test:U2Test.dll
 0002:00001014       __imp_?qt_metacall@GTest@U2@@UAEHW4Call@QMetaObject@@HPAPAX@Z 10027014     U2Test:U2Test.dll
 0002:00001018       __imp_?qt_metacast@GTest@U2@@UAEPAXPBD@Z 10027018     U2Test:U2Test.dll
 0002:0000101c       __imp_?failMissingValue@GTest@U2@@IAEXABVQString@@@Z 1002701c     U2Test:U2Test.dll
 0002:00001020       __imp_?getContext@GTest@U2@@QBEPAVQObject@@ABVQString@@@Z 10027020     U2Test:U2Test.dll
 0002:00001024       __imp_?staticMetaObject@XMLTestFormat@U2@@2UQMetaObject@@B 10027024     U2Test:U2Test.dll
 0002:00001028       __imp_??1XmlTest@U2@@UAE@XZ 10027028     U2Test:U2Test.dll
 0002:0000102c       __imp_??0XmlTest@U2@@QAE@ABVQString@@PAVGTest@1@PBVGTestEnvironment@1@V?$QFlags@W4TaskFlag@U2@@@@ABV?$QList@PAVGTest@U2@@@@@Z 1002702c     U2Test:U2Test.dll
 0002:00001030       __imp_??1XMLTestFactory@U2@@UAE@XZ 10027030     U2Test:U2Test.dll
 0002:00001034       __imp_??0XMLTestFactory@U2@@QAE@ABVQString@@@Z 10027034     U2Test:U2Test.dll
 0002:00001038       \177U2Test_NULL_THUNK_DATA 10027038     U2Test:U2Test.dll
 0002:0000103c       __imp_?qt_metacast@ADVGlobalAction@U2@@UAEPAXPBD@Z 1002703c     U2View:U2View.dll
 0002:00001040       __imp_?qt_metacall@ADVGlobalAction@U2@@UAEHW4Call@QMetaObject@@HPAPAX@Z 10027040     U2View:U2View.dll
 0002:00001044       __imp_?metaObject@ADVGlobalAction@U2@@UBEPBUQMetaObject@@XZ 10027044     U2View:U2View.dll
 0002:00001048       __imp_?getSequenceInFocus@AnnotatedDNAView@U2@@QBEPAVADVSequenceObjectContext@2@XZ 10027048     U2View:U2View.dll
 0002:0000104c       __imp_??1ADVGlobalAction@U2@@UAE@XZ 1002704c     U2View:U2View.dll
 0002:00001050       __imp_?addAlphabetFilter@ADVGlobalAction@U2@@QAEXW4DNAAlphabetType@@@Z 10027050     U2View:U2View.dll
 0002:00001054       __imp_??0ADVGlobalAction@U2@@QAE@PAVAnnotatedDNAView@1@ABVQIcon@@ABVQString@@HV?$QFlags@W4ADVGlobalActionFlag@U2@@@@@Z 10027054     U2View:U2View.dll
 0002:00001058       __imp_?tryAddObject@AnnotatedDNAView@U2@@QAE?AVQString@@PAVGObject@2@@Z 10027058     U2View:U2View.dll
 0002:0000105c       __imp_?createGeneticCodeMenu@SequenceObjectContext@U2@@QAEPAVQMenu@@XZ 1002705c     U2View:U2View.dll
 0002:00001060       __imp_?getSequenceLength@SequenceObjectContext@U2@@QBE_JXZ 10027060     U2View:U2View.dll
 0002:00001064       __imp_?triggerAutoAnnotationsUpdate@AutoAnnotationUtils@U2@@SAXPAVADVSequenceObjectContext@2@ABVQString@@@Z 10027064     U2View:U2View.dll
 0002:00001068       __imp_?staticMetaObject@AnnotatedDNAView@U2@@2UQMetaObject@@B 10027068     U2View:U2View.dll
 0002:0000106c       \177U2View_NULL_THUNK_DATA 1002706c     U2View:U2View.dll
 0002:00001070       ___xc_a                    10027070     MSVCRT:cinitexe.obj
 0002:000013ac       ___xc_z                    100273ac     MSVCRT:cinitexe.obj
 0002:000013b0       ___xi_a                    100273b0     MSVCRT:cinitexe.obj
 0002:000013bc       ___xi_z                    100273bc     MSVCRT:cinitexe.obj
 0002:000013fc       ??_7error_category@std@@6B@ 100273fc     ORFDialog.obj
 0002:00001418       ??_7_Generic_error_category@std@@6B@ 10027418     ORFDialog.obj
 0002:00001430       ??_C@_07DCLBNMLN@generic?$AA@ 10027430     ORFDialog.obj
 0002:00001438       ??_C@_0O@BFJCFAAK@unknown?5error?$AA@ 10027438     ORFDialog.obj
 0002:0000144c       ??_7_Iostream_error_category@std@@6B@ 1002744c     ORFDialog.obj
 0002:00001464       ??_C@_08LLGCOLLL@iostream?$AA@ 10027464     ORFDialog.obj
 0002:00001470       ??_C@_0BG@PADBLCHM@iostream?5stream?5error?$AA@ 10027470     ORFDialog.obj
 0002:0000148c       ??_7_System_error_category@std@@6B@ 1002748c     ORFDialog.obj
 0002:000014a4       ??_C@_06FHFOAHML@system?$AA@ 100274a4     ORFDialog.obj
 0002:000014b4       ??_SQWidget@@6BQObject@@@  100274b4     ORFDialog.obj
 0002:0000156c       ??_SQWidget@@6BQPaintDevice@@@ 1002756c     ORFDialog.obj
 0002:0000158c       ??_SQCheckBox@@6BQObject@@@ 1002758c     ORFDialog.obj
 0002:00001650       ??_SQCheckBox@@6BQPaintDevice@@@ 10027650     ORFDialog.obj
 0002:00001674       ??_SQTabWidget@@6BQObject@@@ 10027674     ORFDialog.obj
 0002:00001734       ??_SQTabWidget@@6BQPaintDevice@@@ 10027734     ORFDialog.obj
 0002:00001754       ??_SQComboBox@@6BQObject@@@ 10027754     ORFDialog.obj
 0002:00001814       ??_SQComboBox@@6BQPaintDevice@@@ 10027814     ORFDialog.obj
 0002:00001834       ??_SQDialogButtonBox@@6BQObject@@@ 10027834     ORFDialog.obj
 0002:000018ec       ??_SQDialogButtonBox@@6BQPaintDevice@@@ 100278ec     ORFDialog.obj
 0002:0000190c       ??_SQSpacerItem@@6B@       1002790c     ORFDialog.obj
 0002:00001954       ??_SQHBoxLayout@@6BQObject@@@ 10027954     ORFDialog.obj
 0002:0000199c       ??_SQHBoxLayout@@6BQLayoutItem@@@ 1002799c     ORFDialog.obj
 0002:000019e4       ??_SQVBoxLayout@@6BQObject@@@ 100279e4     ORFDialog.obj
 0002:00001a2c       ??_SQVBoxLayout@@6BQLayoutItem@@@ 10027a2c     ORFDialog.obj
 0002:00001a74       ??_SQGridLayout@@6BQObject@@@ 10027a74     ORFDialog.obj
 0002:00001abc       ??_SQGridLayout@@6BQLayoutItem@@@ 10027abc     ORFDialog.obj
 0002:00001b04       ??_SQGroupBox@@6BQObject@@@ 10027b04     ORFDialog.obj
 0002:00001bbc       ??_SQGroupBox@@6BQPaintDevice@@@ 10027bbc     ORFDialog.obj
 0002:00001bdc       ??_SQLabel@@6BQObject@@@   10027bdc     ORFDialog.obj
 0002:00001c94       ??_SQLabel@@6BQPaintDevice@@@ 10027c94     ORFDialog.obj
 0002:00001cb4       ??_SQPushButton@@6BQObject@@@ 10027cb4     ORFDialog.obj
 0002:00001d78       ??_SQPushButton@@6BQPaintDevice@@@ 10027d78     ORFDialog.obj
 0002:00001d9c       ??_SQRadioButton@@6BQObject@@@ 10027d9c     ORFDialog.obj
 0002:00001e60       ??_SQRadioButton@@6BQPaintDevice@@@ 10027e60     ORFDialog.obj
 0002:00001e84       ??_SQSpinBox@@6BQObject@@@ 10027e84     ORFDialog.obj
 0002:00001f58       ??_SQSpinBox@@6BQPaintDevice@@@ 10027f58     ORFDialog.obj
 0002:00001f7c       ??_SQTextEdit@@6BQObject@@@ 10027f7c     ORFDialog.obj
 0002:00002058       ??_SQTextEdit@@6BQPaintDevice@@@ 10028058     ORFDialog.obj
 0002:0000207c       ??_SQTreeWidget@@6BQObject@@@ 1002807c     ORFDialog.obj
 0002:000021f4       ??_SQTreeWidget@@6BQPaintDevice@@@ 100281f4     ORFDialog.obj
 0002:00002210       ??_C@_09DMINLBG@1accept?$CI?$CJ?$AA@ 10028210     ORFDialog.obj
 0002:0000221c       ??_C@_0M@MBACPLBI@2accepted?$CI?$CJ?$AA@ 1002821c     ORFDialog.obj
 0002:00002228       ??_C@_09OCDCAEKE@1reject?$CI?$CJ?$AA@ 10028228     ORFDialog.obj
 0002:00002234       ??_C@_0M@BJNBJJN@2rejected?$CI?$CJ?$AA@ 10028234     ORFDialog.obj
 0002:00002240       ??_C@_0L@OCIDPEMA@ORF?5Marker?$AA@ 10028240     ORFDialog.obj
 0002:0000224c       ??_C@_0O@IPEFOBJL@ORFDialogBase?$AA@ 1002824c     ORFDialog.obj
 0002:0000225c       ??_C@_0CF@KNNKHNPF@Find?5Open?5Reading?5Frames?5in?5sequ@ 1002825c     ORFDialog.obj
 0002:00002284       ??_C@_06KDENPHDM@Strand?$AA@ 10028284     ORFDialog.obj
 0002:0000228c       ??_C@_0BH@ONHDDBKG@Search?5in?5both?5strands?$AA@ 1002828c     ORFDialog.obj
 0002:000022a4       ??_C@_04IGHHMFLN@Both?$AA@ 100282a4     ORFDialog.obj
 0002:000022ac       ??_C@_0CE@NHBJLAMG@Search?5frames?5in?5direct?5strand?5o@ 100282ac     ORFDialog.obj
 0002:000022d0       ??_C@_06HDAEFCGM@Direct?$AA@ 100282d0     ORFDialog.obj
 0002:000022d8       ??_C@_0CI@DAAJKLCI@Search?5frames?5in?5complement?5stra@ 100282d8     ORFDialog.obj
 0002:00002300       ??_C@_0L@IKCNMPAO@Complement?$AA@ 10028300     ORFDialog.obj
 0002:0000230c       ??_C@_0BA@OPIBFEIO@Search?5Settings?$AA@ 1002830c     ORFDialog.obj
 0002:0000231c       ??_C@_0CO@JEKKMGNK@Ignore?5ORFs?5shorter?5than?5the?5spe@ 1002831c     ORFDialog.obj
 0002:0000234c       ??_C@_0BA@MOGIPOIE@Min?5length?0?5bp?3?$AA@ 1002834c     ORFDialog.obj
 0002:00002360       ??_C@_0HC@EGNJOGHC@Ignore?5boundary?5ORFs?5which?5last?5@ 10028360     ORFDialog.obj
 0002:000023d4       ??_C@_0BN@KPKPLGJ@Must?5terminate?5within?5region?$AA@ 100283d4     ORFDialog.obj
 0002:000023f4       ??_C@_0DO@HAIJKOOM@Specifies?5that?5each?5ORF?5found?5mu@ 100283f4     ORFDialog.obj
 0002:00002434       ??_C@_0BL@INGEEJAA@Must?5start?5with?5init?5codon?$AA@ 10028434     ORFDialog.obj
 0002:00002450       ??_C@_0NB@DFOJGGEI@?6?5?5?5?5?5?5?5?5?5?5?5?5?5?5?5Allow?5alternativ@ 10028450     ORFDialog.obj
 0002:00002524       ??_C@_0P@FCPFMHFA@Allow?5overlaps?$AA@ 10028524     ORFDialog.obj
 0002:00002538       ??_C@_0JD@DEMGFOKD@?6?5?5?5?5?5?5?5?5?5?5?5?5?5?5?5Allow?5ORFs?5start@ 10028538     ORFDialog.obj
 0002:000025cc       ??_C@_0BO@IECFIIA@Allow?5alternative?5init?5codons?$AA@ 100285cc     ORFDialog.obj
 0002:000025f0       ??_C@_0CBJ@IJFHNNBJ@?$DM?$CBDOCTYPE?5HTML?5PUBLIC?5?$CC?9?1?1W3C?1?1D@ 100285f0     ORFDialog.obj
 0002:0000280c       ??_C@_0BD@LMOHNJLI@Include?5stop?5codon?$AA@ 1002880c     ORFDialog.obj
 0002:00002820       ??_C@_0L@MOEPGNMC@Max?5result?$AA@ 10028820     ORFDialog.obj
 0002:0000282c       ??_C@_0BF@DDGNPIME@Start?5searching?5ORFs?$AA@ 1002882c     ORFDialog.obj
 0002:00002844       ??_C@_07PCOLMHKH@Preview?$AA@ 10028844     ORFDialog.obj
 0002:0000284c       ??_C@_0O@HLFGPFCM@Clear?5results?$AA@ 1002884c     ORFDialog.obj
 0002:0000285c       ??_C@_06MHCOIGNA@Length?$AA@ 1002885c     ORFDialog.obj
 0002:00002864       ??_C@_06FLCJJPBG@Region?$AA@ 10028864     ORFDialog.obj
 0002:0000286c       ??_C@_08EEOHOBEO@Settings?$AA@ 1002886c     ORFDialog.obj
 0002:00002878       ??_C@_06PFDLEJLJ@Output?$AA@ 10028878     ORFDialog.obj
 0002:00002ec0       ??_7?$AbstractId@H@U2@@6B@ 10028ec0     ORFDialog.obj
 0002:00002ecc       ??_7AbstractInt32Id@U2@@6B@ 10028ecc     ORFDialog.obj
 0002:00002ed8       ??_7ServiceType@U2@@6B@    10028ed8     ORFDialog.obj
 0002:00002ee4       ??_SRegionSelector@U2@@6BQObject@@@ 10028ee4     ORFDialog.obj
 0002:00002f9c       ??_SRegionSelector@U2@@6BQPaintDevice@@@ 10028f9c     ORFDialog.obj
 0002:00002fbc       ??_SQTimer@@6B@            10028fbc     ORFDialog.obj
 0002:00002fe8       ??_C@_0L@JLHNEGIN@Algorithms?$AA@ 10028fe8     ORFDialog.obj
 0002:00002ff4       ??_C@_07PGLPGHFC@Console?$AA@ 10028ff4     ORFDialog.obj
 0002:00002ffc       ??_C@_0O@BOFHOPCF@Core?5Services?$AA@ 10028ffc     ORFDialog.obj
 0002:0000300c       ??_C@_0N@PPADAKBM@Input?1Output?$AA@ 1002900c     ORFDialog.obj
 0002:0000301c       ??_C@_0M@KPPBKPKK@Performance?$AA@ 1002901c     ORFDialog.obj
 0002:00003028       ??_C@_07BFDHHBBI@Scripts?$AA@ 10029028     ORFDialog.obj
 0002:00003030       ??_C@_05EEGKELMG@Tasks?$AA@ 10029030     ORFDialog.obj
 0002:00003038       ??_C@_0P@NIIOBHGA@User?5Interface?$AA@ 10029038     ORFDialog.obj
 0002:00003048       ??_C@_0N@JINCGGMN@User?5Actions?$AA@ 10029048     ORFDialog.obj
 0002:0000305c       ??_SORFFindTask@U2@@6BTask@1@@ 1002905c     ORFDialog.obj
 0002:000030ec       ??_SORFFindTask@U2@@6BORFFindResultsListener@1@@ 100290ec     ORFDialog.obj
 0002:000030f8       ??_7ORFDialog@U2@@6BQObject@@@ 100290f8     ORFDialog.obj
 0002:000031c4       ??_7ORFDialog@U2@@6BQPaintDevice@@@ 100291c4     ORFDialog.obj
 0002:000031e0       ??_C@_01CLKCMJKC@?5?$AA@   100291e0     ORFDialog.obj
 0002:000031e8       ??_SCreateAnnotationWidgetController@U2@@6B@ 100291e8     ORFDialog.obj
 0002:00003218       ??_SHelpButton@U2@@6B@     10029218     ORFDialog.obj
 0002:00003248       ??_C@_09HNEPIKCN@QAction?5?$CK?$AA@ 10029248     ORFDialog.obj
 0002:00003258       ??_7ORFListItem@U2@@6B@    10029258     ORFDialog.obj
 0002:00003274       ??_C@_08EGAMPJHA@23331164?$AA@ 10029274     ORFDialog.obj
 0002:00003280       ??_C@_02GIPFHKNO@OK?$AA@   10029280     ORFDialog.obj
 0002:00003284       ??_C@_06FMBNCPDL@Cancel?$AA@ 10029284     ORFDialog.obj
 0002:0000328c       ??_C@_0BK@BMDBLFKM@1sl_onTaskFinished?$CITask?$CK?$CJ?$AA@ 1002928c     ORFDialog.obj
 0002:000032a8       ??_C@_0BI@OCJIPCIK@2si_stateChanged?$CITask?$CK?$CJ?$AA@ 100292a8     ORFDialog.obj
 0002:000032c0       ??_C@_0O@PECEMOAH@1sl_onTimer?$CI?$CJ?$AA@ 100292c0     ORFDialog.obj
 0002:000032d0       ??_C@_0L@CHKJBFLD@2timeout?$CI?$CJ?$AA@ 100292d0     ORFDialog.obj
 0002:000032dc       ??_C@_0BJ@MGGMBPBM@1sl_translationChanged?$CI?$CJ?$AA@ 100292dc     ORFDialog.obj
 0002:000032f8       ??_C@_0BN@GJEBGMAM@2currentIndexChanged?5?$CI?5int?5?$CJ?$AA@ 100292f8     ORFDialog.obj
 0002:00003318       ??_C@_08LHPBPOIK@?$DM?1table?$DO?$AA@ 10029318     ORFDialog.obj
 0002:00003324       ??_C@_0P@PGGJDOJG@?$DM?1b?$DO?$DM?1td?$DO?$DM?1tr?$DO?$AA@ 10029324     ORFDialog.obj
 0002:00003334       ??_C@_0BP@CGDBAMHI@?$CGnbsp?$DL?$CGnbsp?$DL?$CGnbsp?$DL?$DM?1td?$DO?$DMtd?$DO?$DMb?$DO?$AA@ 10029334     ORFDialog.obj
 0002:00003354       ??_C@_0M@KCFNHPFD@Stop?5codons?$AA@ 10029354     ORFDialog.obj
 0002:00003360       ??_C@_08DCPJPKOP@?$DMtr?$DO?$DMtd?$DO?$AA@ 10029360     ORFDialog.obj
 0002:0000336c       ??_C@_0BJ@NPBBGMEP@Alternative?5start?5codons?$AA@ 1002936c     ORFDialog.obj
 0002:00003388       ??_C@_0N@FOAIKFKL@Start?5codons?$AA@ 10029388     ORFDialog.obj
 0002:00003398       ??_C@_0BB@NOHPIHBL@?$DMtable?5border?$DN0?$DO?$AA@ 10029398     ORFDialog.obj
 0002:000033ac       ??_C@_0BC@FCKEKKGE@1sl_onClearList?$CI?$CJ?$AA@ 100293ac     ORFDialog.obj
 0002:000033c0       ??_C@_0L@OELOHDKG@2clicked?$CI?$CJ?$AA@ 100293c0     ORFDialog.obj
 0002:000033cc       ??_C@_0BA@MJHBHLOA@1sl_onFindAll?$CI?$CJ?$AA@ 100293cc     ORFDialog.obj
 0002:000033dc       ??_C@_0CN@POLJMCFM@1sl_onResultActivated?$CIQTreeWidge@ 100293dc     ORFDialog.obj
 0002:0000340c       ??_C@_0CG@LPAMFNML@2itemActivated?$CIQTreeWidgetItem?$CK?0@ 1002940c     ORFDialog.obj
 0002:00003434       ??_C@_0N@EMHIDDIN@Progress?5?$CF1?$CF?$AA@ 10029434     ORFDialog.obj
 0002:00003444       ??_C@_0BC@LPKCGDFP@?$CF1?5results?5found?4?$AA@ 10029444     ORFDialog.obj
 0002:00003458       ??_C@_0DP@MIFBBEOI@Results?5list?5contains?5results?5fr@ 10029458     ORFDialog.obj
 0002:00003498       ??_C@_05NAOIJFC@Error?$AA@ 10029498     ORFDialog.obj
 0002:000034a0       ??_C@_0DK@NFDOGBNG@Cannot?5create?5an?5annotation?5obje@ 100294a0     ORFDialog.obj
 0002:000034dc       ??_C@_0CK@IGBIANDN@Trying?5to?5recover?5from?5error?3?5?$CF1@ 100294dc     ORFDialog.obj
 0002:00003508       ??_C@_0BI@JONIHIHH@Sequence?5object?5is?5NULL?$AA@ 10029508     ORFDialog.obj
 0002:00003520       ??_C@_0BC@LCFODOKG@src?2ORFDialog?4cpp?$AA@ 10029520     ORFDialog.obj
 0002:00003534       ??_C@_0DG@HABLGPNH@Bad?5conversion?5from?5Task?5to?5Auto@ 10029534     ORFDialog.obj
 0002:0000356c       ??_C@_0L@NCNGAHOM@?5?$FL?$CF1?4?4?$CF2?$FN?5?$AA@ 1002956c     ORFDialog.obj
 0002:00003578       ??_C@_0BF@JBHLLBBO@?5?$FL?$CF1?4?4?$CF2?$FN?0?5?$FL?$CF3?4?4?$CF4?$FN?5?$AA@ 10029578     ORFDialog.obj
 0002:00003590       ??_C@_0BA@JFNIOLAK@string?5too?5long?$AA@ 10029590     ORFDialog.obj
 0002:000035a0       ??_C@_0BI@CFPLBAOH@invalid?5string?5position?$AA@ 100295a0     ORFDialog.obj
 0002:000035bc       ??_SADVGlobalAction@U2@@6B@ 100295bc     ORFMarkerPlugin.obj
 0002:000035ec       ??_7ORFMarkerPlugin@U2@@6B@ 100295ec     ORFMarkerPlugin.obj
 0002:0000361c       ??_7ORFViewContext@U2@@6BQObject@@@ 1002961c     ORFMarkerPlugin.obj
 0002:0000366c       ??_7ORFViewContext@U2@@6BGObjectViewObjectHandler@1@@ 1002966c     ORFMarkerPlugin.obj
 0002:00003680       ??_7GTest_ORFMarkerTaskFactory@GTest_ORFMarkerTask@U2@@6B@ 10029680     ORFMarkerPlugin.obj
 0002:0000368c       ??_7GTest_ORFMarkerTask@U2@@6B@ 1002968c     ORFMarkerPlugin.obj
 0002:00003718       ??_C@_0BJ@OBGCHOF@plugin_orf?9marker?9search?$AA@ 10029718     ORFMarkerPlugin.obj
 0002:00003734       ??_C@_0CC@NEGBEPMD@?3orf_marker?1images?1orf_marker?4pn@ 10029734     ORFMarkerPlugin.obj
 0002:00003758       ??_C@_0DK@MMEJLADJ@Searches?5for?5open?5reading?5frames@ 10029758     ORFMarkerPlugin.obj
 0002:00003794       ??_C@_03PEIMBJDE@XML?$AA@  10029794     ORFMarkerPlugin.obj
 0002:0000379c       ??_7?$GAutoDeleteList@VXMLTestFactory@U2@@@U2@@6B@ 1002979c     ORFMarkerPlugin.obj
 0002:000037c8       ??_C@_0BB@JDMPMKOK@AnnotatedDNAView?$AA@ 100297c8     ORFMarkerPlugin.obj
 0002:000037dc       ??_C@_0N@FKPKNLHP@Find?5ORFs?4?4?4?$AA@ 100297dc     ORFMarkerPlugin.obj
 0002:000037ec       ??_C@_09JIHNLCO@Find?5ORFs?$AA@ 100297ec     ORFMarkerPlugin.obj
 0002:000037f8       ??_C@_0BB@CHMBMKNM@1sl_showDialog?$CI?$CJ?$AA@ 100297f8     ORFMarkerPlugin.obj
 0002:0000380c       ??_C@_0N@NBJIAFIH@2triggered?$CI?$CJ?$AA@ 1002980c     ORFMarkerPlugin.obj
 0002:00003819       ??_C@_00CNPNBAHC@?$AA@     10029819     ORFMarkerTask.obj
 0002:0000381c       ??_C@_0N@GPLPHLED@U2?3?3U2Region?$AA@ 1002981c     ORFMarkerTask.obj
 0002:00003834       ??_SCreateAnnotationsTask@U2@@6B@ 10029834     ORFMarkerTask.obj
 0002:000038c4       ??_7FindORFsToAnnotationsTask@U2@@6B@ 100298c4     ORFMarkerTask.obj
 0002:00003954       ??_7ORFAutoAnnotationsUpdater@U2@@6B@ 10029954     ORFMarkerTask.obj
 0002:00003988       ??_C@_0BC@JCKADFML@orf_finder?1strand?$AA@ 10029988     ORFMarkerTask.obj
 0002:0000399c       ??_C@_0BL@KAEOCAPG@orf_finder?1allow_alt_start?$AA@ 1002999c     ORFMarkerTask.obj
 0002:000039b8       ??_C@_0BJ@BOBJGNHD@orf_finder?1allow_overlap?$AA@ 100299b8     ORFMarkerTask.obj
 0002:000039d4       ??_C@_0BI@OJGBFPBB@orf_finder?1amino_transl?$AA@ 100299d4     ORFMarkerTask.obj
 0002:000039ec       ??_C@_0BG@OFGFPAHL@orf_finder?1min_length?$AA@ 100299ec     ORFMarkerTask.obj
 0002:00003a04       ??_C@_0BE@BJGEEMAH@orf_finder?1must_fit?$AA@ 10029a04     ORFMarkerTask.obj
 0002:00003a18       ??_C@_0BF@NOFHNCFG@orf_finder?1must_init?$AA@ 10029a18     ORFMarkerTask.obj
 0002:00003a30       ??_C@_0BC@GKMEFNOB@orf_finder?1region?$AA@ 10029a30     ORFMarkerTask.obj
 0002:00003a44       ??_C@_0BO@MELLDODI@orf_finder?1incldue_stop_codon?$AA@ 10029a44     ORFMarkerTask.obj
 0002:00003a64       ??_C@_0BG@IIKLAPFF@orf_finder?1max_result?$AA@ 10029a64     ORFMarkerTask.obj
 0002:00003a7c       ??_C@_0BN@PCFNBNAO@orf_finder?1is_result_limited?$AA@ 10029a7c     ORFMarkerTask.obj
 0002:00003a9c       ??_C@_0CC@EIOINLNM@Find?5ORFs?5and?5save?5to?5annotation@ 10029a9c     ORFMarkerTask.obj
 0002:00003ac0       ??_C@_0CB@LCDMMNCG@Annotation?5table?5object?5is?5NULL?$CB@ 10029ac0     ORFMarkerTask.obj
 0002:00003ae4       ??_C@_04PCHPNLBE@ORFs?$AA@ 10029ae4     ORFMarkerTask.obj
 0002:00003aec       ??_C@_05LAPONLG@false?$AA@ 10029aec     ORFMarkerTests.obj
 0002:00003af4       ??_C@_04LOAJBDKD@true?$AA@ 10029af4     ORFMarkerTests.obj
 0002:00003afc       ??_C@_0P@PMGBHMNA@NCBI?9GenBank?5?$CD?$AA@ 10029afc     ORFMarkerTests.obj
 0002:00003b0c       ??_C@_03NPAJGOON@seq?$AA@  10029b0c     ORFMarkerTests.obj
 0002:00003b10       ??_C@_0BB@HOHIPJMP@expected_results?$AA@ 10029b10     ORFMarkerTests.obj
 0002:00003b24       ??_C@_02FMCJJKJH@?2?0?$AA@ 10029b24     ORFMarkerTests.obj
 0002:00003b28       ??_C@_03GGLEPCDP@?2?4?4?$AA@ 10029b28     ORFMarkerTests.obj
 0002:00003b2c       ??_C@_0BD@KFLBPKCI@wrong?5value?5for?5?$CF1?$AA@ 10029b2c     ORFMarkerTests.obj
 0002:00003b40       ??_C@_06GMPAMOKA@strand?$AA@ 10029b40     ORFMarkerTests.obj
 0002:00003b48       ??_C@_06LMLJGLPA@direct?$AA@ 10029b48     ORFMarkerTests.obj
 0002:00003b50       ??_C@_0L@HLHDIAKC@compliment?$AA@ 10029b50     ORFMarkerTests.obj
 0002:00003b5c       ??_C@_04EHLGOKLJ@both?$AA@ 10029b5c     ORFMarkerTests.obj
 0002:00003b64       ??_C@_0BF@NBBMDMMA@value?5not?5correct?5?$CF1?$AA@ 10029b64     ORFMarkerTests.obj
 0002:00003b7c       ??_C@_0L@FAGNJOAH@min_length?$AA@ 10029b7c     ORFMarkerTests.obj
 0002:00003b88       ??_C@_0CC@BPKGOACI@Unable?5to?5convert?4?5Value?5wrong?5?$CF@ 10029b88     ORFMarkerTests.obj
 0002:00003bac       ??_C@_0BH@LDHJLCKA@terminates_with_region?$AA@ 10029bac     ORFMarkerTests.obj
 0002:00003bc4       ??_C@_0BH@CAOIGML@starts_with_init_codon?$AA@ 10029bc4     ORFMarkerTests.obj
 0002:00003bdc       ??_C@_0BD@NGJNBBOL@include_stop_codon?$AA@ 10029bdc     ORFMarkerTests.obj
 0002:00003bf0       ??_C@_0BG@NKJGOGNO@allow_alt_init_codons?$AA@ 10029bf0     ORFMarkerTests.obj
 0002:00003c08       ??_C@_0P@GGGFGOBO@translation_id?$AA@ 10029c08     ORFMarkerTests.obj
 0002:00003c18       ??_C@_0CE@EKPFDHP@Can?8t?5cast?5to?5sequence?5from?5GObj@ 10029c18     ORFMarkerTests.obj
 0002:00003c3c       ??_C@_0DK@JABDGHFK@Expected?5and?5Actual?5lists?5of?5reg@ 10029c3c     ORFMarkerTests.obj
 0002:00003c78       ??_C@_0DB@DGHNLACP@One?5of?5the?5expected?5regions?5not?5@ 10029c78     ORFMarkerTests.obj
 0002:00003cb4       ??_STask@U2@@6B@           10029cb4     ORFQuery.obj
 0002:00003d44       ??_SAttribute@U2@@6B@      10029d44     ORFQuery.obj
 0002:00003d70       ??_7QDORFActor@U2@@6B@     10029d70     ORFQuery.obj
 0002:00003dc4       ??_7QDORFActorPrototype@U2@@6B@ 10029dc4     ORFQuery.obj
 0002:00003dd4       ??_SDelegateEditor@U2@@6B@ 10029dd4     ORFQuery.obj
 0002:00003e2c       ??_SSpinBoxDelegate@U2@@6B@ 10029e2c     ORFQuery.obj
 0002:00003eac       ??_SComboBoxDelegate@U2@@6B@ 10029eac     ORFQuery.obj
 0002:00003f2c       ??_STaskSignalMapper@U2@@6B@ 10029f2c     ORFQuery.obj
 0002:00003f5c       ??_SFailTask@U2@@6B@       10029f5c     ORFQuery.obj
 0002:00003fe8       ??_C@_08OPEOHFOO@trans?9id?$AA@ 10029fe8     ORFQuery.obj
 0002:00003ff4       ??_C@_0L@LOBIAIOK@min?9length?$AA@ 10029ff4     ORFQuery.obj
 0002:00004000       ??_C@_0BB@BCJGPBEB@starts?9with?9init?$AA@ 1002a000     ORFQuery.obj
 0002:00004014       ??_C@_0L@BEEJOPLC@stop?9codon?$AA@ 1002a014     ORFQuery.obj
 0002:00004020       ??_C@_09CPOEIL@alt?9start?$AA@ 1002a020     ORFQuery.obj
 0002:0000402c       ??_C@_0L@HCBFHDOF@max?9length?$AA@ 1002a02c     ORFQuery.obj
 0002:00004038       ??_C@_0BF@IPIPHCJL@max?9result?9attribute?$AA@ 1002a038     ORFQuery.obj
 0002:00004050       ??_C@_0O@LNBHIKLK@limit?9results?$AA@ 1002a050     ORFQuery.obj
 0002:00004060       ??_C@_03NJCMLHKJ@orf?$AA@  1002a060     ORFQuery.obj
 0002:00004064       ??_C@_03NENHHKNF@ORF?$AA@  1002a064     ORFQuery.obj
 0002:00004068       ??_C@_0N@ICKNJLMC@both?5strands?$AA@ 1002a068     ORFQuery.obj
 0002:00004078       ??_C@_0O@LLCLNCHA@direct?5strand?$AA@ 1002a078     ORFQuery.obj
 0002:00004088       ??_C@_0BC@KBGHFOJB@complement?5strand?$AA@ 1002a088     ORFQuery.obj
 0002:0000409c       ??_C@_0BC@OFGBKPMA@?$DMa?5href?$DN?$CF1?$DO?$CF2?$DM?1a?$DO?$AA@ 1002a09c     ORFQuery.obj
 0002:000040b0       ??_C@_0EC@EAJHOALJ@?0?5allow?5ORFs?5?$DMu?$DOstarting?5with?5an@ 1002a0b0     ORFQuery.obj
 0002:000040f4       ??_C@_0DE@MGCJHKEG@?0?5take?5into?5account?5?$DMu?$DOalternati@ 1002a0f4     ORFQuery.obj
 0002:00004128       ??_C@_0CE@IIMHGOHP@?0?5?$DMu?$DOignore?5non?9terminated?$DM?1u?$DO?5O@ 1002a128     ORFQuery.obj
 0002:0000414c       ??_C@_0BG@BGLMAAFO@?$DMa?5href?$DN?$CF1?$DO?$CF2?5bps?$DM?1a?$DO?$AA@ 1002a14c     ORFQuery.obj
 0002:00004168       ??_C@_0HE@JLOPJEJD@Finds?5ORFs?5in?5?$DMu?$DO?$CF1?$DM?1u?$DO?5using?5th@ 1002a168     ORFQuery.obj
 0002:000041dc       ??_C@_0N@KJBINPCE@Bad?5sequence?$AA@ 1002a1dc     ORFQuery.obj
 0002:000041ec       ??_C@_08DMCNOEKE@ORF?5find?$AA@ 1002a1ec     ORFQuery.obj
 0002:000041f8       ??_C@_0CD@LIIDOBKP@1sl_onAlgorithmTaskFinished?$CITask@ 1002a1f8     ORFQuery.obj
 0002:0000421c       ??_C@_0BI@KGADHDJC@2si_taskFinished?$CITask?$CK?$CJ?$AA@ 1002a21c     ORFQuery.obj
 0002:00004234       ??_C@_01HIHLOKLC@1?$AA@    1002a234     ORFQuery.obj
 0002:00004238       ??_C@_0BOO@EIPPEIOK@Finds?5Open?5Reading?5Frames?5?$CIORFs?$CJ@ 1002a238     ORFQuery.obj
 0002:00004428       ??_C@_0FB@KNJDAFMM@Which?5genetic?5code?5should?5be?5use@ 1002a428     ORFQuery.obj
 0002:0000447c       ??_C@_0N@IAHCCLEN@Genetic?5code?$AA@ 1002a47c     ORFQuery.obj
 0002:00004490       ??_C@_0GH@FKGPJGCL@?6Ignore?5boundary?5ORFs?5which?5last@ 1002a490     ORFQuery.obj
 0002:000044f8       ??_C@_0BD@BENGIIGF@Require?5init?5codon?$AA@ 1002a4f8     ORFQuery.obj
 0002:00004510       ??_C@_0IG@FILHLMKI@?6?5?5?5?5?5?5?5?5?5?5?5?5?5?5?5Allow?5ORFs?5start@ 1002a510     ORFQuery.obj
 0002:00004598       ??_C@_0BJ@JCJBFOFO@Allow?5alternative?5codons?$AA@ 1002a598     ORFQuery.obj
 0002:000045b4       ??_C@_0CG@LLLKDOJP@Maximum?5length?5of?5annotation?5all@ 1002a5b4     ORFQuery.obj
 0002:000045dc       ??_C@_0L@GPIMOJOD@Max?5length?$AA@ 1002a5dc     ORFQuery.obj
 0002:000045e8       ??_C@_0BE@MMEPPCOK@Require?5stop?5codon?4?$AA@ 1002a5e8     ORFQuery.obj
 0002:000045fc       ??_C@_0BD@JPFDHCHL@Require?5stop?5codon?$AA@ 1002a5fc     ORFQuery.obj
 0002:00004610       ??_C@_0CO@MGHNAPNA@Find?5results?5not?5achieved?5by?5spe@ 1002a610     ORFQuery.obj
 0002:00004640       ??_C@_0DP@NHBMKOEC@The?5amount?5of?5results?5will?5be?5li@ 1002a640     ORFQuery.obj
 0002:00004680       ??_C@_0O@IBDMBFDF@Limit?5results?$AA@ 1002a680     ORFQuery.obj
 0002:00004690       ??_C@_0BA@EAHCLEBK@NCBI?9GenBank?5?$CD1?$AA@ 1002a690     ORFQuery.obj
 0002:000046a0       ??_C@_07CCOEHHFD@minimum?$AA@ 1002a6a0     ORFQuery.obj
 0002:000046a8       ??_C@_07MEIENILC@maximum?$AA@ 1002a6a8     ORFQuery.obj
 0002:000046b0       ??_C@_06EMCDFPCG@suffix?$AA@ 1002a6b0     ORFQuery.obj
 0002:000046bc       ??_SDescriptor@U2@@6B@     1002a6bc     ORFWorker.obj
 0002:000046c4       ??_SMapDataType@U2@@6B@    1002a6c4     ORFWorker.obj
 0002:000046d8       ??_C@_0CD@LMLLOHBG@U2?3?3Workflow?3?3SharedDbiDataHandl@ 1002a6d8     ORFWorker.obj
 0002:000046fc       ??_C@_0BF@COKBMJP@Script?5task?5canceled?$AA@ 1002a6fc     ORFWorker.obj
 0002:00004718       ??_SPortDescriptor@Workflow@U2@@6B@ 1002a718     ORFWorker.obj
 0002:00004728       ??_SIntegralBusActorPrototype@Workflow@U2@@6B@ 1002a728     ORFWorker.obj
 0002:0000473c       ??_7?$PrompterBase@VORFPrompter@LocalWorkflow@U2@@@U2@@6BActorDocument@Workflow@1@@ 1002a73c     ORFWorker.obj
 0002:00004784       ??_7?$PrompterBase@VORFPrompter@LocalWorkflow@U2@@@U2@@6BPrompter@Workflow@1@@ 1002a784     ORFWorker.obj
 0002:00004790       ??_7ORFPrompter@LocalWorkflow@U2@@6BActorDocument@Workflow@2@@ 1002a790     ORFWorker.obj
 0002:000047d8       ??_7ORFPrompter@LocalWorkflow@U2@@6BPrompter@Workflow@2@@ 1002a7d8     ORFWorker.obj
 0002:000047e4       ??_7ORFWorker@LocalWorkflow@U2@@6BQObject@@@ 1002a7e4     ORFWorker.obj
 0002:00004828       ??_7ORFWorker@LocalWorkflow@U2@@6BWorker@Workflow@2@@ 1002a828     ORFWorker.obj
 0002:00004844       ??_7ORFWorker@LocalWorkflow@U2@@6BCommunicationSubject@Workflow@2@@ 1002a844     ORFWorker.obj
 0002:00004854       ??_7ORFWorkerFactory@LocalWorkflow@U2@@6B?$IdRegistry@VDomainFactory@Workflow@U2@@@2@@ 1002a854     ORFWorker.obj
 0002:00004880       ??_7ORFWorkerFactory@LocalWorkflow@U2@@6BDescriptor@2@@ 1002a880     ORFWorker.obj
 0002:00004884       ??_C@_0M@BDNOGNHP@result?9name?$AA@ 1002a884     ORFWorker.obj
 0002:00004890       ??_C@_0N@IPJCHDGG@genetic?9code?$AA@ 1002a890     ORFWorker.obj
 0002:000048a0       ??_C@_0BD@EGKPGEEB@require?9stop?9codon?$AA@ 1002a8a0     ORFWorker.obj
 0002:000048b4       ??_C@_0BD@MNCKJOFP@require?9init?9codon?$AA@ 1002a8b4     ORFWorker.obj
 0002:000048c8       ??_C@_0BJ@POLADPO@allow?9alternative?9codons?$AA@ 1002a8c8     ORFWorker.obj
 0002:000048e4       ??_C@_0BD@GFBLMPIC@include?9stop?9codon?$AA@ 1002a8e4     ORFWorker.obj
 0002:000048f8       ??_C@_0L@OPIKAAIC@orf?9search?$AA@ 1002a8f8     ORFWorker.obj
 0002:00004908       ??_C@_0EI@LBNACHPJ@A?5nucleotide?5sequence?5to?5search?5@ 1002a908     ORFWorker.obj
 0002:00004950       ??_C@_0BA@GLOOOALC@Input?5sequences?$AA@ 1002a950     ORFWorker.obj
 0002:00004960       ??_C@_0DJ@DNJEHCOK@A?5set?5of?5annotations?5marking?5ORF@ 1002a960     ORFWorker.obj
 0002:0000499c       ??_C@_0BA@EGDPMJAO@ORF?5annotations?$AA@ 1002a99c     ORFWorker.obj
 0002:000049ac       ??_C@_0N@GAGJECNB@orf?4sequence?$AA@ 1002a9ac     ORFWorker.obj
 0002:000049bc       ??_C@_0BA@OOEHPIIF@orf?4annotations?$AA@ 1002a9bc     ORFWorker.obj
 0002:000049cc       ??_C@_0DD@IHHCJGGN@Name?5of?5the?5result?5annotations?5m@ 1002a9cc     ORFWorker.obj
 0002:00004a00       ??_C@_0M@EIDFEOEK@Annotate?5as?$AA@ 1002aa00     ORFWorker.obj
 0002:00004a0c       ??_C@_0CP@GNJFJICA@Ignore?5ORFs?5shorter?5than?5the?5spe@ 1002aa0c     ORFWorker.obj
 0002:00004a40       ??_C@_0EG@MCIEJPFG@The?5result?5annotation?5will?5inclu@ 1002aa40     ORFWorker.obj
 0002:00004a88       ??_C@_0EA@JDACDFDO@The?5amount?5of?5results?5will?5be?5li@ 1002aa88     ORFWorker.obj
 0002:00004ac8       ??_C@_0CAF@EMIENMLI@Finds?5Open?5Reading?5Frames?5?$CIORFs?$CJ@ 1002aac8     ORFWorker.obj
 0002:00004cd0       ??_C@_07HNEBHIML@?$DM?1font?$DO?$AA@ 1002acd0     ORFWorker.obj
 0002:00004cd8       ??_C@_05EPBFLBEJ@unset?$AA@ 1002acd8     ORFWorker.obj
 0002:00004ce0       ??_C@_0BD@HCEOAMGB@?$DMfont?5color?$DN?8red?8?$DO?$AA@ 1002ace0     ORFWorker.obj
 0002:00004cf4       ??_C@_0BA@PDDMPIAN@?5from?5?$DMu?$DO?$CF1?$DM?1u?$DO?$AA@ 1002acf4     ORFWorker.obj
 0002:00004d04       ??_C@_0BI@JADCNBNE@starting?5with?5any?5codon?$AA@ 1002ad04     ORFWorker.obj
 0002:00004d1c       ??_C@_0CG@COHCIFFG@?0?5allow?5ORFs?5?$CF1?5other?5than?5termi@ 1002ad1c     ORFWorker.obj
 0002:00004d44       ??_C@_0BJ@GPDPCCJD@alternative?5start?5codons?$AA@ 1002ad44     ORFWorker.obj
 0002:00004d60       ??_C@_0BH@NMCLMPM@?0?5take?5into?5account?5?$CF1?$AA@ 1002ad60     ORFWorker.obj
 0002:00004d78       ??_C@_0BG@DLNGKIJJ@ignore?5non?9terminated?$AA@ 1002ad78     ORFWorker.obj
 0002:00004d90       ??_C@_09LIGJOCGA@?0?5?$CF1?5ORFs?$AA@ 1002ad90     ORFWorker.obj
 0002:00004da0       ??_C@_0LO@GJDBIFJJ@For?5each?5nucleotide?5sequence?$CF1?0?5@ 1002ada0     ORFWorker.obj
 0002:00004e60       ??_C@_0CN@FMIACCHB@ORF?3?5result?5name?5is?5empty?0?5defau@ 1002ae60     ORFWorker.obj
 0002:00004e90       ??_C@_0N@OPLKHDBO@misc_feature?$AA@ 1002ae90     ORFWorker.obj
 0002:00004ea0       ??_C@_0DL@ODLAHPEL@ORF?3?5Incorrect?5value?3?5min?9length@ 1002aea0     ORFWorker.obj
 0002:00004edc       ??_C@_0DG@MBKLONAJ@Incorrect?5value?3?5min?9length?5must@ 1002aedc     ORFWorker.obj
 0002:00004f14       ??_C@_0BD@GBNMGBMK@1sl_taskFinished?$CI?$CJ?$AA@ 1002af14     ORFWorker.obj
 0002:00004f28       ??_C@_0BD@PFECGAMD@2si_stateChanged?$CI?$CJ?$AA@ 1002af28     ORFWorker.obj
 0002:00004f3c       ??_C@_0CH@BHOCGDJK@Bad?5sequence?5supplied?5to?5ORFWork@ 1002af3c     ORFWorker.obj
 0002:00004f64       ??_C@_0M@EFOOKMBN@Annotations?$AA@ 1002af64     ORFWorker.obj
 0002:00004f70       ??_C@_0O@CJIGEMHD@Found?5?$CF1?5ORFs?$AA@ 1002af70     ORFWorker.obj
 0002:00004f80       ??_C@_0BE@LGBLLFOL@1sl_actorModified?$CI?$CJ?$AA@ 1002af80     ORFWorker.obj
 0002:00004f94       ??_C@_0BD@FGIDJNMI@2si_labelChanged?$CI?$CJ?$AA@ 1002af94     ORFWorker.obj
 0002:00004fa8       ??_C@_0P@DIBOLHGA@2si_modified?$CI?$CJ?$AA@ 1002afa8     ORFWorker.obj
 0002:00004fb8       ??_C@_0BC@HBGBGNIM@2bindingChanged?$CI?$CJ?$AA@ 1002afb8     ORFWorker.obj
 0002:00005264       ??_C@_0BB@BHIDNNBC@Ui_ORFDialogBase?$AA@ 1002b264     moc_ORFDialog.obj
 0002:000059e0       ?value@?$integral_constant@_N$0A@@std@@2_NB 1002b9e0     MSVCRT:ti_inst.obj
 0002:000059e1       ?value@?$integral_constant@_N$00@std@@2_NB 1002b9e1     MSVCRT:ti_inst.obj
 0002:000059e8       ??_7type_info@@6B@         1002b9e8     MSVCRT:ti_inst.obj
 0002:000059ec       __pRawDllMain              1002b9ec     MSVCRT:crtdll.obj
 0002:000059ec       __pDefaultRawDllMain       1002b9ec     MSVCRT:crtdll.obj
 0002:000059f8       ?ProcessDetach@NativeDll@<CrtImplementationDetails>@@0IB 1002b9f8     MSVCRT:initsect.obj
 0002:000059fc       ?ProcessAttach@NativeDll@<CrtImplementationDetails>@@0IB 1002b9fc     MSVCRT:initsect.obj
 0002:00005a00       ?ThreadAttach@NativeDll@<CrtImplementationDetails>@@0IB 1002ba00     MSVCRT:initsect.obj
 0002:00005a04       ?ThreadDetach@NativeDll@<CrtImplementationDetails>@@0IB 1002ba04     MSVCRT:initsect.obj
 0002:00005a08       ?ProcessVerifier@NativeDll@<CrtImplementationDetails>@@0IB 1002ba08     MSVCRT:initsect.obj
 0002:00005a10       __load_config_used         1002ba10     MSVCRT:loadcfg.obj
 0002:00005ac8       ??_R4error_category@std@@6B@ 1002bac8     ORFDialog.obj
 0002:00005adc       ??_R3error_category@std@@8 1002badc     ORFDialog.obj
 0002:00005aec       ??_R2error_category@std@@8 1002baec     ORFDialog.obj
 0002:00005af4       ??_R1A@?0A@EA@error_category@std@@8 1002baf4     ORFDialog.obj
 0002:00005b10       ??_R4_Generic_error_category@std@@6B@ 1002bb10     ORFDialog.obj
 0002:00005b24       ??_R3_Generic_error_category@std@@8 1002bb24     ORFDialog.obj
 0002:00005b34       ??_R2_Generic_error_category@std@@8 1002bb34     ORFDialog.obj
 0002:00005b40       ??_R1A@?0A@EA@_Generic_error_category@std@@8 1002bb40     ORFDialog.obj
 0002:00005b5c       ??_R4_Iostream_error_category@std@@6B@ 1002bb5c     ORFDialog.obj
 0002:00005b70       ??_R3_Iostream_error_category@std@@8 1002bb70     ORFDialog.obj
 0002:00005b80       ??_R2_Iostream_error_category@std@@8 1002bb80     ORFDialog.obj
 0002:00005b90       ??_R1A@?0A@EA@_Iostream_error_category@std@@8 1002bb90     ORFDialog.obj
 0002:00005bac       ??_R4_System_error_category@std@@6B@ 1002bbac     ORFDialog.obj
 0002:00005bc0       ??_R3_System_error_category@std@@8 1002bbc0     ORFDialog.obj
 0002:00005bd0       ??_R2_System_error_category@std@@8 1002bbd0     ORFDialog.obj
 0002:00005be0       ??_R1A@?0A@EA@_System_error_category@std@@8 1002bbe0     ORFDialog.obj
 0002:00005bfc       ??_R4QWidget@@6BQObject@@@ 1002bbfc     ORFDialog.obj
 0002:00005c10       ??_R3QWidget@@8            1002bc10     ORFDialog.obj
 0002:00005c20       ??_R2QWidget@@8            1002bc20     ORFDialog.obj
 0002:00005c30       ??_R1A@?0A@EA@QWidget@@8   1002bc30     ORFDialog.obj
 0002:00005c4c       ??_R1A@?0A@EA@QObject@@8   1002bc4c     ORFDialog.obj
 0002:00005c68       ??_R3QObject@@8            1002bc68     ORFDialog.obj
 0002:00005c78       ??_R2QObject@@8            1002bc78     ORFDialog.obj
 0002:00005c80       ??_R17?0A@EA@QPaintDevice@@8 1002bc80     ORFDialog.obj
 0002:00005c9c       ??_R3QPaintDevice@@8       1002bc9c     ORFDialog.obj
 0002:00005cac       ??_R2QPaintDevice@@8       1002bcac     ORFDialog.obj
 0002:00005cb4       ??_R1A@?0A@EA@QPaintDevice@@8 1002bcb4     ORFDialog.obj
 0002:00005cd0       ??_R4QWidget@@6BQPaintDevice@@@ 1002bcd0     ORFDialog.obj
 0002:00005ce4       ??_R4QTimer@@6B@           1002bce4     ORFDialog.obj
 0002:00005cf8       ??_R3QTimer@@8             1002bcf8     ORFDialog.obj
 0002:00005d08       ??_R2QTimer@@8             1002bd08     ORFDialog.obj
 0002:00005d14       ??_R1A@?0A@EA@QTimer@@8    1002bd14     ORFDialog.obj
 0002:00005d30       ??_R4QCheckBox@@6BQObject@@@ 1002bd30     ORFDialog.obj
 0002:00005d44       ??_R3QCheckBox@@8          1002bd44     ORFDialog.obj
 0002:00005d54       ??_R2QCheckBox@@8          1002bd54     ORFDialog.obj
 0002:00005d6c       ??_R1A@?0A@EA@QCheckBox@@8 1002bd6c     ORFDialog.obj
 0002:00005d88       ??_R1A@?0A@EA@QAbstractButton@@8 1002bd88     ORFDialog.obj
 0002:00005da4       ??_R3QAbstractButton@@8    1002bda4     ORFDialog.obj
 0002:00005db4       ??_R2QAbstractButton@@8    1002bdb4     ORFDialog.obj
 0002:00005dc8       ??_R4QCheckBox@@6BQPaintDevice@@@ 1002bdc8     ORFDialog.obj
 0002:00005ddc       ??_R4QTabWidget@@6BQObject@@@ 1002bddc     ORFDialog.obj
 0002:00005df0       ??_R3QTabWidget@@8         1002bdf0     ORFDialog.obj
 0002:00005e00       ??_R2QTabWidget@@8         1002be00     ORFDialog.obj
 0002:00005e14       ??_R1A@?0A@EA@QTabWidget@@8 1002be14     ORFDialog.obj
 0002:00005e30       ??_R4QTabWidget@@6BQPaintDevice@@@ 1002be30     ORFDialog.obj
 0002:00005e44       ??_R4QComboBox@@6BQObject@@@ 1002be44     ORFDialog.obj
 0002:00005e58       ??_R3QComboBox@@8          1002be58     ORFDialog.obj
 0002:00005e68       ??_R2QComboBox@@8          1002be68     ORFDialog.obj
 0002:00005e7c       ??_R1A@?0A@EA@QComboBox@@8 1002be7c     ORFDialog.obj
 0002:00005e98       ??_R4QComboBox@@6BQPaintDevice@@@ 1002be98     ORFDialog.obj
 0002:00005eac       ??_R4QPushButton@@6BQObject@@@ 1002beac     ORFDialog.obj
 0002:00005ec0       ??_R3QPushButton@@8        1002bec0     ORFDialog.obj
 0002:00005ed0       ??_R2QPushButton@@8        1002bed0     ORFDialog.obj
 0002:00005ee8       ??_R1A@?0A@EA@QPushButton@@8 1002bee8     ORFDialog.obj
 0002:00005f04       ??_R4QPushButton@@6BQPaintDevice@@@ 1002bf04     ORFDialog.obj
 0002:00005f18       ??_R4QDialogButtonBox@@6BQObject@@@ 1002bf18     ORFDialog.obj
 0002:00005f2c       ??_R3QDialogButtonBox@@8   1002bf2c     ORFDialog.obj
 0002:00005f3c       ??_R2QDialogButtonBox@@8   1002bf3c     ORFDialog.obj
 0002:00005f50       ??_R1A@?0A@EA@QDialogButtonBox@@8 1002bf50     ORFDialog.obj
 0002:00005f6c       ??_R4QDialogButtonBox@@6BQPaintDevice@@@ 1002bf6c     ORFDialog.obj
 0002:00005f80       ??_R4QSpacerItem@@6B@      1002bf80     ORFDialog.obj
 0002:00005f94       ??_R3QSpacerItem@@8        1002bf94     ORFDialog.obj
 0002:00005fa4       ??_R2QSpacerItem@@8        1002bfa4     ORFDialog.obj
 0002:00005fb0       ??_R1A@?0A@EA@QSpacerItem@@8 1002bfb0     ORFDialog.obj
 0002:00005fcc       ??_R1A@?0A@EA@QLayoutItem@@8 1002bfcc     ORFDialog.obj
 0002:00005fe8       ??_R3QLayoutItem@@8        1002bfe8     ORFDialog.obj
 0002:00005ff8       ??_R2QLayoutItem@@8        1002bff8     ORFDialog.obj
 0002:00006000       ??_R4QHBoxLayout@@6BQObject@@@ 1002c000     ORFDialog.obj
 0002:00006014       ??_R3QHBoxLayout@@8        1002c014     ORFDialog.obj
 0002:00006024       ??_R2QHBoxLayout@@8        1002c024     ORFDialog.obj
 0002:0000603c       ??_R1A@?0A@EA@QHBoxLayout@@8 1002c03c     ORFDialog.obj
 0002:00006058       ??_R1A@?0A@EA@QBoxLayout@@8 1002c058     ORFDialog.obj
 0002:00006074       ??_R3QBoxLayout@@8         1002c074     ORFDialog.obj
 0002:00006084       ??_R2QBoxLayout@@8         1002c084     ORFDialog.obj
 0002:00006098       ??_R1A@?0A@EA@QLayout@@8   1002c098     ORFDialog.obj
 0002:000060b4       ??_R3QLayout@@8            1002c0b4     ORFDialog.obj
 0002:000060c4       ??_R2QLayout@@8            1002c0c4     ORFDialog.obj
 0002:000060d4       ??_R17?0A@EA@QLayoutItem@@8 1002c0d4     ORFDialog.obj
 0002:000060f0       ??_R4QHBoxLayout@@6BQLayoutItem@@@ 1002c0f0     ORFDialog.obj
 0002:00006104       ??_R4QVBoxLayout@@6BQObject@@@ 1002c104     ORFDialog.obj
 0002:00006118       ??_R3QVBoxLayout@@8        1002c118     ORFDialog.obj
 0002:00006128       ??_R2QVBoxLayout@@8        1002c128     ORFDialog.obj
 0002:00006140       ??_R1A@?0A@EA@QVBoxLayout@@8 1002c140     ORFDialog.obj
 0002:0000615c       ??_R4QVBoxLayout@@6BQLayoutItem@@@ 1002c15c     ORFDialog.obj
 0002:00006170       ??_R4QGridLayout@@6BQObject@@@ 1002c170     ORFDialog.obj
 0002:00006184       ??_R3QGridLayout@@8        1002c184     ORFDialog.obj
 0002:00006194       ??_R2QGridLayout@@8        1002c194     ORFDialog.obj
 0002:000061a8       ??_R1A@?0A@EA@QGridLayout@@8 1002c1a8     ORFDialog.obj
 0002:000061c4       ??_R4QGridLayout@@6BQLayoutItem@@@ 1002c1c4     ORFDialog.obj
 0002:000061d8       ??_R4QGroupBox@@6BQObject@@@ 1002c1d8     ORFDialog.obj
 0002:000061ec       ??_R3QGroupBox@@8          1002c1ec     ORFDialog.obj
 0002:000061fc       ??_R2QGroupBox@@8          1002c1fc     ORFDialog.obj
 0002:00006210       ??_R1A@?0A@EA@QGroupBox@@8 1002c210     ORFDialog.obj
 0002:0000622c       ??_R4QGroupBox@@6BQPaintDevice@@@ 1002c22c     ORFDialog.obj
 0002:00006240       ??_R4QLabel@@6BQObject@@@  1002c240     ORFDialog.obj
 0002:00006254       ??_R3QLabel@@8             1002c254     ORFDialog.obj
 0002:00006264       ??_R2QLabel@@8             1002c264     ORFDialog.obj
 0002:0000627c       ??_R1A@?0A@EA@QLabel@@8    1002c27c     ORFDialog.obj
 0002:00006298       ??_R1A@?0A@EA@QFrame@@8    1002c298     ORFDialog.obj
 0002:000062b4       ??_R3QFrame@@8             1002c2b4     ORFDialog.obj
 0002:000062c4       ??_R2QFrame@@8             1002c2c4     ORFDialog.obj
 0002:000062d8       ??_R4QLabel@@6BQPaintDevice@@@ 1002c2d8     ORFDialog.obj
 0002:000062ec       ??_R4QRadioButton@@6BQObject@@@ 1002c2ec     ORFDialog.obj
 0002:00006300       ??_R3QRadioButton@@8       1002c300     ORFDialog.obj
 0002:00006310       ??_R2QRadioButton@@8       1002c310     ORFDialog.obj
 0002:00006328       ??_R1A@?0A@EA@QRadioButton@@8 1002c328     ORFDialog.obj
 0002:00006344       ??_R4QRadioButton@@6BQPaintDevice@@@ 1002c344     ORFDialog.obj
 0002:00006358       ??_R4QSpinBox@@6BQObject@@@ 1002c358     ORFDialog.obj
 0002:0000636c       ??_R3QSpinBox@@8           1002c36c     ORFDialog.obj
 0002:0000637c       ??_R2QSpinBox@@8           1002c37c     ORFDialog.obj
 0002:00006394       ??_R1A@?0A@EA@QSpinBox@@8  1002c394     ORFDialog.obj
 0002:000063b0       ??_R1A@?0A@EA@QAbstractSpinBox@@8 1002c3b0     ORFDialog.obj
 0002:000063cc       ??_R3QAbstractSpinBox@@8   1002c3cc     ORFDialog.obj
 0002:000063dc       ??_R2QAbstractSpinBox@@8   1002c3dc     ORFDialog.obj
 0002:000063f0       ??_R4QSpinBox@@6BQPaintDevice@@@ 1002c3f0     ORFDialog.obj
 0002:00006404       ??_R4QTextEdit@@6BQObject@@@ 1002c404     ORFDialog.obj
 0002:00006418       ??_R3QTextEdit@@8          1002c418     ORFDialog.obj
 0002:00006428       ??_R2QTextEdit@@8          1002c428     ORFDialog.obj
 0002:00006444       ??_R1A@?0A@EA@QTextEdit@@8 1002c444     ORFDialog.obj
 0002:00006460       ??_R1A@?0A@EA@QAbstractScrollArea@@8 1002c460     ORFDialog.obj
 0002:0000647c       ??_R3QAbstractScrollArea@@8 1002c47c     ORFDialog.obj
 0002:0000648c       ??_R2QAbstractScrollArea@@8 1002c48c     ORFDialog.obj
 0002:000064a4       ??_R4QTextEdit@@6BQPaintDevice@@@ 1002c4a4     ORFDialog.obj
 0002:000064b8       ??_R4QTreeWidget@@6BQObject@@@ 1002c4b8     ORFDialog.obj
 0002:000064cc       ??_R3QTreeWidget@@8        1002c4cc     ORFDialog.obj
 0002:000064dc       ??_R2QTreeWidget@@8        1002c4dc     ORFDialog.obj
 0002:00006500       ??_R1A@?0A@EA@QTreeWidget@@8 1002c500     ORFDialog.obj
 0002:0000651c       ??_R1A@?0A@EA@QTreeView@@8 1002c51c     ORFDialog.obj
 0002:00006538       ??_R3QTreeView@@8          1002c538     ORFDialog.obj
 0002:00006548       ??_R2QTreeView@@8          1002c548     ORFDialog.obj
 0002:00006568       ??_R1A@?0A@EA@QAbstractItemView@@8 1002c568     ORFDialog.obj
 0002:00006584       ??_R3QAbstractItemView@@8  1002c584     ORFDialog.obj
 0002:00006594       ??_R2QAbstractItemView@@8  1002c594     ORFDialog.obj
 0002:000065b0       ??_R4QTreeWidget@@6BQPaintDevice@@@ 1002c5b0     ORFDialog.obj
 0002:000065c4       ??_R4AbstractInt32Id@U2@@6B@ 1002c5c4     ORFDialog.obj
 0002:000065d8       ??_R3AbstractInt32Id@U2@@8 1002c5d8     ORFDialog.obj
 0002:000065e8       ??_R2AbstractInt32Id@U2@@8 1002c5e8     ORFDialog.obj
 0002:000065f4       ??_R1A@?0A@EA@AbstractInt32Id@U2@@8 1002c5f4     ORFDialog.obj
 0002:00006610       ??_R1A@?0A@EA@?$AbstractId@H@U2@@8 1002c610     ORFDialog.obj
 0002:0000662c       ??_R3?$AbstractId@H@U2@@8  1002c62c     ORFDialog.obj
 0002:0000663c       ??_R2?$AbstractId@H@U2@@8  1002c63c     ORFDialog.obj
 0002:00006644       ??_R4?$AbstractId@H@U2@@6B@ 1002c644     ORFDialog.obj
 0002:00006658       ??_R4ServiceType@U2@@6B@   1002c658     ORFDialog.obj
 0002:0000666c       ??_R3ServiceType@U2@@8     1002c66c     ORFDialog.obj
 0002:0000667c       ??_R2ServiceType@U2@@8     1002c67c     ORFDialog.obj
 0002:0000668c       ??_R1A@?0A@EA@ServiceType@U2@@8 1002c68c     ORFDialog.obj
 0002:000066a8       ??_R4RegionSelector@U2@@6BQObject@@@ 1002c6a8     ORFDialog.obj
 0002:000066bc       ??_R3RegionSelector@U2@@8  1002c6bc     ORFDialog.obj
 0002:000066cc       ??_R2RegionSelector@U2@@8  1002c6cc     ORFDialog.obj
 0002:000066e0       ??_R1A@?0A@EA@RegionSelector@U2@@8 1002c6e0     ORFDialog.obj
 0002:000066fc       ??_R4RegionSelector@U2@@6BQPaintDevice@@@ 1002c6fc     ORFDialog.obj
 0002:00006710       ??_R4ORFFindTask@U2@@6BTask@1@@ 1002c710     ORFDialog.obj
 0002:00006724       ??_R3ORFFindTask@U2@@8     1002c724     ORFDialog.obj
 0002:00006734       ??_R2ORFFindTask@U2@@8     1002c734     ORFDialog.obj
 0002:00006748       ??_R1A@?0A@EA@ORFFindTask@U2@@8 1002c748     ORFDialog.obj
 0002:00006764       ??_R1A@?0A@EA@Task@U2@@8   1002c764     ORFDialog.obj
 0002:00006780       ??_R3Task@U2@@8            1002c780     ORFDialog.obj
 0002:00006790       ??_R2Task@U2@@8            1002c790     ORFDialog.obj
 0002:0000679c       ??_R1JA@?0A@EA@ORFFindResultsListener@U2@@8 1002c79c     ORFDialog.obj
 0002:000067b8       ??_R3ORFFindResultsListener@U2@@8 1002c7b8     ORFDialog.obj
 0002:000067c8       ??_R2ORFFindResultsListener@U2@@8 1002c7c8     ORFDialog.obj
 0002:000067d0       ??_R1A@?0A@EA@ORFFindResultsListener@U2@@8 1002c7d0     ORFDialog.obj
 0002:000067ec       ??_R4ORFFindTask@U2@@6BORFFindResultsListener@1@@ 1002c7ec     ORFDialog.obj
 0002:00006800       ??_R4CreateAnnotationWidgetController@U2@@6B@ 1002c800     ORFDialog.obj
 0002:00006814       ??_R3CreateAnnotationWidgetController@U2@@8 1002c814     ORFDialog.obj
 0002:00006824       ??_R2CreateAnnotationWidgetController@U2@@8 1002c824     ORFDialog.obj
 0002:00006830       ??_R1A@?0A@EA@CreateAnnotationWidgetController@U2@@8 1002c830     ORFDialog.obj
 0002:0000684c       ??_R4ORFDialog@U2@@6BQObject@@@ 1002c84c     ORFDialog.obj
 0002:00006860       ??_R3ORFDialog@U2@@8       1002c860     ORFDialog.obj
 0002:00006870       ??_R2ORFDialog@U2@@8       1002c870     ORFDialog.obj
 0002:0000688c       ??_R1A@?0A@EA@ORFDialog@U2@@8 1002c88c     ORFDialog.obj
 0002:000068a8       ??_R1A@?0A@EA@QDialog@@8   1002c8a8     ORFDialog.obj
 0002:000068c4       ??_R3QDialog@@8            1002c8c4     ORFDialog.obj
 0002:000068d4       ??_R2QDialog@@8            1002c8d4     ORFDialog.obj
 0002:000068e8       ??_R1BI@?0A@EA@Ui_ORFDialogBase@@8 1002c8e8     ORFDialog.obj
 0002:00006904       ??_R3Ui_ORFDialogBase@@8   1002c904     ORFDialog.obj
 0002:00006914       ??_R2Ui_ORFDialogBase@@8   1002c914     ORFDialog.obj
 0002:0000691c       ??_R1A@?0A@EA@Ui_ORFDialogBase@@8 1002c91c     ORFDialog.obj
 0002:00006938       ??_R4ORFDialog@U2@@6BQPaintDevice@@@ 1002c938     ORFDialog.obj
 0002:0000694c       ??_R4HelpButton@U2@@6B@    1002c94c     ORFDialog.obj
 0002:00006960       ??_R3HelpButton@U2@@8      1002c960     ORFDialog.obj
 0002:00006970       ??_R2HelpButton@U2@@8      1002c970     ORFDialog.obj
 0002:0000697c       ??_R1A@?0A@EA@HelpButton@U2@@8 1002c97c     ORFDialog.obj
 0002:00006998       ??_R4ORFListItem@U2@@6B@   1002c998     ORFDialog.obj
 0002:000069ac       ??_R3ORFListItem@U2@@8     1002c9ac     ORFDialog.obj
 0002:000069bc       ??_R2ORFListItem@U2@@8     1002c9bc     ORFDialog.obj
 0002:000069c8       ??_R1A@?0A@EA@ORFListItem@U2@@8 1002c9c8     ORFDialog.obj
 0002:000069e4       ??_R1A@?0A@EA@QTreeWidgetItem@@8 1002c9e4     ORFDialog.obj
 0002:00006a00       ??_R3QTreeWidgetItem@@8    1002ca00     ORFDialog.obj
 0002:00006a10       ??_R2QTreeWidgetItem@@8    1002ca10     ORFDialog.obj
 0002:00006a18       ??_R4ADVGlobalAction@U2@@6B@ 1002ca18     ORFMarkerPlugin.obj
 0002:00006a2c       ??_R3ADVGlobalAction@U2@@8 1002ca2c     ORFMarkerPlugin.obj
 0002:00006a3c       ??_R2ADVGlobalAction@U2@@8 1002ca3c     ORFMarkerPlugin.obj
 0002:00006a50       ??_R1A@?0A@EA@ADVGlobalAction@U2@@8 1002ca50     ORFMarkerPlugin.obj
 0002:00006a6c       ??_R1A@?0A@EA@GObjectViewAction@U2@@8 1002ca6c     ORFMarkerPlugin.obj
 0002:00006a88       ??_R3GObjectViewAction@U2@@8 1002ca88     ORFMarkerPlugin.obj
 0002:00006a98       ??_R2GObjectViewAction@U2@@8 1002ca98     ORFMarkerPlugin.obj
 0002:00006aa8       ??_R1A@?0A@EA@QAction@@8   1002caa8     ORFMarkerPlugin.obj
 0002:00006ac4       ??_R3QAction@@8            1002cac4     ORFMarkerPlugin.obj
 0002:00006ad4       ??_R2QAction@@8            1002cad4     ORFMarkerPlugin.obj
 0002:00006ae0       ??_R4ORFMarkerPlugin@U2@@6B@ 1002cae0     ORFMarkerPlugin.obj
 0002:00006af4       ??_R3ORFMarkerPlugin@U2@@8 1002caf4     ORFMarkerPlugin.obj
 0002:00006b04       ??_R2ORFMarkerPlugin@U2@@8 1002cb04     ORFMarkerPlugin.obj
 0002:00006b14       ??_R1A@?0A@EA@ORFMarkerPlugin@U2@@8 1002cb14     ORFMarkerPlugin.obj
 0002:00006b30       ??_R1A@?0A@EA@Plugin@U2@@8 1002cb30     ORFMarkerPlugin.obj
 0002:00006b4c       ??_R3Plugin@U2@@8          1002cb4c     ORFMarkerPlugin.obj
 0002:00006b5c       ??_R2Plugin@U2@@8          1002cb5c     ORFMarkerPlugin.obj
 0002:00006b68       ??_R4ORFViewContext@U2@@6BQObject@@@ 1002cb68     ORFMarkerPlugin.obj
 0002:00006b7c       ??_R3ORFViewContext@U2@@8  1002cb7c     ORFMarkerPlugin.obj
 0002:00006b8c       ??_R2ORFViewContext@U2@@8  1002cb8c     ORFMarkerPlugin.obj
 0002:00006ba0       ??_R1A@?0A@EA@ORFViewContext@U2@@8 1002cba0     ORFMarkerPlugin.obj
 0002:00006bbc       ??_R1A@?0A@EA@GObjectViewWindowContext@U2@@8 1002cbbc     ORFMarkerPlugin.obj
 0002:00006bd8       ??_R3GObjectViewWindowContext@U2@@8 1002cbd8     ORFMarkerPlugin.obj
 0002:00006be8       ??_R2GObjectViewWindowContext@U2@@8 1002cbe8     ORFMarkerPlugin.obj
 0002:00006bf8       ??_R17?0A@EA@GObjectViewObjectHandler@U2@@8 1002cbf8     ORFMarkerPlugin.obj
 0002:00006c14       ??_R3GObjectViewObjectHandler@U2@@8 1002cc14     ORFMarkerPlugin.obj
 0002:00006c24       ??_R2GObjectViewObjectHandler@U2@@8 1002cc24     ORFMarkerPlugin.obj
 0002:00006c2c       ??_R1A@?0A@EA@GObjectViewObjectHandler@U2@@8 1002cc2c     ORFMarkerPlugin.obj
 0002:00006c48       ??_R4ORFViewContext@U2@@6BGObjectViewObjectHandler@1@@ 1002cc48     ORFMarkerPlugin.obj
 0002:00006c5c       ??_R1A@?0A@EA@XmlTest@U2@@8 1002cc5c     ORFMarkerPlugin.obj
 0002:00006c78       ??_R3XmlTest@U2@@8         1002cc78     ORFMarkerPlugin.obj
 0002:00006c88       ??_R2XmlTest@U2@@8         1002cc88     ORFMarkerPlugin.obj
 0002:00006c9c       ??_R1A@?0A@EA@GTest@U2@@8  1002cc9c     ORFMarkerPlugin.obj
 0002:00006cb8       ??_R3GTest@U2@@8           1002ccb8     ORFMarkerPlugin.obj
 0002:00006cc8       ??_R2GTest@U2@@8           1002ccc8     ORFMarkerPlugin.obj
 0002:00006cd8       ??_R1A@?0A@EA@XMLTestFactory@U2@@8 1002ccd8     ORFMarkerPlugin.obj
 0002:00006cf4       ??_R3XMLTestFactory@U2@@8  1002ccf4     ORFMarkerPlugin.obj
 0002:00006d04       ??_R2XMLTestFactory@U2@@8  1002cd04     ORFMarkerPlugin.obj
 0002:00006d0c       ??_R4GTest_ORFMarkerTask@U2@@6B@ 1002cd0c     ORFMarkerPlugin.obj
 0002:00006d20       ??_R3GTest_ORFMarkerTask@U2@@8 1002cd20     ORFMarkerPlugin.obj
 0002:00006d30       ??_R2GTest_ORFMarkerTask@U2@@8 1002cd30     ORFMarkerPlugin.obj
 0002:00006d48       ??_R1A@?0A@EA@GTest_ORFMarkerTask@U2@@8 1002cd48     ORFMarkerPlugin.obj
 0002:00006d64       ??_R4GTest_ORFMarkerTaskFactory@GTest_ORFMarkerTask@U2@@6B@ 1002cd64     ORFMarkerPlugin.obj
 0002:00006d78       ??_R3GTest_ORFMarkerTaskFactory@GTest_ORFMarkerTask@U2@@8 1002cd78     ORFMarkerPlugin.obj
 0002:00006d88       ??_R2GTest_ORFMarkerTaskFactory@GTest_ORFMarkerTask@U2@@8 1002cd88     ORFMarkerPlugin.obj
 0002:00006d94       ??_R1A@?0A@EA@GTest_ORFMarkerTaskFactory@GTest_ORFMarkerTask@U2@@8 1002cd94     ORFMarkerPlugin.obj
 0002:00006db0       ??_R4?$GAutoDeleteList@VXMLTestFactory@U2@@@U2@@6B@ 1002cdb0     ORFMarkerPlugin.obj
 0002:00006dc4       ??_R3?$GAutoDeleteList@VXMLTestFactory@U2@@@U2@@8 1002cdc4     ORFMarkerPlugin.obj
 0002:00006dd4       ??_R2?$GAutoDeleteList@VXMLTestFactory@U2@@@U2@@8 1002cdd4     ORFMarkerPlugin.obj
 0002:00006de0       ??_R1A@?0A@EA@?$GAutoDeleteList@VXMLTestFactory@U2@@@U2@@8 1002cde0     ORFMarkerPlugin.obj
 0002:00006dfc       ??_R4CreateAnnotationsTask@U2@@6B@ 1002cdfc     ORFMarkerTask.obj
 0002:00006e10       ??_R3CreateAnnotationsTask@U2@@8 1002ce10     ORFMarkerTask.obj
 0002:00006e20       ??_R2CreateAnnotationsTask@U2@@8 1002ce20     ORFMarkerTask.obj
 0002:00006e30       ??_R1A@?0A@EA@CreateAnnotationsTask@U2@@8 1002ce30     ORFMarkerTask.obj
 0002:00006e4c       ??_R4FindORFsToAnnotationsTask@U2@@6B@ 1002ce4c     ORFMarkerTask.obj
 0002:00006e60       ??_R3FindORFsToAnnotationsTask@U2@@8 1002ce60     ORFMarkerTask.obj
 0002:00006e70       ??_R2FindORFsToAnnotationsTask@U2@@8 1002ce70     ORFMarkerTask.obj
 0002:00006e80       ??_R1A@?0A@EA@FindORFsToAnnotationsTask@U2@@8 1002ce80     ORFMarkerTask.obj
 0002:00006e9c       ??_R4ORFAutoAnnotationsUpdater@U2@@6B@ 1002ce9c     ORFMarkerTask.obj
 0002:00006eb0       ??_R3ORFAutoAnnotationsUpdater@U2@@8 1002ceb0     ORFMarkerTask.obj
 0002:00006ec0       ??_R2ORFAutoAnnotationsUpdater@U2@@8 1002cec0     ORFMarkerTask.obj
 0002:00006ed0       ??_R1A@?0A@EA@ORFAutoAnnotationsUpdater@U2@@8 1002ced0     ORFMarkerTask.obj
 0002:00006eec       ??_R1A@?0A@EA@AutoAnnotationsUpdater@U2@@8 1002ceec     ORFMarkerTask.obj
 0002:00006f08       ??_R3AutoAnnotationsUpdater@U2@@8 1002cf08     ORFMarkerTask.obj
 0002:00006f18       ??_R2AutoAnnotationsUpdater@U2@@8 1002cf18     ORFMarkerTask.obj
 0002:00006f24       ??_R4Task@U2@@6B@          1002cf24     ORFQuery.obj
 0002:00006f38       ??_R3Descriptor@U2@@8      1002cf38     ORFQuery.obj
 0002:00006f48       ??_R2Descriptor@U2@@8      1002cf48     ORFQuery.obj
 0002:00006f50       ??_R1A@?0A@EA@Descriptor@U2@@8 1002cf50     ORFQuery.obj
 0002:00006f6c       ??_R4Attribute@U2@@6B@     1002cf6c     ORFQuery.obj
 0002:00006f80       ??_R3Attribute@U2@@8       1002cf80     ORFQuery.obj
 0002:00006f90       ??_R2Attribute@U2@@8       1002cf90     ORFQuery.obj
 0002:00006f9c       ??_R1A@?0A@EA@Attribute@U2@@8 1002cf9c     ORFQuery.obj
 0002:00006fb8       ??_R3ConfigurationEditor@U2@@8 1002cfb8     ORFQuery.obj
 0002:00006fc8       ??_R2ConfigurationEditor@U2@@8 1002cfc8     ORFQuery.obj
 0002:00006fd4       ??_R1A@?0A@EA@ConfigurationEditor@U2@@8 1002cfd4     ORFQuery.obj
 0002:00006ff0       ??_R4QDORFActor@U2@@6B@    1002cff0     ORFQuery.obj
 0002:00007004       ??_R3QDORFActor@U2@@8      1002d004     ORFQuery.obj
 0002:00007014       ??_R2QDORFActor@U2@@8      1002d014     ORFQuery.obj
 0002:00007024       ??_R1A@?0A@EA@QDORFActor@U2@@8 1002d024     ORFQuery.obj
 0002:00007040       ??_R1A@?0A@EA@QDActor@U2@@8 1002d040     ORFQuery.obj
 0002:0000705c       ??_R3QDActor@U2@@8         1002d05c     ORFQuery.obj
 0002:0000706c       ??_R2QDActor@U2@@8         1002d06c     ORFQuery.obj
 0002:00007078       ??_R4QDORFActorPrototype@U2@@6B@ 1002d078     ORFQuery.obj
 0002:0000708c       ??_R3QDORFActorPrototype@U2@@8 1002d08c     ORFQuery.obj
 0002:0000709c       ??_R2QDORFActorPrototype@U2@@8 1002d09c     ORFQuery.obj
 0002:000070a8       ??_R1A@?0A@EA@QDORFActorPrototype@U2@@8 1002d0a8     ORFQuery.obj
 0002:000070c4       ??_R1A@?0A@EA@QDActorPrototype@U2@@8 1002d0c4     ORFQuery.obj
 0002:000070e0       ??_R3QDActorPrototype@U2@@8 1002d0e0     ORFQuery.obj
 0002:000070f0       ??_R2QDActorPrototype@U2@@8 1002d0f0     ORFQuery.obj
 0002:000070f8       ??_R4DelegateEditor@U2@@6B@ 1002d0f8     ORFQuery.obj
 0002:0000710c       ??_R3DelegateEditor@U2@@8  1002d10c     ORFQuery.obj
 0002:0000711c       ??_R2DelegateEditor@U2@@8  1002d11c     ORFQuery.obj
 0002:0000712c       ??_R1A@?0A@EA@DelegateEditor@U2@@8 1002d12c     ORFQuery.obj
 0002:00007148       ??_R4SpinBoxDelegate@U2@@6B@ 1002d148     ORFQuery.obj
 0002:0000715c       ??_R3SpinBoxDelegate@U2@@8 1002d15c     ORFQuery.obj
 0002:0000716c       ??_R2SpinBoxDelegate@U2@@8 1002d16c     ORFQuery.obj
 0002:00007184       ??_R1A@?0A@EA@SpinBoxDelegate@U2@@8 1002d184     ORFQuery.obj
 0002:000071a0       ??_R1A@?0A@EA@PropertyDelegate@U2@@8 1002d1a0     ORFQuery.obj
 0002:000071bc       ??_R3PropertyDelegate@U2@@8 1002d1bc     ORFQuery.obj
 0002:000071cc       ??_R2PropertyDelegate@U2@@8 1002d1cc     ORFQuery.obj
 0002:000071e0       ??_R1A@?0A@EA@QItemDelegate@@8 1002d1e0     ORFQuery.obj
 0002:000071fc       ??_R3QItemDelegate@@8      1002d1fc     ORFQuery.obj
 0002:0000720c       ??_R2QItemDelegate@@8      1002d20c     ORFQuery.obj
 0002:0000721c       ??_R1A@?0A@EA@QAbstractItemDelegate@@8 1002d21c     ORFQuery.obj
 0002:00007238       ??_R3QAbstractItemDelegate@@8 1002d238     ORFQuery.obj
 0002:00007248       ??_R2QAbstractItemDelegate@@8 1002d248     ORFQuery.obj
 0002:00007254       ??_R4ComboBoxDelegate@U2@@6B@ 1002d254     ORFQuery.obj
 0002:00007268       ??_R3ComboBoxDelegate@U2@@8 1002d268     ORFQuery.obj
 0002:00007278       ??_R2ComboBoxDelegate@U2@@8 1002d278     ORFQuery.obj
 0002:00007290       ??_R1A@?0A@EA@ComboBoxDelegate@U2@@8 1002d290     ORFQuery.obj
 0002:000072ac       ??_R4TaskSignalMapper@U2@@6B@ 1002d2ac     ORFQuery.obj
 0002:000072c0       ??_R3TaskSignalMapper@U2@@8 1002d2c0     ORFQuery.obj
 0002:000072d0       ??_R2TaskSignalMapper@U2@@8 1002d2d0     ORFQuery.obj
 0002:000072dc       ??_R1A@?0A@EA@TaskSignalMapper@U2@@8 1002d2dc     ORFQuery.obj
 0002:000072f8       ??_R4FailTask@U2@@6B@      1002d2f8     ORFQuery.obj
 0002:0000730c       ??_R3FailTask@U2@@8        1002d30c     ORFQuery.obj
 0002:0000731c       ??_R2FailTask@U2@@8        1002d31c     ORFQuery.obj
 0002:0000732c       ??_R1A@?0A@EA@FailTask@U2@@8 1002d32c     ORFQuery.obj
 0002:00007348       ??_R4Descriptor@U2@@6B@    1002d348     ORFWorker.obj
 0002:0000735c       ??_R4MapDataType@U2@@6B@   1002d35c     ORFWorker.obj
 0002:00007370       ??_R3MapDataType@U2@@8     1002d370     ORFWorker.obj
 0002:00007380       ??_R2MapDataType@U2@@8     1002d380     ORFWorker.obj
 0002:00007394       ??_R1A@?0A@EA@MapDataType@U2@@8 1002d394     ORFWorker.obj
 0002:000073b0       ??_R1A@?0A@EA@DataType@U2@@8 1002d3b0     ORFWorker.obj
 0002:000073cc       ??_R3DataType@U2@@8        1002d3cc     ORFWorker.obj
 0002:000073dc       ??_R2DataType@U2@@8        1002d3dc     ORFWorker.obj
 0002:000073ec       ??_R1BA@?0A@EA@QSharedData@@8 1002d3ec     ORFWorker.obj
 0002:00007408       ??_R3QSharedData@@8        1002d408     ORFWorker.obj
 0002:00007418       ??_R2QSharedData@@8        1002d418     ORFWorker.obj
 0002:00007420       ??_R1A@?0A@EA@QSharedData@@8 1002d420     ORFWorker.obj
 0002:0000743c       ??_R4PortDescriptor@Workflow@U2@@6B@ 1002d43c     ORFWorker.obj
 0002:00007450       ??_R3PortDescriptor@Workflow@U2@@8 1002d450     ORFWorker.obj
 0002:00007460       ??_R2PortDescriptor@Workflow@U2@@8 1002d460     ORFWorker.obj
 0002:0000746c       ??_R1A@?0A@EA@PortDescriptor@Workflow@U2@@8 1002d46c     ORFWorker.obj
 0002:00007488       ??_R17?0A@EA@Descriptor@U2@@8 1002d488     ORFWorker.obj
 0002:000074a4       ??_R4IntegralBusActorPrototype@Workflow@U2@@6B@ 1002d4a4     ORFWorker.obj
 0002:000074b8       ??_R3IntegralBusActorPrototype@Workflow@U2@@8 1002d4b8     ORFWorker.obj
 0002:000074c8       ??_R2IntegralBusActorPrototype@Workflow@U2@@8 1002d4c8     ORFWorker.obj
 0002:000074dc       ??_R1A@?0A@EA@IntegralBusActorPrototype@Workflow@U2@@8 1002d4dc     ORFWorker.obj
 0002:000074f8       ??_R1A@?0A@EA@ActorPrototype@Workflow@U2@@8 1002d4f8     ORFWorker.obj
 0002:00007514       ??_R3ActorPrototype@Workflow@U2@@8 1002d514     ORFWorker.obj
 0002:00007524       ??_R2ActorPrototype@Workflow@U2@@8 1002d524     ORFWorker.obj
 0002:00007534       ??_R1A@?0A@EA@VisualDescriptor@U2@@8 1002d534     ORFWorker.obj
 0002:00007550       ??_R3VisualDescriptor@U2@@8 1002d550     ORFWorker.obj
 0002:00007560       ??_R2VisualDescriptor@U2@@8 1002d560     ORFWorker.obj
 0002:0000756c       ??_R4ORFPrompter@LocalWorkflow@U2@@6BActorDocument@Workflow@2@@ 1002d56c     ORFWorker.obj
 0002:00007580       ??_R3ORFPrompter@LocalWorkflow@U2@@8 1002d580     ORFWorker.obj
 0002:00007590       ??_R2ORFPrompter@LocalWorkflow@U2@@8 1002d590     ORFWorker.obj
 0002:000075b0       ??_R1A@?0A@EA@ORFPrompter@LocalWorkflow@U2@@8 1002d5b0     ORFWorker.obj
 0002:000075cc       ??_R1A@?0A@EA@?$PrompterBase@VORFPrompter@LocalWorkflow@U2@@@U2@@8 1002d5cc     ORFWorker.obj
 0002:000075e8       ??_R3?$PrompterBase@VORFPrompter@LocalWorkflow@U2@@@U2@@8 1002d5e8     ORFWorker.obj
 0002:000075f8       ??_R2?$PrompterBase@VORFPrompter@LocalWorkflow@U2@@@U2@@8 1002d5f8     ORFWorker.obj
 0002:00007614       ??_R1A@?0A@EA@PrompterBaseImpl@U2@@8 1002d614     ORFWorker.obj
 0002:00007630       ??_R3PrompterBaseImpl@U2@@8 1002d630     ORFWorker.obj
 0002:00007640       ??_R2PrompterBaseImpl@U2@@8 1002d640     ORFWorker.obj
 0002:00007658       ??_R1A@?0A@EA@ActorDocument@Workflow@U2@@8 1002d658     ORFWorker.obj
 0002:00007674       ??_R3ActorDocument@Workflow@U2@@8 1002d674     ORFWorker.obj
 0002:00007684       ??_R2ActorDocument@Workflow@U2@@8 1002d684     ORFWorker.obj
 0002:00007694       ??_R1A@?0A@EA@QTextDocument@@8 1002d694     ORFWorker.obj
 0002:000076b0       ??_R3QTextDocument@@8      1002d6b0     ORFWorker.obj
 0002:000076c0       ??_R2QTextDocument@@8      1002d6c0     ORFWorker.obj
 0002:000076cc       ??_R1M@?0A@EA@Prompter@Workflow@U2@@8 1002d6cc     ORFWorker.obj
 0002:000076e8       ??_R3Prompter@Workflow@U2@@8 1002d6e8     ORFWorker.obj
 0002:000076f8       ??_R2Prompter@Workflow@U2@@8 1002d6f8     ORFWorker.obj
 0002:00007700       ??_R1A@?0A@EA@Prompter@Workflow@U2@@8 1002d700     ORFWorker.obj
 0002:0000771c       ??_R4ORFPrompter@LocalWorkflow@U2@@6BPrompter@Workflow@2@@ 1002d71c     ORFWorker.obj
 0002:00007730       ??_R4?$PrompterBase@VORFPrompter@LocalWorkflow@U2@@@U2@@6BActorDocument@Workflow@1@@ 1002d730     ORFWorker.obj
 0002:00007744       ??_R4?$PrompterBase@VORFPrompter@LocalWorkflow@U2@@@U2@@6BPrompter@Workflow@1@@ 1002d744     ORFWorker.obj
 0002:00007758       ??_R4ORFWorker@LocalWorkflow@U2@@6BQObject@@@ 1002d758     ORFWorker.obj
 0002:0000776c       ??_R3ORFWorker@LocalWorkflow@U2@@8 1002d76c     ORFWorker.obj
 0002:0000777c       ??_R2ORFWorker@LocalWorkflow@U2@@8 1002d77c     ORFWorker.obj
 0002:00007794       ??_R1A@?0A@EA@ORFWorker@LocalWorkflow@U2@@8 1002d794     ORFWorker.obj
 0002:000077b0       ??_R1A@?0A@EA@BaseWorker@LocalWorkflow@U2@@8 1002d7b0     ORFWorker.obj
 0002:000077cc       ??_R3BaseWorker@LocalWorkflow@U2@@8 1002d7cc     ORFWorker.obj
 0002:000077dc       ??_R2BaseWorker@LocalWorkflow@U2@@8 1002d7dc     ORFWorker.obj
 0002:000077f0       ??_R17?0A@EA@Worker@Workflow@U2@@8 1002d7f0     ORFWorker.obj
 0002:0000780c       ??_R3Worker@Workflow@U2@@8 1002d80c     ORFWorker.obj
 0002:0000781c       ??_R2Worker@Workflow@U2@@8 1002d81c     ORFWorker.obj
 0002:00007824       ??_R1A@?0A@EA@Worker@Workflow@U2@@8 1002d824     ORFWorker.obj
 0002:00007840       ??_R1BA@?0A@EA@CommunicationSubject@Workflow@U2@@8 1002d840     ORFWorker.obj
 0002:0000785c       ??_R3CommunicationSubject@Workflow@U2@@8 1002d85c     ORFWorker.obj
 0002:0000786c       ??_R2CommunicationSubject@Workflow@U2@@8 1002d86c     ORFWorker.obj
 0002:00007874       ??_R1A@?0A@EA@CommunicationSubject@Workflow@U2@@8 1002d874     ORFWorker.obj
 0002:00007890       ??_R4ORFWorker@LocalWorkflow@U2@@6BWorker@Workflow@2@@ 1002d890     ORFWorker.obj
 0002:000078a4       ??_R4ORFWorker@LocalWorkflow@U2@@6BCommunicationSubject@Workflow@2@@ 1002d8a4     ORFWorker.obj
 0002:000078b8       ??_R4ORFWorkerFactory@LocalWorkflow@U2@@6B?$IdRegistry@VDomainFactory@Workflow@U2@@@2@@ 1002d8b8     ORFWorker.obj
 0002:000078cc       ??_R3ORFWorkerFactory@LocalWorkflow@U2@@8 1002d8cc     ORFWorker.obj
 0002:000078dc       ??_R2ORFWorkerFactory@LocalWorkflow@U2@@8 1002d8dc     ORFWorker.obj
 0002:000078f0       ??_R1A@?0A@EA@ORFWorkerFactory@LocalWorkflow@U2@@8 1002d8f0     ORFWorker.obj
 0002:0000790c       ??_R1A@?0A@EA@DomainFactory@Workflow@U2@@8 1002d90c     ORFWorker.obj
 0002:00007928       ??_R3DomainFactory@Workflow@U2@@8 1002d928     ORFWorker.obj
 0002:00007938       ??_R2DomainFactory@Workflow@U2@@8 1002d938     ORFWorker.obj
 0002:00007948       ??_R1A@?0A@EA@?$IdRegistry@VDomainFactory@Workflow@U2@@@U2@@8 1002d948     ORFWorker.obj
 0002:00007964       ??_R3?$IdRegistry@VDomainFactory@Workflow@U2@@@U2@@8 1002d964     ORFWorker.obj
 0002:00007974       ??_R2?$IdRegistry@VDomainFactory@Workflow@U2@@@U2@@8 1002d974     ORFWorker.obj
 0002:0000797c       ??_R4ORFWorkerFactory@LocalWorkflow@U2@@6BDescriptor@2@@ 1002d97c     ORFWorker.obj
 0002:00007990       ??_R4type_info@@6B@        1002d990     MSVCRT:ti_inst.obj
 0002:000079a4       ??_R3type_info@@8          1002d9a4     MSVCRT:ti_inst.obj
 0002:000079b4       ??_R2type_info@@8          1002d9b4     MSVCRT:ti_inst.obj
 0002:000079bc       ??_R1A@?0A@EA@type_info@@8 1002d9bc     MSVCRT:ti_inst.obj
 0002:000079e0       ___safe_se_handler_table   1002d9e0     <linker-defined>
 0002:00007d98       ___rtc_iaa                 1002dd98     MSVCRT:initsect.obj
 0002:00007d9c       ___rtc_izz                 1002dd9c     MSVCRT:initsect.obj
 0002:00007da0       ___rtc_taa                 1002dda0     MSVCRT:initsect.obj
 0002:00007da4       ___rtc_tzz                 1002dda4     MSVCRT:initsect.obj
 0002:0000cf64       __IMPORT_DESCRIPTOR_U2Core 10032f64     U2Core:U2Core.dll
 0002:0000cf78       __IMPORT_DESCRIPTOR_U2Algorithm 10032f78     U2Algorithm:U2Algorithm.dll
 0002:0000cf8c       __IMPORT_DESCRIPTOR_U2Gui  10032f8c     U2Gui:U2Gui.dll
 0002:0000cfa0       __IMPORT_DESCRIPTOR_U2View 10032fa0     U2View:U2View.dll
 0002:0000cfb4       __IMPORT_DESCRIPTOR_U2Test 10032fb4     U2Test:U2Test.dll
 0002:0000cfc8       __IMPORT_DESCRIPTOR_U2Lang 10032fc8     U2Lang:U2Lang.dll
 0002:0000cfdc       __IMPORT_DESCRIPTOR_U2Designer 10032fdc     U2Designer:U2Designer.dll
 0002:0000cff0       __IMPORT_DESCRIPTOR_Qt5Widgets 10032ff0     Qt5Widgets:Qt5Widgets.dll
 0002:0000d004       __IMPORT_DESCRIPTOR_Qt5Gui 10033004     Qt5Gui:Qt5Gui.dll
 0002:0000d018       __IMPORT_DESCRIPTOR_Qt5Script 10033018     Qt5Script:Qt5Script.dll
 0002:0000d02c       __IMPORT_DESCRIPTOR_Qt5Xml 1003302c     Qt5Xml:Qt5Xml.dll
 0002:0000d040       __IMPORT_DESCRIPTOR_Qt5Core 10033040     Qt5Core:Qt5Core.dll
 0002:0000d054       __IMPORT_DESCRIPTOR_MSVCP120 10033054     msvcprt:MSVCP120.dll
 0002:0000d068       __IMPORT_DESCRIPTOR_MSVCR120 10033068     MSVCRT:MSVCR120.dll
 0002:0000d07c       __IMPORT_DESCRIPTOR_KERNEL32 1003307c     kernel32:KERNEL32.dll
 0002:0000d090       __NULL_IMPORT_DESCRIPTOR   10033090     U2Core:U2Core.dll
 0003:00000000       ?_Generic_object@?$_Error_objects@H@std@@2V_Generic_error_category@2@A 10042000     ORFDialog.obj
 0003:00000004       ?_Iostream_object@?$_Error_objects@H@std@@2V_Iostream_error_category@2@A 10042004     ORFDialog.obj
 0003:00000008       ?_System_object@?$_Error_objects@H@std@@2V_System_error_category@2@A 10042008     ORFDialog.obj
 0003:00000144       ?staticMetaObject@ORFDialog@U2@@2UQMetaObject@@B 10042144     moc_ORFDialog.obj
 0003:000001c4       ?staticMetaObject@ORFMarkerPlugin@U2@@2UQMetaObject@@B 100421c4     moc_ORFMarkerPlugin.obj
 0003:000001dc       ?staticMetaObject@ORFViewContext@U2@@2UQMetaObject@@B 100421dc     moc_ORFMarkerPlugin.obj
 0003:000001f4       ?staticMetaObject@FindORFsToAnnotationsTask@U2@@2UQMetaObject@@B 100421f4     moc_ORFMarkerTask.obj
 0003:0000020c       ?staticMetaObject@ORFAutoAnnotationsUpdater@U2@@2UQMetaObject@@B 1004220c     moc_ORFMarkerTask.obj
 0003:0000028c       ?staticMetaObject@GTest_ORFMarkerTask@U2@@2UQMetaObject@@B 1004228c     moc_ORFMarkerTests.obj
 0003:000002a4       ?staticMetaObject@QDORFActor@U2@@2UQMetaObject@@B 100422a4     moc_ORFQuery.obj
 0003:000002bc       ?staticMetaObject@ORFPrompter@LocalWorkflow@U2@@2UQMetaObject@@B 100422bc     moc_ORFWorker.obj
 0003:000002d4       ?staticMetaObject@ORFWorker@LocalWorkflow@U2@@2UQMetaObject@@B 100422d4     moc_ORFWorker.obj
 0003:000002ec       ___security_cookie         100422ec     MSVCRT:gs_cookie.obj
 0003:000002f0       ___security_cookie_complement 100422f0     MSVCRT:gs_cookie.obj
 0003:00000300       ___native_dllmain_reason   10042300     MSVCRT:natstart.obj
 0003:00000308       ??_R0?AVerror_category@std@@@8 10042308     ORFDialog.obj
 0003:0000032c       ??_R0?AV_Generic_error_category@std@@@8 1004232c     ORFDialog.obj
 0003:00000358       ??_R0?AV_Iostream_error_category@std@@@8 10042358     ORFDialog.obj
 0003:00000384       ??_R0?AV_System_error_category@std@@@8 10042384     ORFDialog.obj
 0003:000003b0       ??_R0?AVQWidget@@@8        100423b0     ORFDialog.obj
 0003:000003c8       ??_R0?AVQObject@@@8        100423c8     ORFDialog.obj
 0003:000003e0       ??_R0?AVQPaintDevice@@@8   100423e0     ORFDialog.obj
 0003:000003fc       ??_R0?AVQTimer@@@8         100423fc     ORFDialog.obj
 0003:00000414       ??_R0?AVQCheckBox@@@8      10042414     ORFDialog.obj
 0003:0000042c       ??_R0?AVQAbstractButton@@@8 1004242c     ORFDialog.obj
 0003:0000044c       ??_R0?AVQTabWidget@@@8     1004244c     ORFDialog.obj
 0003:00000468       ??_R0?AVQComboBox@@@8      10042468     ORFDialog.obj
 0003:00000480       ??_R0?AVQPushButton@@@8    10042480     ORFDialog.obj
 0003:0000049c       ??_R0?AVQDialogButtonBox@@@8 1004249c     ORFDialog.obj
 0003:000004bc       ??_R0?AVQSpacerItem@@@8    100424bc     ORFDialog.obj
 0003:000004d8       ??_R0?AVQLayoutItem@@@8    100424d8     ORFDialog.obj
 0003:000004f4       ??_R0?AVQHBoxLayout@@@8    100424f4     ORFDialog.obj
 0003:00000510       ??_R0?AVQBoxLayout@@@8     10042510     ORFDialog.obj
 0003:0000052c       ??_R0?AVQLayout@@@8        1004252c     ORFDialog.obj
 0003:00000544       ??_R0?AVQVBoxLayout@@@8    10042544     ORFDialog.obj
 0003:00000560       ??_R0?AVQGridLayout@@@8    10042560     ORFDialog.obj
 0003:0000057c       ??_R0?AVQGroupBox@@@8      1004257c     ORFDialog.obj
 0003:00000594       ??_R0?AVQLabel@@@8         10042594     ORFDialog.obj
 0003:000005ac       ??_R0?AVQFrame@@@8         100425ac     ORFDialog.obj
 0003:000005c4       ??_R0?AVQRadioButton@@@8   100425c4     ORFDialog.obj
 0003:000005e0       ??_R0?AVQSpinBox@@@8       100425e0     ORFDialog.obj
 0003:000005f8       ??_R0?AVQAbstractSpinBox@@@8 100425f8     ORFDialog.obj
 0003:00000618       ??_R0?AVQTextEdit@@@8      10042618     ORFDialog.obj
 0003:00000630       ??_R0?AVQAbstractScrollArea@@@8 10042630     ORFDialog.obj
 0003:00000654       ??_R0?AVQTreeWidget@@@8    10042654     ORFDialog.obj
 0003:00000670       ??_R0?AVQTreeView@@@8      10042670     ORFDialog.obj
 0003:00000688       ??_R0?AVQAbstractItemView@@@8 10042688     ORFDialog.obj
 0003:000006a8       ??_R0?AVAbstractInt32Id@U2@@@8 100426a8     ORFDialog.obj
 0003:000006cc       ??_R0?AV?$AbstractId@H@U2@@@8 100426cc     ORFDialog.obj
 0003:000006ec       ??_R0?AVServiceType@U2@@@8 100426ec     ORFDialog.obj
 0003:0000070c       ??_R0?AVRegionSelector@U2@@@8 1004270c     ORFDialog.obj
 0003:0000072c       ??_R0?AVORFFindTask@U2@@@8 1004272c     ORFDialog.obj
 0003:0000074c       ??_R0?AVTask@U2@@@8        1004274c     ORFDialog.obj
 0003:00000764       ??_R0?AVORFFindResultsListener@U2@@@8 10042764     ORFDialog.obj
 0003:0000078c       ??_R0?AVCreateAnnotationWidgetController@U2@@@8 1004278c     ORFDialog.obj
 0003:000007c0       ??_R0?AVORFDialog@U2@@@8   100427c0     ORFDialog.obj
 0003:000007dc       ??_R0?AVQDialog@@@8        100427dc     ORFDialog.obj
 0003:000007f4       ??_R0?AVUi_ORFDialogBase@@@8 100427f4     ORFDialog.obj
 0003:00000814       ??_R0?AVHelpButton@U2@@@8  10042814     ORFDialog.obj
 0003:00000830       ??_R0?AVORFListItem@U2@@@8 10042830     ORFDialog.obj
 0003:00000850       ??_R0?AVQTreeWidgetItem@@@8 10042850     ORFDialog.obj
 0003:00000870       ??_R0?AVADVGlobalAction@U2@@@8 10042870     ORFMarkerPlugin.obj
 0003:00000894       ??_R0?AVGObjectViewAction@U2@@@8 10042894     ORFMarkerPlugin.obj
 0003:000008b8       ??_R0?AVQAction@@@8        100428b8     ORFMarkerPlugin.obj
 0003:000008d0       ??_R0?AVORFMarkerPlugin@U2@@@8 100428d0     ORFMarkerPlugin.obj
 0003:000008f4       ??_R0?AVPlugin@U2@@@8      100428f4     ORFMarkerPlugin.obj
 0003:0000090c       ??_R0?AVORFViewContext@U2@@@8 1004290c     ORFMarkerPlugin.obj
 0003:0000092c       ??_R0?AVGObjectViewWindowContext@U2@@@8 1004292c     ORFMarkerPlugin.obj
 0003:00000958       ??_R0?AVGObjectViewObjectHandler@U2@@@8 10042958     ORFMarkerPlugin.obj
 0003:00000984       ??_R0?AVXmlTest@U2@@@8     10042984     ORFMarkerPlugin.obj
 0003:000009a0       ??_R0?AVGTest@U2@@@8       100429a0     ORFMarkerPlugin.obj
 0003:000009b8       ??_R0?AVXMLTestFactory@U2@@@8 100429b8     ORFMarkerPlugin.obj
 0003:000009d8       ??_R0?AVGTest_ORFMarkerTask@U2@@@8 100429d8     ORFMarkerPlugin.obj
 0003:00000a00       ??_R0?AVGTest_ORFMarkerTaskFactory@GTest_ORFMarkerTask@U2@@@8 10042a00     ORFMarkerPlugin.obj
 0003:00000a40       ??_R0?AV?$GAutoDeleteList@VXMLTestFactory@U2@@@U2@@@8 10042a40     ORFMarkerPlugin.obj
 0003:00000a78       ??_R0?AVCreateAnnotationsTask@U2@@@8 10042a78     ORFMarkerTask.obj
 0003:00000aa0       ??_R0?AVFindORFsToAnnotationsTask@U2@@@8 10042aa0     ORFMarkerTask.obj
 0003:00000acc       ??_R0?AVORFAutoAnnotationsUpdater@U2@@@8 10042acc     ORFMarkerTask.obj
 0003:00000af8       ??_R0?AVAutoAnnotationsUpdater@U2@@@8 10042af8     ORFMarkerTask.obj
 0003:00000b20       ??_R0?AVDescriptor@U2@@@8  10042b20     ORFQuery.obj
 0003:00000b3c       ??_R0?AVAttribute@U2@@@8   10042b3c     ORFQuery.obj
 0003:00000b58       ??_R0?AVConfigurationEditor@U2@@@8 10042b58     ORFQuery.obj
 0003:00000b80       ??_R0?AVQDORFActor@U2@@@8  10042b80     ORFQuery.obj
 0003:00000b9c       ??_R0?AVQDActor@U2@@@8     10042b9c     ORFQuery.obj
 0003:00000bb8       ??_R0?AVQDORFActorPrototype@U2@@@8 10042bb8     ORFQuery.obj
 0003:00000be0       ??_R0?AVQDActorPrototype@U2@@@8 10042be0     ORFQuery.obj
 0003:00000c04       ??_R0?AVDelegateEditor@U2@@@8 10042c04     ORFQuery.obj
 0003:00000c24       ??_R0?AVSpinBoxDelegate@U2@@@8 10042c24     ORFQuery.obj
 0003:00000c48       ??_R0?AVPropertyDelegate@U2@@@8 10042c48     ORFQuery.obj
 0003:00000c6c       ??_R0?AVQItemDelegate@@@8  10042c6c     ORFQuery.obj
 0003:00000c88       ??_R0?AVQAbstractItemDelegate@@@8 10042c88     ORFQuery.obj
 0003:00000cac       ??_R0?AVComboBoxDelegate@U2@@@8 10042cac     ORFQuery.obj
 0003:00000cd0       ??_R0?AVTaskSignalMapper@U2@@@8 10042cd0     ORFQuery.obj
 0003:00000cf4       ??_R0?AVFailTask@U2@@@8    10042cf4     ORFQuery.obj
 0003:00000d10       ??_R0?AVMapDataType@U2@@@8 10042d10     ORFWorker.obj
 0003:00000d30       ??_R0?AVDataType@U2@@@8    10042d30     ORFWorker.obj
 0003:00000d4c       ??_R0?AVQSharedData@@@8    10042d4c     ORFWorker.obj
 0003:00000d68       ??_R0?AVPortDescriptor@Workflow@U2@@@8 10042d68     ORFWorker.obj
 0003:00000d94       ??_R0?AVIntegralBusActorPrototype@Workflow@U2@@@8 10042d94     ORFWorker.obj
 0003:00000dc8       ??_R0?AVActorPrototype@Workflow@U2@@@8 10042dc8     ORFWorker.obj
 0003:00000df4       ??_R0?AVVisualDescriptor@U2@@@8 10042df4     ORFWorker.obj
 0003:00000e18       ??_R0?AVORFPrompter@LocalWorkflow@U2@@@8 10042e18     ORFWorker.obj
 0003:00000e48       ??_R0?AV?$PrompterBase@VORFPrompter@LocalWorkflow@U2@@@U2@@@8 10042e48     ORFWorker.obj
 0003:00000e88       ??_R0?AVPrompterBaseImpl@U2@@@8 10042e88     ORFWorker.obj
 0003:00000eac       ??_R0?AVActorDocument@Workflow@U2@@@8 10042eac     ORFWorker.obj
 0003:00000ed4       ??_R0?AVQTextDocument@@@8  10042ed4     ORFWorker.obj
 0003:00000ef0       ??_R0?AVPrompter@Workflow@U2@@@8 10042ef0     ORFWorker.obj
 0003:00000f14       ??_R0?AVORFWorker@LocalWorkflow@U2@@@8 10042f14     ORFWorker.obj
 0003:00000f40       ??_R0?AVBaseWorker@LocalWorkflow@U2@@@8 10042f40     ORFWorker.obj
 0003:00000f6c       ??_R0?AVWorker@Workflow@U2@@@8 10042f6c     ORFWorker.obj
 0003:00000f90       ??_R0?AVCommunicationSubject@Workflow@U2@@@8 10042f90     ORFWorker.obj
 0003:00000fc0       ??_R0?AVORFWorkerFactory@LocalWorkflow@U2@@@8 10042fc0     ORFWorker.obj
 0003:00000ff0       ??_R0?AVDomainFactory@Workflow@U2@@@8 10042ff0     ORFWorker.obj
 0003:00001018       ??_R0?AV?$IdRegistry@VDomainFactory@Workflow@U2@@@U2@@@8 10043018     ORFWorker.obj
 0003:00001054       ??_R0?AVtype_info@@@8      10043054     MSVCRT:ti_inst.obj
 0003:000010bc       ?id@?$num_put@DV?$back_insert_iterator@V?$basic_string@DU?$char_traits@D@std@@V?$allocator@D@2@@std@@@std@@@std@@2V0locale@2@A 100430bc     ORFDialog.obj
 0003:000010c0       ?id@?$num_put@_WV?$back_insert_iterator@V?$basic_string@_WU?$char_traits@_W@std@@V?$allocator@_W@2@@std@@@std@@@std@@2V0locale@2@A 100430c0     ORFDialog.obj
 0003:000010c4       ?metatype_id@?1??qt_metatype_id@?$QMetaTypeId@PAVQAction@@@@SAHXZ@4V?$QBasicAtomicInteger@H@@A 100430c4     ORFDialog.obj
 0003:00001120       ?AMINO_TRANSL@ORFSettingsKeys@U2@@2VQString@@B 10043120     ORFMarkerTask.obj
 0003:00001144       ?ALLOW_ALT_START@ORFSettingsKeys@U2@@2VQString@@B 10043144     ORFMarkerTask.obj
 0003:00001158       ?MAX_RESULT@ORFSettingsKeys@U2@@2VQString@@B 10043158     ORFMarkerTask.obj
 0003:0000115c       ?MUST_INIT@ORFSettingsKeys@U2@@2VQString@@B 1004315c     ORFMarkerTask.obj
 0003:00001168       ?SEARCH_REGION@ORFSettingsKeys@U2@@2VQString@@B 10043168     ORFMarkerTask.obj
 0003:0000116c       ?MIN_LEN@ORFSettingsKeys@U2@@2VQString@@B 1004316c     ORFMarkerTask.obj
 0003:00001170       ?STRAND@ORFSettingsKeys@U2@@2VQString@@B 10043170     ORFMarkerTask.obj
 0003:0000117c       ?IS_RESULT_LIMITED@ORFSettingsKeys@U2@@2VQString@@B 1004317c     ORFMarkerTask.obj
 0003:00001180       ?ALLOW_OVERLAP@ORFSettingsKeys@U2@@2VQString@@B 10043180     ORFMarkerTask.obj
 0003:00001184       ?INCLUDE_STOP_CODON@ORFSettingsKeys@U2@@2VQString@@B 10043184     ORFMarkerTask.obj
 0003:00001188       ?MUST_FIT@ORFSettingsKeys@U2@@2VQString@@B 10043188     ORFMarkerTask.obj
 0003:0000118c       ?metatype_id@?1??qt_metatype_id@?$QMetaTypeId@VU2Region@U2@@@@SAHXZ@4V?$QBasicAtomicInteger@H@@A 1004318c     ORFMarkerTask.obj
 0003:000012b8       ?ACTOR_ID@ORFWorkerFactory@LocalWorkflow@U2@@2VQString@@B 100432b8     ORFWorker.obj
 0003:000012bc       ?metatype_id@?1??qt_metatype_id@?$QMetaTypeId@V?$QSharedDataPointer@VDbiDataHandler@Workflow@U2@@@@@@SAHXZ@4V?$QBasicAtomicInteger@H@@A 100432bc     ORFWorker.obj
 0003:0000130c       ?metatype_id@?1??qt_metatype_id@?$QMetaTypeIdQObject@PAVTask@U2@@$00@@SAHXZ@4V?$QBasicAtomicInteger@H@@A 1004330c     moc_ORFDialog.obj
 0003:00001444       ?dummy@?A0xaf06a44c@@3Uinitializer@1@A 10043444     qrc_orf_marker.obj
 0003:00001770       ?__type_info_root_node@@3U__type_info_node@@A 10043770     MSVCRT:tncleanup.obj
 0003:00001778       ___native_startup_lock     10043778     <common>
 0003:0000177c       ___native_startup_state    1004377c     <common>
 0003:00001780       ___dyn_tls_init_callback   10043780     <common>
 0003:00001784       ___onexitend               10043784     <common>
 0003:00001788       ___onexitbegin             10043788     <common>

 entry point at        0001:0001eba0

 Static symbols

 0000:fffb5000       .debug$S                   10000000     MSVCRT:MSVCR120.dll
 0000:fffb5000       .debug$S                   10000000     MSVCRT:MSVCR120.dll
 0000:fffb5000       .debug$S                   10000000     MSVCRT:MSVCR120.dll
 0000:fffb5000       .debug$S                   10000000     MSVCRT:MSVCR120.dll
 0000:fffb5000       .debug$S                   10000000     MSVCRT:MSVCR120.dll
 0000:fffb5000       .debug$S                   10000000     MSVCRT:MSVCR120.dll
 0000:fffb5000       .debug$S                   10000000     MSVCRT:MSVCR120.dll
 0000:fffb5000       .debug$S                   10000000     MSVCRT:MSVCR120.dll
 0000:fffb5000       .debug$S                   10000000     MSVCRT:MSVCR120.dll
 0000:fffb5000       .debug$S                   10000000     MSVCRT:MSVCR120.dll
 0001:fffff000       __ehhandler$?node_copy@?$QList@VORFFindResult@U2@@@@AAEXPAUNode@1@00@Z 10000000 f   ORFMarkerTask.obj
 0000:fffb5000       .debug$S                   10000000     MSVCRT:MSVCR120.dll
 0000:fffb5000       .debug$S                   10000000     MSVCRT:MSVCR120.dll
 0000:fffb5000       .debug$S                   10000000     MSVCRT:MSVCR120.dll
 0000:fffb5000       .debug$S                   10000000     MSVCRT:MSVCR120.dll
 0000:fffb5000       .debug$S                   10000000     MSVCRT:MSVCR120.dll
 0000:fffb5000       .debug$S                   10000000     MSVCRT:MSVCR120.dll
 0001:fffff000       __ehhandler$??0?$QList@VORFFindResult@U2@@@@QAE@ABV0@@Z 10000000 f   ORFMarkerTask.obj
 0000:fffb5000       .debug$S                   10000000     MSVCRT:MSVCR120.dll
 0001:fffff000       __ehhandler$??0?$QList@PAVTask@U2@@@@QAE@ABV0@@Z 10000000 f   ORFMarkerTask.obj
 0000:fffb5000       .debug$S                   10000000     MSVCRT:MSVCR120.dll
 0001:fffff000       __ehhandler$?_Copy@?$basic_string@DU?$char_traits@D@std@@V?$allocator@D@2@@std@@QAEXII@Z 10000000 f   ORFMarkerTask.obj
 0000:fffb5000       .debug$S                   10000000     MSVCRT:MSVCR120.dll
 0002:fffda000       ?_System_object$initializer$@?$_Error_objects@H@std@@2P6AXXZA 10000000     ORFMarkerTests.obj
 0000:fffb5000       .debug$S                   10000000     MSVCRT:MSVCR120.dll
 0002:fffda000       ?_Iostream_object$initializer$@?$_Error_objects@H@std@@2P6AXXZA 10000000     ORFMarkerTests.obj
 0000:fffb5000       .debug$S                   10000000     MSVCRT:MSVCR120.dll
 0002:fffda000       ?_Generic_object$initializer$@?$_Error_objects@H@std@@2P6AXXZA 10000000     ORFMarkerTests.obj
 0000:fffb5000       .debug$S                   10000000     MSVCRT:MSVCR120.dll
 0002:fffda000       __catchsym$?_Copy@?$basic_string@DU?$char_traits@D@std@@V?$allocator@D@2@@std@@QAEXII@Z$5 10000000     ORFMarkerTask.obj
 0000:fffb5000       .debug$S                   10000000     MSVCRT:MSVCR120.dll
 0002:fffda000       __catchsym$??0?$QList@PAVTask@U2@@@@QAE@ABV0@@Z$2 10000000     ORFMarkerTask.obj
 0000:fffb5000       .debug$S                   10000000     MSVCRT:MSVCR120.dll
 0002:fffda000       __catchsym$??0?$QList@VORFFindResult@U2@@@@QAE@ABV0@@Z$2 10000000     ORFMarkerTask.obj
 0000:fffb5000       .debug$S                   10000000     MSVCRT:MSVCR120.dll
 0002:fffda000       __catchsym$?node_copy@?$QList@VORFFindResult@U2@@@@AAEXPAUNode@1@00@Z$4 10000000     ORFMarkerTask.obj
 0002:fffda000       ?_Generic_object$initializer$@?$_Error_objects@H@std@@2P6AXXZA 10000000     ORFMarkerTask.obj
 0002:fffda000       ?_Iostream_object$initializer$@?$_Error_objects@H@std@@2P6AXXZA 10000000     ORFMarkerTask.obj
 0000:fffb5000       .debug$S                   10000000     MSVCRT:MSVCR120.dll
 0002:fffda000       ?_System_object$initializer$@?$_Error_objects@H@std@@2P6AXXZA 10000000     ORFMarkerTask.obj
 0000:fffb5000       .debug$S                   10000000     MSVCRT:MSVCR120.dll
 0002:fffda000       __catchsym$?node_copy@?$QList@VORFFindResult@U2@@@@AAEXPAUNode@1@00@Z$4 10000000     ORFMarkerTests.obj
 0002:fffda000       __catchsym$??0?$QList@VORFFindResult@U2@@@@QAE@ABV0@@Z$2 10000000     ORFMarkerTests.obj
 0001:fffff000       __ehhandler$?_Copy@?$basic_string@DU?$char_traits@D@std@@V?$allocator@D@2@@std@@QAEXII@Z 10000000 f   moc_ORFWorker.obj
 0001:fffff000       __ehhandler$?_Copy@?$basic_string@DU?$char_traits@D@std@@V?$allocator@D@2@@std@@QAEXII@Z 10000000 f   ORFMarkerPlugin.obj
 0002:fffda000       __unwindtable$??H@YA?BVQString@@PBDABV0@@Z 10000000     ORFMarkerTests.obj
 0002:fffda000       __catchsym$?_Copy@?$basic_string@DU?$char_traits@D@std@@V?$allocator@D@2@@std@@QAEXII@Z$5 10000000     ORFMarkerTests.obj
 0002:fffda000       __catchsym$?_Copy@?$basic_string@DU?$char_traits@D@std@@V?$allocator@D@2@@std@@QAEXII@Z$5 10000000     ORFMarkerPlugin.obj
 0002:fffda000       ?_Generic_object$initializer$@?$_Error_objects@H@std@@2P6AXXZA 10000000     ORFMarkerPlugin.obj
 0000:fffb5000       .debug$S                   10000000     msvcprt:MSVCP120.dll
 0000:fffb5000       .debug$S                   10000000     msvcprt:MSVCP120.dll
 0000:fffb5000       .debug$S                   10000000     msvcprt:MSVCP120.dll
 0000:fffb5000       .debug$S                   10000000     msvcprt:MSVCP120.dll
 0000:fffb5000       .debug$S                   10000000     msvcprt:MSVCP120.dll
 0000:fffb5000       .debug$S                   10000000     kernel32:KERNEL32.dll
 0000:fffb5000       .debug$S                   10000000     kernel32:KERNEL32.dll
 0000:fffb5000       .debug$S                   10000000     kernel32:KERNEL32.dll
 0000:fffb5000       .debug$S                   10000000     kernel32:KERNEL32.dll
 0000:fffb5000       .debug$S                   10000000     kernel32:KERNEL32.dll
 0000:fffb5000       .debug$S                   10000000     kernel32:KERNEL32.dll
 0000:fffb5000       .debug$S                   10000000     kernel32:KERNEL32.dll
 0000:fffb5000       .debug$S                   10000000     kernel32:KERNEL32.dll
 0000:fffb5000       .debug$S                   10000000     kernel32:KERNEL32.dll
 0000:fffb5000       .debug$S                   10000000     Qt5Core:Qt5Core.dll
 0002:fffda000       ?_Iostream_object$initializer$@?$_Error_objects@H@std@@2P6AXXZA 10000000     ORFMarkerPlugin.obj
 0002:fffda000       ?_System_object$initializer$@?$_Error_objects@H@std@@2P6AXXZA 10000000     ORFMarkerPlugin.obj
 0001:fffff000       __ehhandler$?node_copy@?$QList@VORFFindResult@U2@@@@AAEXPAUNode@1@00@Z 10000000 f   ORFMarkerTests.obj
 0001:fffff000       __ehhandler$??0?$QList@VORFFindResult@U2@@@@QAE@ABV0@@Z 10000000 f   ORFMarkerTests.obj
 0002:fffda000       __catchsym$?_Copy@?$basic_string@DU?$char_traits@D@std@@V?$allocator@D@2@@std@@QAEXII@Z$5 10000000     moc_ORFWorker.obj
 0000:fffb5000       .debug$S                   10000000     Qt5Core:Qt5Core.dll
 0000:fffb5000       .debug$S                   10000000     Qt5Core:Qt5Core.dll
 0000:fffb5000       .debug$S                   10000000     Qt5Core:Qt5Core.dll
 0000:fffb5000       .debug$S                   10000000     Qt5Core:Qt5Core.dll
 0000:fffb5000       .debug$S                   10000000     Qt5Core:Qt5Core.dll
 0000:fffb5000       .debug$S                   10000000     Qt5Core:Qt5Core.dll
 0000:fffb5000       .debug$S                   10000000     Qt5Core:Qt5Core.dll
 0000:fffb5000       .debug$S                   10000000     Qt5Core:Qt5Core.dll
 0000:fffb5000       .debug$S                   10000000     Qt5Core:Qt5Core.dll
 0000:fffb5000       .debug$S                   10000000     Qt5Core:Qt5Core.dll
 0000:fffb5000       .debug$S                   10000000     Qt5Core:Qt5Core.dll
 0000:fffb5000       .debug$S                   10000000     Qt5Core:Qt5Core.dll
 0000:fffb5000       .debug$S                   10000000     Qt5Core:Qt5Core.dll
 0000:fffb5000       .debug$S                   10000000     Qt5Core:Qt5Core.dll
 0000:fffb5000       .debug$S                   10000000     Qt5Core:Qt5Core.dll
 0000:fffb5000       .debug$S                   10000000     Qt5Core:Qt5Core.dll
 0000:fffb5000       .debug$S                   10000000     Qt5Core:Qt5Core.dll
 0000:fffb5000       .debug$S                   10000000     Qt5Core:Qt5Core.dll
 0000:fffb5000       .debug$S                   10000000     Qt5Core:Qt5Core.dll
 0000:fffb5000       .debug$S                   10000000     Qt5Core:Qt5Core.dll
 0000:fffb5000       .debug$S                   10000000     Qt5Core:Qt5Core.dll
 0000:fffb5000       .debug$S                   10000000     Qt5Core:Qt5Core.dll
 0000:fffb5000       .debug$S                   10000000     Qt5Core:Qt5Core.dll
 0000:fffb5000       .debug$S                   10000000     Qt5Core:Qt5Core.dll
 0000:fffb5000       .debug$S                   10000000     Qt5Core:Qt5Core.dll
 0000:fffb5000       .debug$S                   10000000     Qt5Core:Qt5Core.dll
 0000:fffb5000       .debug$S                   10000000     Qt5Core:Qt5Core.dll
 0000:fffb5000       .debug$S                   10000000     Qt5Core:Qt5Core.dll
 0000:fffb5000       .debug$S                   10000000     Qt5Core:Qt5Core.dll
 0000:fffb5000       .debug$S                   10000000     Qt5Core:Qt5Core.dll
 0000:fffb5000       .debug$S                   10000000     Qt5Core:Qt5Core.dll
 0000:fffb5000       .debug$S                   10000000     Qt5Core:Qt5Core.dll
 0000:fffb5000       .debug$S                   10000000     Qt5Core:Qt5Core.dll
 0000:fffb5000       .debug$S                   10000000     Qt5Core:Qt5Core.dll
 0000:fffb5000       .debug$S                   10000000     Qt5Core:Qt5Core.dll
 0000:fffb5000       .debug$S                   10000000     Qt5Core:Qt5Core.dll
 0000:fffb5000       .debug$S                   10000000     Qt5Core:Qt5Core.dll
 0000:fffb5000       .debug$S                   10000000     Qt5Core:Qt5Core.dll
 0000:fffb5000       .debug$S                   10000000     Qt5Core:Qt5Core.dll
 0000:fffb5000       .debug$S                   10000000     Qt5Core:Qt5Core.dll
 0000:fffb5000       .debug$S                   10000000     Qt5Core:Qt5Core.dll
 0000:fffb5000       .debug$S                   10000000     Qt5Core:Qt5Core.dll
 0002:fffda000       ?_Generic_object$initializer$@?$_Error_objects@H@std@@2P6AXXZA 10000000     moc_ORFWorker.obj
 0002:fffda000       ?_Iostream_object$initializer$@?$_Error_objects@H@std@@2P6AXXZA 10000000     moc_ORFWorker.obj
 0002:fffda000       ?_System_object$initializer$@?$_Error_objects@H@std@@2P6AXXZA 10000000     moc_ORFWorker.obj
 0000:fffb5000       .debug$S                   10000000     Qt5Core:Qt5Core.dll
 0000:fffb5000       .debug$S                   10000000     Qt5Core:Qt5Core.dll
 0001:fffff000       __unwindfunclet$??H@YA?BVQString@@PBDABV0@@Z$0 10000000 f   ORFMarkerTests.obj
 0000:fffb5000       .debug$S                   10000000     Qt5Core:Qt5Core.dll
 0001:fffff000       __ehhandler$?_Copy@?$basic_string@DU?$char_traits@D@std@@V?$allocator@D@2@@std@@QAEXII@Z 10000000 f   ORFMarkerTests.obj
 0000:fffb5000       .debug$S                   10000000     Qt5Core:Qt5Core.dll
 0002:fffda000       ?_System_object$initializer$@?$_Error_objects@H@std@@2P6AXXZA 10000000     ORFQuery.obj
 0000:fffb5000       .debug$S                   10000000     Qt5Core:Qt5Core.dll
 0002:fffda000       ?_Iostream_object$initializer$@?$_Error_objects@H@std@@2P6AXXZA 10000000     ORFQuery.obj
 0000:fffb5000       .debug$S                   10000000     Qt5Core:Qt5Core.dll
 0002:fffda000       ?_Generic_object$initializer$@?$_Error_objects@H@std@@2P6AXXZA 10000000     ORFQuery.obj
 0000:fffb5000       .debug$S                   10000000     Qt5Core:Qt5Core.dll
 0002:fffda000       __catchsym$?node_copy@?$QList@VORFFindResult@U2@@@@AAEXPAUNode@1@00@Z$4 10000000     ORFQuery.obj
 0000:fffb5000       .debug$S                   10000000     Qt5Core:Qt5Core.dll
 0002:fffda000       __catchsym$??0?$QList@VORFFindResult@U2@@@@QAE@ABV0@@Z$2 10000000     ORFQuery.obj
 0000:fffb5000       .debug$S                   10000000     Qt5Core:Qt5Core.dll
 0002:fffda000       __catchsym$?_Copy@?$basic_string@DU?$char_traits@D@std@@V?$allocator@D@2@@std@@QAEXII@Z$5 10000000     ORFQuery.obj
 0000:fffb5000       .debug$S                   10000000     Qt5Core:Qt5Core.dll
 0001:fffff000       __ehhandler$?node_copy@?$QList@VORFFindResult@U2@@@@AAEXPAUNode@1@00@Z 10000000 f   ORFQuery.obj
 0000:fffb5000       .debug$S                   10000000     Qt5Core:Qt5Core.dll
 0001:fffff000       __ehhandler$??0?$QList@VORFFindResult@U2@@@@QAE@ABV0@@Z 10000000 f   ORFQuery.obj
 0000:fffb5000       .debug$S                   10000000     U2Core:U2Core.dll
 0000:fffb5000       .debug$S                   10000000     Qt5Core:Qt5Core.dll
 0000:fffb5000       .debug$S                   10000000     U2Core:U2Core.dll
 0000:fffb5000       .debug$S                   10000000     Qt5Core:Qt5Core.dll
 0000:fffb5000       .debug$S                   10000000     U2Core:U2Core.dll
 0000:fffb5000       .debug$S                   10000000     Qt5Core:Qt5Core.dll
 0001:fffff000       __ehhandler$?_Copy@?$basic_string@DU?$char_traits@D@std@@V?$allocator@D@2@@std@@QAEXII@Z 10000000 f   moc_ORFQuery.obj
 0000:fffb5000       .debug$S                   10000000     U2Core:U2Core.dll
 0000:fffb5000       .debug$S                   10000000     U2Core:U2Core.dll
 0000:fffb5000       .debug$S                   10000000     Qt5Core:Qt5Core.dll
 0000:fffb5000       .debug$S                   10000000     Qt5Core:Qt5Core.dll
 0000:fffb5000       .debug$S                   10000000     Qt5Core:Qt5Core.dll
 0000:fffb5000       .debug$S                   10000000     Qt5Core:Qt5Core.dll
 0000:fffb5000       .debug$S                   10000000     Qt5Core:Qt5Core.dll
 0000:fffb5000       .debug$S                   10000000     Qt5Core:Qt5Core.dll
 0000:fffb5000       .debug$S                   10000000     Qt5Core:Qt5Core.dll
 0000:fffb5000       .debug$S                   10000000     Qt5Core:Qt5Core.dll
 0000:fffb5000       .debug$S                   10000000     Qt5Core:Qt5Core.dll
 0000:fffb5000       .debug$S                   10000000     Qt5Core:Qt5Core.dll
 0000:fffb5000       .debug$S                   10000000     Qt5Core:Qt5Core.dll
 0000:fffb5000       .debug$S                   10000000     Qt5Core:Qt5Core.dll
 0000:fffb5000       .debug$S                   10000000     Qt5Core:Qt5Core.dll
 0000:fffb5000       .debug$S                   10000000     Qt5Core:Qt5Core.dll
 0000:fffb5000       .debug$S                   10000000     Qt5Core:Qt5Core.dll
 0000:fffb5000       .debug$S                   10000000     Qt5Core:Qt5Core.dll
 0000:fffb5000       .debug$S                   10000000     Qt5Core:Qt5Core.dll
 0000:fffb5000       .debug$S                   10000000     Qt5Core:Qt5Core.dll
 0000:fffb5000       .debug$S                   10000000     U2Core:U2Core.dll
 0001:fffff000       __unwindfunclet$?qt_metatype_id@?$QMetaTypeIdQObject@PAVTask@U2@@$00@@SAHXZ$0 10000000 f   moc_ORFQuery.obj
 0000:fffb5000       .debug$S                   10000000     U2Core:U2Core.dll
 0000:fffb5000       .debug$S                   10000000     U2Core:U2Core.dll
 0000:fffb5000       .debug$S                   10000000     U2Core:U2Core.dll
 0000:fffb5000       .debug$S                   10000000     U2Core:U2Core.dll
 0002:fffda000       __catchsym$?_Copy@?$basic_string@DU?$char_traits@D@std@@V?$allocator@D@2@@std@@QAEXII@Z$5 10000000     moc_ORFQuery.obj
 0000:fffb5000       .debug$S                   10000000     Qt5Core:Qt5Core.dll
 0000:fffb5000       .debug$S                   10000000     Qt5Core:Qt5Core.dll
 0000:fffb5000       .debug$S                   10000000     Qt5Core:Qt5Core.dll
 0000:fffb5000       .debug$S                   10000000     Qt5Core:Qt5Core.dll
 0000:fffb5000       .debug$S                   10000000     Qt5Core:Qt5Core.dll
 0000:fffb5000       .debug$S                   10000000     Qt5Core:Qt5Core.dll
 0000:fffb5000       .debug$S                   10000000     Qt5Core:Qt5Core.dll
 0000:fffb5000       .debug$S                   10000000     Qt5Core:Qt5Core.dll
 0000:fffb5000       .debug$S                   10000000     Qt5Core:Qt5Core.dll
 0000:fffb5000       .debug$S                   10000000     Qt5Core:Qt5Core.dll
 0000:fffb5000       .debug$S                   10000000     Qt5Core:Qt5Core.dll
 0000:fffb5000       .debug$S                   10000000     Qt5Core:Qt5Core.dll
 0000:fffb5000       .debug$S                   10000000     Qt5Core:Qt5Core.dll
 0000:fffb5000       .debug$S                   10000000     Qt5Core:Qt5Core.dll
 0000:fffb5000       .debug$S                   10000000     Qt5Core:Qt5Core.dll
 0000:fffb5000       .debug$S                   10000000     Qt5Core:Qt5Core.dll
 0000:fffb5000       .debug$S                   10000000     Qt5Core:Qt5Core.dll
 0000:fffb5000       .debug$S                   10000000     Qt5Core:Qt5Core.dll
 0000:fffb5000       .debug$S                   10000000     U2Core:U2Core.dll
 0002:fffda000       __unwindtable$?qt_metatype_id@?$QMetaTypeIdQObject@PAVTask@U2@@$00@@SAHXZ 10000000     moc_ORFQuery.obj
 0000:fffb5000       .debug$S                   10000000     Qt5Core:Qt5Core.dll
 0000:fffb5000       .debug$S                   10000000     Qt5Core:Qt5Core.dll
 0000:fffb5000       .debug$S                   10000000     Qt5Core:Qt5Core.dll
 0000:fffb5000       .debug$S                   10000000     Qt5Core:Qt5Core.dll
 0000:fffb5000       .debug$S                   10000000     Qt5Core:Qt5Core.dll
 0000:fffb5000       .debug$S                   10000000     Qt5Core:Qt5Core.dll
 0000:fffb5000       .debug$S                   10000000     Qt5Core:Qt5Core.dll
 0000:fffb5000       .debug$S                   10000000     Qt5Core:Qt5Core.dll
 0000:fffb5000       .debug$S                   10000000     Qt5Core:Qt5Core.dll
 0000:fffb5000       .debug$S                   10000000     Qt5Core:Qt5Core.dll
 0000:fffb5000       .debug$S                   10000000     Qt5Core:Qt5Core.dll
 0000:fffb5000       .debug$S                   10000000     Qt5Core:Qt5Core.dll
 0000:fffb5000       .debug$S                   10000000     Qt5Core:Qt5Core.dll
 0000:fffb5000       .debug$S                   10000000     Qt5Core:Qt5Core.dll
 0000:fffb5000       .debug$S                   10000000     Qt5Core:Qt5Core.dll
 0000:fffb5000       .debug$S                   10000000     Qt5Core:Qt5Core.dll
 0000:fffb5000       .debug$S                   10000000     Qt5Xml:Qt5Xml.dll
 0000:fffb5000       .debug$S                   10000000     Qt5Script:Qt5Script.dll
 0000:fffb5000       .debug$S                   10000000     Qt5Script:Qt5Script.dll
 0000:fffb5000       .debug$S                   10000000     Qt5Script:Qt5Script.dll
 0000:fffb5000       .debug$S                   10000000     Qt5Script:Qt5Script.dll
 0000:fffb5000       .debug$S                   10000000     Qt5Script:Qt5Script.dll
 0000:fffb5000       .debug$S                   10000000     Qt5Script:Qt5Script.dll
 0002:fffda000       ?_Generic_object$initializer$@?$_Error_objects@H@std@@2P6AXXZA 10000000     moc_ORFQuery.obj
 0002:fffda000       ?_Iostream_object$initializer$@?$_Error_objects@H@std@@2P6AXXZA 10000000     moc_ORFQuery.obj
 0002:fffda000       ?_System_object$initializer$@?$_Error_objects@H@std@@2P6AXXZA 10000000     moc_ORFQuery.obj
 0000:fffb5000       .debug$S                   10000000     Qt5Script:Qt5Script.dll
 0000:fffb5000       .debug$S                   10000000     Qt5Script:Qt5Script.dll
 0000:fffb5000       .debug$S                   10000000     U2Core:U2Core.dll
 0000:fffb5000       .debug$S                   10000000     Qt5Script:Qt5Script.dll
 0000:fffb5000       .debug$S                   10000000     U2Core:U2Core.dll
 0000:fffb5000       .debug$S                   10000000     Qt5Script:Qt5Script.dll
 0000:fffb5000       .debug$S                   10000000     U2Core:U2Core.dll
 0000:fffb5000       .debug$S                   10000000     Qt5Gui:Qt5Gui.dll
 0000:fffb5000       .debug$S                   10000000     U2Core:U2Core.dll
 0000:fffb5000       .debug$S                   10000000     Qt5Gui:Qt5Gui.dll
 0000:fffb5000       .debug$S                   10000000     U2Core:U2Core.dll
 0000:fffb5000       .debug$S                   10000000     Qt5Gui:Qt5Gui.dll
 0000:fffb5000       .debug$S                   10000000     U2Core:U2Core.dll
 0000:fffb5000       .debug$S                   10000000     Qt5Gui:Qt5Gui.dll
 0000:fffb5000       .debug$S                   10000000     U2Core:U2Core.dll
 0000:fffb5000       .debug$S                   10000000     Qt5Gui:Qt5Gui.dll
 0000:fffb5000       .debug$S                   10000000     U2Core:U2Core.dll
 0000:fffb5000       .debug$S                   10000000     Qt5Gui:Qt5Gui.dll
 0000:fffb5000       .debug$S                   10000000     U2Core:U2Core.dll
 0000:fffb5000       .debug$S                   10000000     Qt5Gui:Qt5Gui.dll
 0000:fffb5000       .debug$S                   10000000     U2Core:U2Core.dll
 0000:fffb5000       .debug$S                   10000000     Qt5Gui:Qt5Gui.dll
 0000:fffb5000       .debug$S                   10000000     U2Core:U2Core.dll
 0000:fffb5000       .debug$S                   10000000     Qt5Gui:Qt5Gui.dll
 0000:fffb5000       .debug$S                   10000000     U2Core:U2Core.dll
 0000:fffb5000       .debug$S                   10000000     Qt5Widgets:Qt5Widgets.dll
 0001:fffff000       __ehhandler$?_Copy@?$basic_string@DU?$char_traits@D@std@@V?$allocator@D@2@@std@@QAEXII@Z 10000000 f   ORFQuery.obj
 0000:fffb5000       .debug$S                   10000000     Qt5Widgets:Qt5Widgets.dll
 0000:fffb5000       .debug$S                   10000000     U2Core:U2Core.dll
 0000:fffb5000       .debug$S                   10000000     Qt5Widgets:Qt5Widgets.dll
 0000:fffb5000       .debug$S                   10000000     U2Core:U2Core.dll
 0000:fffb5000       .debug$S                   10000000     Qt5Widgets:Qt5Widgets.dll
 0000:fffb5000       .debug$S                   10000000     U2Core:U2Core.dll
 0000:fffb5000       .debug$S                   10000000     Qt5Widgets:Qt5Widgets.dll
 0000:fffb5000       .debug$S                   10000000     U2Core:U2Core.dll
 0000:fffb5000       .debug$S                   10000000     Qt5Widgets:Qt5Widgets.dll
 0000:fffb5000       .debug$S                   10000000     U2Core:U2Core.dll
 0000:fffb5000       .debug$S                   10000000     Qt5Widgets:Qt5Widgets.dll
 0000:fffb5000       .debug$S                   10000000     U2Core:U2Core.dll
 0000:fffb5000       .debug$S                   10000000     Qt5Widgets:Qt5Widgets.dll
 0000:fffb5000       .debug$S                   10000000     U2Core:U2Core.dll
 0000:fffb5000       .debug$S                   10000000     Qt5Widgets:Qt5Widgets.dll
 0000:fffb5000       .debug$S                   10000000     U2Core:U2Core.dll
 0000:fffb5000       .debug$S                   10000000     Qt5Widgets:Qt5Widgets.dll
 0000:fffb5000       .debug$S                   10000000     U2Core:U2Core.dll
 0000:fffb5000       .debug$S                   10000000     Qt5Widgets:Qt5Widgets.dll
 0000:fffb5000       .debug$S                   10000000     U2Core:U2Core.dll
 0000:fffb5000       .debug$S                   10000000     U2Core:U2Core.dll
 0000:fffb5000       .debug$S                   10000000     Qt5Widgets:Qt5Widgets.dll
 0000:fffb5000       .debug$S                   10000000     U2Core:U2Core.dll
 0000:fffb5000       .debug$S                   10000000     Qt5Widgets:Qt5Widgets.dll
 0000:fffb5000       .debug$S                   10000000     U2Core:U2Core.dll
 0000:fffb5000       .debug$S                   10000000     Qt5Widgets:Qt5Widgets.dll
 0001:fffff000       __ehhandler$?_Copy@?$basic_string@DU?$char_traits@D@std@@V?$allocator@D@2@@std@@QAEXII@Z 10000000 f   moc_ORFMarkerTests.obj
 0000:fffb5000       .debug$S                   10000000     U2Core:U2Core.dll
 0000:fffb5000       .debug$S                   10000000     U2Core:U2Core.dll
 0000:fffb5000       .debug$S                   10000000     Qt5Widgets:Qt5Widgets.dll
 0000:fffb5000       .debug$S                   10000000     Qt5Widgets:Qt5Widgets.dll
 0000:fffb5000       .debug$S                   10000000     Qt5Widgets:Qt5Widgets.dll
 0000:fffb5000       .debug$S                   10000000     Qt5Widgets:Qt5Widgets.dll
 0000:fffb5000       .debug$S                   10000000     Qt5Widgets:Qt5Widgets.dll
 0000:fffb5000       .debug$S                   10000000     Qt5Widgets:Qt5Widgets.dll
 0000:fffb5000       .debug$S                   10000000     Qt5Widgets:Qt5Widgets.dll
 0000:fffb5000       .debug$S                   10000000     Qt5Widgets:Qt5Widgets.dll
 0000:fffb5000       .debug$S                   10000000     Qt5Widgets:Qt5Widgets.dll
 0000:fffb5000       .debug$S                   10000000     Qt5Widgets:Qt5Widgets.dll
 0000:fffb5000       .debug$S                   10000000     Qt5Widgets:Qt5Widgets.dll
 0000:fffb5000       .debug$S                   10000000     Qt5Widgets:Qt5Widgets.dll
 0000:fffb5000       .debug$S                   10000000     Qt5Widgets:Qt5Widgets.dll
 0000:fffb5000       .debug$S                   10000000     Qt5Widgets:Qt5Widgets.dll
 0000:fffb5000       .debug$S                   10000000     Qt5Widgets:Qt5Widgets.dll
 0000:fffb5000       .debug$S                   10000000     Qt5Widgets:Qt5Widgets.dll
 0000:fffb5000       .debug$S                   10000000     Qt5Widgets:Qt5Widgets.dll
 0000:fffb5000       .debug$S                   10000000     Qt5Widgets:Qt5Widgets.dll
 0000:fffb5000       .debug$S                   10000000     U2Core:U2Core.dll
 0000:fffb5000       .debug$S                   10000000     U2Core:U2Core.dll
 0000:fffb5000       .debug$S                   10000000     U2Core:U2Core.dll
 0000:fffb5000       .debug$S                   10000000     U2Core:U2Core.dll
 0002:fffda000       __catchsym$?_Copy@?$basic_string@DU?$char_traits@D@std@@V?$allocator@D@2@@std@@QAEXII@Z$5 10000000     moc_ORFMarkerTests.obj
 0000:fffb5000       .debug$S                   10000000     Qt5Widgets:Qt5Widgets.dll
 0000:fffb5000       .debug$S                   10000000     Qt5Widgets:Qt5Widgets.dll
 0000:fffb5000       .debug$S                   10000000     Qt5Widgets:Qt5Widgets.dll
 0000:fffb5000       .debug$S                   10000000     Qt5Widgets:Qt5Widgets.dll
 0000:fffb5000       .debug$S                   10000000     Qt5Widgets:Qt5Widgets.dll
 0000:fffb5000       .debug$S                   10000000     Qt5Widgets:Qt5Widgets.dll
 0000:fffb5000       .debug$S                   10000000     Qt5Widgets:Qt5Widgets.dll
 0000:fffb5000       .debug$S                   10000000     Qt5Widgets:Qt5Widgets.dll
 0000:fffb5000       .debug$S                   10000000     Qt5Widgets:Qt5Widgets.dll
 0000:fffb5000       .debug$S                   10000000     Qt5Widgets:Qt5Widgets.dll
 0000:fffb5000       .debug$S                   10000000     Qt5Widgets:Qt5Widgets.dll
 0000:fffb5000       .debug$S                   10000000     Qt5Widgets:Qt5Widgets.dll
 0000:fffb5000       .debug$S                   10000000     Qt5Widgets:Qt5Widgets.dll
 0000:fffb5000       .debug$S                   10000000     Qt5Widgets:Qt5Widgets.dll
 0000:fffb5000       .debug$S                   10000000     Qt5Widgets:Qt5Widgets.dll
 0000:fffb5000       .debug$S                   10000000     Qt5Widgets:Qt5Widgets.dll
 0000:fffb5000       .debug$S                   10000000     Qt5Widgets:Qt5Widgets.dll
 0000:fffb5000       .debug$S                   10000000     Qt5Widgets:Qt5Widgets.dll
 0000:fffb5000       .debug$S                   10000000     Qt5Widgets:Qt5Widgets.dll
 0000:fffb5000       .debug$S                   10000000     Qt5Widgets:Qt5Widgets.dll
 0000:fffb5000       .debug$S                   10000000     Qt5Widgets:Qt5Widgets.dll
 0000:fffb5000       .debug$S                   10000000     Qt5Widgets:Qt5Widgets.dll
 0000:fffb5000       .debug$S                   10000000     Qt5Widgets:Qt5Widgets.dll
 0000:fffb5000       .debug$S                   10000000     Qt5Widgets:Qt5Widgets.dll
 0000:fffb5000       .debug$S                   10000000     Qt5Widgets:Qt5Widgets.dll
 0000:fffb5000       .debug$S                   10000000     Qt5Widgets:Qt5Widgets.dll
 0000:fffb5000       .debug$S                   10000000     Qt5Widgets:Qt5Widgets.dll
 0000:fffb5000       .debug$S                   10000000     Qt5Widgets:Qt5Widgets.dll
 0000:fffb5000       .debug$S                   10000000     Qt5Widgets:Qt5Widgets.dll
 0000:fffb5000       .debug$S                   10000000     Qt5Widgets:Qt5Widgets.dll
 0000:fffb5000       .debug$S                   10000000     Qt5Widgets:Qt5Widgets.dll
 0000:fffb5000       .debug$S                   10000000     Qt5Widgets:Qt5Widgets.dll
 0000:fffb5000       .debug$S                   10000000     Qt5Widgets:Qt5Widgets.dll
 0000:fffb5000       .debug$S                   10000000     Qt5Widgets:Qt5Widgets.dll
 0000:fffb5000       .debug$S                   10000000     Qt5Widgets:Qt5Widgets.dll
 0000:fffb5000       .debug$S                   10000000     Qt5Widgets:Qt5Widgets.dll
 0000:fffb5000       .debug$S                   10000000     Qt5Widgets:Qt5Widgets.dll
 0000:fffb5000       .debug$S                   10000000     Qt5Widgets:Qt5Widgets.dll
 0000:fffb5000       .debug$S                   10000000     Qt5Widgets:Qt5Widgets.dll
 0000:fffb5000       .debug$S                   10000000     Qt5Widgets:Qt5Widgets.dll
 0000:fffb5000       .debug$S                   10000000     Qt5Widgets:Qt5Widgets.dll
 0000:fffb5000       .debug$S                   10000000     Qt5Widgets:Qt5Widgets.dll
 0000:fffb5000       .debug$S                   10000000     Qt5Widgets:Qt5Widgets.dll
 0000:fffb5000       .debug$S                   10000000     Qt5Widgets:Qt5Widgets.dll
 0000:fffb5000       .debug$S                   10000000     Qt5Widgets:Qt5Widgets.dll
 0000:fffb5000       .debug$S                   10000000     Qt5Widgets:Qt5Widgets.dll
 0000:fffb5000       .debug$S                   10000000     Qt5Widgets:Qt5Widgets.dll
 0000:fffb5000       .debug$S                   10000000     Qt5Widgets:Qt5Widgets.dll
 0000:fffb5000       .debug$S                   10000000     Qt5Widgets:Qt5Widgets.dll
 0000:fffb5000       .debug$S                   10000000     Qt5Widgets:Qt5Widgets.dll
 0000:fffb5000       .debug$S                   10000000     Qt5Widgets:Qt5Widgets.dll
 0000:fffb5000       .debug$S                   10000000     Qt5Widgets:Qt5Widgets.dll
 0000:fffb5000       .debug$S                   10000000     Qt5Widgets:Qt5Widgets.dll
 0000:fffb5000       .debug$S                   10000000     Qt5Widgets:Qt5Widgets.dll
 0000:fffb5000       .debug$S                   10000000     Qt5Widgets:Qt5Widgets.dll
 0000:fffb5000       .debug$S                   10000000     Qt5Widgets:Qt5Widgets.dll
 0000:fffb5000       .debug$S                   10000000     Qt5Widgets:Qt5Widgets.dll
 0000:fffb5000       .debug$S                   10000000     Qt5Widgets:Qt5Widgets.dll
 0000:fffb5000       .debug$S                   10000000     Qt5Widgets:Qt5Widgets.dll
 0000:fffb5000       .debug$S                   10000000     Qt5Widgets:Qt5Widgets.dll
 0000:fffb5000       .debug$S                   10000000     Qt5Widgets:Qt5Widgets.dll
 0000:fffb5000       .debug$S                   10000000     Qt5Widgets:Qt5Widgets.dll
 0000:fffb5000       .debug$S                   10000000     Qt5Widgets:Qt5Widgets.dll
 0000:fffb5000       .debug$S                   10000000     Qt5Widgets:Qt5Widgets.dll
 0000:fffb5000       .debug$S                   10000000     Qt5Widgets:Qt5Widgets.dll
 0000:fffb5000       .debug$S                   10000000     Qt5Widgets:Qt5Widgets.dll
 0000:fffb5000       .debug$S                   10000000     Qt5Widgets:Qt5Widgets.dll
 0002:fffda000       ?_Generic_object$initializer$@?$_Error_objects@H@std@@2P6AXXZA 10000000     moc_ORFMarkerTests.obj
 0002:fffda000       ?_Iostream_object$initializer$@?$_Error_objects@H@std@@2P6AXXZA 10000000     moc_ORFMarkerTests.obj
 0002:fffda000       ?_System_object$initializer$@?$_Error_objects@H@std@@2P6AXXZA 10000000     moc_ORFMarkerTests.obj
 0000:fffb5000       .debug$S                   10000000     Qt5Widgets:Qt5Widgets.dll
 0000:fffb5000       .debug$S                   10000000     Qt5Widgets:Qt5Widgets.dll
 0000:fffb5000       .debug$S                   10000000     Qt5Widgets:Qt5Widgets.dll
 0000:fffb5000       .debug$S                   10000000     Qt5Widgets:Qt5Widgets.dll
 0000:fffb5000       .debug$S                   10000000     U2Core:U2Core.dll
 0000:fffb5000       .debug$S                   10000000     Qt5Widgets:Qt5Widgets.dll
 0002:fffda000       ?_System_object$initializer$@?$_Error_objects@H@std@@2P6AXXZA 10000000     ORFWorker.obj
 0000:fffb5000       .debug$S                   10000000     Qt5Widgets:Qt5Widgets.dll
 0002:fffda000       ?_Iostream_object$initializer$@?$_Error_objects@H@std@@2P6AXXZA 10000000     ORFWorker.obj
 0000:fffb5000       .debug$S                   10000000     Qt5Widgets:Qt5Widgets.dll
 0002:fffda000       ?_Generic_object$initializer$@?$_Error_objects@H@std@@2P6AXXZA 10000000     ORFWorker.obj
 0000:fffb5000       .debug$S                   10000000     Qt5Widgets:Qt5Widgets.dll
 0000:fffb5000       .debug$S                   10000000     U2Core:U2Core.dll
 0000:fffb5000       .debug$S                   10000000     Qt5Widgets:Qt5Widgets.dll
 0000:fffb5000       .debug$S                   10000000     U2Core:U2Core.dll
 0000:fffb5000       .debug$S                   10000000     Qt5Widgets:Qt5Widgets.dll
 0000:fffb5000       .debug$S                   10000000     U2Core:U2Core.dll
 0000:fffb5000       .debug$S                   10000000     Qt5Widgets:Qt5Widgets.dll
 0000:fffb5000       .debug$S                   10000000     U2Core:U2Core.dll
 0000:fffb5000       .debug$S                   10000000     Qt5Widgets:Qt5Widgets.dll
 0000:fffb5000       .debug$S                   10000000     U2Core:U2Core.dll
 0000:fffb5000       .debug$S                   10000000     Qt5Widgets:Qt5Widgets.dll
 0000:fffb5000       .debug$S                   10000000     U2Core:U2Core.dll
 0000:fffb5000       .debug$S                   10000000     U2Core:U2Core.dll
 0000:fffb5000       .debug$S                   10000000     U2Core:U2Core.dll
 0000:fffb5000       .debug$S                   10000000     Qt5Widgets:Qt5Widgets.dll
 0000:fffb5000       .debug$S                   10000000     U2Core:U2Core.dll
 0000:fffb5000       .debug$S                   10000000     Qt5Widgets:Qt5Widgets.dll
 0000:fffb5000       .debug$S                   10000000     U2Core:U2Core.dll
 0000:fffb5000       .debug$S                   10000000     Qt5Widgets:Qt5Widgets.dll
 0001:fffff000       __ehhandler$?_Copy@?$basic_string@DU?$char_traits@D@std@@V?$allocator@D@2@@std@@QAEXII@Z 10000000 f   moc_ORFMarkerTask.obj
 0000:fffb5000       .debug$S                   10000000     U2Core:U2Core.dll
 0000:fffb5000       .debug$S                   10000000     U2Core:U2Core.dll
 0000:fffb5000       .debug$S                   10000000     Qt5Widgets:Qt5Widgets.dll
 0000:fffb5000       .debug$S                   10000000     Qt5Widgets:Qt5Widgets.dll
 0000:fffb5000       .debug$S                   10000000     Qt5Widgets:Qt5Widgets.dll
 0000:fffb5000       .debug$S                   10000000     Qt5Widgets:Qt5Widgets.dll
 0000:fffb5000       .debug$S                   10000000     Qt5Widgets:Qt5Widgets.dll
 0000:fffb5000       .debug$S                   10000000     Qt5Widgets:Qt5Widgets.dll
 0000:fffb5000       .debug$S                   10000000     Qt5Widgets:Qt5Widgets.dll
 0000:fffb5000       .debug$S                   10000000     Qt5Widgets:Qt5Widgets.dll
 0000:fffb5000       .debug$S                   10000000     Qt5Widgets:Qt5Widgets.dll
 0000:fffb5000       .debug$S                   10000000     Qt5Widgets:Qt5Widgets.dll
 0000:fffb5000       .debug$S                   10000000     Qt5Widgets:Qt5Widgets.dll
 0000:fffb5000       .debug$S                   10000000     Qt5Widgets:Qt5Widgets.dll
 0000:fffb5000       .debug$S                   10000000     Qt5Widgets:Qt5Widgets.dll
 0000:fffb5000       .debug$S                   10000000     Qt5Widgets:Qt5Widgets.dll
 0000:fffb5000       .debug$S                   10000000     Qt5Widgets:Qt5Widgets.dll
 0000:fffb5000       .debug$S                   10000000     Qt5Widgets:Qt5Widgets.dll
 0000:fffb5000       .debug$S                   10000000     Qt5Widgets:Qt5Widgets.dll
 0000:fffb5000       .debug$S                   10000000     Qt5Widgets:Qt5Widgets.dll
 0000:fffb5000       .debug$S                   10000000     U2Core:U2Core.dll
 0000:fffb5000       .debug$S                   10000000     U2Core:U2Core.dll
 0000:fffb5000       .debug$S                   10000000     U2Core:U2Core.dll
 0000:fffb5000       .debug$S                   10000000     U2Core:U2Core.dll
 0002:fffda000       __catchsym$?_Copy@?$basic_string@DU?$char_traits@D@std@@V?$allocator@D@2@@std@@QAEXII@Z$5 10000000     moc_ORFMarkerTask.obj
 0000:fffb5000       .debug$S                   10000000     Qt5Widgets:Qt5Widgets.dll
 0000:fffb5000       .debug$S                   10000000     Qt5Widgets:Qt5Widgets.dll
 0000:fffb5000       .debug$S                   10000000     Qt5Widgets:Qt5Widgets.dll
 0000:fffb5000       .debug$S                   10000000     Qt5Widgets:Qt5Widgets.dll
 0000:fffb5000       .debug$S                   10000000     Qt5Widgets:Qt5Widgets.dll
 0000:fffb5000       .debug$S                   10000000     Qt5Widgets:Qt5Widgets.dll
 0000:fffb5000       .debug$S                   10000000     Qt5Widgets:Qt5Widgets.dll
 0000:fffb5000       .debug$S                   10000000     Qt5Widgets:Qt5Widgets.dll
 0000:fffb5000       .debug$S                   10000000     Qt5Widgets:Qt5Widgets.dll
 0000:fffb5000       .debug$S                   10000000     Qt5Widgets:Qt5Widgets.dll
 0000:fffb5000       .debug$S                   10000000     Qt5Widgets:Qt5Widgets.dll
 0000:fffb5000       .debug$S                   10000000     Qt5Widgets:Qt5Widgets.dll
 0000:fffb5000       .debug$S                   10000000     Qt5Widgets:Qt5Widgets.dll
 0000:fffb5000       .debug$S                   10000000     Qt5Widgets:Qt5Widgets.dll
 0000:fffb5000       .debug$S                   10000000     Qt5Widgets:Qt5Widgets.dll
 0000:fffb5000       .debug$S                   10000000     Qt5Widgets:Qt5Widgets.dll
 0000:fffb5000       .debug$S                   10000000     Qt5Widgets:Qt5Widgets.dll
 0000:fffb5000       .debug$S                   10000000     Qt5Widgets:Qt5Widgets.dll
 0000:fffb5000       .debug$S                   10000000     Qt5Widgets:Qt5Widgets.dll
 0000:fffb5000       .debug$S                   10000000     Qt5Widgets:Qt5Widgets.dll
 0000:fffb5000       .debug$S                   10000000     Qt5Widgets:Qt5Widgets.dll
 0000:fffb5000       .debug$S                   10000000     Qt5Widgets:Qt5Widgets.dll
 0000:fffb5000       .debug$S                   10000000     Qt5Widgets:Qt5Widgets.dll
 0000:fffb5000       .debug$S                   10000000     Qt5Widgets:Qt5Widgets.dll
 0000:fffb5000       .debug$S                   10000000     Qt5Widgets:Qt5Widgets.dll
 0000:fffb5000       .debug$S                   10000000     Qt5Widgets:Qt5Widgets.dll
 0000:fffb5000       .debug$S                   10000000     Qt5Widgets:Qt5Widgets.dll
 0000:fffb5000       .debug$S                   10000000     Qt5Widgets:Qt5Widgets.dll
 0000:fffb5000       .debug$S                   10000000     Qt5Widgets:Qt5Widgets.dll
 0000:fffb5000       .debug$S                   10000000     Qt5Widgets:Qt5Widgets.dll
 0000:fffb5000       .debug$S                   10000000     Qt5Widgets:Qt5Widgets.dll
 0000:fffb5000       .debug$S                   10000000     Qt5Widgets:Qt5Widgets.dll
 0000:fffb5000       .debug$S                   10000000     Qt5Widgets:Qt5Widgets.dll
 0000:fffb5000       .debug$S                   10000000     Qt5Widgets:Qt5Widgets.dll
 0000:fffb5000       .debug$S                   10000000     Qt5Widgets:Qt5Widgets.dll
 0000:fffb5000       .debug$S                   10000000     Qt5Widgets:Qt5Widgets.dll
 0000:fffb5000       .debug$S                   10000000     Qt5Widgets:Qt5Widgets.dll
 0000:fffb5000       .debug$S                   10000000     Qt5Widgets:Qt5Widgets.dll
 0000:fffb5000       .debug$S                   10000000     Qt5Widgets:Qt5Widgets.dll
 0000:fffb5000       .debug$S                   10000000     Qt5Widgets:Qt5Widgets.dll
 0000:fffb5000       .debug$S                   10000000     Qt5Widgets:Qt5Widgets.dll
 0000:fffb5000       .debug$S                   10000000     Qt5Widgets:Qt5Widgets.dll
 0002:fffda000       ?_Generic_object$initializer$@?$_Error_objects@H@std@@2P6AXXZA 10000000     moc_ORFMarkerTask.obj
 0002:fffda000       ?_Iostream_object$initializer$@?$_Error_objects@H@std@@2P6AXXZA 10000000     moc_ORFMarkerTask.obj
 0002:fffda000       ?_System_object$initializer$@?$_Error_objects@H@std@@2P6AXXZA 10000000     moc_ORFMarkerTask.obj
 0000:fffb5000       .debug$S                   10000000     Qt5Widgets:Qt5Widgets.dll
 0000:fffb5000       .debug$S                   10000000     Qt5Widgets:Qt5Widgets.dll
 0000:fffb5000       .debug$S                   10000000     Qt5Widgets:Qt5Widgets.dll
 0000:fffb5000       .debug$S                   10000000     Qt5Widgets:Qt5Widgets.dll
 0000:fffb5000       .debug$S                   10000000     U2Core:U2Core.dll
 0000:fffb5000       .debug$S                   10000000     Qt5Widgets:Qt5Widgets.dll
 0000:fffb5000       .debug$S                   10000000     U2Core:U2Core.dll
 0000:fffb5000       .debug$S                   10000000     Qt5Widgets:Qt5Widgets.dll
 0000:fffb5000       .debug$S                   10000000     U2Core:U2Core.dll
 0000:fffb5000       .debug$S                   10000000     Qt5Widgets:Qt5Widgets.dll
 0000:fffb5000       .debug$S                   10000000     U2Core:U2Core.dll
 0000:fffb5000       .debug$S                   10000000     Qt5Widgets:Qt5Widgets.dll
 0000:fffb5000       .debug$S                   10000000     U2Core:U2Core.dll
 0000:fffb5000       .debug$S                   10000000     Qt5Widgets:Qt5Widgets.dll
 0000:fffb5000       .debug$S                   10000000     U2Core:U2Core.dll
 0000:fffb5000       .debug$S                   10000000     Qt5Widgets:Qt5Widgets.dll
 0000:fffb5000       .debug$S                   10000000     U2Core:U2Core.dll
 0000:fffb5000       .debug$S                   10000000     Qt5Widgets:Qt5Widgets.dll
 0000:fffb5000       .debug$S                   10000000     U2Core:U2Core.dll
 0000:fffb5000       .debug$S                   10000000     Qt5Widgets:Qt5Widgets.dll
 0000:fffb5000       .debug$S                   10000000     U2Core:U2Core.dll
 0000:fffb5000       .debug$S                   10000000     Qt5Widgets:Qt5Widgets.dll
 0000:fffb5000       .debug$S                   10000000     U2Core:U2Core.dll
 0000:fffb5000       .debug$S                   10000000     Qt5Widgets:Qt5Widgets.dll
 0000:fffb5000       .debug$S                   10000000     U2Core:U2Core.dll
 0000:fffb5000       .debug$S                   10000000     Qt5Widgets:Qt5Widgets.dll
 0000:fffb5000       .debug$S                   10000000     U2Core:U2Core.dll
 0000:fffb5000       .debug$S                   10000000     Qt5Widgets:Qt5Widgets.dll
 0000:fffb5000       .debug$S                   10000000     U2Core:U2Core.dll
 0000:fffb5000       .debug$S                   10000000     Qt5Widgets:Qt5Widgets.dll
 0000:fffb5000       .debug$S                   10000000     U2Core:U2Core.dll
 0000:fffb5000       .debug$S                   10000000     U2Core:U2Core.dll
 0000:fffb5000       .debug$S                   10000000     U2Core:U2Core.dll
 0000:fffb5000       .debug$S                   10000000     Qt5Widgets:Qt5Widgets.dll
 0000:fffb5000       .debug$S                   10000000     U2Core:U2Core.dll
 0000:fffb5000       .debug$S                   10000000     Qt5Widgets:Qt5Widgets.dll
 0000:fffb5000       .debug$S                   10000000     U2Core:U2Core.dll
 0000:fffb5000       .debug$S                   10000000     Qt5Widgets:Qt5Widgets.dll
 0001:fffff000       __ehhandler$?_Copy@?$basic_string@DU?$char_traits@D@std@@V?$allocator@D@2@@std@@QAEXII@Z 10000000 f   moc_ORFMarkerPlugin.obj
 0000:fffb5000       .debug$S                   10000000     U2Core:U2Core.dll
 0000:fffb5000       .debug$S                   10000000     U2Core:U2Core.dll
 0000:fffb5000       .debug$S                   10000000     U2Core:U2Core.dll
 0000:fffb5000       .debug$S                   10000000     U2Core:U2Core.dll
 0000:fffb5000       .debug$S                   10000000     U2Core:U2Core.dll
 0000:fffb5000       .debug$S                   10000000     U2Core:U2Core.dll
 0002:fffda000       __catchsym$?_Copy@?$basic_string@DU?$char_traits@D@std@@V?$allocator@D@2@@std@@QAEXII@Z$5 10000000     moc_ORFMarkerPlugin.obj
 0000:fffb5000       .debug$S                   10000000     Qt5Widgets:Qt5Widgets.dll
 0000:fffb5000       .debug$S                   10000000     Qt5Widgets:Qt5Widgets.dll
 0000:fffb5000       .debug$S                   10000000     Qt5Widgets:Qt5Widgets.dll
 0000:fffb5000       .debug$S                   10000000     Qt5Widgets:Qt5Widgets.dll
 0000:fffb5000       .debug$S                   10000000     Qt5Widgets:Qt5Widgets.dll
 0000:fffb5000       .debug$S                   10000000     Qt5Widgets:Qt5Widgets.dll
 0000:fffb5000       .debug$S                   10000000     Qt5Widgets:Qt5Widgets.dll
 0000:fffb5000       .debug$S                   10000000     Qt5Widgets:Qt5Widgets.dll
 0000:fffb5000       .debug$S                   10000000     Qt5Widgets:Qt5Widgets.dll
 0000:fffb5000       .debug$S                   10000000     Qt5Widgets:Qt5Widgets.dll
 0000:fffb5000       .debug$S                   10000000     Qt5Widgets:Qt5Widgets.dll
 0000:fffb5000       .debug$S                   10000000     Qt5Widgets:Qt5Widgets.dll
 0000:fffb5000       .debug$S                   10000000     Qt5Widgets:Qt5Widgets.dll
 0000:fffb5000       .debug$S                   10000000     Qt5Widgets:Qt5Widgets.dll
 0000:fffb5000       .debug$S                   10000000     Qt5Widgets:Qt5Widgets.dll
 0000:fffb5000       .debug$S                   10000000     Qt5Widgets:Qt5Widgets.dll
 0000:fffb5000       .debug$S                   10000000     Qt5Widgets:Qt5Widgets.dll
 0000:fffb5000       .debug$S                   10000000     Qt5Widgets:Qt5Widgets.dll
 0000:fffb5000       .debug$S                   10000000     Qt5Widgets:Qt5Widgets.dll
 0000:fffb5000       .debug$S                   10000000     Qt5Widgets:Qt5Widgets.dll
 0000:fffb5000       .debug$S                   10000000     Qt5Widgets:Qt5Widgets.dll
 0000:fffb5000       .debug$S                   10000000     Qt5Widgets:Qt5Widgets.dll
 0000:fffb5000       .debug$S                   10000000     Qt5Widgets:Qt5Widgets.dll
 0000:fffb5000       .debug$S                   10000000     Qt5Widgets:Qt5Widgets.dll
 0000:fffb5000       .debug$S                   10000000     Qt5Widgets:Qt5Widgets.dll
 0000:fffb5000       .debug$S                   10000000     Qt5Widgets:Qt5Widgets.dll
 0000:fffb5000       .debug$S                   10000000     Qt5Widgets:Qt5Widgets.dll
 0000:fffb5000       .debug$S                   10000000     Qt5Widgets:Qt5Widgets.dll
 0000:fffb5000       .debug$S                   10000000     Qt5Widgets:Qt5Widgets.dll
 0000:fffb5000       .debug$S                   10000000     Qt5Widgets:Qt5Widgets.dll
 0000:fffb5000       .debug$S                   10000000     Qt5Widgets:Qt5Widgets.dll
 0000:fffb5000       .debug$S                   10000000     Qt5Widgets:Qt5Widgets.dll
 0002:fffda000       ?_Generic_object$initializer$@?$_Error_objects@H@std@@2P6AXXZA 10000000     moc_ORFMarkerPlugin.obj
 0002:fffda000       ?_Iostream_object$initializer$@?$_Error_objects@H@std@@2P6AXXZA 10000000     moc_ORFMarkerPlugin.obj
 0002:fffda000       ?_System_object$initializer$@?$_Error_objects@H@std@@2P6AXXZA 10000000     moc_ORFMarkerPlugin.obj
 0000:fffb5000       .debug$S                   10000000     Qt5Widgets:Qt5Widgets.dll
 0000:fffb5000       .debug$S                   10000000     Qt5Widgets:Qt5Widgets.dll
 0000:fffb5000       .debug$S                   10000000     U2Core:U2Core.dll
 0000:fffb5000       .debug$S                   10000000     Qt5Widgets:Qt5Widgets.dll
 0000:fffb5000       .debug$S                   10000000     U2Core:U2Core.dll
 0000:fffb5000       .debug$S                   10000000     Qt5Widgets:Qt5Widgets.dll
 0000:fffb5000       .debug$S                   10000000     U2Core:U2Core.dll
 0000:fffb5000       .debug$S                   10000000     Qt5Widgets:Qt5Widgets.dll
 0002:fffda000       __unwindtable$?metaType@?$QVariantValueHelper@VQString@@@QtPrivate@@SA?AVQString@@ABVQVariant@@@Z 10000000     ORFWorker.obj
 0000:fffb5000       .debug$S                   10000000     Qt5Widgets:Qt5Widgets.dll
 0002:fffda000       __catchsym$?createNode@?$QMapData@VQString@@PAVPropertyDelegate@U2@@@@QAEPAU?$QMapNode@VQString@@PAVPropertyDelegate@U2@@@@ABVQString@@ABQAVPropertyDelegate@U2@@PAU2@_N@Z$5 10000000     ORFWorker.obj
 0000:fffb5000       .debug$S                   10000000     Qt5Widgets:Qt5Widgets.dll
 0000:fffb5000       .debug$S                   10000000     U2Core:U2Core.dll
 0000:fffb5000       .debug$S                   10000000     Qt5Widgets:Qt5Widgets.dll
 0000:fffb5000       .debug$S                   10000000     U2Core:U2Core.dll
 0000:fffb5000       .debug$S                   10000000     Qt5Widgets:Qt5Widgets.dll
 0000:fffb5000       .debug$S                   10000000     U2Core:U2Core.dll
 0000:fffb5000       .debug$S                   10000000     Qt5Widgets:Qt5Widgets.dll
 0000:fffb5000       .debug$S                   10000000     U2Core:U2Core.dll
 0000:fffb5000       .debug$S                   10000000     Qt5Widgets:Qt5Widgets.dll
 0000:fffb5000       .debug$S                   10000000     U2Core:U2Core.dll
 0000:fffb5000       .debug$S                   10000000     U2Core:U2Core.dll
 0000:fffb5000       .debug$S                   10000000     Qt5Widgets:Qt5Widgets.dll
 0000:fffb5000       .debug$S                   10000000     U2Core:U2Core.dll
 0000:fffb5000       .debug$S                   10000000     Qt5Widgets:Qt5Widgets.dll
 0000:fffb5000       .debug$S                   10000000     U2Core:U2Core.dll
 0000:fffb5000       .debug$S                   10000000     Qt5Widgets:Qt5Widgets.dll
 0001:fffff000       __ehhandler$?_Copy@?$basic_string@DU?$char_traits@D@std@@V?$allocator@D@2@@std@@QAEXII@Z 10000000 f   moc_ORFDialog.obj
 0000:fffb5000       .debug$S                   10000000     U2Core:U2Core.dll
 0000:fffb5000       .debug$S                   10000000     U2Core:U2Core.dll
 0000:fffb5000       .debug$S                   10000000     Qt5Widgets:Qt5Widgets.dll
 0000:fffb5000       .debug$S                   10000000     Qt5Widgets:Qt5Widgets.dll
 0000:fffb5000       .debug$S                   10000000     Qt5Widgets:Qt5Widgets.dll
 0000:fffb5000       .debug$S                   10000000     Qt5Widgets:Qt5Widgets.dll
 0000:fffb5000       .debug$S                   10000000     Qt5Widgets:Qt5Widgets.dll
 0000:fffb5000       .debug$S                   10000000     Qt5Widgets:Qt5Widgets.dll
 0000:fffb5000       .debug$S                   10000000     Qt5Widgets:Qt5Widgets.dll
 0000:fffb5000       .debug$S                   10000000     Qt5Widgets:Qt5Widgets.dll
 0000:fffb5000       .debug$S                   10000000     Qt5Widgets:Qt5Widgets.dll
 0000:fffb5000       .debug$S                   10000000     Qt5Widgets:Qt5Widgets.dll
 0000:fffb5000       .debug$S                   10000000     Qt5Widgets:Qt5Widgets.dll
 0000:fffb5000       .debug$S                   10000000     Qt5Widgets:Qt5Widgets.dll
 0000:fffb5000       .debug$S                   10000000     Qt5Widgets:Qt5Widgets.dll
 0000:fffb5000       .debug$S                   10000000     Qt5Widgets:Qt5Widgets.dll
 0000:fffb5000       .debug$S                   10000000     Qt5Widgets:Qt5Widgets.dll
 0000:fffb5000       .debug$S                   10000000     Qt5Widgets:Qt5Widgets.dll
 0000:fffb5000       .debug$S                   10000000     Qt5Widgets:Qt5Widgets.dll
 0000:fffb5000       .debug$S                   10000000     Qt5Widgets:Qt5Widgets.dll
 0000:fffb5000       .debug$S                   10000000     U2Core:U2Core.dll
 0000:fffb5000       .debug$S                   10000000     Qt5Widgets:Qt5Widgets.dll
 0000:fffb5000       .debug$S                   10000000     Qt5Widgets:Qt5Widgets.dll
 0000:fffb5000       .debug$S                   10000000     U2Core:U2Core.dll
 0000:fffb5000       .debug$S                   10000000     U2Core:U2Core.dll
 0002:fffda000       __catchsym$?createNode@?$QMapData@VQString@@VQVariant@@@@QAEPAU?$QMapNode@VQString@@VQVariant@@@@ABVQString@@ABVQVariant@@PAU2@_N@Z$7 10000000     ORFWorker.obj
 0000:fffb5000       .debug$S                   10000000     U2Core:U2Core.dll
 0002:fffda000       __catchsym$?_Copy@?$basic_string@DU?$char_traits@D@std@@V?$allocator@D@2@@std@@QAEXII@Z$5 10000000     moc_ORFDialog.obj
 0000:fffb5000       .debug$S                   10000000     Qt5Widgets:Qt5Widgets.dll
 0000:fffb5000       .debug$S                   10000000     Qt5Widgets:Qt5Widgets.dll
 0000:fffb5000       .debug$S                   10000000     Qt5Widgets:Qt5Widgets.dll
 0000:fffb5000       .debug$S                   10000000     Qt5Widgets:Qt5Widgets.dll
 0000:fffb5000       .debug$S                   10000000     Qt5Widgets:Qt5Widgets.dll
 0000:fffb5000       .debug$S                   10000000     Qt5Widgets:Qt5Widgets.dll
 0000:fffb5000       .debug$S                   10000000     Qt5Widgets:Qt5Widgets.dll
 0000:fffb5000       .debug$S                   10000000     Qt5Widgets:Qt5Widgets.dll
 0000:fffb5000       .debug$S                   10000000     Qt5Widgets:Qt5Widgets.dll
 0000:fffb5000       .debug$S                   10000000     Qt5Widgets:Qt5Widgets.dll
 0000:fffb5000       .debug$S                   10000000     Qt5Widgets:Qt5Widgets.dll
 0000:fffb5000       .debug$S                   10000000     Qt5Widgets:Qt5Widgets.dll
 0000:fffb5000       .debug$S                   10000000     Qt5Widgets:Qt5Widgets.dll
 0000:fffb5000       .debug$S                   10000000     Qt5Widgets:Qt5Widgets.dll
 0000:fffb5000       .debug$S                   10000000     Qt5Widgets:Qt5Widgets.dll
 0000:fffb5000       .debug$S                   10000000     Qt5Widgets:Qt5Widgets.dll
 0000:fffb5000       .debug$S                   10000000     Qt5Widgets:Qt5Widgets.dll
 0000:fffb5000       .debug$S                   10000000     Qt5Widgets:Qt5Widgets.dll
 0000:fffb5000       .debug$S                   10000000     Qt5Widgets:Qt5Widgets.dll
 0000:fffb5000       .debug$S                   10000000     Qt5Widgets:Qt5Widgets.dll
 0000:fffb5000       .debug$S                   10000000     Qt5Widgets:Qt5Widgets.dll
 0000:fffb5000       .debug$S                   10000000     Qt5Widgets:Qt5Widgets.dll
 0000:fffb5000       .debug$S                   10000000     Qt5Widgets:Qt5Widgets.dll
 0000:fffb5000       .debug$S                   10000000     Qt5Widgets:Qt5Widgets.dll
 0000:fffb5000       .debug$S                   10000000     Qt5Widgets:Qt5Widgets.dll
 0000:fffb5000       .debug$S                   10000000     Qt5Widgets:Qt5Widgets.dll
 0000:fffb5000       .debug$S                   10000000     Qt5Widgets:Qt5Widgets.dll
 0000:fffb5000       .debug$S                   10000000     Qt5Widgets:Qt5Widgets.dll
 0000:fffb5000       .debug$S                   10000000     Qt5Widgets:Qt5Widgets.dll
 0000:fffb5000       .debug$S                   10000000     Qt5Widgets:Qt5Widgets.dll
 0000:fffb5000       .debug$S                   10000000     Qt5Widgets:Qt5Widgets.dll
 0000:fffb5000       .debug$S                   10000000     Qt5Widgets:Qt5Widgets.dll
 0000:fffb5000       .debug$S                   10000000     Qt5Widgets:Qt5Widgets.dll
 0000:fffb5000       .debug$S                   10000000     Qt5Widgets:Qt5Widgets.dll
 0000:fffb5000       .debug$S                   10000000     Qt5Widgets:Qt5Widgets.dll
 0000:fffb5000       .debug$S                   10000000     Qt5Widgets:Qt5Widgets.dll
 0000:fffb5000       .debug$S                   10000000     Qt5Widgets:Qt5Widgets.dll
 0000:fffb5000       .debug$S                   10000000     Qt5Widgets:Qt5Widgets.dll
 0000:fffb5000       .debug$S                   10000000     Qt5Widgets:Qt5Widgets.dll
 0000:fffb5000       .debug$S                   10000000     Qt5Widgets:Qt5Widgets.dll
 0000:fffb5000       .debug$S                   10000000     Qt5Widgets:Qt5Widgets.dll
 0000:fffb5000       .debug$S                   10000000     Qt5Widgets:Qt5Widgets.dll
 0000:fffb5000       .debug$S                   10000000     Qt5Widgets:Qt5Widgets.dll
 0002:fffda000       ?_Generic_object$initializer$@?$_Error_objects@H@std@@2P6AXXZA 10000000     moc_ORFDialog.obj
 0002:fffda000       ?_Iostream_object$initializer$@?$_Error_objects@H@std@@2P6AXXZA 10000000     moc_ORFDialog.obj
 0002:fffda000       ?_System_object$initializer$@?$_Error_objects@H@std@@2P6AXXZA 10000000     moc_ORFDialog.obj
 0000:fffb5000       .debug$S                   10000000     U2Core:U2Core.dll
 0000:fffb5000       .debug$S                   10000000     Qt5Widgets:Qt5Widgets.dll
 0000:fffb5000       .debug$S                   10000000     U2Core:U2Core.dll
 0000:fffb5000       .debug$S                   10000000     Qt5Widgets:Qt5Widgets.dll
 0000:fffb5000       .debug$S                   10000000     U2Core:U2Core.dll
 0000:fffb5000       .debug$S                   10000000     Qt5Widgets:Qt5Widgets.dll
 0000:fffb5000       .debug$S                   10000000     U2Core:U2Core.dll
 0000:fffb5000       .debug$S                   10000000     Qt5Widgets:Qt5Widgets.dll
 0000:fffb5000       .debug$S                   10000000     U2Core:U2Core.dll
 0000:fffb5000       .debug$S                   10000000     Qt5Widgets:Qt5Widgets.dll
 0000:fffb5000       .debug$S                   10000000     U2Core:U2Core.dll
 0000:fffb5000       .debug$S                   10000000     Qt5Widgets:Qt5Widgets.dll
 0000:fffb5000       .debug$S                   10000000     U2Core:U2Core.dll
 0000:fffb5000       .debug$S                   10000000     Qt5Widgets:Qt5Widgets.dll
 0000:fffb5000       .debug$S                   10000000     U2Core:U2Core.dll
 0000:fffb5000       .debug$S                   10000000     Qt5Widgets:Qt5Widgets.dll
 0000:fffb5000       .debug$S                   10000000     U2Core:U2Core.dll
 0000:fffb5000       .debug$S                   10000000     Qt5Widgets:Qt5Widgets.dll
 0000:fffb5000       .debug$S                   10000000     U2Core:U2Core.dll
 0000:fffb5000       .debug$S                   10000000     Qt5Widgets:Qt5Widgets.dll
 0000:fffb5000       .debug$S                   10000000     U2Core:U2Core.dll
 0000:fffb5000       .debug$S                   10000000     Qt5Widgets:Qt5Widgets.dll
 0002:fffda000       __catchsym$??0?$QList@PAVDNATranslation@U2@@@@QAE@ABV0@@Z$2 10000000     ORFWorker.obj
 0000:fffb5000       .debug$S                   10000000     Qt5Widgets:Qt5Widgets.dll
 0000:fffb5000       .debug$S                   10000000     U2Core:U2Core.dll
 0000:fffb5000       .debug$S                   10000000     Qt5Widgets:Qt5Widgets.dll
 0000:fffb5000       .debug$S                   10000000     U2Algorithm:U2Algorithm.dll
 0000:fffb5000       .debug$S                   10000000     Qt5Widgets:Qt5Widgets.dll
 0000:fffb5000       .debug$S                   10000000     U2Algorithm:U2Algorithm.dll
 0000:fffb5000       .debug$S                   10000000     Qt5Widgets:Qt5Widgets.dll
 0000:fffb5000       .debug$S                   10000000     U2Algorithm:U2Algorithm.dll
 0000:fffb5000       .debug$S                   10000000     Qt5Widgets:Qt5Widgets.dll
 0000:fffb5000       .debug$S                   10000000     U2Algorithm:U2Algorithm.dll
 0000:fffb5000       .debug$S                   10000000     Qt5Widgets:Qt5Widgets.dll
 0000:fffb5000       .debug$S                   10000000     U2Algorithm:U2Algorithm.dll
 0000:fffb5000       .debug$S                   10000000     Qt5Widgets:Qt5Widgets.dll
 0000:fffb5000       .debug$S                   10000000     U2Algorithm:U2Algorithm.dll
 0000:fffb5000       .debug$S                   10000000     Qt5Widgets:Qt5Widgets.dll
 0000:fffb5000       .debug$S                   10000000     U2Algorithm:U2Algorithm.dll
 0000:fffb5000       .debug$S                   10000000     U2Algorithm:U2Algorithm.dll
 0000:fffb5000       .debug$S                   10000000     Qt5Widgets:Qt5Widgets.dll
 0000:fffb5000       .debug$S                   10000000     U2Algorithm:U2Algorithm.dll
 0000:fffb5000       .debug$S                   10000000     Qt5Widgets:Qt5Widgets.dll
 0000:fffb5000       .debug$S                   10000000     U2Algorithm:U2Algorithm.dll
 0000:fffb5000       .debug$S                   10000000     Qt5Widgets:Qt5Widgets.dll
 0001:fffff000       __ehhandler$?_Copy@?$basic_string@DU?$char_traits@D@std@@V?$allocator@D@2@@std@@QAEXII@Z 10000000 f   ORFWorker.obj
 0000:fffb5000       .debug$S                   10000000     U2Algorithm:U2Algorithm.dll
 0000:fffb5000       .debug$S                   10000000     U2Algorithm:U2Algorithm.dll
 0000:fffb5000       .debug$S                   10000000     U2Algorithm:U2Algorithm.dll
 0001:fffff000       __unwindfunclet$??H@YA?BVQString@@ABV0@PBD@Z$0 10000000 f   ORFWorker.obj
 0000:fffb5000       .debug$S                   10000000     U2Algorithm:U2Algorithm.dll
 0000:fffb5000       .debug$S                   10000000     U2Algorithm:U2Algorithm.dll
 0001:fffff000       __unwindfunclet$??H@YA?BVQString@@PBDABV0@@Z$0 10000000 f   ORFWorker.obj
 0000:fffb5000       .debug$S                   10000000     U2Gui:U2Gui.dll
 0001:fffff000       __unwindfunclet$??A?$QMap@VQString@@VQVariant@@@@QAEAAVQVariant@@ABVQString@@@Z$0 10000000 f   ORFWorker.obj
 0000:fffb5000       .debug$S                   10000000     Qt5Widgets:Qt5Widgets.dll
 0000:fffb5000       .debug$S                   10000000     Qt5Widgets:Qt5Widgets.dll
 0000:fffb5000       .debug$S                   10000000     Qt5Widgets:Qt5Widgets.dll
 0000:fffb5000       .debug$S                   10000000     Qt5Widgets:Qt5Widgets.dll
 0000:fffb5000       .debug$S                   10000000     Qt5Widgets:Qt5Widgets.dll
 0000:fffb5000       .debug$S                   10000000     Qt5Widgets:Qt5Widgets.dll
 0000:fffb5000       .debug$S                   10000000     Qt5Widgets:Qt5Widgets.dll
 0000:fffb5000       .debug$S                   10000000     Qt5Widgets:Qt5Widgets.dll
 0000:fffb5000       .debug$S                   10000000     Qt5Widgets:Qt5Widgets.dll
 0000:fffb5000       .debug$S                   10000000     Qt5Widgets:Qt5Widgets.dll
 0000:fffb5000       .debug$S                   10000000     Qt5Widgets:Qt5Widgets.dll
 0000:fffb5000       .debug$S                   10000000     Qt5Widgets:Qt5Widgets.dll
 0000:fffb5000       .debug$S                   10000000     Qt5Widgets:Qt5Widgets.dll
 0000:fffb5000       .debug$S                   10000000     Qt5Widgets:Qt5Widgets.dll
 0000:fffb5000       .debug$S                   10000000     Qt5Widgets:Qt5Widgets.dll
 0000:fffb5000       .debug$S                   10000000     Qt5Widgets:Qt5Widgets.dll
 0000:fffb5000       .debug$S                   10000000     Qt5Widgets:Qt5Widgets.dll
 0000:fffb5000       .debug$S                   10000000     Qt5Widgets:Qt5Widgets.dll
 0000:fffb5000       .debug$S                   10000000     Qt5Widgets:Qt5Widgets.dll
 0000:fffb5000       .debug$S                   10000000     Qt5Widgets:Qt5Widgets.dll
 0000:fffb5000       .debug$S                   10000000     Qt5Widgets:Qt5Widgets.dll
 0000:fffb5000       .debug$S                   10000000     U2Gui:U2Gui.dll
 0000:fffb5000       .debug$S                   10000000     Qt5Widgets:Qt5Widgets.dll
 0000:fffb5000       .debug$S                   10000000     U2Gui:U2Gui.dll
 0000:fffb5000       .debug$S                   10000000     Qt5Widgets:Qt5Widgets.dll
 0000:fffb5000       .debug$S                   10000000     U2Gui:U2Gui.dll
 0000:fffb5000       .debug$S                   10000000     Qt5Widgets:Qt5Widgets.dll
 0000:fffb5000       .debug$S                   10000000     U2Gui:U2Gui.dll
 0000:fffb5000       .debug$S                   10000000     U2Gui:U2Gui.dll
 0000:fffb5000       .debug$S                   10000000     Qt5Widgets:Qt5Widgets.dll
 0000:fffb5000       .debug$S                   10000000     U2Gui:U2Gui.dll
 0000:fffb5000       .debug$S                   10000000     Qt5Widgets:Qt5Widgets.dll
 0000:fffb5000       .debug$S                   10000000     Qt5Widgets:Qt5Widgets.dll
 0000:fffb5000       .debug$S                   10000000     Qt5Widgets:Qt5Widgets.dll
 0000:fffb5000       .debug$S                   10000000     U2Gui:U2Gui.dll
 0000:fffb5000       .debug$S                   10000000     Qt5Widgets:Qt5Widgets.dll
 0000:fffb5000       .debug$S                   10000000     Qt5Widgets:Qt5Widgets.dll
 0000:fffb5000       .debug$S                   10000000     Qt5Widgets:Qt5Widgets.dll
 0000:fffb5000       .debug$S                   10000000     Qt5Widgets:Qt5Widgets.dll
 0000:fffb5000       .debug$S                   10000000     Qt5Widgets:Qt5Widgets.dll
 0000:fffb5000       .debug$S                   10000000     Qt5Widgets:Qt5Widgets.dll
 0000:fffb5000       .debug$S                   10000000     Qt5Widgets:Qt5Widgets.dll
 0000:fffb5000       .debug$S                   10000000     Qt5Widgets:Qt5Widgets.dll
 0000:fffb5000       .debug$S                   10000000     Qt5Widgets:Qt5Widgets.dll
 0000:fffb5000       .debug$S                   10000000     Qt5Widgets:Qt5Widgets.dll
 0000:fffb5000       .debug$S                   10000000     Qt5Widgets:Qt5Widgets.dll
 0000:fffb5000       .debug$S                   10000000     Qt5Widgets:Qt5Widgets.dll
 0000:fffb5000       .debug$S                   10000000     Qt5Widgets:Qt5Widgets.dll
 0000:fffb5000       .debug$S                   10000000     Qt5Widgets:Qt5Widgets.dll
 0000:fffb5000       .debug$S                   10000000     Qt5Widgets:Qt5Widgets.dll
 0000:fffb5000       .debug$S                   10000000     Qt5Widgets:Qt5Widgets.dll
 0000:fffb5000       .debug$S                   10000000     Qt5Widgets:Qt5Widgets.dll
 0000:fffb5000       .debug$S                   10000000     Qt5Widgets:Qt5Widgets.dll
 0000:fffb5000       .debug$S                   10000000     Qt5Widgets:Qt5Widgets.dll
 0000:fffb5000       .debug$S                   10000000     Qt5Widgets:Qt5Widgets.dll
 0000:fffb5000       .debug$S                   10000000     Qt5Widgets:Qt5Widgets.dll
 0000:fffb5000       .debug$S                   10000000     Qt5Widgets:Qt5Widgets.dll
 0000:fffb5000       .debug$S                   10000000     Qt5Widgets:Qt5Widgets.dll
 0000:fffb5000       .debug$S                   10000000     Qt5Widgets:Qt5Widgets.dll
 0000:fffb5000       .debug$S                   10000000     Qt5Widgets:Qt5Widgets.dll
 0000:fffb5000       .debug$S                   10000000     Qt5Widgets:Qt5Widgets.dll
 0000:fffb5000       .debug$S                   10000000     Qt5Widgets:Qt5Widgets.dll
 0000:fffb5000       .debug$S                   10000000     Qt5Widgets:Qt5Widgets.dll
 0000:fffb5000       .debug$S                   10000000     Qt5Widgets:Qt5Widgets.dll
 0000:fffb5000       .debug$S                   10000000     Qt5Widgets:Qt5Widgets.dll
 0000:fffb5000       .debug$S                   10000000     Qt5Widgets:Qt5Widgets.dll
 0000:fffb5000       .debug$S                   10000000     Qt5Widgets:Qt5Widgets.dll
 0000:fffb5000       .debug$S                   10000000     Qt5Widgets:Qt5Widgets.dll
 0000:fffb5000       .debug$S                   10000000     Qt5Widgets:Qt5Widgets.dll
 0000:fffb5000       .debug$S                   10000000     Qt5Widgets:Qt5Widgets.dll
 0000:fffb5000       .debug$S                   10000000     Qt5Widgets:Qt5Widgets.dll
 0001:fffff000       __ehhandler$?append@?$QList@PAVAttribute@U2@@@@QAEXABQAVAttribute@U2@@@Z 10000000 f   ORFWorker.obj
 0000:fffb5000       .debug$S                   10000000     U2Gui:U2Gui.dll
 0001:fffff000       __ehhandler$?detach_helper_grow@?$QList@PAVAttribute@U2@@@@AAEPAUNode@1@HH@Z 10000000 f   ORFWorker.obj
 0000:fffb5000       .debug$S                   10000000     U2Gui:U2Gui.dll
 0000:fffb5000       .debug$S                   10000000     U2Gui:U2Gui.dll
 0000:fffb5000       .debug$S                   10000000     Qt5Widgets:Qt5Widgets.dll
 0000:fffb5000       .debug$S                   10000000     U2Gui:U2Gui.dll
 0000:fffb5000       .debug$S                   10000000     Qt5Widgets:Qt5Widgets.dll
 0000:fffb5000       .debug$S                   10000000     U2Gui:U2Gui.dll
 0000:fffb5000       .debug$S                   10000000     U2Gui:U2Gui.dll
 0000:fffb5000       .debug$S                   10000000     Qt5Widgets:Qt5Widgets.dll
 0000:fffb5000       .debug$S                   10000000     Qt5Widgets:Qt5Widgets.dll
 0000:fffb5000       .debug$S                   10000000     Qt5Widgets:Qt5Widgets.dll
 0000:fffb5000       .debug$S                   10000000     Qt5Widgets:Qt5Widgets.dll
 0000:fffb5000       .debug$S                   10000000     Qt5Widgets:Qt5Widgets.dll
 0000:fffb5000       .debug$S                   10000000     Qt5Widgets:Qt5Widgets.dll
 0000:fffb5000       .debug$S                   10000000     Qt5Widgets:Qt5Widgets.dll
 0000:fffb5000       .debug$S                   10000000     Qt5Widgets:Qt5Widgets.dll
 0000:fffb5000       .debug$S                   10000000     Qt5Widgets:Qt5Widgets.dll
 0000:fffb5000       .debug$S                   10000000     Qt5Widgets:Qt5Widgets.dll
 0000:fffb5000       .debug$S                   10000000     Qt5Widgets:Qt5Widgets.dll
 0000:fffb5000       .debug$S                   10000000     Qt5Widgets:Qt5Widgets.dll
 0000:fffb5000       .debug$S                   10000000     Qt5Widgets:Qt5Widgets.dll
 0000:fffb5000       .debug$S                   10000000     Qt5Widgets:Qt5Widgets.dll
 0000:fffb5000       .debug$S                   10000000     Qt5Widgets:Qt5Widgets.dll
 0000:fffb5000       .debug$S                   10000000     Qt5Widgets:Qt5Widgets.dll
 0000:fffb5000       .debug$S                   10000000     Qt5Widgets:Qt5Widgets.dll
 0000:fffb5000       .debug$S                   10000000     Qt5Widgets:Qt5Widgets.dll
 0000:fffb5000       .debug$S                   10000000     Qt5Widgets:Qt5Widgets.dll
 0000:fffb5000       .debug$S                   10000000     Qt5Widgets:Qt5Widgets.dll
 0000:fffb5000       .debug$S                   10000000     Qt5Widgets:Qt5Widgets.dll
 0000:fffb5000       .debug$S                   10000000     Qt5Widgets:Qt5Widgets.dll
 0000:fffb5000       .debug$S                   10000000     Qt5Widgets:Qt5Widgets.dll
 0000:fffb5000       .debug$S                   10000000     Qt5Widgets:Qt5Widgets.dll
 0000:fffb5000       .debug$S                   10000000     Qt5Widgets:Qt5Widgets.dll
 0000:fffb5000       .debug$S                   10000000     Qt5Widgets:Qt5Widgets.dll
 0000:fffb5000       .debug$S                   10000000     Qt5Widgets:Qt5Widgets.dll
 0000:fffb5000       .debug$S                   10000000     Qt5Widgets:Qt5Widgets.dll
 0000:fffb5000       .debug$S                   10000000     Qt5Widgets:Qt5Widgets.dll
 0000:fffb5000       .debug$S                   10000000     Qt5Widgets:Qt5Widgets.dll
 0000:fffb5000       .debug$S                   10000000     Qt5Widgets:Qt5Widgets.dll
 0000:fffb5000       .debug$S                   10000000     Qt5Widgets:Qt5Widgets.dll
 0000:fffb5000       .debug$S                   10000000     Qt5Widgets:Qt5Widgets.dll
 0000:fffb5000       .debug$S                   10000000     Qt5Widgets:Qt5Widgets.dll
 0000:fffb5000       .debug$S                   10000000     Qt5Widgets:Qt5Widgets.dll
 0000:fffb5000       .debug$S                   10000000     Qt5Widgets:Qt5Widgets.dll
 0000:fffb5000       .debug$S                   10000000     Qt5Widgets:Qt5Widgets.dll
 0000:fffb5000       .debug$S                   10000000     Qt5Widgets:Qt5Widgets.dll
 0000:fffb5000       .debug$S                   10000000     Qt5Widgets:Qt5Widgets.dll
 0000:fffb5000       .debug$S                   10000000     Qt5Widgets:Qt5Widgets.dll
 0000:fffb5000       .debug$S                   10000000     Qt5Widgets:Qt5Widgets.dll
 0000:fffb5000       .debug$S                   10000000     Qt5Widgets:Qt5Widgets.dll
 0000:fffb5000       .debug$S                   10000000     Qt5Widgets:Qt5Widgets.dll
 0000:fffb5000       .debug$S                   10000000     Qt5Widgets:Qt5Widgets.dll
 0000:fffb5000       .debug$S                   10000000     Qt5Widgets:Qt5Widgets.dll
 0000:fffb5000       .debug$S                   10000000     Qt5Widgets:Qt5Widgets.dll
 0000:fffb5000       .debug$S                   10000000     Qt5Widgets:Qt5Widgets.dll
 0000:fffb5000       .debug$S                   10000000     Qt5Widgets:Qt5Widgets.dll
 0000:fffb5000       .debug$S                   10000000     Qt5Widgets:Qt5Widgets.dll
 0000:fffb5000       .debug$S                   10000000     Qt5Widgets:Qt5Widgets.dll
 0000:fffb5000       .debug$S                   10000000     Qt5Widgets:Qt5Widgets.dll
 0000:fffb5000       .debug$S                   10000000     Qt5Widgets:Qt5Widgets.dll
 0000:fffb5000       .debug$S                   10000000     Qt5Widgets:Qt5Widgets.dll
 0000:fffb5000       .debug$S                   10000000     Qt5Widgets:Qt5Widgets.dll
 0000:fffb5000       .debug$S                   10000000     Qt5Widgets:Qt5Widgets.dll
 0000:fffb5000       .debug$S                   10000000     Qt5Widgets:Qt5Widgets.dll
 0000:fffb5000       .debug$S                   10000000     Qt5Widgets:Qt5Widgets.dll
 0000:fffb5000       .debug$S                   10000000     Qt5Widgets:Qt5Widgets.dll
 0000:fffb5000       .debug$S                   10000000     Qt5Widgets:Qt5Widgets.dll
 0000:fffb5000       .debug$S                   10000000     Qt5Widgets:Qt5Widgets.dll
 0000:fffb5000       .debug$S                   10000000     Qt5Widgets:Qt5Widgets.dll
 0000:fffb5000       .debug$S                   10000000     Qt5Widgets:Qt5Widgets.dll
 0000:fffb5000       .debug$S                   10000000     Qt5Widgets:Qt5Widgets.dll
 0000:fffb5000       .debug$S                   10000000     Qt5Widgets:Qt5Widgets.dll
 0000:fffb5000       .debug$S                   10000000     Qt5Widgets:Qt5Widgets.dll
 0000:fffb5000       .debug$S                   10000000     Qt5Widgets:Qt5Widgets.dll
 0000:fffb5000       .debug$S                   10000000     Qt5Widgets:Qt5Widgets.dll
 0000:fffb5000       .debug$S                   10000000     Qt5Widgets:Qt5Widgets.dll
 0000:fffb5000       .debug$S                   10000000     Qt5Widgets:Qt5Widgets.dll
 0000:fffb5000       .debug$S                   10000000     Qt5Widgets:Qt5Widgets.dll
 0000:fffb5000       .debug$S                   10000000     Qt5Widgets:Qt5Widgets.dll
 0000:fffb5000       .debug$S                   10000000     Qt5Widgets:Qt5Widgets.dll
 0000:fffb5000       .debug$S                   10000000     Qt5Widgets:Qt5Widgets.dll
 0000:fffb5000       .debug$S                   10000000     Qt5Widgets:Qt5Widgets.dll
 0000:fffb5000       .debug$S                   10000000     Qt5Widgets:Qt5Widgets.dll
 0000:fffb5000       .debug$S                   10000000     Qt5Widgets:Qt5Widgets.dll
 0000:fffb5000       .debug$S                   10000000     Qt5Widgets:Qt5Widgets.dll
 0000:fffb5000       .debug$S                   10000000     Qt5Widgets:Qt5Widgets.dll
 0000:fffb5000       .debug$S                   10000000     Qt5Widgets:Qt5Widgets.dll
 0000:fffb5000       .debug$S                   10000000     Qt5Widgets:Qt5Widgets.dll
 0000:fffb5000       .debug$S                   10000000     Qt5Widgets:Qt5Widgets.dll
 0000:fffb5000       .debug$S                   10000000     Qt5Widgets:Qt5Widgets.dll
 0000:fffb5000       .debug$S                   10000000     Qt5Widgets:Qt5Widgets.dll
 0000:fffb5000       .debug$S                   10000000     Qt5Widgets:Qt5Widgets.dll
 0000:fffb5000       .debug$S                   10000000     Qt5Widgets:Qt5Widgets.dll
 0000:fffb5000       .debug$S                   10000000     Qt5Widgets:Qt5Widgets.dll
 0000:fffb5000       .debug$S                   10000000     Qt5Widgets:Qt5Widgets.dll
 0000:fffb5000       .debug$S                   10000000     Qt5Widgets:Qt5Widgets.dll
 0000:fffb5000       .debug$S                   10000000     Qt5Widgets:Qt5Widgets.dll
 0000:fffb5000       .debug$S                   10000000     Qt5Widgets:Qt5Widgets.dll
 0000:fffb5000       .debug$S                   10000000     Qt5Widgets:Qt5Widgets.dll
 0000:fffb5000       .debug$S                   10000000     Qt5Widgets:Qt5Widgets.dll
 0000:fffb5000       .debug$S                   10000000     Qt5Widgets:Qt5Widgets.dll
 0000:fffb5000       .debug$S                   10000000     Qt5Widgets:Qt5Widgets.dll
 0000:fffb5000       .debug$S                   10000000     Qt5Widgets:Qt5Widgets.dll
 0000:fffb5000       .debug$S                   10000000     Qt5Widgets:Qt5Widgets.dll
 0000:fffb5000       .debug$S                   10000000     Qt5Widgets:Qt5Widgets.dll
 0000:fffb5000       .debug$S                   10000000     Qt5Widgets:Qt5Widgets.dll
 0000:fffb5000       .debug$S                   10000000     Qt5Widgets:Qt5Widgets.dll
 0000:fffb5000       .debug$S                   10000000     Qt5Widgets:Qt5Widgets.dll
 0000:fffb5000       .debug$S                   10000000     Qt5Widgets:Qt5Widgets.dll
 0000:fffb5000       .debug$S                   10000000     Qt5Widgets:Qt5Widgets.dll
 0000:fffb5000       .debug$S                   10000000     Qt5Widgets:Qt5Widgets.dll
 0000:fffb5000       .debug$S                   10000000     Qt5Widgets:Qt5Widgets.dll
 0000:fffb5000       .debug$S                   10000000     Qt5Widgets:Qt5Widgets.dll
 0000:fffb5000       .debug$S                   10000000     Qt5Widgets:Qt5Widgets.dll
 0000:fffb5000       .debug$S                   10000000     Qt5Widgets:Qt5Widgets.dll
 0000:fffb5000       .debug$S                   10000000     Qt5Widgets:Qt5Widgets.dll
 0000:fffb5000       .debug$S                   10000000     Qt5Widgets:Qt5Widgets.dll
 0000:fffb5000       .debug$S                   10000000     U2Designer:U2Designer.dll
 0000:fffb5000       .debug$S                   10000000     U2Designer:U2Designer.dll
 0000:fffb5000       .debug$S                   10000000     U2Designer:U2Designer.dll
 0000:fffb5000       .debug$S                   10000000     U2Designer:U2Designer.dll
 0000:fffb5000       .debug$S                   10000000     U2Designer:U2Designer.dll
 0000:fffb5000       .debug$S                   10000000     U2Designer:U2Designer.dll
 0000:fffb5000       .debug$S                   10000000     U2Designer:U2Designer.dll
 0000:fffb5000       .debug$S                   10000000     U2Designer:U2Designer.dll
 0000:fffb5000       .debug$S                   10000000     U2Designer:U2Designer.dll
 0000:fffb5000       .debug$S                   10000000     U2Designer:U2Designer.dll
 0000:fffb5000       .debug$S                   10000000     U2Designer:U2Designer.dll
 0000:fffb5000       .debug$S                   10000000     U2Designer:U2Designer.dll
 0000:fffb5000       .debug$S                   10000000     U2Designer:U2Designer.dll
 0000:fffb5000       .debug$S                   10000000     U2Designer:U2Designer.dll
 0000:fffb5000       .debug$S                   10000000     U2Designer:U2Designer.dll
 0000:fffb5000       .debug$S                   10000000     U2Designer:U2Designer.dll
 0000:fffb5000       .debug$S                   10000000     U2Designer:U2Designer.dll
 0000:fffb5000       .debug$S                   10000000     U2Designer:U2Designer.dll
 0000:fffb5000       .debug$S                   10000000     U2Designer:U2Designer.dll
 0000:fffb5000       .debug$S                   10000000     U2Designer:U2Designer.dll
 0000:fffb5000       .debug$S                   10000000     U2Designer:U2Designer.dll
 0000:fffb5000       .debug$S                   10000000     U2Designer:U2Designer.dll
 0000:fffb5000       .debug$S                   10000000     U2Designer:U2Designer.dll
 0000:fffb5000       .debug$S                   10000000     U2Designer:U2Designer.dll
 0000:fffb5000       .debug$S                   10000000     U2Designer:U2Designer.dll
 0000:fffb5000       .debug$S                   10000000     U2Designer:U2Designer.dll
 0000:fffb5000       .debug$S                   10000000     U2Designer:U2Designer.dll
 0000:fffb5000       .debug$S                   10000000     U2Designer:U2Designer.dll
 0000:fffb5000       .debug$S                   10000000     U2Designer:U2Designer.dll
 0000:fffb5000       .debug$S                   10000000     U2Designer:U2Designer.dll
 0000:fffb5000       .debug$S                   10000000     U2Designer:U2Designer.dll
 0000:fffb5000       .debug$S                   10000000     U2Designer:U2Designer.dll
 0000:fffb5000       .debug$S                   10000000     U2Designer:U2Designer.dll
 0000:fffb5000       .debug$S                   10000000     U2Designer:U2Designer.dll
 0000:fffb5000       .debug$S                   10000000     U2Designer:U2Designer.dll
 0000:fffb5000       .debug$S                   10000000     U2Designer:U2Designer.dll
 0000:fffb5000       .debug$S                   10000000     U2Designer:U2Designer.dll
 0000:fffb5000       .debug$S                   10000000     U2Lang:U2Lang.dll
 0000:fffb5000       .debug$S                   10000000     U2Lang:U2Lang.dll
 0000:fffb5000       .debug$S                   10000000     U2Lang:U2Lang.dll
 0000:fffb5000       .debug$S                   10000000     U2Lang:U2Lang.dll
 0000:fffb5000       .debug$S                   10000000     U2Lang:U2Lang.dll
 0000:fffb5000       .debug$S                   10000000     U2Lang:U2Lang.dll
 0000:fffb5000       .debug$S                   10000000     U2Lang:U2Lang.dll
 0000:fffb5000       .debug$S                   10000000     U2Lang:U2Lang.dll
 0000:fffb5000       .debug$S                   10000000     U2Lang:U2Lang.dll
 0000:fffb5000       .debug$S                   10000000     U2Lang:U2Lang.dll
 0000:fffb5000       .debug$S                   10000000     U2Lang:U2Lang.dll
 0000:fffb5000       .debug$S                   10000000     U2Lang:U2Lang.dll
 0000:fffb5000       .debug$S                   10000000     U2Lang:U2Lang.dll
 0000:fffb5000       .debug$S                   10000000     U2Lang:U2Lang.dll
 0000:fffb5000       .debug$S                   10000000     U2Lang:U2Lang.dll
 0000:fffb5000       .debug$S                   10000000     U2Lang:U2Lang.dll
 0000:fffb5000       .debug$S                   10000000     U2Lang:U2Lang.dll
 0000:fffb5000       .debug$S                   10000000     U2Lang:U2Lang.dll
 0000:fffb5000       .debug$S                   10000000     U2Lang:U2Lang.dll
 0000:fffb5000       .debug$S                   10000000     U2Lang:U2Lang.dll
 0000:fffb5000       .debug$S                   10000000     U2Lang:U2Lang.dll
 0000:fffb5000       .debug$S                   10000000     U2Lang:U2Lang.dll
 0000:fffb5000       .debug$S                   10000000     U2Lang:U2Lang.dll
 0000:fffb5000       .debug$S                   10000000     U2Lang:U2Lang.dll
 0000:fffb5000       .debug$S                   10000000     U2Lang:U2Lang.dll
 0000:fffb5000       .debug$S                   10000000     U2Lang:U2Lang.dll
 0000:fffb5000       .debug$S                   10000000     U2Lang:U2Lang.dll
 0000:fffb5000       .debug$S                   10000000     U2Lang:U2Lang.dll
 0000:fffb5000       .debug$S                   10000000     U2Lang:U2Lang.dll
 0000:fffb5000       .debug$S                   10000000     U2Lang:U2Lang.dll
 0000:fffb5000       .debug$S                   10000000     U2Lang:U2Lang.dll
 0000:fffb5000       .debug$S                   10000000     U2Lang:U2Lang.dll
 0000:fffb5000       .debug$S                   10000000     U2Lang:U2Lang.dll
 0000:fffb5000       .debug$S                   10000000     U2Lang:U2Lang.dll
 0000:fffb5000       .debug$S                   10000000     U2Lang:U2Lang.dll
 0000:fffb5000       .debug$S                   10000000     U2Lang:U2Lang.dll
 0000:fffb5000       .debug$S                   10000000     U2Lang:U2Lang.dll
 0000:fffb5000       .debug$S                   10000000     U2Lang:U2Lang.dll
 0000:fffb5000       .debug$S                   10000000     U2Lang:U2Lang.dll
 0000:fffb5000       .debug$S                   10000000     U2Lang:U2Lang.dll
 0000:fffb5000       .debug$S                   10000000     U2Lang:U2Lang.dll
 0000:fffb5000       .debug$S                   10000000     U2Lang:U2Lang.dll
 0000:fffb5000       .debug$S                   10000000     U2Lang:U2Lang.dll
 0000:fffb5000       .debug$S                   10000000     U2Lang:U2Lang.dll
 0000:fffb5000       .debug$S                   10000000     U2Lang:U2Lang.dll
 0000:fffb5000       .debug$S                   10000000     U2Lang:U2Lang.dll
 0000:fffb5000       .debug$S                   10000000     U2Lang:U2Lang.dll
 0000:fffb5000       .debug$S                   10000000     U2Lang:U2Lang.dll
 0000:fffb5000       .debug$S                   10000000     U2Lang:U2Lang.dll
 0000:fffb5000       .debug$S                   10000000     U2Lang:U2Lang.dll
 0000:fffb5000       .debug$S                   10000000     U2Lang:U2Lang.dll
 0000:fffb5000       .debug$S                   10000000     U2Lang:U2Lang.dll
 0000:fffb5000       .debug$S                   10000000     U2Lang:U2Lang.dll
 0000:fffb5000       .debug$S                   10000000     U2Lang:U2Lang.dll
 0000:fffb5000       .debug$S                   10000000     U2Lang:U2Lang.dll
 0000:fffb5000       .debug$S                   10000000     U2Lang:U2Lang.dll
 0000:fffb5000       .debug$S                   10000000     U2Lang:U2Lang.dll
 0000:fffb5000       .debug$S                   10000000     U2Lang:U2Lang.dll
 0000:fffb5000       .debug$S                   10000000     U2Lang:U2Lang.dll
 0000:fffb5000       .debug$S                   10000000     U2Lang:U2Lang.dll
 0000:fffb5000       .debug$S                   10000000     U2Lang:U2Lang.dll
 0000:fffb5000       .debug$S                   10000000     U2Lang:U2Lang.dll
 0000:fffb5000       .debug$S                   10000000     U2Lang:U2Lang.dll
 0000:fffb5000       .debug$S                   10000000     U2Lang:U2Lang.dll
 0000:fffb5000       .debug$S                   10000000     U2Lang:U2Lang.dll
 0000:fffb5000       .debug$S                   10000000     U2Lang:U2Lang.dll
 0000:fffb5000       .debug$S                   10000000     U2Lang:U2Lang.dll
 0000:fffb5000       .debug$S                   10000000     U2Lang:U2Lang.dll
 0000:fffb5000       .debug$S                   10000000     U2Lang:U2Lang.dll
 0000:fffb5000       .debug$S                   10000000     U2Lang:U2Lang.dll
 0000:fffb5000       .debug$S                   10000000     U2Lang:U2Lang.dll
 0000:fffb5000       .debug$S                   10000000     U2Lang:U2Lang.dll
 0000:fffb5000       .debug$S                   10000000     U2Lang:U2Lang.dll
 0000:fffb5000       .debug$S                   10000000     U2Gui:U2Gui.dll
 0000:fffb5000       .debug$S                   10000000     U2Gui:U2Gui.dll
 0000:fffb5000       .debug$S                   10000000     U2Lang:U2Lang.dll
 0000:fffb5000       .debug$S                   10000000     U2Gui:U2Gui.dll
 0000:fffb5000       .debug$S                   10000000     U2Gui:U2Gui.dll
 0000:fffb5000       .debug$S                   10000000     U2Lang:U2Lang.dll
 0000:fffb5000       .debug$S                   10000000     U2Lang:U2Lang.dll
 0000:fffb5000       .debug$S                   10000000     U2Lang:U2Lang.dll
 0000:fffb5000       .debug$S                   10000000     U2Lang:U2Lang.dll
 0000:fffb5000       .debug$S                   10000000     U2Lang:U2Lang.dll
 0000:fffb5000       .debug$S                   10000000     U2Lang:U2Lang.dll
 0000:fffb5000       .debug$S                   10000000     U2Gui:U2Gui.dll
 0000:fffb5000       .debug$S                   10000000     U2Lang:U2Lang.dll
 0000:fffb5000       .debug$S                   10000000     U2Lang:U2Lang.dll
 0000:fffb5000       .debug$S                   10000000     U2Lang:U2Lang.dll
 0000:fffb5000       .debug$S                   10000000     U2Lang:U2Lang.dll
 0000:fffb5000       .debug$S                   10000000     U2Lang:U2Lang.dll
 0001:fffff000       __ehhandler$??0?$QList@PAVDNATranslation@U2@@@@QAE@ABV0@@Z 10000000 f   ORFWorker.obj
 0000:fffb5000       .debug$S                   10000000     U2Gui:U2Gui.dll
 0000:fffb5000       .debug$S                   10000000     U2Lang:U2Lang.dll
 0000:fffb5000       .debug$S                   10000000     U2Lang:U2Lang.dll
 0000:fffb5000       .debug$S                   10000000     U2Lang:U2Lang.dll
 0000:fffb5000       .debug$S                   10000000     U2Lang:U2Lang.dll
 0000:fffb5000       .debug$S                   10000000     U2Lang:U2Lang.dll
 0000:fffb5000       .debug$S                   10000000     U2Lang:U2Lang.dll
 0000:fffb5000       .debug$S                   10000000     U2Lang:U2Lang.dll
 0000:fffb5000       .debug$S                   10000000     U2Lang:U2Lang.dll
 0000:fffb5000       .debug$S                   10000000     U2Lang:U2Lang.dll
 0000:fffb5000       .debug$S                   10000000     U2Lang:U2Lang.dll
 0000:fffb5000       .debug$S                   10000000     U2Lang:U2Lang.dll
 0000:fffb5000       .debug$S                   10000000     U2Lang:U2Lang.dll
 0000:fffb5000       .debug$S                   10000000     U2Lang:U2Lang.dll
 0000:fffb5000       .debug$S                   10000000     U2Lang:U2Lang.dll
 0000:fffb5000       .debug$S                   10000000     U2Lang:U2Lang.dll
 0000:fffb5000       .debug$S                   10000000     U2Gui:U2Gui.dll
 0000:fffb5000       .debug$S                   10000000     U2Gui:U2Gui.dll
 0000:fffb5000       .debug$S                   10000000     U2Gui:U2Gui.dll
 0001:fffff000       __unwindfunclet$?createNode@?$QMapData@VQString@@VQVariant@@@@QAEPAU?$QMapNode@VQString@@VQVariant@@@@ABVQString@@ABVQVariant@@PAU2@_N@Z$4 10000000 f   ORFWorker.obj
 0000:fffb5000       .debug$S                   10000000     U2Gui:U2Gui.dll
 0000:fffb5000       .debug$S                   10000000     U2Lang:U2Lang.dll
 0000:fffb5000       .debug$S                   10000000     U2Gui:U2Gui.dll
 0000:fffb5000       .debug$S                   10000000     U2Gui:U2Gui.dll
 0000:fffb5000       .debug$S                   10000000     U2Lang:U2Lang.dll
 0000:fffb5000       .debug$S                   10000000     U2Lang:U2Lang.dll
 0000:fffb5000       .debug$S                   10000000     U2Lang:U2Lang.dll
 0000:fffb5000       .debug$S                   10000000     U2Gui:U2Gui.dll
 0000:fffb5000       .debug$S                   10000000     U2Lang:U2Lang.dll
 0000:fffb5000       .debug$S                   10000000     U2Lang:U2Lang.dll
 0000:fffb5000       .debug$S                   10000000     U2Gui:U2Gui.dll
 0000:fffb5000       .debug$S                   10000000     U2Gui:U2Gui.dll
 0000:fffb5000       .debug$S                   10000000     U2Gui:U2Gui.dll
 0001:fffff000       __unwindfunclet$?createNode@?$QMapData@VQString@@PAVPropertyDelegate@U2@@@@QAEPAU?$QMapNode@VQString@@PAVPropertyDelegate@U2@@@@ABVQString@@ABQAVPropertyDelegate@U2@@PAU2@_N@Z$4 10000000 f   ORFWorker.obj
 0000:fffb5000       .debug$S                   10000000     U2Gui:U2Gui.dll
 0001:fffff000       __unwindfunclet$?metaType@?$QVariantValueHelper@VQString@@@QtPrivate@@SA?AVQString@@ABVQVariant@@@Z$0 10000000 f   ORFWorker.obj
 0000:fffb5000       .debug$S                   10000000     U2Gui:U2Gui.dll
 0000:fffb5000       .debug$S                   10000000     U2Lang:U2Lang.dll
 0000:fffb5000       .debug$S                   10000000     U2Lang:U2Lang.dll
 0000:fffb5000       .debug$S                   10000000     U2Lang:U2Lang.dll
 0000:fffb5000       .debug$S                   10000000     U2Gui:U2Gui.dll
 0000:fffb5000       .debug$S                   10000000     U2Gui:U2Gui.dll
 0000:fffb5000       .debug$S                   10000000     U2Gui:U2Gui.dll
 0000:fffb5000       .debug$S                   10000000     U2Gui:U2Gui.dll
 0002:fffda000       __catchsym$?_Copy@?$basic_string@DU?$char_traits@D@std@@V?$allocator@D@2@@std@@QAEXII@Z$5 10000000     ORFWorker.obj
 0000:fffb5000       .debug$S                   10000000     U2Gui:U2Gui.dll
 0002:fffda000       __unwindtable$??H@YA?BVQString@@ABV0@PBD@Z 10000000     ORFWorker.obj
 0002:fffda000       __catchsym$?detach_helper_grow@?$QList@PAVAttribute@U2@@@@AAEPAUNode@1@HH@Z$5 10000000     ORFWorker.obj
 0002:fffda000       __unwindtable$??H@YA?BVQString@@PBDABV0@@Z 10000000     ORFWorker.obj
 0002:fffda000       __catchsym$?append@?$QList@PAVAttribute@U2@@@@QAEXABQAVAttribute@U2@@@Z$6 10000000     ORFWorker.obj
 0002:fffda000       __unwindtable$??A?$QMap@VQString@@VQVariant@@@@QAEAAVQVariant@@ABVQString@@@Z 10000000     ORFWorker.obj
 0000:fffb5000       .debug$S                   10000000     U2Lang:U2Lang.dll
 0000:fffb5000       .debug$S                   10000000     U2Lang:U2Lang.dll
 0000:fffb5000       .debug$S                   10000000     U2Lang:U2Lang.dll
 0000:fffb5000       .debug$S                   10000000     U2Lang:U2Lang.dll
 0000:fffb5000       .debug$S                   10000000     U2Lang:U2Lang.dll
 0000:fffb5000       .debug$S                   10000000     U2Lang:U2Lang.dll
 0000:fffb5000       .debug$S                   10000000     U2Lang:U2Lang.dll
 0000:fffb5000       .debug$S                   10000000     U2Lang:U2Lang.dll
 0000:fffb5000       .debug$S                   10000000     U2Lang:U2Lang.dll
 0000:fffb5000       .debug$S                   10000000     U2Lang:U2Lang.dll
 0000:fffb5000       .debug$S                   10000000     U2Lang:U2Lang.dll
 0000:fffb5000       .debug$S                   10000000     U2Lang:U2Lang.dll
 0000:fffb5000       .debug$S                   10000000     U2Lang:U2Lang.dll
 0000:fffb5000       .debug$S                   10000000     U2Lang:U2Lang.dll
 0000:fffb5000       .debug$S                   10000000     U2Lang:U2Lang.dll
 0000:fffb5000       .debug$S                   10000000     U2Lang:U2Lang.dll
 0000:fffb5000       .debug$S                   10000000     U2Lang:U2Lang.dll
 0000:fffb5000       .debug$S                   10000000     U2Lang:U2Lang.dll
 0000:fffb5000       .debug$S                   10000000     U2Lang:U2Lang.dll
 0000:fffb5000       .debug$S                   10000000     U2Lang:U2Lang.dll
 0000:fffb5000       .debug$S                   10000000     U2Lang:U2Lang.dll
 0000:fffb5000       .debug$S                   10000000     U2Lang:U2Lang.dll
 0000:fffb5000       .debug$S                   10000000     U2Lang:U2Lang.dll
 0000:fffb5000       .debug$S                   10000000     U2Lang:U2Lang.dll
 0000:fffb5000       .debug$S                   10000000     U2Lang:U2Lang.dll
 0000:fffb5000       .debug$S                   10000000     U2Lang:U2Lang.dll
 0000:fffb5000       .debug$S                   10000000     U2Test:U2Test.dll
 0000:fffb5000       .debug$S                   10000000     U2Test:U2Test.dll
 0000:fffb5000       .debug$S                   10000000     U2Test:U2Test.dll
 0000:fffb5000       .debug$S                   10000000     U2Test:U2Test.dll
 0000:fffb5000       .debug$S                   10000000     U2Test:U2Test.dll
 0000:fffb5000       .debug$S                   10000000     U2Test:U2Test.dll
 0000:fffb5000       .debug$S                   10000000     U2Test:U2Test.dll
 0000:fffb5000       .debug$S                   10000000     U2Test:U2Test.dll
 0000:fffb5000       .debug$S                   10000000     U2Test:U2Test.dll
 0000:fffb5000       .debug$S                   10000000     U2Test:U2Test.dll
 0000:fffb5000       .debug$S                   10000000     U2Test:U2Test.dll
 0000:fffb5000       .debug$S                   10000000     U2View:U2View.dll
 0000:fffb5000       .debug$S                   10000000     U2View:U2View.dll
 0000:fffb5000       .debug$S                   10000000     U2View:U2View.dll
 0000:fffb5000       .debug$S                   10000000     U2View:U2View.dll
 0000:fffb5000       .debug$S                   10000000     U2View:U2View.dll
 0000:fffb5000       .debug$S                   10000000     U2View:U2View.dll
 0000:fffb5000       .debug$S                   10000000     U2View:U2View.dll
 0000:fffb5000       .debug$S                   10000000     U2View:U2View.dll
 0000:fffb5000       .debug$S                   10000000     U2View:U2View.dll
 0000:fffb5000       .debug$S                   10000000     U2View:U2View.dll
 0000:fffb5000       .debug$S                   10000000     U2View:U2View.dll
 0000:fffb5000       .debug$S                   10000000     U2View:U2View.dll
 0000:fffb5000       .debug$S                   10000000     U2Gui:U2Gui.dll
 0000:fffb5000       .debug$S                   10000000     U2Gui:U2Gui.dll
 0000:fffb5000       .debug$S                   10000000     U2Gui:U2Gui.dll
 0000:fffb5000       .debug$S                   10000000     U2Gui:U2Gui.dll
 0000:fffb5000       .debug$S                   10000000     U2Gui:U2Gui.dll
 0000:fffb5000       .debug$S                   10000000     U2Gui:U2Gui.dll
 0000:fffb5000       .debug$S                   10000000     U2Gui:U2Gui.dll
 0002:fffda008       __ehfuncinfo$?qt_metatype_id@?$QMetaTypeIdQObject@PAVTask@U2@@$00@@SAHXZ 10000008     moc_ORFQuery.obj
 0002:fffda008       __ehfuncinfo$??H@YA?BVQString@@PBDABV0@@Z 10000008     ORFMarkerTests.obj
 0002:fffda008       __ehfuncinfo$??A?$QMap@VQString@@VQVariant@@@@QAEAAVQVariant@@ABVQString@@@Z 10000008     ORFWorker.obj
 0002:fffda008       __ehfuncinfo$??H@YA?BVQString@@PBDABV0@@Z 10000008     ORFWorker.obj
 0001:fffff009       __ehhandler$?qt_metatype_id@?$QMetaTypeIdQObject@PAVTask@U2@@$00@@SAHXZ 10000009 f   moc_ORFQuery.obj
 0001:fffff009       __ehhandler$??A?$QMap@VQString@@VQVariant@@@@QAEAAVQVariant@@ABVQString@@@Z 10000009 f   ORFWorker.obj
 0002:fffda010       __catchsym$?_Copy@?$basic_string@DU?$char_traits@D@std@@V?$allocator@D@2@@std@@QAEXII@Z$4 10000010     ORFMarkerTests.obj
 0002:fffda010       __unwindtable$??0?$QList@VORFFindResult@U2@@@@QAE@ABV0@@Z 10000010     ORFQuery.obj
 0002:fffda010       __catchsym$?_Copy@?$basic_string@DU?$char_traits@D@std@@V?$allocator@D@2@@std@@QAEXII@Z$4 10000010     moc_ORFQuery.obj
 0002:fffda010       __ehfuncinfo$??H@YA?BVQString@@ABV0@PBD@Z 10000010     ORFWorker.obj
 0002:fffda010       __catchsym$?_Copy@?$basic_string@DU?$char_traits@D@std@@V?$allocator@D@2@@std@@QAEXII@Z$4 10000010     ORFWorker.obj
 0002:fffda010       __tryblocktable$?append@?$QList@PAVAttribute@U2@@@@QAEXABQAVAttribute@U2@@@Z 10000010     ORFWorker.obj
 0002:fffda010       __catchsym$?_Copy@?$basic_string@DU?$char_traits@D@std@@V?$allocator@D@2@@std@@QAEXII@Z$4 10000010     ORFQuery.obj
 0002:fffda010       __catchsym$?_Copy@?$basic_string@DU?$char_traits@D@std@@V?$allocator@D@2@@std@@QAEXII@Z$4 10000010     moc_ORFDialog.obj
 0002:fffda010       __catchsym$?detach_helper_grow@?$QList@PAVAttribute@U2@@@@AAEPAUNode@1@HH@Z$4 10000010     ORFWorker.obj
 0002:fffda010       __tryblocktable$?node_copy@?$QList@VORFFindResult@U2@@@@AAEXPAUNode@1@00@Z 10000010     ORFQuery.obj
 0002:fffda010       __tryblocktable$?createNode@?$QMapData@VQString@@PAVPropertyDelegate@U2@@@@QAEPAU?$QMapNode@VQString@@PAVPropertyDelegate@U2@@@@ABVQString@@ABQAVPropertyDelegate@U2@@PAU2@_N@Z 10000010     ORFWorker.obj
 0002:fffda010       __unwindtable$??0?$QList@PAVDNATranslation@U2@@@@QAE@ABV0@@Z 10000010     ORFWorker.obj
 0002:fffda010       __unwindtable$??0?$QList@VORFFindResult@U2@@@@QAE@ABV0@@Z 10000010     ORFMarkerTests.obj
 0002:fffda010       __catchsym$?_Copy@?$basic_string@DU?$char_traits@D@std@@V?$allocator@D@2@@std@@QAEXII@Z$4 10000010     ORFMarkerTask.obj
 0002:fffda010       __ehfuncinfo$?metaType@?$QVariantValueHelper@VQString@@@QtPrivate@@SA?AVQString@@ABVQVariant@@@Z 10000010     ORFWorker.obj
 0002:fffda010       __tryblocktable$?node_copy@?$QList@VORFFindResult@U2@@@@AAEXPAUNode@1@00@Z 10000010     ORFMarkerTests.obj
 0002:fffda010       __unwindtable$??0?$QList@PAVTask@U2@@@@QAE@ABV0@@Z 10000010     ORFMarkerTask.obj
 0002:fffda010       __tryblocktable$?node_copy@?$QList@VORFFindResult@U2@@@@AAEXPAUNode@1@00@Z 10000010     ORFMarkerTask.obj
 0002:fffda010       __catchsym$?_Copy@?$basic_string@DU?$char_traits@D@std@@V?$allocator@D@2@@std@@QAEXII@Z$4 10000010     moc_ORFMarkerPlugin.obj
 0002:fffda010       __catchsym$?_Copy@?$basic_string@DU?$char_traits@D@std@@V?$allocator@D@2@@std@@QAEXII@Z$4 10000010     moc_ORFMarkerTests.obj
 0002:fffda010       __catchsym$?_Copy@?$basic_string@DU?$char_traits@D@std@@V?$allocator@D@2@@std@@QAEXII@Z$4 10000010     moc_ORFWorker.obj
 0002:fffda010       __unwindtable$??0?$QList@VORFFindResult@U2@@@@QAE@ABV0@@Z 10000010     ORFMarkerTask.obj
 0002:fffda010       __catchsym$?_Copy@?$basic_string@DU?$char_traits@D@std@@V?$allocator@D@2@@std@@QAEXII@Z$4 10000010     moc_ORFMarkerTask.obj
 0002:fffda010       __catchsym$?_Copy@?$basic_string@DU?$char_traits@D@std@@V?$allocator@D@2@@std@@QAEXII@Z$4 10000010     ORFMarkerPlugin.obj
 0002:fffda010       __catchsym$?createNode@?$QMapData@VQString@@VQVariant@@@@QAEPAU?$QMapNode@VQString@@VQVariant@@@@ABVQString@@ABVQVariant@@PAU2@_N@Z$6 10000010     ORFWorker.obj
 0001:fffff014       __ehhandler$?createNode@?$QMapData@VQString@@PAVPropertyDelegate@U2@@@@QAEPAU?$QMapNode@VQString@@PAVPropertyDelegate@U2@@@@ABVQString@@ABQAVPropertyDelegate@U2@@PAU2@_N@Z 10000014 f   ORFWorker.obj
 0001:fffff014       __unwindfunclet$?createNode@?$QMapData@VQString@@VQVariant@@@@QAEPAU?$QMapNode@VQString@@VQVariant@@@@ABVQString@@ABVQVariant@@PAU2@_N@Z$5 10000014 f   ORFWorker.obj
 0001:fffff01a       __ehhandler$??H@YA?BVQString@@PBDABV0@@Z 1000001a f   ORFMarkerTests.obj
 0001:fffff01a       __unwindfunclet$??H@YA?BVQString@@ABV0@PBD@Z$1 1000001a f   ORFWorker.obj
 0001:fffff01a       __unwindfunclet$?metaType@?$QVariantValueHelper@VQString@@@QtPrivate@@SA?AVQString@@ABVQVariant@@@Z$1 1000001a f   ORFWorker.obj
 0001:fffff01a       __ehhandler$??H@YA?BVQString@@PBDABV0@@Z 1000001a f   ORFWorker.obj
 0002:fffda020       __tryblocktable$??0?$QList@PAVTask@U2@@@@QAE@ABV0@@Z 10000020     ORFMarkerTask.obj
 0002:fffda020       __tryblocktable$??0?$QList@PAVDNATranslation@U2@@@@QAE@ABV0@@Z 10000020     ORFWorker.obj
 0002:fffda020       __unwindtable$?_Copy@?$basic_string@DU?$char_traits@D@std@@V?$allocator@D@2@@std@@QAEXII@Z 10000020     moc_ORFMarkerPlugin.obj
 0002:fffda020       __unwindtable$?_Copy@?$basic_string@DU?$char_traits@D@std@@V?$allocator@D@2@@std@@QAEXII@Z 10000020     ORFMarkerTask.obj
 0002:fffda020       __tryblocktable$??0?$QList@VORFFindResult@U2@@@@QAE@ABV0@@Z 10000020     ORFMarkerTask.obj
 0002:fffda020       __unwindtable$?_Copy@?$basic_string@DU?$char_traits@D@std@@V?$allocator@D@2@@std@@QAEXII@Z 10000020     moc_ORFDialog.obj
 0002:fffda020       __unwindtable$?_Copy@?$basic_string@DU?$char_traits@D@std@@V?$allocator@D@2@@std@@QAEXII@Z 10000020     moc_ORFMarkerTests.obj
 0002:fffda020       __tryblocktable$??0?$QList@VORFFindResult@U2@@@@QAE@ABV0@@Z 10000020     ORFQuery.obj
 0002:fffda020       __unwindtable$?_Copy@?$basic_string@DU?$char_traits@D@std@@V?$allocator@D@2@@std@@QAEXII@Z 10000020     moc_ORFWorker.obj
 0002:fffda020       __unwindtable$?_Copy@?$basic_string@DU?$char_traits@D@std@@V?$allocator@D@2@@std@@QAEXII@Z 10000020     moc_ORFMarkerTask.obj
 0002:fffda020       __tryblocktable$??0?$QList@VORFFindResult@U2@@@@QAE@ABV0@@Z 10000020     ORFMarkerTests.obj
 0002:fffda020       __unwindtable$?_Copy@?$basic_string@DU?$char_traits@D@std@@V?$allocator@D@2@@std@@QAEXII@Z 10000020     ORFWorker.obj
 0002:fffda020       __unwindtable$?detach_helper_grow@?$QList@PAVAttribute@U2@@@@AAEPAUNode@1@HH@Z 10000020     ORFWorker.obj
 0002:fffda020       __ehfuncinfo$?createNode@?$QMapData@VQString@@VQVariant@@@@QAEPAU?$QMapNode@VQString@@VQVariant@@@@ABVQString@@ABVQVariant@@PAU2@_N@Z 10000020     ORFWorker.obj
 0002:fffda020       __unwindtable$?_Copy@?$basic_string@DU?$char_traits@D@std@@V?$allocator@D@2@@std@@QAEXII@Z 10000020     ORFMarkerTests.obj
 0002:fffda020       __unwindtable$?_Copy@?$basic_string@DU?$char_traits@D@std@@V?$allocator@D@2@@std@@QAEXII@Z 10000020     ORFQuery.obj
 0002:fffda020       __unwindtable$?_Copy@?$basic_string@DU?$char_traits@D@std@@V?$allocator@D@2@@std@@QAEXII@Z 10000020     moc_ORFQuery.obj
 0002:fffda020       __unwindtable$?_Copy@?$basic_string@DU?$char_traits@D@std@@V?$allocator@D@2@@std@@QAEXII@Z 10000020     ORFMarkerPlugin.obj
 0001:fffff023       __ehhandler$??H@YA?BVQString@@ABV0@PBD@Z 10000023 f   ORFWorker.obj
 0001:fffff023       __ehhandler$?metaType@?$QVariantValueHelper@VQString@@@QtPrivate@@SA?AVQString@@ABVQVariant@@@Z 10000023 f   ORFWorker.obj
 0002:fffda024       __unwindtable$?node_copy@?$QList@VORFFindResult@U2@@@@AAEXPAUNode@1@00@Z 10000024     ORFMarkerTask.obj
 0002:fffda024       __unwindtable$?node_copy@?$QList@VORFFindResult@U2@@@@AAEXPAUNode@1@00@Z 10000024     ORFMarkerTests.obj
 0002:fffda024       __ehfuncinfo$?createNode@?$QMapData@VQString@@PAVPropertyDelegate@U2@@@@QAEPAU?$QMapNode@VQString@@PAVPropertyDelegate@U2@@@@ABVQString@@ABQAVPropertyDelegate@U2@@PAU2@_N@Z 10000024     ORFWorker.obj
 0002:fffda024       __ehfuncinfo$?append@?$QList@PAVAttribute@U2@@@@QAEXABQAVAttribute@U2@@@Z 10000024     ORFWorker.obj
 0002:fffda024       __unwindtable$?node_copy@?$QList@VORFFindResult@U2@@@@AAEXPAUNode@1@00@Z 10000024     ORFQuery.obj
 0001:fffff028       __ehhandler$?createNode@?$QMapData@VQString@@VQVariant@@@@QAEPAU?$QMapNode@VQString@@VQVariant@@@@ABVQString@@ABVQVariant@@PAU2@_N@Z 10000028 f   ORFWorker.obj
 0002:fffda034       __ehfuncinfo$??0?$QList@PAVTask@U2@@@@QAE@ABV0@@Z 10000034     ORFMarkerTask.obj
 0002:fffda034       __ehfuncinfo$??0?$QList@VORFFindResult@U2@@@@QAE@ABV0@@Z 10000034     ORFMarkerTask.obj
 0002:fffda034       __ehfuncinfo$??0?$QList@VORFFindResult@U2@@@@QAE@ABV0@@Z 10000034     ORFQuery.obj
 0002:fffda034       __ehfuncinfo$??0?$QList@PAVDNATranslation@U2@@@@QAE@ABV0@@Z 10000034     ORFWorker.obj
 0002:fffda034       __ehfuncinfo$??0?$QList@VORFFindResult@U2@@@@QAE@ABV0@@Z 10000034     ORFMarkerTests.obj
 0002:fffda040       __ehfuncinfo$?_Copy@?$basic_string@DU?$char_traits@D@std@@V?$allocator@D@2@@std@@QAEXII@Z 10000040     moc_ORFMarkerPlugin.obj
 0002:fffda040       __ehfuncinfo$?_Copy@?$basic_string@DU?$char_traits@D@std@@V?$allocator@D@2@@std@@QAEXII@Z 10000040     moc_ORFMarkerTests.obj
 0002:fffda040       __ehfuncinfo$?_Copy@?$basic_string@DU?$char_traits@D@std@@V?$allocator@D@2@@std@@QAEXII@Z 10000040     ORFMarkerTask.obj
 0002:fffda040       __ehfuncinfo$?_Copy@?$basic_string@DU?$char_traits@D@std@@V?$allocator@D@2@@std@@QAEXII@Z 10000040     ORFQuery.obj
 0002:fffda040       __ehfuncinfo$?_Copy@?$basic_string@DU?$char_traits@D@std@@V?$allocator@D@2@@std@@QAEXII@Z 10000040     ORFMarkerPlugin.obj
 0002:fffda040       __ehfuncinfo$?_Copy@?$basic_string@DU?$char_traits@D@std@@V?$allocator@D@2@@std@@QAEXII@Z 10000040     moc_ORFWorker.obj
 0002:fffda040       __ehfuncinfo$?_Copy@?$basic_string@DU?$char_traits@D@std@@V?$allocator@D@2@@std@@QAEXII@Z 10000040     moc_ORFQuery.obj
 0002:fffda040       __ehfuncinfo$?_Copy@?$basic_string@DU?$char_traits@D@std@@V?$allocator@D@2@@std@@QAEXII@Z 10000040     moc_ORFDialog.obj
 0002:fffda040       __ehfuncinfo$?_Copy@?$basic_string@DU?$char_traits@D@std@@V?$allocator@D@2@@std@@QAEXII@Z 10000040     moc_ORFMarkerTask.obj
 0002:fffda040       __ehfuncinfo$?_Copy@?$basic_string@DU?$char_traits@D@std@@V?$allocator@D@2@@std@@QAEXII@Z 10000040     ORFWorker.obj
 0002:fffda040       __ehfuncinfo$?detach_helper_grow@?$QList@PAVAttribute@U2@@@@AAEPAUNode@1@HH@Z 10000040     ORFWorker.obj
 0002:fffda040       __ehfuncinfo$?_Copy@?$basic_string@DU?$char_traits@D@std@@V?$allocator@D@2@@std@@QAEXII@Z 10000040     ORFMarkerTests.obj
 0002:fffda044       __tryblocktable$?createNode@?$QMapData@VQString@@VQVariant@@@@QAEPAU?$QMapNode@VQString@@VQVariant@@@@ABVQString@@ABVQVariant@@PAU2@_N@Z 10000044     ORFWorker.obj
 0002:fffda044       __ehfuncinfo$?node_copy@?$QList@VORFFindResult@U2@@@@AAEXPAUNode@1@00@Z 10000044     ORFMarkerTests.obj
 0002:fffda044       __ehfuncinfo$?node_copy@?$QList@VORFFindResult@U2@@@@AAEXPAUNode@1@00@Z 10000044     ORFMarkerTask.obj
 0002:fffda044       __ehfuncinfo$?node_copy@?$QList@VORFFindResult@U2@@@@AAEXPAUNode@1@00@Z 10000044     ORFQuery.obj
 0002:fffda048       __unwindtable$?append@?$QList@PAVAttribute@U2@@@@QAEXABQAVAttribute@U2@@@Z 10000048     ORFWorker.obj
 0002:fffda048       __unwindtable$?createNode@?$QMapData@VQString@@PAVPropertyDelegate@U2@@@@QAEPAU?$QMapNode@VQString@@PAVPropertyDelegate@U2@@@@ABVQString@@ABQAVPropertyDelegate@U2@@PAU2@_N@Z 10000048     ORFWorker.obj
 0002:fffda064       __tryblocktable$?_Copy@?$basic_string@DU?$char_traits@D@std@@V?$allocator@D@2@@std@@QAEXII@Z 10000064     ORFMarkerTask.obj
 0002:fffda064       __tryblocktable$?_Copy@?$basic_string@DU?$char_traits@D@std@@V?$allocator@D@2@@std@@QAEXII@Z 10000064     ORFWorker.obj
 0002:fffda064       __tryblocktable$?detach_helper_grow@?$QList@PAVAttribute@U2@@@@AAEPAUNode@1@HH@Z 10000064     ORFWorker.obj
 0002:fffda064       __tryblocktable$?_Copy@?$basic_string@DU?$char_traits@D@std@@V?$allocator@D@2@@std@@QAEXII@Z 10000064     ORFMarkerTests.obj
 0002:fffda064       __tryblocktable$?_Copy@?$basic_string@DU?$char_traits@D@std@@V?$allocator@D@2@@std@@QAEXII@Z 10000064     ORFQuery.obj
 0002:fffda064       __tryblocktable$?_Copy@?$basic_string@DU?$char_traits@D@std@@V?$allocator@D@2@@std@@QAEXII@Z 10000064     moc_ORFWorker.obj
 0002:fffda064       __tryblocktable$?_Copy@?$basic_string@DU?$char_traits@D@std@@V?$allocator@D@2@@std@@QAEXII@Z 10000064     moc_ORFMarkerPlugin.obj
 0002:fffda064       __tryblocktable$?_Copy@?$basic_string@DU?$char_traits@D@std@@V?$allocator@D@2@@std@@QAEXII@Z 10000064     moc_ORFQuery.obj
 0002:fffda064       __tryblocktable$?_Copy@?$basic_string@DU?$char_traits@D@std@@V?$allocator@D@2@@std@@QAEXII@Z 10000064     ORFMarkerPlugin.obj
 0002:fffda064       __tryblocktable$?_Copy@?$basic_string@DU?$char_traits@D@std@@V?$allocator@D@2@@std@@QAEXII@Z 10000064     moc_ORFDialog.obj
 0002:fffda064       __tryblocktable$?_Copy@?$basic_string@DU?$char_traits@D@std@@V?$allocator@D@2@@std@@QAEXII@Z 10000064     moc_ORFMarkerTask.obj
 0002:fffda064       __tryblocktable$?_Copy@?$basic_string@DU?$char_traits@D@std@@V?$allocator@D@2@@std@@QAEXII@Z 10000064     moc_ORFMarkerTests.obj
 0002:fffda06c       __unwindtable$?createNode@?$QMapData@VQString@@VQVariant@@@@QAEPAU?$QMapNode@VQString@@VQVariant@@@@ABVQString@@ABVQVariant@@PAU2@_N@Z 1000006c     ORFWorker.obj
 0001:fffff084       __catch$?node_copy@?$QList@VORFFindResult@U2@@@@AAEXPAUNode@1@00@Z$0 10000084 f   ORFMarkerTask.obj
 0001:fffff084       __catch$?node_copy@?$QList@VORFFindResult@U2@@@@AAEXPAUNode@1@00@Z$0 10000084 f   ORFMarkerTests.obj
 0001:fffff084       __catch$?node_copy@?$QList@VORFFindResult@U2@@@@AAEXPAUNode@1@00@Z$0 10000084 f   ORFQuery.obj
 0001:fffff085       __catch$?append@?$QList@PAVAttribute@U2@@@@QAEXABQAVAttribute@U2@@@Z$4 10000085 f   ORFWorker.obj
 0001:fffff085       __catch$?createNode@?$QMapData@VQString@@PAVPropertyDelegate@U2@@@@QAEPAU?$QMapNode@VQString@@PAVPropertyDelegate@U2@@@@ABVQString@@ABQAVPropertyDelegate@U2@@PAU2@_N@Z$2 10000085 f   ORFWorker.obj
 0001:fffff08e       __catch$?createNode@?$QMapData@VQString@@VQVariant@@@@QAEPAU?$QMapNode@VQString@@VQVariant@@@@ABVQString@@ABVQVariant@@PAU2@_N@Z$0 1000008e f   ORFWorker.obj
 0001:fffff096       __catch$?_Copy@?$basic_string@DU?$char_traits@D@std@@V?$allocator@D@2@@std@@QAEXII@Z$0 10000096 f   moc_ORFMarkerTests.obj
 0001:fffff096       __catch$?_Copy@?$basic_string@DU?$char_traits@D@std@@V?$allocator@D@2@@std@@QAEXII@Z$0 10000096 f   ORFQuery.obj
 0001:fffff096       __catch$?_Copy@?$basic_string@DU?$char_traits@D@std@@V?$allocator@D@2@@std@@QAEXII@Z$0 10000096 f   ORFMarkerTests.obj
 0001:fffff096       __catch$?_Copy@?$basic_string@DU?$char_traits@D@std@@V?$allocator@D@2@@std@@QAEXII@Z$0 10000096 f   moc_ORFWorker.obj
 0001:fffff096       __catch$?_Copy@?$basic_string@DU?$char_traits@D@std@@V?$allocator@D@2@@std@@QAEXII@Z$0 10000096 f   ORFWorker.obj
 0001:fffff096       __catch$?_Copy@?$basic_string@DU?$char_traits@D@std@@V?$allocator@D@2@@std@@QAEXII@Z$0 10000096 f   moc_ORFMarkerPlugin.obj
 0001:fffff096       __catch$?_Copy@?$basic_string@DU?$char_traits@D@std@@V?$allocator@D@2@@std@@QAEXII@Z$0 10000096 f   ORFMarkerPlugin.obj
 0001:fffff096       __catch$?_Copy@?$basic_string@DU?$char_traits@D@std@@V?$allocator@D@2@@std@@QAEXII@Z$0 10000096 f   moc_ORFQuery.obj
 0001:fffff096       __catch$?_Copy@?$basic_string@DU?$char_traits@D@std@@V?$allocator@D@2@@std@@QAEXII@Z$0 10000096 f   ORFMarkerTask.obj
 0001:fffff096       __catch$?_Copy@?$basic_string@DU?$char_traits@D@std@@V?$allocator@D@2@@std@@QAEXII@Z$0 10000096 f   moc_ORFDialog.obj
 0001:fffff096       __catch$?_Copy@?$basic_string@DU?$char_traits@D@std@@V?$allocator@D@2@@std@@QAEXII@Z$0 10000096 f   moc_ORFMarkerTask.obj
 0001:fffff09e       __catch$??0?$QList@VORFFindResult@U2@@@@QAE@ABV0@@Z$0 1000009e f   ORFMarkerTests.obj
 0001:fffff09e       __catch$??0?$QList@VORFFindResult@U2@@@@QAE@ABV0@@Z$0 1000009e f   ORFQuery.obj
 0001:fffff09e       __catch$??0?$QList@PAVDNATranslation@U2@@@@QAE@ABV0@@Z$0 1000009e f   ORFWorker.obj
 0001:fffff09e       __catch$??0?$QList@VORFFindResult@U2@@@@QAE@ABV0@@Z$0 1000009e f   ORFMarkerTask.obj
 0001:fffff09e       __catch$??0?$QList@PAVTask@U2@@@@QAE@ABV0@@Z$0 1000009e f   ORFMarkerTask.obj
 0001:fffff0a3       __catch$?createNode@?$QMapData@VQString@@VQVariant@@@@QAEPAU?$QMapNode@VQString@@VQVariant@@@@ABVQString@@ABVQVariant@@PAU2@_N@Z$2 100000a3 f   ORFWorker.obj
 0001:fffff0d3       __catch$?_Copy@?$basic_string@DU?$char_traits@D@std@@V?$allocator@D@2@@std@@QAEXII@Z$1 100000d3 f   ORFMarkerTests.obj
 0001:fffff0d3       __catch$?_Copy@?$basic_string@DU?$char_traits@D@std@@V?$allocator@D@2@@std@@QAEXII@Z$1 100000d3 f   moc_ORFMarkerTests.obj
 0001:fffff0d3       __catch$?_Copy@?$basic_string@DU?$char_traits@D@std@@V?$allocator@D@2@@std@@QAEXII@Z$1 100000d3 f   ORFWorker.obj
 0001:fffff0d3       __catch$?_Copy@?$basic_string@DU?$char_traits@D@std@@V?$allocator@D@2@@std@@QAEXII@Z$1 100000d3 f   moc_ORFMarkerPlugin.obj
 0001:fffff0d3       __catch$?_Copy@?$basic_string@DU?$char_traits@D@std@@V?$allocator@D@2@@std@@QAEXII@Z$1 100000d3 f   moc_ORFDialog.obj
 0001:fffff0d3       __catch$?_Copy@?$basic_string@DU?$char_traits@D@std@@V?$allocator@D@2@@std@@QAEXII@Z$1 100000d3 f   ORFMarkerTask.obj
 0001:fffff0d3       __catch$?_Copy@?$basic_string@DU?$char_traits@D@std@@V?$allocator@D@2@@std@@QAEXII@Z$1 100000d3 f   ORFMarkerPlugin.obj
 0001:fffff0d3       __catch$?_Copy@?$basic_string@DU?$char_traits@D@std@@V?$allocator@D@2@@std@@QAEXII@Z$1 100000d3 f   ORFQuery.obj
 0001:fffff0d3       __catch$?_Copy@?$basic_string@DU?$char_traits@D@std@@V?$allocator@D@2@@std@@QAEXII@Z$1 100000d3 f   moc_ORFMarkerTask.obj
 0001:fffff0d3       __catch$?_Copy@?$basic_string@DU?$char_traits@D@std@@V?$allocator@D@2@@std@@QAEXII@Z$1 100000d3 f   moc_ORFQuery.obj
 0001:fffff0d3       __catch$?_Copy@?$basic_string@DU?$char_traits@D@std@@V?$allocator@D@2@@std@@QAEXII@Z$1 100000d3 f   moc_ORFWorker.obj
 0001:fffff0f1       __catch$?detach_helper_grow@?$QList@PAVAttribute@U2@@@@AAEPAUNode@1@HH@Z$2 100000f1 f   ORFWorker.obj
 0001:fffff0f1       __catch$?detach_helper_grow@?$QList@PAVAttribute@U2@@@@AAEPAUNode@1@HH@Z$0 100000f1 f   ORFWorker.obj
 0001:00000000       ??__E?_Generic_object@?$_Error_objects@H@std@@2V_Generic_error_category@2@A@@YAXXZ 10001000 f   ORFDialog.obj
 0001:00000010       ??__E?_Iostream_object@?$_Error_objects@H@std@@2V_Iostream_error_category@2@A@@YAXXZ 10001010 f   ORFDialog.obj
 0001:00000020       ??__E?_System_object@?$_Error_objects@H@std@@2V_System_error_category@2@A@@YAXXZ 10001020 f   ORFDialog.obj
 0001:00000030       ??__EService_DNAExport@U2@@YAXXZ 10001030 f   ORFDialog.obj
 0001:00000040       ??__EService_DNAGraphPack@U2@@YAXXZ 10001040 f   ORFDialog.obj
 0001:00000050       ??__EService_ExternalToolSupport@U2@@YAXXZ 10001050 f   ORFDialog.obj
 0001:00000060       ??__EService_GUITesting@U2@@YAXXZ 10001060 f   ORFDialog.obj
 0001:00000070       ??__EService_MaxCoreServiceId@U2@@YAXXZ 10001070 f   ORFDialog.obj
 0001:00000080       ??__EService_MinCoreServiceId@U2@@YAXXZ 10001080 f   ORFDialog.obj
 0001:00000090       ??__EService_PluginViewer@U2@@YAXXZ 10001090 f   ORFDialog.obj
 0001:000000a0       ??__EService_Project@U2@@YAXXZ 100010a0 f   ORFDialog.obj
 0001:000000b0       ??__EService_ProjectView@U2@@YAXXZ 100010b0 f   ORFDialog.obj
 0001:000000c0       ??__EService_QueryDesigner@U2@@YAXXZ 100010c0 f   ORFDialog.obj
 0001:000000d0       ??__EService_ScriptRegistry@U2@@YAXXZ 100010d0 f   ORFDialog.obj
 0001:000000e0       ??__EService_TestRunner@U2@@YAXXZ 100010e0 f   ORFDialog.obj
 0001:000000f0       ??__EService_WorkflowDesigner@U2@@YAXXZ 100010f0 f   ORFDialog.obj
 0001:00000100       ??__EalgoLog@U2@@YAXXZ     10001100 f   ORFDialog.obj
 0001:00000180       ??__EcmdLog@U2@@YAXXZ      10001180 f   ORFDialog.obj
 0001:00000200       ??__EcoreLog@U2@@YAXXZ     10001200 f   ORFDialog.obj
 0001:00000280       ??__EioLog@U2@@YAXXZ       10001280 f   ORFDialog.obj
 0001:00000300       ??__EperfLog@U2@@YAXXZ     10001300 f   ORFDialog.obj
 0001:00000380       ??__EscriptLog@U2@@YAXXZ   10001380 f   ORFDialog.obj
 0001:00000400       ??__EtaskLog@U2@@YAXXZ     10001400 f   ORFDialog.obj
 0001:00000480       ??__EuiLog@U2@@YAXXZ       10001480 f   ORFDialog.obj
 0001:00000500       ??__EuserActLog@U2@@YAXXZ  10001500 f   ORFDialog.obj
 0001:00000580       ??__E?_Generic_object@?$_Error_objects@H@std@@2V_Generic_error_category@2@A@@YAXXZ 10001580 f   ORFMarkerPlugin.obj
 0001:00000590       ??__E?_Iostream_object@?$_Error_objects@H@std@@2V_Iostream_error_category@2@A@@YAXXZ 10001590 f   ORFMarkerPlugin.obj
 0001:000005a0       ??__E?_System_object@?$_Error_objects@H@std@@2V_System_error_category@2@A@@YAXXZ 100015a0 f   ORFMarkerPlugin.obj
 0001:000005b0       ??__EService_DNAExport@U2@@YAXXZ 100015b0 f   ORFMarkerPlugin.obj
 0001:000005c0       ??__EService_DNAGraphPack@U2@@YAXXZ 100015c0 f   ORFMarkerPlugin.obj
 0001:000005d0       ??__EService_ExternalToolSupport@U2@@YAXXZ 100015d0 f   ORFMarkerPlugin.obj
 0001:000005e0       ??__EService_GUITesting@U2@@YAXXZ 100015e0 f   ORFMarkerPlugin.obj
 0001:000005f0       ??__EService_MaxCoreServiceId@U2@@YAXXZ 100015f0 f   ORFMarkerPlugin.obj
 0001:00000600       ??__EService_MinCoreServiceId@U2@@YAXXZ 10001600 f   ORFMarkerPlugin.obj
 0001:00000610       ??__EService_PluginViewer@U2@@YAXXZ 10001610 f   ORFMarkerPlugin.obj
 0001:00000620       ??__EService_Project@U2@@YAXXZ 10001620 f   ORFMarkerPlugin.obj
 0001:00000630       ??__EService_ProjectView@U2@@YAXXZ 10001630 f   ORFMarkerPlugin.obj
 0001:00000640       ??__EService_QueryDesigner@U2@@YAXXZ 10001640 f   ORFMarkerPlugin.obj
 0001:00000650       ??__EService_ScriptRegistry@U2@@YAXXZ 10001650 f   ORFMarkerPlugin.obj
 0001:00000660       ??__EService_TestRunner@U2@@YAXXZ 10001660 f   ORFMarkerPlugin.obj
 0001:00000670       ??__EService_WorkflowDesigner@U2@@YAXXZ 10001670 f   ORFMarkerPlugin.obj
 0001:00000680       ??__EalgoLog@U2@@YAXXZ     10001680 f   ORFMarkerPlugin.obj
 0001:00000700       ??__EcmdLog@U2@@YAXXZ      10001700 f   ORFMarkerPlugin.obj
 0001:00000780       ??__EcoreLog@U2@@YAXXZ     10001780 f   ORFMarkerPlugin.obj
 0001:00000800       ??__EioLog@U2@@YAXXZ       10001800 f   ORFMarkerPlugin.obj
 0001:00000880       ??__EperfLog@U2@@YAXXZ     10001880 f   ORFMarkerPlugin.obj
 0001:00000900       ??__EscriptLog@U2@@YAXXZ   10001900 f   ORFMarkerPlugin.obj
 0001:00000980       ??__EtaskLog@U2@@YAXXZ     10001980 f   ORFMarkerPlugin.obj
 0001:00000a00       ??__EuiLog@U2@@YAXXZ       10001a00 f   ORFMarkerPlugin.obj
 0001:00000a80       ??__EuserActLog@U2@@YAXXZ  10001a80 f   ORFMarkerPlugin.obj
 0001:00000b00       ??__E?ALLOW_ALT_START@ORFSettingsKeys@U2@@2VQString@@B@@YAXXZ 10001b00 f   ORFMarkerTask.obj
 0001:00000b20       ??__E?ALLOW_OVERLAP@ORFSettingsKeys@U2@@2VQString@@B@@YAXXZ 10001b20 f   ORFMarkerTask.obj
 0001:00000b40       ??__E?AMINO_TRANSL@ORFSettingsKeys@U2@@2VQString@@B@@YAXXZ 10001b40 f   ORFMarkerTask.obj
 0001:00000b60       ??__E?INCLUDE_STOP_CODON@ORFSettingsKeys@U2@@2VQString@@B@@YAXXZ 10001b60 f   ORFMarkerTask.obj
 0001:00000b80       ??__E?IS_RESULT_LIMITED@ORFSettingsKeys@U2@@2VQString@@B@@YAXXZ 10001b80 f   ORFMarkerTask.obj
 0001:00000ba0       ??__E?MAX_RESULT@ORFSettingsKeys@U2@@2VQString@@B@@YAXXZ 10001ba0 f   ORFMarkerTask.obj
 0001:00000bc0       ??__E?MIN_LEN@ORFSettingsKeys@U2@@2VQString@@B@@YAXXZ 10001bc0 f   ORFMarkerTask.obj
 0001:00000be0       ??__E?MUST_FIT@ORFSettingsKeys@U2@@2VQString@@B@@YAXXZ 10001be0 f   ORFMarkerTask.obj
 0001:00000c00       ??__E?MUST_INIT@ORFSettingsKeys@U2@@2VQString@@B@@YAXXZ 10001c00 f   ORFMarkerTask.obj
 0001:00000c20       ??__E?SEARCH_REGION@ORFSettingsKeys@U2@@2VQString@@B@@YAXXZ 10001c20 f   ORFMarkerTask.obj
 0001:00000c40       ??__E?STRAND@ORFSettingsKeys@U2@@2VQString@@B@@YAXXZ 10001c40 f   ORFMarkerTask.obj
 0001:00000c60       ??__E?_Generic_object@?$_Error_objects@H@std@@2V_Generic_error_category@2@A@@YAXXZ 10001c60 f   ORFMarkerTask.obj
 0001:00000c70       ??__E?_Iostream_object@?$_Error_objects@H@std@@2V_Iostream_error_category@2@A@@YAXXZ 10001c70 f   ORFMarkerTask.obj
 0001:00000c80       ??__E?_System_object@?$_Error_objects@H@std@@2V_System_error_category@2@A@@YAXXZ 10001c80 f   ORFMarkerTask.obj
 0001:00000c90       ??__EalgoLog@U2@@YAXXZ     10001c90 f   ORFMarkerTask.obj
 0001:00000d10       ??__EcmdLog@U2@@YAXXZ      10001d10 f   ORFMarkerTask.obj
 0001:00000d90       ??__EcoreLog@U2@@YAXXZ     10001d90 f   ORFMarkerTask.obj
 0001:00000e10       ??__EioLog@U2@@YAXXZ       10001e10 f   ORFMarkerTask.obj
 0001:00000e90       ??__EperfLog@U2@@YAXXZ     10001e90 f   ORFMarkerTask.obj
 0001:00000f10       ??__EscriptLog@U2@@YAXXZ   10001f10 f   ORFMarkerTask.obj
 0001:00000f90       ??__EtaskLog@U2@@YAXXZ     10001f90 f   ORFMarkerTask.obj
 0001:00001010       ??__EuiLog@U2@@YAXXZ       10002010 f   ORFMarkerTask.obj
 0001:00001090       ??__EuserActLog@U2@@YAXXZ  10002090 f   ORFMarkerTask.obj
 0001:00001110       ??__E?_Generic_object@?$_Error_objects@H@std@@2V_Generic_error_category@2@A@@YAXXZ 10002110 f   ORFMarkerTests.obj
 0001:00001120       ??__E?_Iostream_object@?$_Error_objects@H@std@@2V_Iostream_error_category@2@A@@YAXXZ 10002120 f   ORFMarkerTests.obj
 0001:00001130       ??__E?_System_object@?$_Error_objects@H@std@@2V_System_error_category@2@A@@YAXXZ 10002130 f   ORFMarkerTests.obj
 0001:00001140       ??__EService_DNAExport@U2@@YAXXZ 10002140 f   ORFMarkerTests.obj
 0001:00001150       ??__EService_DNAGraphPack@U2@@YAXXZ 10002150 f   ORFMarkerTests.obj
 0001:00001160       ??__EService_ExternalToolSupport@U2@@YAXXZ 10002160 f   ORFMarkerTests.obj
 0001:00001170       ??__EService_GUITesting@U2@@YAXXZ 10002170 f   ORFMarkerTests.obj
 0001:00001180       ??__EService_MaxCoreServiceId@U2@@YAXXZ 10002180 f   ORFMarkerTests.obj
 0001:00001190       ??__EService_MinCoreServiceId@U2@@YAXXZ 10002190 f   ORFMarkerTests.obj
 0001:000011a0       ??__EService_PluginViewer@U2@@YAXXZ 100021a0 f   ORFMarkerTests.obj
 0001:000011b0       ??__EService_Project@U2@@YAXXZ 100021b0 f   ORFMarkerTests.obj
 0001:000011c0       ??__EService_ProjectView@U2@@YAXXZ 100021c0 f   ORFMarkerTests.obj
 0001:000011d0       ??__EService_QueryDesigner@U2@@YAXXZ 100021d0 f   ORFMarkerTests.obj
 0001:000011e0       ??__EService_ScriptRegistry@U2@@YAXXZ 100021e0 f   ORFMarkerTests.obj
 0001:000011f0       ??__EService_TestRunner@U2@@YAXXZ 100021f0 f   ORFMarkerTests.obj
 0001:00001200       ??__EService_WorkflowDesigner@U2@@YAXXZ 10002200 f   ORFMarkerTests.obj
 0001:00001210       ??__EalgoLog@U2@@YAXXZ     10002210 f   ORFMarkerTests.obj
 0001:00001290       ??__EcmdLog@U2@@YAXXZ      10002290 f   ORFMarkerTests.obj
 0001:00001310       ??__EcoreLog@U2@@YAXXZ     10002310 f   ORFMarkerTests.obj
 0001:00001390       ??__EioLog@U2@@YAXXZ       10002390 f   ORFMarkerTests.obj
 0001:00001410       ??__EperfLog@U2@@YAXXZ     10002410 f   ORFMarkerTests.obj
 0001:00001490       ??__EscriptLog@U2@@YAXXZ   10002490 f   ORFMarkerTests.obj
 0001:00001510       ??__EtaskLog@U2@@YAXXZ     10002510 f   ORFMarkerTests.obj
 0001:00001590       ??__EuiLog@U2@@YAXXZ       10002590 f   ORFMarkerTests.obj
 0001:00001610       ??__EuserActLog@U2@@YAXXZ  10002610 f   ORFMarkerTests.obj
 0001:00001690       ??__E?_Generic_object@?$_Error_objects@H@std@@2V_Generic_error_category@2@A@@YAXXZ 10002690 f   ORFQuery.obj
 0001:000016a0       ??__E?_Iostream_object@?$_Error_objects@H@std@@2V_Iostream_error_category@2@A@@YAXXZ 100026a0 f   ORFQuery.obj
 0001:000016b0       ??__E?_System_object@?$_Error_objects@H@std@@2V_System_error_category@2@A@@YAXXZ 100026b0 f   ORFQuery.obj
 0001:000016c0       ??__EALT_ATTR@U2@@YAXXZ    100026c0 f   ORFQuery.obj
 0001:000016e0       ??__EFIT_ATTR@U2@@YAXXZ    100026e0 f   ORFQuery.obj
 0001:00001700       ??__EID_ATTR@U2@@YAXXZ     10002700 f   ORFQuery.obj
 0001:00001720       ??__EINIT_ATTR@U2@@YAXXZ   10002720 f   ORFQuery.obj
 0001:00001740       ??__ELEN_ATTR@U2@@YAXXZ    10002740 f   ORFQuery.obj
 0001:00001760       ??__ELIMIT_ATTR@U2@@YAXXZ  10002760 f   ORFQuery.obj
 0001:00001780       ??__EMAX_LENGTH_ATTR@U2@@YAXXZ 10002780 f   ORFQuery.obj
 0001:000017a0       ??__ERES_ATTR@U2@@YAXXZ    100027a0 f   ORFQuery.obj
 0001:000017c0       ??__EalgoLog@U2@@YAXXZ     100027c0 f   ORFQuery.obj
 0001:00001840       ??__EcmdLog@U2@@YAXXZ      10002840 f   ORFQuery.obj
 0001:000018c0       ??__EcoreLog@U2@@YAXXZ     100028c0 f   ORFQuery.obj
 0001:00001940       ??__EioLog@U2@@YAXXZ       10002940 f   ORFQuery.obj
 0001:000019c0       ??__EperfLog@U2@@YAXXZ     100029c0 f   ORFQuery.obj
 0001:00001a40       ??__EscriptLog@U2@@YAXXZ   10002a40 f   ORFQuery.obj
 0001:00001ac0       ??__EtaskLog@U2@@YAXXZ     10002ac0 f   ORFQuery.obj
 0001:00001b40       ??__EuiLog@U2@@YAXXZ       10002b40 f   ORFQuery.obj
 0001:00001bc0       ??__EuserActLog@U2@@YAXXZ  10002bc0 f   ORFQuery.obj
 0001:00001c40       ??__E?ACTOR_ID@ORFWorkerFactory@LocalWorkflow@U2@@2VQString@@B@@YAXXZ 10002c40 f   ORFWorker.obj
 0001:00001c60       ??__E?_Generic_object@?$_Error_objects@H@std@@2V_Generic_error_category@2@A@@YAXXZ 10002c60 f   ORFWorker.obj
 0001:00001c70       ??__E?_Iostream_object@?$_Error_objects@H@std@@2V_Iostream_error_category@2@A@@YAXXZ 10002c70 f   ORFWorker.obj
 0001:00001c80       ??__E?_System_object@?$_Error_objects@H@std@@2V_System_error_category@2@A@@YAXXZ 10002c80 f   ORFWorker.obj
 0001:00001c90       ??__EALT_ATTR@LocalWorkflow@U2@@YAXXZ 10002c90 f   ORFWorker.obj
 0001:00001cb0       ??__EFIT_ATTR@LocalWorkflow@U2@@YAXXZ 10002cb0 f   ORFWorker.obj
 0001:00001cd0       ??__EID_ATTR@LocalWorkflow@U2@@YAXXZ 10002cd0 f   ORFWorker.obj
 0001:00001cf0       ??__EINIT_ATTR@LocalWorkflow@U2@@YAXXZ 10002cf0 f   ORFWorker.obj
 0001:00001d10       ??__EISC_ATTR@LocalWorkflow@U2@@YAXXZ 10002d10 f   ORFWorker.obj
 0001:00001d30       ??__ELEN_ATTR@LocalWorkflow@U2@@YAXXZ 10002d30 f   ORFWorker.obj
 0001:00001d50       ??__ELIMIT_ATTR@LocalWorkflow@U2@@YAXXZ 10002d50 f   ORFWorker.obj
 0001:00001d70       ??__ENAME_ATTR@LocalWorkflow@U2@@YAXXZ 10002d70 f   ORFWorker.obj
 0001:00001d90       ??__ERES_ATTR@LocalWorkflow@U2@@YAXXZ 10002d90 f   ORFWorker.obj
 0001:00001db0       ??__EalgoLog@U2@@YAXXZ     10002db0 f   ORFWorker.obj
 0001:00001e30       ??__EcmdLog@U2@@YAXXZ      10002e30 f   ORFWorker.obj
 0001:00001eb0       ??__EcoreLog@U2@@YAXXZ     10002eb0 f   ORFWorker.obj
 0001:00001f30       ??__EioLog@U2@@YAXXZ       10002f30 f   ORFWorker.obj
 0001:00001fb0       ??__EperfLog@U2@@YAXXZ     10002fb0 f   ORFWorker.obj
 0001:00002030       ??__EscriptLog@U2@@YAXXZ   10003030 f   ORFWorker.obj
 0001:000020b0       ??__EtaskLog@U2@@YAXXZ     100030b0 f   ORFWorker.obj
 0001:00002130       ??__EuiLog@U2@@YAXXZ       10003130 f   ORFWorker.obj
 0001:000021b0       ??__EuserActLog@U2@@YAXXZ  100031b0 f   ORFWorker.obj
 0001:00002230       ??__E?_Generic_object@?$_Error_objects@H@std@@2V_Generic_error_category@2@A@@YAXXZ 10003230 f   moc_ORFDialog.obj
 0001:00002240       ??__E?_Iostream_object@?$_Error_objects@H@std@@2V_Iostream_error_category@2@A@@YAXXZ 10003240 f   moc_ORFDialog.obj
 0001:00002250       ??__E?_System_object@?$_Error_objects@H@std@@2V_System_error_category@2@A@@YAXXZ 10003250 f   moc_ORFDialog.obj
 0001:00002260       ??__E?staticMetaObject@ORFDialog@U2@@2UQMetaObject@@B@@YAXXZ 10003260 f   moc_ORFDialog.obj
 0001:00002270       ??__EalgoLog@U2@@YAXXZ     10003270 f   moc_ORFDialog.obj
 0001:000022f0       ??__EcmdLog@U2@@YAXXZ      100032f0 f   moc_ORFDialog.obj
 0001:00002370       ??__EcoreLog@U2@@YAXXZ     10003370 f   moc_ORFDialog.obj
 0001:000023f0       ??__EioLog@U2@@YAXXZ       100033f0 f   moc_ORFDialog.obj
 0001:00002470       ??__EperfLog@U2@@YAXXZ     10003470 f   moc_ORFDialog.obj
 0001:000024f0       ??__EscriptLog@U2@@YAXXZ   100034f0 f   moc_ORFDialog.obj
 0001:00002570       ??__EtaskLog@U2@@YAXXZ     10003570 f   moc_ORFDialog.obj
 0001:000025f0       ??__EuiLog@U2@@YAXXZ       100035f0 f   moc_ORFDialog.obj
 0001:00002670       ??__EuserActLog@U2@@YAXXZ  10003670 f   moc_ORFDialog.obj
 0001:000026f0       ??__E?_Generic_object@?$_Error_objects@H@std@@2V_Generic_error_category@2@A@@YAXXZ 100036f0 f   moc_ORFMarkerPlugin.obj
 0001:00002700       ??__E?_Iostream_object@?$_Error_objects@H@std@@2V_Iostream_error_category@2@A@@YAXXZ 10003700 f   moc_ORFMarkerPlugin.obj
 0001:00002710       ??__E?_System_object@?$_Error_objects@H@std@@2V_System_error_category@2@A@@YAXXZ 10003710 f   moc_ORFMarkerPlugin.obj
 0001:00002720       ??__E?staticMetaObject@ORFMarkerPlugin@U2@@2UQMetaObject@@B@@YAXXZ 10003720 f   moc_ORFMarkerPlugin.obj
 0001:00002730       ??__E?staticMetaObject@ORFViewContext@U2@@2UQMetaObject@@B@@YAXXZ 10003730 f   moc_ORFMarkerPlugin.obj
 0001:00002740       ??__EService_DNAExport@U2@@YAXXZ 10003740 f   moc_ORFMarkerPlugin.obj
 0001:00002750       ??__EService_DNAGraphPack@U2@@YAXXZ 10003750 f   moc_ORFMarkerPlugin.obj
 0001:00002760       ??__EService_ExternalToolSupport@U2@@YAXXZ 10003760 f   moc_ORFMarkerPlugin.obj
 0001:00002770       ??__EService_GUITesting@U2@@YAXXZ 10003770 f   moc_ORFMarkerPlugin.obj
 0001:00002780       ??__EService_MaxCoreServiceId@U2@@YAXXZ 10003780 f   moc_ORFMarkerPlugin.obj
 0001:00002790       ??__EService_MinCoreServiceId@U2@@YAXXZ 10003790 f   moc_ORFMarkerPlugin.obj
 0001:000027a0       ??__EService_PluginViewer@U2@@YAXXZ 100037a0 f   moc_ORFMarkerPlugin.obj
 0001:000027b0       ??__EService_Project@U2@@YAXXZ 100037b0 f   moc_ORFMarkerPlugin.obj
 0001:000027c0       ??__EService_ProjectView@U2@@YAXXZ 100037c0 f   moc_ORFMarkerPlugin.obj
 0001:000027d0       ??__EService_QueryDesigner@U2@@YAXXZ 100037d0 f   moc_ORFMarkerPlugin.obj
 0001:000027e0       ??__EService_ScriptRegistry@U2@@YAXXZ 100037e0 f   moc_ORFMarkerPlugin.obj
 0001:000027f0       ??__EService_TestRunner@U2@@YAXXZ 100037f0 f   moc_ORFMarkerPlugin.obj
 0001:00002800       ??__EService_WorkflowDesigner@U2@@YAXXZ 10003800 f   moc_ORFMarkerPlugin.obj
 0001:00002810       ??__E?_Generic_object@?$_Error_objects@H@std@@2V_Generic_error_category@2@A@@YAXXZ 10003810 f   moc_ORFMarkerTask.obj
 0001:00002820       ??__E?_Iostream_object@?$_Error_objects@H@std@@2V_Iostream_error_category@2@A@@YAXXZ 10003820 f   moc_ORFMarkerTask.obj
 0001:00002830       ??__E?_System_object@?$_Error_objects@H@std@@2V_System_error_category@2@A@@YAXXZ 10003830 f   moc_ORFMarkerTask.obj
 0001:00002840       ??__E?staticMetaObject@FindORFsToAnnotationsTask@U2@@2UQMetaObject@@B@@YAXXZ 10003840 f   moc_ORFMarkerTask.obj
 0001:00002850       ??__E?staticMetaObject@ORFAutoAnnotationsUpdater@U2@@2UQMetaObject@@B@@YAXXZ 10003850 f   moc_ORFMarkerTask.obj
 0001:00002860       ??__EalgoLog@U2@@YAXXZ     10003860 f   moc_ORFMarkerTask.obj
 0001:000028e0       ??__EcmdLog@U2@@YAXXZ      100038e0 f   moc_ORFMarkerTask.obj
 0001:00002960       ??__EcoreLog@U2@@YAXXZ     10003960 f   moc_ORFMarkerTask.obj
 0001:000029e0       ??__EioLog@U2@@YAXXZ       100039e0 f   moc_ORFMarkerTask.obj
 0001:00002a60       ??__EperfLog@U2@@YAXXZ     10003a60 f   moc_ORFMarkerTask.obj
 0001:00002ae0       ??__EscriptLog@U2@@YAXXZ   10003ae0 f   moc_ORFMarkerTask.obj
 0001:00002b60       ??__EtaskLog@U2@@YAXXZ     10003b60 f   moc_ORFMarkerTask.obj
 0001:00002be0       ??__EuiLog@U2@@YAXXZ       10003be0 f   moc_ORFMarkerTask.obj
 0001:00002c60       ??__EuserActLog@U2@@YAXXZ  10003c60 f   moc_ORFMarkerTask.obj
 0001:00002ce0       ??__E?_Generic_object@?$_Error_objects@H@std@@2V_Generic_error_category@2@A@@YAXXZ 10003ce0 f   moc_ORFMarkerTests.obj
 0001:00002cf0       ??__E?_Iostream_object@?$_Error_objects@H@std@@2V_Iostream_error_category@2@A@@YAXXZ 10003cf0 f   moc_ORFMarkerTests.obj
 0001:00002d00       ??__E?_System_object@?$_Error_objects@H@std@@2V_System_error_category@2@A@@YAXXZ 10003d00 f   moc_ORFMarkerTests.obj
 0001:00002d10       ??__E?staticMetaObject@GTest_ORFMarkerTask@U2@@2UQMetaObject@@B@@YAXXZ 10003d10 f   moc_ORFMarkerTests.obj
 0001:00002d20       ??__EService_DNAExport@U2@@YAXXZ 10003d20 f   moc_ORFMarkerTests.obj
 0001:00002d30       ??__EService_DNAGraphPack@U2@@YAXXZ 10003d30 f   moc_ORFMarkerTests.obj
 0001:00002d40       ??__EService_ExternalToolSupport@U2@@YAXXZ 10003d40 f   moc_ORFMarkerTests.obj
 0001:00002d50       ??__EService_GUITesting@U2@@YAXXZ 10003d50 f   moc_ORFMarkerTests.obj
 0001:00002d60       ??__EService_MaxCoreServiceId@U2@@YAXXZ 10003d60 f   moc_ORFMarkerTests.obj
 0001:00002d70       ??__EService_MinCoreServiceId@U2@@YAXXZ 10003d70 f   moc_ORFMarkerTests.obj
 0001:00002d80       ??__EService_PluginViewer@U2@@YAXXZ 10003d80 f   moc_ORFMarkerTests.obj
 0001:00002d90       ??__EService_Project@U2@@YAXXZ 10003d90 f   moc_ORFMarkerTests.obj
 0001:00002da0       ??__EService_ProjectView@U2@@YAXXZ 10003da0 f   moc_ORFMarkerTests.obj
 0001:00002db0       ??__EService_QueryDesigner@U2@@YAXXZ 10003db0 f   moc_ORFMarkerTests.obj
 0001:00002dc0       ??__EService_ScriptRegistry@U2@@YAXXZ 10003dc0 f   moc_ORFMarkerTests.obj
 0001:00002dd0       ??__EService_TestRunner@U2@@YAXXZ 10003dd0 f   moc_ORFMarkerTests.obj
 0001:00002de0       ??__EService_WorkflowDesigner@U2@@YAXXZ 10003de0 f   moc_ORFMarkerTests.obj
 0001:00002df0       ??__EalgoLog@U2@@YAXXZ     10003df0 f   moc_ORFMarkerTests.obj
 0001:00002e70       ??__EcmdLog@U2@@YAXXZ      10003e70 f   moc_ORFMarkerTests.obj
 0001:00002ef0       ??__EcoreLog@U2@@YAXXZ     10003ef0 f   moc_ORFMarkerTests.obj
 0001:00002f70       ??__EioLog@U2@@YAXXZ       10003f70 f   moc_ORFMarkerTests.obj
 0001:00002ff0       ??__EperfLog@U2@@YAXXZ     10003ff0 f   moc_ORFMarkerTests.obj
 0001:00003070       ??__EscriptLog@U2@@YAXXZ   10004070 f   moc_ORFMarkerTests.obj
 0001:000030f0       ??__EtaskLog@U2@@YAXXZ     100040f0 f   moc_ORFMarkerTests.obj
 0001:00003170       ??__EuiLog@U2@@YAXXZ       10004170 f   moc_ORFMarkerTests.obj
 0001:000031f0       ??__EuserActLog@U2@@YAXXZ  100041f0 f   moc_ORFMarkerTests.obj
 0001:00003270       ??__E?_Generic_object@?$_Error_objects@H@std@@2V_Generic_error_category@2@A@@YAXXZ 10004270 f   moc_ORFQuery.obj
 0001:00003280       ??__E?_Iostream_object@?$_Error_objects@H@std@@2V_Iostream_error_category@2@A@@YAXXZ 10004280 f   moc_ORFQuery.obj
 0001:00003290       ??__E?_System_object@?$_Error_objects@H@std@@2V_System_error_category@2@A@@YAXXZ 10004290 f   moc_ORFQuery.obj
 0001:000032a0       ??__E?staticMetaObject@QDORFActor@U2@@2UQMetaObject@@B@@YAXXZ 100042a0 f   moc_ORFQuery.obj
 0001:000032b0       ??__EalgoLog@U2@@YAXXZ     100042b0 f   moc_ORFQuery.obj
 0001:00003330       ??__EcmdLog@U2@@YAXXZ      10004330 f   moc_ORFQuery.obj
 0001:000033b0       ??__EcoreLog@U2@@YAXXZ     100043b0 f   moc_ORFQuery.obj
 0001:00003430       ??__EioLog@U2@@YAXXZ       10004430 f   moc_ORFQuery.obj
 0001:000034b0       ??__EperfLog@U2@@YAXXZ     100044b0 f   moc_ORFQuery.obj
 0001:00003530       ??__EscriptLog@U2@@YAXXZ   10004530 f   moc_ORFQuery.obj
 0001:000035b0       ??__EtaskLog@U2@@YAXXZ     100045b0 f   moc_ORFQuery.obj
 0001:00003630       ??__EuiLog@U2@@YAXXZ       10004630 f   moc_ORFQuery.obj
 0001:000036b0       ??__EuserActLog@U2@@YAXXZ  100046b0 f   moc_ORFQuery.obj
 0001:00003730       ??__E?_Generic_object@?$_Error_objects@H@std@@2V_Generic_error_category@2@A@@YAXXZ 10004730 f   moc_ORFWorker.obj
 0001:00003740       ??__E?_Iostream_object@?$_Error_objects@H@std@@2V_Iostream_error_category@2@A@@YAXXZ 10004740 f   moc_ORFWorker.obj
 0001:00003750       ??__E?_System_object@?$_Error_objects@H@std@@2V_System_error_category@2@A@@YAXXZ 10004750 f   moc_ORFWorker.obj
 0001:00003760       ??__E?staticMetaObject@ORFPrompter@LocalWorkflow@U2@@2UQMetaObject@@B@@YAXXZ 10004760 f   moc_ORFWorker.obj
 0001:00003770       ??__E?staticMetaObject@ORFWorker@LocalWorkflow@U2@@2UQMetaObject@@B@@YAXXZ 10004770 f   moc_ORFWorker.obj
 0001:00003780       ??__EalgoLog@U2@@YAXXZ     10004780 f   moc_ORFWorker.obj
 0001:00003800       ??__EcmdLog@U2@@YAXXZ      10004800 f   moc_ORFWorker.obj
 0001:00003880       ??__EcoreLog@U2@@YAXXZ     10004880 f   moc_ORFWorker.obj
 0001:00003900       ??__EioLog@U2@@YAXXZ       10004900 f   moc_ORFWorker.obj
 0001:00003980       ??__EperfLog@U2@@YAXXZ     10004980 f   moc_ORFWorker.obj
 0001:00003a00       ??__EscriptLog@U2@@YAXXZ   10004a00 f   moc_ORFWorker.obj
 0001:00003a80       ??__EtaskLog@U2@@YAXXZ     10004a80 f   moc_ORFWorker.obj
 0001:00003b00       ??__EuiLog@U2@@YAXXZ       10004b00 f   moc_ORFWorker.obj
 0001:00003b80       ??__EuserActLog@U2@@YAXXZ  10004b80 f   moc_ORFWorker.obj
 0001:00003c00       ??__Edummy@?A0xaf06a44c@@YAXXZ 10004c00 f   qrc_orf_marker.obj
 0001:000041ce       __catch$??0?$QList@PAVQAction@@@@QAE@ABV0@@Z$0 100051ce f i ORFDialog.obj
 0001:0000428e       __catch$??0?$QList@PAVTask@U2@@@@QAE@ABV0@@Z$0 1000528e f i ORFDialog.obj
 0001:0000435e       __catch$??0?$QList@UTriplet@U2@@@@QAE@ABV0@@Z$0 1000535e f i ORFDialog.obj
 0001:0000442e       __catch$??0?$QList@VORFFindResult@U2@@@@QAE@ABV0@@Z$0 1000542e f i ORFDialog.obj
 0001:000057b0       ??R<lambda_0a0e7f32f0abf4fe998f0c4219dad45a>@@QBE?AVQString@@XZ 100067b0 f   ORFDialog.obj
 0001:000057d0       ??R<lambda_0ff5d552fbbf7817874d60f1df8acf29>@@QBE?AVQString@@XZ 100067d0 f   ORFDialog.obj
 0001:000057f0       ??R<lambda_1dd36e8e753f070291a4e308cf29c03c>@@QBE?AVQString@@XZ 100067f0 f   ORFDialog.obj
 0001:00005810       ??R<lambda_220f8f8c5ecf4ac023635268940e37e3>@@QBE?AVQString@@XZ 10006810 f   ORFDialog.obj
 0001:00005830       ??R<lambda_341cb0a24dbb67dcf78c26228121c09a>@@QBE?AVQString@@XZ 10006830 f   ORFDialog.obj
 0001:00005850       ??R<lambda_3bd8f2f42d9c55363ea1b95aa573d950>@@QBE?AVQString@@XZ 10006850 f   ORFDialog.obj
 0001:00005870       ??R<lambda_44e65958acee4170841d4644da5d91a6>@@QBE?AVQString@@XZ 10006870 f   ORFDialog.obj
 0001:00005890       ??R<lambda_4655343fe23bb4b3b7882e1f3316a452>@@QBE?AVQString@@XZ 10006890 f   ORFDialog.obj
 0001:000058b0       ??R<lambda_46cc8f107b08cda0fe36f9525d4f10d7>@@QBE?AVQString@@XZ 100068b0 f   ORFDialog.obj
 0001:000058d0       ??R<lambda_50b3e03a63dfd75480240ba88917e908>@@QBE?AVQString@@XZ 100068d0 f   ORFDialog.obj
 0001:000058f0       ??R<lambda_52fe59cca71e9c144ba25b49fc880329>@@QBE?AVQString@@XZ 100068f0 f   ORFDialog.obj
 0001:00005910       ??R<lambda_633eb662894a0f52b681d98c902f4666>@@QBE?AVQString@@XZ 10006910 f   ORFDialog.obj
 0001:00005930       ??R<lambda_6b04bc410d0484eb77773aabbb2121e7>@@QBE?AVQString@@XZ 10006930 f   ORFDialog.obj
 0001:00005950       ??R<lambda_6cda75d66740ac343a5306b8d47f27c7>@@QBE?AVQString@@XZ 10006950 f   ORFDialog.obj
 0001:00005970       ??R<lambda_6e91e825d1cfc04223738cd463f9b99e>@@QBE?AVQString@@XZ 10006970 f   ORFDialog.obj
 0001:00005990       ??R<lambda_727dfb955ba445b1d6e1c6e761ef9880>@@QBE?AVQString@@XZ 10006990 f   ORFDialog.obj
 0001:000059b0       ??R<lambda_7a879637595ff6229c926fc23ea90814>@@QBE?AVQString@@XZ 100069b0 f   ORFDialog.obj
 0001:000059d0       ??R<lambda_81b46f5ffcbd23e97e4414d4b5d9aa96>@@QBE?AVQString@@XZ 100069d0 f   ORFDialog.obj
 0001:000059f0       ??R<lambda_95d7ce4a46ac2420c3ef42b00d6e46c6>@@QBE?AVQString@@XZ 100069f0 f   ORFDialog.obj
 0001:00005a10       ??R<lambda_9f8f56f1a1953070dc5e6b8678d8115f>@@QBE?AVQString@@XZ 10006a10 f   ORFDialog.obj
 0001:00005a30       ??R<lambda_a9859d689698127f97835ff63b5de490>@@QBE?AVQString@@XZ 10006a30 f   ORFDialog.obj
 0001:00005a50       ??R<lambda_bd58d910664159c2d4adc7a129b025ac>@@QBE?AVQString@@XZ 10006a50 f   ORFDialog.obj
 0001:00005a70       ??R<lambda_c5b2208d484aab5eeda4b4e8d9e81a71>@@QBE?AVQString@@XZ 10006a70 f   ORFDialog.obj
 0001:00005a90       ??R<lambda_c934430d2d61852a3610e57fc7181a03>@@QBE?AVQString@@XZ 10006a90 f   ORFDialog.obj
 0001:00005ab0       ??R<lambda_c9ff954e0b34c3c8e5fae69c2fe05e0b>@@QBE?AVQString@@XZ 10006ab0 f   ORFDialog.obj
 0001:00005ad0       ??R<lambda_ca85f9d6613aef30f18329a26b64b6d3>@@QBE?AVQString@@XZ 10006ad0 f   ORFDialog.obj
 0001:00005af0       ??R<lambda_cb8147e3c8b49d91b9201acf92d06490>@@QBE?AVQString@@XZ 10006af0 f   ORFDialog.obj
 0001:00005b10       ??R<lambda_cb920ba896b73d37c549d63b6b5320cc>@@QBE?AVQString@@XZ 10006b10 f   ORFDialog.obj
 0001:00005b30       ??R<lambda_cd7c1f4a134beb52c9cbdd3b6ce610db>@@QBE?AVQString@@XZ 10006b30 f   ORFDialog.obj
 0001:00005b50       ??R<lambda_cf8fd9af3f824ea42de5b8d51851b3e7>@@QBE?AVQString@@XZ 10006b50 f   ORFDialog.obj
 0001:00005b70       ??R<lambda_d0d42478d3362983368102e03c7eeecb>@@QBE?AVQString@@XZ 10006b70 f   ORFDialog.obj
 0001:00005b90       ??R<lambda_d9d5d6d4341da3ae04a63bbef4f4d8fd>@@QBE?AVQString@@XZ 10006b90 f   ORFDialog.obj
 0001:00005bb0       ??R<lambda_e114dfc637b50f53a12623c298138117>@@QBE?AVQString@@XZ 10006bb0 f   ORFDialog.obj
 0001:00005bd0       ??R<lambda_e38c0bfbbb0434d86bd5f34b32af9382>@@QBE?AVQString@@XZ 10006bd0 f   ORFDialog.obj
 0001:00005bf0       ??R<lambda_e718f0b57f7aaf937d0d3b715c431104>@@QBE?AVQString@@XZ 10006bf0 f   ORFDialog.obj
 0001:00005c10       ??R<lambda_ea7e40f3c293bc0745c9796f572004af>@@QBE?AVQString@@XZ 10006c10 f   ORFDialog.obj
 0001:00005c30       ??R<lambda_f4b85fea6c6cf4d9c35c782cf8237f89>@@QBE?AVQString@@XZ 10006c30 f   ORFDialog.obj
 0001:00005c50       ??R<lambda_f746202d42af9037ea860442f08e949b>@@QBE?AVQString@@XZ 10006c50 f   ORFDialog.obj
 0001:000064a6       __catch$?_Copy@?$basic_string@DU?$char_traits@D@std@@V?$allocator@D@2@@std@@QAEXII@Z$0 100074a6 f i ORFDialog.obj
 0001:000064e3       __catch$?_Copy@?$basic_string@DU?$char_traits@D@std@@V?$allocator@D@2@@std@@QAEXII@Z$1 100074e3 f i ORFDialog.obj
 0001:00007134       __catch$?createNode@?$QMapData@W4DNATranslationRole@U2@@V?$QList@UTriplet@U2@@@@@@QAEPAU?$QMapNode@W4DNATranslationRole@U2@@V?$QList@UTriplet@U2@@@@@@ABW4DNATranslationRole@U2@@ABV?$QList@UTriplet@U2@@@@PAU2@_N@Z$2 10008134 f i ORFDialog.obj
 0001:00007140       __catch$?createNode@?$QMapData@W4DNATranslationRole@U2@@V?$QList@UTriplet@U2@@@@@@QAEPAU?$QMapNode@W4DNATranslationRole@U2@@V?$QList@UTriplet@U2@@@@@@ABW4DNATranslationRole@U2@@ABV?$QList@UTriplet@U2@@@@PAU2@_N@Z$0 10008140 f i ORFDialog.obj
 0001:00008544       __catch$?node_copy@?$QList@UTriplet@U2@@@@AAEXPAUNode@1@00@Z$0 10009544 f i ORFDialog.obj
 0001:00008604       __catch$?node_copy@?$QList@VORFFindResult@U2@@@@AAEXPAUNode@1@00@Z$0 10009604 f i ORFDialog.obj
 0001:0000b6b0       ?triplet2str@U2@@YA?AVQString@@ABUTriplet@1@@Z 1000c6b0 f   ORFDialog.obj
 0001:0000bc3e       __catch$??0?$QList@PAVXMLTestFactory@U2@@@@QAE@ABV0@@Z$0 1000cc3e f i ORFMarkerPlugin.obj
 0001:0000c7f5       __catch$?append@?$QList@PAVXMLTestFactory@U2@@@@QAEXABQAVXMLTestFactory@U2@@@Z$4 1000d7f5 f i ORFMarkerPlugin.obj
 0001:0000cb51       __catch$?detach_helper_grow@?$QList@PAVXMLTestFactory@U2@@@@AAEPAUNode@1@HH@Z$0 1000db51 f i ORFMarkerPlugin.obj
 0001:0000cb51       __catch$?detach_helper_grow@?$QList@PAVXMLTestFactory@U2@@@@AAEPAUNode@1@HH@Z$2 1000db51 f i ORFMarkerPlugin.obj
 0001:0000d885       __catch$?append@?$QList@PAVTask@U2@@@@QAEXABQAVTask@U2@@@Z$4 1000e885 f i ORFMarkerTask.obj
 0001:0000d942       __catch$?append@?$QList@V?$QSharedDataPointer@VAnnotationData@U2@@@@@@QAEXABV?$QSharedDataPointer@VAnnotationData@U2@@@@@Z$4 1000e942 f i ORFMarkerTask.obj
 0001:0000dcc1       __catch$?detach_helper_grow@?$QList@PAVTask@U2@@@@AAEPAUNode@1@HH@Z$0 1000ecc1 f i ORFMarkerTask.obj
 0001:0000dcc1       __catch$?detach_helper_grow@?$QList@PAVTask@U2@@@@AAEPAUNode@1@HH@Z$2 1000ecc1 f i ORFMarkerTask.obj
 0001:0000ddec       __catch$?detach_helper_grow@?$QList@V?$QSharedDataPointer@VAnnotationData@U2@@@@@@AAEPAUNode@1@HH@Z$2 1000edec f i ORFMarkerTask.obj
 0001:0000de27       __catch$?detach_helper_grow@?$QList@V?$QSharedDataPointer@VAnnotationData@U2@@@@@@AAEPAUNode@1@HH@Z$0 1000ee27 f i ORFMarkerTask.obj
 0001:0000efde       __catch$??0?$QList@VQString@@@@QAE@ABV0@@Z$0 1000ffde f i ORFMarkerTests.obj
 0001:0000f5f1       __catch$?detach_helper@?$QList@VQString@@@@AAEXH@Z$0 100105f1 f i ORFMarkerTests.obj
 0001:00010492       __catch$?node_copy@?$QList@VQString@@@@AAEXPAUNode@1@00@Z$2 10011492 f i ORFMarkerTests.obj
 0001:00010825       __catch$?reallocData@?$QVector@VU2Region@U2@@@@AAEXHHV?$QFlags@W4AllocationOption@QArrayData@@@@@Z$0 10011825 f i ORFMarkerTests.obj
 0001:00010837       __catch$?reallocData@?$QVector@VU2Region@U2@@@@AAEXHHV?$QFlags@W4AllocationOption@QArrayData@@@@@Z$2 10011837 f i ORFMarkerTests.obj
 0001:0001116e       __catch$??0?$QList@PAVDNATranslation@U2@@@@QAE@ABV0@@Z$0 1001216e f i ORFQuery.obj
 0001:0001122e       __catch$??0?$QList@PAVORFFindTask@U2@@@@QAE@ABV0@@Z$0 1001222e f i ORFQuery.obj
 0001:000112fe       __catch$??0?$QList@V?$QSharedDataPointer@VAnnotationData@U2@@@@@@QAE@ABV0@@Z$0 100122fe f i ORFQuery.obj
 0001:00012cda       __catch$??Y?$QList@VORFFindResult@U2@@@@QAEAAV0@ABV0@@Z$0 10013cda f i ORFQuery.obj
 0001:00013045       __catch$?append@?$QList@PAVAttribute@U2@@@@QAEXABQAVAttribute@U2@@@Z$4 10014045 f i ORFQuery.obj
 0001:000130d5       __catch$?append@?$QList@PAVORFFindTask@U2@@@@QAEXABQAVORFFindTask@U2@@@Z$4 100140d5 f i ORFQuery.obj
 0001:000135a5       __catch$?createNode@?$QMapData@VQString@@PAVPropertyDelegate@U2@@@@QAEPAU?$QMapNode@VQString@@PAVPropertyDelegate@U2@@@@ABVQString@@ABQAVPropertyDelegate@U2@@PAU2@_N@Z$2 100145a5 f i ORFQuery.obj
 0001:00013645       __catch$?createNode@?$QMapData@VQString@@PAVQDSchemeUnit@U2@@@@QAEPAU?$QMapNode@VQString@@PAVQDSchemeUnit@U2@@@@ABVQString@@ABQAVQDSchemeUnit@U2@@PAU2@_N@Z$2 10014645 f i ORFQuery.obj
 0001:000136ee       __catch$?createNode@?$QMapData@VQString@@VQVariant@@@@QAEPAU?$QMapNode@VQString@@VQVariant@@@@ABVQString@@ABVQVariant@@PAU2@_N@Z$0 100146ee f i ORFQuery.obj
 0001:00013703       __catch$?createNode@?$QMapData@VQString@@VQVariant@@@@QAEPAU?$QMapNode@VQString@@VQVariant@@@@ABVQString@@ABVQVariant@@PAU2@_N@Z$2 10014703 f i ORFQuery.obj
 0001:00013df1       __catch$?detach_helper_grow@?$QList@PAVAttribute@U2@@@@AAEPAUNode@1@HH@Z$0 10014df1 f i ORFQuery.obj
 0001:00013df1       __catch$?detach_helper_grow@?$QList@PAVAttribute@U2@@@@AAEPAUNode@1@HH@Z$2 10014df1 f i ORFQuery.obj
 0001:00013f01       __catch$?detach_helper_grow@?$QList@PAVORFFindTask@U2@@@@AAEPAUNode@1@HH@Z$2 10014f01 f i ORFQuery.obj
 0001:00013f01       __catch$?detach_helper_grow@?$QList@PAVORFFindTask@U2@@@@AAEPAUNode@1@HH@Z$0 10014f01 f i ORFQuery.obj
 0001:00014041       __catch$?detach_helper_grow@?$QList@VORFFindResult@U2@@@@AAEPAUNode@1@HH@Z$2 10015041 f i ORFQuery.obj
 0001:0001407c       __catch$?detach_helper_grow@?$QList@VORFFindResult@U2@@@@AAEPAUNode@1@HH@Z$0 1001507c f i ORFQuery.obj
 0001:00016c3e       __catch$??0?$QList@PAVPort@Workflow@U2@@@@QAE@ABV0@@Z$0 10017c3e f i ORFWorker.obj
 0001:00016d3e       __catch$??0?$QList@VDescriptor@U2@@@@QAE@ABV0@@Z$0 10017d3e f i ORFWorker.obj
 0001:00017ba5       __catch$?append@?$QList@PAVPortDescriptor@Workflow@U2@@@@QAEXABQAVPortDescriptor@Workflow@U2@@@Z$4 10018ba5 f i ORFWorker.obj
 0001:00017c02       __catch$?append@?$QList@U?$QPair@VQString@@VQVariant@@@@@@QAEXABU?$QPair@VQString@@VQVariant@@@@@Z$0 10018c02 f i ORFWorker.obj
 0001:00017c02       __catch$?append@?$QList@U?$QPair@VQString@@VQVariant@@@@@@QAEXABU?$QPair@VQString@@VQVariant@@@@@Z$2 10018c02 f i ORFWorker.obj
 0001:00017cec       __catch$?append@?$QList@VDescriptor@U2@@@@QAEXABVDescriptor@U2@@@Z$0 10018cec f i ORFWorker.obj
 0001:00017cec       __catch$?append@?$QList@VDescriptor@U2@@@@QAEXABVDescriptor@U2@@@Z$2 10018cec f i ORFWorker.obj
 0001:00018b5d       __catch$?createNode@?$QMapData@VDescriptor@U2@@V?$QExplicitlySharedDataPointer@VDataType@U2@@@@@@QAEPAU?$QMapNode@VDescriptor@U2@@V?$QExplicitlySharedDataPointer@VDataType@U2@@@@@@ABVDescriptor@U2@@ABV?$QExplicitlySharedDataPointer@VDataType@U2@@@@PAU2@_N@Z$2 10019b5d f i ORFWorker.obj
 0001:00018c0e       __catch$?createNode@?$QMapData@VQString@@VQScriptValue@@@@QAEPAU?$QMapNode@VQString@@VQScriptValue@@@@ABVQString@@ABVQScriptValue@@PAU2@_N@Z$0 10019c0e f i ORFWorker.obj
 0001:00018c23       __catch$?createNode@?$QMapData@VQString@@VQScriptValue@@@@QAEPAU?$QMapNode@VQString@@VQScriptValue@@@@ABVQString@@ABVQScriptValue@@PAU2@_N@Z$2 10019c23 f i ORFWorker.obj
 0001:00018f4a       __catch$?detach_helper@?$QList@VDescriptor@U2@@@@AAEXH@Z$0 10019f4a f i ORFWorker.obj
 0001:00019161       __catch$?detach_helper_grow@?$QList@PAVPortDescriptor@Workflow@U2@@@@AAEPAUNode@1@HH@Z$2 1001a161 f i ORFWorker.obj
 0001:00019161       __catch$?detach_helper_grow@?$QList@PAVPortDescriptor@Workflow@U2@@@@AAEPAUNode@1@HH@Z$0 1001a161 f i ORFWorker.obj
 0001:0001928c       __catch$?detach_helper_grow@?$QList@U?$QPair@VQString@@VQVariant@@@@@@AAEPAUNode@1@HH@Z$2 1001a28c f i ORFWorker.obj
 0001:000192c7       __catch$?detach_helper_grow@?$QList@U?$QPair@VQString@@VQVariant@@@@@@AAEPAUNode@1@HH@Z$0 1001a2c7 f i ORFWorker.obj
 0001:000193df       __catch$?detach_helper_grow@?$QList@VDescriptor@U2@@@@AAEPAUNode@1@HH@Z$2 1001a3df f i ORFWorker.obj
 0001:0001941a       __catch$?detach_helper_grow@?$QList@VDescriptor@U2@@@@AAEPAUNode@1@HH@Z$0 1001a41a f i ORFWorker.obj
 0001:000195d0       ?getStrand@LocalWorkflow@U2@@YA?AW4ORFAlgorithmStrand@2@ABVQString@@@Z 1001a5d0 f   ORFWorker.obj
 0001:0001b59b       __catch$?node_copy@?$QList@U?$QPair@VQString@@VQVariant@@@@@@AAEXPAUNode@1@00@Z$0 1001c59b f i ORFWorker.obj
 0001:0001b685       __catch$?node_copy@?$QList@VDescriptor@U2@@@@AAEXPAUNode@1@00@Z$0 1001c685 f i ORFWorker.obj
 0001:0001c980       $LN35                      1001d980     moc_ORFDialog.obj
 0001:0001e956       _pre_c_init                1001f956 f   MSVCRT:crtdll.obj
 0001:0001ebc3       ___DllMainCRTStartup       1001fbc3 f   MSVCRT:crtdll.obj
 0001:0001ed10       $$000000                   1001fd10     MSVCRT:sehprolg4.obj
 0001:0001f125       ?ArrayUnwindFilter@@YAHPAU_EXCEPTION_POINTERS@@@Z 10020125 f   MSVCRT:ehvecdtr.obj
 0001:0001f470       __unwindfunclet$??$qRegisterMetaType@PAVQAction@@@@YAHPBDPAPAVQAction@@W4DefinedType@?$MetaTypeDefinedHelper@PAVQAction@@$00@QtPrivate@@@Z$0 10020470 f   ORFDialog.obj
 0001:0001f479       __ehhandler$??$qRegisterMetaType@PAVQAction@@@@YAHPBDPAPAVQAction@@W4DefinedType@?$MetaTypeDefinedHelper@PAVQAction@@$00@QtPrivate@@@Z 10020479 f   ORFDialog.obj
 0001:0001f4a0       __ehhandler$??0?$QList@PAVQAction@@@@QAE@ABV0@@Z 100204a0 f   ORFDialog.obj
 0001:0001f4c0       __ehhandler$??0?$QList@PAVTask@U2@@@@QAE@ABV0@@Z 100204c0 f   ORFDialog.obj
 0001:0001f4e0       __ehhandler$??0?$QList@UTriplet@U2@@@@QAE@ABV0@@Z 100204e0 f   ORFDialog.obj
 0001:0001f500       __ehhandler$??0?$QList@VORFFindResult@U2@@@@QAE@ABV0@@Z 10020500 f   ORFDialog.obj
 0001:0001f520       __unwindfunclet$??0ORFDialog@U2@@QAE@PAVADVSequenceObjectContext@1@@Z$0 10020520 f   ORFDialog.obj
 0001:0001f529       __unwindfunclet$??0ORFDialog@U2@@QAE@PAVADVSequenceObjectContext@1@@Z$1 10020529 f   ORFDialog.obj
 0001:0001f534       __unwindfunclet$??0ORFDialog@U2@@QAE@PAVADVSequenceObjectContext@1@@Z$2 10020534 f   ORFDialog.obj
 0001:0001f54e       __unwindfunclet$??0ORFDialog@U2@@QAE@PAVADVSequenceObjectContext@1@@Z$3 1002054e f   ORFDialog.obj
 0001:0001f557       __unwindfunclet$??0ORFDialog@U2@@QAE@PAVADVSequenceObjectContext@1@@Z$4 10020557 f   ORFDialog.obj
 0001:0001f560       __unwindfunclet$??0ORFDialog@U2@@QAE@PAVADVSequenceObjectContext@1@@Z$5 10020560 f   ORFDialog.obj
 0001:0001f56b       __unwindfunclet$??0ORFDialog@U2@@QAE@PAVADVSequenceObjectContext@1@@Z$7 1002056b f   ORFDialog.obj
 0001:0001f576       __unwindfunclet$??0ORFDialog@U2@@QAE@PAVADVSequenceObjectContext@1@@Z$10 10020576 f   ORFDialog.obj
 0001:0001f57e       __unwindfunclet$??0ORFDialog@U2@@QAE@PAVADVSequenceObjectContext@1@@Z$11 1002057e f   ORFDialog.obj
 0001:0001f586       __unwindfunclet$??0ORFDialog@U2@@QAE@PAVADVSequenceObjectContext@1@@Z$12 10020586 f   ORFDialog.obj
 0001:0001f58f       __unwindfunclet$??0ORFDialog@U2@@QAE@PAVADVSequenceObjectContext@1@@Z$13 1002058f f   ORFDialog.obj
 0001:0001f598       __unwindfunclet$??0ORFDialog@U2@@QAE@PAVADVSequenceObjectContext@1@@Z$16 10020598 f   ORFDialog.obj
 0001:0001f5a1       __ehhandler$??0ORFDialog@U2@@QAE@PAVADVSequenceObjectContext@1@@Z 100205a1 f   ORFDialog.obj
 0001:0001f5c0       __unwindfunclet$??0ORFListItem@U2@@QAE@ABVORFFindResult@1@@Z$0 100205c0 f   ORFDialog.obj
 0001:0001f5c9       __unwindfunclet$??0ORFListItem@U2@@QAE@ABVORFFindResult@1@@Z$1 100205c9 f   ORFDialog.obj
 0001:0001f5d2       __unwindfunclet$??0ORFListItem@U2@@QAE@ABVORFFindResult@1@@Z$2 100205d2 f   ORFDialog.obj
 0001:0001f5db       __unwindfunclet$??0ORFListItem@U2@@QAE@ABVORFFindResult@1@@Z$3 100205db f   ORFDialog.obj
 0001:0001f5e4       __unwindfunclet$??0ORFListItem@U2@@QAE@ABVORFFindResult@1@@Z$4 100205e4 f   ORFDialog.obj
 0001:0001f5ed       __unwindfunclet$??0ORFListItem@U2@@QAE@ABVORFFindResult@1@@Z$5 100205ed f   ORFDialog.obj
 0001:0001f5f6       __unwindfunclet$??0ORFListItem@U2@@QAE@ABVORFFindResult@1@@Z$6 100205f6 f   ORFDialog.obj
 0001:0001f5ff       __unwindfunclet$??0ORFListItem@U2@@QAE@ABVORFFindResult@1@@Z$7 100205ff f   ORFDialog.obj
 0001:0001f608       __unwindfunclet$??0ORFListItem@U2@@QAE@ABVORFFindResult@1@@Z$8 10020608 f   ORFDialog.obj
 0001:0001f611       __unwindfunclet$??0ORFListItem@U2@@QAE@ABVORFFindResult@1@@Z$9 10020611 f   ORFDialog.obj
 0001:0001f62b       __unwindfunclet$??0ORFListItem@U2@@QAE@ABVORFFindResult@1@@Z$10 1002062b f   ORFDialog.obj
 0001:0001f645       __unwindfunclet$??0ORFListItem@U2@@QAE@ABVORFFindResult@1@@Z$11 10020645 f   ORFDialog.obj
 0001:0001f64e       __unwindfunclet$??0ORFListItem@U2@@QAE@ABVORFFindResult@1@@Z$12 1002064e f   ORFDialog.obj
 0001:0001f657       __unwindfunclet$??0ORFListItem@U2@@QAE@ABVORFFindResult@1@@Z$13 10020657 f   ORFDialog.obj
 0001:0001f660       __unwindfunclet$??0ORFListItem@U2@@QAE@ABVORFFindResult@1@@Z$14 10020660 f   ORFDialog.obj
 0001:0001f669       __unwindfunclet$??0ORFListItem@U2@@QAE@ABVORFFindResult@1@@Z$15 10020669 f   ORFDialog.obj
 0001:0001f672       __ehhandler$??0ORFListItem@U2@@QAE@ABVORFFindResult@1@@Z 10020672 f   ORFDialog.obj
 0001:0001f690       __unwindfunclet$??A?$QMap@W4DNATranslationRole@U2@@V?$QList@UTriplet@U2@@@@@@QAEAAV?$QList@UTriplet@U2@@@@ABW4DNATranslationRole@U2@@@Z$0 10020690 f   ORFDialog.obj
 0001:0001f698       __ehhandler$??A?$QMap@W4DNATranslationRole@U2@@V?$QList@UTriplet@U2@@@@@@QAEAAV?$QList@UTriplet@U2@@@@ABW4DNATranslationRole@U2@@@Z 10020698 f   ORFDialog.obj
 0001:0001f6c0       __unwindfunclet$??H@YA?BVQString@@ABV0@0@Z$0 100206c0 f   ORFDialog.obj
 0001:0001f6da       __ehhandler$??H@YA?BVQString@@ABV0@0@Z 100206da f   ORFDialog.obj
 0001:0001f700       __unwindfunclet$??H@YA?BVQString@@ABV0@PBD@Z$0 10020700 f   ORFDialog.obj
 0001:0001f71a       __unwindfunclet$??H@YA?BVQString@@ABV0@PBD@Z$1 1002071a f   ORFDialog.obj
 0001:0001f723       __ehhandler$??H@YA?BVQString@@ABV0@PBD@Z 10020723 f   ORFDialog.obj
 0001:0001f740       __unwindfunclet$??H@YA?BVQString@@PBDABV0@@Z$0 10020740 f   ORFDialog.obj
 0001:0001f75a       __ehhandler$??H@YA?BVQString@@PBDABV0@@Z 1002075a f   ORFDialog.obj
 0001:0001f780       __unwindfunclet$??MORFListItem@U2@@UBE_NABVQTreeWidgetItem@@@Z$0 10020780 f   ORFDialog.obj
 0001:0001f789       __unwindfunclet$??MORFListItem@U2@@UBE_NABVQTreeWidgetItem@@@Z$1 10020789 f   ORFDialog.obj
 0001:0001f792       __ehhandler$??MORFListItem@U2@@UBE_NABVQTreeWidgetItem@@@Z 10020792 f   ORFDialog.obj
 0001:0001f7b0       __unwindfunclet$??__EalgoLog@U2@@YAXXZ$0 100207b0 f   ORFDialog.obj
 0001:0001f7b9       __ehhandler$??__EalgoLog@U2@@YAXXZ 100207b9 f   ORFDialog.obj
 0001:0001f7e0       __unwindfunclet$??__EcmdLog@U2@@YAXXZ$0 100207e0 f   ORFDialog.obj
 0001:0001f7e9       __ehhandler$??__EcmdLog@U2@@YAXXZ 100207e9 f   ORFDialog.obj
 0001:0001f810       __unwindfunclet$??__EcoreLog@U2@@YAXXZ$0 10020810 f   ORFDialog.obj
 0001:0001f819       __ehhandler$??__EcoreLog@U2@@YAXXZ 10020819 f   ORFDialog.obj
 0001:0001f840       __unwindfunclet$??__EioLog@U2@@YAXXZ$0 10020840 f   ORFDialog.obj
 0001:0001f849       __ehhandler$??__EioLog@U2@@YAXXZ 10020849 f   ORFDialog.obj
 0001:0001f870       __unwindfunclet$??__EperfLog@U2@@YAXXZ$0 10020870 f   ORFDialog.obj
 0001:0001f879       __ehhandler$??__EperfLog@U2@@YAXXZ 10020879 f   ORFDialog.obj
 0001:0001f8a0       __unwindfunclet$??__EscriptLog@U2@@YAXXZ$0 100208a0 f   ORFDialog.obj
 0001:0001f8a9       __ehhandler$??__EscriptLog@U2@@YAXXZ 100208a9 f   ORFDialog.obj
 0001:0001f8d0       __unwindfunclet$??__EtaskLog@U2@@YAXXZ$0 100208d0 f   ORFDialog.obj
 0001:0001f8d9       __ehhandler$??__EtaskLog@U2@@YAXXZ 100208d9 f   ORFDialog.obj
 0001:0001f900       __unwindfunclet$??__EuiLog@U2@@YAXXZ$0 10020900 f   ORFDialog.obj
 0001:0001f909       __ehhandler$??__EuiLog@U2@@YAXXZ 10020909 f   ORFDialog.obj
 0001:0001f930       __unwindfunclet$??__EuserActLog@U2@@YAXXZ$0 10020930 f   ORFDialog.obj
 0001:0001f939       __ehhandler$??__EuserActLog@U2@@YAXXZ 10020939 f   ORFDialog.obj
 0001:0001f960       __ehhandler$?_Copy@?$basic_string@DU?$char_traits@D@std@@V?$allocator@D@2@@std@@QAEXII@Z 10020960 f   ORFDialog.obj
 0001:0001f980       __unwindfunclet$?accept@ORFDialog@U2@@UAEXXZ$0 10020980 f   ORFDialog.obj
 0001:0001f989       __unwindfunclet$?accept@ORFDialog@U2@@UAEXXZ$1 10020989 f   ORFDialog.obj
 0001:0001f992       __unwindfunclet$?accept@ORFDialog@U2@@UAEXXZ$2 10020992 f   ORFDialog.obj
 0001:0001f99b       __unwindfunclet$?accept@ORFDialog@U2@@UAEXXZ$3 1002099b f   ORFDialog.obj
 0001:0001f9a4       __unwindfunclet$?accept@ORFDialog@U2@@UAEXXZ$5 100209a4 f   ORFDialog.obj
 0001:0001f9af       __ehhandler$?accept@ORFDialog@U2@@UAEXXZ 100209af f   ORFDialog.obj
 0001:0001f9d0       __unwindfunclet$?clone@?$QSharedDataPointer@VAnnotationData@U2@@@@IAEPAVAnnotationData@U2@@XZ$0 100209d0 f   ORFDialog.obj
 0001:0001f9db       __ehhandler$?clone@?$QSharedDataPointer@VAnnotationData@U2@@@@IAEPAVAnnotationData@U2@@XZ 100209db f   ORFDialog.obj
 0001:0001fa00       __unwindfunclet$?createAnnotationWidget@ORFDialog@U2@@AAEXXZ$0 10020a00 f   ORFDialog.obj
 0001:0001fa0c       __unwindfunclet$?createAnnotationWidget@ORFDialog@U2@@AAEXXZ$1 10020a0c f   ORFDialog.obj
 0001:0001fa18       __unwindfunclet$?createAnnotationWidget@ORFDialog@U2@@AAEXXZ$2 10020a18 f   ORFDialog.obj
 0001:0001fa23       __unwindfunclet$?createAnnotationWidget@ORFDialog@U2@@AAEXXZ$3 10020a23 f   ORFDialog.obj
 0001:0001fa2e       __ehhandler$?createAnnotationWidget@ORFDialog@U2@@AAEXXZ 10020a2e f   ORFDialog.obj
 0001:0001fa50       __unwindfunclet$?createNode@?$QMapData@W4DNATranslationRole@U2@@V?$QList@UTriplet@U2@@@@@@QAEPAU?$QMapNode@W4DNATranslationRole@U2@@V?$QList@UTriplet@U2@@@@@@ABW4DNATranslationRole@U2@@ABV?$QList@UTriplet@U2@@@@PAU2@_N@Z$4 10020a50 f   ORFDialog.obj
 0001:0001fa64       __ehhandler$?createNode@?$QMapData@W4DNATranslationRole@U2@@V?$QList@UTriplet@U2@@@@@@QAEPAU?$QMapNode@W4DNATranslationRole@U2@@V?$QList@UTriplet@U2@@@@@@ABW4DNATranslationRole@U2@@ABV?$QList@UTriplet@U2@@@@PAU2@_N@Z 10020a64 f   ORFDialog.obj
 0001:0001fa80       __unwindfunclet$?detach_helper@?$QSharedDataPointer@VAnnotationData@U2@@@@AAEXXZ$0 10020a80 f   ORFDialog.obj
 0001:0001fa8b       __ehhandler$?detach_helper@?$QSharedDataPointer@VAnnotationData@U2@@@@AAEXXZ 10020a8b f   ORFDialog.obj
 0001:0001fab0       __unwindfunclet$?findStartedAAUpdateTask@ORFDialog@U2@@AAEXXZ$0 10020ab0 f   ORFDialog.obj
 0001:0001fab8       __unwindfunclet$?findStartedAAUpdateTask@ORFDialog@U2@@AAEXXZ$1 10020ab8 f   ORFDialog.obj
 0001:0001fac1       __unwindfunclet$?findStartedAAUpdateTask@ORFDialog@U2@@AAEXXZ$2 10020ac1 f   ORFDialog.obj
 0001:0001faca       __unwindfunclet$?findStartedAAUpdateTask@ORFDialog@U2@@AAEXXZ$3 10020aca f   ORFDialog.obj
 0001:0001fad3       __unwindfunclet$?findStartedAAUpdateTask@ORFDialog@U2@@AAEXXZ$4 10020ad3 f   ORFDialog.obj
 0001:0001fadc       __unwindfunclet$?findStartedAAUpdateTask@ORFDialog@U2@@AAEXXZ$5 10020adc f   ORFDialog.obj
 0001:0001fae5       __unwindfunclet$?findStartedAAUpdateTask@ORFDialog@U2@@AAEXXZ$6 10020ae5 f   ORFDialog.obj
 0001:0001faee       __unwindfunclet$?findStartedAAUpdateTask@ORFDialog@U2@@AAEXXZ$7 10020aee f   ORFDialog.obj
 0001:0001faf7       __ehhandler$?findStartedAAUpdateTask@ORFDialog@U2@@AAEXXZ 10020af7 f   ORFDialog.obj
 0001:0001fb20       __unwindfunclet$?getSettings@ORFDialog@U2@@AAEXAAVORFAlgorithmSettings@2@@Z$0 10020b20 f   ORFDialog.obj
 0001:0001fb29       __unwindfunclet$?getSettings@ORFDialog@U2@@AAEXAAVORFAlgorithmSettings@2@@Z$1 10020b29 f   ORFDialog.obj
 0001:0001fb32       __unwindfunclet$?getSettings@ORFDialog@U2@@AAEXAAVORFAlgorithmSettings@2@@Z$2 10020b32 f   ORFDialog.obj
 0001:0001fb3b       __unwindfunclet$?getSettings@ORFDialog@U2@@AAEXAAVORFAlgorithmSettings@2@@Z$3 10020b3b f   ORFDialog.obj
 0001:0001fb44       __unwindfunclet$?getSettings@ORFDialog@U2@@AAEXAAVORFAlgorithmSettings@2@@Z$4 10020b44 f   ORFDialog.obj
 0001:0001fb4d       __unwindfunclet$?getSettings@ORFDialog@U2@@AAEXAAVORFAlgorithmSettings@2@@Z$5 10020b4d f   ORFDialog.obj
 0001:0001fb56       __ehhandler$?getSettings@ORFDialog@U2@@AAEXAAVORFAlgorithmSettings@2@@Z 10020b56 f   ORFDialog.obj
 0001:0001fb80       __unwindfunclet$?importResults@ORFDialog@U2@@AAEXXZ$0 10020b80 f   ORFDialog.obj
 0001:0001fb88       __unwindfunclet$?importResults@ORFDialog@U2@@AAEXXZ$1 10020b88 f   ORFDialog.obj
 0001:0001fb90       __unwindfunclet$?importResults@ORFDialog@U2@@AAEXXZ$2 10020b90 f   ORFDialog.obj
 0001:0001fb9b       __ehhandler$?importResults@ORFDialog@U2@@AAEXXZ 10020b9b f   ORFDialog.obj
 0001:0001fbc0       __ehhandler$?node_copy@?$QList@UTriplet@U2@@@@AAEXPAUNode@1@00@Z 10020bc0 f   ORFDialog.obj
 0001:0001fbe0       __ehhandler$?node_copy@?$QList@VORFFindResult@U2@@@@AAEXPAUNode@1@00@Z 10020be0 f   ORFDialog.obj
 0001:0001fc00       __unwindfunclet$?qt_metatype_id@?$QMetaTypeId@PAVQAction@@@@SAHXZ$0 10020c00 f   ORFDialog.obj
 0001:0001fc09       __ehhandler$?qt_metatype_id@?$QMetaTypeId@PAVQAction@@@@SAHXZ 10020c09 f   ORFDialog.obj
 0001:0001fc30       __unwindfunclet$?retranslateUi@Ui_ORFDialogBase@@QAEXPAVQDialog@@@Z$0 10020c30 f   ORFDialog.obj
 0001:0001fc39       __unwindfunclet$?retranslateUi@Ui_ORFDialogBase@@QAEXPAVQDialog@@@Z$1 10020c39 f   ORFDialog.obj
 0001:0001fc42       __unwindfunclet$?retranslateUi@Ui_ORFDialogBase@@QAEXPAVQDialog@@@Z$2 10020c42 f   ORFDialog.obj
 0001:0001fc4b       __unwindfunclet$?retranslateUi@Ui_ORFDialogBase@@QAEXPAVQDialog@@@Z$3 10020c4b f   ORFDialog.obj
 0001:0001fc54       __unwindfunclet$?retranslateUi@Ui_ORFDialogBase@@QAEXPAVQDialog@@@Z$4 10020c54 f   ORFDialog.obj
 0001:0001fc5d       __unwindfunclet$?retranslateUi@Ui_ORFDialogBase@@QAEXPAVQDialog@@@Z$5 10020c5d f   ORFDialog.obj
 0001:0001fc66       __unwindfunclet$?retranslateUi@Ui_ORFDialogBase@@QAEXPAVQDialog@@@Z$6 10020c66 f   ORFDialog.obj
 0001:0001fc6f       __unwindfunclet$?retranslateUi@Ui_ORFDialogBase@@QAEXPAVQDialog@@@Z$7 10020c6f f   ORFDialog.obj
 0001:0001fc78       __unwindfunclet$?retranslateUi@Ui_ORFDialogBase@@QAEXPAVQDialog@@@Z$8 10020c78 f   ORFDialog.obj
 0001:0001fc81       __unwindfunclet$?retranslateUi@Ui_ORFDialogBase@@QAEXPAVQDialog@@@Z$9 10020c81 f   ORFDialog.obj
 0001:0001fc8a       __unwindfunclet$?retranslateUi@Ui_ORFDialogBase@@QAEXPAVQDialog@@@Z$10 10020c8a f   ORFDialog.obj
 0001:0001fc93       __unwindfunclet$?retranslateUi@Ui_ORFDialogBase@@QAEXPAVQDialog@@@Z$11 10020c93 f   ORFDialog.obj
 0001:0001fc9c       __unwindfunclet$?retranslateUi@Ui_ORFDialogBase@@QAEXPAVQDialog@@@Z$12 10020c9c f   ORFDialog.obj
 0001:0001fca5       __unwindfunclet$?retranslateUi@Ui_ORFDialogBase@@QAEXPAVQDialog@@@Z$13 10020ca5 f   ORFDialog.obj
 0001:0001fcae       __unwindfunclet$?retranslateUi@Ui_ORFDialogBase@@QAEXPAVQDialog@@@Z$14 10020cae f   ORFDialog.obj
 0001:0001fcb7       __unwindfunclet$?retranslateUi@Ui_ORFDialogBase@@QAEXPAVQDialog@@@Z$15 10020cb7 f   ORFDialog.obj
 0001:0001fcc0       __unwindfunclet$?retranslateUi@Ui_ORFDialogBase@@QAEXPAVQDialog@@@Z$16 10020cc0 f   ORFDialog.obj
 0001:0001fcc9       __unwindfunclet$?retranslateUi@Ui_ORFDialogBase@@QAEXPAVQDialog@@@Z$17 10020cc9 f   ORFDialog.obj
 0001:0001fcd2       __unwindfunclet$?retranslateUi@Ui_ORFDialogBase@@QAEXPAVQDialog@@@Z$18 10020cd2 f   ORFDialog.obj
 0001:0001fcdb       __unwindfunclet$?retranslateUi@Ui_ORFDialogBase@@QAEXPAVQDialog@@@Z$19 10020cdb f   ORFDialog.obj
 0001:0001fce4       __unwindfunclet$?retranslateUi@Ui_ORFDialogBase@@QAEXPAVQDialog@@@Z$20 10020ce4 f   ORFDialog.obj
 0001:0001fced       __unwindfunclet$?retranslateUi@Ui_ORFDialogBase@@QAEXPAVQDialog@@@Z$21 10020ced f   ORFDialog.obj
 0001:0001fcf6       __unwindfunclet$?retranslateUi@Ui_ORFDialogBase@@QAEXPAVQDialog@@@Z$22 10020cf6 f   ORFDialog.obj
 0001:0001fcff       __unwindfunclet$?retranslateUi@Ui_ORFDialogBase@@QAEXPAVQDialog@@@Z$23 10020cff f   ORFDialog.obj
 0001:0001fd08       __unwindfunclet$?retranslateUi@Ui_ORFDialogBase@@QAEXPAVQDialog@@@Z$24 10020d08 f   ORFDialog.obj
 0001:0001fd11       __unwindfunclet$?retranslateUi@Ui_ORFDialogBase@@QAEXPAVQDialog@@@Z$25 10020d11 f   ORFDialog.obj
 0001:0001fd1a       __unwindfunclet$?retranslateUi@Ui_ORFDialogBase@@QAEXPAVQDialog@@@Z$26 10020d1a f   ORFDialog.obj
 0001:0001fd23       __unwindfunclet$?retranslateUi@Ui_ORFDialogBase@@QAEXPAVQDialog@@@Z$27 10020d23 f   ORFDialog.obj
 0001:0001fd2c       __unwindfunclet$?retranslateUi@Ui_ORFDialogBase@@QAEXPAVQDialog@@@Z$28 10020d2c f   ORFDialog.obj
 0001:0001fd35       __unwindfunclet$?retranslateUi@Ui_ORFDialogBase@@QAEXPAVQDialog@@@Z$29 10020d35 f   ORFDialog.obj
 0001:0001fd3e       __unwindfunclet$?retranslateUi@Ui_ORFDialogBase@@QAEXPAVQDialog@@@Z$30 10020d3e f   ORFDialog.obj
 0001:0001fd47       __unwindfunclet$?retranslateUi@Ui_ORFDialogBase@@QAEXPAVQDialog@@@Z$31 10020d47 f   ORFDialog.obj
 0001:0001fd50       __unwindfunclet$?retranslateUi@Ui_ORFDialogBase@@QAEXPAVQDialog@@@Z$32 10020d50 f   ORFDialog.obj
 0001:0001fd59       __unwindfunclet$?retranslateUi@Ui_ORFDialogBase@@QAEXPAVQDialog@@@Z$33 10020d59 f   ORFDialog.obj
 0001:0001fd62       __unwindfunclet$?retranslateUi@Ui_ORFDialogBase@@QAEXPAVQDialog@@@Z$34 10020d62 f   ORFDialog.obj
 0001:0001fd6b       __unwindfunclet$?retranslateUi@Ui_ORFDialogBase@@QAEXPAVQDialog@@@Z$35 10020d6b f   ORFDialog.obj
 0001:0001fd74       __unwindfunclet$?retranslateUi@Ui_ORFDialogBase@@QAEXPAVQDialog@@@Z$36 10020d74 f   ORFDialog.obj
 0001:0001fd7d       __unwindfunclet$?retranslateUi@Ui_ORFDialogBase@@QAEXPAVQDialog@@@Z$37 10020d7d f   ORFDialog.obj
 0001:0001fd86       __unwindfunclet$?retranslateUi@Ui_ORFDialogBase@@QAEXPAVQDialog@@@Z$38 10020d86 f   ORFDialog.obj
 0001:0001fd8f       __unwindfunclet$?retranslateUi@Ui_ORFDialogBase@@QAEXPAVQDialog@@@Z$39 10020d8f f   ORFDialog.obj
 0001:0001fd98       __unwindfunclet$?retranslateUi@Ui_ORFDialogBase@@QAEXPAVQDialog@@@Z$40 10020d98 f   ORFDialog.obj
 0001:0001fda1       __unwindfunclet$?retranslateUi@Ui_ORFDialogBase@@QAEXPAVQDialog@@@Z$41 10020da1 f   ORFDialog.obj
 0001:0001fdaa       __unwindfunclet$?retranslateUi@Ui_ORFDialogBase@@QAEXPAVQDialog@@@Z$42 10020daa f   ORFDialog.obj
 0001:0001fdb3       __unwindfunclet$?retranslateUi@Ui_ORFDialogBase@@QAEXPAVQDialog@@@Z$43 10020db3 f   ORFDialog.obj
 0001:0001fdbc       __unwindfunclet$?retranslateUi@Ui_ORFDialogBase@@QAEXPAVQDialog@@@Z$44 10020dbc f   ORFDialog.obj
 0001:0001fdc5       __unwindfunclet$?retranslateUi@Ui_ORFDialogBase@@QAEXPAVQDialog@@@Z$45 10020dc5 f   ORFDialog.obj
 0001:0001fdce       __unwindfunclet$?retranslateUi@Ui_ORFDialogBase@@QAEXPAVQDialog@@@Z$46 10020dce f   ORFDialog.obj
 0001:0001fdd7       __unwindfunclet$?retranslateUi@Ui_ORFDialogBase@@QAEXPAVQDialog@@@Z$47 10020dd7 f   ORFDialog.obj
 0001:0001fde0       __unwindfunclet$?retranslateUi@Ui_ORFDialogBase@@QAEXPAVQDialog@@@Z$48 10020de0 f   ORFDialog.obj
 0001:0001fde9       __unwindfunclet$?retranslateUi@Ui_ORFDialogBase@@QAEXPAVQDialog@@@Z$49 10020de9 f   ORFDialog.obj
 0001:0001fdf2       __unwindfunclet$?retranslateUi@Ui_ORFDialogBase@@QAEXPAVQDialog@@@Z$50 10020df2 f   ORFDialog.obj
 0001:0001fdfb       __unwindfunclet$?retranslateUi@Ui_ORFDialogBase@@QAEXPAVQDialog@@@Z$51 10020dfb f   ORFDialog.obj
 0001:0001fe04       __ehhandler$?retranslateUi@Ui_ORFDialogBase@@QAEXPAVQDialog@@@Z 10020e04 f   ORFDialog.obj
 0001:0001fe20       __unwindfunclet$?runTask@ORFDialog@U2@@AAEXXZ$0 10020e20 f   ORFDialog.obj
 0001:0001fe2b       __ehhandler$?runTask@ORFDialog@U2@@AAEXXZ 10020e2b f   ORFDialog.obj
 0001:0001fe50       __unwindfunclet$?setupUi@Ui_ORFDialogBase@@QAEXPAVQDialog@@@Z$1 10020e50 f   ORFDialog.obj
 0001:0001fe59       __unwindfunclet$?setupUi@Ui_ORFDialogBase@@QAEXPAVQDialog@@@Z$2 10020e59 f   ORFDialog.obj
 0001:0001fe64       __unwindfunclet$?setupUi@Ui_ORFDialogBase@@QAEXPAVQDialog@@@Z$3 10020e64 f   ORFDialog.obj
 0001:0001fe6d       __unwindfunclet$?setupUi@Ui_ORFDialogBase@@QAEXPAVQDialog@@@Z$4 10020e6d f   ORFDialog.obj
 0001:0001fe78       __unwindfunclet$?setupUi@Ui_ORFDialogBase@@QAEXPAVQDialog@@@Z$5 10020e78 f   ORFDialog.obj
 0001:0001fe81       __unwindfunclet$?setupUi@Ui_ORFDialogBase@@QAEXPAVQDialog@@@Z$6 10020e81 f   ORFDialog.obj
 0001:0001fe8c       __unwindfunclet$?setupUi@Ui_ORFDialogBase@@QAEXPAVQDialog@@@Z$7 10020e8c f   ORFDialog.obj
 0001:0001fe95       __unwindfunclet$?setupUi@Ui_ORFDialogBase@@QAEXPAVQDialog@@@Z$8 10020e95 f   ORFDialog.obj
 0001:0001fea0       __unwindfunclet$?setupUi@Ui_ORFDialogBase@@QAEXPAVQDialog@@@Z$9 10020ea0 f   ORFDialog.obj
 0001:0001fea9       __unwindfunclet$?setupUi@Ui_ORFDialogBase@@QAEXPAVQDialog@@@Z$10 10020ea9 f   ORFDialog.obj
 0001:0001feb4       __unwindfunclet$?setupUi@Ui_ORFDialogBase@@QAEXPAVQDialog@@@Z$11 10020eb4 f   ORFDialog.obj
 0001:0001febd       __unwindfunclet$?setupUi@Ui_ORFDialogBase@@QAEXPAVQDialog@@@Z$12 10020ebd f   ORFDialog.obj
 0001:0001fec8       __unwindfunclet$?setupUi@Ui_ORFDialogBase@@QAEXPAVQDialog@@@Z$13 10020ec8 f   ORFDialog.obj
 0001:0001fed1       __unwindfunclet$?setupUi@Ui_ORFDialogBase@@QAEXPAVQDialog@@@Z$14 10020ed1 f   ORFDialog.obj
 0001:0001fedc       __unwindfunclet$?setupUi@Ui_ORFDialogBase@@QAEXPAVQDialog@@@Z$15 10020edc f   ORFDialog.obj
 0001:0001fee5       __unwindfunclet$?setupUi@Ui_ORFDialogBase@@QAEXPAVQDialog@@@Z$16 10020ee5 f   ORFDialog.obj
 0001:0001fef0       __unwindfunclet$?setupUi@Ui_ORFDialogBase@@QAEXPAVQDialog@@@Z$17 10020ef0 f   ORFDialog.obj
 0001:0001fef9       __unwindfunclet$?setupUi@Ui_ORFDialogBase@@QAEXPAVQDialog@@@Z$18 10020ef9 f   ORFDialog.obj
 0001:0001ff04       __unwindfunclet$?setupUi@Ui_ORFDialogBase@@QAEXPAVQDialog@@@Z$19 10020f04 f   ORFDialog.obj
 0001:0001ff0d       __unwindfunclet$?setupUi@Ui_ORFDialogBase@@QAEXPAVQDialog@@@Z$20 10020f0d f   ORFDialog.obj
 0001:0001ff18       __unwindfunclet$?setupUi@Ui_ORFDialogBase@@QAEXPAVQDialog@@@Z$21 10020f18 f   ORFDialog.obj
 0001:0001ff21       __unwindfunclet$?setupUi@Ui_ORFDialogBase@@QAEXPAVQDialog@@@Z$22 10020f21 f   ORFDialog.obj
 0001:0001ff2c       __unwindfunclet$?setupUi@Ui_ORFDialogBase@@QAEXPAVQDialog@@@Z$23 10020f2c f   ORFDialog.obj
 0001:0001ff35       __unwindfunclet$?setupUi@Ui_ORFDialogBase@@QAEXPAVQDialog@@@Z$24 10020f35 f   ORFDialog.obj
 0001:0001ff40       __unwindfunclet$?setupUi@Ui_ORFDialogBase@@QAEXPAVQDialog@@@Z$25 10020f40 f   ORFDialog.obj
 0001:0001ff49       __unwindfunclet$?setupUi@Ui_ORFDialogBase@@QAEXPAVQDialog@@@Z$26 10020f49 f   ORFDialog.obj
 0001:0001ff54       __unwindfunclet$?setupUi@Ui_ORFDialogBase@@QAEXPAVQDialog@@@Z$27 10020f54 f   ORFDialog.obj
 0001:0001ff5d       __unwindfunclet$?setupUi@Ui_ORFDialogBase@@QAEXPAVQDialog@@@Z$28 10020f5d f   ORFDialog.obj
 0001:0001ff68       __unwindfunclet$?setupUi@Ui_ORFDialogBase@@QAEXPAVQDialog@@@Z$29 10020f68 f   ORFDialog.obj
 0001:0001ff71       __unwindfunclet$?setupUi@Ui_ORFDialogBase@@QAEXPAVQDialog@@@Z$30 10020f71 f   ORFDialog.obj
 0001:0001ff7c       __unwindfunclet$?setupUi@Ui_ORFDialogBase@@QAEXPAVQDialog@@@Z$31 10020f7c f   ORFDialog.obj
 0001:0001ff85       __unwindfunclet$?setupUi@Ui_ORFDialogBase@@QAEXPAVQDialog@@@Z$32 10020f85 f   ORFDialog.obj
 0001:0001ff90       __unwindfunclet$?setupUi@Ui_ORFDialogBase@@QAEXPAVQDialog@@@Z$33 10020f90 f   ORFDialog.obj
 0001:0001ff99       __unwindfunclet$?setupUi@Ui_ORFDialogBase@@QAEXPAVQDialog@@@Z$34 10020f99 f   ORFDialog.obj
 0001:0001ffa4       __unwindfunclet$?setupUi@Ui_ORFDialogBase@@QAEXPAVQDialog@@@Z$35 10020fa4 f   ORFDialog.obj
 0001:0001ffad       __unwindfunclet$?setupUi@Ui_ORFDialogBase@@QAEXPAVQDialog@@@Z$36 10020fad f   ORFDialog.obj
 0001:0001ffb8       __unwindfunclet$?setupUi@Ui_ORFDialogBase@@QAEXPAVQDialog@@@Z$37 10020fb8 f   ORFDialog.obj
 0001:0001ffc1       __unwindfunclet$?setupUi@Ui_ORFDialogBase@@QAEXPAVQDialog@@@Z$38 10020fc1 f   ORFDialog.obj
 0001:0001ffcc       __unwindfunclet$?setupUi@Ui_ORFDialogBase@@QAEXPAVQDialog@@@Z$39 10020fcc f   ORFDialog.obj
 0001:0001ffd5       __unwindfunclet$?setupUi@Ui_ORFDialogBase@@QAEXPAVQDialog@@@Z$40 10020fd5 f   ORFDialog.obj
 0001:0001ffe0       __unwindfunclet$?setupUi@Ui_ORFDialogBase@@QAEXPAVQDialog@@@Z$41 10020fe0 f   ORFDialog.obj
 0001:0001ffe9       __unwindfunclet$?setupUi@Ui_ORFDialogBase@@QAEXPAVQDialog@@@Z$42 10020fe9 f   ORFDialog.obj
 0001:0001fff4       __unwindfunclet$?setupUi@Ui_ORFDialogBase@@QAEXPAVQDialog@@@Z$43 10020ff4 f   ORFDialog.obj
 0001:0001fffd       __unwindfunclet$?setupUi@Ui_ORFDialogBase@@QAEXPAVQDialog@@@Z$44 10020ffd f   ORFDialog.obj
 0001:00020008       __unwindfunclet$?setupUi@Ui_ORFDialogBase@@QAEXPAVQDialog@@@Z$45 10021008 f   ORFDialog.obj
 0001:00020011       __unwindfunclet$?setupUi@Ui_ORFDialogBase@@QAEXPAVQDialog@@@Z$46 10021011 f   ORFDialog.obj
 0001:0002001c       __unwindfunclet$?setupUi@Ui_ORFDialogBase@@QAEXPAVQDialog@@@Z$47 1002101c f   ORFDialog.obj
 0001:00020025       __unwindfunclet$?setupUi@Ui_ORFDialogBase@@QAEXPAVQDialog@@@Z$48 10021025 f   ORFDialog.obj
 0001:00020030       __unwindfunclet$?setupUi@Ui_ORFDialogBase@@QAEXPAVQDialog@@@Z$49 10021030 f   ORFDialog.obj
 0001:00020039       __unwindfunclet$?setupUi@Ui_ORFDialogBase@@QAEXPAVQDialog@@@Z$50 10021039 f   ORFDialog.obj
 0001:00020044       __unwindfunclet$?setupUi@Ui_ORFDialogBase@@QAEXPAVQDialog@@@Z$51 10021044 f   ORFDialog.obj
 0001:0002004d       __unwindfunclet$?setupUi@Ui_ORFDialogBase@@QAEXPAVQDialog@@@Z$52 1002104d f   ORFDialog.obj
 0001:00020058       __unwindfunclet$?setupUi@Ui_ORFDialogBase@@QAEXPAVQDialog@@@Z$53 10021058 f   ORFDialog.obj
 0001:00020061       __unwindfunclet$?setupUi@Ui_ORFDialogBase@@QAEXPAVQDialog@@@Z$54 10021061 f   ORFDialog.obj
 0001:0002006c       __unwindfunclet$?setupUi@Ui_ORFDialogBase@@QAEXPAVQDialog@@@Z$55 1002106c f   ORFDialog.obj
 0001:00020075       __unwindfunclet$?setupUi@Ui_ORFDialogBase@@QAEXPAVQDialog@@@Z$56 10021075 f   ORFDialog.obj
 0001:00020080       __unwindfunclet$?setupUi@Ui_ORFDialogBase@@QAEXPAVQDialog@@@Z$57 10021080 f   ORFDialog.obj
 0001:0002008b       __unwindfunclet$?setupUi@Ui_ORFDialogBase@@QAEXPAVQDialog@@@Z$58 1002108b f   ORFDialog.obj
 0001:00020094       __unwindfunclet$?setupUi@Ui_ORFDialogBase@@QAEXPAVQDialog@@@Z$59 10021094 f   ORFDialog.obj
 0001:0002009f       __unwindfunclet$?setupUi@Ui_ORFDialogBase@@QAEXPAVQDialog@@@Z$60 1002109f f   ORFDialog.obj
 0001:000200a8       __unwindfunclet$?setupUi@Ui_ORFDialogBase@@QAEXPAVQDialog@@@Z$61 100210a8 f   ORFDialog.obj
 0001:000200b3       __unwindfunclet$?setupUi@Ui_ORFDialogBase@@QAEXPAVQDialog@@@Z$62 100210b3 f   ORFDialog.obj
 0001:000200bc       __unwindfunclet$?setupUi@Ui_ORFDialogBase@@QAEXPAVQDialog@@@Z$63 100210bc f   ORFDialog.obj
 0001:000200c7       __unwindfunclet$?setupUi@Ui_ORFDialogBase@@QAEXPAVQDialog@@@Z$64 100210c7 f   ORFDialog.obj
 0001:000200d0       __unwindfunclet$?setupUi@Ui_ORFDialogBase@@QAEXPAVQDialog@@@Z$65 100210d0 f   ORFDialog.obj
 0001:000200d9       __unwindfunclet$?setupUi@Ui_ORFDialogBase@@QAEXPAVQDialog@@@Z$66 100210d9 f   ORFDialog.obj
 0001:000200e4       __unwindfunclet$?setupUi@Ui_ORFDialogBase@@QAEXPAVQDialog@@@Z$67 100210e4 f   ORFDialog.obj
 0001:000200ed       __unwindfunclet$?setupUi@Ui_ORFDialogBase@@QAEXPAVQDialog@@@Z$68 100210ed f   ORFDialog.obj
 0001:000200f8       __unwindfunclet$?setupUi@Ui_ORFDialogBase@@QAEXPAVQDialog@@@Z$69 100210f8 f   ORFDialog.obj
 0001:00020101       __unwindfunclet$?setupUi@Ui_ORFDialogBase@@QAEXPAVQDialog@@@Z$70 10021101 f   ORFDialog.obj
 0001:0002010c       __unwindfunclet$?setupUi@Ui_ORFDialogBase@@QAEXPAVQDialog@@@Z$71 1002110c f   ORFDialog.obj
 0001:00020115       __unwindfunclet$?setupUi@Ui_ORFDialogBase@@QAEXPAVQDialog@@@Z$72 10021115 f   ORFDialog.obj
 0001:00020120       __unwindfunclet$?setupUi@Ui_ORFDialogBase@@QAEXPAVQDialog@@@Z$73 10021120 f   ORFDialog.obj
 0001:00020129       __unwindfunclet$?setupUi@Ui_ORFDialogBase@@QAEXPAVQDialog@@@Z$74 10021129 f   ORFDialog.obj
 0001:00020134       __unwindfunclet$?setupUi@Ui_ORFDialogBase@@QAEXPAVQDialog@@@Z$75 10021134 f   ORFDialog.obj
 0001:0002013d       __unwindfunclet$?setupUi@Ui_ORFDialogBase@@QAEXPAVQDialog@@@Z$76 1002113d f   ORFDialog.obj
 0001:00020148       __unwindfunclet$?setupUi@Ui_ORFDialogBase@@QAEXPAVQDialog@@@Z$77 10021148 f   ORFDialog.obj
 0001:00020151       __unwindfunclet$?setupUi@Ui_ORFDialogBase@@QAEXPAVQDialog@@@Z$78 10021151 f   ORFDialog.obj
 0001:0002015c       __unwindfunclet$?setupUi@Ui_ORFDialogBase@@QAEXPAVQDialog@@@Z$79 1002115c f   ORFDialog.obj
 0001:00020165       __ehhandler$?setupUi@Ui_ORFDialogBase@@QAEXPAVQDialog@@@Z 10021165 f   ORFDialog.obj
 0001:00020180       __unwindfunclet$?sl_onFindAll@ORFDialog@U2@@AAEXXZ$0 10021180 f   ORFDialog.obj
 0001:00020189       __unwindfunclet$?sl_onFindAll@ORFDialog@U2@@AAEXXZ$1 10021189 f   ORFDialog.obj
 0001:00020192       __ehhandler$?sl_onFindAll@ORFDialog@U2@@AAEXXZ 10021192 f   ORFDialog.obj
 0001:000201b0       __unwindfunclet$?sl_translationChanged@ORFDialog@U2@@AAEXXZ$0 100211b0 f   ORFDialog.obj
 0001:000201bc       __unwindfunclet$?sl_translationChanged@ORFDialog@U2@@AAEXXZ$1 100211bc f   ORFDialog.obj
 0001:000201c4       __unwindfunclet$?sl_translationChanged@ORFDialog@U2@@AAEXXZ$2 100211c4 f   ORFDialog.obj
 0001:000201cd       __unwindfunclet$?sl_translationChanged@ORFDialog@U2@@AAEXXZ$3 100211cd f   ORFDialog.obj
 0001:000201d6       __unwindfunclet$?sl_translationChanged@ORFDialog@U2@@AAEXXZ$4 100211d6 f   ORFDialog.obj
 0001:000201df       __unwindfunclet$?sl_translationChanged@ORFDialog@U2@@AAEXXZ$5 100211df f   ORFDialog.obj
 0001:000201e8       __unwindfunclet$?sl_translationChanged@ORFDialog@U2@@AAEXXZ$6 100211e8 f   ORFDialog.obj
 0001:000201f1       __unwindfunclet$?sl_translationChanged@ORFDialog@U2@@AAEXXZ$7 100211f1 f   ORFDialog.obj
 0001:000201fa       __unwindfunclet$?sl_translationChanged@ORFDialog@U2@@AAEXXZ$8 100211fa f   ORFDialog.obj
 0001:00020203       __unwindfunclet$?sl_translationChanged@ORFDialog@U2@@AAEXXZ$9 10021203 f   ORFDialog.obj
 0001:0002020c       __unwindfunclet$?sl_translationChanged@ORFDialog@U2@@AAEXXZ$10 1002120c f   ORFDialog.obj
 0001:00020215       __unwindfunclet$?sl_translationChanged@ORFDialog@U2@@AAEXXZ$11 10021215 f   ORFDialog.obj
 0001:0002021e       __unwindfunclet$?sl_translationChanged@ORFDialog@U2@@AAEXXZ$12 1002121e f   ORFDialog.obj
 0001:00020227       __unwindfunclet$?sl_translationChanged@ORFDialog@U2@@AAEXXZ$13 10021227 f   ORFDialog.obj
 0001:00020230       __unwindfunclet$?sl_translationChanged@ORFDialog@U2@@AAEXXZ$14 10021230 f   ORFDialog.obj
 0001:00020239       __unwindfunclet$?sl_translationChanged@ORFDialog@U2@@AAEXXZ$15 10021239 f   ORFDialog.obj
 0001:00020242       __unwindfunclet$?sl_translationChanged@ORFDialog@U2@@AAEXXZ$16 10021242 f   ORFDialog.obj
 0001:0002024b       __unwindfunclet$?sl_translationChanged@ORFDialog@U2@@AAEXXZ$17 1002124b f   ORFDialog.obj
 0001:00020254       __unwindfunclet$?sl_translationChanged@ORFDialog@U2@@AAEXXZ$18 10021254 f   ORFDialog.obj
 0001:0002025d       __unwindfunclet$?sl_translationChanged@ORFDialog@U2@@AAEXXZ$19 1002125d f   ORFDialog.obj
 0001:00020266       __unwindfunclet$?sl_translationChanged@ORFDialog@U2@@AAEXXZ$20 10021266 f   ORFDialog.obj
 0001:0002026f       __unwindfunclet$?sl_translationChanged@ORFDialog@U2@@AAEXXZ$21 1002126f f   ORFDialog.obj
 0001:00020278       __unwindfunclet$?sl_translationChanged@ORFDialog@U2@@AAEXXZ$22 10021278 f   ORFDialog.obj
 0001:00020281       __unwindfunclet$?sl_translationChanged@ORFDialog@U2@@AAEXXZ$23 10021281 f   ORFDialog.obj
 0001:0002028a       __unwindfunclet$?sl_translationChanged@ORFDialog@U2@@AAEXXZ$24 1002128a f   ORFDialog.obj
 0001:00020293       __unwindfunclet$?sl_translationChanged@ORFDialog@U2@@AAEXXZ$25 10021293 f   ORFDialog.obj
 0001:0002029c       __unwindfunclet$?sl_translationChanged@ORFDialog@U2@@AAEXXZ$26 1002129c f   ORFDialog.obj
 0001:000202a5       __unwindfunclet$?sl_translationChanged@ORFDialog@U2@@AAEXXZ$27 100212a5 f   ORFDialog.obj
 0001:000202ae       __unwindfunclet$?sl_translationChanged@ORFDialog@U2@@AAEXXZ$28 100212ae f   ORFDialog.obj
 0001:000202b7       __ehhandler$?sl_translationChanged@ORFDialog@U2@@AAEXXZ 100212b7 f   ORFDialog.obj
 0001:000202e0       __unwindfunclet$?triplet2str@U2@@YA?AVQString@@ABUTriplet@1@@Z$0 100212e0 f   ORFDialog.obj
 0001:000202fa       __ehhandler$?triplet2str@U2@@YA?AVQString@@ABUTriplet@1@@Z 100212fa f   ORFDialog.obj
 0001:00020320       __unwindfunclet$?updateStatus@ORFDialog@U2@@AAEXXZ$0 10021320 f   ORFDialog.obj
 0001:00020329       __unwindfunclet$?updateStatus@ORFDialog@U2@@AAEXXZ$1 10021329 f   ORFDialog.obj
 0001:00020332       __unwindfunclet$?updateStatus@ORFDialog@U2@@AAEXXZ$2 10021332 f   ORFDialog.obj
 0001:0002033b       __unwindfunclet$?updateStatus@ORFDialog@U2@@AAEXXZ$3 1002133b f   ORFDialog.obj
 0001:00020344       __unwindfunclet$?updateStatus@ORFDialog@U2@@AAEXXZ$4 10021344 f   ORFDialog.obj
 0001:0002034d       __ehhandler$?updateStatus@ORFDialog@U2@@AAEXXZ 1002134d f   ORFDialog.obj
 0001:00020370       __ehhandler$??0?$QList@PAVXMLTestFactory@U2@@@@QAE@ABV0@@Z 10021370 f   ORFMarkerPlugin.obj
 0001:00020390       __unwindfunclet$??0GTest_ORFMarkerTask@U2@@QAE@PAVXMLTestFormat@1@ABVQString@@PAVGTest@1@PBVGTestEnvironment@1@ABV?$QList@PAVGTest@U2@@@@ABVQDomElement@@@Z$0 10021390 f   ORFMarkerPlugin.obj
 0001:00020399       __unwindfunclet$??0GTest_ORFMarkerTask@U2@@QAE@PAVXMLTestFormat@1@ABVQString@@PAVGTest@1@PBVGTestEnvironment@1@ABV?$QList@PAVGTest@U2@@@@ABVQDomElement@@@Z$1 10021399 f   ORFMarkerPlugin.obj
 0001:000203a8       __unwindfunclet$??0GTest_ORFMarkerTask@U2@@QAE@PAVXMLTestFormat@1@ABVQString@@PAVGTest@1@PBVGTestEnvironment@1@ABV?$QList@PAVGTest@U2@@@@ABVQDomElement@@@Z$2 100213a8 f   ORFMarkerPlugin.obj
 0001:000203b7       __unwindfunclet$??0GTest_ORFMarkerTask@U2@@QAE@PAVXMLTestFormat@1@ABVQString@@PAVGTest@1@PBVGTestEnvironment@1@ABV?$QList@PAVGTest@U2@@@@ABVQDomElement@@@Z$3 100213b7 f   ORFMarkerPlugin.obj
 0001:000203c5       __ehhandler$??0GTest_ORFMarkerTask@U2@@QAE@PAVXMLTestFormat@1@ABVQString@@PAVGTest@1@PBVGTestEnvironment@1@ABV?$QList@PAVGTest@U2@@@@ABVQDomElement@@@Z 100213c5 f   ORFMarkerPlugin.obj
 0001:000203e0       __unwindfunclet$??0GTest_ORFMarkerTaskFactory@GTest_ORFMarkerTask@U2@@QAE@XZ$0 100213e0 f   ORFMarkerPlugin.obj
 0001:000203e9       __unwindfunclet$??0GTest_ORFMarkerTaskFactory@GTest_ORFMarkerTask@U2@@QAE@XZ$1 100213e9 f   ORFMarkerPlugin.obj
 0001:000203f2       __ehhandler$??0GTest_ORFMarkerTaskFactory@GTest_ORFMarkerTask@U2@@QAE@XZ 100213f2 f   ORFMarkerPlugin.obj
 0001:00020410       __unwindfunclet$??0ORFMarkerPlugin@U2@@QAE@XZ$0 10021410 f   ORFMarkerPlugin.obj
 0001:00020419       __unwindfunclet$??0ORFMarkerPlugin@U2@@QAE@XZ$1 10021419 f   ORFMarkerPlugin.obj
 0001:00020422       __unwindfunclet$??0ORFMarkerPlugin@U2@@QAE@XZ$2 10021422 f   ORFMarkerPlugin.obj
 0001:0002042b       __unwindfunclet$??0ORFMarkerPlugin@U2@@QAE@XZ$3 1002142b f   ORFMarkerPlugin.obj
 0001:00020436       __unwindfunclet$??0ORFMarkerPlugin@U2@@QAE@XZ$4 10021436 f   ORFMarkerPlugin.obj
 0001:00020441       __unwindfunclet$??0ORFMarkerPlugin@U2@@QAE@XZ$5 10021441 f   ORFMarkerPlugin.obj
 0001:0002044c       __unwindfunclet$??0ORFMarkerPlugin@U2@@QAE@XZ$6 1002144c f   ORFMarkerPlugin.obj
 0001:00020455       __unwindfunclet$??0ORFMarkerPlugin@U2@@QAE@XZ$7 10021455 f   ORFMarkerPlugin.obj
 0001:00020460       __unwindfunclet$??0ORFMarkerPlugin@U2@@QAE@XZ$9 10021460 f   ORFMarkerPlugin.obj
 0001:00020468       __ehhandler$??0ORFMarkerPlugin@U2@@QAE@XZ 10021468 f   ORFMarkerPlugin.obj
 0001:00020490       __unwindfunclet$??0ORFViewContext@U2@@QAE@PAVQObject@@@Z$0 10021490 f   ORFMarkerPlugin.obj
 0001:00020498       __unwindfunclet$??0ORFViewContext@U2@@QAE@PAVQObject@@@Z$1 10021498 f   ORFMarkerPlugin.obj
 0001:000204a1       __ehhandler$??0ORFViewContext@U2@@QAE@PAVQObject@@@Z 100214a1 f   ORFMarkerPlugin.obj
 0001:000204c0       __unwindfunclet$??1?$GAutoDeleteList@VXMLTestFactory@U2@@@U2@@UAE@XZ$0 100214c0 f   ORFMarkerPlugin.obj
 0001:000204c9       __unwindfunclet$??1?$GAutoDeleteList@VXMLTestFactory@U2@@@U2@@UAE@XZ$1 100214c9 f   ORFMarkerPlugin.obj
 0001:000204d4       __ehhandler$??1?$GAutoDeleteList@VXMLTestFactory@U2@@@U2@@UAE@XZ 100214d4 f   ORFMarkerPlugin.obj
 0001:000204f0       __unwindfunclet$??1?$QObjectScopedPointer@VORFDialog@U2@@@U2@@QAE@XZ$0 100214f0 f   ORFMarkerPlugin.obj
 0001:000204f8       __ehhandler$??1?$QObjectScopedPointer@VORFDialog@U2@@@U2@@QAE@XZ 100214f8 f   ORFMarkerPlugin.obj
 0001:00020520       __unwindfunclet$??1GTest_ORFMarkerTask@U2@@UAE@XZ$0 10021520 f   ORFMarkerPlugin.obj
 0001:00020529       __unwindfunclet$??1GTest_ORFMarkerTask@U2@@UAE@XZ$1 10021529 f   ORFMarkerPlugin.obj
 0001:00020538       __unwindfunclet$??1GTest_ORFMarkerTask@U2@@UAE@XZ$2 10021538 f   ORFMarkerPlugin.obj
 0001:00020547       __ehhandler$??1GTest_ORFMarkerTask@U2@@UAE@XZ 10021547 f   ORFMarkerPlugin.obj
 0001:00020570       __unwindfunclet$??__EalgoLog@U2@@YAXXZ$0 10021570 f   ORFMarkerPlugin.obj
 0001:00020579       __ehhandler$??__EalgoLog@U2@@YAXXZ 10021579 f   ORFMarkerPlugin.obj
 0001:000205a0       __unwindfunclet$??__EcmdLog@U2@@YAXXZ$0 100215a0 f   ORFMarkerPlugin.obj
 0001:000205a9       __ehhandler$??__EcmdLog@U2@@YAXXZ 100215a9 f   ORFMarkerPlugin.obj
 0001:000205d0       __unwindfunclet$??__EcoreLog@U2@@YAXXZ$0 100215d0 f   ORFMarkerPlugin.obj
 0001:000205d9       __ehhandler$??__EcoreLog@U2@@YAXXZ 100215d9 f   ORFMarkerPlugin.obj
 0001:00020600       __unwindfunclet$??__EioLog@U2@@YAXXZ$0 10021600 f   ORFMarkerPlugin.obj
 0001:00020609       __ehhandler$??__EioLog@U2@@YAXXZ 10021609 f   ORFMarkerPlugin.obj
 0001:00020630       __unwindfunclet$??__EperfLog@U2@@YAXXZ$0 10021630 f   ORFMarkerPlugin.obj
 0001:00020639       __ehhandler$??__EperfLog@U2@@YAXXZ 10021639 f   ORFMarkerPlugin.obj
 0001:00020660       __unwindfunclet$??__EscriptLog@U2@@YAXXZ$0 10021660 f   ORFMarkerPlugin.obj
 0001:00020669       __ehhandler$??__EscriptLog@U2@@YAXXZ 10021669 f   ORFMarkerPlugin.obj
 0001:00020690       __unwindfunclet$??__EtaskLog@U2@@YAXXZ$0 10021690 f   ORFMarkerPlugin.obj
 0001:00020699       __ehhandler$??__EtaskLog@U2@@YAXXZ 10021699 f   ORFMarkerPlugin.obj
 0001:000206c0       __unwindfunclet$??__EuiLog@U2@@YAXXZ$0 100216c0 f   ORFMarkerPlugin.obj
 0001:000206c9       __ehhandler$??__EuiLog@U2@@YAXXZ 100216c9 f   ORFMarkerPlugin.obj
 0001:000206f0       __unwindfunclet$??__EuserActLog@U2@@YAXXZ$0 100216f0 f   ORFMarkerPlugin.obj
 0001:000206f9       __ehhandler$??__EuserActLog@U2@@YAXXZ 100216f9 f   ORFMarkerPlugin.obj
 0001:00020720       __ehhandler$?append@?$QList@PAVXMLTestFactory@U2@@@@QAEXABQAVXMLTestFactory@U2@@@Z 10021720 f   ORFMarkerPlugin.obj
 0001:00020740       __unwindfunclet$?createFactory@GTest_ORFMarkerTask@U2@@SAPAVXMLTestFactory@2@XZ$0 10021740 f   ORFMarkerPlugin.obj
 0001:0002074b       __unwindfunclet$?createFactory@GTest_ORFMarkerTask@U2@@SAPAVXMLTestFactory@2@XZ$1 1002174b f   ORFMarkerPlugin.obj
 0001:00020754       __unwindfunclet$?createFactory@GTest_ORFMarkerTask@U2@@SAPAVXMLTestFactory@2@XZ$2 10021754 f   ORFMarkerPlugin.obj
 0001:0002075d       __ehhandler$?createFactory@GTest_ORFMarkerTask@U2@@SAPAVXMLTestFactory@2@XZ 1002175d f   ORFMarkerPlugin.obj
 0001:00020780       __unwindfunclet$?createTest@GTest_ORFMarkerTaskFactory@GTest_ORFMarkerTask@U2@@UAEPAVGTest@3@PAVXMLTestFormat@3@ABVQString@@PAV43@PBVGTestEnvironment@3@ABV?$QList@PAVGTest@U2@@@@ABVQDomElement@@@Z$0 10021780 f   ORFMarkerPlugin.obj
 0001:0002078b       __ehhandler$?createTest@GTest_ORFMarkerTaskFactory@GTest_ORFMarkerTask@U2@@UAEPAVGTest@3@PAVXMLTestFormat@3@ABVQString@@PAV43@PBVGTestEnvironment@3@ABV?$QList@PAVGTest@U2@@@@ABVQDomElement@@@Z 1002178b f   ORFMarkerPlugin.obj
 0001:000207b0       __unwindfunclet$?createTestFactories@ORFMarkerTests@U2@@SA?AV?$QList@PAVXMLTestFactory@U2@@@@XZ$0 100217b0 f   ORFMarkerPlugin.obj
 0001:000207c9       __ehhandler$?createTestFactories@ORFMarkerTests@U2@@SA?AV?$QList@PAVXMLTestFactory@U2@@@@XZ 100217c9 f   ORFMarkerPlugin.obj
 0001:000207f0       __ehhandler$?detach_helper_grow@?$QList@PAVXMLTestFactory@U2@@@@AAEPAUNode@1@HH@Z 100217f0 f   ORFMarkerPlugin.obj
 0001:00020810       __unwindfunclet$?initViewContext@ORFViewContext@U2@@MAEXPAVGObjectView@2@@Z$0 10021810 f   ORFMarkerPlugin.obj
 0001:0002081b       __unwindfunclet$?initViewContext@ORFViewContext@U2@@MAEXPAVGObjectView@2@@Z$1 1002181b f   ORFMarkerPlugin.obj
 0001:00020835       __unwindfunclet$?initViewContext@ORFViewContext@U2@@MAEXPAVGObjectView@2@@Z$2 10021835 f   ORFMarkerPlugin.obj
 0001:0002084f       __unwindfunclet$?initViewContext@ORFViewContext@U2@@MAEXPAVGObjectView@2@@Z$3 1002184f f   ORFMarkerPlugin.obj
 0001:00020869       __unwindfunclet$?initViewContext@ORFViewContext@U2@@MAEXPAVGObjectView@2@@Z$4 10021869 f   ORFMarkerPlugin.obj
 0001:00020872       __ehhandler$?initViewContext@ORFViewContext@U2@@MAEXPAVGObjectView@2@@Z 10021872 f   ORFMarkerPlugin.obj
 0001:00020890       __unwindfunclet$?sl_showDialog@ORFViewContext@U2@@IAEXXZ$0 10021890 f   ORFMarkerPlugin.obj
 0001:0002089b       __unwindfunclet$?sl_showDialog@ORFViewContext@U2@@IAEXXZ$1 1002189b f   ORFMarkerPlugin.obj
 0001:000208a3       __unwindfunclet$?sl_showDialog@ORFViewContext@U2@@IAEXXZ$4 100218a3 f   ORFMarkerPlugin.obj
 0001:000208ab       __ehhandler$?sl_showDialog@ORFViewContext@U2@@IAEXXZ 100218ab f   ORFMarkerPlugin.obj
 0001:000208d0       __unwindfunclet$??$qRegisterMetaType@VU2Region@U2@@@@YAHPBDPAVU2Region@U2@@W4DefinedType@?$MetaTypeDefinedHelper@VU2Region@U2@@$00@QtPrivate@@@Z$0 100218d0 f   ORFMarkerTask.obj
 0001:000208d9       __ehhandler$??$qRegisterMetaType@VU2Region@U2@@@@YAHPBDPAVU2Region@U2@@W4DefinedType@?$MetaTypeDefinedHelper@VU2Region@U2@@$00@QtPrivate@@@Z 100218d9 f   ORFMarkerTask.obj
 0001:00020900       __unwindfunclet$??0FindORFsToAnnotationsTask@U2@@QAE@PAVAnnotationTableObject@1@ABVU2EntityRef@1@ABVORFAlgorithmSettings@1@ABVQString@@3@Z$0 10021900 f   ORFMarkerTask.obj
 0001:00020909       __unwindfunclet$??0FindORFsToAnnotationsTask@U2@@QAE@PAVAnnotationTableObject@1@ABVU2EntityRef@1@ABVORFAlgorithmSettings@1@ABVQString@@3@Z$1 10021909 f   ORFMarkerTask.obj
 0001:00020912       __unwindfunclet$??0FindORFsToAnnotationsTask@U2@@QAE@PAVAnnotationTableObject@1@ABVU2EntityRef@1@ABVORFAlgorithmSettings@1@ABVQString@@3@Z$2 10021912 f   ORFMarkerTask.obj
 0001:00020920       __unwindfunclet$??0FindORFsToAnnotationsTask@U2@@QAE@PAVAnnotationTableObject@1@ABVU2EntityRef@1@ABVORFAlgorithmSettings@1@ABVQString@@3@Z$3 10021920 f   ORFMarkerTask.obj
 0001:0002092f       __unwindfunclet$??0FindORFsToAnnotationsTask@U2@@QAE@PAVAnnotationTableObject@1@ABVU2EntityRef@1@ABVORFAlgorithmSettings@1@ABVQString@@3@Z$4 1002192f f   ORFMarkerTask.obj
 0001:0002093e       __unwindfunclet$??0FindORFsToAnnotationsTask@U2@@QAE@PAVAnnotationTableObject@1@ABVU2EntityRef@1@ABVORFAlgorithmSettings@1@ABVQString@@3@Z$5 1002193e f   ORFMarkerTask.obj
 0001:0002094d       __unwindfunclet$??0FindORFsToAnnotationsTask@U2@@QAE@PAVAnnotationTableObject@1@ABVU2EntityRef@1@ABVORFAlgorithmSettings@1@ABVQString@@3@Z$6 1002194d f   ORFMarkerTask.obj
 0001:00020956       __unwindfunclet$??0FindORFsToAnnotationsTask@U2@@QAE@PAVAnnotationTableObject@1@ABVU2EntityRef@1@ABVORFAlgorithmSettings@1@ABVQString@@3@Z$7 10021956 f   ORFMarkerTask.obj
 0001:00020961       __ehhandler$??0FindORFsToAnnotationsTask@U2@@QAE@PAVAnnotationTableObject@1@ABVU2EntityRef@1@ABVORFAlgorithmSettings@1@ABVQString@@3@Z 10021961 f   ORFMarkerTask.obj
 0001:00020980       __unwindfunclet$??0ORFAutoAnnotationsUpdater@U2@@QAE@XZ$0 10021980 f   ORFMarkerTask.obj
 0001:00020989       __unwindfunclet$??0ORFAutoAnnotationsUpdater@U2@@QAE@XZ$1 10021989 f   ORFMarkerTask.obj
 0001:00020992       __ehhandler$??0ORFAutoAnnotationsUpdater@U2@@QAE@XZ 10021992 f   ORFMarkerTask.obj
 0001:000209b0       __unwindfunclet$??1FindORFsToAnnotationsTask@U2@@UAE@XZ$0 100219b0 f   ORFMarkerTask.obj
 0001:000209b9       __unwindfunclet$??1FindORFsToAnnotationsTask@U2@@UAE@XZ$1 100219b9 f   ORFMarkerTask.obj
 0001:000209c7       __unwindfunclet$??1FindORFsToAnnotationsTask@U2@@UAE@XZ$2 100219c7 f   ORFMarkerTask.obj
 0001:000209d6       __unwindfunclet$??1FindORFsToAnnotationsTask@U2@@UAE@XZ$3 100219d6 f   ORFMarkerTask.obj
 0001:000209e5       __ehhandler$??1FindORFsToAnnotationsTask@U2@@UAE@XZ 100219e5 f   ORFMarkerTask.obj
 0001:00020a00       __unwindfunclet$??__EalgoLog@U2@@YAXXZ$0 10021a00 f   ORFMarkerTask.obj
 0001:00020a09       __ehhandler$??__EalgoLog@U2@@YAXXZ 10021a09 f   ORFMarkerTask.obj
 0001:00020a30       __unwindfunclet$??__EcmdLog@U2@@YAXXZ$0 10021a30 f   ORFMarkerTask.obj
 0001:00020a39       __ehhandler$??__EcmdLog@U2@@YAXXZ 10021a39 f   ORFMarkerTask.obj
 0001:00020a60       __unwindfunclet$??__EcoreLog@U2@@YAXXZ$0 10021a60 f   ORFMarkerTask.obj
 0001:00020a69       __ehhandler$??__EcoreLog@U2@@YAXXZ 10021a69 f   ORFMarkerTask.obj
 0001:00020a90       __unwindfunclet$??__EioLog@U2@@YAXXZ$0 10021a90 f   ORFMarkerTask.obj
 0001:00020a99       __ehhandler$??__EioLog@U2@@YAXXZ 10021a99 f   ORFMarkerTask.obj
 0001:00020ac0       __unwindfunclet$??__EperfLog@U2@@YAXXZ$0 10021ac0 f   ORFMarkerTask.obj
 0001:00020ac9       __ehhandler$??__EperfLog@U2@@YAXXZ 10021ac9 f   ORFMarkerTask.obj
 0001:00020af0       __unwindfunclet$??__EscriptLog@U2@@YAXXZ$0 10021af0 f   ORFMarkerTask.obj
 0001:00020af9       __ehhandler$??__EscriptLog@U2@@YAXXZ 10021af9 f   ORFMarkerTask.obj
 0001:00020b20       __unwindfunclet$??__EtaskLog@U2@@YAXXZ$0 10021b20 f   ORFMarkerTask.obj
 0001:00020b29       __ehhandler$??__EtaskLog@U2@@YAXXZ 10021b29 f   ORFMarkerTask.obj
 0001:00020b50       __unwindfunclet$??__EuiLog@U2@@YAXXZ$0 10021b50 f   ORFMarkerTask.obj
 0001:00020b59       __ehhandler$??__EuiLog@U2@@YAXXZ 10021b59 f   ORFMarkerTask.obj
 0001:00020b80       __unwindfunclet$??__EuserActLog@U2@@YAXXZ$0 10021b80 f   ORFMarkerTask.obj
 0001:00020b89       __ehhandler$??__EuserActLog@U2@@YAXXZ 10021b89 f   ORFMarkerTask.obj
 0001:00020bb0       __ehhandler$?append@?$QList@PAVTask@U2@@@@QAEXABQAVTask@U2@@@Z 10021bb0 f   ORFMarkerTask.obj
 0001:00020bd0       __ehhandler$?append@?$QList@V?$QSharedDataPointer@VAnnotationData@U2@@@@@@QAEXABV?$QSharedDataPointer@VAnnotationData@U2@@@@@Z 10021bd0 f   ORFMarkerTask.obj
 0001:00020bf0       __unwindfunclet$?createAutoAnnotationsUpdateTask@ORFAutoAnnotationsUpdater@U2@@UAEPAVTask@2@PBVAutoAnnotationObject@2@@Z$0 10021bf0 f   ORFMarkerTask.obj
 0001:00020bfb       __unwindfunclet$?createAutoAnnotationsUpdateTask@ORFAutoAnnotationsUpdater@U2@@UAEPAVTask@2@PBVAutoAnnotationObject@2@@Z$1 10021bfb f   ORFMarkerTask.obj
 0001:00020c15       __unwindfunclet$?createAutoAnnotationsUpdateTask@ORFAutoAnnotationsUpdater@U2@@UAEPAVTask@2@PBVAutoAnnotationObject@2@@Z$2 10021c15 f   ORFMarkerTask.obj
 0001:00020c2f       __unwindfunclet$?createAutoAnnotationsUpdateTask@ORFAutoAnnotationsUpdater@U2@@UAEPAVTask@2@PBVAutoAnnotationObject@2@@Z$3 10021c2f f   ORFMarkerTask.obj
 0001:00020c49       __ehhandler$?createAutoAnnotationsUpdateTask@ORFAutoAnnotationsUpdater@U2@@UAEPAVTask@2@PBVAutoAnnotationObject@2@@Z 10021c49 f   ORFMarkerTask.obj
 0001:00020c70       __ehhandler$?detach_helper_grow@?$QList@PAVTask@U2@@@@AAEPAUNode@1@HH@Z 10021c70 f   ORFMarkerTask.obj
 0001:00020c90       __ehhandler$?detach_helper_grow@?$QList@V?$QSharedDataPointer@VAnnotationData@U2@@@@@@AAEPAUNode@1@HH@Z 10021c90 f   ORFMarkerTask.obj
 0001:00020cb0       __unwindfunclet$?onSubTaskFinished@FindORFsToAnnotationsTask@U2@@UAE?AV?$QList@PAVTask@U2@@@@PAVTask@2@@Z$0 10021cb0 f   ORFMarkerTask.obj
 0001:00020cc9       __unwindfunclet$?onSubTaskFinished@FindORFsToAnnotationsTask@U2@@UAE?AV?$QList@PAVTask@U2@@@@PAVTask@2@@Z$1 10021cc9 f   ORFMarkerTask.obj
 0001:00020cd1       __unwindfunclet$?onSubTaskFinished@FindORFsToAnnotationsTask@U2@@UAE?AV?$QList@PAVTask@U2@@@@PAVTask@2@@Z$2 10021cd1 f   ORFMarkerTask.obj
 0001:00020cd9       __unwindfunclet$?onSubTaskFinished@FindORFsToAnnotationsTask@U2@@UAE?AV?$QList@PAVTask@U2@@@@PAVTask@2@@Z$3 10021cd9 f   ORFMarkerTask.obj
 0001:00020ce1       __unwindfunclet$?onSubTaskFinished@FindORFsToAnnotationsTask@U2@@UAE?AV?$QList@PAVTask@U2@@@@PAVTask@2@@Z$4 10021ce1 f   ORFMarkerTask.obj
 0001:00020ce9       __unwindfunclet$?onSubTaskFinished@FindORFsToAnnotationsTask@U2@@UAE?AV?$QList@PAVTask@U2@@@@PAVTask@2@@Z$5 10021ce9 f   ORFMarkerTask.obj
 0001:00020cf4       __unwindfunclet$?onSubTaskFinished@FindORFsToAnnotationsTask@U2@@UAE?AV?$QList@PAVTask@U2@@@@PAVTask@2@@Z$6 10021cf4 f   ORFMarkerTask.obj
 0001:00020cfc       __ehhandler$?onSubTaskFinished@FindORFsToAnnotationsTask@U2@@UAE?AV?$QList@PAVTask@U2@@@@PAVTask@2@@Z 10021cfc f   ORFMarkerTask.obj
 0001:00020d20       __unwindfunclet$?qt_metatype_id@?$QMetaTypeId@VU2Region@U2@@@@SAHXZ$0 10021d20 f   ORFMarkerTask.obj
 0001:00020d29       __ehhandler$?qt_metatype_id@?$QMetaTypeId@VU2Region@U2@@@@SAHXZ 10021d29 f   ORFMarkerTask.obj
 0001:00020d50       __unwindfunclet$?read@ORFSettingsKeys@U2@@SAXAAVORFAlgorithmSettings@2@PBVSettings@2@@Z$0 10021d50 f   ORFMarkerTask.obj
 0001:00020d59       __unwindfunclet$?read@ORFSettingsKeys@U2@@SAXAAVORFAlgorithmSettings@2@PBVSettings@2@@Z$1 10021d59 f   ORFMarkerTask.obj
 0001:00020d62       __unwindfunclet$?read@ORFSettingsKeys@U2@@SAXAAVORFAlgorithmSettings@2@PBVSettings@2@@Z$2 10021d62 f   ORFMarkerTask.obj
 0001:00020d6b       __unwindfunclet$?read@ORFSettingsKeys@U2@@SAXAAVORFAlgorithmSettings@2@PBVSettings@2@@Z$3 10021d6b f   ORFMarkerTask.obj
 0001:00020d74       __unwindfunclet$?read@ORFSettingsKeys@U2@@SAXAAVORFAlgorithmSettings@2@PBVSettings@2@@Z$4 10021d74 f   ORFMarkerTask.obj
 0001:00020d7d       __unwindfunclet$?read@ORFSettingsKeys@U2@@SAXAAVORFAlgorithmSettings@2@PBVSettings@2@@Z$5 10021d7d f   ORFMarkerTask.obj
 0001:00020d86       __unwindfunclet$?read@ORFSettingsKeys@U2@@SAXAAVORFAlgorithmSettings@2@PBVSettings@2@@Z$6 10021d86 f   ORFMarkerTask.obj
 0001:00020d8f       __unwindfunclet$?read@ORFSettingsKeys@U2@@SAXAAVORFAlgorithmSettings@2@PBVSettings@2@@Z$7 10021d8f f   ORFMarkerTask.obj
 0001:00020d98       __unwindfunclet$?read@ORFSettingsKeys@U2@@SAXAAVORFAlgorithmSettings@2@PBVSettings@2@@Z$8 10021d98 f   ORFMarkerTask.obj
 0001:00020da1       __unwindfunclet$?read@ORFSettingsKeys@U2@@SAXAAVORFAlgorithmSettings@2@PBVSettings@2@@Z$9 10021da1 f   ORFMarkerTask.obj
 0001:00020daa       __unwindfunclet$?read@ORFSettingsKeys@U2@@SAXAAVORFAlgorithmSettings@2@PBVSettings@2@@Z$10 10021daa f   ORFMarkerTask.obj
 0001:00020db3       __unwindfunclet$?read@ORFSettingsKeys@U2@@SAXAAVORFAlgorithmSettings@2@PBVSettings@2@@Z$11 10021db3 f   ORFMarkerTask.obj
 0001:00020dbc       __unwindfunclet$?read@ORFSettingsKeys@U2@@SAXAAVORFAlgorithmSettings@2@PBVSettings@2@@Z$12 10021dbc f   ORFMarkerTask.obj
 0001:00020dc5       __unwindfunclet$?read@ORFSettingsKeys@U2@@SAXAAVORFAlgorithmSettings@2@PBVSettings@2@@Z$13 10021dc5 f   ORFMarkerTask.obj
 0001:00020dce       __unwindfunclet$?read@ORFSettingsKeys@U2@@SAXAAVORFAlgorithmSettings@2@PBVSettings@2@@Z$14 10021dce f   ORFMarkerTask.obj
 0001:00020dd7       __unwindfunclet$?read@ORFSettingsKeys@U2@@SAXAAVORFAlgorithmSettings@2@PBVSettings@2@@Z$15 10021dd7 f   ORFMarkerTask.obj
 0001:00020de0       __unwindfunclet$?read@ORFSettingsKeys@U2@@SAXAAVORFAlgorithmSettings@2@PBVSettings@2@@Z$16 10021de0 f   ORFMarkerTask.obj
 0001:00020de9       __unwindfunclet$?read@ORFSettingsKeys@U2@@SAXAAVORFAlgorithmSettings@2@PBVSettings@2@@Z$17 10021de9 f   ORFMarkerTask.obj
 0001:00020df2       __unwindfunclet$?read@ORFSettingsKeys@U2@@SAXAAVORFAlgorithmSettings@2@PBVSettings@2@@Z$18 10021df2 f   ORFMarkerTask.obj
 0001:00020dfe       __unwindfunclet$?read@ORFSettingsKeys@U2@@SAXAAVORFAlgorithmSettings@2@PBVSettings@2@@Z$19 10021dfe f   ORFMarkerTask.obj
 0001:00020e07       __unwindfunclet$?read@ORFSettingsKeys@U2@@SAXAAVORFAlgorithmSettings@2@PBVSettings@2@@Z$20 10021e07 f   ORFMarkerTask.obj
 0001:00020e10       __unwindfunclet$?read@ORFSettingsKeys@U2@@SAXAAVORFAlgorithmSettings@2@PBVSettings@2@@Z$21 10021e10 f   ORFMarkerTask.obj
 0001:00020e19       __unwindfunclet$?read@ORFSettingsKeys@U2@@SAXAAVORFAlgorithmSettings@2@PBVSettings@2@@Z$22 10021e19 f   ORFMarkerTask.obj
 0001:00020e25       __unwindfunclet$?read@ORFSettingsKeys@U2@@SAXAAVORFAlgorithmSettings@2@PBVSettings@2@@Z$23 10021e25 f   ORFMarkerTask.obj
 0001:00020e2e       __ehhandler$?read@ORFSettingsKeys@U2@@SAXAAVORFAlgorithmSettings@2@PBVSettings@2@@Z 10021e2e f   ORFMarkerTask.obj
 0001:00020e50       __unwindfunclet$?save@ORFSettingsKeys@U2@@SAXABVORFAlgorithmSettings@2@PAVSettings@2@@Z$0 10021e50 f   ORFMarkerTask.obj
 0001:00020e59       __unwindfunclet$?save@ORFSettingsKeys@U2@@SAXABVORFAlgorithmSettings@2@PAVSettings@2@@Z$1 10021e59 f   ORFMarkerTask.obj
 0001:00020e62       __unwindfunclet$?save@ORFSettingsKeys@U2@@SAXABVORFAlgorithmSettings@2@PAVSettings@2@@Z$2 10021e62 f   ORFMarkerTask.obj
 0001:00020e6b       __unwindfunclet$?save@ORFSettingsKeys@U2@@SAXABVORFAlgorithmSettings@2@PAVSettings@2@@Z$3 10021e6b f   ORFMarkerTask.obj
 0001:00020e74       __unwindfunclet$?save@ORFSettingsKeys@U2@@SAXABVORFAlgorithmSettings@2@PAVSettings@2@@Z$4 10021e74 f   ORFMarkerTask.obj
 0001:00020e7d       __unwindfunclet$?save@ORFSettingsKeys@U2@@SAXABVORFAlgorithmSettings@2@PAVSettings@2@@Z$5 10021e7d f   ORFMarkerTask.obj
 0001:00020e86       __unwindfunclet$?save@ORFSettingsKeys@U2@@SAXABVORFAlgorithmSettings@2@PAVSettings@2@@Z$6 10021e86 f   ORFMarkerTask.obj
 0001:00020e8f       __unwindfunclet$?save@ORFSettingsKeys@U2@@SAXABVORFAlgorithmSettings@2@PAVSettings@2@@Z$7 10021e8f f   ORFMarkerTask.obj
 0001:00020e98       __unwindfunclet$?save@ORFSettingsKeys@U2@@SAXABVORFAlgorithmSettings@2@PAVSettings@2@@Z$8 10021e98 f   ORFMarkerTask.obj
 0001:00020ea1       __unwindfunclet$?save@ORFSettingsKeys@U2@@SAXABVORFAlgorithmSettings@2@PAVSettings@2@@Z$9 10021ea1 f   ORFMarkerTask.obj
 0001:00020eaa       __unwindfunclet$?save@ORFSettingsKeys@U2@@SAXABVORFAlgorithmSettings@2@PAVSettings@2@@Z$10 10021eaa f   ORFMarkerTask.obj
 0001:00020eb3       __unwindfunclet$?save@ORFSettingsKeys@U2@@SAXABVORFAlgorithmSettings@2@PAVSettings@2@@Z$11 10021eb3 f   ORFMarkerTask.obj
 0001:00020ebc       __ehhandler$?save@ORFSettingsKeys@U2@@SAXABVORFAlgorithmSettings@2@PAVSettings@2@@Z 10021ebc f   ORFMarkerTask.obj
 0001:00020ee0       __ehhandler$??0?$QList@VQString@@@@QAE@ABV0@@Z 10021ee0 f   ORFMarkerTests.obj
 0001:00020f00       __unwindfunclet$??0Translator@U2@@QAE@PBVU2SequenceObject@1@ABVQString@@@Z$0 10021f00 f   ORFMarkerTests.obj
 0001:00020f09       __ehhandler$??0Translator@U2@@QAE@PBVU2SequenceObject@1@ABVQString@@@Z 10021f09 f   ORFMarkerTests.obj
 0001:00020f30       __unwindfunclet$??__EalgoLog@U2@@YAXXZ$0 10021f30 f   ORFMarkerTests.obj
 0001:00020f39       __ehhandler$??__EalgoLog@U2@@YAXXZ 10021f39 f   ORFMarkerTests.obj
 0001:00020f60       __unwindfunclet$??__EcmdLog@U2@@YAXXZ$0 10021f60 f   ORFMarkerTests.obj
 0001:00020f69       __ehhandler$??__EcmdLog@U2@@YAXXZ 10021f69 f   ORFMarkerTests.obj
 0001:00020f90       __unwindfunclet$??__EcoreLog@U2@@YAXXZ$0 10021f90 f   ORFMarkerTests.obj
 0001:00020f99       __ehhandler$??__EcoreLog@U2@@YAXXZ 10021f99 f   ORFMarkerTests.obj
 0001:00020fc0       __unwindfunclet$??__EioLog@U2@@YAXXZ$0 10021fc0 f   ORFMarkerTests.obj
 0001:00020fc9       __ehhandler$??__EioLog@U2@@YAXXZ 10021fc9 f   ORFMarkerTests.obj
 0001:00020ff0       __unwindfunclet$??__EperfLog@U2@@YAXXZ$0 10021ff0 f   ORFMarkerTests.obj
 0001:00020ff9       __ehhandler$??__EperfLog@U2@@YAXXZ 10021ff9 f   ORFMarkerTests.obj
 0001:00021020       __unwindfunclet$??__EscriptLog@U2@@YAXXZ$0 10022020 f   ORFMarkerTests.obj
 0001:00021029       __ehhandler$??__EscriptLog@U2@@YAXXZ 10022029 f   ORFMarkerTests.obj
 0001:00021050       __unwindfunclet$??__EtaskLog@U2@@YAXXZ$0 10022050 f   ORFMarkerTests.obj
 0001:00021059       __ehhandler$??__EtaskLog@U2@@YAXXZ 10022059 f   ORFMarkerTests.obj
 0001:00021080       __unwindfunclet$??__EuiLog@U2@@YAXXZ$0 10022080 f   ORFMarkerTests.obj
 0001:00021089       __ehhandler$??__EuiLog@U2@@YAXXZ 10022089 f   ORFMarkerTests.obj
 0001:000210b0       __unwindfunclet$??__EuserActLog@U2@@YAXXZ$0 100220b0 f   ORFMarkerTests.obj
 0001:000210b9       __ehhandler$??__EuserActLog@U2@@YAXXZ 100220b9 f   ORFMarkerTests.obj
 0001:000210e0       __ehhandler$?detach_helper@?$QList@VQString@@@@AAEXH@Z 100220e0 f   ORFMarkerTests.obj
 0001:00021100       __unwindfunclet$?init@GTest_ORFMarkerTask@U2@@QAEXPAVXMLTestFormat@2@ABVQDomElement@@@Z$0 10022100 f   ORFMarkerTests.obj
 0001:00021109       __unwindfunclet$?init@GTest_ORFMarkerTask@U2@@QAEXPAVXMLTestFormat@2@ABVQDomElement@@@Z$1 10022109 f   ORFMarkerTests.obj
 0001:00021112       __unwindfunclet$?init@GTest_ORFMarkerTask@U2@@QAEXPAVXMLTestFormat@2@ABVQDomElement@@@Z$2 10022112 f   ORFMarkerTests.obj
 0001:0002111b       __unwindfunclet$?init@GTest_ORFMarkerTask@U2@@QAEXPAVXMLTestFormat@2@ABVQDomElement@@@Z$3 1002211b f   ORFMarkerTests.obj
 0001:00021124       __unwindfunclet$?init@GTest_ORFMarkerTask@U2@@QAEXPAVXMLTestFormat@2@ABVQDomElement@@@Z$4 10022124 f   ORFMarkerTests.obj
 0001:0002112d       __unwindfunclet$?init@GTest_ORFMarkerTask@U2@@QAEXPAVXMLTestFormat@2@ABVQDomElement@@@Z$5 1002212d f   ORFMarkerTests.obj
 0001:00021139       __unwindfunclet$?init@GTest_ORFMarkerTask@U2@@QAEXPAVXMLTestFormat@2@ABVQDomElement@@@Z$6 10022139 f   ORFMarkerTests.obj
 0001:00021142       __unwindfunclet$?init@GTest_ORFMarkerTask@U2@@QAEXPAVXMLTestFormat@2@ABVQDomElement@@@Z$7 10022142 f   ORFMarkerTests.obj
 0001:0002114b       __unwindfunclet$?init@GTest_ORFMarkerTask@U2@@QAEXPAVXMLTestFormat@2@ABVQDomElement@@@Z$8 1002214b f   ORFMarkerTests.obj
 0001:00021154       __unwindfunclet$?init@GTest_ORFMarkerTask@U2@@QAEXPAVXMLTestFormat@2@ABVQDomElement@@@Z$9 10022154 f   ORFMarkerTests.obj
 0001:0002115c       __unwindfunclet$?init@GTest_ORFMarkerTask@U2@@QAEXPAVXMLTestFormat@2@ABVQDomElement@@@Z$10 1002215c f   ORFMarkerTests.obj
 0001:00021164       __unwindfunclet$?init@GTest_ORFMarkerTask@U2@@QAEXPAVXMLTestFormat@2@ABVQDomElement@@@Z$11 10022164 f   ORFMarkerTests.obj
 0001:0002116d       __unwindfunclet$?init@GTest_ORFMarkerTask@U2@@QAEXPAVXMLTestFormat@2@ABVQDomElement@@@Z$12 1002216d f   ORFMarkerTests.obj
 0001:00021176       __unwindfunclet$?init@GTest_ORFMarkerTask@U2@@QAEXPAVXMLTestFormat@2@ABVQDomElement@@@Z$13 10022176 f   ORFMarkerTests.obj
 0001:0002117f       __unwindfunclet$?init@GTest_ORFMarkerTask@U2@@QAEXPAVXMLTestFormat@2@ABVQDomElement@@@Z$14 1002217f f   ORFMarkerTests.obj
 0001:00021187       __unwindfunclet$?init@GTest_ORFMarkerTask@U2@@QAEXPAVXMLTestFormat@2@ABVQDomElement@@@Z$18 10022187 f   ORFMarkerTests.obj
 0001:00021190       __unwindfunclet$?init@GTest_ORFMarkerTask@U2@@QAEXPAVXMLTestFormat@2@ABVQDomElement@@@Z$19 10022190 f   ORFMarkerTests.obj
 0001:00021199       __unwindfunclet$?init@GTest_ORFMarkerTask@U2@@QAEXPAVXMLTestFormat@2@ABVQDomElement@@@Z$20 10022199 f   ORFMarkerTests.obj
 0001:000211a2       __unwindfunclet$?init@GTest_ORFMarkerTask@U2@@QAEXPAVXMLTestFormat@2@ABVQDomElement@@@Z$15 100221a2 f   ORFMarkerTests.obj
 0001:000211ab       __unwindfunclet$?init@GTest_ORFMarkerTask@U2@@QAEXPAVXMLTestFormat@2@ABVQDomElement@@@Z$16 100221ab f   ORFMarkerTests.obj
 0001:000211b4       __unwindfunclet$?init@GTest_ORFMarkerTask@U2@@QAEXPAVXMLTestFormat@2@ABVQDomElement@@@Z$17 100221b4 f   ORFMarkerTests.obj
 0001:000211bd       __unwindfunclet$?init@GTest_ORFMarkerTask@U2@@QAEXPAVXMLTestFormat@2@ABVQDomElement@@@Z$21 100221bd f   ORFMarkerTests.obj
 0001:000211c6       __unwindfunclet$?init@GTest_ORFMarkerTask@U2@@QAEXPAVXMLTestFormat@2@ABVQDomElement@@@Z$22 100221c6 f   ORFMarkerTests.obj
 0001:000211cf       __unwindfunclet$?init@GTest_ORFMarkerTask@U2@@QAEXPAVXMLTestFormat@2@ABVQDomElement@@@Z$23 100221cf f   ORFMarkerTests.obj
 0001:000211d8       __unwindfunclet$?init@GTest_ORFMarkerTask@U2@@QAEXPAVXMLTestFormat@2@ABVQDomElement@@@Z$27 100221d8 f   ORFMarkerTests.obj
 0001:000211e1       __unwindfunclet$?init@GTest_ORFMarkerTask@U2@@QAEXPAVXMLTestFormat@2@ABVQDomElement@@@Z$28 100221e1 f   ORFMarkerTests.obj
 0001:000211ea       __unwindfunclet$?init@GTest_ORFMarkerTask@U2@@QAEXPAVXMLTestFormat@2@ABVQDomElement@@@Z$29 100221ea f   ORFMarkerTests.obj
 0001:000211f3       __unwindfunclet$?init@GTest_ORFMarkerTask@U2@@QAEXPAVXMLTestFormat@2@ABVQDomElement@@@Z$30 100221f3 f   ORFMarkerTests.obj
 0001:000211fc       __unwindfunclet$?init@GTest_ORFMarkerTask@U2@@QAEXPAVXMLTestFormat@2@ABVQDomElement@@@Z$31 100221fc f   ORFMarkerTests.obj
 0001:00021205       __unwindfunclet$?init@GTest_ORFMarkerTask@U2@@QAEXPAVXMLTestFormat@2@ABVQDomElement@@@Z$32 10022205 f   ORFMarkerTests.obj
 0001:0002120e       __unwindfunclet$?init@GTest_ORFMarkerTask@U2@@QAEXPAVXMLTestFormat@2@ABVQDomElement@@@Z$33 1002220e f   ORFMarkerTests.obj
 0001:00021217       __unwindfunclet$?init@GTest_ORFMarkerTask@U2@@QAEXPAVXMLTestFormat@2@ABVQDomElement@@@Z$34 10022217 f   ORFMarkerTests.obj
 0001:00021220       __unwindfunclet$?init@GTest_ORFMarkerTask@U2@@QAEXPAVXMLTestFormat@2@ABVQDomElement@@@Z$35 10022220 f   ORFMarkerTests.obj
 0001:0002122c       __unwindfunclet$?init@GTest_ORFMarkerTask@U2@@QAEXPAVXMLTestFormat@2@ABVQDomElement@@@Z$36 1002222c f   ORFMarkerTests.obj
 0001:00021235       __unwindfunclet$?init@GTest_ORFMarkerTask@U2@@QAEXPAVXMLTestFormat@2@ABVQDomElement@@@Z$37 10022235 f   ORFMarkerTests.obj
 0001:0002123e       __unwindfunclet$?init@GTest_ORFMarkerTask@U2@@QAEXPAVXMLTestFormat@2@ABVQDomElement@@@Z$41 1002223e f   ORFMarkerTests.obj
 0001:00021247       __unwindfunclet$?init@GTest_ORFMarkerTask@U2@@QAEXPAVXMLTestFormat@2@ABVQDomElement@@@Z$42 10022247 f   ORFMarkerTests.obj
 0001:00021253       __unwindfunclet$?init@GTest_ORFMarkerTask@U2@@QAEXPAVXMLTestFormat@2@ABVQDomElement@@@Z$43 10022253 f   ORFMarkerTests.obj
 0001:0002125c       __unwindfunclet$?init@GTest_ORFMarkerTask@U2@@QAEXPAVXMLTestFormat@2@ABVQDomElement@@@Z$44 1002225c f   ORFMarkerTests.obj
 0001:00021265       __unwindfunclet$?init@GTest_ORFMarkerTask@U2@@QAEXPAVXMLTestFormat@2@ABVQDomElement@@@Z$48 10022265 f   ORFMarkerTests.obj
 0001:0002126e       __unwindfunclet$?init@GTest_ORFMarkerTask@U2@@QAEXPAVXMLTestFormat@2@ABVQDomElement@@@Z$49 1002226e f   ORFMarkerTests.obj
 0001:0002127a       __unwindfunclet$?init@GTest_ORFMarkerTask@U2@@QAEXPAVXMLTestFormat@2@ABVQDomElement@@@Z$50 1002227a f   ORFMarkerTests.obj
 0001:00021283       __unwindfunclet$?init@GTest_ORFMarkerTask@U2@@QAEXPAVXMLTestFormat@2@ABVQDomElement@@@Z$51 10022283 f   ORFMarkerTests.obj
 0001:0002128c       __unwindfunclet$?init@GTest_ORFMarkerTask@U2@@QAEXPAVXMLTestFormat@2@ABVQDomElement@@@Z$52 1002228c f   ORFMarkerTests.obj
 0001:00021298       __unwindfunclet$?init@GTest_ORFMarkerTask@U2@@QAEXPAVXMLTestFormat@2@ABVQDomElement@@@Z$53 10022298 f   ORFMarkerTests.obj
 0001:000212a1       __unwindfunclet$?init@GTest_ORFMarkerTask@U2@@QAEXPAVXMLTestFormat@2@ABVQDomElement@@@Z$54 100222a1 f   ORFMarkerTests.obj
 0001:000212aa       __unwindfunclet$?init@GTest_ORFMarkerTask@U2@@QAEXPAVXMLTestFormat@2@ABVQDomElement@@@Z$58 100222aa f   ORFMarkerTests.obj
 0001:000212b3       __unwindfunclet$?init@GTest_ORFMarkerTask@U2@@QAEXPAVXMLTestFormat@2@ABVQDomElement@@@Z$59 100222b3 f   ORFMarkerTests.obj
 0001:000212bc       __unwindfunclet$?init@GTest_ORFMarkerTask@U2@@QAEXPAVXMLTestFormat@2@ABVQDomElement@@@Z$60 100222bc f   ORFMarkerTests.obj
 0001:000212c5       __unwindfunclet$?init@GTest_ORFMarkerTask@U2@@QAEXPAVXMLTestFormat@2@ABVQDomElement@@@Z$61 100222c5 f   ORFMarkerTests.obj
 0001:000212ce       __unwindfunclet$?init@GTest_ORFMarkerTask@U2@@QAEXPAVXMLTestFormat@2@ABVQDomElement@@@Z$62 100222ce f   ORFMarkerTests.obj
 0001:000212d7       __unwindfunclet$?init@GTest_ORFMarkerTask@U2@@QAEXPAVXMLTestFormat@2@ABVQDomElement@@@Z$63 100222d7 f   ORFMarkerTests.obj
 0001:000212e0       __unwindfunclet$?init@GTest_ORFMarkerTask@U2@@QAEXPAVXMLTestFormat@2@ABVQDomElement@@@Z$64 100222e0 f   ORFMarkerTests.obj
 0001:000212e9       __unwindfunclet$?init@GTest_ORFMarkerTask@U2@@QAEXPAVXMLTestFormat@2@ABVQDomElement@@@Z$55 100222e9 f   ORFMarkerTests.obj
 0001:000212f2       __unwindfunclet$?init@GTest_ORFMarkerTask@U2@@QAEXPAVXMLTestFormat@2@ABVQDomElement@@@Z$56 100222f2 f   ORFMarkerTests.obj
 0001:000212fb       __unwindfunclet$?init@GTest_ORFMarkerTask@U2@@QAEXPAVXMLTestFormat@2@ABVQDomElement@@@Z$57 100222fb f   ORFMarkerTests.obj
 0001:00021304       __unwindfunclet$?init@GTest_ORFMarkerTask@U2@@QAEXPAVXMLTestFormat@2@ABVQDomElement@@@Z$45 10022304 f   ORFMarkerTests.obj
 0001:0002130d       __unwindfunclet$?init@GTest_ORFMarkerTask@U2@@QAEXPAVXMLTestFormat@2@ABVQDomElement@@@Z$46 1002230d f   ORFMarkerTests.obj
 0001:00021316       __unwindfunclet$?init@GTest_ORFMarkerTask@U2@@QAEXPAVXMLTestFormat@2@ABVQDomElement@@@Z$47 10022316 f   ORFMarkerTests.obj
 0001:0002131f       __unwindfunclet$?init@GTest_ORFMarkerTask@U2@@QAEXPAVXMLTestFormat@2@ABVQDomElement@@@Z$38 1002231f f   ORFMarkerTests.obj
 0001:00021328       __unwindfunclet$?init@GTest_ORFMarkerTask@U2@@QAEXPAVXMLTestFormat@2@ABVQDomElement@@@Z$39 10022328 f   ORFMarkerTests.obj
 0001:00021331       __unwindfunclet$?init@GTest_ORFMarkerTask@U2@@QAEXPAVXMLTestFormat@2@ABVQDomElement@@@Z$40 10022331 f   ORFMarkerTests.obj
 0001:0002133a       __unwindfunclet$?init@GTest_ORFMarkerTask@U2@@QAEXPAVXMLTestFormat@2@ABVQDomElement@@@Z$24 1002233a f   ORFMarkerTests.obj
 0001:00021343       __unwindfunclet$?init@GTest_ORFMarkerTask@U2@@QAEXPAVXMLTestFormat@2@ABVQDomElement@@@Z$25 10022343 f   ORFMarkerTests.obj
 0001:0002134c       __unwindfunclet$?init@GTest_ORFMarkerTask@U2@@QAEXPAVXMLTestFormat@2@ABVQDomElement@@@Z$26 1002234c f   ORFMarkerTests.obj
 0001:00021355       __ehhandler$?init@GTest_ORFMarkerTask@U2@@QAEXPAVXMLTestFormat@2@ABVQDomElement@@@Z 10022355 f   ORFMarkerTests.obj
 0001:00021380       __unwindfunclet$?node_copy@?$QList@VQString@@@@AAEXPAUNode@1@00@Z$5 10022380 f   ORFMarkerTests.obj
 0001:00021391       __ehhandler$?node_copy@?$QList@VQString@@@@AAEXPAUNode@1@00@Z 10022391 f   ORFMarkerTests.obj
 0001:000213b0       __unwindfunclet$?prepare@GTest_ORFMarkerTask@U2@@UAEXXZ$0 100223b0 f   ORFMarkerTests.obj
 0001:000213b9       __unwindfunclet$?prepare@GTest_ORFMarkerTask@U2@@UAEXXZ$1 100223b9 f   ORFMarkerTests.obj
 0001:000213c4       __unwindfunclet$?prepare@GTest_ORFMarkerTask@U2@@UAEXXZ$2 100223c4 f   ORFMarkerTests.obj
 0001:000213de       __ehhandler$?prepare@GTest_ORFMarkerTask@U2@@UAEXXZ 100223de f   ORFMarkerTests.obj
 0001:00021400       __ehhandler$?reallocData@?$QVector@VU2Region@U2@@@@AAEXHHV?$QFlags@W4AllocationOption@QArrayData@@@@@Z 10022400 f   ORFMarkerTests.obj
 0001:00021420       __unwindfunclet$?report@GTest_ORFMarkerTask@U2@@UAE?AW4ReportResult@Task@2@XZ$0 10022420 f   ORFMarkerTests.obj
 0001:00021428       __unwindfunclet$?report@GTest_ORFMarkerTask@U2@@UAE?AW4ReportResult@Task@2@XZ$1 10022428 f   ORFMarkerTests.obj
 0001:00021430       __unwindfunclet$?report@GTest_ORFMarkerTask@U2@@UAE?AW4ReportResult@Task@2@XZ$2 10022430 f   ORFMarkerTests.obj
 0001:00021438       __unwindfunclet$?report@GTest_ORFMarkerTask@U2@@UAE?AW4ReportResult@Task@2@XZ$3 10022438 f   ORFMarkerTests.obj
 0001:00021441       __unwindfunclet$?report@GTest_ORFMarkerTask@U2@@UAE?AW4ReportResult@Task@2@XZ$4 10022441 f   ORFMarkerTests.obj
 0001:0002144a       __unwindfunclet$?report@GTest_ORFMarkerTask@U2@@UAE?AW4ReportResult@Task@2@XZ$5 1002244a f   ORFMarkerTests.obj
 0001:00021453       __unwindfunclet$?report@GTest_ORFMarkerTask@U2@@UAE?AW4ReportResult@Task@2@XZ$6 10022453 f   ORFMarkerTests.obj
 0001:0002145c       __ehhandler$?report@GTest_ORFMarkerTask@U2@@UAE?AW4ReportResult@Task@2@XZ 1002245c f   ORFMarkerTests.obj
 0001:00021480       __unwindfunclet$??0?$QForeachContainer@$$CBV?$QVector@VU2Region@U2@@@@@@QAE@ABV?$QVector@VU2Region@U2@@@@@Z$0 10022480 f   ORFQuery.obj
 0001:00021488       __ehhandler$??0?$QForeachContainer@$$CBV?$QVector@VU2Region@U2@@@@@@QAE@ABV?$QVector@VU2Region@U2@@@@@Z 10022488 f   ORFQuery.obj
 0001:000214b0       __ehhandler$??0?$QList@PAVDNATranslation@U2@@@@QAE@ABV0@@Z 100224b0 f   ORFQuery.obj
 0001:000214d0       __ehhandler$??0?$QList@PAVORFFindTask@U2@@@@QAE@ABV0@@Z 100224d0 f   ORFQuery.obj
 0001:000214f0       __ehhandler$??0?$QList@V?$QSharedDataPointer@VAnnotationData@U2@@@@@@QAE@ABV0@@Z 100224f0 f   ORFQuery.obj
 0001:00021510       __unwindfunclet$??0QDORFActor@U2@@QAE@PBVQDActorPrototype@1@@Z$0 10022510 f   ORFQuery.obj
 0001:00021519       __unwindfunclet$??0QDORFActor@U2@@QAE@PBVQDActorPrototype@1@@Z$1 10022519 f   ORFQuery.obj
 0001:00021524       __unwindfunclet$??0QDORFActor@U2@@QAE@PBVQDActorPrototype@1@@Z$2 10022524 f   ORFQuery.obj
 0001:0002152f       __unwindfunclet$??0QDORFActor@U2@@QAE@PBVQDActorPrototype@1@@Z$3 1002252f f   ORFQuery.obj
 0001:00021538       __unwindfunclet$??0QDORFActor@U2@@QAE@PBVQDActorPrototype@1@@Z$4 10022538 f   ORFQuery.obj
 0001:00021541       __ehhandler$??0QDORFActor@U2@@QAE@PBVQDActorPrototype@1@@Z 10022541 f   ORFQuery.obj
 0001:00021560       __unwindfunclet$??0QDORFActorPrototype@U2@@QAE@XZ$0 10022560 f   ORFQuery.obj
 0001:00021569       __unwindfunclet$??0QDORFActorPrototype@U2@@QAE@XZ$1 10022569 f   ORFQuery.obj
 0001:00021572       __unwindfunclet$??0QDORFActorPrototype@U2@@QAE@XZ$2 10022572 f   ORFQuery.obj
 0001:0002157b       __unwindfunclet$??0QDORFActorPrototype@U2@@QAE@XZ$3 1002257b f   ORFQuery.obj
 0001:00021584       __unwindfunclet$??0QDORFActorPrototype@U2@@QAE@XZ$4 10022584 f   ORFQuery.obj
 0001:0002158d       __unwindfunclet$??0QDORFActorPrototype@U2@@QAE@XZ$5 1002258d f   ORFQuery.obj
 0001:00021599       __unwindfunclet$??0QDORFActorPrototype@U2@@QAE@XZ$6 10022599 f   ORFQuery.obj
 0001:000215a5       __unwindfunclet$??0QDORFActorPrototype@U2@@QAE@XZ$7 100225a5 f   ORFQuery.obj
 0001:000215ae       __unwindfunclet$??0QDORFActorPrototype@U2@@QAE@XZ$8 100225ae f   ORFQuery.obj
 0001:000215b7       __unwindfunclet$??0QDORFActorPrototype@U2@@QAE@XZ$9 100225b7 f   ORFQuery.obj
 0001:000215c3       __unwindfunclet$??0QDORFActorPrototype@U2@@QAE@XZ$10 100225c3 f   ORFQuery.obj
 0001:000215cc       __unwindfunclet$??0QDORFActorPrototype@U2@@QAE@XZ$11 100225cc f   ORFQuery.obj
 0001:000215d8       __unwindfunclet$??0QDORFActorPrototype@U2@@QAE@XZ$12 100225d8 f   ORFQuery.obj
 0001:000215e4       __unwindfunclet$??0QDORFActorPrototype@U2@@QAE@XZ$13 100225e4 f   ORFQuery.obj
 0001:000215ed       __unwindfunclet$??0QDORFActorPrototype@U2@@QAE@XZ$14 100225ed f   ORFQuery.obj
 0001:000215f6       __unwindfunclet$??0QDORFActorPrototype@U2@@QAE@XZ$15 100225f6 f   ORFQuery.obj
 0001:00021602       __unwindfunclet$??0QDORFActorPrototype@U2@@QAE@XZ$16 10022602 f   ORFQuery.obj
 0001:0002160b       __unwindfunclet$??0QDORFActorPrototype@U2@@QAE@XZ$17 1002260b f   ORFQuery.obj
 0001:00021614       __unwindfunclet$??0QDORFActorPrototype@U2@@QAE@XZ$18 10022614 f   ORFQuery.obj
 0001:00021620       __unwindfunclet$??0QDORFActorPrototype@U2@@QAE@XZ$19 10022620 f   ORFQuery.obj
 0001:00021629       __unwindfunclet$??0QDORFActorPrototype@U2@@QAE@XZ$20 10022629 f   ORFQuery.obj
 0001:00021632       __unwindfunclet$??0QDORFActorPrototype@U2@@QAE@XZ$21 10022632 f   ORFQuery.obj
 0001:0002163e       __unwindfunclet$??0QDORFActorPrototype@U2@@QAE@XZ$22 1002263e f   ORFQuery.obj
 0001:00021647       __unwindfunclet$??0QDORFActorPrototype@U2@@QAE@XZ$23 10022647 f   ORFQuery.obj
 0001:00021653       __unwindfunclet$??0QDORFActorPrototype@U2@@QAE@XZ$24 10022653 f   ORFQuery.obj
 0001:0002165f       __unwindfunclet$??0QDORFActorPrototype@U2@@QAE@XZ$25 1002265f f   ORFQuery.obj
 0001:00021668       __unwindfunclet$??0QDORFActorPrototype@U2@@QAE@XZ$26 10022668 f   ORFQuery.obj
 0001:00021674       __unwindfunclet$??0QDORFActorPrototype@U2@@QAE@XZ$27 10022674 f   ORFQuery.obj
 0001:00021680       __unwindfunclet$??0QDORFActorPrototype@U2@@QAE@XZ$28 10022680 f   ORFQuery.obj
 0001:0002168b       __unwindfunclet$??0QDORFActorPrototype@U2@@QAE@XZ$29 1002268b f   ORFQuery.obj
 0001:000216a5       __unwindfunclet$??0QDORFActorPrototype@U2@@QAE@XZ$31 100226a5 f   ORFQuery.obj
 0001:000216b0       __unwindfunclet$??0QDORFActorPrototype@U2@@QAE@XZ$32 100226b0 f   ORFQuery.obj
 0001:000216ca       __unwindfunclet$??0QDORFActorPrototype@U2@@QAE@XZ$34 100226ca f   ORFQuery.obj
 0001:000216d5       __unwindfunclet$??0QDORFActorPrototype@U2@@QAE@XZ$35 100226d5 f   ORFQuery.obj
 0001:000216ef       __unwindfunclet$??0QDORFActorPrototype@U2@@QAE@XZ$37 100226ef f   ORFQuery.obj
 0001:000216fa       __unwindfunclet$??0QDORFActorPrototype@U2@@QAE@XZ$38 100226fa f   ORFQuery.obj
 0001:00021714       __unwindfunclet$??0QDORFActorPrototype@U2@@QAE@XZ$40 10022714 f   ORFQuery.obj
 0001:0002171f       __unwindfunclet$??0QDORFActorPrototype@U2@@QAE@XZ$41 1002271f f   ORFQuery.obj
 0001:00021739       __unwindfunclet$??0QDORFActorPrototype@U2@@QAE@XZ$43 10022739 f   ORFQuery.obj
 0001:00021744       __unwindfunclet$??0QDORFActorPrototype@U2@@QAE@XZ$44 10022744 f   ORFQuery.obj
 0001:0002175e       __unwindfunclet$??0QDORFActorPrototype@U2@@QAE@XZ$46 1002275e f   ORFQuery.obj
 0001:00021769       __unwindfunclet$??0QDORFActorPrototype@U2@@QAE@XZ$47 10022769 f   ORFQuery.obj
 0001:00021783       __unwindfunclet$??0QDORFActorPrototype@U2@@QAE@XZ$49 10022783 f   ORFQuery.obj
 0001:0002178e       __unwindfunclet$??0QDORFActorPrototype@U2@@QAE@XZ$50 1002278e f   ORFQuery.obj
 0001:000217ad       __unwindfunclet$??0QDORFActorPrototype@U2@@QAE@XZ$52 100227ad f   ORFQuery.obj
 0001:000217b5       __unwindfunclet$??0QDORFActorPrototype@U2@@QAE@XZ$53 100227b5 f   ORFQuery.obj
 0001:000217bd       __unwindfunclet$??0QDORFActorPrototype@U2@@QAE@XZ$54 100227bd f   ORFQuery.obj
 0001:000217c6       __unwindfunclet$??0QDORFActorPrototype@U2@@QAE@XZ$55 100227c6 f   ORFQuery.obj
 0001:000217cf       __unwindfunclet$??0QDORFActorPrototype@U2@@QAE@XZ$56 100227cf f   ORFQuery.obj
 0001:000217d8       __unwindfunclet$??0QDORFActorPrototype@U2@@QAE@XZ$57 100227d8 f   ORFQuery.obj
 0001:000217e1       __unwindfunclet$??0QDORFActorPrototype@U2@@QAE@XZ$58 100227e1 f   ORFQuery.obj
 0001:000217ea       __unwindfunclet$??0QDORFActorPrototype@U2@@QAE@XZ$59 100227ea f   ORFQuery.obj
 0001:000217f3       __unwindfunclet$??0QDORFActorPrototype@U2@@QAE@XZ$60 100227f3 f   ORFQuery.obj
 0001:000217fc       __unwindfunclet$??0QDORFActorPrototype@U2@@QAE@XZ$61 100227fc f   ORFQuery.obj
 0001:00021807       __unwindfunclet$??0QDORFActorPrototype@U2@@QAE@XZ$62 10022807 f   ORFQuery.obj
 0001:00021812       __unwindfunclet$??0QDORFActorPrototype@U2@@QAE@XZ$63 10022812 f   ORFQuery.obj
 0001:0002181a       __unwindfunclet$??0QDORFActorPrototype@U2@@QAE@XZ$64 1002281a f   ORFQuery.obj
 0001:00021823       __unwindfunclet$??0QDORFActorPrototype@U2@@QAE@XZ$65 10022823 f   ORFQuery.obj
 0001:0002182b       __unwindfunclet$??0QDORFActorPrototype@U2@@QAE@XZ$66 1002282b f   ORFQuery.obj
 0001:00021833       __unwindfunclet$??0QDORFActorPrototype@U2@@QAE@XZ$67 10022833 f   ORFQuery.obj
 0001:0002183c       __unwindfunclet$??0QDORFActorPrototype@U2@@QAE@XZ$68 1002283c f   ORFQuery.obj
 0001:00021847       __unwindfunclet$??0QDORFActorPrototype@U2@@QAE@XZ$69 10022847 f   ORFQuery.obj
 0001:00021852       __ehhandler$??0QDORFActorPrototype@U2@@QAE@XZ 10022852 f   ORFQuery.obj
 0001:00021870       __unwindfunclet$??1QDORFActor@U2@@UAE@XZ$0 10022870 f   ORFQuery.obj
 0001:00021879       __ehhandler$??1QDORFActor@U2@@UAE@XZ 10022879 f   ORFQuery.obj
 0001:000218a0       __unwindfunclet$??A?$QMap@VQString@@VQVariant@@@@QAEAAVQVariant@@ABVQString@@@Z$0 100228a0 f   ORFQuery.obj
 0001:000218a9       __ehhandler$??A?$QMap@VQString@@VQVariant@@@@QAEAAVQVariant@@ABVQString@@@Z 100228a9 f   ORFQuery.obj
 0001:000218d0       __ehhandler$??Y?$QList@VORFFindResult@U2@@@@QAEAAV0@ABV0@@Z 100228d0 f   ORFQuery.obj
 0001:000218f0       __unwindfunclet$??_GQDORFActor@U2@@UAEPAXI@Z$0 100228f0 f   ORFQuery.obj
 0001:000218f9       __ehhandler$??_GQDORFActor@U2@@UAEPAXI@Z 100228f9 f   ORFQuery.obj
 0001:00021920       __unwindfunclet$??__EalgoLog@U2@@YAXXZ$0 10022920 f   ORFQuery.obj
 0001:00021929       __ehhandler$??__EalgoLog@U2@@YAXXZ 10022929 f   ORFQuery.obj
 0001:00021950       __unwindfunclet$??__EcmdLog@U2@@YAXXZ$0 10022950 f   ORFQuery.obj
 0001:00021959       __ehhandler$??__EcmdLog@U2@@YAXXZ 10022959 f   ORFQuery.obj
 0001:00021980       __unwindfunclet$??__EcoreLog@U2@@YAXXZ$0 10022980 f   ORFQuery.obj
 0001:00021989       __ehhandler$??__EcoreLog@U2@@YAXXZ 10022989 f   ORFQuery.obj
 0001:000219b0       __unwindfunclet$??__EioLog@U2@@YAXXZ$0 100229b0 f   ORFQuery.obj
 0001:000219b9       __ehhandler$??__EioLog@U2@@YAXXZ 100229b9 f   ORFQuery.obj
 0001:000219e0       __unwindfunclet$??__EperfLog@U2@@YAXXZ$0 100229e0 f   ORFQuery.obj
 0001:000219e9       __ehhandler$??__EperfLog@U2@@YAXXZ 100229e9 f   ORFQuery.obj
 0001:00021a10       __unwindfunclet$??__EscriptLog@U2@@YAXXZ$0 10022a10 f   ORFQuery.obj
 0001:00021a19       __ehhandler$??__EscriptLog@U2@@YAXXZ 10022a19 f   ORFQuery.obj
 0001:00021a40       __unwindfunclet$??__EtaskLog@U2@@YAXXZ$0 10022a40 f   ORFQuery.obj
 0001:00021a49       __ehhandler$??__EtaskLog@U2@@YAXXZ 10022a49 f   ORFQuery.obj
 0001:00021a70       __unwindfunclet$??__EuiLog@U2@@YAXXZ$0 10022a70 f   ORFQuery.obj
 0001:00021a79       __ehhandler$??__EuiLog@U2@@YAXXZ 10022a79 f   ORFQuery.obj
 0001:00021aa0       __unwindfunclet$??__EuserActLog@U2@@YAXXZ$0 10022aa0 f   ORFQuery.obj
 0001:00021aa9       __ehhandler$??__EuserActLog@U2@@YAXXZ 10022aa9 f   ORFQuery.obj
 0001:00021ad0       __ehhandler$?append@?$QList@PAVAttribute@U2@@@@QAEXABQAVAttribute@U2@@@Z 10022ad0 f   ORFQuery.obj
 0001:00021af0       __ehhandler$?append@?$QList@PAVORFFindTask@U2@@@@QAEXABQAVORFFindTask@U2@@@Z 10022af0 f   ORFQuery.obj
 0001:00021b10       __unwindfunclet$?clone@?$QSharedDataPointer@VQDResultUnitData@U2@@@@IAEPAVQDResultUnitData@U2@@XZ$0 10022b10 f   ORFQuery.obj
 0001:00021b1b       __ehhandler$?clone@?$QSharedDataPointer@VQDResultUnitData@U2@@@@IAEPAVQDResultUnitData@U2@@XZ 10022b1b f   ORFQuery.obj
 0001:00021b40       __unwindfunclet$?copyConstruct@?$QVector@VU2Qualifier@U2@@@@AAEXPBVU2Qualifier@U2@@0PAV23@@Z$0 10022b40 f   ORFQuery.obj
 0001:00021b51       __ehhandler$?copyConstruct@?$QVector@VU2Qualifier@U2@@@@AAEXPBVU2Qualifier@U2@@0PAV23@@Z 10022b51 f   ORFQuery.obj
 0001:00021b70       __unwindfunclet$?createInstance@QDORFActorPrototype@U2@@UBEPAVQDActor@2@XZ$0 10022b70 f   ORFQuery.obj
 0001:00021b7b       __ehhandler$?createInstance@QDORFActorPrototype@U2@@UBEPAVQDActor@2@XZ 10022b7b f   ORFQuery.obj
 0001:00021ba0       __unwindfunclet$?createNode@?$QMapData@VQString@@PAVPropertyDelegate@U2@@@@QAEPAU?$QMapNode@VQString@@PAVPropertyDelegate@U2@@@@ABVQString@@ABQAVPropertyDelegate@U2@@PAU2@_N@Z$4 10022ba0 f   ORFQuery.obj
 0001:00021bb4       __ehhandler$?createNode@?$QMapData@VQString@@PAVPropertyDelegate@U2@@@@QAEPAU?$QMapNode@VQString@@PAVPropertyDelegate@U2@@@@ABVQString@@ABQAVPropertyDelegate@U2@@PAU2@_N@Z 10022bb4 f   ORFQuery.obj
 0001:00021bd0       __unwindfunclet$?createNode@?$QMapData@VQString@@PAVQDSchemeUnit@U2@@@@QAEPAU?$QMapNode@VQString@@PAVQDSchemeUnit@U2@@@@ABVQString@@ABQAVQDSchemeUnit@U2@@PAU2@_N@Z$4 10022bd0 f   ORFQuery.obj
 0001:00021be4       __ehhandler$?createNode@?$QMapData@VQString@@PAVQDSchemeUnit@U2@@@@QAEPAU?$QMapNode@VQString@@PAVQDSchemeUnit@U2@@@@ABVQString@@ABQAVQDSchemeUnit@U2@@PAU2@_N@Z 10022be4 f   ORFQuery.obj
 0001:00021c00       __unwindfunclet$?createNode@?$QMapData@VQString@@VQVariant@@@@QAEPAU?$QMapNode@VQString@@VQVariant@@@@ABVQString@@ABVQVariant@@PAU2@_N@Z$4 10022c00 f   ORFQuery.obj
 0001:00021c14       __unwindfunclet$?createNode@?$QMapData@VQString@@VQVariant@@@@QAEPAU?$QMapNode@VQString@@VQVariant@@@@ABVQString@@ABVQVariant@@PAU2@_N@Z$5 10022c14 f   ORFQuery.obj
 0001:00021c28       __ehhandler$?createNode@?$QMapData@VQString@@VQVariant@@@@QAEPAU?$QMapNode@VQString@@VQVariant@@@@ABVQString@@ABVQVariant@@PAU2@_N@Z 10022c28 f   ORFQuery.obj
 0001:00021c50       __unwindfunclet$?detach_helper@?$QSharedDataPointer@VQDResultUnitData@U2@@@@AAEXXZ$0 10022c50 f   ORFQuery.obj
 0001:00021c5b       __ehhandler$?detach_helper@?$QSharedDataPointer@VQDResultUnitData@U2@@@@AAEXXZ 10022c5b f   ORFQuery.obj
 0001:00021c80       __ehhandler$?detach_helper_grow@?$QList@PAVAttribute@U2@@@@AAEPAUNode@1@HH@Z 10022c80 f   ORFQuery.obj
 0001:00021ca0       __ehhandler$?detach_helper_grow@?$QList@PAVORFFindTask@U2@@@@AAEPAUNode@1@HH@Z 10022ca0 f   ORFQuery.obj
 0001:00021cc0       __ehhandler$?detach_helper_grow@?$QList@VORFFindResult@U2@@@@AAEPAUNode@1@HH@Z 10022cc0 f   ORFQuery.obj
 0001:00021ce0       __unwindfunclet$?getAlgorithmTask@QDORFActor@U2@@UAEPAVTask@2@ABV?$QVector@VU2Region@U2@@@@@Z$0 10022ce0 f   ORFQuery.obj
 0001:00021ce8       __unwindfunclet$?getAlgorithmTask@QDORFActor@U2@@UAEPAVTask@2@ABV?$QVector@VU2Region@U2@@@@@Z$1 10022ce8 f   ORFQuery.obj
 0001:00021cf1       __unwindfunclet$?getAlgorithmTask@QDORFActor@U2@@UAEPAVTask@2@ABV?$QVector@VU2Region@U2@@@@@Z$2 10022cf1 f   ORFQuery.obj
 0001:00021cfc       __unwindfunclet$?getAlgorithmTask@QDORFActor@U2@@UAEPAVTask@2@ABV?$QVector@VU2Region@U2@@@@@Z$3 10022cfc f   ORFQuery.obj
 0001:00021d16       __unwindfunclet$?getAlgorithmTask@QDORFActor@U2@@UAEPAVTask@2@ABV?$QVector@VU2Region@U2@@@@@Z$4 10022d16 f   ORFQuery.obj
 0001:00021d21       __unwindfunclet$?getAlgorithmTask@QDORFActor@U2@@UAEPAVTask@2@ABV?$QVector@VU2Region@U2@@@@@Z$5 10022d21 f   ORFQuery.obj
 0001:00021d3b       __unwindfunclet$?getAlgorithmTask@QDORFActor@U2@@UAEPAVTask@2@ABV?$QVector@VU2Region@U2@@@@@Z$11 10022d3b f   ORFQuery.obj
 0001:00021d43       __unwindfunclet$?getAlgorithmTask@QDORFActor@U2@@UAEPAVTask@2@ABV?$QVector@VU2Region@U2@@@@@Z$6 10022d43 f   ORFQuery.obj
 0001:00021d4b       __unwindfunclet$?getAlgorithmTask@QDORFActor@U2@@UAEPAVTask@2@ABV?$QVector@VU2Region@U2@@@@@Z$7 10022d4b f   ORFQuery.obj
 0001:00021d56       __unwindfunclet$?getAlgorithmTask@QDORFActor@U2@@UAEPAVTask@2@ABV?$QVector@VU2Region@U2@@@@@Z$8 10022d56 f   ORFQuery.obj
 0001:00021d70       __unwindfunclet$?getAlgorithmTask@QDORFActor@U2@@UAEPAVTask@2@ABV?$QVector@VU2Region@U2@@@@@Z$9 10022d70 f   ORFQuery.obj
 0001:00021d7b       __ehhandler$?getAlgorithmTask@QDORFActor@U2@@UAEPAVTask@2@ABV?$QVector@VU2Region@U2@@@@@Z 10022d7b f   ORFQuery.obj
 0001:00021da0       __unwindfunclet$?getIcon@QDORFActorPrototype@U2@@UBE?AVQIcon@@XZ$0 10022da0 f   ORFQuery.obj
 0001:00021da9       __unwindfunclet$?getIcon@QDORFActorPrototype@U2@@UBE?AVQIcon@@XZ$1 10022da9 f   ORFQuery.obj
 0001:00021dc3       __ehhandler$?getIcon@QDORFActorPrototype@U2@@UBE?AVQIcon@@XZ 10022dc3 f   ORFQuery.obj
 0001:00021de0       __unwindfunclet$?getText@QDORFActor@U2@@UBE?AVQString@@XZ$0 10022de0 f   ORFQuery.obj
 0001:00021de8       __unwindfunclet$?getText@QDORFActor@U2@@UBE?AVQString@@XZ$1 10022de8 f   ORFQuery.obj
 0001:00021df1       __unwindfunclet$?getText@QDORFActor@U2@@UBE?AVQString@@XZ$2 10022df1 f   ORFQuery.obj
 0001:00021dfa       __unwindfunclet$?getText@QDORFActor@U2@@UBE?AVQString@@XZ$4 10022dfa f   ORFQuery.obj
 0001:00021e03       __unwindfunclet$?getText@QDORFActor@U2@@UBE?AVQString@@XZ$3 10022e03 f   ORFQuery.obj
 0001:00021e0c       __unwindfunclet$?getText@QDORFActor@U2@@UBE?AVQString@@XZ$5 10022e0c f   ORFQuery.obj
 0001:00021e14       __unwindfunclet$?getText@QDORFActor@U2@@UBE?AVQString@@XZ$6 10022e14 f   ORFQuery.obj
 0001:00021e1d       __unwindfunclet$?getText@QDORFActor@U2@@UBE?AVQString@@XZ$7 10022e1d f   ORFQuery.obj
 0001:00021e26       __unwindfunclet$?getText@QDORFActor@U2@@UBE?AVQString@@XZ$8 10022e26 f   ORFQuery.obj
 0001:00021e2f       __unwindfunclet$?getText@QDORFActor@U2@@UBE?AVQString@@XZ$9 10022e2f f   ORFQuery.obj
 0001:00021e38       __unwindfunclet$?getText@QDORFActor@U2@@UBE?AVQString@@XZ$10 10022e38 f   ORFQuery.obj
 0001:00021e41       __unwindfunclet$?getText@QDORFActor@U2@@UBE?AVQString@@XZ$11 10022e41 f   ORFQuery.obj
 0001:00021e4a       __unwindfunclet$?getText@QDORFActor@U2@@UBE?AVQString@@XZ$12 10022e4a f   ORFQuery.obj
 0001:00021e53       __unwindfunclet$?getText@QDORFActor@U2@@UBE?AVQString@@XZ$13 10022e53 f   ORFQuery.obj
 0001:00021e5c       __unwindfunclet$?getText@QDORFActor@U2@@UBE?AVQString@@XZ$14 10022e5c f   ORFQuery.obj
 0001:00021e65       __unwindfunclet$?getText@QDORFActor@U2@@UBE?AVQString@@XZ$15 10022e65 f   ORFQuery.obj
 0001:00021e6e       __unwindfunclet$?getText@QDORFActor@U2@@UBE?AVQString@@XZ$16 10022e6e f   ORFQuery.obj
 0001:00021e77       __unwindfunclet$?getText@QDORFActor@U2@@UBE?AVQString@@XZ$17 10022e77 f   ORFQuery.obj
 0001:00021e80       __unwindfunclet$?getText@QDORFActor@U2@@UBE?AVQString@@XZ$18 10022e80 f   ORFQuery.obj
 0001:00021e89       __unwindfunclet$?getText@QDORFActor@U2@@UBE?AVQString@@XZ$19 10022e89 f   ORFQuery.obj
 0001:00021e92       __unwindfunclet$?getText@QDORFActor@U2@@UBE?AVQString@@XZ$20 10022e92 f   ORFQuery.obj
 0001:00021e9b       __unwindfunclet$?getText@QDORFActor@U2@@UBE?AVQString@@XZ$21 10022e9b f   ORFQuery.obj
 0001:00021ea4       __unwindfunclet$?getText@QDORFActor@U2@@UBE?AVQString@@XZ$22 10022ea4 f   ORFQuery.obj
 0001:00021ead       __unwindfunclet$?getText@QDORFActor@U2@@UBE?AVQString@@XZ$23 10022ead f   ORFQuery.obj
 0001:00021eb6       __unwindfunclet$?getText@QDORFActor@U2@@UBE?AVQString@@XZ$24 10022eb6 f   ORFQuery.obj
 0001:00021ebf       __unwindfunclet$?getText@QDORFActor@U2@@UBE?AVQString@@XZ$25 10022ebf f   ORFQuery.obj
 0001:00021ec8       __unwindfunclet$?getText@QDORFActor@U2@@UBE?AVQString@@XZ$26 10022ec8 f   ORFQuery.obj
 0001:00021ed1       __unwindfunclet$?getText@QDORFActor@U2@@UBE?AVQString@@XZ$27 10022ed1 f   ORFQuery.obj
 0001:00021eeb       __ehhandler$?getText@QDORFActor@U2@@UBE?AVQString@@XZ 10022eeb f   ORFQuery.obj
 0001:00021f10       __unwindfunclet$?metaType@?$QVariantValueHelper@VQString@@@QtPrivate@@SA?AVQString@@ABVQVariant@@@Z$0 10022f10 f   ORFQuery.obj
 0001:00021f2a       __unwindfunclet$?metaType@?$QVariantValueHelper@VQString@@@QtPrivate@@SA?AVQString@@ABVQVariant@@@Z$1 10022f2a f   ORFQuery.obj
 0001:00021f33       __ehhandler$?metaType@?$QVariantValueHelper@VQString@@@QtPrivate@@SA?AVQString@@ABVQVariant@@@Z 10022f33 f   ORFQuery.obj
 0001:00021f50       __unwindfunclet$?sl_onAlgorithmTaskFinished@QDORFActor@U2@@AAEXPAVTask@2@@Z$0 10022f50 f   ORFQuery.obj
 0001:00021f58       __unwindfunclet$?sl_onAlgorithmTaskFinished@QDORFActor@U2@@AAEXPAVTask@2@@Z$1 10022f58 f   ORFQuery.obj
 0001:00021f60       __unwindfunclet$?sl_onAlgorithmTaskFinished@QDORFActor@U2@@AAEXPAVTask@2@@Z$2 10022f60 f   ORFQuery.obj
 0001:00021f68       __unwindfunclet$?sl_onAlgorithmTaskFinished@QDORFActor@U2@@AAEXPAVTask@2@@Z$3 10022f68 f   ORFQuery.obj
 0001:00021f71       __unwindfunclet$?sl_onAlgorithmTaskFinished@QDORFActor@U2@@AAEXPAVTask@2@@Z$4 10022f71 f   ORFQuery.obj
 0001:00021f79       __unwindfunclet$?sl_onAlgorithmTaskFinished@QDORFActor@U2@@AAEXPAVTask@2@@Z$5 10022f79 f   ORFQuery.obj
 0001:00021f81       __unwindfunclet$?sl_onAlgorithmTaskFinished@QDORFActor@U2@@AAEXPAVTask@2@@Z$6 10022f81 f   ORFQuery.obj
 0001:00021f8c       __unwindfunclet$?sl_onAlgorithmTaskFinished@QDORFActor@U2@@AAEXPAVTask@2@@Z$7 10022f8c f   ORFQuery.obj
 0001:00021f94       __unwindfunclet$?sl_onAlgorithmTaskFinished@QDORFActor@U2@@AAEXPAVTask@2@@Z$12 10022f94 f   ORFQuery.obj
 0001:00021f9f       __unwindfunclet$?sl_onAlgorithmTaskFinished@QDORFActor@U2@@AAEXPAVTask@2@@Z$13 10022f9f f   ORFQuery.obj
 0001:00021faa       __unwindfunclet$?sl_onAlgorithmTaskFinished@QDORFActor@U2@@AAEXPAVTask@2@@Z$15 10022faa f   ORFQuery.obj
 0001:00021fb5       __unwindfunclet$?sl_onAlgorithmTaskFinished@QDORFActor@U2@@AAEXPAVTask@2@@Z$8 10022fb5 f   ORFQuery.obj
 0001:00021fbe       __unwindfunclet$?sl_onAlgorithmTaskFinished@QDORFActor@U2@@AAEXPAVTask@2@@Z$16 10022fbe f   ORFQuery.obj
 0001:00021fc9       __ehhandler$?sl_onAlgorithmTaskFinished@QDORFActor@U2@@AAEXPAVTask@2@@Z 10022fc9 f   ORFQuery.obj
 0001:00021ff0       __unwindfunclet$??$?0VQString@@V0@@?$QPair@VQString@@VQVariant@@@@QAE@$$QAU?$QPair@VQString@@V1@@@@Z$0 10022ff0 f   ORFWorker.obj
 0001:00021ff9       __ehhandler$??$?0VQString@@V0@@?$QPair@VQString@@VQVariant@@@@QAE@$$QAU?$QPair@VQString@@V1@@@@Z 10022ff9 f   ORFWorker.obj
 0001:00022020       __unwindfunclet$??$getAttributeValue@H@Attribute@U2@@QBEHPAVWorkflowContext@Workflow@1@@Z$0 10023020 f   ORFWorker.obj
 0001:00022029       __unwindfunclet$??$getAttributeValue@H@Attribute@U2@@QBEHPAVWorkflowContext@Workflow@1@@Z$1 10023029 f   ORFWorker.obj
 0001:00022031       __unwindfunclet$??$getAttributeValue@H@Attribute@U2@@QBEHPAVWorkflowContext@Workflow@1@@Z$2 10023031 f   ORFWorker.obj
 0001:00022039       __unwindfunclet$??$getAttributeValue@H@Attribute@U2@@QBEHPAVWorkflowContext@Workflow@1@@Z$3 10023039 f   ORFWorker.obj
 0001:00022041       __unwindfunclet$??$getAttributeValue@H@Attribute@U2@@QBEHPAVWorkflowContext@Workflow@1@@Z$4 10023041 f   ORFWorker.obj
 0001:0002204a       __unwindfunclet$??$getAttributeValue@H@Attribute@U2@@QBEHPAVWorkflowContext@Workflow@1@@Z$5 1002304a f   ORFWorker.obj
 0001:00022053       __unwindfunclet$??$getAttributeValue@H@Attribute@U2@@QBEHPAVWorkflowContext@Workflow@1@@Z$6 10023053 f   ORFWorker.obj
 0001:0002205c       __unwindfunclet$??$getAttributeValue@H@Attribute@U2@@QBEHPAVWorkflowContext@Workflow@1@@Z$7 1002305c f   ORFWorker.obj
 0001:00022065       __unwindfunclet$??$getAttributeValue@H@Attribute@U2@@QBEHPAVWorkflowContext@Workflow@1@@Z$8 10023065 f   ORFWorker.obj
 0001:0002206e       __unwindfunclet$??$getAttributeValue@H@Attribute@U2@@QBEHPAVWorkflowContext@Workflow@1@@Z$9 1002306e f   ORFWorker.obj
 0001:00022077       __unwindfunclet$??$getAttributeValue@H@Attribute@U2@@QBEHPAVWorkflowContext@Workflow@1@@Z$10 10023077 f   ORFWorker.obj
 0001:00022080       __unwindfunclet$??$getAttributeValue@H@Attribute@U2@@QBEHPAVWorkflowContext@Workflow@1@@Z$11 10023080 f   ORFWorker.obj
 0001:00022089       __ehhandler$??$getAttributeValue@H@Attribute@U2@@QBEHPAVWorkflowContext@Workflow@1@@Z 10023089 f   ORFWorker.obj
 0001:000220b0       __unwindfunclet$??$getAttributeValue@VQString@@@Attribute@U2@@QBE?AVQString@@PAVWorkflowContext@Workflow@1@@Z$0 100230b0 f   ORFWorker.obj
 0001:000220ca       __unwindfunclet$??$getAttributeValue@VQString@@@Attribute@U2@@QBE?AVQString@@PAVWorkflowContext@Workflow@1@@Z$1 100230ca f   ORFWorker.obj
 0001:000220d3       __unwindfunclet$??$getAttributeValue@VQString@@@Attribute@U2@@QBE?AVQString@@PAVWorkflowContext@Workflow@1@@Z$2 100230d3 f   ORFWorker.obj
 0001:000220db       __unwindfunclet$??$getAttributeValue@VQString@@@Attribute@U2@@QBE?AVQString@@PAVWorkflowContext@Workflow@1@@Z$3 100230db f   ORFWorker.obj
 0001:000220e3       __unwindfunclet$??$getAttributeValue@VQString@@@Attribute@U2@@QBE?AVQString@@PAVWorkflowContext@Workflow@1@@Z$4 100230e3 f   ORFWorker.obj
 0001:000220eb       __unwindfunclet$??$getAttributeValue@VQString@@@Attribute@U2@@QBE?AVQString@@PAVWorkflowContext@Workflow@1@@Z$5 100230eb f   ORFWorker.obj
 0001:000220f4       __unwindfunclet$??$getAttributeValue@VQString@@@Attribute@U2@@QBE?AVQString@@PAVWorkflowContext@Workflow@1@@Z$6 100230f4 f   ORFWorker.obj
 0001:000220fd       __unwindfunclet$??$getAttributeValue@VQString@@@Attribute@U2@@QBE?AVQString@@PAVWorkflowContext@Workflow@1@@Z$7 100230fd f   ORFWorker.obj
 0001:00022106       __unwindfunclet$??$getAttributeValue@VQString@@@Attribute@U2@@QBE?AVQString@@PAVWorkflowContext@Workflow@1@@Z$8 10023106 f   ORFWorker.obj
 0001:0002210f       __unwindfunclet$??$getAttributeValue@VQString@@@Attribute@U2@@QBE?AVQString@@PAVWorkflowContext@Workflow@1@@Z$9 1002310f f   ORFWorker.obj
 0001:00022118       __unwindfunclet$??$getAttributeValue@VQString@@@Attribute@U2@@QBE?AVQString@@PAVWorkflowContext@Workflow@1@@Z$10 10023118 f   ORFWorker.obj
 0001:00022121       __unwindfunclet$??$getAttributeValue@VQString@@@Attribute@U2@@QBE?AVQString@@PAVWorkflowContext@Workflow@1@@Z$11 10023121 f   ORFWorker.obj
 0001:0002212a       __unwindfunclet$??$getAttributeValue@VQString@@@Attribute@U2@@QBE?AVQString@@PAVWorkflowContext@Workflow@1@@Z$12 1002312a f   ORFWorker.obj
 0001:00022133       __ehhandler$??$getAttributeValue@VQString@@@Attribute@U2@@QBE?AVQString@@PAVWorkflowContext@Workflow@1@@Z 10023133 f   ORFWorker.obj
 0001:00022160       __unwindfunclet$??$qMakePair@VQString@@V1@@@YA?AU?$QPair@VQString@@V1@@@ABVQString@@0@Z$1 10023160 f   ORFWorker.obj
 0001:00022169       __ehhandler$??$qMakePair@VQString@@V1@@@YA?AU?$QPair@VQString@@V1@@@ABVQString@@0@Z 10023169 f   ORFWorker.obj
 0001:00022190       __unwindfunclet$??$qRegisterMetaType@V?$QSharedDataPointer@VDbiDataHandler@Workflow@U2@@@@@@YAHPBDPAV?$QSharedDataPointer@VDbiDataHandler@Workflow@U2@@@@W4DefinedType@?$MetaTypeDefinedHelper@V?$QSharedDataPointer@VDbiDataHandler@Workflow@U2@@@@$00@QtPrivate@@@Z$0 10023190 f   ORFWorker.obj
 0001:00022199       __ehhandler$??$qRegisterMetaType@V?$QSharedDataPointer@VDbiDataHandler@Workflow@U2@@@@@@YAHPBDPAV?$QSharedDataPointer@VDbiDataHandler@Workflow@U2@@@@W4DefinedType@?$MetaTypeDefinedHelper@V?$QSharedDataPointer@VDbiDataHandler@Workflow@U2@@@@$00@QtPrivate@@@Z 10023199 f   ORFWorker.obj
 0001:000221c0       __ehhandler$??0?$QList@PAVPort@Workflow@U2@@@@QAE@ABV0@@Z 100231c0 f   ORFWorker.obj
 0001:000221e0       __ehhandler$??0?$QList@VDescriptor@U2@@@@QAE@ABV0@@Z 100231e0 f   ORFWorker.obj
 0001:00022200       __unwindfunclet$??0?$QPair@VQString@@V1@@@QAE@ABVQString@@0@Z$0 10023200 f   ORFWorker.obj
 0001:00022209       __ehhandler$??0?$QPair@VQString@@V1@@@QAE@ABVQString@@0@Z 10023209 f   ORFWorker.obj
 0001:00022230       __unwindfunclet$??0?$QPair@VQString@@VQVariant@@@@QAE@ABU0@@Z$0 10023230 f   ORFWorker.obj
 0001:00022239       __ehhandler$??0?$QPair@VQString@@VQVariant@@@@QAE@ABU0@@Z 10023239 f   ORFWorker.obj
 0001:00022260       __unwindfunclet$??0ORFWorker@LocalWorkflow@U2@@QAE@PAVActor@Workflow@2@@Z$0 10023260 f   ORFWorker.obj
 0001:00022269       __unwindfunclet$??0ORFWorker@LocalWorkflow@U2@@QAE@PAVActor@Workflow@2@@Z$1 10023269 f   ORFWorker.obj
 0001:00022275       __ehhandler$??0ORFWorker@LocalWorkflow@U2@@QAE@PAVActor@Workflow@2@@Z 10023275 f   ORFWorker.obj
 0001:00022290       __unwindfunclet$??1?$QPair@VQString@@V1@@@QAE@XZ$0 10023290 f   ORFWorker.obj
 0001:00022299       __ehhandler$??1?$QPair@VQString@@V1@@@QAE@XZ 10023299 f   ORFWorker.obj
 0001:000222c0       __unwindfunclet$??1?$QPair@VQString@@VQVariant@@@@QAE@XZ$0 100232c0 f   ORFWorker.obj
 0001:000222c9       __ehhandler$??1?$QPair@VQString@@VQVariant@@@@QAE@XZ 100232c9 f   ORFWorker.obj
 0001:000222f0       __unwindfunclet$??1ORFWorker@LocalWorkflow@U2@@UAE@XZ$0 100232f0 f   ORFWorker.obj
 0001:000222f9       __unwindfunclet$??1ORFWorker@LocalWorkflow@U2@@UAE@XZ$1 100232f9 f   ORFWorker.obj
 0001:00022305       __ehhandler$??1ORFWorker@LocalWorkflow@U2@@UAE@XZ 10023305 f   ORFWorker.obj
 0001:00022320       __unwindfunclet$??A?$QMap@VDescriptor@U2@@V?$QExplicitlySharedDataPointer@VDataType@U2@@@@@@QAEAAV?$QExplicitlySharedDataPointer@VDataType@U2@@@@ABVDescriptor@U2@@@Z$0 10023320 f   ORFWorker.obj
 0001:00022328       __ehhandler$??A?$QMap@VDescriptor@U2@@V?$QExplicitlySharedDataPointer@VDataType@U2@@@@@@QAEAAV?$QExplicitlySharedDataPointer@VDataType@U2@@@@ABVDescriptor@U2@@@Z 10023328 f   ORFWorker.obj
 0001:00022350       __unwindfunclet$??A?$QMap@VQString@@VQScriptValue@@@@QAEAAVQScriptValue@@ABVQString@@@Z$0 10023350 f   ORFWorker.obj
 0001:00022359       __ehhandler$??A?$QMap@VQString@@VQScriptValue@@@@QAEAAVQScriptValue@@ABVQString@@@Z 10023359 f   ORFWorker.obj
 0001:00022380       __unwindfunclet$??_G?$QPair@VQString@@VQVariant@@@@QAEPAXI@Z$0 10023380 f   ORFWorker.obj
 0001:00022389       __ehhandler$??_G?$QPair@VQString@@VQVariant@@@@QAEPAXI@Z 10023389 f   ORFWorker.obj
 0001:000223b0       __unwindfunclet$??_GORFWorker@LocalWorkflow@U2@@UAEPAXI@Z$0 100233b0 f   ORFWorker.obj
 0001:000223b9       __unwindfunclet$??_GORFWorker@LocalWorkflow@U2@@UAEPAXI@Z$1 100233b9 f   ORFWorker.obj
 0001:000223c5       __ehhandler$??_GORFWorker@LocalWorkflow@U2@@UAEPAXI@Z 100233c5 f   ORFWorker.obj
 0001:000223e0       __unwindfunclet$??__EalgoLog@U2@@YAXXZ$0 100233e0 f   ORFWorker.obj
 0001:000223e9       __ehhandler$??__EalgoLog@U2@@YAXXZ 100233e9 f   ORFWorker.obj
 0001:00022410       __unwindfunclet$??__EcmdLog@U2@@YAXXZ$0 10023410 f   ORFWorker.obj
 0001:00022419       __ehhandler$??__EcmdLog@U2@@YAXXZ 10023419 f   ORFWorker.obj
 0001:00022440       __unwindfunclet$??__EcoreLog@U2@@YAXXZ$0 10023440 f   ORFWorker.obj
 0001:00022449       __ehhandler$??__EcoreLog@U2@@YAXXZ 10023449 f   ORFWorker.obj
 0001:00022470       __unwindfunclet$??__EioLog@U2@@YAXXZ$0 10023470 f   ORFWorker.obj
 0001:00022479       __ehhandler$??__EioLog@U2@@YAXXZ 10023479 f   ORFWorker.obj
 0001:000224a0       __unwindfunclet$??__EperfLog@U2@@YAXXZ$0 100234a0 f   ORFWorker.obj
 0001:000224a9       __ehhandler$??__EperfLog@U2@@YAXXZ 100234a9 f   ORFWorker.obj
 0001:000224d0       __unwindfunclet$??__EscriptLog@U2@@YAXXZ$0 100234d0 f   ORFWorker.obj
 0001:000224d9       __ehhandler$??__EscriptLog@U2@@YAXXZ 100234d9 f   ORFWorker.obj
 0001:00022500       __unwindfunclet$??__EtaskLog@U2@@YAXXZ$0 10023500 f   ORFWorker.obj
 0001:00022509       __ehhandler$??__EtaskLog@U2@@YAXXZ 10023509 f   ORFWorker.obj
 0001:00022530       __unwindfunclet$??__EuiLog@U2@@YAXXZ$0 10023530 f   ORFWorker.obj
 0001:00022539       __ehhandler$??__EuiLog@U2@@YAXXZ 10023539 f   ORFWorker.obj
 0001:00022560       __unwindfunclet$??__EuserActLog@U2@@YAXXZ$0 10023560 f   ORFWorker.obj
 0001:00022569       __ehhandler$??__EuserActLog@U2@@YAXXZ 10023569 f   ORFWorker.obj
 0001:00022590       __ehhandler$?append@?$QList@PAVPortDescriptor@Workflow@U2@@@@QAEXABQAVPortDescriptor@Workflow@U2@@@Z 10023590 f   ORFWorker.obj
 0001:000225b0       __ehhandler$?append@?$QList@U?$QPair@VQString@@VQVariant@@@@@@QAEXABU?$QPair@VQString@@VQVariant@@@@@Z 100235b0 f   ORFWorker.obj
 0001:000225d0       __unwindfunclet$?append@?$QList@VDescriptor@U2@@@@QAEXABVDescriptor@U2@@@Z$6 100235d0 f   ORFWorker.obj
 0001:000225db       __ehhandler$?append@?$QList@VDescriptor@U2@@@@QAEXABVDescriptor@U2@@@Z 100235db f   ORFWorker.obj
 0001:00022600       __unwindfunclet$?composeRichDoc@ORFPrompter@LocalWorkflow@U2@@MAE?AVQString@@XZ$0 10023600 f   ORFWorker.obj
 0001:00022609       __unwindfunclet$?composeRichDoc@ORFPrompter@LocalWorkflow@U2@@MAE?AVQString@@XZ$1 10023609 f   ORFWorker.obj
 0001:00022615       __unwindfunclet$?composeRichDoc@ORFPrompter@LocalWorkflow@U2@@MAE?AVQString@@XZ$2 10023615 f   ORFWorker.obj
 0001:0002261e       __unwindfunclet$?composeRichDoc@ORFPrompter@LocalWorkflow@U2@@MAE?AVQString@@XZ$3 1002361e f   ORFWorker.obj
 0001:00022627       __unwindfunclet$?composeRichDoc@ORFPrompter@LocalWorkflow@U2@@MAE?AVQString@@XZ$4 10023627 f   ORFWorker.obj
 0001:00022630       __unwindfunclet$?composeRichDoc@ORFPrompter@LocalWorkflow@U2@@MAE?AVQString@@XZ$5 10023630 f   ORFWorker.obj
 0001:00022639       __unwindfunclet$?composeRichDoc@ORFPrompter@LocalWorkflow@U2@@MAE?AVQString@@XZ$6 10023639 f   ORFWorker.obj
 0001:00022653       __unwindfunclet$?composeRichDoc@ORFPrompter@LocalWorkflow@U2@@MAE?AVQString@@XZ$7 10023653 f   ORFWorker.obj
 0001:0002266d       __unwindfunclet$?composeRichDoc@ORFPrompter@LocalWorkflow@U2@@MAE?AVQString@@XZ$8 1002366d f   ORFWorker.obj
 0001:00022676       __unwindfunclet$?composeRichDoc@ORFPrompter@LocalWorkflow@U2@@MAE?AVQString@@XZ$9 10023676 f   ORFWorker.obj
 0001:0002267f       __unwindfunclet$?composeRichDoc@ORFPrompter@LocalWorkflow@U2@@MAE?AVQString@@XZ$10 1002367f f   ORFWorker.obj
 0001:00022688       __unwindfunclet$?composeRichDoc@ORFPrompter@LocalWorkflow@U2@@MAE?AVQString@@XZ$11 10023688 f   ORFWorker.obj
 0001:00022691       __unwindfunclet$?composeRichDoc@ORFPrompter@LocalWorkflow@U2@@MAE?AVQString@@XZ$12 10023691 f   ORFWorker.obj
 0001:0002269d       __unwindfunclet$?composeRichDoc@ORFPrompter@LocalWorkflow@U2@@MAE?AVQString@@XZ$13 1002369d f   ORFWorker.obj
 0001:000226a6       __unwindfunclet$?composeRichDoc@ORFPrompter@LocalWorkflow@U2@@MAE?AVQString@@XZ$14 100236a6 f   ORFWorker.obj
 0001:000226af       __unwindfunclet$?composeRichDoc@ORFPrompter@LocalWorkflow@U2@@MAE?AVQString@@XZ$15 100236af f   ORFWorker.obj
 0001:000226b8       __unwindfunclet$?composeRichDoc@ORFPrompter@LocalWorkflow@U2@@MAE?AVQString@@XZ$16 100236b8 f   ORFWorker.obj
 0001:000226c1       __unwindfunclet$?composeRichDoc@ORFPrompter@LocalWorkflow@U2@@MAE?AVQString@@XZ$17 100236c1 f   ORFWorker.obj
 0001:000226ca       __unwindfunclet$?composeRichDoc@ORFPrompter@LocalWorkflow@U2@@MAE?AVQString@@XZ$18 100236ca f   ORFWorker.obj
 0001:000226d3       __unwindfunclet$?composeRichDoc@ORFPrompter@LocalWorkflow@U2@@MAE?AVQString@@XZ$19 100236d3 f   ORFWorker.obj
 0001:000226dc       __unwindfunclet$?composeRichDoc@ORFPrompter@LocalWorkflow@U2@@MAE?AVQString@@XZ$20 100236dc f   ORFWorker.obj
 0001:000226e5       __unwindfunclet$?composeRichDoc@ORFPrompter@LocalWorkflow@U2@@MAE?AVQString@@XZ$21 100236e5 f   ORFWorker.obj
 0001:000226ee       __unwindfunclet$?composeRichDoc@ORFPrompter@LocalWorkflow@U2@@MAE?AVQString@@XZ$22 100236ee f   ORFWorker.obj
 0001:000226f7       __unwindfunclet$?composeRichDoc@ORFPrompter@LocalWorkflow@U2@@MAE?AVQString@@XZ$23 100236f7 f   ORFWorker.obj
 0001:00022700       __unwindfunclet$?composeRichDoc@ORFPrompter@LocalWorkflow@U2@@MAE?AVQString@@XZ$24 10023700 f   ORFWorker.obj
 0001:00022709       __unwindfunclet$?composeRichDoc@ORFPrompter@LocalWorkflow@U2@@MAE?AVQString@@XZ$25 10023709 f   ORFWorker.obj
 0001:00022712       __unwindfunclet$?composeRichDoc@ORFPrompter@LocalWorkflow@U2@@MAE?AVQString@@XZ$26 10023712 f   ORFWorker.obj
 0001:0002271b       __unwindfunclet$?composeRichDoc@ORFPrompter@LocalWorkflow@U2@@MAE?AVQString@@XZ$27 1002371b f   ORFWorker.obj
 0001:00022724       __unwindfunclet$?composeRichDoc@ORFPrompter@LocalWorkflow@U2@@MAE?AVQString@@XZ$28 10023724 f   ORFWorker.obj
 0001:0002272d       __unwindfunclet$?composeRichDoc@ORFPrompter@LocalWorkflow@U2@@MAE?AVQString@@XZ$29 1002372d f   ORFWorker.obj
 0001:00022736       __unwindfunclet$?composeRichDoc@ORFPrompter@LocalWorkflow@U2@@MAE?AVQString@@XZ$30 10023736 f   ORFWorker.obj
 0001:0002273f       __unwindfunclet$?composeRichDoc@ORFPrompter@LocalWorkflow@U2@@MAE?AVQString@@XZ$31 1002373f f   ORFWorker.obj
 0001:00022748       __unwindfunclet$?composeRichDoc@ORFPrompter@LocalWorkflow@U2@@MAE?AVQString@@XZ$32 10023748 f   ORFWorker.obj
 0001:00022751       __unwindfunclet$?composeRichDoc@ORFPrompter@LocalWorkflow@U2@@MAE?AVQString@@XZ$35 10023751 f   ORFWorker.obj
 0001:0002275a       __unwindfunclet$?composeRichDoc@ORFPrompter@LocalWorkflow@U2@@MAE?AVQString@@XZ$34 1002375a f   ORFWorker.obj
 0001:00022763       __unwindfunclet$?composeRichDoc@ORFPrompter@LocalWorkflow@U2@@MAE?AVQString@@XZ$33 10023763 f   ORFWorker.obj
 0001:0002276c       __unwindfunclet$?composeRichDoc@ORFPrompter@LocalWorkflow@U2@@MAE?AVQString@@XZ$36 1002376c f   ORFWorker.obj
 0001:00022775       __unwindfunclet$?composeRichDoc@ORFPrompter@LocalWorkflow@U2@@MAE?AVQString@@XZ$37 10023775 f   ORFWorker.obj
 0001:0002277e       __unwindfunclet$?composeRichDoc@ORFPrompter@LocalWorkflow@U2@@MAE?AVQString@@XZ$38 1002377e f   ORFWorker.obj
 0001:00022787       __unwindfunclet$?composeRichDoc@ORFPrompter@LocalWorkflow@U2@@MAE?AVQString@@XZ$39 10023787 f   ORFWorker.obj
 0001:00022790       __unwindfunclet$?composeRichDoc@ORFPrompter@LocalWorkflow@U2@@MAE?AVQString@@XZ$40 10023790 f   ORFWorker.obj
 0001:00022799       __unwindfunclet$?composeRichDoc@ORFPrompter@LocalWorkflow@U2@@MAE?AVQString@@XZ$41 10023799 f   ORFWorker.obj
 0001:000227a2       __unwindfunclet$?composeRichDoc@ORFPrompter@LocalWorkflow@U2@@MAE?AVQString@@XZ$42 100237a2 f   ORFWorker.obj
 0001:000227ab       __unwindfunclet$?composeRichDoc@ORFPrompter@LocalWorkflow@U2@@MAE?AVQString@@XZ$43 100237ab f   ORFWorker.obj
 0001:000227b4       __unwindfunclet$?composeRichDoc@ORFPrompter@LocalWorkflow@U2@@MAE?AVQString@@XZ$44 100237b4 f   ORFWorker.obj
 0001:000227bd       __unwindfunclet$?composeRichDoc@ORFPrompter@LocalWorkflow@U2@@MAE?AVQString@@XZ$45 100237bd f   ORFWorker.obj
 0001:000227c6       __unwindfunclet$?composeRichDoc@ORFPrompter@LocalWorkflow@U2@@MAE?AVQString@@XZ$46 100237c6 f   ORFWorker.obj
 0001:000227cf       __unwindfunclet$?composeRichDoc@ORFPrompter@LocalWorkflow@U2@@MAE?AVQString@@XZ$47 100237cf f   ORFWorker.obj
 0001:000227d8       __unwindfunclet$?composeRichDoc@ORFPrompter@LocalWorkflow@U2@@MAE?AVQString@@XZ$48 100237d8 f   ORFWorker.obj
 0001:000227e4       __unwindfunclet$?composeRichDoc@ORFPrompter@LocalWorkflow@U2@@MAE?AVQString@@XZ$49 100237e4 f   ORFWorker.obj
 0001:000227ed       __unwindfunclet$?composeRichDoc@ORFPrompter@LocalWorkflow@U2@@MAE?AVQString@@XZ$50 100237ed f   ORFWorker.obj
 0001:000227f6       __unwindfunclet$?composeRichDoc@ORFPrompter@LocalWorkflow@U2@@MAE?AVQString@@XZ$51 100237f6 f   ORFWorker.obj
 0001:000227ff       __unwindfunclet$?composeRichDoc@ORFPrompter@LocalWorkflow@U2@@MAE?AVQString@@XZ$52 100237ff f   ORFWorker.obj
 0001:00022808       __unwindfunclet$?composeRichDoc@ORFPrompter@LocalWorkflow@U2@@MAE?AVQString@@XZ$53 10023808 f   ORFWorker.obj
 0001:00022822       __ehhandler$?composeRichDoc@ORFPrompter@LocalWorkflow@U2@@MAE?AVQString@@XZ 10023822 f   ORFWorker.obj
 0001:00022840       __unwindfunclet$?createDescription@?$PrompterBase@VORFPrompter@LocalWorkflow@U2@@@U2@@UAEPAVActorDocument@Workflow@2@PAVActor@42@@Z$0 10023840 f   ORFWorker.obj
 0001:0002284b       __unwindfunclet$?createDescription@?$PrompterBase@VORFPrompter@LocalWorkflow@U2@@@U2@@UAEPAVActorDocument@Workflow@2@PAVActor@42@@Z$3 1002384b f   ORFWorker.obj
 0001:00022853       __unwindfunclet$?createDescription@?$PrompterBase@VORFPrompter@LocalWorkflow@U2@@@U2@@UAEPAVActorDocument@Workflow@2@PAVActor@42@@Z$4 10023853 f   ORFWorker.obj
 0001:0002285b       __unwindfunclet$?createDescription@?$PrompterBase@VORFPrompter@LocalWorkflow@U2@@@U2@@UAEPAVActorDocument@Workflow@2@PAVActor@42@@Z$6 1002385b f   ORFWorker.obj
 0001:00022863       __unwindfunclet$?createDescription@?$PrompterBase@VORFPrompter@LocalWorkflow@U2@@@U2@@UAEPAVActorDocument@Workflow@2@PAVActor@42@@Z$7 10023863 f   ORFWorker.obj
 0001:0002286b       __ehhandler$?createDescription@?$PrompterBase@VORFPrompter@LocalWorkflow@U2@@@U2@@UAEPAVActorDocument@Workflow@2@PAVActor@42@@Z 1002386b f   ORFWorker.obj
 0001:00022890       __unwindfunclet$?createNode@?$QMapData@VDescriptor@U2@@V?$QExplicitlySharedDataPointer@VDataType@U2@@@@@@QAEPAU?$QMapNode@VDescriptor@U2@@V?$QExplicitlySharedDataPointer@VDataType@U2@@@@@@ABVDescriptor@U2@@ABV?$QExplicitlySharedDataPointer@VDataType@U2@@@@PAU2@_N@Z$4 10023890 f   ORFWorker.obj
 0001:000228a4       __ehhandler$?createNode@?$QMapData@VDescriptor@U2@@V?$QExplicitlySharedDataPointer@VDataType@U2@@@@@@QAEPAU?$QMapNode@VDescriptor@U2@@V?$QExplicitlySharedDataPointer@VDataType@U2@@@@@@ABVDescriptor@U2@@ABV?$QExplicitlySharedDataPointer@VDataType@U2@@@@PAU2@_N@Z 100238a4 f   ORFWorker.obj
 0001:000228c0       __unwindfunclet$?createNode@?$QMapData@VQString@@VQScriptValue@@@@QAEPAU?$QMapNode@VQString@@VQScriptValue@@@@ABVQString@@ABVQScriptValue@@PAU2@_N@Z$4 100238c0 f   ORFWorker.obj
 0001:000228d4       __unwindfunclet$?createNode@?$QMapData@VQString@@VQScriptValue@@@@QAEPAU?$QMapNode@VQString@@VQScriptValue@@@@ABVQString@@ABVQScriptValue@@PAU2@_N@Z$5 100238d4 f   ORFWorker.obj
 0001:000228e8       __ehhandler$?createNode@?$QMapData@VQString@@VQScriptValue@@@@QAEPAU?$QMapNode@VQString@@VQScriptValue@@@@ABVQString@@ABVQScriptValue@@PAU2@_N@Z 100238e8 f   ORFWorker.obj
 0001:00022910       __unwindfunclet$?createWorker@ORFWorkerFactory@LocalWorkflow@U2@@UAEPAVWorker@Workflow@3@PAVActor@53@@Z$0 10023910 f   ORFWorker.obj
 0001:0002291b       __ehhandler$?createWorker@ORFWorkerFactory@LocalWorkflow@U2@@UAEPAVWorker@Workflow@3@PAVActor@53@@Z 1002391b f   ORFWorker.obj
 0001:00022940       __ehhandler$?detach_helper@?$QList@VDescriptor@U2@@@@AAEXH@Z 10023940 f   ORFWorker.obj
 0001:00022960       __ehhandler$?detach_helper_grow@?$QList@PAVPortDescriptor@Workflow@U2@@@@AAEPAUNode@1@HH@Z 10023960 f   ORFWorker.obj
 0001:00022980       __ehhandler$?detach_helper_grow@?$QList@U?$QPair@VQString@@VQVariant@@@@@@AAEPAUNode@1@HH@Z 10023980 f   ORFWorker.obj
 0001:000229a0       __ehhandler$?detach_helper_grow@?$QList@VDescriptor@U2@@@@AAEPAUNode@1@HH@Z 100239a0 f   ORFWorker.obj
 0001:000229c0       __unwindfunclet$?getStrand@LocalWorkflow@U2@@YA?AW4ORFAlgorithmStrand@2@ABVQString@@@Z$0 100239c0 f   ORFWorker.obj
 0001:000229c9       __unwindfunclet$?getStrand@LocalWorkflow@U2@@YA?AW4ORFAlgorithmStrand@2@ABVQString@@@Z$1 100239c9 f   ORFWorker.obj
 0001:000229d2       __unwindfunclet$?getStrand@LocalWorkflow@U2@@YA?AW4ORFAlgorithmStrand@2@ABVQString@@@Z$2 100239d2 f   ORFWorker.obj
 0001:000229db       __unwindfunclet$?getStrand@LocalWorkflow@U2@@YA?AW4ORFAlgorithmStrand@2@ABVQString@@@Z$3 100239db f   ORFWorker.obj
 0001:000229e4       __ehhandler$?getStrand@LocalWorkflow@U2@@YA?AW4ORFAlgorithmStrand@2@ABVQString@@@Z 100239e4 f   ORFWorker.obj
 0001:00022a00       __unwindfunclet$?init@ORFWorker@LocalWorkflow@U2@@UAEXXZ$0 10023a00 f   ORFWorker.obj
 0001:00022a09       __unwindfunclet$?init@ORFWorker@LocalWorkflow@U2@@UAEXXZ$1 10023a09 f   ORFWorker.obj
 0001:00022a12       __ehhandler$?init@ORFWorker@LocalWorkflow@U2@@UAEXXZ 10023a12 f   ORFWorker.obj
 0001:00022a30       __unwindfunclet$?init@ORFWorkerFactory@LocalWorkflow@U2@@SAXXZ$0 10023a30 f   ORFWorker.obj
 0001:00022a38       __unwindfunclet$?init@ORFWorkerFactory@LocalWorkflow@U2@@SAXXZ$1 10023a38 f   ORFWorker.obj
 0001:00022a40       __unwindfunclet$?init@ORFWorkerFactory@LocalWorkflow@U2@@SAXXZ$2 10023a40 f   ORFWorker.obj
 0001:00022a49       __unwindfunclet$?init@ORFWorkerFactory@LocalWorkflow@U2@@SAXXZ$3 10023a49 f   ORFWorker.obj
 0001:00022a55       __unwindfunclet$?init@ORFWorkerFactory@LocalWorkflow@U2@@SAXXZ$4 10023a55 f   ORFWorker.obj
 0001:00022a5e       __unwindfunclet$?init@ORFWorkerFactory@LocalWorkflow@U2@@SAXXZ$5 10023a5e f   ORFWorker.obj
 0001:00022a6a       __unwindfunclet$?init@ORFWorkerFactory@LocalWorkflow@U2@@SAXXZ$6 10023a6a f   ORFWorker.obj
 0001:00022a76       __unwindfunclet$?init@ORFWorkerFactory@LocalWorkflow@U2@@SAXXZ$7 10023a76 f   ORFWorker.obj
 0001:00022a82       __unwindfunclet$?init@ORFWorkerFactory@LocalWorkflow@U2@@SAXXZ$8 10023a82 f   ORFWorker.obj
 0001:00022a8e       __unwindfunclet$?init@ORFWorkerFactory@LocalWorkflow@U2@@SAXXZ$9 10023a8e f   ORFWorker.obj
 0001:00022a97       __unwindfunclet$?init@ORFWorkerFactory@LocalWorkflow@U2@@SAXXZ$10 10023a97 f   ORFWorker.obj
 0001:00022a9f       __unwindfunclet$?init@ORFWorkerFactory@LocalWorkflow@U2@@SAXXZ$11 10023a9f f   ORFWorker.obj
 0001:00022aa7       __unwindfunclet$?init@ORFWorkerFactory@LocalWorkflow@U2@@SAXXZ$12 10023aa7 f   ORFWorker.obj
 0001:00022ab3       __unwindfunclet$?init@ORFWorkerFactory@LocalWorkflow@U2@@SAXXZ$13 10023ab3 f   ORFWorker.obj
 0001:00022abe       __unwindfunclet$?init@ORFWorkerFactory@LocalWorkflow@U2@@SAXXZ$14 10023abe f   ORFWorker.obj
 0001:00022ac9       __unwindfunclet$?init@ORFWorkerFactory@LocalWorkflow@U2@@SAXXZ$15 10023ac9 f   ORFWorker.obj
 0001:00022ae3       __unwindfunclet$?init@ORFWorkerFactory@LocalWorkflow@U2@@SAXXZ$17 10023ae3 f   ORFWorker.obj
 0001:00022aeb       __unwindfunclet$?init@ORFWorkerFactory@LocalWorkflow@U2@@SAXXZ$18 10023aeb f   ORFWorker.obj
 0001:00022af3       __unwindfunclet$?init@ORFWorkerFactory@LocalWorkflow@U2@@SAXXZ$19 10023af3 f   ORFWorker.obj
 0001:00022aff       __unwindfunclet$?init@ORFWorkerFactory@LocalWorkflow@U2@@SAXXZ$20 10023aff f   ORFWorker.obj
 0001:00022b0a       __unwindfunclet$?init@ORFWorkerFactory@LocalWorkflow@U2@@SAXXZ$21 10023b0a f   ORFWorker.obj
 0001:00022b15       __unwindfunclet$?init@ORFWorkerFactory@LocalWorkflow@U2@@SAXXZ$22 10023b15 f   ORFWorker.obj
 0001:00022b2f       __unwindfunclet$?init@ORFWorkerFactory@LocalWorkflow@U2@@SAXXZ$24 10023b2f f   ORFWorker.obj
 0001:00022b3b       __unwindfunclet$?init@ORFWorkerFactory@LocalWorkflow@U2@@SAXXZ$25 10023b3b f   ORFWorker.obj
 0001:00022b47       __unwindfunclet$?init@ORFWorkerFactory@LocalWorkflow@U2@@SAXXZ$26 10023b47 f   ORFWorker.obj
 0001:00022b53       __unwindfunclet$?init@ORFWorkerFactory@LocalWorkflow@U2@@SAXXZ$27 10023b53 f   ORFWorker.obj
 0001:00022b5c       __unwindfunclet$?init@ORFWorkerFactory@LocalWorkflow@U2@@SAXXZ$28 10023b5c f   ORFWorker.obj
 0001:00022b68       __unwindfunclet$?init@ORFWorkerFactory@LocalWorkflow@U2@@SAXXZ$29 10023b68 f   ORFWorker.obj
 0001:00022b74       __unwindfunclet$?init@ORFWorkerFactory@LocalWorkflow@U2@@SAXXZ$30 10023b74 f   ORFWorker.obj
 0001:00022b7d       __unwindfunclet$?init@ORFWorkerFactory@LocalWorkflow@U2@@SAXXZ$31 10023b7d f   ORFWorker.obj
 0001:00022b89       __unwindfunclet$?init@ORFWorkerFactory@LocalWorkflow@U2@@SAXXZ$32 10023b89 f   ORFWorker.obj
 0001:00022b95       __unwindfunclet$?init@ORFWorkerFactory@LocalWorkflow@U2@@SAXXZ$33 10023b95 f   ORFWorker.obj
 0001:00022b9e       __unwindfunclet$?init@ORFWorkerFactory@LocalWorkflow@U2@@SAXXZ$34 10023b9e f   ORFWorker.obj
 0001:00022ba7       __unwindfunclet$?init@ORFWorkerFactory@LocalWorkflow@U2@@SAXXZ$35 10023ba7 f   ORFWorker.obj
 0001:00022bb3       __unwindfunclet$?init@ORFWorkerFactory@LocalWorkflow@U2@@SAXXZ$36 10023bb3 f   ORFWorker.obj
 0001:00022bbf       __unwindfunclet$?init@ORFWorkerFactory@LocalWorkflow@U2@@SAXXZ$37 10023bbf f   ORFWorker.obj
 0001:00022bcb       __unwindfunclet$?init@ORFWorkerFactory@LocalWorkflow@U2@@SAXXZ$38 10023bcb f   ORFWorker.obj
 0001:00022bd7       __unwindfunclet$?init@ORFWorkerFactory@LocalWorkflow@U2@@SAXXZ$39 10023bd7 f   ORFWorker.obj
 0001:00022be3       __unwindfunclet$?init@ORFWorkerFactory@LocalWorkflow@U2@@SAXXZ$40 10023be3 f   ORFWorker.obj
 0001:00022bef       __unwindfunclet$?init@ORFWorkerFactory@LocalWorkflow@U2@@SAXXZ$41 10023bef f   ORFWorker.obj
 0001:00022bfb       __unwindfunclet$?init@ORFWorkerFactory@LocalWorkflow@U2@@SAXXZ$42 10023bfb f   ORFWorker.obj
 0001:00022c07       __unwindfunclet$?init@ORFWorkerFactory@LocalWorkflow@U2@@SAXXZ$43 10023c07 f   ORFWorker.obj
 0001:00022c13       __unwindfunclet$?init@ORFWorkerFactory@LocalWorkflow@U2@@SAXXZ$44 10023c13 f   ORFWorker.obj
 0001:00022c1f       __unwindfunclet$?init@ORFWorkerFactory@LocalWorkflow@U2@@SAXXZ$45 10023c1f f   ORFWorker.obj
 0001:00022c2b       __unwindfunclet$?init@ORFWorkerFactory@LocalWorkflow@U2@@SAXXZ$46 10023c2b f   ORFWorker.obj
 0001:00022c37       __unwindfunclet$?init@ORFWorkerFactory@LocalWorkflow@U2@@SAXXZ$47 10023c37 f   ORFWorker.obj
 0001:00022c43       __unwindfunclet$?init@ORFWorkerFactory@LocalWorkflow@U2@@SAXXZ$48 10023c43 f   ORFWorker.obj
 0001:00022c4c       __unwindfunclet$?init@ORFWorkerFactory@LocalWorkflow@U2@@SAXXZ$49 10023c4c f   ORFWorker.obj
 0001:00022c55       __unwindfunclet$?init@ORFWorkerFactory@LocalWorkflow@U2@@SAXXZ$50 10023c55 f   ORFWorker.obj
 0001:00022c5e       __unwindfunclet$?init@ORFWorkerFactory@LocalWorkflow@U2@@SAXXZ$51 10023c5e f   ORFWorker.obj
 0001:00022c69       __unwindfunclet$?init@ORFWorkerFactory@LocalWorkflow@U2@@SAXXZ$52 10023c69 f   ORFWorker.obj
 0001:00022c86       __unwindfunclet$?init@ORFWorkerFactory@LocalWorkflow@U2@@SAXXZ$54 10023c86 f   ORFWorker.obj
 0001:00022c91       __unwindfunclet$?init@ORFWorkerFactory@LocalWorkflow@U2@@SAXXZ$55 10023c91 f   ORFWorker.obj
 0001:00022cae       __unwindfunclet$?init@ORFWorkerFactory@LocalWorkflow@U2@@SAXXZ$57 10023cae f   ORFWorker.obj
 0001:00022cb9       __unwindfunclet$?init@ORFWorkerFactory@LocalWorkflow@U2@@SAXXZ$58 10023cb9 f   ORFWorker.obj
 0001:00022cd6       __unwindfunclet$?init@ORFWorkerFactory@LocalWorkflow@U2@@SAXXZ$60 10023cd6 f   ORFWorker.obj
 0001:00022ce1       __unwindfunclet$?init@ORFWorkerFactory@LocalWorkflow@U2@@SAXXZ$61 10023ce1 f   ORFWorker.obj
 0001:00022cfb       __unwindfunclet$?init@ORFWorkerFactory@LocalWorkflow@U2@@SAXXZ$62 10023cfb f   ORFWorker.obj
 0001:00022d18       __unwindfunclet$?init@ORFWorkerFactory@LocalWorkflow@U2@@SAXXZ$63 10023d18 f   ORFWorker.obj
 0001:00022d20       __unwindfunclet$?init@ORFWorkerFactory@LocalWorkflow@U2@@SAXXZ$64 10023d20 f   ORFWorker.obj
 0001:00022d3f       __unwindfunclet$?init@ORFWorkerFactory@LocalWorkflow@U2@@SAXXZ$65 10023d3f f   ORFWorker.obj
 0001:00022d4a       __unwindfunclet$?init@ORFWorkerFactory@LocalWorkflow@U2@@SAXXZ$66 10023d4a f   ORFWorker.obj
 0001:00022d69       __unwindfunclet$?init@ORFWorkerFactory@LocalWorkflow@U2@@SAXXZ$68 10023d69 f   ORFWorker.obj
 0001:00022d74       __unwindfunclet$?init@ORFWorkerFactory@LocalWorkflow@U2@@SAXXZ$69 10023d74 f   ORFWorker.obj
 0001:00022d93       __unwindfunclet$?init@ORFWorkerFactory@LocalWorkflow@U2@@SAXXZ$71 10023d93 f   ORFWorker.obj
 0001:00022d9e       __unwindfunclet$?init@ORFWorkerFactory@LocalWorkflow@U2@@SAXXZ$72 10023d9e f   ORFWorker.obj
 0001:00022dbd       __unwindfunclet$?init@ORFWorkerFactory@LocalWorkflow@U2@@SAXXZ$74 10023dbd f   ORFWorker.obj
 0001:00022dc8       __unwindfunclet$?init@ORFWorkerFactory@LocalWorkflow@U2@@SAXXZ$75 10023dc8 f   ORFWorker.obj
 0001:00022de7       __unwindfunclet$?init@ORFWorkerFactory@LocalWorkflow@U2@@SAXXZ$77 10023de7 f   ORFWorker.obj
 0001:00022df2       __unwindfunclet$?init@ORFWorkerFactory@LocalWorkflow@U2@@SAXXZ$78 10023df2 f   ORFWorker.obj
 0001:00022e14       __unwindfunclet$?init@ORFWorkerFactory@LocalWorkflow@U2@@SAXXZ$80 10023e14 f   ORFWorker.obj
 0001:00022e1f       __unwindfunclet$?init@ORFWorkerFactory@LocalWorkflow@U2@@SAXXZ$81 10023e1f f   ORFWorker.obj
 0001:00022e3e       __unwindfunclet$?init@ORFWorkerFactory@LocalWorkflow@U2@@SAXXZ$83 10023e3e f   ORFWorker.obj
 0001:00022e47       __unwindfunclet$?init@ORFWorkerFactory@LocalWorkflow@U2@@SAXXZ$84 10023e47 f   ORFWorker.obj
 0001:00022e50       __unwindfunclet$?init@ORFWorkerFactory@LocalWorkflow@U2@@SAXXZ$85 10023e50 f   ORFWorker.obj
 0001:00022e5c       __unwindfunclet$?init@ORFWorkerFactory@LocalWorkflow@U2@@SAXXZ$86 10023e5c f   ORFWorker.obj
 0001:00022e67       __unwindfunclet$?init@ORFWorkerFactory@LocalWorkflow@U2@@SAXXZ$87 10023e67 f   ORFWorker.obj
 0001:00022e6f       __unwindfunclet$?init@ORFWorkerFactory@LocalWorkflow@U2@@SAXXZ$88 10023e6f f   ORFWorker.obj
 0001:00022e77       __unwindfunclet$?init@ORFWorkerFactory@LocalWorkflow@U2@@SAXXZ$89 10023e77 f   ORFWorker.obj
 0001:00022e80       __unwindfunclet$?init@ORFWorkerFactory@LocalWorkflow@U2@@SAXXZ$90 10023e80 f   ORFWorker.obj
 0001:00022e89       __unwindfunclet$?init@ORFWorkerFactory@LocalWorkflow@U2@@SAXXZ$91 10023e89 f   ORFWorker.obj
 0001:00022e92       __unwindfunclet$?init@ORFWorkerFactory@LocalWorkflow@U2@@SAXXZ$92 10023e92 f   ORFWorker.obj
 0001:00022e9b       __unwindfunclet$?init@ORFWorkerFactory@LocalWorkflow@U2@@SAXXZ$93 10023e9b f   ORFWorker.obj
 0001:00022ea4       __unwindfunclet$?init@ORFWorkerFactory@LocalWorkflow@U2@@SAXXZ$94 10023ea4 f   ORFWorker.obj
 0001:00022eb0       __unwindfunclet$?init@ORFWorkerFactory@LocalWorkflow@U2@@SAXXZ$95 10023eb0 f   ORFWorker.obj
 0001:00022eb9       __unwindfunclet$?init@ORFWorkerFactory@LocalWorkflow@U2@@SAXXZ$96 10023eb9 f   ORFWorker.obj
 0001:00022ec4       __unwindfunclet$?init@ORFWorkerFactory@LocalWorkflow@U2@@SAXXZ$97 10023ec4 f   ORFWorker.obj
 0001:00022ecf       __unwindfunclet$?init@ORFWorkerFactory@LocalWorkflow@U2@@SAXXZ$98 10023ecf f   ORFWorker.obj
 0001:00022eed       __unwindfunclet$?init@ORFWorkerFactory@LocalWorkflow@U2@@SAXXZ$99 10023eed f   ORFWorker.obj
 0001:00022ef6       __unwindfunclet$?init@ORFWorkerFactory@LocalWorkflow@U2@@SAXXZ$100 10023ef6 f   ORFWorker.obj
 0001:00022eff       __unwindfunclet$?init@ORFWorkerFactory@LocalWorkflow@U2@@SAXXZ$101 10023eff f   ORFWorker.obj
 0001:00022f07       __unwindfunclet$?init@ORFWorkerFactory@LocalWorkflow@U2@@SAXXZ$102 10023f07 f   ORFWorker.obj
 0001:00022f10       __unwindfunclet$?init@ORFWorkerFactory@LocalWorkflow@U2@@SAXXZ$103 10023f10 f   ORFWorker.obj
 0001:00022f18       __unwindfunclet$?init@ORFWorkerFactory@LocalWorkflow@U2@@SAXXZ$104 10023f18 f   ORFWorker.obj
 0001:00022f20       __unwindfunclet$?init@ORFWorkerFactory@LocalWorkflow@U2@@SAXXZ$105 10023f20 f   ORFWorker.obj
 0001:00022f28       __unwindfunclet$?init@ORFWorkerFactory@LocalWorkflow@U2@@SAXXZ$115 10023f28 f   ORFWorker.obj
 0001:00022f31       __unwindfunclet$?init@ORFWorkerFactory@LocalWorkflow@U2@@SAXXZ$106 10023f31 f   ORFWorker.obj
 0001:00022f39       __unwindfunclet$?init@ORFWorkerFactory@LocalWorkflow@U2@@SAXXZ$117 10023f39 f   ORFWorker.obj
 0001:00022f42       __unwindfunclet$?init@ORFWorkerFactory@LocalWorkflow@U2@@SAXXZ$119 10023f42 f   ORFWorker.obj
 0001:00022f4b       __unwindfunclet$?init@ORFWorkerFactory@LocalWorkflow@U2@@SAXXZ$107 10023f4b f   ORFWorker.obj
 0001:00022f56       __unwindfunclet$?init@ORFWorkerFactory@LocalWorkflow@U2@@SAXXZ$108 10023f56 f   ORFWorker.obj
 0001:00022f61       __unwindfunclet$?init@ORFWorkerFactory@LocalWorkflow@U2@@SAXXZ$109 10023f61 f   ORFWorker.obj
 0001:00022f6c       __unwindfunclet$?init@ORFWorkerFactory@LocalWorkflow@U2@@SAXXZ$110 10023f6c f   ORFWorker.obj
 0001:00022f75       __unwindfunclet$?init@ORFWorkerFactory@LocalWorkflow@U2@@SAXXZ$111 10023f75 f   ORFWorker.obj
 0001:00022f7e       __unwindfunclet$?init@ORFWorkerFactory@LocalWorkflow@U2@@SAXXZ$112 10023f7e f   ORFWorker.obj
 0001:00022f89       __ehhandler$?init@ORFWorkerFactory@LocalWorkflow@U2@@SAXXZ 10023f89 f   ORFWorker.obj
 0001:00022fb0       __unwindfunclet$?metaType@?$QVariantValueHelper@V?$QSharedDataPointer@VDbiDataHandler@Workflow@U2@@@@@QtPrivate@@SA?AV?$QSharedDataPointer@VDbiDataHandler@Workflow@U2@@@@ABVQVariant@@@Z$0 10023fb0 f   ORFWorker.obj
 0001:00022fc9       __unwindfunclet$?metaType@?$QVariantValueHelper@V?$QSharedDataPointer@VDbiDataHandler@Workflow@U2@@@@@QtPrivate@@SA?AV?$QSharedDataPointer@VDbiDataHandler@Workflow@U2@@@@ABVQVariant@@@Z$1 10023fc9 f   ORFWorker.obj
 0001:00022fd1       __ehhandler$?metaType@?$QVariantValueHelper@V?$QSharedDataPointer@VDbiDataHandler@Workflow@U2@@@@@QtPrivate@@SA?AV?$QSharedDataPointer@VDbiDataHandler@Workflow@U2@@@@ABVQVariant@@@Z 10023fd1 f   ORFWorker.obj
 0001:00022ff0       __unwindfunclet$?node_construct@?$QList@U?$QPair@VQString@@VQVariant@@@@@@AAEXPAUNode@1@ABU?$QPair@VQString@@VQVariant@@@@@Z$0 10023ff0 f   ORFWorker.obj
 0001:00022ffb       __unwindfunclet$?node_construct@?$QList@U?$QPair@VQString@@VQVariant@@@@@@AAEXPAUNode@1@ABU?$QPair@VQString@@VQVariant@@@@@Z$2 10023ffb f   ORFWorker.obj
 0001:00023004       __ehhandler$?node_construct@?$QList@U?$QPair@VQString@@VQVariant@@@@@@AAEXPAUNode@1@ABU?$QPair@VQString@@VQVariant@@@@@Z 10024004 f   ORFWorker.obj
 0001:00023020       __unwindfunclet$?node_construct@?$QList@VDescriptor@U2@@@@AAEXPAUNode@1@ABVDescriptor@U2@@@Z$0 10024020 f   ORFWorker.obj
 0001:0002302b       __ehhandler$?node_construct@?$QList@VDescriptor@U2@@@@AAEXPAUNode@1@ABVDescriptor@U2@@@Z 1002402b f   ORFWorker.obj
 0001:00023050       __unwindfunclet$?node_copy@?$QList@U?$QPair@VQString@@VQVariant@@@@@@AAEXPAUNode@1@00@Z$4 10024050 f   ORFWorker.obj
 0001:0002305b       __unwindfunclet$?node_copy@?$QList@U?$QPair@VQString@@VQVariant@@@@@@AAEXPAUNode@1@00@Z$6 1002405b f   ORFWorker.obj
 0001:00023064       __unwindfunclet$?node_copy@?$QList@U?$QPair@VQString@@VQVariant@@@@@@AAEXPAUNode@1@00@Z$8 10024064 f   ORFWorker.obj
 0001:0002306d       __ehhandler$?node_copy@?$QList@U?$QPair@VQString@@VQVariant@@@@@@AAEXPAUNode@1@00@Z 1002406d f   ORFWorker.obj
 0001:00023090       __unwindfunclet$?node_copy@?$QList@VDescriptor@U2@@@@AAEXPAUNode@1@00@Z$4 10024090 f   ORFWorker.obj
 0001:0002309b       __ehhandler$?node_copy@?$QList@VDescriptor@U2@@@@AAEXPAUNode@1@00@Z 1002409b f   ORFWorker.obj
 0001:000230c0       __unwindfunclet$?node_destruct@?$QList@U?$QPair@VQString@@VQVariant@@@@@@AAEXPAUNode@1@0@Z$0 100240c0 f   ORFWorker.obj
 0001:000230c9       __ehhandler$?node_destruct@?$QList@U?$QPair@VQString@@VQVariant@@@@@@AAEXPAUNode@1@0@Z 100240c9 f   ORFWorker.obj
 0001:000230f0       __unwindfunclet$?node_destruct@?$QList@U?$QPair@VQString@@VQVariant@@@@@@AAEXPAUNode@1@@Z$0 100240f0 f   ORFWorker.obj
 0001:000230f9       __ehhandler$?node_destruct@?$QList@U?$QPair@VQString@@VQVariant@@@@@@AAEXPAUNode@1@@Z 100240f9 f   ORFWorker.obj
 0001:00023120       __unwindfunclet$?qt_metatype_id@?$QMetaTypeId@V?$QSharedDataPointer@VDbiDataHandler@Workflow@U2@@@@@@SAHXZ$0 10024120 f   ORFWorker.obj
 0001:00023129       __ehhandler$?qt_metatype_id@?$QMetaTypeId@V?$QSharedDataPointer@VDbiDataHandler@Workflow@U2@@@@@@SAHXZ 10024129 f   ORFWorker.obj
 0001:00023150       __unwindfunclet$?sl_taskFinished@ORFWorker@LocalWorkflow@U2@@AAEXXZ$0 10024150 f   ORFWorker.obj
 0001:00023158       __unwindfunclet$?sl_taskFinished@ORFWorker@LocalWorkflow@U2@@AAEXXZ$1 10024158 f   ORFWorker.obj
 0001:00023160       __unwindfunclet$?sl_taskFinished@ORFWorker@LocalWorkflow@U2@@AAEXXZ$3 10024160 f   ORFWorker.obj
 0001:00023168       __unwindfunclet$?sl_taskFinished@ORFWorker@LocalWorkflow@U2@@AAEXXZ$4 10024168 f   ORFWorker.obj
 0001:00023171       __unwindfunclet$?sl_taskFinished@ORFWorker@LocalWorkflow@U2@@AAEXXZ$6 10024171 f   ORFWorker.obj
 0001:0002317a       __unwindfunclet$?sl_taskFinished@ORFWorker@LocalWorkflow@U2@@AAEXXZ$7 1002417a f   ORFWorker.obj
 0001:00023183       __unwindfunclet$?sl_taskFinished@ORFWorker@LocalWorkflow@U2@@AAEXXZ$8 10024183 f   ORFWorker.obj
 0001:0002318c       __ehhandler$?sl_taskFinished@ORFWorker@LocalWorkflow@U2@@AAEXXZ 1002418c f   ORFWorker.obj
 0001:000231b0       __unwindfunclet$?tick@ORFWorker@LocalWorkflow@U2@@UAEPAVTask@3@XZ$0 100241b0 f   ORFWorker.obj
 0001:000231bc       __unwindfunclet$?tick@ORFWorker@LocalWorkflow@U2@@UAEPAVTask@3@XZ$1 100241bc f   ORFWorker.obj
 0001:000231c8       __unwindfunclet$?tick@ORFWorker@LocalWorkflow@U2@@UAEPAVTask@3@XZ$2 100241c8 f   ORFWorker.obj
 0001:000231d1       __unwindfunclet$?tick@ORFWorker@LocalWorkflow@U2@@UAEPAVTask@3@XZ$3 100241d1 f   ORFWorker.obj
 0001:000231da       __unwindfunclet$?tick@ORFWorker@LocalWorkflow@U2@@UAEPAVTask@3@XZ$4 100241da f   ORFWorker.obj
 0001:000231e3       __unwindfunclet$?tick@ORFWorker@LocalWorkflow@U2@@UAEPAVTask@3@XZ$5 100241e3 f   ORFWorker.obj
 0001:000231ec       __unwindfunclet$?tick@ORFWorker@LocalWorkflow@U2@@UAEPAVTask@3@XZ$6 100241ec f   ORFWorker.obj
 0001:000231f5       __unwindfunclet$?tick@ORFWorker@LocalWorkflow@U2@@UAEPAVTask@3@XZ$7 100241f5 f   ORFWorker.obj
 0001:000231fe       __unwindfunclet$?tick@ORFWorker@LocalWorkflow@U2@@UAEPAVTask@3@XZ$8 100241fe f   ORFWorker.obj
 0001:00023207       __unwindfunclet$?tick@ORFWorker@LocalWorkflow@U2@@UAEPAVTask@3@XZ$9 10024207 f   ORFWorker.obj
 0001:00023212       __unwindfunclet$?tick@ORFWorker@LocalWorkflow@U2@@UAEPAVTask@3@XZ$10 10024212 f   ORFWorker.obj
 0001:0002322c       __unwindfunclet$?tick@ORFWorker@LocalWorkflow@U2@@UAEPAVTask@3@XZ$11 1002422c f   ORFWorker.obj
 0001:00023238       __unwindfunclet$?tick@ORFWorker@LocalWorkflow@U2@@UAEPAVTask@3@XZ$12 10024238 f   ORFWorker.obj
 0001:00023244       __unwindfunclet$?tick@ORFWorker@LocalWorkflow@U2@@UAEPAVTask@3@XZ$13 10024244 f   ORFWorker.obj
 0001:0002324d       __unwindfunclet$?tick@ORFWorker@LocalWorkflow@U2@@UAEPAVTask@3@XZ$14 1002424d f   ORFWorker.obj
 0001:00023259       __unwindfunclet$?tick@ORFWorker@LocalWorkflow@U2@@UAEPAVTask@3@XZ$15 10024259 f   ORFWorker.obj
 0001:00023261       __unwindfunclet$?tick@ORFWorker@LocalWorkflow@U2@@UAEPAVTask@3@XZ$16 10024261 f   ORFWorker.obj
 0001:0002326a       __unwindfunclet$?tick@ORFWorker@LocalWorkflow@U2@@UAEPAVTask@3@XZ$17 1002426a f   ORFWorker.obj
 0001:00023272       __unwindfunclet$?tick@ORFWorker@LocalWorkflow@U2@@UAEPAVTask@3@XZ$18 10024272 f   ORFWorker.obj
 0001:0002327a       __unwindfunclet$?tick@ORFWorker@LocalWorkflow@U2@@UAEPAVTask@3@XZ$19 1002427a f   ORFWorker.obj
 0001:00023285       __unwindfunclet$?tick@ORFWorker@LocalWorkflow@U2@@UAEPAVTask@3@XZ$21 10024285 f   ORFWorker.obj
 0001:0002328e       __unwindfunclet$?tick@ORFWorker@LocalWorkflow@U2@@UAEPAVTask@3@XZ$22 1002428e f   ORFWorker.obj
 0001:00023297       __unwindfunclet$?tick@ORFWorker@LocalWorkflow@U2@@UAEPAVTask@3@XZ$23 10024297 f   ORFWorker.obj
 0001:000232a0       __unwindfunclet$?tick@ORFWorker@LocalWorkflow@U2@@UAEPAVTask@3@XZ$24 100242a0 f   ORFWorker.obj
 0001:000232ab       __ehhandler$?tick@ORFWorker@LocalWorkflow@U2@@UAEPAVTask@3@XZ 100242ab f   ORFWorker.obj
 0001:000232d0       __unwindfunclet$?uniqueKeys@?$QMap@VDescriptor@U2@@VQVariant@@@@QBE?AV?$QList@VDescriptor@U2@@@@XZ$1 100242d0 f   ORFWorker.obj
 0001:000232e9       __ehhandler$?uniqueKeys@?$QMap@VDescriptor@U2@@VQVariant@@@@QBE?AV?$QList@VDescriptor@U2@@@@XZ 100242e9 f   ORFWorker.obj
 0001:00023310       __unwindfunclet$??__EalgoLog@U2@@YAXXZ$0 10024310 f   moc_ORFDialog.obj
 0001:00023319       __ehhandler$??__EalgoLog@U2@@YAXXZ 10024319 f   moc_ORFDialog.obj
 0001:00023340       __unwindfunclet$??__EcmdLog@U2@@YAXXZ$0 10024340 f   moc_ORFDialog.obj
 0001:00023349       __ehhandler$??__EcmdLog@U2@@YAXXZ 10024349 f   moc_ORFDialog.obj
 0001:00023370       __unwindfunclet$??__EcoreLog@U2@@YAXXZ$0 10024370 f   moc_ORFDialog.obj
 0001:00023379       __ehhandler$??__EcoreLog@U2@@YAXXZ 10024379 f   moc_ORFDialog.obj
 0001:000233a0       __unwindfunclet$??__EioLog@U2@@YAXXZ$0 100243a0 f   moc_ORFDialog.obj
 0001:000233a9       __ehhandler$??__EioLog@U2@@YAXXZ 100243a9 f   moc_ORFDialog.obj
 0001:000233d0       __unwindfunclet$??__EperfLog@U2@@YAXXZ$0 100243d0 f   moc_ORFDialog.obj
 0001:000233d9       __ehhandler$??__EperfLog@U2@@YAXXZ 100243d9 f   moc_ORFDialog.obj
 0001:00023400       __unwindfunclet$??__EscriptLog@U2@@YAXXZ$0 10024400 f   moc_ORFDialog.obj
 0001:00023409       __ehhandler$??__EscriptLog@U2@@YAXXZ 10024409 f   moc_ORFDialog.obj
 0001:00023430       __unwindfunclet$??__EtaskLog@U2@@YAXXZ$0 10024430 f   moc_ORFDialog.obj
 0001:00023439       __ehhandler$??__EtaskLog@U2@@YAXXZ 10024439 f   moc_ORFDialog.obj
 0001:00023460       __unwindfunclet$??__EuiLog@U2@@YAXXZ$0 10024460 f   moc_ORFDialog.obj
 0001:00023469       __ehhandler$??__EuiLog@U2@@YAXXZ 10024469 f   moc_ORFDialog.obj
 0001:00023490       __unwindfunclet$??__EuserActLog@U2@@YAXXZ$0 10024490 f   moc_ORFDialog.obj
 0001:00023499       __ehhandler$??__EuserActLog@U2@@YAXXZ 10024499 f   moc_ORFDialog.obj
 0001:000234c0       __unwindfunclet$?qt_metatype_id@?$QMetaTypeIdQObject@PAVTask@U2@@$00@@SAHXZ$0 100244c0 f   moc_ORFDialog.obj
 0001:000234c9       __ehhandler$?qt_metatype_id@?$QMetaTypeIdQObject@PAVTask@U2@@$00@@SAHXZ 100244c9 f   moc_ORFDialog.obj
 0001:000234f0       __unwindfunclet$??__EalgoLog@U2@@YAXXZ$0 100244f0 f   moc_ORFMarkerTask.obj
 0001:000234f9       __ehhandler$??__EalgoLog@U2@@YAXXZ 100244f9 f   moc_ORFMarkerTask.obj
 0001:00023520       __unwindfunclet$??__EcmdLog@U2@@YAXXZ$0 10024520 f   moc_ORFMarkerTask.obj
 0001:00023529       __ehhandler$??__EcmdLog@U2@@YAXXZ 10024529 f   moc_ORFMarkerTask.obj
 0001:00023550       __unwindfunclet$??__EcoreLog@U2@@YAXXZ$0 10024550 f   moc_ORFMarkerTask.obj
 0001:00023559       __ehhandler$??__EcoreLog@U2@@YAXXZ 10024559 f   moc_ORFMarkerTask.obj
 0001:00023580       __unwindfunclet$??__EioLog@U2@@YAXXZ$0 10024580 f   moc_ORFMarkerTask.obj
 0001:00023589       __ehhandler$??__EioLog@U2@@YAXXZ 10024589 f   moc_ORFMarkerTask.obj
 0001:000235b0       __unwindfunclet$??__EperfLog@U2@@YAXXZ$0 100245b0 f   moc_ORFMarkerTask.obj
 0001:000235b9       __ehhandler$??__EperfLog@U2@@YAXXZ 100245b9 f   moc_ORFMarkerTask.obj
 0001:000235e0       __unwindfunclet$??__EscriptLog@U2@@YAXXZ$0 100245e0 f   moc_ORFMarkerTask.obj
 0001:000235e9       __ehhandler$??__EscriptLog@U2@@YAXXZ 100245e9 f   moc_ORFMarkerTask.obj
 0001:00023610       __unwindfunclet$??__EtaskLog@U2@@YAXXZ$0 10024610 f   moc_ORFMarkerTask.obj
 0001:00023619       __ehhandler$??__EtaskLog@U2@@YAXXZ 10024619 f   moc_ORFMarkerTask.obj
 0001:00023640       __unwindfunclet$??__EuiLog@U2@@YAXXZ$0 10024640 f   moc_ORFMarkerTask.obj
 0001:00023649       __ehhandler$??__EuiLog@U2@@YAXXZ 10024649 f   moc_ORFMarkerTask.obj
 0001:00023670       __unwindfunclet$??__EuserActLog@U2@@YAXXZ$0 10024670 f   moc_ORFMarkerTask.obj
 0001:00023679       __ehhandler$??__EuserActLog@U2@@YAXXZ 10024679 f   moc_ORFMarkerTask.obj
 0001:000236a0       __unwindfunclet$??__EalgoLog@U2@@YAXXZ$0 100246a0 f   moc_ORFMarkerTests.obj
 0001:000236a9       __ehhandler$??__EalgoLog@U2@@YAXXZ 100246a9 f   moc_ORFMarkerTests.obj
 0001:000236d0       __unwindfunclet$??__EcmdLog@U2@@YAXXZ$0 100246d0 f   moc_ORFMarkerTests.obj
 0001:000236d9       __ehhandler$??__EcmdLog@U2@@YAXXZ 100246d9 f   moc_ORFMarkerTests.obj
 0001:00023700       __unwindfunclet$??__EcoreLog@U2@@YAXXZ$0 10024700 f   moc_ORFMarkerTests.obj
 0001:00023709       __ehhandler$??__EcoreLog@U2@@YAXXZ 10024709 f   moc_ORFMarkerTests.obj
 0001:00023730       __unwindfunclet$??__EioLog@U2@@YAXXZ$0 10024730 f   moc_ORFMarkerTests.obj
 0001:00023739       __ehhandler$??__EioLog@U2@@YAXXZ 10024739 f   moc_ORFMarkerTests.obj
 0001:00023760       __unwindfunclet$??__EperfLog@U2@@YAXXZ$0 10024760 f   moc_ORFMarkerTests.obj
 0001:00023769       __ehhandler$??__EperfLog@U2@@YAXXZ 10024769 f   moc_ORFMarkerTests.obj
 0001:00023790       __unwindfunclet$??__EscriptLog@U2@@YAXXZ$0 10024790 f   moc_ORFMarkerTests.obj
 0001:00023799       __ehhandler$??__EscriptLog@U2@@YAXXZ 10024799 f   moc_ORFMarkerTests.obj
 0001:000237c0       __unwindfunclet$??__EtaskLog@U2@@YAXXZ$0 100247c0 f   moc_ORFMarkerTests.obj
 0001:000237c9       __ehhandler$??__EtaskLog@U2@@YAXXZ 100247c9 f   moc_ORFMarkerTests.obj
 0001:000237f0       __unwindfunclet$??__EuiLog@U2@@YAXXZ$0 100247f0 f   moc_ORFMarkerTests.obj
 0001:000237f9       __ehhandler$??__EuiLog@U2@@YAXXZ 100247f9 f   moc_ORFMarkerTests.obj
 0001:00023820       __unwindfunclet$??__EuserActLog@U2@@YAXXZ$0 10024820 f   moc_ORFMarkerTests.obj
 0001:00023829       __ehhandler$??__EuserActLog@U2@@YAXXZ 10024829 f   moc_ORFMarkerTests.obj
 0001:00023850       __unwindfunclet$??__EalgoLog@U2@@YAXXZ$0 10024850 f   moc_ORFQuery.obj
 0001:00023859       __ehhandler$??__EalgoLog@U2@@YAXXZ 10024859 f   moc_ORFQuery.obj
 0001:00023880       __unwindfunclet$??__EcmdLog@U2@@YAXXZ$0 10024880 f   moc_ORFQuery.obj
 0001:00023889       __ehhandler$??__EcmdLog@U2@@YAXXZ 10024889 f   moc_ORFQuery.obj
 0001:000238b0       __unwindfunclet$??__EcoreLog@U2@@YAXXZ$0 100248b0 f   moc_ORFQuery.obj
 0001:000238b9       __ehhandler$??__EcoreLog@U2@@YAXXZ 100248b9 f   moc_ORFQuery.obj
 0001:000238e0       __unwindfunclet$??__EioLog@U2@@YAXXZ$0 100248e0 f   moc_ORFQuery.obj
 0001:000238e9       __ehhandler$??__EioLog@U2@@YAXXZ 100248e9 f   moc_ORFQuery.obj
 0001:00023910       __unwindfunclet$??__EperfLog@U2@@YAXXZ$0 10024910 f   moc_ORFQuery.obj
 0001:00023919       __ehhandler$??__EperfLog@U2@@YAXXZ 10024919 f   moc_ORFQuery.obj
 0001:00023940       __unwindfunclet$??__EscriptLog@U2@@YAXXZ$0 10024940 f   moc_ORFQuery.obj
 0001:00023949       __ehhandler$??__EscriptLog@U2@@YAXXZ 10024949 f   moc_ORFQuery.obj
 0001:00023970       __unwindfunclet$??__EtaskLog@U2@@YAXXZ$0 10024970 f   moc_ORFQuery.obj
 0001:00023979       __ehhandler$??__EtaskLog@U2@@YAXXZ 10024979 f   moc_ORFQuery.obj
 0001:000239a0       __unwindfunclet$??__EuiLog@U2@@YAXXZ$0 100249a0 f   moc_ORFQuery.obj
 0001:000239a9       __ehhandler$??__EuiLog@U2@@YAXXZ 100249a9 f   moc_ORFQuery.obj
 0001:000239d0       __unwindfunclet$??__EuserActLog@U2@@YAXXZ$0 100249d0 f   moc_ORFQuery.obj
 0001:000239d9       __ehhandler$??__EuserActLog@U2@@YAXXZ 100249d9 f   moc_ORFQuery.obj
 0001:00023a00       __unwindfunclet$??__EalgoLog@U2@@YAXXZ$0 10024a00 f   moc_ORFWorker.obj
 0001:00023a09       __ehhandler$??__EalgoLog@U2@@YAXXZ 10024a09 f   moc_ORFWorker.obj
 0001:00023a30       __unwindfunclet$??__EcmdLog@U2@@YAXXZ$0 10024a30 f   moc_ORFWorker.obj
 0001:00023a39       __ehhandler$??__EcmdLog@U2@@YAXXZ 10024a39 f   moc_ORFWorker.obj
 0001:00023a60       __unwindfunclet$??__EcoreLog@U2@@YAXXZ$0 10024a60 f   moc_ORFWorker.obj
 0001:00023a69       __ehhandler$??__EcoreLog@U2@@YAXXZ 10024a69 f   moc_ORFWorker.obj
 0001:00023a90       __unwindfunclet$??__EioLog@U2@@YAXXZ$0 10024a90 f   moc_ORFWorker.obj
 0001:00023a99       __ehhandler$??__EioLog@U2@@YAXXZ 10024a99 f   moc_ORFWorker.obj
 0001:00023ac0       __unwindfunclet$??__EperfLog@U2@@YAXXZ$0 10024ac0 f   moc_ORFWorker.obj
 0001:00023ac9       __ehhandler$??__EperfLog@U2@@YAXXZ 10024ac9 f   moc_ORFWorker.obj
 0001:00023af0       __unwindfunclet$??__EscriptLog@U2@@YAXXZ$0 10024af0 f   moc_ORFWorker.obj
 0001:00023af9       __ehhandler$??__EscriptLog@U2@@YAXXZ 10024af9 f   moc_ORFWorker.obj
 0001:00023b20       __unwindfunclet$??__EtaskLog@U2@@YAXXZ$0 10024b20 f   moc_ORFWorker.obj
 0001:00023b29       __ehhandler$??__EtaskLog@U2@@YAXXZ 10024b29 f   moc_ORFWorker.obj
 0001:00023b50       __unwindfunclet$??__EuiLog@U2@@YAXXZ$0 10024b50 f   moc_ORFWorker.obj
 0001:00023b59       __ehhandler$??__EuiLog@U2@@YAXXZ 10024b59 f   moc_ORFWorker.obj
 0001:00023b80       __unwindfunclet$??__EuserActLog@U2@@YAXXZ$0 10024b80 f   moc_ORFWorker.obj
 0001:00023b89       __ehhandler$??__EuserActLog@U2@@YAXXZ 10024b89 f   moc_ORFWorker.obj
 0001:00023bb0       ??__F?_Generic_object@?$_Error_objects@H@std@@2V_Generic_error_category@2@A@@YAXXZ 10024bb0 f   ORFDialog.obj
 0001:00023bc0       ??__F?_Iostream_object@?$_Error_objects@H@std@@2V_Iostream_error_category@2@A@@YAXXZ 10024bc0 f   ORFDialog.obj
 0001:00023bd0       ??__F?_System_object@?$_Error_objects@H@std@@2V_System_error_category@2@A@@YAXXZ 10024bd0 f   ORFDialog.obj
 0001:00023be0       ??__FService_DNAExport@U2@@YAXXZ 10024be0 f   ORFDialog.obj
 0001:00023bf0       ??__FService_DNAGraphPack@U2@@YAXXZ 10024bf0 f   ORFDialog.obj
 0001:00023c00       ??__FService_ExternalToolSupport@U2@@YAXXZ 10024c00 f   ORFDialog.obj
 0001:00023c10       ??__FService_GUITesting@U2@@YAXXZ 10024c10 f   ORFDialog.obj
 0001:00023c20       ??__FService_MaxCoreServiceId@U2@@YAXXZ 10024c20 f   ORFDialog.obj
 0001:00023c30       ??__FService_MinCoreServiceId@U2@@YAXXZ 10024c30 f   ORFDialog.obj
 0001:00023c40       ??__FService_PluginViewer@U2@@YAXXZ 10024c40 f   ORFDialog.obj
 0001:00023c50       ??__FService_Project@U2@@YAXXZ 10024c50 f   ORFDialog.obj
 0001:00023c60       ??__FService_ProjectView@U2@@YAXXZ 10024c60 f   ORFDialog.obj
 0001:00023c70       ??__FService_QueryDesigner@U2@@YAXXZ 10024c70 f   ORFDialog.obj
 0001:00023c80       ??__FService_ScriptRegistry@U2@@YAXXZ 10024c80 f   ORFDialog.obj
 0001:00023c90       ??__FService_TestRunner@U2@@YAXXZ 10024c90 f   ORFDialog.obj
 0001:00023ca0       ??__FService_WorkflowDesigner@U2@@YAXXZ 10024ca0 f   ORFDialog.obj
 0001:00023cb0       ??__FalgoLog@U2@@YAXXZ     10024cb0 f   ORFDialog.obj
 0001:00023cc0       ??__FcmdLog@U2@@YAXXZ      10024cc0 f   ORFDialog.obj
 0001:00023cd0       ??__FcoreLog@U2@@YAXXZ     10024cd0 f   ORFDialog.obj
 0001:00023ce0       ??__FioLog@U2@@YAXXZ       10024ce0 f   ORFDialog.obj
 0001:00023cf0       ??__FperfLog@U2@@YAXXZ     10024cf0 f   ORFDialog.obj
 0001:00023d00       ??__FscriptLog@U2@@YAXXZ   10024d00 f   ORFDialog.obj
 0001:00023d10       ??__FtaskLog@U2@@YAXXZ     10024d10 f   ORFDialog.obj
 0001:00023d20       ??__FuiLog@U2@@YAXXZ       10024d20 f   ORFDialog.obj
 0001:00023d30       ??__FuserActLog@U2@@YAXXZ  10024d30 f   ORFDialog.obj
 0001:00023d40       ??__F?_Generic_object@?$_Error_objects@H@std@@2V_Generic_error_category@2@A@@YAXXZ 10024d40 f   ORFMarkerPlugin.obj
 0001:00023d50       ??__F?_Iostream_object@?$_Error_objects@H@std@@2V_Iostream_error_category@2@A@@YAXXZ 10024d50 f   ORFMarkerPlugin.obj
 0001:00023d60       ??__F?_System_object@?$_Error_objects@H@std@@2V_System_error_category@2@A@@YAXXZ 10024d60 f   ORFMarkerPlugin.obj
 0001:00023d70       ??__FService_DNAExport@U2@@YAXXZ 10024d70 f   ORFMarkerPlugin.obj
 0001:00023d80       ??__FService_DNAGraphPack@U2@@YAXXZ 10024d80 f   ORFMarkerPlugin.obj
 0001:00023d90       ??__FService_ExternalToolSupport@U2@@YAXXZ 10024d90 f   ORFMarkerPlugin.obj
 0001:00023da0       ??__FService_GUITesting@U2@@YAXXZ 10024da0 f   ORFMarkerPlugin.obj
 0001:00023db0       ??__FService_MaxCoreServiceId@U2@@YAXXZ 10024db0 f   ORFMarkerPlugin.obj
 0001:00023dc0       ??__FService_MinCoreServiceId@U2@@YAXXZ 10024dc0 f   ORFMarkerPlugin.obj
 0001:00023dd0       ??__FService_PluginViewer@U2@@YAXXZ 10024dd0 f   ORFMarkerPlugin.obj
 0001:00023de0       ??__FService_Project@U2@@YAXXZ 10024de0 f   ORFMarkerPlugin.obj
 0001:00023df0       ??__FService_ProjectView@U2@@YAXXZ 10024df0 f   ORFMarkerPlugin.obj
 0001:00023e00       ??__FService_QueryDesigner@U2@@YAXXZ 10024e00 f   ORFMarkerPlugin.obj
 0001:00023e10       ??__FService_ScriptRegistry@U2@@YAXXZ 10024e10 f   ORFMarkerPlugin.obj
 0001:00023e20       ??__FService_TestRunner@U2@@YAXXZ 10024e20 f   ORFMarkerPlugin.obj
 0001:00023e30       ??__FService_WorkflowDesigner@U2@@YAXXZ 10024e30 f   ORFMarkerPlugin.obj
 0001:00023e40       ??__FalgoLog@U2@@YAXXZ     10024e40 f   ORFMarkerPlugin.obj
 0001:00023e50       ??__FcmdLog@U2@@YAXXZ      10024e50 f   ORFMarkerPlugin.obj
 0001:00023e60       ??__FcoreLog@U2@@YAXXZ     10024e60 f   ORFMarkerPlugin.obj
 0001:00023e70       ??__FioLog@U2@@YAXXZ       10024e70 f   ORFMarkerPlugin.obj
 0001:00023e80       ??__FperfLog@U2@@YAXXZ     10024e80 f   ORFMarkerPlugin.obj
 0001:00023e90       ??__FscriptLog@U2@@YAXXZ   10024e90 f   ORFMarkerPlugin.obj
 0001:00023ea0       ??__FtaskLog@U2@@YAXXZ     10024ea0 f   ORFMarkerPlugin.obj
 0001:00023eb0       ??__FuiLog@U2@@YAXXZ       10024eb0 f   ORFMarkerPlugin.obj
 0001:00023ec0       ??__FuserActLog@U2@@YAXXZ  10024ec0 f   ORFMarkerPlugin.obj
 0001:00023ed0       ??__F?ALLOW_ALT_START@ORFSettingsKeys@U2@@2VQString@@B@@YAXXZ 10024ed0 f   ORFMarkerTask.obj
 0001:00023ee0       ??__F?ALLOW_OVERLAP@ORFSettingsKeys@U2@@2VQString@@B@@YAXXZ 10024ee0 f   ORFMarkerTask.obj
 0001:00023ef0       ??__F?AMINO_TRANSL@ORFSettingsKeys@U2@@2VQString@@B@@YAXXZ 10024ef0 f   ORFMarkerTask.obj
 0001:00023f00       ??__F?INCLUDE_STOP_CODON@ORFSettingsKeys@U2@@2VQString@@B@@YAXXZ 10024f00 f   ORFMarkerTask.obj
 0001:00023f10       ??__F?IS_RESULT_LIMITED@ORFSettingsKeys@U2@@2VQString@@B@@YAXXZ 10024f10 f   ORFMarkerTask.obj
 0001:00023f20       ??__F?MAX_RESULT@ORFSettingsKeys@U2@@2VQString@@B@@YAXXZ 10024f20 f   ORFMarkerTask.obj
 0001:00023f30       ??__F?MIN_LEN@ORFSettingsKeys@U2@@2VQString@@B@@YAXXZ 10024f30 f   ORFMarkerTask.obj
 0001:00023f40       ??__F?MUST_FIT@ORFSettingsKeys@U2@@2VQString@@B@@YAXXZ 10024f40 f   ORFMarkerTask.obj
 0001:00023f50       ??__F?MUST_INIT@ORFSettingsKeys@U2@@2VQString@@B@@YAXXZ 10024f50 f   ORFMarkerTask.obj
 0001:00023f60       ??__F?SEARCH_REGION@ORFSettingsKeys@U2@@2VQString@@B@@YAXXZ 10024f60 f   ORFMarkerTask.obj
 0001:00023f70       ??__F?STRAND@ORFSettingsKeys@U2@@2VQString@@B@@YAXXZ 10024f70 f   ORFMarkerTask.obj
 0001:00023f80       ??__F?_Generic_object@?$_Error_objects@H@std@@2V_Generic_error_category@2@A@@YAXXZ 10024f80 f   ORFMarkerTask.obj
 0001:00023f90       ??__F?_Iostream_object@?$_Error_objects@H@std@@2V_Iostream_error_category@2@A@@YAXXZ 10024f90 f   ORFMarkerTask.obj
 0001:00023fa0       ??__F?_System_object@?$_Error_objects@H@std@@2V_System_error_category@2@A@@YAXXZ 10024fa0 f   ORFMarkerTask.obj
 0001:00023fb0       ??__FalgoLog@U2@@YAXXZ     10024fb0 f   ORFMarkerTask.obj
 0001:00023fc0       ??__FcmdLog@U2@@YAXXZ      10024fc0 f   ORFMarkerTask.obj
 0001:00023fd0       ??__FcoreLog@U2@@YAXXZ     10024fd0 f   ORFMarkerTask.obj
 0001:00023fe0       ??__FioLog@U2@@YAXXZ       10024fe0 f   ORFMarkerTask.obj
 0001:00023ff0       ??__FperfLog@U2@@YAXXZ     10024ff0 f   ORFMarkerTask.obj
 0001:00024000       ??__FscriptLog@U2@@YAXXZ   10025000 f   ORFMarkerTask.obj
 0001:00024010       ??__FtaskLog@U2@@YAXXZ     10025010 f   ORFMarkerTask.obj
 0001:00024020       ??__FuiLog@U2@@YAXXZ       10025020 f   ORFMarkerTask.obj
 0001:00024030       ??__FuserActLog@U2@@YAXXZ  10025030 f   ORFMarkerTask.obj
 0001:00024040       ??__F?_Generic_object@?$_Error_objects@H@std@@2V_Generic_error_category@2@A@@YAXXZ 10025040 f   ORFMarkerTests.obj
 0001:00024050       ??__F?_Iostream_object@?$_Error_objects@H@std@@2V_Iostream_error_category@2@A@@YAXXZ 10025050 f   ORFMarkerTests.obj
 0001:00024060       ??__F?_System_object@?$_Error_objects@H@std@@2V_System_error_category@2@A@@YAXXZ 10025060 f   ORFMarkerTests.obj
 0001:00024070       ??__FService_DNAExport@U2@@YAXXZ 10025070 f   ORFMarkerTests.obj
 0001:00024080       ??__FService_DNAGraphPack@U2@@YAXXZ 10025080 f   ORFMarkerTests.obj
 0001:00024090       ??__FService_ExternalToolSupport@U2@@YAXXZ 10025090 f   ORFMarkerTests.obj
 0001:000240a0       ??__FService_GUITesting@U2@@YAXXZ 100250a0 f   ORFMarkerTests.obj
 0001:000240b0       ??__FService_MaxCoreServiceId@U2@@YAXXZ 100250b0 f   ORFMarkerTests.obj
 0001:000240c0       ??__FService_MinCoreServiceId@U2@@YAXXZ 100250c0 f   ORFMarkerTests.obj
 0001:000240d0       ??__FService_PluginViewer@U2@@YAXXZ 100250d0 f   ORFMarkerTests.obj
 0001:000240e0       ??__FService_Project@U2@@YAXXZ 100250e0 f   ORFMarkerTests.obj
 0001:000240f0       ??__FService_ProjectView@U2@@YAXXZ 100250f0 f   ORFMarkerTests.obj
 0001:00024100       ??__FService_QueryDesigner@U2@@YAXXZ 10025100 f   ORFMarkerTests.obj
 0001:00024110       ??__FService_ScriptRegistry@U2@@YAXXZ 10025110 f   ORFMarkerTests.obj
 0001:00024120       ??__FService_TestRunner@U2@@YAXXZ 10025120 f   ORFMarkerTests.obj
 0001:00024130       ??__FService_WorkflowDesigner@U2@@YAXXZ 10025130 f   ORFMarkerTests.obj
 0001:00024140       ??__FalgoLog@U2@@YAXXZ     10025140 f   ORFMarkerTests.obj
 0001:00024150       ??__FcmdLog@U2@@YAXXZ      10025150 f   ORFMarkerTests.obj
 0001:00024160       ??__FcoreLog@U2@@YAXXZ     10025160 f   ORFMarkerTests.obj
 0001:00024170       ??__FioLog@U2@@YAXXZ       10025170 f   ORFMarkerTests.obj
 0001:00024180       ??__FperfLog@U2@@YAXXZ     10025180 f   ORFMarkerTests.obj
 0001:00024190       ??__FscriptLog@U2@@YAXXZ   10025190 f   ORFMarkerTests.obj
 0001:000241a0       ??__FtaskLog@U2@@YAXXZ     100251a0 f   ORFMarkerTests.obj
 0001:000241b0       ??__FuiLog@U2@@YAXXZ       100251b0 f   ORFMarkerTests.obj
 0001:000241c0       ??__FuserActLog@U2@@YAXXZ  100251c0 f   ORFMarkerTests.obj
 0001:000241d0       ??__F?_Generic_object@?$_Error_objects@H@std@@2V_Generic_error_category@2@A@@YAXXZ 100251d0 f   ORFQuery.obj
 0001:000241e0       ??__F?_Iostream_object@?$_Error_objects@H@std@@2V_Iostream_error_category@2@A@@YAXXZ 100251e0 f   ORFQuery.obj
 0001:000241f0       ??__F?_System_object@?$_Error_objects@H@std@@2V_System_error_category@2@A@@YAXXZ 100251f0 f   ORFQuery.obj
 0001:00024200       ??__FALT_ATTR@U2@@YAXXZ    10025200 f   ORFQuery.obj
 0001:00024210       ??__FFIT_ATTR@U2@@YAXXZ    10025210 f   ORFQuery.obj
 0001:00024220       ??__FID_ATTR@U2@@YAXXZ     10025220 f   ORFQuery.obj
 0001:00024230       ??__FINIT_ATTR@U2@@YAXXZ   10025230 f   ORFQuery.obj
 0001:00024240       ??__FLEN_ATTR@U2@@YAXXZ    10025240 f   ORFQuery.obj
 0001:00024250       ??__FLIMIT_ATTR@U2@@YAXXZ  10025250 f   ORFQuery.obj
 0001:00024260       ??__FMAX_LENGTH_ATTR@U2@@YAXXZ 10025260 f   ORFQuery.obj
 0001:00024270       ??__FRES_ATTR@U2@@YAXXZ    10025270 f   ORFQuery.obj
 0001:00024280       ??__FalgoLog@U2@@YAXXZ     10025280 f   ORFQuery.obj
 0001:00024290       ??__FcmdLog@U2@@YAXXZ      10025290 f   ORFQuery.obj
 0001:000242a0       ??__FcoreLog@U2@@YAXXZ     100252a0 f   ORFQuery.obj
 0001:000242b0       ??__FioLog@U2@@YAXXZ       100252b0 f   ORFQuery.obj
 0001:000242c0       ??__FperfLog@U2@@YAXXZ     100252c0 f   ORFQuery.obj
 0001:000242d0       ??__FscriptLog@U2@@YAXXZ   100252d0 f   ORFQuery.obj
 0001:000242e0       ??__FtaskLog@U2@@YAXXZ     100252e0 f   ORFQuery.obj
 0001:000242f0       ??__FuiLog@U2@@YAXXZ       100252f0 f   ORFQuery.obj
 0001:00024300       ??__FuserActLog@U2@@YAXXZ  10025300 f   ORFQuery.obj
 0001:00024310       ??__F?ACTOR_ID@ORFWorkerFactory@LocalWorkflow@U2@@2VQString@@B@@YAXXZ 10025310 f   ORFWorker.obj
 0001:00024320       ??__F?_Generic_object@?$_Error_objects@H@std@@2V_Generic_error_category@2@A@@YAXXZ 10025320 f   ORFWorker.obj
 0001:00024330       ??__F?_Iostream_object@?$_Error_objects@H@std@@2V_Iostream_error_category@2@A@@YAXXZ 10025330 f   ORFWorker.obj
 0001:00024340       ??__F?_System_object@?$_Error_objects@H@std@@2V_System_error_category@2@A@@YAXXZ 10025340 f   ORFWorker.obj
 0001:00024350       ??__FALT_ATTR@LocalWorkflow@U2@@YAXXZ 10025350 f   ORFWorker.obj
 0001:00024360       ??__FFIT_ATTR@LocalWorkflow@U2@@YAXXZ 10025360 f   ORFWorker.obj
 0001:00024370       ??__FID_ATTR@LocalWorkflow@U2@@YAXXZ 10025370 f   ORFWorker.obj
 0001:00024380       ??__FINIT_ATTR@LocalWorkflow@U2@@YAXXZ 10025380 f   ORFWorker.obj
 0001:00024390       ??__FISC_ATTR@LocalWorkflow@U2@@YAXXZ 10025390 f   ORFWorker.obj
 0001:000243a0       ??__FLEN_ATTR@LocalWorkflow@U2@@YAXXZ 100253a0 f   ORFWorker.obj
 0001:000243b0       ??__FLIMIT_ATTR@LocalWorkflow@U2@@YAXXZ 100253b0 f   ORFWorker.obj
 0001:000243c0       ??__FNAME_ATTR@LocalWorkflow@U2@@YAXXZ 100253c0 f   ORFWorker.obj
 0001:000243d0       ??__FRES_ATTR@LocalWorkflow@U2@@YAXXZ 100253d0 f   ORFWorker.obj
 0001:000243e0       ??__FalgoLog@U2@@YAXXZ     100253e0 f   ORFWorker.obj
 0001:000243f0       ??__FcmdLog@U2@@YAXXZ      100253f0 f   ORFWorker.obj
 0001:00024400       ??__FcoreLog@U2@@YAXXZ     10025400 f   ORFWorker.obj
 0001:00024410       ??__FioLog@U2@@YAXXZ       10025410 f   ORFWorker.obj
 0001:00024420       ??__FperfLog@U2@@YAXXZ     10025420 f   ORFWorker.obj
 0001:00024430       ??__FscriptLog@U2@@YAXXZ   10025430 f   ORFWorker.obj
 0001:00024440       ??__FtaskLog@U2@@YAXXZ     10025440 f   ORFWorker.obj
 0001:00024450       ??__FuiLog@U2@@YAXXZ       10025450 f   ORFWorker.obj
 0001:00024460       ??__FuserActLog@U2@@YAXXZ  10025460 f   ORFWorker.obj
 0001:00024470       ??__F?_Generic_object@?$_Error_objects@H@std@@2V_Generic_error_category@2@A@@YAXXZ 10025470 f   moc_ORFDialog.obj
 0001:00024480       ??__F?_Iostream_object@?$_Error_objects@H@std@@2V_Iostream_error_category@2@A@@YAXXZ 10025480 f   moc_ORFDialog.obj
 0001:00024490       ??__F?_System_object@?$_Error_objects@H@std@@2V_System_error_category@2@A@@YAXXZ 10025490 f   moc_ORFDialog.obj
 0001:000244a0       ??__FalgoLog@U2@@YAXXZ     100254a0 f   moc_ORFDialog.obj
 0001:000244b0       ??__FcmdLog@U2@@YAXXZ      100254b0 f   moc_ORFDialog.obj
 0001:000244c0       ??__FcoreLog@U2@@YAXXZ     100254c0 f   moc_ORFDialog.obj
 0001:000244d0       ??__FioLog@U2@@YAXXZ       100254d0 f   moc_ORFDialog.obj
 0001:000244e0       ??__FperfLog@U2@@YAXXZ     100254e0 f   moc_ORFDialog.obj
 0001:000244f0       ??__FscriptLog@U2@@YAXXZ   100254f0 f   moc_ORFDialog.obj
 0001:00024500       ??__FtaskLog@U2@@YAXXZ     10025500 f   moc_ORFDialog.obj
 0001:00024510       ??__FuiLog@U2@@YAXXZ       10025510 f   moc_ORFDialog.obj
 0001:00024520       ??__FuserActLog@U2@@YAXXZ  10025520 f   moc_ORFDialog.obj
 0001:00024530       ??__F?_Generic_object@?$_Error_objects@H@std@@2V_Generic_error_category@2@A@@YAXXZ 10025530 f   moc_ORFMarkerPlugin.obj
 0001:00024540       ??__F?_Iostream_object@?$_Error_objects@H@std@@2V_Iostream_error_category@2@A@@YAXXZ 10025540 f   moc_ORFMarkerPlugin.obj
 0001:00024550       ??__F?_System_object@?$_Error_objects@H@std@@2V_System_error_category@2@A@@YAXXZ 10025550 f   moc_ORFMarkerPlugin.obj
 0001:00024560       ??__FService_DNAExport@U2@@YAXXZ 10025560 f   moc_ORFMarkerPlugin.obj
 0001:00024570       ??__FService_DNAGraphPack@U2@@YAXXZ 10025570 f   moc_ORFMarkerPlugin.obj
 0001:00024580       ??__FService_ExternalToolSupport@U2@@YAXXZ 10025580 f   moc_ORFMarkerPlugin.obj
 0001:00024590       ??__FService_GUITesting@U2@@YAXXZ 10025590 f   moc_ORFMarkerPlugin.obj
 0001:000245a0       ??__FService_MaxCoreServiceId@U2@@YAXXZ 100255a0 f   moc_ORFMarkerPlugin.obj
 0001:000245b0       ??__FService_MinCoreServiceId@U2@@YAXXZ 100255b0 f   moc_ORFMarkerPlugin.obj
 0001:000245c0       ??__FService_PluginViewer@U2@@YAXXZ 100255c0 f   moc_ORFMarkerPlugin.obj
 0001:000245d0       ??__FService_Project@U2@@YAXXZ 100255d0 f   moc_ORFMarkerPlugin.obj
 0001:000245e0       ??__FService_ProjectView@U2@@YAXXZ 100255e0 f   moc_ORFMarkerPlugin.obj
 0001:000245f0       ??__FService_QueryDesigner@U2@@YAXXZ 100255f0 f   moc_ORFMarkerPlugin.obj
 0001:00024600       ??__FService_ScriptRegistry@U2@@YAXXZ 10025600 f   moc_ORFMarkerPlugin.obj
 0001:00024610       ??__FService_TestRunner@U2@@YAXXZ 10025610 f   moc_ORFMarkerPlugin.obj
 0001:00024620       ??__FService_WorkflowDesigner@U2@@YAXXZ 10025620 f   moc_ORFMarkerPlugin.obj
 0001:00024630       ??__F?_Generic_object@?$_Error_objects@H@std@@2V_Generic_error_category@2@A@@YAXXZ 10025630 f   moc_ORFMarkerTask.obj
 0001:00024640       ??__F?_Iostream_object@?$_Error_objects@H@std@@2V_Iostream_error_category@2@A@@YAXXZ 10025640 f   moc_ORFMarkerTask.obj
 0001:00024650       ??__F?_System_object@?$_Error_objects@H@std@@2V_System_error_category@2@A@@YAXXZ 10025650 f   moc_ORFMarkerTask.obj
 0001:00024660       ??__FalgoLog@U2@@YAXXZ     10025660 f   moc_ORFMarkerTask.obj
 0001:00024670       ??__FcmdLog@U2@@YAXXZ      10025670 f   moc_ORFMarkerTask.obj
 0001:00024680       ??__FcoreLog@U2@@YAXXZ     10025680 f   moc_ORFMarkerTask.obj
 0001:00024690       ??__FioLog@U2@@YAXXZ       10025690 f   moc_ORFMarkerTask.obj
 0001:000246a0       ??__FperfLog@U2@@YAXXZ     100256a0 f   moc_ORFMarkerTask.obj
 0001:000246b0       ??__FscriptLog@U2@@YAXXZ   100256b0 f   moc_ORFMarkerTask.obj
 0001:000246c0       ??__FtaskLog@U2@@YAXXZ     100256c0 f   moc_ORFMarkerTask.obj
 0001:000246d0       ??__FuiLog@U2@@YAXXZ       100256d0 f   moc_ORFMarkerTask.obj
 0001:000246e0       ??__FuserActLog@U2@@YAXXZ  100256e0 f   moc_ORFMarkerTask.obj
 0001:000246f0       ??__F?_Generic_object@?$_Error_objects@H@std@@2V_Generic_error_category@2@A@@YAXXZ 100256f0 f   moc_ORFMarkerTests.obj
 0001:00024700       ??__F?_Iostream_object@?$_Error_objects@H@std@@2V_Iostream_error_category@2@A@@YAXXZ 10025700 f   moc_ORFMarkerTests.obj
 0001:00024710       ??__F?_System_object@?$_Error_objects@H@std@@2V_System_error_category@2@A@@YAXXZ 10025710 f   moc_ORFMarkerTests.obj
 0001:00024720       ??__FService_DNAExport@U2@@YAXXZ 10025720 f   moc_ORFMarkerTests.obj
 0001:00024730       ??__FService_DNAGraphPack@U2@@YAXXZ 10025730 f   moc_ORFMarkerTests.obj
 0001:00024740       ??__FService_ExternalToolSupport@U2@@YAXXZ 10025740 f   moc_ORFMarkerTests.obj
 0001:00024750       ??__FService_GUITesting@U2@@YAXXZ 10025750 f   moc_ORFMarkerTests.obj
 0001:00024760       ??__FService_MaxCoreServiceId@U2@@YAXXZ 10025760 f   moc_ORFMarkerTests.obj
 0001:00024770       ??__FService_MinCoreServiceId@U2@@YAXXZ 10025770 f   moc_ORFMarkerTests.obj
 0001:00024780       ??__FService_PluginViewer@U2@@YAXXZ 10025780 f   moc_ORFMarkerTests.obj
 0001:00024790       ??__FService_Project@U2@@YAXXZ 10025790 f   moc_ORFMarkerTests.obj
 0001:000247a0       ??__FService_ProjectView@U2@@YAXXZ 100257a0 f   moc_ORFMarkerTests.obj
 0001:000247b0       ??__FService_QueryDesigner@U2@@YAXXZ 100257b0 f   moc_ORFMarkerTests.obj
 0001:000247c0       ??__FService_ScriptRegistry@U2@@YAXXZ 100257c0 f   moc_ORFMarkerTests.obj
 0001:000247d0       ??__FService_TestRunner@U2@@YAXXZ 100257d0 f   moc_ORFMarkerTests.obj
 0001:000247e0       ??__FService_WorkflowDesigner@U2@@YAXXZ 100257e0 f   moc_ORFMarkerTests.obj
 0001:000247f0       ??__FalgoLog@U2@@YAXXZ     100257f0 f   moc_ORFMarkerTests.obj
 0001:00024800       ??__FcmdLog@U2@@YAXXZ      10025800 f   moc_ORFMarkerTests.obj
 0001:00024810       ??__FcoreLog@U2@@YAXXZ     10025810 f   moc_ORFMarkerTests.obj
 0001:00024820       ??__FioLog@U2@@YAXXZ       10025820 f   moc_ORFMarkerTests.obj
 0001:00024830       ??__FperfLog@U2@@YAXXZ     10025830 f   moc_ORFMarkerTests.obj
 0001:00024840       ??__FscriptLog@U2@@YAXXZ   10025840 f   moc_ORFMarkerTests.obj
 0001:00024850       ??__FtaskLog@U2@@YAXXZ     10025850 f   moc_ORFMarkerTests.obj
 0001:00024860       ??__FuiLog@U2@@YAXXZ       10025860 f   moc_ORFMarkerTests.obj
 0001:00024870       ??__FuserActLog@U2@@YAXXZ  10025870 f   moc_ORFMarkerTests.obj
 0001:00024880       ??__F?_Generic_object@?$_Error_objects@H@std@@2V_Generic_error_category@2@A@@YAXXZ 10025880 f   moc_ORFQuery.obj
 0001:00024890       ??__F?_Iostream_object@?$_Error_objects@H@std@@2V_Iostream_error_category@2@A@@YAXXZ 10025890 f   moc_ORFQuery.obj
 0001:000248a0       ??__F?_System_object@?$_Error_objects@H@std@@2V_System_error_category@2@A@@YAXXZ 100258a0 f   moc_ORFQuery.obj
 0001:000248b0       ??__FalgoLog@U2@@YAXXZ     100258b0 f   moc_ORFQuery.obj
 0001:000248c0       ??__FcmdLog@U2@@YAXXZ      100258c0 f   moc_ORFQuery.obj
 0001:000248d0       ??__FcoreLog@U2@@YAXXZ     100258d0 f   moc_ORFQuery.obj
 0001:000248e0       ??__FioLog@U2@@YAXXZ       100258e0 f   moc_ORFQuery.obj
 0001:000248f0       ??__FperfLog@U2@@YAXXZ     100258f0 f   moc_ORFQuery.obj
 0001:00024900       ??__FscriptLog@U2@@YAXXZ   10025900 f   moc_ORFQuery.obj
 0001:00024910       ??__FtaskLog@U2@@YAXXZ     10025910 f   moc_ORFQuery.obj
 0001:00024920       ??__FuiLog@U2@@YAXXZ       10025920 f   moc_ORFQuery.obj
 0001:00024930       ??__FuserActLog@U2@@YAXXZ  10025930 f   moc_ORFQuery.obj
 0001:00024940       ??__F?_Generic_object@?$_Error_objects@H@std@@2V_Generic_error_category@2@A@@YAXXZ 10025940 f   moc_ORFWorker.obj
 0001:00024950       ??__F?_Iostream_object@?$_Error_objects@H@std@@2V_Iostream_error_category@2@A@@YAXXZ 10025950 f   moc_ORFWorker.obj
 0001:00024960       ??__F?_System_object@?$_Error_objects@H@std@@2V_System_error_category@2@A@@YAXXZ 10025960 f   moc_ORFWorker.obj
 0001:00024970       ??__FalgoLog@U2@@YAXXZ     10025970 f   moc_ORFWorker.obj
 0001:00024980       ??__FcmdLog@U2@@YAXXZ      10025980 f   moc_ORFWorker.obj
 0001:00024990       ??__FcoreLog@U2@@YAXXZ     10025990 f   moc_ORFWorker.obj
 0001:000249a0       ??__FioLog@U2@@YAXXZ       100259a0 f   moc_ORFWorker.obj
 0001:000249b0       ??__FperfLog@U2@@YAXXZ     100259b0 f   moc_ORFWorker.obj
 0001:000249c0       ??__FscriptLog@U2@@YAXXZ   100259c0 f   moc_ORFWorker.obj
 0001:000249d0       ??__FtaskLog@U2@@YAXXZ     100259d0 f   moc_ORFWorker.obj
 0001:000249e0       ??__FuiLog@U2@@YAXXZ       100259e0 f   moc_ORFWorker.obj
 0001:000249f0       ??__FuserActLog@U2@@YAXXZ  100259f0 f   moc_ORFWorker.obj
 0001:00024a00       ??__Fdummy@?A0xaf06a44c@@YAXXZ 10025a00 f   qrc_orf_marker.obj
 0002:00001074       _algoLog$initializer$      10027074     ORFDialog.obj
 0002:00001078       _cmdLog$initializer$       10027078     ORFDialog.obj
 0002:0000107c       _coreLog$initializer$      1002707c     ORFDialog.obj
 0002:00001080       _ioLog$initializer$        10027080     ORFDialog.obj
 0002:00001084       _perfLog$initializer$      10027084     ORFDialog.obj
 0002:00001088       _scriptLog$initializer$    10027088     ORFDialog.obj
 0002:0000108c       _taskLog$initializer$      1002708c     ORFDialog.obj
 0002:00001090       _uiLog$initializer$        10027090     ORFDialog.obj
 0002:00001094       _userActLog$initializer$   10027094     ORFDialog.obj
 0002:00001098       _Service_PluginViewer$initializer$ 10027098     ORFDialog.obj
 0002:0000109c       _Service_Project$initializer$ 1002709c     ORFDialog.obj
 0002:000010a0       _Service_ProjectView$initializer$ 100270a0     ORFDialog.obj
 0002:000010a4       _Service_DNAGraphPack$initializer$ 100270a4     ORFDialog.obj
 0002:000010a8       _Service_DNAExport$initializer$ 100270a8     ORFDialog.obj
 0002:000010ac       _Service_TestRunner$initializer$ 100270ac     ORFDialog.obj
 0002:000010b0       _Service_ScriptRegistry$initializer$ 100270b0     ORFDialog.obj
 0002:000010b4       _Service_ExternalToolSupport$initializer$ 100270b4     ORFDialog.obj
 0002:000010b8       _Service_GUITesting$initializer$ 100270b8     ORFDialog.obj
 0002:000010bc       _Service_WorkflowDesigner$initializer$ 100270bc     ORFDialog.obj
 0002:000010c0       _Service_QueryDesigner$initializer$ 100270c0     ORFDialog.obj
 0002:000010c4       _Service_MinCoreServiceId$initializer$ 100270c4     ORFDialog.obj
 0002:000010c8       _Service_MaxCoreServiceId$initializer$ 100270c8     ORFDialog.obj
 0002:000010cc       ?_Generic_object$initializer$@?$_Error_objects@H@std@@2P6AXXZA 100270cc     ORFDialog.obj
 0002:000010d0       ?_Iostream_object$initializer$@?$_Error_objects@H@std@@2P6AXXZA 100270d0     ORFDialog.obj
 0002:000010d4       ?_System_object$initializer$@?$_Error_objects@H@std@@2P6AXXZA 100270d4     ORFDialog.obj
 0002:000010d8       _algoLog$initializer$      100270d8     ORFMarkerPlugin.obj
 0002:000010dc       _cmdLog$initializer$       100270dc     ORFMarkerPlugin.obj
 0002:000010e0       _coreLog$initializer$      100270e0     ORFMarkerPlugin.obj
 0002:000010e4       _ioLog$initializer$        100270e4     ORFMarkerPlugin.obj
 0002:000010e8       _perfLog$initializer$      100270e8     ORFMarkerPlugin.obj
 0002:000010ec       _scriptLog$initializer$    100270ec     ORFMarkerPlugin.obj
 0002:000010f0       _taskLog$initializer$      100270f0     ORFMarkerPlugin.obj
 0002:000010f4       _uiLog$initializer$        100270f4     ORFMarkerPlugin.obj
 0002:000010f8       _userActLog$initializer$   100270f8     ORFMarkerPlugin.obj
 0002:000010fc       _Service_PluginViewer$initializer$ 100270fc     ORFMarkerPlugin.obj
 0002:00001100       _Service_Project$initializer$ 10027100     ORFMarkerPlugin.obj
 0002:00001104       _Service_ProjectView$initializer$ 10027104     ORFMarkerPlugin.obj
 0002:00001108       _Service_DNAGraphPack$initializer$ 10027108     ORFMarkerPlugin.obj
 0002:0000110c       _Service_DNAExport$initializer$ 1002710c     ORFMarkerPlugin.obj
 0002:00001110       _Service_TestRunner$initializer$ 10027110     ORFMarkerPlugin.obj
 0002:00001114       _Service_ScriptRegistry$initializer$ 10027114     ORFMarkerPlugin.obj
 0002:00001118       _Service_ExternalToolSupport$initializer$ 10027118     ORFMarkerPlugin.obj
 0002:0000111c       _Service_GUITesting$initializer$ 1002711c     ORFMarkerPlugin.obj
 0002:00001120       _Service_WorkflowDesigner$initializer$ 10027120     ORFMarkerPlugin.obj
 0002:00001124       _Service_QueryDesigner$initializer$ 10027124     ORFMarkerPlugin.obj
 0002:00001128       _Service_MinCoreServiceId$initializer$ 10027128     ORFMarkerPlugin.obj
 0002:0000112c       _Service_MaxCoreServiceId$initializer$ 1002712c     ORFMarkerPlugin.obj
 0002:00001130       _algoLog$initializer$      10027130     ORFMarkerTask.obj
 0002:00001134       _cmdLog$initializer$       10027134     ORFMarkerTask.obj
 0002:00001138       _coreLog$initializer$      10027138     ORFMarkerTask.obj
 0002:0000113c       _ioLog$initializer$        1002713c     ORFMarkerTask.obj
 0002:00001140       _perfLog$initializer$      10027140     ORFMarkerTask.obj
 0002:00001144       _scriptLog$initializer$    10027144     ORFMarkerTask.obj
 0002:00001148       _taskLog$initializer$      10027148     ORFMarkerTask.obj
 0002:0000114c       _uiLog$initializer$        1002714c     ORFMarkerTask.obj
 0002:00001150       _userActLog$initializer$   10027150     ORFMarkerTask.obj
 0002:00001154       ?STRAND$initializer$@ORFSettingsKeys@U2@@2P6AXXZA 10027154     ORFMarkerTask.obj
 0002:00001158       ?ALLOW_ALT_START$initializer$@ORFSettingsKeys@U2@@2P6AXXZA 10027158     ORFMarkerTask.obj
 0002:0000115c       ?ALLOW_OVERLAP$initializer$@ORFSettingsKeys@U2@@2P6AXXZA 1002715c     ORFMarkerTask.obj
 0002:00001160       ?AMINO_TRANSL$initializer$@ORFSettingsKeys@U2@@2P6AXXZA 10027160     ORFMarkerTask.obj
 0002:00001164       ?MIN_LEN$initializer$@ORFSettingsKeys@U2@@2P6AXXZA 10027164     ORFMarkerTask.obj
 0002:00001168       ?MUST_FIT$initializer$@ORFSettingsKeys@U2@@2P6AXXZA 10027168     ORFMarkerTask.obj
 0002:0000116c       ?MUST_INIT$initializer$@ORFSettingsKeys@U2@@2P6AXXZA 1002716c     ORFMarkerTask.obj
 0002:00001170       ?SEARCH_REGION$initializer$@ORFSettingsKeys@U2@@2P6AXXZA 10027170     ORFMarkerTask.obj
 0002:00001174       ?INCLUDE_STOP_CODON$initializer$@ORFSettingsKeys@U2@@2P6AXXZA 10027174     ORFMarkerTask.obj
 0002:00001178       ?MAX_RESULT$initializer$@ORFSettingsKeys@U2@@2P6AXXZA 10027178     ORFMarkerTask.obj
 0002:0000117c       ?IS_RESULT_LIMITED$initializer$@ORFSettingsKeys@U2@@2P6AXXZA 1002717c     ORFMarkerTask.obj
 0002:00001180       _algoLog$initializer$      10027180     ORFMarkerTests.obj
 0002:00001184       _cmdLog$initializer$       10027184     ORFMarkerTests.obj
 0002:00001188       _coreLog$initializer$      10027188     ORFMarkerTests.obj
 0002:0000118c       _ioLog$initializer$        1002718c     ORFMarkerTests.obj
 0002:00001190       _perfLog$initializer$      10027190     ORFMarkerTests.obj
 0002:00001194       _scriptLog$initializer$    10027194     ORFMarkerTests.obj
 0002:00001198       _taskLog$initializer$      10027198     ORFMarkerTests.obj
 0002:0000119c       _uiLog$initializer$        1002719c     ORFMarkerTests.obj
 0002:000011a0       _userActLog$initializer$   100271a0     ORFMarkerTests.obj
 0002:000011a4       _Service_PluginViewer$initializer$ 100271a4     ORFMarkerTests.obj
 0002:000011a8       _Service_Project$initializer$ 100271a8     ORFMarkerTests.obj
 0002:000011ac       _Service_ProjectView$initializer$ 100271ac     ORFMarkerTests.obj
 0002:000011b0       _Service_DNAGraphPack$initializer$ 100271b0     ORFMarkerTests.obj
 0002:000011b4       _Service_DNAExport$initializer$ 100271b4     ORFMarkerTests.obj
 0002:000011b8       _Service_TestRunner$initializer$ 100271b8     ORFMarkerTests.obj
 0002:000011bc       _Service_ScriptRegistry$initializer$ 100271bc     ORFMarkerTests.obj
 0002:000011c0       _Service_ExternalToolSupport$initializer$ 100271c0     ORFMarkerTests.obj
 0002:000011c4       _Service_GUITesting$initializer$ 100271c4     ORFMarkerTests.obj
 0002:000011c8       _Service_WorkflowDesigner$initializer$ 100271c8     ORFMarkerTests.obj
 0002:000011cc       _Service_QueryDesigner$initializer$ 100271cc     ORFMarkerTests.obj
 0002:000011d0       _Service_MinCoreServiceId$initializer$ 100271d0     ORFMarkerTests.obj
 0002:000011d4       _Service_MaxCoreServiceId$initializer$ 100271d4     ORFMarkerTests.obj
 0002:000011d8       _algoLog$initializer$      100271d8     ORFQuery.obj
 0002:000011dc       _cmdLog$initializer$       100271dc     ORFQuery.obj
 0002:000011e0       _coreLog$initializer$      100271e0     ORFQuery.obj
 0002:000011e4       _ioLog$initializer$        100271e4     ORFQuery.obj
 0002:000011e8       _perfLog$initializer$      100271e8     ORFQuery.obj
 0002:000011ec       _scriptLog$initializer$    100271ec     ORFQuery.obj
 0002:000011f0       _taskLog$initializer$      100271f0     ORFQuery.obj
 0002:000011f4       _uiLog$initializer$        100271f4     ORFQuery.obj
 0002:000011f8       _userActLog$initializer$   100271f8     ORFQuery.obj
 0002:000011fc       _ID_ATTR$initializer$      100271fc     ORFQuery.obj
 0002:00001200       _LEN_ATTR$initializer$     10027200     ORFQuery.obj
 0002:00001204       _INIT_ATTR$initializer$    10027204     ORFQuery.obj
 0002:00001208       _FIT_ATTR$initializer$     10027208     ORFQuery.obj
 0002:0000120c       _ALT_ATTR$initializer$     1002720c     ORFQuery.obj
 0002:00001210       _MAX_LENGTH_ATTR$initializer$ 10027210     ORFQuery.obj
 0002:00001214       _RES_ATTR$initializer$     10027214     ORFQuery.obj
 0002:00001218       _LIMIT_ATTR$initializer$   10027218     ORFQuery.obj
 0002:0000121c       _algoLog$initializer$      1002721c     ORFWorker.obj
 0002:00001220       _cmdLog$initializer$       10027220     ORFWorker.obj
 0002:00001224       _coreLog$initializer$      10027224     ORFWorker.obj
 0002:00001228       _ioLog$initializer$        10027228     ORFWorker.obj
 0002:0000122c       _perfLog$initializer$      1002722c     ORFWorker.obj
 0002:00001230       _scriptLog$initializer$    10027230     ORFWorker.obj
 0002:00001234       _taskLog$initializer$      10027234     ORFWorker.obj
 0002:00001238       _uiLog$initializer$        10027238     ORFWorker.obj
 0002:0000123c       _userActLog$initializer$   1002723c     ORFWorker.obj
 0002:00001240       _NAME_ATTR$initializer$    10027240     ORFWorker.obj
 0002:00001244       _ID_ATTR$initializer$      10027244     ORFWorker.obj
 0002:00001248       _LEN_ATTR$initializer$     10027248     ORFWorker.obj
 0002:0000124c       _FIT_ATTR$initializer$     1002724c     ORFWorker.obj
 0002:00001250       _INIT_ATTR$initializer$    10027250     ORFWorker.obj
 0002:00001254       _ALT_ATTR$initializer$     10027254     ORFWorker.obj
 0002:00001258       _ISC_ATTR$initializer$     10027258     ORFWorker.obj
 0002:0000125c       _RES_ATTR$initializer$     1002725c     ORFWorker.obj
 0002:00001260       _LIMIT_ATTR$initializer$   10027260     ORFWorker.obj
 0002:00001264       ?ACTOR_ID$initializer$@ORFWorkerFactory@LocalWorkflow@U2@@2P6AXXZA 10027264     ORFWorker.obj
 0002:00001268       _algoLog$initializer$      10027268     moc_ORFDialog.obj
 0002:0000126c       _cmdLog$initializer$       1002726c     moc_ORFDialog.obj
 0002:00001270       _coreLog$initializer$      10027270     moc_ORFDialog.obj
 0002:00001274       _ioLog$initializer$        10027274     moc_ORFDialog.obj
 0002:00001278       _perfLog$initializer$      10027278     moc_ORFDialog.obj
 0002:0000127c       _scriptLog$initializer$    1002727c     moc_ORFDialog.obj
 0002:00001280       _taskLog$initializer$      10027280     moc_ORFDialog.obj
 0002:00001284       _uiLog$initializer$        10027284     moc_ORFDialog.obj
 0002:00001288       _userActLog$initializer$   10027288     moc_ORFDialog.obj
 0002:0000128c       ?staticMetaObject$initializer$@ORFDialog@U2@@2P6AXXZA 1002728c     moc_ORFDialog.obj
 0002:00001290       _Service_PluginViewer$initializer$ 10027290     moc_ORFMarkerPlugin.obj
 0002:00001294       _Service_Project$initializer$ 10027294     moc_ORFMarkerPlugin.obj
 0002:00001298       _Service_ProjectView$initializer$ 10027298     moc_ORFMarkerPlugin.obj
 0002:0000129c       _Service_DNAGraphPack$initializer$ 1002729c     moc_ORFMarkerPlugin.obj
 0002:000012a0       _Service_DNAExport$initializer$ 100272a0     moc_ORFMarkerPlugin.obj
 0002:000012a4       _Service_TestRunner$initializer$ 100272a4     moc_ORFMarkerPlugin.obj
 0002:000012a8       _Service_ScriptRegistry$initializer$ 100272a8     moc_ORFMarkerPlugin.obj
 0002:000012ac       _Service_ExternalToolSupport$initializer$ 100272ac     moc_ORFMarkerPlugin.obj
 0002:000012b0       _Service_GUITesting$initializer$ 100272b0     moc_ORFMarkerPlugin.obj
 0002:000012b4       _Service_WorkflowDesigner$initializer$ 100272b4     moc_ORFMarkerPlugin.obj
 0002:000012b8       _Service_QueryDesigner$initializer$ 100272b8     moc_ORFMarkerPlugin.obj
 0002:000012bc       _Service_MinCoreServiceId$initializer$ 100272bc     moc_ORFMarkerPlugin.obj
 0002:000012c0       _Service_MaxCoreServiceId$initializer$ 100272c0     moc_ORFMarkerPlugin.obj
 0002:000012c4       ?staticMetaObject$initializer$@ORFMarkerPlugin@U2@@2P6AXXZA 100272c4     moc_ORFMarkerPlugin.obj
 0002:000012c8       ?staticMetaObject$initializer$@ORFViewContext@U2@@2P6AXXZA 100272c8     moc_ORFMarkerPlugin.obj
 0002:000012cc       _algoLog$initializer$      100272cc     moc_ORFMarkerTask.obj
 0002:000012d0       _cmdLog$initializer$       100272d0     moc_ORFMarkerTask.obj
 0002:000012d4       _coreLog$initializer$      100272d4     moc_ORFMarkerTask.obj
 0002:000012d8       _ioLog$initializer$        100272d8     moc_ORFMarkerTask.obj
 0002:000012dc       _perfLog$initializer$      100272dc     moc_ORFMarkerTask.obj
 0002:000012e0       _scriptLog$initializer$    100272e0     moc_ORFMarkerTask.obj
 0002:000012e4       _taskLog$initializer$      100272e4     moc_ORFMarkerTask.obj
 0002:000012e8       _uiLog$initializer$        100272e8     moc_ORFMarkerTask.obj
 0002:000012ec       _userActLog$initializer$   100272ec     moc_ORFMarkerTask.obj
 0002:000012f0       ?staticMetaObject$initializer$@FindORFsToAnnotationsTask@U2@@2P6AXXZA 100272f0     moc_ORFMarkerTask.obj
 0002:000012f4       ?staticMetaObject$initializer$@ORFAutoAnnotationsUpdater@U2@@2P6AXXZA 100272f4     moc_ORFMarkerTask.obj
 0002:000012f8       _algoLog$initializer$      100272f8     moc_ORFMarkerTests.obj
 0002:000012fc       _cmdLog$initializer$       100272fc     moc_ORFMarkerTests.obj
 0002:00001300       _coreLog$initializer$      10027300     moc_ORFMarkerTests.obj
 0002:00001304       _ioLog$initializer$        10027304     moc_ORFMarkerTests.obj
 0002:00001308       _perfLog$initializer$      10027308     moc_ORFMarkerTests.obj
 0002:0000130c       _scriptLog$initializer$    1002730c     moc_ORFMarkerTests.obj
 0002:00001310       _taskLog$initializer$      10027310     moc_ORFMarkerTests.obj
 0002:00001314       _uiLog$initializer$        10027314     moc_ORFMarkerTests.obj
 0002:00001318       _userActLog$initializer$   10027318     moc_ORFMarkerTests.obj
 0002:0000131c       _Service_PluginViewer$initializer$ 1002731c     moc_ORFMarkerTests.obj
 0002:00001320       _Service_Project$initializer$ 10027320     moc_ORFMarkerTests.obj
 0002:00001324       _Service_ProjectView$initializer$ 10027324     moc_ORFMarkerTests.obj
 0002:00001328       _Service_DNAGraphPack$initializer$ 10027328     moc_ORFMarkerTests.obj
 0002:0000132c       _Service_DNAExport$initializer$ 1002732c     moc_ORFMarkerTests.obj
 0002:00001330       _Service_TestRunner$initializer$ 10027330     moc_ORFMarkerTests.obj
 0002:00001334       _Service_ScriptRegistry$initializer$ 10027334     moc_ORFMarkerTests.obj
 0002:00001338       _Service_ExternalToolSupport$initializer$ 10027338     moc_ORFMarkerTests.obj
 0002:0000133c       _Service_GUITesting$initializer$ 1002733c     moc_ORFMarkerTests.obj
 0002:00001340       _Service_WorkflowDesigner$initializer$ 10027340     moc_ORFMarkerTests.obj
 0002:00001344       _Service_QueryDesigner$initializer$ 10027344     moc_ORFMarkerTests.obj
 0002:00001348       _Service_MinCoreServiceId$initializer$ 10027348     moc_ORFMarkerTests.obj
 0002:0000134c       _Service_MaxCoreServiceId$initializer$ 1002734c     moc_ORFMarkerTests.obj
 0002:00001350       ?staticMetaObject$initializer$@GTest_ORFMarkerTask@U2@@2P6AXXZA 10027350     moc_ORFMarkerTests.obj
 0002:00001354       _algoLog$initializer$      10027354     moc_ORFQuery.obj
 0002:00001358       _cmdLog$initializer$       10027358     moc_ORFQuery.obj
 0002:0000135c       _coreLog$initializer$      1002735c     moc_ORFQuery.obj
 0002:00001360       _ioLog$initializer$        10027360     moc_ORFQuery.obj
 0002:00001364       _perfLog$initializer$      10027364     moc_ORFQuery.obj
 0002:00001368       _scriptLog$initializer$    10027368     moc_ORFQuery.obj
 0002:0000136c       _taskLog$initializer$      1002736c     moc_ORFQuery.obj
 0002:00001370       _uiLog$initializer$        10027370     moc_ORFQuery.obj
 0002:00001374       _userActLog$initializer$   10027374     moc_ORFQuery.obj
 0002:00001378       ?staticMetaObject$initializer$@QDORFActor@U2@@2P6AXXZA 10027378     moc_ORFQuery.obj
 0002:0000137c       _algoLog$initializer$      1002737c     moc_ORFWorker.obj
 0002:00001380       _cmdLog$initializer$       10027380     moc_ORFWorker.obj
 0002:00001384       _coreLog$initializer$      10027384     moc_ORFWorker.obj
 0002:00001388       _ioLog$initializer$        10027388     moc_ORFWorker.obj
 0002:0000138c       _perfLog$initializer$      1002738c     moc_ORFWorker.obj
 0002:00001390       _scriptLog$initializer$    10027390     moc_ORFWorker.obj
 0002:00001394       _taskLog$initializer$      10027394     moc_ORFWorker.obj
 0002:00001398       _uiLog$initializer$        10027398     moc_ORFWorker.obj
 0002:0000139c       _userActLog$initializer$   1002739c     moc_ORFWorker.obj
 0002:000013a0       ?staticMetaObject$initializer$@ORFPrompter@LocalWorkflow@U2@@2P6AXXZA 100273a0     moc_ORFWorker.obj
 0002:000013a4       ?staticMetaObject$initializer$@ORFWorker@LocalWorkflow@U2@@2P6AXXZA 100273a4     moc_ORFWorker.obj
 0002:000013a8       _dummy$initializer$        100273a8     qrc_orf_marker.obj
 0002:000013b4       _pcinit                    100273b4     MSVCRT:crtdll.obj
 0002:000013b8       _pinit                     100273b8     MSVCRT:atonexit.obj
 0002:00002880       ?qstring_literal@?6???R<lambda_a9859d689698127f97835ff63b5de490>@@QBE?AVQString@@XZ@4U?$QStaticStringData@$0N@@@B 10028880     ORFDialog.obj
 0002:000028ac       ?qstring_literal@?7???R<lambda_e114dfc637b50f53a12623c298138117>@@QBE?AVQString@@XZ@4U?$QStaticStringData@$0BA@@@B 100288ac     ORFDialog.obj
 0002:000028e0       ?qstring_literal@?8???R<lambda_f746202d42af9037ea860442f08e949b>@@QBE?AVQString@@XZ@4U?$QStaticStringData@$08@@B 100288e0     ORFDialog.obj
 0002:00002904       ?qstring_literal@?9???R<lambda_ea7e40f3c293bc0745c9796f572004af>@@QBE?AVQString@@XZ@4U?$QStaticStringData@$04@@B 10028904     ORFDialog.obj
 0002:00002920       ?qstring_literal@?L@???R<lambda_4655343fe23bb4b3b7882e1f3316a452>@@QBE?AVQString@@XZ@4U?$QStaticStringData@$0BA@@@B 10028920     ORFDialog.obj
 0002:00002954       ?qstring_literal@?M@???R<lambda_81b46f5ffcbd23e97e4414d4b5d9aa96>@@QBE?AVQString@@XZ@4U?$QStaticStringData@$09@@B 10028954     ORFDialog.obj
 0002:0000297c       ?qstring_literal@?N@???R<lambda_0ff5d552fbbf7817874d60f1df8acf29>@@QBE?AVQString@@XZ@4U?$QStaticStringData@$0BC@@@B 1002897c     ORFDialog.obj
 0002:000029b4       ?qstring_literal@?O@???R<lambda_ca85f9d6613aef30f18329a26b64b6d3>@@QBE?AVQString@@XZ@4U?$QStaticStringData@$07@@B 100289b4     ORFDialog.obj
 0002:000029d8       ?qstring_literal@?P@???R<lambda_cb8147e3c8b49d91b9201acf92d06490>@@QBE?AVQString@@XZ@4U?$QStaticStringData@$0O@@@B 100289d8     ORFDialog.obj
 0002:00002a08       ?qstring_literal@?BA@???R<lambda_9f8f56f1a1953070dc5e6b8678d8115f>@@QBE?AVQString@@XZ@4U?$QStaticStringData@$05@@B 10028a08     ORFDialog.obj
 0002:00002a28       ?qstring_literal@?BB@???R<lambda_d9d5d6d4341da3ae04a63bbef4f4d8fd>@@QBE?AVQString@@XZ@4U?$QStaticStringData@$07@@B 10028a28     ORFDialog.obj
 0002:00002a4c       ?qstring_literal@?BC@???R<lambda_44e65958acee4170841d4644da5d91a6>@@QBE?AVQString@@XZ@4U?$QStaticStringData@$0M@@@B 10028a4c     ORFDialog.obj
 0002:00002a78       ?qstring_literal@?BD@???R<lambda_7a879637595ff6229c926fc23ea90814>@@QBE?AVQString@@XZ@4U?$QStaticStringData@$07@@B 10028a78     ORFDialog.obj
 0002:00002a9c       ?qstring_literal@?BE@???R<lambda_f4b85fea6c6cf4d9c35c782cf8237f89>@@QBE?AVQString@@XZ@4U?$QStaticStringData@$0BA@@@B 10028a9c     ORFDialog.obj
 0002:00002ad0       ?qstring_literal@?BF@???R<lambda_0a0e7f32f0abf4fe998f0c4219dad45a>@@QBE?AVQString@@XZ@4U?$QStaticStringData@$0BA@@@B 10028ad0     ORFDialog.obj
 0002:00002b04       ?qstring_literal@?BG@???R<lambda_3bd8f2f42d9c55363ea1b95aa573d950>@@QBE?AVQString@@XZ@4U?$QStaticStringData@$07@@B 10028b04     ORFDialog.obj
 0002:00002b28       ?qstring_literal@?BH@???R<lambda_341cb0a24dbb67dcf78c26228121c09a>@@QBE?AVQString@@XZ@4U?$QStaticStringData@$07@@B 10028b28     ORFDialog.obj
 0002:00002b4c       ?qstring_literal@?BI@???R<lambda_c5b2208d484aab5eeda4b4e8d9e81a71>@@QBE?AVQString@@XZ@4U?$QStaticStringData@$04@@B 10028b4c     ORFDialog.obj
 0002:00002b68       ?qstring_literal@?BJ@???R<lambda_cd7c1f4a134beb52c9cbdd3b6ce610db>@@QBE?AVQString@@XZ@4U?$QStaticStringData@$05@@B 10028b68     ORFDialog.obj
 0002:00002b88       ?qstring_literal@?BK@???R<lambda_6cda75d66740ac343a5306b8d47f27c7>@@QBE?AVQString@@XZ@4U?$QStaticStringData@$08@@B 10028b88     ORFDialog.obj
 0002:00002bac       ?qstring_literal@?BL@???R<lambda_220f8f8c5ecf4ac023635268940e37e3>@@QBE?AVQString@@XZ@4U?$QStaticStringData@$04@@B 10028bac     ORFDialog.obj
 0002:00002bc8       ?qstring_literal@?BM@???R<lambda_cf8fd9af3f824ea42de5b8d51851b3e7>@@QBE?AVQString@@XZ@4U?$QStaticStringData@$0O@@@B 10028bc8     ORFDialog.obj
 0002:00002bf8       ?qstring_literal@?BN@???R<lambda_95d7ce4a46ac2420c3ef42b00d6e46c6>@@QBE?AVQString@@XZ@4U?$QStaticStringData@$0BC@@@B 10028bf8     ORFDialog.obj
 0002:00002c30       ?qstring_literal@?BO@???R<lambda_e718f0b57f7aaf937d0d3b715c431104>@@QBE?AVQString@@XZ@4U?$QStaticStringData@$08@@B 10028c30     ORFDialog.obj
 0002:00002c54       ?qstring_literal@?BP@???R<lambda_1dd36e8e753f070291a4e308cf29c03c>@@QBE?AVQString@@XZ@4U?$QStaticStringData@$0O@@@B 10028c54     ORFDialog.obj
 0002:00002c84       ?qstring_literal@?CA@???R<lambda_6e91e825d1cfc04223738cd463f9b99e>@@QBE?AVQString@@XZ@4U?$QStaticStringData@$0BA@@@B 10028c84     ORFDialog.obj
 0002:00002cb8       ?qstring_literal@?CB@???R<lambda_46cc8f107b08cda0fe36f9525d4f10d7>@@QBE?AVQString@@XZ@4U?$QStaticStringData@$08@@B 10028cb8     ORFDialog.obj
 0002:00002cdc       ?qstring_literal@?CC@???R<lambda_c9ff954e0b34c3c8e5fae69c2fe05e0b>@@QBE?AVQString@@XZ@4U?$QStaticStringData@$0L@@@B 10028cdc     ORFDialog.obj
 0002:00002d04       ?qstring_literal@?CD@???R<lambda_bd58d910664159c2d4adc7a129b025ac>@@QBE?AVQString@@XZ@4U?$QStaticStringData@$09@@B 10028d04     ORFDialog.obj
 0002:00002d2c       ?qstring_literal@?CE@???R<lambda_6b04bc410d0484eb77773aabbb2121e7>@@QBE?AVQString@@XZ@4U?$QStaticStringData@$09@@B 10028d2c     ORFDialog.obj
 0002:00002d54       ?qstring_literal@?CF@???R<lambda_727dfb955ba445b1d6e1c6e761ef9880>@@QBE?AVQString@@XZ@4U?$QStaticStringData@$0BD@@@B 10028d54     ORFDialog.obj
 0002:00002d8c       ?qstring_literal@?CG@???R<lambda_e38c0bfbbb0434d86bd5f34b32af9382>@@QBE?AVQString@@XZ@4U?$QStaticStringData@$0L@@@B 10028d8c     ORFDialog.obj
 0002:00002db4       ?qstring_literal@?CH@???R<lambda_c934430d2d61852a3610e57fc7181a03>@@QBE?AVQString@@XZ@4U?$QStaticStringData@$04@@B 10028db4     ORFDialog.obj
 0002:00002dd0       ?qstring_literal@?CI@???R<lambda_633eb662894a0f52b681d98c902f4666>@@QBE?AVQString@@XZ@4U?$QStaticStringData@$0BA@@@B 10028dd0     ORFDialog.obj
 0002:00002e04       ?qstring_literal@?CJ@???R<lambda_52fe59cca71e9c144ba25b49fc880329>@@QBE?AVQString@@XZ@4U?$QStaticStringData@$0BB@@@B 10028e04     ORFDialog.obj
 0002:00002e38       ?qstring_literal@?CK@???R<lambda_d0d42478d3362983368102e03c7eeecb>@@QBE?AVQString@@XZ@4U?$QStaticStringData@$0BC@@@B 10028e38     ORFDialog.obj
 0002:00002e70       ?qstring_literal@?CL@???R<lambda_50b3e03a63dfd75480240ba88917e908>@@QBE?AVQString@@XZ@4U?$QStaticStringData@$0L@@@B 10028e70     ORFDialog.obj
 0002:00002e98       ?qstring_literal@?CM@???R<lambda_cb920ba896b73d37c549d63b6b5320cc>@@QBE?AVQString@@XZ@4U?$QStaticStringData@$08@@B 10028e98     ORFDialog.obj
 0002:00004fd0       _qt_meta_stringdata_U2__ORFDialog 1002afd0     moc_ORFDialog.obj
 0002:00005150       _qt_meta_data_U2__ORFDialog 1002b150     moc_ORFDialog.obj
 0002:00005278       _qt_meta_stringdata_U2__ORFMarkerPlugin 1002b278     moc_ORFMarkerPlugin.obj
 0002:0000529c       _qt_meta_data_U2__ORFMarkerPlugin 1002b29c     moc_ORFMarkerPlugin.obj
 0002:000052d8       _qt_meta_stringdata_U2__ORFViewContext 1002b2d8     moc_ORFMarkerPlugin.obj
 0002:00005330       _qt_meta_data_U2__ORFViewContext 1002b330     moc_ORFMarkerPlugin.obj
 0002:00005384       _qt_meta_stringdata_U2__FindORFsToAnnotationsTask 1002b384     moc_ORFMarkerTask.obj
 0002:000053b4       _qt_meta_data_U2__FindORFsToAnnotationsTask 1002b3b4     moc_ORFMarkerTask.obj
 0002:000053f0       _qt_meta_stringdata_U2__ORFAutoAnnotationsUpdater 1002b3f0     moc_ORFMarkerTask.obj
 0002:00005420       _qt_meta_data_U2__ORFAutoAnnotationsUpdater 1002b420     moc_ORFMarkerTask.obj
 0002:0000545c       _qt_meta_stringdata_U2__GTest_ORFMarkerTask 1002b45c     moc_ORFMarkerTests.obj
 0002:00005484       _qt_meta_data_U2__GTest_ORFMarkerTask 1002b484     moc_ORFMarkerTests.obj
 0002:000054c0       _qt_meta_stringdata_U2__QDORFActor 1002b4c0     moc_ORFQuery.obj
 0002:00005538       _qt_meta_data_U2__QDORFActor 1002b538     moc_ORFQuery.obj
 0002:00005598       _qt_meta_stringdata_U2__LocalWorkflow__ORFPrompter 1002b598     moc_ORFWorker.obj
 0002:000055c8       _qt_meta_data_U2__LocalWorkflow__ORFPrompter 1002b5c8     moc_ORFWorker.obj
 0002:00005608       _qt_meta_stringdata_U2__LocalWorkflow__ORFWorker 1002b608     moc_ORFWorker.obj
 0002:00005668       _qt_meta_data_U2__LocalWorkflow__ORFWorker 1002b668     moc_ORFWorker.obj
 0002:000056c0       _qt_resource_data          1002b6c0     qrc_orf_marker.obj
 0002:00005958       _qt_resource_name          1002b958     qrc_orf_marker.obj
 0002:000059a8       _qt_resource_struct        1002b9a8     qrc_orf_marker.obj
 0002:000059f0       _GS_ExceptionPointers      1002b9f0     MSVCRT:gs_report.obj
 0002:00007da8       __catchsym$?_Copy@?$basic_string@DU?$char_traits@D@std@@V?$allocator@D@2@@std@@QAEXII@Z$5 1002dda8     ORFDialog.obj
 0002:00007db8       __catchsym$?_Copy@?$basic_string@DU?$char_traits@D@std@@V?$allocator@D@2@@std@@QAEXII@Z$4 1002ddb8     ORFDialog.obj
 0002:00007dc8       __unwindtable$?_Copy@?$basic_string@DU?$char_traits@D@std@@V?$allocator@D@2@@std@@QAEXII@Z 1002ddc8     ORFDialog.obj
 0002:00007de8       __ehfuncinfo$?_Copy@?$basic_string@DU?$char_traits@D@std@@V?$allocator@D@2@@std@@QAEXII@Z 1002dde8     ORFDialog.obj
 0002:00007e0c       __tryblocktable$?_Copy@?$basic_string@DU?$char_traits@D@std@@V?$allocator@D@2@@std@@QAEXII@Z 1002de0c     ORFDialog.obj
 0002:00007e34       __unwindtable$??H@YA?BVQString@@ABV0@0@Z 1002de34     ORFDialog.obj
 0002:00007e3c       __ehfuncinfo$??H@YA?BVQString@@ABV0@0@Z 1002de3c     ORFDialog.obj
 0002:00007e60       __unwindtable$??H@YA?BVQString@@ABV0@PBD@Z 1002de60     ORFDialog.obj
 0002:00007e70       __ehfuncinfo$??H@YA?BVQString@@ABV0@PBD@Z 1002de70     ORFDialog.obj
 0002:00007e94       __unwindtable$??H@YA?BVQString@@PBDABV0@@Z 1002de94     ORFDialog.obj
 0002:00007e9c       __ehfuncinfo$??H@YA?BVQString@@PBDABV0@@Z 1002de9c     ORFDialog.obj
 0002:00007ec0       __ehfuncinfo$?setupUi@Ui_ORFDialogBase@@QAEXPAVQDialog@@@Z 1002dec0     ORFDialog.obj
 0002:00007ee4       __unwindtable$?setupUi@Ui_ORFDialogBase@@QAEXPAVQDialog@@@Z 1002dee4     ORFDialog.obj
 0002:0000815c       __ehfuncinfo$?retranslateUi@Ui_ORFDialogBase@@QAEXPAVQDialog@@@Z 1002e15c     ORFDialog.obj
 0002:00008180       __unwindtable$?retranslateUi@Ui_ORFDialogBase@@QAEXPAVQDialog@@@Z 1002e180     ORFDialog.obj
 0002:00008320       __unwindtable$??__EalgoLog@U2@@YAXXZ 1002e320     ORFDialog.obj
 0002:00008328       __ehfuncinfo$??__EalgoLog@U2@@YAXXZ 1002e328     ORFDialog.obj
 0002:0000834c       __unwindtable$??__EcmdLog@U2@@YAXXZ 1002e34c     ORFDialog.obj
 0002:00008354       __ehfuncinfo$??__EcmdLog@U2@@YAXXZ 1002e354     ORFDialog.obj
 0002:00008378       __unwindtable$??__EcoreLog@U2@@YAXXZ 1002e378     ORFDialog.obj
 0002:00008380       __ehfuncinfo$??__EcoreLog@U2@@YAXXZ 1002e380     ORFDialog.obj
 0002:000083a4       __unwindtable$??__EioLog@U2@@YAXXZ 1002e3a4     ORFDialog.obj
 0002:000083ac       __ehfuncinfo$??__EioLog@U2@@YAXXZ 1002e3ac     ORFDialog.obj
 0002:000083d0       __unwindtable$??__EperfLog@U2@@YAXXZ 1002e3d0     ORFDialog.obj
 0002:000083d8       __ehfuncinfo$??__EperfLog@U2@@YAXXZ 1002e3d8     ORFDialog.obj
 0002:000083fc       __unwindtable$??__EscriptLog@U2@@YAXXZ 1002e3fc     ORFDialog.obj
 0002:00008404       __ehfuncinfo$??__EscriptLog@U2@@YAXXZ 1002e404     ORFDialog.obj
 0002:00008428       __unwindtable$??__EtaskLog@U2@@YAXXZ 1002e428     ORFDialog.obj
 0002:00008430       __ehfuncinfo$??__EtaskLog@U2@@YAXXZ 1002e430     ORFDialog.obj
 0002:00008454       __unwindtable$??__EuiLog@U2@@YAXXZ 1002e454     ORFDialog.obj
 0002:0000845c       __ehfuncinfo$??__EuiLog@U2@@YAXXZ 1002e45c     ORFDialog.obj
 0002:00008480       __unwindtable$??__EuserActLog@U2@@YAXXZ 1002e480     ORFDialog.obj
 0002:00008488       __ehfuncinfo$??__EuserActLog@U2@@YAXXZ 1002e488     ORFDialog.obj
 0002:000084ac       __catchsym$??0?$QList@PAVTask@U2@@@@QAE@ABV0@@Z$2 1002e4ac     ORFDialog.obj
 0002:000084bc       __unwindtable$??0?$QList@PAVTask@U2@@@@QAE@ABV0@@Z 1002e4bc     ORFDialog.obj
 0002:000084cc       __tryblocktable$??0?$QList@PAVTask@U2@@@@QAE@ABV0@@Z 1002e4cc     ORFDialog.obj
 0002:000084e0       __ehfuncinfo$??0?$QList@PAVTask@U2@@@@QAE@ABV0@@Z 1002e4e0     ORFDialog.obj
 0002:00008504       __unwindtable$?clone@?$QSharedDataPointer@VAnnotationData@U2@@@@IAEPAVAnnotationData@U2@@XZ 1002e504     ORFDialog.obj
 0002:0000850c       __ehfuncinfo$?clone@?$QSharedDataPointer@VAnnotationData@U2@@@@IAEPAVAnnotationData@U2@@XZ 1002e50c     ORFDialog.obj
 0002:00008530       __unwindtable$?detach_helper@?$QSharedDataPointer@VAnnotationData@U2@@@@AAEXXZ 1002e530     ORFDialog.obj
 0002:00008538       __ehfuncinfo$?detach_helper@?$QSharedDataPointer@VAnnotationData@U2@@@@AAEXXZ 1002e538     ORFDialog.obj
 0002:0000855c       __catchsym$??0?$QList@VORFFindResult@U2@@@@QAE@ABV0@@Z$2 1002e55c     ORFDialog.obj
 0002:0000856c       __unwindtable$??0?$QList@VORFFindResult@U2@@@@QAE@ABV0@@Z 1002e56c     ORFDialog.obj
 0002:0000857c       __tryblocktable$??0?$QList@VORFFindResult@U2@@@@QAE@ABV0@@Z 1002e57c     ORFDialog.obj
 0002:00008590       __ehfuncinfo$??0?$QList@VORFFindResult@U2@@@@QAE@ABV0@@Z 1002e590     ORFDialog.obj
 0002:000085b4       __catchsym$?node_copy@?$QList@VORFFindResult@U2@@@@AAEXPAUNode@1@00@Z$4 1002e5b4     ORFDialog.obj
 0002:000085c4       __tryblocktable$?node_copy@?$QList@VORFFindResult@U2@@@@AAEXPAUNode@1@00@Z 1002e5c4     ORFDialog.obj
 0002:000085d8       __unwindtable$?node_copy@?$QList@VORFFindResult@U2@@@@AAEXPAUNode@1@00@Z 1002e5d8     ORFDialog.obj
 0002:000085f8       __ehfuncinfo$?node_copy@?$QList@VORFFindResult@U2@@@@AAEXPAUNode@1@00@Z 1002e5f8     ORFDialog.obj
 0002:0000861c       __ehfuncinfo$??0ORFDialog@U2@@QAE@PAVADVSequenceObjectContext@1@@Z 1002e61c     ORFDialog.obj
 0002:00008640       __unwindtable$??0ORFDialog@U2@@QAE@PAVADVSequenceObjectContext@1@@Z 1002e640     ORFDialog.obj
 0002:000086b0       __ehfuncinfo$?accept@ORFDialog@U2@@UAEXXZ 1002e6b0     ORFDialog.obj
 0002:000086d4       __unwindtable$?accept@ORFDialog@U2@@UAEXXZ 1002e6d4     ORFDialog.obj
 0002:000086fc       __unwindtable$?sl_onFindAll@ORFDialog@U2@@AAEXXZ 1002e6fc     ORFDialog.obj
 0002:0000870c       __ehfuncinfo$?sl_onFindAll@ORFDialog@U2@@AAEXXZ 1002e70c     ORFDialog.obj
 0002:00008730       __ehfuncinfo$?sl_translationChanged@ORFDialog@U2@@AAEXXZ 1002e730     ORFDialog.obj
 0002:00008754       __unwindtable$?sl_translationChanged@ORFDialog@U2@@AAEXXZ 1002e754     ORFDialog.obj
 0002:000088d4       __ehfuncinfo$?updateStatus@ORFDialog@U2@@AAEXXZ 1002e8d4     ORFDialog.obj
 0002:000088f8       __unwindtable$?updateStatus@ORFDialog@U2@@AAEXXZ 1002e8f8     ORFDialog.obj
 0002:00008920       __ehfuncinfo$?getSettings@ORFDialog@U2@@AAEXAAVORFAlgorithmSettings@2@@Z 1002e920     ORFDialog.obj
 0002:00008944       __unwindtable$?getSettings@ORFDialog@U2@@AAEXAAVORFAlgorithmSettings@2@@Z 1002e944     ORFDialog.obj
 0002:00008974       __unwindtable$?runTask@ORFDialog@U2@@AAEXXZ 1002e974     ORFDialog.obj
 0002:0000897c       __ehfuncinfo$?runTask@ORFDialog@U2@@AAEXXZ 1002e97c     ORFDialog.obj
 0002:000089a0       __unwindtable$?importResults@ORFDialog@U2@@AAEXXZ 1002e9a0     ORFDialog.obj
 0002:000089b8       __ehfuncinfo$?importResults@ORFDialog@U2@@AAEXXZ 1002e9b8     ORFDialog.obj
 0002:000089dc       __unwindtable$?createAnnotationWidget@ORFDialog@U2@@AAEXXZ 1002e9dc     ORFDialog.obj
 0002:000089fc       __ehfuncinfo$?createAnnotationWidget@ORFDialog@U2@@AAEXXZ 1002e9fc     ORFDialog.obj
 0002:00008a20       __ehfuncinfo$?findStartedAAUpdateTask@ORFDialog@U2@@AAEXXZ 1002ea20     ORFDialog.obj
 0002:00008a44       __unwindtable$?findStartedAAUpdateTask@ORFDialog@U2@@AAEXXZ 1002ea44     ORFDialog.obj
 0002:00008a84       __unwindtable$??A?$QMap@W4DNATranslationRole@U2@@V?$QList@UTriplet@U2@@@@@@QAEAAV?$QList@UTriplet@U2@@@@ABW4DNATranslationRole@U2@@@Z 1002ea84     ORFDialog.obj
 0002:00008a8c       __ehfuncinfo$??A?$QMap@W4DNATranslationRole@U2@@V?$QList@UTriplet@U2@@@@@@QAEAAV?$QList@UTriplet@U2@@@@ABW4DNATranslationRole@U2@@@Z 1002ea8c     ORFDialog.obj
 0002:00008ab0       __catchsym$??0?$QList@PAVQAction@@@@QAE@ABV0@@Z$2 1002eab0     ORFDialog.obj
 0002:00008ac0       __unwindtable$??0?$QList@PAVQAction@@@@QAE@ABV0@@Z 1002eac0     ORFDialog.obj
 0002:00008ad0       __tryblocktable$??0?$QList@PAVQAction@@@@QAE@ABV0@@Z 1002ead0     ORFDialog.obj
 0002:00008ae4       __ehfuncinfo$??0?$QList@PAVQAction@@@@QAE@ABV0@@Z 1002eae4     ORFDialog.obj
 0002:00008b08       __unwindtable$?qt_metatype_id@?$QMetaTypeId@PAVQAction@@@@SAHXZ 1002eb08     ORFDialog.obj
 0002:00008b10       __ehfuncinfo$?qt_metatype_id@?$QMetaTypeId@PAVQAction@@@@SAHXZ 1002eb10     ORFDialog.obj
 0002:00008b34       __unwindtable$??$qRegisterMetaType@PAVQAction@@@@YAHPBDPAPAVQAction@@W4DefinedType@?$MetaTypeDefinedHelper@PAVQAction@@$00@QtPrivate@@@Z 1002eb34     ORFDialog.obj
 0002:00008b3c       __ehfuncinfo$??$qRegisterMetaType@PAVQAction@@@@YAHPBDPAPAVQAction@@W4DefinedType@?$MetaTypeDefinedHelper@PAVQAction@@$00@QtPrivate@@@Z 1002eb3c     ORFDialog.obj
 0002:00008b60       __ehfuncinfo$??0ORFListItem@U2@@QAE@ABVORFFindResult@1@@Z 1002eb60     ORFDialog.obj
 0002:00008b84       __unwindtable$??0ORFListItem@U2@@QAE@ABVORFFindResult@1@@Z 1002eb84     ORFDialog.obj
 0002:00008c14       __unwindtable$??MORFListItem@U2@@UBE_NABVQTreeWidgetItem@@@Z 1002ec14     ORFDialog.obj
 0002:00008c24       __ehfuncinfo$??MORFListItem@U2@@UBE_NABVQTreeWidgetItem@@@Z 1002ec24     ORFDialog.obj
 0002:00008c48       __unwindtable$?triplet2str@U2@@YA?AVQString@@ABUTriplet@1@@Z 1002ec48     ORFDialog.obj
 0002:00008c50       __ehfuncinfo$?triplet2str@U2@@YA?AVQString@@ABUTriplet@1@@Z 1002ec50     ORFDialog.obj
 0002:00008c74       __catchsym$??0?$QList@UTriplet@U2@@@@QAE@ABV0@@Z$2 1002ec74     ORFDialog.obj
 0002:00008c84       __unwindtable$??0?$QList@UTriplet@U2@@@@QAE@ABV0@@Z 1002ec84     ORFDialog.obj
 0002:00008c94       __tryblocktable$??0?$QList@UTriplet@U2@@@@QAE@ABV0@@Z 1002ec94     ORFDialog.obj
 0002:00008ca8       __ehfuncinfo$??0?$QList@UTriplet@U2@@@@QAE@ABV0@@Z 1002eca8     ORFDialog.obj
 0002:00008ccc       __catchsym$?node_copy@?$QList@UTriplet@U2@@@@AAEXPAUNode@1@00@Z$4 1002eccc     ORFDialog.obj
 0002:00008cdc       __tryblocktable$?node_copy@?$QList@UTriplet@U2@@@@AAEXPAUNode@1@00@Z 1002ecdc     ORFDialog.obj
 0002:00008cf0       __unwindtable$?node_copy@?$QList@UTriplet@U2@@@@AAEXPAUNode@1@00@Z 1002ecf0     ORFDialog.obj
 0002:00008d10       __ehfuncinfo$?node_copy@?$QList@UTriplet@U2@@@@AAEXPAUNode@1@00@Z 1002ed10     ORFDialog.obj
 0002:00008d34       __catchsym$?createNode@?$QMapData@W4DNATranslationRole@U2@@V?$QList@UTriplet@U2@@@@@@QAEPAU?$QMapNode@W4DNATranslationRole@U2@@V?$QList@UTriplet@U2@@@@@@ABW4DNATranslationRole@U2@@ABV?$QList@UTriplet@U2@@@@PAU2@_N@Z$6 1002ed34     ORFDialog.obj
 0002:00008d44       __catchsym$?createNode@?$QMapData@W4DNATranslationRole@U2@@V?$QList@UTriplet@U2@@@@@@QAEPAU?$QMapNode@W4DNATranslationRole@U2@@V?$QList@UTriplet@U2@@@@@@ABW4DNATranslationRole@U2@@ABV?$QList@UTriplet@U2@@@@PAU2@_N@Z$5 1002ed44     ORFDialog.obj
 0002:00008d54       __ehfuncinfo$?createNode@?$QMapData@W4DNATranslationRole@U2@@V?$QList@UTriplet@U2@@@@@@QAEPAU?$QMapNode@W4DNATranslationRole@U2@@V?$QList@UTriplet@U2@@@@@@ABW4DNATranslationRole@U2@@ABV?$QList@UTriplet@U2@@@@PAU2@_N@Z 1002ed54     ORFDialog.obj
 0002:00008d78       __tryblocktable$?createNode@?$QMapData@W4DNATranslationRole@U2@@V?$QList@UTriplet@U2@@@@@@QAEPAU?$QMapNode@W4DNATranslationRole@U2@@V?$QList@UTriplet@U2@@@@@@ABW4DNATranslationRole@U2@@ABV?$QList@UTriplet@U2@@@@PAU2@_N@Z 1002ed78     ORFDialog.obj
 0002:00008da0       __unwindtable$?createNode@?$QMapData@W4DNATranslationRole@U2@@V?$QList@UTriplet@U2@@@@@@QAEPAU?$QMapNode@W4DNATranslationRole@U2@@V?$QList@UTriplet@U2@@@@@@ABW4DNATranslationRole@U2@@ABV?$QList@UTriplet@U2@@@@PAU2@_N@Z 1002eda0     ORFDialog.obj
 0002:00008dc8       __unwindtable$??__EalgoLog@U2@@YAXXZ 1002edc8     ORFMarkerPlugin.obj
 0002:00008dd0       __ehfuncinfo$??__EalgoLog@U2@@YAXXZ 1002edd0     ORFMarkerPlugin.obj
 0002:00008df4       __unwindtable$??__EcmdLog@U2@@YAXXZ 1002edf4     ORFMarkerPlugin.obj
 0002:00008dfc       __ehfuncinfo$??__EcmdLog@U2@@YAXXZ 1002edfc     ORFMarkerPlugin.obj
 0002:00008e20       __unwindtable$??__EcoreLog@U2@@YAXXZ 1002ee20     ORFMarkerPlugin.obj
 0002:00008e28       __ehfuncinfo$??__EcoreLog@U2@@YAXXZ 1002ee28     ORFMarkerPlugin.obj
 0002:00008e4c       __unwindtable$??__EioLog@U2@@YAXXZ 1002ee4c     ORFMarkerPlugin.obj
 0002:00008e54       __ehfuncinfo$??__EioLog@U2@@YAXXZ 1002ee54     ORFMarkerPlugin.obj
 0002:00008e78       __unwindtable$??__EperfLog@U2@@YAXXZ 1002ee78     ORFMarkerPlugin.obj
 0002:00008e80       __ehfuncinfo$??__EperfLog@U2@@YAXXZ 1002ee80     ORFMarkerPlugin.obj
 0002:00008ea4       __unwindtable$??__EscriptLog@U2@@YAXXZ 1002eea4     ORFMarkerPlugin.obj
 0002:00008eac       __ehfuncinfo$??__EscriptLog@U2@@YAXXZ 1002eeac     ORFMarkerPlugin.obj
 0002:00008ed0       __unwindtable$??__EtaskLog@U2@@YAXXZ 1002eed0     ORFMarkerPlugin.obj
 0002:00008ed8       __ehfuncinfo$??__EtaskLog@U2@@YAXXZ 1002eed8     ORFMarkerPlugin.obj
 0002:00008efc       __unwindtable$??__EuiLog@U2@@YAXXZ 1002eefc     ORFMarkerPlugin.obj
 0002:00008f04       __ehfuncinfo$??__EuiLog@U2@@YAXXZ 1002ef04     ORFMarkerPlugin.obj
 0002:00008f28       __unwindtable$??__EuserActLog@U2@@YAXXZ 1002ef28     ORFMarkerPlugin.obj
 0002:00008f30       __ehfuncinfo$??__EuserActLog@U2@@YAXXZ 1002ef30     ORFMarkerPlugin.obj
 0002:00008f54       __ehfuncinfo$??0ORFMarkerPlugin@U2@@QAE@XZ 1002ef54     ORFMarkerPlugin.obj
 0002:00008f78       __unwindtable$??0ORFMarkerPlugin@U2@@QAE@XZ 1002ef78     ORFMarkerPlugin.obj
 0002:00008fd0       __unwindtable$??0ORFViewContext@U2@@QAE@PAVQObject@@@Z 1002efd0     ORFMarkerPlugin.obj
 0002:00008fe8       __ehfuncinfo$??0ORFViewContext@U2@@QAE@PAVQObject@@@Z 1002efe8     ORFMarkerPlugin.obj
 0002:0000900c       __unwindtable$?sl_showDialog@ORFViewContext@U2@@IAEXXZ 1002f00c     ORFMarkerPlugin.obj
 0002:00009024       __ehfuncinfo$?sl_showDialog@ORFViewContext@U2@@IAEXXZ 1002f024     ORFMarkerPlugin.obj
 0002:00009048       __ehfuncinfo$?initViewContext@ORFViewContext@U2@@MAEXPAVGObjectView@2@@Z 1002f048     ORFMarkerPlugin.obj
 0002:0000906c       __unwindtable$?initViewContext@ORFViewContext@U2@@MAEXPAVGObjectView@2@@Z 1002f06c     ORFMarkerPlugin.obj
 0002:000090ac       __unwindtable$?createTestFactories@ORFMarkerTests@U2@@SA?AV?$QList@PAVXMLTestFactory@U2@@@@XZ 1002f0ac     ORFMarkerPlugin.obj
 0002:000090b4       __ehfuncinfo$?createTestFactories@ORFMarkerTests@U2@@SA?AV?$QList@PAVXMLTestFactory@U2@@@@XZ 1002f0b4     ORFMarkerPlugin.obj
 0002:000090d8       __unwindtable$??0GTest_ORFMarkerTask@U2@@QAE@PAVXMLTestFormat@1@ABVQString@@PAVGTest@1@PBVGTestEnvironment@1@ABV?$QList@PAVGTest@U2@@@@ABVQDomElement@@@Z 1002f0d8     ORFMarkerPlugin.obj
 0002:000090f8       __ehfuncinfo$??0GTest_ORFMarkerTask@U2@@QAE@PAVXMLTestFormat@1@ABVQString@@PAVGTest@1@PBVGTestEnvironment@1@ABV?$QList@PAVGTest@U2@@@@ABVQDomElement@@@Z 1002f0f8     ORFMarkerPlugin.obj
 0002:0000911c       __unwindtable$??0GTest_ORFMarkerTaskFactory@GTest_ORFMarkerTask@U2@@QAE@XZ 1002f11c     ORFMarkerPlugin.obj
 0002:00009134       __ehfuncinfo$??0GTest_ORFMarkerTaskFactory@GTest_ORFMarkerTask@U2@@QAE@XZ 1002f134     ORFMarkerPlugin.obj
 0002:00009158       __unwindtable$?createTest@GTest_ORFMarkerTaskFactory@GTest_ORFMarkerTask@U2@@UAEPAVGTest@3@PAVXMLTestFormat@3@ABVQString@@PAV43@PBVGTestEnvironment@3@ABV?$QList@PAVGTest@U2@@@@ABVQDomElement@@@Z 1002f158     ORFMarkerPlugin.obj
 0002:00009160       __ehfuncinfo$?createTest@GTest_ORFMarkerTaskFactory@GTest_ORFMarkerTask@U2@@UAEPAVGTest@3@PAVXMLTestFormat@3@ABVQString@@PAV43@PBVGTestEnvironment@3@ABV?$QList@PAVGTest@U2@@@@ABVQDomElement@@@Z 1002f160     ORFMarkerPlugin.obj
 0002:00009184       __unwindtable$?createFactory@GTest_ORFMarkerTask@U2@@SAPAVXMLTestFactory@2@XZ 1002f184     ORFMarkerPlugin.obj
 0002:000091a4       __ehfuncinfo$?createFactory@GTest_ORFMarkerTask@U2@@SAPAVXMLTestFactory@2@XZ 1002f1a4     ORFMarkerPlugin.obj
 0002:000091c8       __unwindtable$??1GTest_ORFMarkerTask@U2@@UAE@XZ 1002f1c8     ORFMarkerPlugin.obj
 0002:000091e0       __ehfuncinfo$??1GTest_ORFMarkerTask@U2@@UAE@XZ 1002f1e0     ORFMarkerPlugin.obj
 0002:00009204       __unwindtable$??1?$GAutoDeleteList@VXMLTestFactory@U2@@@U2@@UAE@XZ 1002f204     ORFMarkerPlugin.obj
 0002:00009214       __ehfuncinfo$??1?$GAutoDeleteList@VXMLTestFactory@U2@@@U2@@UAE@XZ 1002f214     ORFMarkerPlugin.obj
 0002:00009238       __catchsym$??0?$QList@PAVXMLTestFactory@U2@@@@QAE@ABV0@@Z$2 1002f238     ORFMarkerPlugin.obj
 0002:00009248       __unwindtable$??0?$QList@PAVXMLTestFactory@U2@@@@QAE@ABV0@@Z 1002f248     ORFMarkerPlugin.obj
 0002:00009258       __tryblocktable$??0?$QList@PAVXMLTestFactory@U2@@@@QAE@ABV0@@Z 1002f258     ORFMarkerPlugin.obj
 0002:0000926c       __ehfuncinfo$??0?$QList@PAVXMLTestFactory@U2@@@@QAE@ABV0@@Z 1002f26c     ORFMarkerPlugin.obj
 0002:00009290       __catchsym$?append@?$QList@PAVXMLTestFactory@U2@@@@QAEXABQAVXMLTestFactory@U2@@@Z$6 1002f290     ORFMarkerPlugin.obj
 0002:000092a0       __tryblocktable$?append@?$QList@PAVXMLTestFactory@U2@@@@QAEXABQAVXMLTestFactory@U2@@@Z 1002f2a0     ORFMarkerPlugin.obj
 0002:000092b4       __ehfuncinfo$?append@?$QList@PAVXMLTestFactory@U2@@@@QAEXABQAVXMLTestFactory@U2@@@Z 1002f2b4     ORFMarkerPlugin.obj
 0002:000092d8       __unwindtable$?append@?$QList@PAVXMLTestFactory@U2@@@@QAEXABQAVXMLTestFactory@U2@@@Z 1002f2d8     ORFMarkerPlugin.obj
 0002:00009308       __catchsym$?detach_helper_grow@?$QList@PAVXMLTestFactory@U2@@@@AAEPAUNode@1@HH@Z$5 1002f308     ORFMarkerPlugin.obj
 0002:00009318       __catchsym$?detach_helper_grow@?$QList@PAVXMLTestFactory@U2@@@@AAEPAUNode@1@HH@Z$4 1002f318     ORFMarkerPlugin.obj
 0002:00009328       __unwindtable$?detach_helper_grow@?$QList@PAVXMLTestFactory@U2@@@@AAEPAUNode@1@HH@Z 1002f328     ORFMarkerPlugin.obj
 0002:00009348       __ehfuncinfo$?detach_helper_grow@?$QList@PAVXMLTestFactory@U2@@@@AAEPAUNode@1@HH@Z 1002f348     ORFMarkerPlugin.obj
 0002:0000936c       __tryblocktable$?detach_helper_grow@?$QList@PAVXMLTestFactory@U2@@@@AAEPAUNode@1@HH@Z 1002f36c     ORFMarkerPlugin.obj
 0002:00009394       __unwindtable$??1?$QObjectScopedPointer@VORFDialog@U2@@@U2@@QAE@XZ 1002f394     ORFMarkerPlugin.obj
 0002:0000939c       __ehfuncinfo$??1?$QObjectScopedPointer@VORFDialog@U2@@@U2@@QAE@XZ 1002f39c     ORFMarkerPlugin.obj
 0002:000093c0       __unwindtable$?qt_metatype_id@?$QMetaTypeId@VU2Region@U2@@@@SAHXZ 1002f3c0     ORFMarkerTask.obj
 0002:000093c8       __ehfuncinfo$?qt_metatype_id@?$QMetaTypeId@VU2Region@U2@@@@SAHXZ 1002f3c8     ORFMarkerTask.obj
 0002:000093ec       __unwindtable$??$qRegisterMetaType@VU2Region@U2@@@@YAHPBDPAVU2Region@U2@@W4DefinedType@?$MetaTypeDefinedHelper@VU2Region@U2@@$00@QtPrivate@@@Z 1002f3ec     ORFMarkerTask.obj
 0002:000093f4       __ehfuncinfo$??$qRegisterMetaType@VU2Region@U2@@@@YAHPBDPAVU2Region@U2@@W4DefinedType@?$MetaTypeDefinedHelper@VU2Region@U2@@$00@QtPrivate@@@Z 1002f3f4     ORFMarkerTask.obj
 0002:00009418       __catchsym$?append@?$QList@V?$QSharedDataPointer@VAnnotationData@U2@@@@@@QAEXABV?$QSharedDataPointer@VAnnotationData@U2@@@@@Z$12 1002f418     ORFMarkerTask.obj
 0002:00009428       __tryblocktable$?append@?$QList@V?$QSharedDataPointer@VAnnotationData@U2@@@@@@QAEXABV?$QSharedDataPointer@VAnnotationData@U2@@@@@Z 1002f428     ORFMarkerTask.obj
 0002:0000943c       __ehfuncinfo$?append@?$QList@V?$QSharedDataPointer@VAnnotationData@U2@@@@@@QAEXABV?$QSharedDataPointer@VAnnotationData@U2@@@@@Z 1002f43c     ORFMarkerTask.obj
 0002:00009460       __unwindtable$?append@?$QList@V?$QSharedDataPointer@VAnnotationData@U2@@@@@@QAEXABV?$QSharedDataPointer@VAnnotationData@U2@@@@@Z 1002f460     ORFMarkerTask.obj
 0002:00009490       __catchsym$?detach_helper_grow@?$QList@V?$QSharedDataPointer@VAnnotationData@U2@@@@@@AAEPAUNode@1@HH@Z$5 1002f490     ORFMarkerTask.obj
 0002:000094a0       __catchsym$?detach_helper_grow@?$QList@V?$QSharedDataPointer@VAnnotationData@U2@@@@@@AAEPAUNode@1@HH@Z$4 1002f4a0     ORFMarkerTask.obj
 0002:000094b0       __unwindtable$?detach_helper_grow@?$QList@V?$QSharedDataPointer@VAnnotationData@U2@@@@@@AAEPAUNode@1@HH@Z 1002f4b0     ORFMarkerTask.obj
 0002:000094d0       __ehfuncinfo$?detach_helper_grow@?$QList@V?$QSharedDataPointer@VAnnotationData@U2@@@@@@AAEPAUNode@1@HH@Z 1002f4d0     ORFMarkerTask.obj
 0002:000094f4       __tryblocktable$?detach_helper_grow@?$QList@V?$QSharedDataPointer@VAnnotationData@U2@@@@@@AAEPAUNode@1@HH@Z 1002f4f4     ORFMarkerTask.obj
 0002:0000951c       __unwindtable$??__EalgoLog@U2@@YAXXZ 1002f51c     ORFMarkerTask.obj
 0002:00009524       __ehfuncinfo$??__EalgoLog@U2@@YAXXZ 1002f524     ORFMarkerTask.obj
 0002:00009548       __unwindtable$??__EcmdLog@U2@@YAXXZ 1002f548     ORFMarkerTask.obj
 0002:00009550       __ehfuncinfo$??__EcmdLog@U2@@YAXXZ 1002f550     ORFMarkerTask.obj
 0002:00009574       __unwindtable$??__EcoreLog@U2@@YAXXZ 1002f574     ORFMarkerTask.obj
 0002:0000957c       __ehfuncinfo$??__EcoreLog@U2@@YAXXZ 1002f57c     ORFMarkerTask.obj
 0002:000095a0       __unwindtable$??__EioLog@U2@@YAXXZ 1002f5a0     ORFMarkerTask.obj
 0002:000095a8       __ehfuncinfo$??__EioLog@U2@@YAXXZ 1002f5a8     ORFMarkerTask.obj
 0002:000095cc       __unwindtable$??__EperfLog@U2@@YAXXZ 1002f5cc     ORFMarkerTask.obj
 0002:000095d4       __ehfuncinfo$??__EperfLog@U2@@YAXXZ 1002f5d4     ORFMarkerTask.obj
 0002:000095f8       __unwindtable$??__EscriptLog@U2@@YAXXZ 1002f5f8     ORFMarkerTask.obj
 0002:00009600       __ehfuncinfo$??__EscriptLog@U2@@YAXXZ 1002f600     ORFMarkerTask.obj
 0002:00009624       __unwindtable$??__EtaskLog@U2@@YAXXZ 1002f624     ORFMarkerTask.obj
 0002:0000962c       __ehfuncinfo$??__EtaskLog@U2@@YAXXZ 1002f62c     ORFMarkerTask.obj
 0002:00009650       __unwindtable$??__EuiLog@U2@@YAXXZ 1002f650     ORFMarkerTask.obj
 0002:00009658       __ehfuncinfo$??__EuiLog@U2@@YAXXZ 1002f658     ORFMarkerTask.obj
 0002:0000967c       __unwindtable$??__EuserActLog@U2@@YAXXZ 1002f67c     ORFMarkerTask.obj
 0002:00009684       __ehfuncinfo$??__EuserActLog@U2@@YAXXZ 1002f684     ORFMarkerTask.obj
 0002:000096a8       __catchsym$?append@?$QList@PAVTask@U2@@@@QAEXABQAVTask@U2@@@Z$6 1002f6a8     ORFMarkerTask.obj
 0002:000096b8       __tryblocktable$?append@?$QList@PAVTask@U2@@@@QAEXABQAVTask@U2@@@Z 1002f6b8     ORFMarkerTask.obj
 0002:000096cc       __ehfuncinfo$?append@?$QList@PAVTask@U2@@@@QAEXABQAVTask@U2@@@Z 1002f6cc     ORFMarkerTask.obj
 0002:000096f0       __unwindtable$?append@?$QList@PAVTask@U2@@@@QAEXABQAVTask@U2@@@Z 1002f6f0     ORFMarkerTask.obj
 0002:00009720       __catchsym$?detach_helper_grow@?$QList@PAVTask@U2@@@@AAEPAUNode@1@HH@Z$5 1002f720     ORFMarkerTask.obj
 0002:00009730       __catchsym$?detach_helper_grow@?$QList@PAVTask@U2@@@@AAEPAUNode@1@HH@Z$4 1002f730     ORFMarkerTask.obj
 0002:00009740       __unwindtable$?detach_helper_grow@?$QList@PAVTask@U2@@@@AAEPAUNode@1@HH@Z 1002f740     ORFMarkerTask.obj
 0002:00009760       __ehfuncinfo$?detach_helper_grow@?$QList@PAVTask@U2@@@@AAEPAUNode@1@HH@Z 1002f760     ORFMarkerTask.obj
 0002:00009784       __tryblocktable$?detach_helper_grow@?$QList@PAVTask@U2@@@@AAEPAUNode@1@HH@Z 1002f784     ORFMarkerTask.obj
 0002:000097ac       __ehfuncinfo$?save@ORFSettingsKeys@U2@@SAXABVORFAlgorithmSettings@2@PAVSettings@2@@Z 1002f7ac     ORFMarkerTask.obj
 0002:000097d0       __unwindtable$?save@ORFSettingsKeys@U2@@SAXABVORFAlgorithmSettings@2@PAVSettings@2@@Z 1002f7d0     ORFMarkerTask.obj
 0002:00009830       __ehfuncinfo$?read@ORFSettingsKeys@U2@@SAXAAVORFAlgorithmSettings@2@PBVSettings@2@@Z 1002f830     ORFMarkerTask.obj
 0002:00009854       __unwindtable$?read@ORFSettingsKeys@U2@@SAXAAVORFAlgorithmSettings@2@PBVSettings@2@@Z 1002f854     ORFMarkerTask.obj
 0002:00009934       __ehfuncinfo$??0FindORFsToAnnotationsTask@U2@@QAE@PAVAnnotationTableObject@1@ABVU2EntityRef@1@ABVORFAlgorithmSettings@1@ABVQString@@3@Z 1002f934     ORFMarkerTask.obj
 0002:00009958       __unwindtable$??0FindORFsToAnnotationsTask@U2@@QAE@PAVAnnotationTableObject@1@ABVU2EntityRef@1@ABVORFAlgorithmSettings@1@ABVQString@@3@Z 1002f958     ORFMarkerTask.obj
 0002:000099a0       __ehfuncinfo$?onSubTaskFinished@FindORFsToAnnotationsTask@U2@@UAE?AV?$QList@PAVTask@U2@@@@PAVTask@2@@Z 1002f9a0     ORFMarkerTask.obj
 0002:000099c4       __unwindtable$?onSubTaskFinished@FindORFsToAnnotationsTask@U2@@UAE?AV?$QList@PAVTask@U2@@@@PAVTask@2@@Z 1002f9c4     ORFMarkerTask.obj
 0002:000099fc       __unwindtable$??1FindORFsToAnnotationsTask@U2@@UAE@XZ 1002f9fc     ORFMarkerTask.obj
 0002:00009a1c       __ehfuncinfo$??1FindORFsToAnnotationsTask@U2@@UAE@XZ 1002fa1c     ORFMarkerTask.obj
 0002:00009a40       __unwindtable$??0ORFAutoAnnotationsUpdater@U2@@QAE@XZ 1002fa40     ORFMarkerTask.obj
 0002:00009a58       __ehfuncinfo$??0ORFAutoAnnotationsUpdater@U2@@QAE@XZ 1002fa58     ORFMarkerTask.obj
 0002:00009a7c       __ehfuncinfo$?createAutoAnnotationsUpdateTask@ORFAutoAnnotationsUpdater@U2@@UAEPAVTask@2@PBVAutoAnnotationObject@2@@Z 1002fa7c     ORFMarkerTask.obj
 0002:00009aa0       __unwindtable$?createAutoAnnotationsUpdateTask@ORFAutoAnnotationsUpdater@U2@@UAEPAVTask@2@PBVAutoAnnotationObject@2@@Z 1002faa0     ORFMarkerTask.obj
 0002:00009ad8       __catchsym$??0?$QList@VQString@@@@QAE@ABV0@@Z$2 1002fad8     ORFMarkerTests.obj
 0002:00009ae8       __unwindtable$??0?$QList@VQString@@@@QAE@ABV0@@Z 1002fae8     ORFMarkerTests.obj
 0002:00009af8       __tryblocktable$??0?$QList@VQString@@@@QAE@ABV0@@Z 1002faf8     ORFMarkerTests.obj
 0002:00009b0c       __ehfuncinfo$??0?$QList@VQString@@@@QAE@ABV0@@Z 1002fb0c     ORFMarkerTests.obj
 0002:00009b30       __catchsym$?detach_helper@?$QList@VQString@@@@AAEXH@Z$2 1002fb30     ORFMarkerTests.obj
 0002:00009b40       __unwindtable$?detach_helper@?$QList@VQString@@@@AAEXH@Z 1002fb40     ORFMarkerTests.obj
 0002:00009b50       __tryblocktable$?detach_helper@?$QList@VQString@@@@AAEXH@Z 1002fb50     ORFMarkerTests.obj
 0002:00009b64       __ehfuncinfo$?detach_helper@?$QList@VQString@@@@AAEXH@Z 1002fb64     ORFMarkerTests.obj
 0002:00009b88       __catchsym$?node_copy@?$QList@VQString@@@@AAEXPAUNode@1@00@Z$6 1002fb88     ORFMarkerTests.obj
 0002:00009b98       __tryblocktable$?node_copy@?$QList@VQString@@@@AAEXPAUNode@1@00@Z 1002fb98     ORFMarkerTests.obj
 0002:00009bac       __ehfuncinfo$?node_copy@?$QList@VQString@@@@AAEXPAUNode@1@00@Z 1002fbac     ORFMarkerTests.obj
 0002:00009bd0       __unwindtable$?node_copy@?$QList@VQString@@@@AAEXPAUNode@1@00@Z 1002fbd0     ORFMarkerTests.obj
 0002:00009c00       __unwindtable$??__EalgoLog@U2@@YAXXZ 1002fc00     ORFMarkerTests.obj
 0002:00009c08       __ehfuncinfo$??__EalgoLog@U2@@YAXXZ 1002fc08     ORFMarkerTests.obj
 0002:00009c2c       __unwindtable$??__EcmdLog@U2@@YAXXZ 1002fc2c     ORFMarkerTests.obj
 0002:00009c34       __ehfuncinfo$??__EcmdLog@U2@@YAXXZ 1002fc34     ORFMarkerTests.obj
 0002:00009c58       __unwindtable$??__EcoreLog@U2@@YAXXZ 1002fc58     ORFMarkerTests.obj
 0002:00009c60       __ehfuncinfo$??__EcoreLog@U2@@YAXXZ 1002fc60     ORFMarkerTests.obj
 0002:00009c84       __unwindtable$??__EioLog@U2@@YAXXZ 1002fc84     ORFMarkerTests.obj
 0002:00009c8c       __ehfuncinfo$??__EioLog@U2@@YAXXZ 1002fc8c     ORFMarkerTests.obj
 0002:00009cb0       __unwindtable$??__EperfLog@U2@@YAXXZ 1002fcb0     ORFMarkerTests.obj
 0002:00009cb8       __ehfuncinfo$??__EperfLog@U2@@YAXXZ 1002fcb8     ORFMarkerTests.obj
 0002:00009cdc       __unwindtable$??__EscriptLog@U2@@YAXXZ 1002fcdc     ORFMarkerTests.obj
 0002:00009ce4       __ehfuncinfo$??__EscriptLog@U2@@YAXXZ 1002fce4     ORFMarkerTests.obj
 0002:00009d08       __unwindtable$??__EtaskLog@U2@@YAXXZ 1002fd08     ORFMarkerTests.obj
 0002:00009d10       __ehfuncinfo$??__EtaskLog@U2@@YAXXZ 1002fd10     ORFMarkerTests.obj
 0002:00009d34       __unwindtable$??__EuiLog@U2@@YAXXZ 1002fd34     ORFMarkerTests.obj
 0002:00009d3c       __ehfuncinfo$??__EuiLog@U2@@YAXXZ 1002fd3c     ORFMarkerTests.obj
 0002:00009d60       __unwindtable$??__EuserActLog@U2@@YAXXZ 1002fd60     ORFMarkerTests.obj
 0002:00009d68       __ehfuncinfo$??__EuserActLog@U2@@YAXXZ 1002fd68     ORFMarkerTests.obj
 0002:00009d8c       __catchsym$?reallocData@?$QVector@VU2Region@U2@@@@AAEXHHV?$QFlags@W4AllocationOption@QArrayData@@@@@Z$5 1002fd8c     ORFMarkerTests.obj
 0002:00009d9c       __catchsym$?reallocData@?$QVector@VU2Region@U2@@@@AAEXHHV?$QFlags@W4AllocationOption@QArrayData@@@@@Z$4 1002fd9c     ORFMarkerTests.obj
 0002:00009dac       __unwindtable$?reallocData@?$QVector@VU2Region@U2@@@@AAEXHHV?$QFlags@W4AllocationOption@QArrayData@@@@@Z 1002fdac     ORFMarkerTests.obj
 0002:00009dcc       __ehfuncinfo$?reallocData@?$QVector@VU2Region@U2@@@@AAEXHHV?$QFlags@W4AllocationOption@QArrayData@@@@@Z 1002fdcc     ORFMarkerTests.obj
 0002:00009df0       __tryblocktable$?reallocData@?$QVector@VU2Region@U2@@@@AAEXHHV?$QFlags@W4AllocationOption@QArrayData@@@@@Z 1002fdf0     ORFMarkerTests.obj
 0002:00009e18       __ehfuncinfo$?init@GTest_ORFMarkerTask@U2@@QAEXPAVXMLTestFormat@2@ABVQDomElement@@@Z 1002fe18     ORFMarkerTests.obj
 0002:00009e3c       __unwindtable$?init@GTest_ORFMarkerTask@U2@@QAEXPAVXMLTestFormat@2@ABVQDomElement@@@Z 1002fe3c     ORFMarkerTests.obj
 0002:0000a0e4       __unwindtable$?prepare@GTest_ORFMarkerTask@U2@@UAEXXZ 100300e4     ORFMarkerTests.obj
 0002:0000a104       __ehfuncinfo$?prepare@GTest_ORFMarkerTask@U2@@UAEXXZ 10030104     ORFMarkerTests.obj
 0002:0000a128       __ehfuncinfo$?report@GTest_ORFMarkerTask@U2@@UAE?AW4ReportResult@Task@2@XZ 10030128     ORFMarkerTests.obj
 0002:0000a14c       __unwindtable$?report@GTest_ORFMarkerTask@U2@@UAE?AW4ReportResult@Task@2@XZ 1003014c     ORFMarkerTests.obj
 0002:0000a18c       __unwindtable$??0Translator@U2@@QAE@PBVU2SequenceObject@1@ABVQString@@@Z 1003018c     ORFMarkerTests.obj
 0002:0000a194       __ehfuncinfo$??0Translator@U2@@QAE@PBVU2SequenceObject@1@ABVQString@@@Z 10030194     ORFMarkerTests.obj
 0002:0000a1b8       __unwindtable$??A?$QMap@VQString@@VQVariant@@@@QAEAAVQVariant@@ABVQString@@@Z 100301b8     ORFQuery.obj
 0002:0000a1c0       __ehfuncinfo$??A?$QMap@VQString@@VQVariant@@@@QAEAAVQVariant@@ABVQString@@@Z 100301c0     ORFQuery.obj
 0002:0000a1e4       __unwindtable$??0?$QForeachContainer@$$CBV?$QVector@VU2Region@U2@@@@@@QAE@ABV?$QVector@VU2Region@U2@@@@@Z 100301e4     ORFQuery.obj
 0002:0000a1ec       __ehfuncinfo$??0?$QForeachContainer@$$CBV?$QVector@VU2Region@U2@@@@@@QAE@ABV?$QVector@VU2Region@U2@@@@@Z 100301ec     ORFQuery.obj
 0002:0000a210       __unwindtable$?copyConstruct@?$QVector@VU2Qualifier@U2@@@@AAEXPBVU2Qualifier@U2@@0PAV23@@Z 10030210     ORFQuery.obj
 0002:0000a218       __ehfuncinfo$?copyConstruct@?$QVector@VU2Qualifier@U2@@@@AAEXPBVU2Qualifier@U2@@0PAV23@@Z 10030218     ORFQuery.obj
 0002:0000a23c       __catchsym$??0?$QList@V?$QSharedDataPointer@VAnnotationData@U2@@@@@@QAE@ABV0@@Z$2 1003023c     ORFQuery.obj
 0002:0000a24c       __unwindtable$??0?$QList@V?$QSharedDataPointer@VAnnotationData@U2@@@@@@QAE@ABV0@@Z 1003024c     ORFQuery.obj
 0002:0000a25c       __tryblocktable$??0?$QList@V?$QSharedDataPointer@VAnnotationData@U2@@@@@@QAE@ABV0@@Z 1003025c     ORFQuery.obj
 0002:0000a270       __ehfuncinfo$??0?$QList@V?$QSharedDataPointer@VAnnotationData@U2@@@@@@QAE@ABV0@@Z 10030270     ORFQuery.obj
 0002:0000a294       __unwindtable$??__EalgoLog@U2@@YAXXZ 10030294     ORFQuery.obj
 0002:0000a29c       __ehfuncinfo$??__EalgoLog@U2@@YAXXZ 1003029c     ORFQuery.obj
 0002:0000a2c0       __unwindtable$??__EcmdLog@U2@@YAXXZ 100302c0     ORFQuery.obj
 0002:0000a2c8       __ehfuncinfo$??__EcmdLog@U2@@YAXXZ 100302c8     ORFQuery.obj
 0002:0000a2ec       __unwindtable$??__EcoreLog@U2@@YAXXZ 100302ec     ORFQuery.obj
 0002:0000a2f4       __ehfuncinfo$??__EcoreLog@U2@@YAXXZ 100302f4     ORFQuery.obj
 0002:0000a318       __unwindtable$??__EioLog@U2@@YAXXZ 10030318     ORFQuery.obj
 0002:0000a320       __ehfuncinfo$??__EioLog@U2@@YAXXZ 10030320     ORFQuery.obj
 0002:0000a344       __unwindtable$??__EperfLog@U2@@YAXXZ 10030344     ORFQuery.obj
 0002:0000a34c       __ehfuncinfo$??__EperfLog@U2@@YAXXZ 1003034c     ORFQuery.obj
 0002:0000a370       __unwindtable$??__EscriptLog@U2@@YAXXZ 10030370     ORFQuery.obj
 0002:0000a378       __ehfuncinfo$??__EscriptLog@U2@@YAXXZ 10030378     ORFQuery.obj
 0002:0000a39c       __unwindtable$??__EtaskLog@U2@@YAXXZ 1003039c     ORFQuery.obj
 0002:0000a3a4       __ehfuncinfo$??__EtaskLog@U2@@YAXXZ 100303a4     ORFQuery.obj
 0002:0000a3c8       __unwindtable$??__EuiLog@U2@@YAXXZ 100303c8     ORFQuery.obj
 0002:0000a3d0       __ehfuncinfo$??__EuiLog@U2@@YAXXZ 100303d0     ORFQuery.obj
 0002:0000a3f4       __unwindtable$??__EuserActLog@U2@@YAXXZ 100303f4     ORFQuery.obj
 0002:0000a3fc       __ehfuncinfo$??__EuserActLog@U2@@YAXXZ 100303fc     ORFQuery.obj
 0002:0000a420       __catchsym$?append@?$QList@PAVAttribute@U2@@@@QAEXABQAVAttribute@U2@@@Z$6 10030420     ORFQuery.obj
 0002:0000a430       __tryblocktable$?append@?$QList@PAVAttribute@U2@@@@QAEXABQAVAttribute@U2@@@Z 10030430     ORFQuery.obj
 0002:0000a444       __ehfuncinfo$?append@?$QList@PAVAttribute@U2@@@@QAEXABQAVAttribute@U2@@@Z 10030444     ORFQuery.obj
 0002:0000a468       __unwindtable$?append@?$QList@PAVAttribute@U2@@@@QAEXABQAVAttribute@U2@@@Z 10030468     ORFQuery.obj
 0002:0000a498       __catchsym$?detach_helper_grow@?$QList@PAVAttribute@U2@@@@AAEPAUNode@1@HH@Z$5 10030498     ORFQuery.obj
 0002:0000a4a8       __catchsym$?detach_helper_grow@?$QList@PAVAttribute@U2@@@@AAEPAUNode@1@HH@Z$4 100304a8     ORFQuery.obj
 0002:0000a4b8       __unwindtable$?detach_helper_grow@?$QList@PAVAttribute@U2@@@@AAEPAUNode@1@HH@Z 100304b8     ORFQuery.obj
 0002:0000a4d8       __ehfuncinfo$?detach_helper_grow@?$QList@PAVAttribute@U2@@@@AAEPAUNode@1@HH@Z 100304d8     ORFQuery.obj
 0002:0000a4fc       __tryblocktable$?detach_helper_grow@?$QList@PAVAttribute@U2@@@@AAEPAUNode@1@HH@Z 100304fc     ORFQuery.obj
 0002:0000a524       __catchsym$??Y?$QList@VORFFindResult@U2@@@@QAEAAV0@ABV0@@Z$3 10030524     ORFQuery.obj
 0002:0000a534       __unwindtable$??Y?$QList@VORFFindResult@U2@@@@QAEAAV0@ABV0@@Z 10030534     ORFQuery.obj
 0002:0000a544       __tryblocktable$??Y?$QList@VORFFindResult@U2@@@@QAEAAV0@ABV0@@Z 10030544     ORFQuery.obj
 0002:0000a558       __ehfuncinfo$??Y?$QList@VORFFindResult@U2@@@@QAEAAV0@ABV0@@Z 10030558     ORFQuery.obj
 0002:0000a57c       __catchsym$?detach_helper_grow@?$QList@VORFFindResult@U2@@@@AAEPAUNode@1@HH@Z$5 1003057c     ORFQuery.obj
 0002:0000a58c       __catchsym$?detach_helper_grow@?$QList@VORFFindResult@U2@@@@AAEPAUNode@1@HH@Z$4 1003058c     ORFQuery.obj
 0002:0000a59c       __unwindtable$?detach_helper_grow@?$QList@VORFFindResult@U2@@@@AAEPAUNode@1@HH@Z 1003059c     ORFQuery.obj
 0002:0000a5bc       __ehfuncinfo$?detach_helper_grow@?$QList@VORFFindResult@U2@@@@AAEPAUNode@1@HH@Z 100305bc     ORFQuery.obj
 0002:0000a5e0       __tryblocktable$?detach_helper_grow@?$QList@VORFFindResult@U2@@@@AAEPAUNode@1@HH@Z 100305e0     ORFQuery.obj
 0002:0000a608       __ehfuncinfo$??0QDORFActor@U2@@QAE@PBVQDActorPrototype@1@@Z 10030608     ORFQuery.obj
 0002:0000a62c       __unwindtable$??0QDORFActor@U2@@QAE@PBVQDActorPrototype@1@@Z 1003062c     ORFQuery.obj
 0002:0000a654       __ehfuncinfo$?getText@QDORFActor@U2@@UBE?AVQString@@XZ 10030654     ORFQuery.obj
 0002:0000a678       __unwindtable$?getText@QDORFActor@U2@@UBE?AVQString@@XZ 10030678     ORFQuery.obj
 0002:0000a788       __ehfuncinfo$?getAlgorithmTask@QDORFActor@U2@@UAEPAVTask@2@ABV?$QVector@VU2Region@U2@@@@@Z 10030788     ORFQuery.obj
 0002:0000a7ac       __unwindtable$?getAlgorithmTask@QDORFActor@U2@@UAEPAVTask@2@ABV?$QVector@VU2Region@U2@@@@@Z 100307ac     ORFQuery.obj
 0002:0000a81c       __ehfuncinfo$?sl_onAlgorithmTaskFinished@QDORFActor@U2@@AAEXPAVTask@2@@Z 1003081c     ORFQuery.obj
 0002:0000a840       __unwindtable$?sl_onAlgorithmTaskFinished@QDORFActor@U2@@AAEXPAVTask@2@@Z 10030840     ORFQuery.obj
 0002:0000a8b0       __catchsym$??0?$QList@PAVORFFindTask@U2@@@@QAE@ABV0@@Z$2 100308b0     ORFQuery.obj
 0002:0000a8c0       __unwindtable$??0?$QList@PAVORFFindTask@U2@@@@QAE@ABV0@@Z 100308c0     ORFQuery.obj
 0002:0000a8d0       __tryblocktable$??0?$QList@PAVORFFindTask@U2@@@@QAE@ABV0@@Z 100308d0     ORFQuery.obj
 0002:0000a8e4       __ehfuncinfo$??0?$QList@PAVORFFindTask@U2@@@@QAE@ABV0@@Z 100308e4     ORFQuery.obj
 0002:0000a908       __catchsym$?append@?$QList@PAVORFFindTask@U2@@@@QAEXABQAVORFFindTask@U2@@@Z$6 10030908     ORFQuery.obj
 0002:0000a918       __tryblocktable$?append@?$QList@PAVORFFindTask@U2@@@@QAEXABQAVORFFindTask@U2@@@Z 10030918     ORFQuery.obj
 0002:0000a92c       __ehfuncinfo$?append@?$QList@PAVORFFindTask@U2@@@@QAEXABQAVORFFindTask@U2@@@Z 1003092c     ORFQuery.obj
 0002:0000a950       __unwindtable$?append@?$QList@PAVORFFindTask@U2@@@@QAEXABQAVORFFindTask@U2@@@Z 10030950     ORFQuery.obj
 0002:0000a980       __catchsym$?detach_helper_grow@?$QList@PAVORFFindTask@U2@@@@AAEPAUNode@1@HH@Z$5 10030980     ORFQuery.obj
 0002:0000a990       __catchsym$?detach_helper_grow@?$QList@PAVORFFindTask@U2@@@@AAEPAUNode@1@HH@Z$4 10030990     ORFQuery.obj
 0002:0000a9a0       __unwindtable$?detach_helper_grow@?$QList@PAVORFFindTask@U2@@@@AAEPAUNode@1@HH@Z 100309a0     ORFQuery.obj
 0002:0000a9c0       __ehfuncinfo$?detach_helper_grow@?$QList@PAVORFFindTask@U2@@@@AAEPAUNode@1@HH@Z 100309c0     ORFQuery.obj
 0002:0000a9e4       __tryblocktable$?detach_helper_grow@?$QList@PAVORFFindTask@U2@@@@AAEPAUNode@1@HH@Z 100309e4     ORFQuery.obj
 0002:0000aa0c       __unwindtable$??1QDORFActor@U2@@UAE@XZ 10030a0c     ORFQuery.obj
 0002:0000aa14       __ehfuncinfo$??1QDORFActor@U2@@UAE@XZ 10030a14     ORFQuery.obj
 0002:0000aa38       __unwindtable$??_GQDORFActor@U2@@UAEPAXI@Z 10030a38     ORFQuery.obj
 0002:0000aa40       __ehfuncinfo$??_GQDORFActor@U2@@UAEPAXI@Z 10030a40     ORFQuery.obj
 0002:0000aa64       __ehfuncinfo$??0QDORFActorPrototype@U2@@QAE@XZ 10030a64     ORFQuery.obj
 0002:0000aa88       __unwindtable$??0QDORFActorPrototype@U2@@QAE@XZ 10030a88     ORFQuery.obj
 0002:0000ad40       __unwindtable$?getIcon@QDORFActorPrototype@U2@@UBE?AVQIcon@@XZ 10030d40     ORFQuery.obj
 0002:0000ad50       __ehfuncinfo$?getIcon@QDORFActorPrototype@U2@@UBE?AVQIcon@@XZ 10030d50     ORFQuery.obj
 0002:0000ad74       __unwindtable$?createInstance@QDORFActorPrototype@U2@@UBEPAVQDActor@2@XZ 10030d74     ORFQuery.obj
 0002:0000ad7c       __ehfuncinfo$?createInstance@QDORFActorPrototype@U2@@UBEPAVQDActor@2@XZ 10030d7c     ORFQuery.obj
 0002:0000ada0       __catchsym$??0?$QList@PAVDNATranslation@U2@@@@QAE@ABV0@@Z$2 10030da0     ORFQuery.obj
 0002:0000adb0       __unwindtable$??0?$QList@PAVDNATranslation@U2@@@@QAE@ABV0@@Z 10030db0     ORFQuery.obj
 0002:0000adc0       __tryblocktable$??0?$QList@PAVDNATranslation@U2@@@@QAE@ABV0@@Z 10030dc0     ORFQuery.obj
 0002:0000add4       __ehfuncinfo$??0?$QList@PAVDNATranslation@U2@@@@QAE@ABV0@@Z 10030dd4     ORFQuery.obj
 0002:0000adf8       __unwindtable$?clone@?$QSharedDataPointer@VQDResultUnitData@U2@@@@IAEPAVQDResultUnitData@U2@@XZ 10030df8     ORFQuery.obj
 0002:0000ae00       __ehfuncinfo$?clone@?$QSharedDataPointer@VQDResultUnitData@U2@@@@IAEPAVQDResultUnitData@U2@@XZ 10030e00     ORFQuery.obj
 0002:0000ae24       __unwindtable$?detach_helper@?$QSharedDataPointer@VQDResultUnitData@U2@@@@AAEXXZ 10030e24     ORFQuery.obj
 0002:0000ae2c       __ehfuncinfo$?detach_helper@?$QSharedDataPointer@VQDResultUnitData@U2@@@@AAEXXZ 10030e2c     ORFQuery.obj
 0002:0000ae50       __catchsym$?createNode@?$QMapData@VQString@@VQVariant@@@@QAEPAU?$QMapNode@VQString@@VQVariant@@@@ABVQString@@ABVQVariant@@PAU2@_N@Z$7 10030e50     ORFQuery.obj
 0002:0000ae60       __catchsym$?createNode@?$QMapData@VQString@@VQVariant@@@@QAEPAU?$QMapNode@VQString@@VQVariant@@@@ABVQString@@ABVQVariant@@PAU2@_N@Z$6 10030e60     ORFQuery.obj
 0002:0000ae70       __ehfuncinfo$?createNode@?$QMapData@VQString@@VQVariant@@@@QAEPAU?$QMapNode@VQString@@VQVariant@@@@ABVQString@@ABVQVariant@@PAU2@_N@Z 10030e70     ORFQuery.obj
 0002:0000ae94       __tryblocktable$?createNode@?$QMapData@VQString@@VQVariant@@@@QAEPAU?$QMapNode@VQString@@VQVariant@@@@ABVQString@@ABVQVariant@@PAU2@_N@Z 10030e94     ORFQuery.obj
 0002:0000aebc       __unwindtable$?createNode@?$QMapData@VQString@@VQVariant@@@@QAEPAU?$QMapNode@VQString@@VQVariant@@@@ABVQString@@ABVQVariant@@PAU2@_N@Z 10030ebc     ORFQuery.obj
 0002:0000aeec       __catchsym$?createNode@?$QMapData@VQString@@PAVPropertyDelegate@U2@@@@QAEPAU?$QMapNode@VQString@@PAVPropertyDelegate@U2@@@@ABVQString@@ABQAVPropertyDelegate@U2@@PAU2@_N@Z$5 10030eec     ORFQuery.obj
 0002:0000aefc       __tryblocktable$?createNode@?$QMapData@VQString@@PAVPropertyDelegate@U2@@@@QAEPAU?$QMapNode@VQString@@PAVPropertyDelegate@U2@@@@ABVQString@@ABQAVPropertyDelegate@U2@@PAU2@_N@Z 10030efc     ORFQuery.obj
 0002:0000af10       __ehfuncinfo$?createNode@?$QMapData@VQString@@PAVPropertyDelegate@U2@@@@QAEPAU?$QMapNode@VQString@@PAVPropertyDelegate@U2@@@@ABVQString@@ABQAVPropertyDelegate@U2@@PAU2@_N@Z 10030f10     ORFQuery.obj
 0002:0000af34       __unwindtable$?createNode@?$QMapData@VQString@@PAVPropertyDelegate@U2@@@@QAEPAU?$QMapNode@VQString@@PAVPropertyDelegate@U2@@@@ABVQString@@ABQAVPropertyDelegate@U2@@PAU2@_N@Z 10030f34     ORFQuery.obj
 0002:0000af5c       __unwindtable$?metaType@?$QVariantValueHelper@VQString@@@QtPrivate@@SA?AVQString@@ABVQVariant@@@Z 10030f5c     ORFQuery.obj
 0002:0000af6c       __ehfuncinfo$?metaType@?$QVariantValueHelper@VQString@@@QtPrivate@@SA?AVQString@@ABVQVariant@@@Z 10030f6c     ORFQuery.obj
 0002:0000af90       __catchsym$?createNode@?$QMapData@VQString@@PAVQDSchemeUnit@U2@@@@QAEPAU?$QMapNode@VQString@@PAVQDSchemeUnit@U2@@@@ABVQString@@ABQAVQDSchemeUnit@U2@@PAU2@_N@Z$5 10030f90     ORFQuery.obj
 0002:0000afa0       __tryblocktable$?createNode@?$QMapData@VQString@@PAVQDSchemeUnit@U2@@@@QAEPAU?$QMapNode@VQString@@PAVQDSchemeUnit@U2@@@@ABVQString@@ABQAVQDSchemeUnit@U2@@PAU2@_N@Z 10030fa0     ORFQuery.obj
 0002:0000afb4       __ehfuncinfo$?createNode@?$QMapData@VQString@@PAVQDSchemeUnit@U2@@@@QAEPAU?$QMapNode@VQString@@PAVQDSchemeUnit@U2@@@@ABVQString@@ABQAVQDSchemeUnit@U2@@PAU2@_N@Z 10030fb4     ORFQuery.obj
 0002:0000afd8       __unwindtable$?createNode@?$QMapData@VQString@@PAVQDSchemeUnit@U2@@@@QAEPAU?$QMapNode@VQString@@PAVQDSchemeUnit@U2@@@@ABVQString@@ABQAVQDSchemeUnit@U2@@PAU2@_N@Z 10030fd8     ORFQuery.obj
 0002:0000b000       __unwindtable$??__EalgoLog@U2@@YAXXZ 10031000     ORFWorker.obj
 0002:0000b008       __ehfuncinfo$??__EalgoLog@U2@@YAXXZ 10031008     ORFWorker.obj
 0002:0000b02c       __unwindtable$??__EcmdLog@U2@@YAXXZ 1003102c     ORFWorker.obj
 0002:0000b034       __ehfuncinfo$??__EcmdLog@U2@@YAXXZ 10031034     ORFWorker.obj
 0002:0000b058       __unwindtable$??__EcoreLog@U2@@YAXXZ 10031058     ORFWorker.obj
 0002:0000b060       __ehfuncinfo$??__EcoreLog@U2@@YAXXZ 10031060     ORFWorker.obj
 0002:0000b084       __unwindtable$??__EioLog@U2@@YAXXZ 10031084     ORFWorker.obj
 0002:0000b08c       __ehfuncinfo$??__EioLog@U2@@YAXXZ 1003108c     ORFWorker.obj
 0002:0000b0b0       __unwindtable$??__EperfLog@U2@@YAXXZ 100310b0     ORFWorker.obj
 0002:0000b0b8       __ehfuncinfo$??__EperfLog@U2@@YAXXZ 100310b8     ORFWorker.obj
 0002:0000b0dc       __unwindtable$??__EscriptLog@U2@@YAXXZ 100310dc     ORFWorker.obj
 0002:0000b0e4       __ehfuncinfo$??__EscriptLog@U2@@YAXXZ 100310e4     ORFWorker.obj
 0002:0000b108       __unwindtable$??__EtaskLog@U2@@YAXXZ 10031108     ORFWorker.obj
 0002:0000b110       __ehfuncinfo$??__EtaskLog@U2@@YAXXZ 10031110     ORFWorker.obj
 0002:0000b134       __unwindtable$??__EuiLog@U2@@YAXXZ 10031134     ORFWorker.obj
 0002:0000b13c       __ehfuncinfo$??__EuiLog@U2@@YAXXZ 1003113c     ORFWorker.obj
 0002:0000b160       __unwindtable$??__EuserActLog@U2@@YAXXZ 10031160     ORFWorker.obj
 0002:0000b168       __ehfuncinfo$??__EuserActLog@U2@@YAXXZ 10031168     ORFWorker.obj
 0002:0000b18c       __unwindtable$??A?$QMap@VQString@@VQScriptValue@@@@QAEAAVQScriptValue@@ABVQString@@@Z 1003118c     ORFWorker.obj
 0002:0000b194       __ehfuncinfo$??A?$QMap@VQString@@VQScriptValue@@@@QAEAAVQScriptValue@@ABVQString@@@Z 10031194     ORFWorker.obj
 0002:0000b1b8       __catchsym$??0?$QList@VDescriptor@U2@@@@QAE@ABV0@@Z$2 100311b8     ORFWorker.obj
 0002:0000b1c8       __unwindtable$??0?$QList@VDescriptor@U2@@@@QAE@ABV0@@Z 100311c8     ORFWorker.obj
 0002:0000b1d8       __tryblocktable$??0?$QList@VDescriptor@U2@@@@QAE@ABV0@@Z 100311d8     ORFWorker.obj
 0002:0000b1ec       __ehfuncinfo$??0?$QList@VDescriptor@U2@@@@QAE@ABV0@@Z 100311ec     ORFWorker.obj
 0002:0000b210       __catchsym$?append@?$QList@VDescriptor@U2@@@@QAEXABVDescriptor@U2@@@Z$9 10031210     ORFWorker.obj
 0002:0000b220       __catchsym$?append@?$QList@VDescriptor@U2@@@@QAEXABVDescriptor@U2@@@Z$8 10031220     ORFWorker.obj
 0002:0000b230       __ehfuncinfo$?append@?$QList@VDescriptor@U2@@@@QAEXABVDescriptor@U2@@@Z 10031230     ORFWorker.obj
 0002:0000b254       __tryblocktable$?append@?$QList@VDescriptor@U2@@@@QAEXABVDescriptor@U2@@@Z 10031254     ORFWorker.obj
 0002:0000b27c       __unwindtable$?append@?$QList@VDescriptor@U2@@@@QAEXABVDescriptor@U2@@@Z 1003127c     ORFWorker.obj
 0002:0000b2bc       __catchsym$?detach_helper_grow@?$QList@VDescriptor@U2@@@@AAEPAUNode@1@HH@Z$5 100312bc     ORFWorker.obj
 0002:0000b2cc       __catchsym$?detach_helper_grow@?$QList@VDescriptor@U2@@@@AAEPAUNode@1@HH@Z$4 100312cc     ORFWorker.obj
 0002:0000b2dc       __unwindtable$?detach_helper_grow@?$QList@VDescriptor@U2@@@@AAEPAUNode@1@HH@Z 100312dc     ORFWorker.obj
 0002:0000b2fc       __ehfuncinfo$?detach_helper_grow@?$QList@VDescriptor@U2@@@@AAEPAUNode@1@HH@Z 100312fc     ORFWorker.obj
 0002:0000b320       __tryblocktable$?detach_helper_grow@?$QList@VDescriptor@U2@@@@AAEPAUNode@1@HH@Z 10031320     ORFWorker.obj
 0002:0000b348       __catchsym$?detach_helper@?$QList@VDescriptor@U2@@@@AAEXH@Z$2 10031348     ORFWorker.obj
 0002:0000b358       __unwindtable$?detach_helper@?$QList@VDescriptor@U2@@@@AAEXH@Z 10031358     ORFWorker.obj
 0002:0000b368       __tryblocktable$?detach_helper@?$QList@VDescriptor@U2@@@@AAEXH@Z 10031368     ORFWorker.obj
 0002:0000b37c       __ehfuncinfo$?detach_helper@?$QList@VDescriptor@U2@@@@AAEXH@Z 1003137c     ORFWorker.obj
 0002:0000b3a0       __unwindtable$?node_construct@?$QList@VDescriptor@U2@@@@AAEXPAUNode@1@ABVDescriptor@U2@@@Z 100313a0     ORFWorker.obj
 0002:0000b3b0       __ehfuncinfo$?node_construct@?$QList@VDescriptor@U2@@@@AAEXPAUNode@1@ABVDescriptor@U2@@@Z 100313b0     ORFWorker.obj
 0002:0000b3d4       __catchsym$?node_copy@?$QList@VDescriptor@U2@@@@AAEXPAUNode@1@00@Z$6 100313d4     ORFWorker.obj
 0002:0000b3e4       __tryblocktable$?node_copy@?$QList@VDescriptor@U2@@@@AAEXPAUNode@1@00@Z 100313e4     ORFWorker.obj
 0002:0000b3f8       __ehfuncinfo$?node_copy@?$QList@VDescriptor@U2@@@@AAEXPAUNode@1@00@Z 100313f8     ORFWorker.obj
 0002:0000b41c       __unwindtable$?node_copy@?$QList@VDescriptor@U2@@@@AAEXPAUNode@1@00@Z 1003141c     ORFWorker.obj
 0002:0000b44c       __unwindtable$??A?$QMap@VDescriptor@U2@@V?$QExplicitlySharedDataPointer@VDataType@U2@@@@@@QAEAAV?$QExplicitlySharedDataPointer@VDataType@U2@@@@ABVDescriptor@U2@@@Z 1003144c     ORFWorker.obj
 0002:0000b454       __ehfuncinfo$??A?$QMap@VDescriptor@U2@@V?$QExplicitlySharedDataPointer@VDataType@U2@@@@@@QAEAAV?$QExplicitlySharedDataPointer@VDataType@U2@@@@ABVDescriptor@U2@@@Z 10031454     ORFWorker.obj
 0002:0000b478       __unwindtable$?qt_metatype_id@?$QMetaTypeId@V?$QSharedDataPointer@VDbiDataHandler@Workflow@U2@@@@@@SAHXZ 10031478     ORFWorker.obj
 0002:0000b480       __ehfuncinfo$?qt_metatype_id@?$QMetaTypeId@V?$QSharedDataPointer@VDbiDataHandler@Workflow@U2@@@@@@SAHXZ 10031480     ORFWorker.obj
 0002:0000b4a4       __unwindtable$??$qRegisterMetaType@V?$QSharedDataPointer@VDbiDataHandler@Workflow@U2@@@@@@YAHPBDPAV?$QSharedDataPointer@VDbiDataHandler@Workflow@U2@@@@W4DefinedType@?$MetaTypeDefinedHelper@V?$QSharedDataPointer@VDbiDataHandler@Workflow@U2@@@@$00@QtPrivate@@@Z 100314a4     ORFWorker.obj
 0002:0000b4ac       __ehfuncinfo$??$qRegisterMetaType@V?$QSharedDataPointer@VDbiDataHandler@Workflow@U2@@@@@@YAHPBDPAV?$QSharedDataPointer@VDbiDataHandler@Workflow@U2@@@@W4DefinedType@?$MetaTypeDefinedHelper@V?$QSharedDataPointer@VDbiDataHandler@Workflow@U2@@@@$00@QtPrivate@@@Z 100314ac     ORFWorker.obj
 0002:0000b4d0       __unwindtable$?uniqueKeys@?$QMap@VDescriptor@U2@@VQVariant@@@@QBE?AV?$QList@VDescriptor@U2@@@@XZ 100314d0     ORFWorker.obj
 0002:0000b4d8       __ehfuncinfo$?uniqueKeys@?$QMap@VDescriptor@U2@@VQVariant@@@@QBE?AV?$QList@VDescriptor@U2@@@@XZ 100314d8     ORFWorker.obj
 0002:0000b4fc       __ehfuncinfo$??$getAttributeValue@VQString@@@Attribute@U2@@QBE?AVQString@@PAVWorkflowContext@Workflow@1@@Z 100314fc     ORFWorker.obj
 0002:0000b520       __unwindtable$??$getAttributeValue@VQString@@@Attribute@U2@@QBE?AVQString@@PAVWorkflowContext@Workflow@1@@Z 10031520     ORFWorker.obj
 0002:0000b590       __ehfuncinfo$??$getAttributeValue@H@Attribute@U2@@QBEHPAVWorkflowContext@Workflow@1@@Z 10031590     ORFWorker.obj
 0002:0000b5b4       __unwindtable$??$getAttributeValue@H@Attribute@U2@@QBEHPAVWorkflowContext@Workflow@1@@Z 100315b4     ORFWorker.obj
 0002:0000b61c       __catchsym$?append@?$QList@PAVPortDescriptor@Workflow@U2@@@@QAEXABQAVPortDescriptor@Workflow@U2@@@Z$6 1003161c     ORFWorker.obj
 0002:0000b62c       __tryblocktable$?append@?$QList@PAVPortDescriptor@Workflow@U2@@@@QAEXABQAVPortDescriptor@Workflow@U2@@@Z 1003162c     ORFWorker.obj
 0002:0000b640       __ehfuncinfo$?append@?$QList@PAVPortDescriptor@Workflow@U2@@@@QAEXABQAVPortDescriptor@Workflow@U2@@@Z 10031640     ORFWorker.obj
 0002:0000b664       __unwindtable$?append@?$QList@PAVPortDescriptor@Workflow@U2@@@@QAEXABQAVPortDescriptor@Workflow@U2@@@Z 10031664     ORFWorker.obj
 0002:0000b694       __catchsym$?detach_helper_grow@?$QList@PAVPortDescriptor@Workflow@U2@@@@AAEPAUNode@1@HH@Z$5 10031694     ORFWorker.obj
 0002:0000b6a4       __catchsym$?detach_helper_grow@?$QList@PAVPortDescriptor@Workflow@U2@@@@AAEPAUNode@1@HH@Z$4 100316a4     ORFWorker.obj
 0002:0000b6b4       __unwindtable$?detach_helper_grow@?$QList@PAVPortDescriptor@Workflow@U2@@@@AAEPAUNode@1@HH@Z 100316b4     ORFWorker.obj
 0002:0000b6d4       __ehfuncinfo$?detach_helper_grow@?$QList@PAVPortDescriptor@Workflow@U2@@@@AAEPAUNode@1@HH@Z 100316d4     ORFWorker.obj
 0002:0000b6f8       __tryblocktable$?detach_helper_grow@?$QList@PAVPortDescriptor@Workflow@U2@@@@AAEPAUNode@1@HH@Z 100316f8     ORFWorker.obj
 0002:0000b720       __unwindtable$??0?$QPair@VQString@@V1@@@QAE@ABVQString@@0@Z 10031720     ORFWorker.obj
 0002:0000b728       __ehfuncinfo$??0?$QPair@VQString@@V1@@@QAE@ABVQString@@0@Z 10031728     ORFWorker.obj
 0002:0000b74c       __unwindtable$??1?$QPair@VQString@@V1@@@QAE@XZ 1003174c     ORFWorker.obj
 0002:0000b754       __ehfuncinfo$??1?$QPair@VQString@@V1@@@QAE@XZ 10031754     ORFWorker.obj
 0002:0000b778       __ehfuncinfo$?createDescription@?$PrompterBase@VORFPrompter@LocalWorkflow@U2@@@U2@@UAEPAVActorDocument@Workflow@2@PAVActor@42@@Z 10031778     ORFWorker.obj
 0002:0000b79c       __unwindtable$?createDescription@?$PrompterBase@VORFPrompter@LocalWorkflow@U2@@@U2@@UAEPAVActorDocument@Workflow@2@PAVActor@42@@Z 1003179c     ORFWorker.obj
 0002:0000b7d4       __ehfuncinfo$?composeRichDoc@ORFPrompter@LocalWorkflow@U2@@MAE?AVQString@@XZ 100317d4     ORFWorker.obj
 0002:0000b7f8       __unwindtable$?composeRichDoc@ORFPrompter@LocalWorkflow@U2@@MAE?AVQString@@XZ 100317f8     ORFWorker.obj
 0002:0000ba00       __unwindtable$??0ORFWorker@LocalWorkflow@U2@@QAE@PAVActor@Workflow@2@@Z 10031a00     ORFWorker.obj
 0002:0000ba10       __ehfuncinfo$??0ORFWorker@LocalWorkflow@U2@@QAE@PAVActor@Workflow@2@@Z 10031a10     ORFWorker.obj
 0002:0000ba34       __unwindtable$?init@ORFWorker@LocalWorkflow@U2@@UAEXXZ 10031a34     ORFWorker.obj
 0002:0000ba44       __ehfuncinfo$?init@ORFWorker@LocalWorkflow@U2@@UAEXXZ 10031a44     ORFWorker.obj
 0002:0000ba68       __ehfuncinfo$?tick@ORFWorker@LocalWorkflow@U2@@UAEPAVTask@3@XZ 10031a68     ORFWorker.obj
 0002:0000ba8c       __unwindtable$?tick@ORFWorker@LocalWorkflow@U2@@UAEPAVTask@3@XZ 10031a8c     ORFWorker.obj
 0002:0000bb94       __ehfuncinfo$?sl_taskFinished@ORFWorker@LocalWorkflow@U2@@AAEXXZ 10031b94     ORFWorker.obj
 0002:0000bbb8       __unwindtable$?sl_taskFinished@ORFWorker@LocalWorkflow@U2@@AAEXXZ 10031bb8     ORFWorker.obj
 0002:0000bbf0       __unwindtable$??1ORFWorker@LocalWorkflow@U2@@UAE@XZ 10031bf0     ORFWorker.obj
 0002:0000bc00       __ehfuncinfo$??1ORFWorker@LocalWorkflow@U2@@UAE@XZ 10031c00     ORFWorker.obj
 0002:0000bc24       __unwindtable$??_GORFWorker@LocalWorkflow@U2@@UAEPAXI@Z 10031c24     ORFWorker.obj
 0002:0000bc34       __ehfuncinfo$??_GORFWorker@LocalWorkflow@U2@@UAEPAXI@Z 10031c34     ORFWorker.obj
 0002:0000bc58       __ehfuncinfo$?init@ORFWorkerFactory@LocalWorkflow@U2@@SAXXZ 10031c58     ORFWorker.obj
 0002:0000bc7c       __unwindtable$?init@ORFWorkerFactory@LocalWorkflow@U2@@SAXXZ 10031c7c     ORFWorker.obj
 0002:0000c12c       __unwindtable$?createWorker@ORFWorkerFactory@LocalWorkflow@U2@@UAEPAVWorker@Workflow@3@PAVActor@53@@Z 1003212c     ORFWorker.obj
 0002:0000c134       __ehfuncinfo$?createWorker@ORFWorkerFactory@LocalWorkflow@U2@@UAEPAVWorker@Workflow@3@PAVActor@53@@Z 10032134     ORFWorker.obj
 0002:0000c158       __catchsym$?append@?$QList@U?$QPair@VQString@@VQVariant@@@@@@QAEXABU?$QPair@VQString@@VQVariant@@@@@Z$7 10032158     ORFWorker.obj
 0002:0000c168       __catchsym$?append@?$QList@U?$QPair@VQString@@VQVariant@@@@@@QAEXABU?$QPair@VQString@@VQVariant@@@@@Z$6 10032168     ORFWorker.obj
 0002:0000c178       __ehfuncinfo$?append@?$QList@U?$QPair@VQString@@VQVariant@@@@@@QAEXABU?$QPair@VQString@@VQVariant@@@@@Z 10032178     ORFWorker.obj
 0002:0000c19c       __tryblocktable$?append@?$QList@U?$QPair@VQString@@VQVariant@@@@@@QAEXABU?$QPair@VQString@@VQVariant@@@@@Z 1003219c     ORFWorker.obj
 0002:0000c1c4       __unwindtable$?append@?$QList@U?$QPair@VQString@@VQVariant@@@@@@QAEXABU?$QPair@VQString@@VQVariant@@@@@Z 100321c4     ORFWorker.obj
 0002:0000c1f4       __catchsym$?detach_helper_grow@?$QList@U?$QPair@VQString@@VQVariant@@@@@@AAEPAUNode@1@HH@Z$5 100321f4     ORFWorker.obj
 0002:0000c204       __catchsym$?detach_helper_grow@?$QList@U?$QPair@VQString@@VQVariant@@@@@@AAEPAUNode@1@HH@Z$4 10032204     ORFWorker.obj
 0002:0000c214       __unwindtable$?detach_helper_grow@?$QList@U?$QPair@VQString@@VQVariant@@@@@@AAEPAUNode@1@HH@Z 10032214     ORFWorker.obj
 0002:0000c234       __ehfuncinfo$?detach_helper_grow@?$QList@U?$QPair@VQString@@VQVariant@@@@@@AAEPAUNode@1@HH@Z 10032234     ORFWorker.obj
 0002:0000c258       __tryblocktable$?detach_helper_grow@?$QList@U?$QPair@VQString@@VQVariant@@@@@@AAEPAUNode@1@HH@Z 10032258     ORFWorker.obj
 0002:0000c280       __unwindtable$?node_construct@?$QList@U?$QPair@VQString@@VQVariant@@@@@@AAEXPAUNode@1@ABU?$QPair@VQString@@VQVariant@@@@@Z 10032280     ORFWorker.obj
 0002:0000c2a0       __ehfuncinfo$?node_construct@?$QList@U?$QPair@VQString@@VQVariant@@@@@@AAEXPAUNode@1@ABU?$QPair@VQString@@VQVariant@@@@@Z 100322a0     ORFWorker.obj
 0002:0000c2c4       __unwindtable$?node_destruct@?$QList@U?$QPair@VQString@@VQVariant@@@@@@AAEXPAUNode@1@@Z 100322c4     ORFWorker.obj
 0002:0000c2d4       __ehfuncinfo$?node_destruct@?$QList@U?$QPair@VQString@@VQVariant@@@@@@AAEXPAUNode@1@@Z 100322d4     ORFWorker.obj
 0002:0000c2f8       __catchsym$?node_copy@?$QList@U?$QPair@VQString@@VQVariant@@@@@@AAEXPAUNode@1@00@Z$14 100322f8     ORFWorker.obj
 0002:0000c308       __tryblocktable$?node_copy@?$QList@U?$QPair@VQString@@VQVariant@@@@@@AAEXPAUNode@1@00@Z 10032308     ORFWorker.obj
 0002:0000c31c       __ehfuncinfo$?node_copy@?$QList@U?$QPair@VQString@@VQVariant@@@@@@AAEXPAUNode@1@00@Z 1003231c     ORFWorker.obj
 0002:0000c340       __unwindtable$?node_copy@?$QList@U?$QPair@VQString@@VQVariant@@@@@@AAEXPAUNode@1@00@Z 10032340     ORFWorker.obj
 0002:0000c390       __unwindtable$?node_destruct@?$QList@U?$QPair@VQString@@VQVariant@@@@@@AAEXPAUNode@1@0@Z 10032390     ORFWorker.obj
 0002:0000c3a0       __ehfuncinfo$?node_destruct@?$QList@U?$QPair@VQString@@VQVariant@@@@@@AAEXPAUNode@1@0@Z 100323a0     ORFWorker.obj
 0002:0000c3c4       __unwindtable$??$qMakePair@VQString@@V1@@@YA?AU?$QPair@VQString@@V1@@@ABVQString@@0@Z 100323c4     ORFWorker.obj
 0002:0000c3cc       __ehfuncinfo$??$qMakePair@VQString@@V1@@@YA?AU?$QPair@VQString@@V1@@@ABVQString@@0@Z 100323cc     ORFWorker.obj
 0002:0000c3f0       __unwindtable$??1?$QPair@VQString@@VQVariant@@@@QAE@XZ 100323f0     ORFWorker.obj
 0002:0000c3f8       __ehfuncinfo$??1?$QPair@VQString@@VQVariant@@@@QAE@XZ 100323f8     ORFWorker.obj
 0002:0000c41c       __unwindtable$??0?$QPair@VQString@@VQVariant@@@@QAE@ABU0@@Z 1003241c     ORFWorker.obj
 0002:0000c424       __ehfuncinfo$??0?$QPair@VQString@@VQVariant@@@@QAE@ABU0@@Z 10032424     ORFWorker.obj
 0002:0000c448       __unwindtable$??_G?$QPair@VQString@@VQVariant@@@@QAEPAXI@Z 10032448     ORFWorker.obj
 0002:0000c450       __ehfuncinfo$??_G?$QPair@VQString@@VQVariant@@@@QAEPAXI@Z 10032450     ORFWorker.obj
 0002:0000c474       __unwindtable$??$?0VQString@@V0@@?$QPair@VQString@@VQVariant@@@@QAE@$$QAU?$QPair@VQString@@V1@@@@Z 10032474     ORFWorker.obj
 0002:0000c47c       __ehfuncinfo$??$?0VQString@@V0@@?$QPair@VQString@@VQVariant@@@@QAE@$$QAU?$QPair@VQString@@V1@@@@Z 1003247c     ORFWorker.obj
 0002:0000c4a0       __unwindtable$?getStrand@LocalWorkflow@U2@@YA?AW4ORFAlgorithmStrand@2@ABVQString@@@Z 100324a0     ORFWorker.obj
 0002:0000c4c0       __ehfuncinfo$?getStrand@LocalWorkflow@U2@@YA?AW4ORFAlgorithmStrand@2@ABVQString@@@Z 100324c0     ORFWorker.obj
 0002:0000c4e4       __catchsym$?createNode@?$QMapData@VQString@@VQScriptValue@@@@QAEPAU?$QMapNode@VQString@@VQScriptValue@@@@ABVQString@@ABVQScriptValue@@PAU2@_N@Z$7 100324e4     ORFWorker.obj
 0002:0000c4f4       __catchsym$?createNode@?$QMapData@VQString@@VQScriptValue@@@@QAEPAU?$QMapNode@VQString@@VQScriptValue@@@@ABVQString@@ABVQScriptValue@@PAU2@_N@Z$6 100324f4     ORFWorker.obj
 0002:0000c504       __ehfuncinfo$?createNode@?$QMapData@VQString@@VQScriptValue@@@@QAEPAU?$QMapNode@VQString@@VQScriptValue@@@@ABVQString@@ABVQScriptValue@@PAU2@_N@Z 10032504     ORFWorker.obj
 0002:0000c528       __tryblocktable$?createNode@?$QMapData@VQString@@VQScriptValue@@@@QAEPAU?$QMapNode@VQString@@VQScriptValue@@@@ABVQString@@ABVQScriptValue@@PAU2@_N@Z 10032528     ORFWorker.obj
 0002:0000c550       __unwindtable$?createNode@?$QMapData@VQString@@VQScriptValue@@@@QAEPAU?$QMapNode@VQString@@VQScriptValue@@@@ABVQString@@ABVQScriptValue@@PAU2@_N@Z 10032550     ORFWorker.obj
 0002:0000c580       __catchsym$?createNode@?$QMapData@VDescriptor@U2@@V?$QExplicitlySharedDataPointer@VDataType@U2@@@@@@QAEPAU?$QMapNode@VDescriptor@U2@@V?$QExplicitlySharedDataPointer@VDataType@U2@@@@@@ABVDescriptor@U2@@ABV?$QExplicitlySharedDataPointer@VDataType@U2@@@@PAU2@_N@Z$6 10032580     ORFWorker.obj
 0002:0000c590       __tryblocktable$?createNode@?$QMapData@VDescriptor@U2@@V?$QExplicitlySharedDataPointer@VDataType@U2@@@@@@QAEPAU?$QMapNode@VDescriptor@U2@@V?$QExplicitlySharedDataPointer@VDataType@U2@@@@@@ABVDescriptor@U2@@ABV?$QExplicitlySharedDataPointer@VDataType@U2@@@@PAU2@_N@Z 10032590     ORFWorker.obj
 0002:0000c5a4       __ehfuncinfo$?createNode@?$QMapData@VDescriptor@U2@@V?$QExplicitlySharedDataPointer@VDataType@U2@@@@@@QAEPAU?$QMapNode@VDescriptor@U2@@V?$QExplicitlySharedDataPointer@VDataType@U2@@@@@@ABVDescriptor@U2@@ABV?$QExplicitlySharedDataPointer@VDataType@U2@@@@PAU2@_N@Z 100325a4     ORFWorker.obj
 0002:0000c5c8       __unwindtable$?createNode@?$QMapData@VDescriptor@U2@@V?$QExplicitlySharedDataPointer@VDataType@U2@@@@@@QAEPAU?$QMapNode@VDescriptor@U2@@V?$QExplicitlySharedDataPointer@VDataType@U2@@@@@@ABVDescriptor@U2@@ABV?$QExplicitlySharedDataPointer@VDataType@U2@@@@PAU2@_N@Z 100325c8     ORFWorker.obj
 0002:0000c5f0       __catchsym$??0?$QList@PAVPort@Workflow@U2@@@@QAE@ABV0@@Z$2 100325f0     ORFWorker.obj
 0002:0000c600       __unwindtable$??0?$QList@PAVPort@Workflow@U2@@@@QAE@ABV0@@Z 10032600     ORFWorker.obj
 0002:0000c610       __tryblocktable$??0?$QList@PAVPort@Workflow@U2@@@@QAE@ABV0@@Z 10032610     ORFWorker.obj
 0002:0000c624       __ehfuncinfo$??0?$QList@PAVPort@Workflow@U2@@@@QAE@ABV0@@Z 10032624     ORFWorker.obj
 0002:0000c648       __unwindtable$?metaType@?$QVariantValueHelper@V?$QSharedDataPointer@VDbiDataHandler@Workflow@U2@@@@@QtPrivate@@SA?AV?$QSharedDataPointer@VDbiDataHandler@Workflow@U2@@@@ABVQVariant@@@Z 10032648     ORFWorker.obj
 0002:0000c658       __ehfuncinfo$?metaType@?$QVariantValueHelper@V?$QSharedDataPointer@VDbiDataHandler@Workflow@U2@@@@@QtPrivate@@SA?AV?$QSharedDataPointer@VDbiDataHandler@Workflow@U2@@@@ABVQVariant@@@Z 10032658     ORFWorker.obj
 0002:0000c67c       __unwindtable$??__EalgoLog@U2@@YAXXZ 1003267c     moc_ORFDialog.obj
 0002:0000c684       __ehfuncinfo$??__EalgoLog@U2@@YAXXZ 10032684     moc_ORFDialog.obj
 0002:0000c6a8       __unwindtable$??__EcmdLog@U2@@YAXXZ 100326a8     moc_ORFDialog.obj
 0002:0000c6b0       __ehfuncinfo$??__EcmdLog@U2@@YAXXZ 100326b0     moc_ORFDialog.obj
 0002:0000c6d4       __unwindtable$??__EcoreLog@U2@@YAXXZ 100326d4     moc_ORFDialog.obj
 0002:0000c6dc       __ehfuncinfo$??__EcoreLog@U2@@YAXXZ 100326dc     moc_ORFDialog.obj
 0002:0000c700       __unwindtable$??__EioLog@U2@@YAXXZ 10032700     moc_ORFDialog.obj
 0002:0000c708       __ehfuncinfo$??__EioLog@U2@@YAXXZ 10032708     moc_ORFDialog.obj
 0002:0000c72c       __unwindtable$??__EperfLog@U2@@YAXXZ 1003272c     moc_ORFDialog.obj
 0002:0000c734       __ehfuncinfo$??__EperfLog@U2@@YAXXZ 10032734     moc_ORFDialog.obj
 0002:0000c758       __unwindtable$??__EscriptLog@U2@@YAXXZ 10032758     moc_ORFDialog.obj
 0002:0000c760       __ehfuncinfo$??__EscriptLog@U2@@YAXXZ 10032760     moc_ORFDialog.obj
 0002:0000c784       __unwindtable$??__EtaskLog@U2@@YAXXZ 10032784     moc_ORFDialog.obj
 0002:0000c78c       __ehfuncinfo$??__EtaskLog@U2@@YAXXZ 1003278c     moc_ORFDialog.obj
 0002:0000c7b0       __unwindtable$??__EuiLog@U2@@YAXXZ 100327b0     moc_ORFDialog.obj
 0002:0000c7b8       __ehfuncinfo$??__EuiLog@U2@@YAXXZ 100327b8     moc_ORFDialog.obj
 0002:0000c7dc       __unwindtable$??__EuserActLog@U2@@YAXXZ 100327dc     moc_ORFDialog.obj
 0002:0000c7e4       __ehfuncinfo$??__EuserActLog@U2@@YAXXZ 100327e4     moc_ORFDialog.obj
 0002:0000c808       __unwindtable$?qt_metatype_id@?$QMetaTypeIdQObject@PAVTask@U2@@$00@@SAHXZ 10032808     moc_ORFDialog.obj
 0002:0000c810       __ehfuncinfo$?qt_metatype_id@?$QMetaTypeIdQObject@PAVTask@U2@@$00@@SAHXZ 10032810     moc_ORFDialog.obj
 0002:0000c834       __unwindtable$??__EalgoLog@U2@@YAXXZ 10032834     moc_ORFMarkerTask.obj
 0002:0000c83c       __ehfuncinfo$??__EalgoLog@U2@@YAXXZ 1003283c     moc_ORFMarkerTask.obj
 0002:0000c860       __unwindtable$??__EcmdLog@U2@@YAXXZ 10032860     moc_ORFMarkerTask.obj
 0002:0000c868       __ehfuncinfo$??__EcmdLog@U2@@YAXXZ 10032868     moc_ORFMarkerTask.obj
 0002:0000c88c       __unwindtable$??__EcoreLog@U2@@YAXXZ 1003288c     moc_ORFMarkerTask.obj
 0002:0000c894       __ehfuncinfo$??__EcoreLog@U2@@YAXXZ 10032894     moc_ORFMarkerTask.obj
 0002:0000c8b8       __unwindtable$??__EioLog@U2@@YAXXZ 100328b8     moc_ORFMarkerTask.obj
 0002:0000c8c0       __ehfuncinfo$??__EioLog@U2@@YAXXZ 100328c0     moc_ORFMarkerTask.obj
 0002:0000c8e4       __unwindtable$??__EperfLog@U2@@YAXXZ 100328e4     moc_ORFMarkerTask.obj
 0002:0000c8ec       __ehfuncinfo$??__EperfLog@U2@@YAXXZ 100328ec     moc_ORFMarkerTask.obj
 0002:0000c910       __unwindtable$??__EscriptLog@U2@@YAXXZ 10032910     moc_ORFMarkerTask.obj
 0002:0000c918       __ehfuncinfo$??__EscriptLog@U2@@YAXXZ 10032918     moc_ORFMarkerTask.obj
 0002:0000c93c       __unwindtable$??__EtaskLog@U2@@YAXXZ 1003293c     moc_ORFMarkerTask.obj
 0002:0000c944       __ehfuncinfo$??__EtaskLog@U2@@YAXXZ 10032944     moc_ORFMarkerTask.obj
 0002:0000c968       __unwindtable$??__EuiLog@U2@@YAXXZ 10032968     moc_ORFMarkerTask.obj
 0002:0000c970       __ehfuncinfo$??__EuiLog@U2@@YAXXZ 10032970     moc_ORFMarkerTask.obj
 0002:0000c994       __unwindtable$??__EuserActLog@U2@@YAXXZ 10032994     moc_ORFMarkerTask.obj
 0002:0000c99c       __ehfuncinfo$??__EuserActLog@U2@@YAXXZ 1003299c     moc_ORFMarkerTask.obj
 0002:0000c9c0       __unwindtable$??__EalgoLog@U2@@YAXXZ 100329c0     moc_ORFMarkerTests.obj
 0002:0000c9c8       __ehfuncinfo$??__EalgoLog@U2@@YAXXZ 100329c8     moc_ORFMarkerTests.obj
 0002:0000c9ec       __unwindtable$??__EcmdLog@U2@@YAXXZ 100329ec     moc_ORFMarkerTests.obj
 0002:0000c9f4       __ehfuncinfo$??__EcmdLog@U2@@YAXXZ 100329f4     moc_ORFMarkerTests.obj
 0002:0000ca18       __unwindtable$??__EcoreLog@U2@@YAXXZ 10032a18     moc_ORFMarkerTests.obj
 0002:0000ca20       __ehfuncinfo$??__EcoreLog@U2@@YAXXZ 10032a20     moc_ORFMarkerTests.obj
 0002:0000ca44       __unwindtable$??__EioLog@U2@@YAXXZ 10032a44     moc_ORFMarkerTests.obj
 0002:0000ca4c       __ehfuncinfo$??__EioLog@U2@@YAXXZ 10032a4c     moc_ORFMarkerTests.obj
 0002:0000ca70       __unwindtable$??__EperfLog@U2@@YAXXZ 10032a70     moc_ORFMarkerTests.obj
 0002:0000ca78       __ehfuncinfo$??__EperfLog@U2@@YAXXZ 10032a78     moc_ORFMarkerTests.obj
 0002:0000ca9c       __unwindtable$??__EscriptLog@U2@@YAXXZ 10032a9c     moc_ORFMarkerTests.obj
 0002:0000caa4       __ehfuncinfo$??__EscriptLog@U2@@YAXXZ 10032aa4     moc_ORFMarkerTests.obj
 0002:0000cac8       __unwindtable$??__EtaskLog@U2@@YAXXZ 10032ac8     moc_ORFMarkerTests.obj
 0002:0000cad0       __ehfuncinfo$??__EtaskLog@U2@@YAXXZ 10032ad0     moc_ORFMarkerTests.obj
 0002:0000caf4       __unwindtable$??__EuiLog@U2@@YAXXZ 10032af4     moc_ORFMarkerTests.obj
 0002:0000cafc       __ehfuncinfo$??__EuiLog@U2@@YAXXZ 10032afc     moc_ORFMarkerTests.obj
 0002:0000cb20       __unwindtable$??__EuserActLog@U2@@YAXXZ 10032b20     moc_ORFMarkerTests.obj
 0002:0000cb28       __ehfuncinfo$??__EuserActLog@U2@@YAXXZ 10032b28     moc_ORFMarkerTests.obj
 0002:0000cb4c       __unwindtable$??__EalgoLog@U2@@YAXXZ 10032b4c     moc_ORFQuery.obj
 0002:0000cb54       __ehfuncinfo$??__EalgoLog@U2@@YAXXZ 10032b54     moc_ORFQuery.obj
 0002:0000cb78       __unwindtable$??__EcmdLog@U2@@YAXXZ 10032b78     moc_ORFQuery.obj
 0002:0000cb80       __ehfuncinfo$??__EcmdLog@U2@@YAXXZ 10032b80     moc_ORFQuery.obj
 0002:0000cba4       __unwindtable$??__EcoreLog@U2@@YAXXZ 10032ba4     moc_ORFQuery.obj
 0002:0000cbac       __ehfuncinfo$??__EcoreLog@U2@@YAXXZ 10032bac     moc_ORFQuery.obj
 0002:0000cbd0       __unwindtable$??__EioLog@U2@@YAXXZ 10032bd0     moc_ORFQuery.obj
 0002:0000cbd8       __ehfuncinfo$??__EioLog@U2@@YAXXZ 10032bd8     moc_ORFQuery.obj
 0002:0000cbfc       __unwindtable$??__EperfLog@U2@@YAXXZ 10032bfc     moc_ORFQuery.obj
 0002:0000cc04       __ehfuncinfo$??__EperfLog@U2@@YAXXZ 10032c04     moc_ORFQuery.obj
 0002:0000cc28       __unwindtable$??__EscriptLog@U2@@YAXXZ 10032c28     moc_ORFQuery.obj
 0002:0000cc30       __ehfuncinfo$??__EscriptLog@U2@@YAXXZ 10032c30     moc_ORFQuery.obj
 0002:0000cc54       __unwindtable$??__EtaskLog@U2@@YAXXZ 10032c54     moc_ORFQuery.obj
 0002:0000cc5c       __ehfuncinfo$??__EtaskLog@U2@@YAXXZ 10032c5c     moc_ORFQuery.obj
 0002:0000cc80       __unwindtable$??__EuiLog@U2@@YAXXZ 10032c80     moc_ORFQuery.obj
 0002:0000cc88       __ehfuncinfo$??__EuiLog@U2@@YAXXZ 10032c88     moc_ORFQuery.obj
 0002:0000ccac       __unwindtable$??__EuserActLog@U2@@YAXXZ 10032cac     moc_ORFQuery.obj
 0002:0000ccb4       __ehfuncinfo$??__EuserActLog@U2@@YAXXZ 10032cb4     moc_ORFQuery.obj
 0002:0000ccd8       __unwindtable$??__EalgoLog@U2@@YAXXZ 10032cd8     moc_ORFWorker.obj
 0002:0000cce0       __ehfuncinfo$??__EalgoLog@U2@@YAXXZ 10032ce0     moc_ORFWorker.obj
 0002:0000cd04       __unwindtable$??__EcmdLog@U2@@YAXXZ 10032d04     moc_ORFWorker.obj
 0002:0000cd0c       __ehfuncinfo$??__EcmdLog@U2@@YAXXZ 10032d0c     moc_ORFWorker.obj
 0002:0000cd30       __unwindtable$??__EcoreLog@U2@@YAXXZ 10032d30     moc_ORFWorker.obj
 0002:0000cd38       __ehfuncinfo$??__EcoreLog@U2@@YAXXZ 10032d38     moc_ORFWorker.obj
 0002:0000cd5c       __unwindtable$??__EioLog@U2@@YAXXZ 10032d5c     moc_ORFWorker.obj
 0002:0000cd64       __ehfuncinfo$??__EioLog@U2@@YAXXZ 10032d64     moc_ORFWorker.obj
 0002:0000cd88       __unwindtable$??__EperfLog@U2@@YAXXZ 10032d88     moc_ORFWorker.obj
 0002:0000cd90       __ehfuncinfo$??__EperfLog@U2@@YAXXZ 10032d90     moc_ORFWorker.obj
 0002:0000cdb4       __unwindtable$??__EscriptLog@U2@@YAXXZ 10032db4     moc_ORFWorker.obj
 0002:0000cdbc       __ehfuncinfo$??__EscriptLog@U2@@YAXXZ 10032dbc     moc_ORFWorker.obj
 0002:0000cde0       __unwindtable$??__EtaskLog@U2@@YAXXZ 10032de0     moc_ORFWorker.obj
 0002:0000cde8       __ehfuncinfo$??__EtaskLog@U2@@YAXXZ 10032de8     moc_ORFWorker.obj
 0002:0000ce0c       __unwindtable$??__EuiLog@U2@@YAXXZ 10032e0c     moc_ORFWorker.obj
 0002:0000ce14       __ehfuncinfo$??__EuiLog@U2@@YAXXZ 10032e14     moc_ORFWorker.obj
 0002:0000ce38       __unwindtable$??__EuserActLog@U2@@YAXXZ 10032e38     moc_ORFWorker.obj
 0002:0000ce40       __ehfuncinfo$??__EuserActLog@U2@@YAXXZ 10032e40     moc_ORFWorker.obj
 0002:0000ce68       __sehtable$__onexit        10032e68     MSVCRT:atonexit.obj
 0002:0000ce88       __sehtable$___DllMainCRTStartup 10032e88     MSVCRT:crtdll.obj
 0002:0000ceb0       __sehtable$??_M@YGXPAXIHP6EX0@Z@Z 10032eb0     MSVCRT:ehvecdtr.obj
 0002:0000ced0       __sehtable$?__ArrayUnwind@@YGXPAXIHP6EX0@Z@Z 10032ed0     MSVCRT:ehvecdtr.obj
 0002:0000cef0       __sehtable$__IsNonwritableInCurrentImage 10032ef0     MSVCRT:pesect.obj
 0002:0000cf10       .edata                     10032f10     orf_marker.exp
 0002:0000cf38       rgpv                       10032f38     orf_marker.exp
 0002:0000cf3c       rgszName                   10032f3c     orf_marker.exp
 0002:0000cf40       rgwOrd                     10032f40     orf_marker.exp
 0002:0000cf42       szName                     10032f42     orf_marker.exp
 0002:0000cf51       $N00001                    10032f51     orf_marker.exp
 0002:0000f7e8       .idata$6                   100357e8     U2Core:U2Core.dll
 0002:0000fbe6       .idata$6                   10035be6     U2Algorithm:U2Algorithm.dll
 0002:00010722       .idata$6                   10036722     U2Gui:U2Gui.dll
 0002:00010a62       .idata$6                   10036a62     U2View:U2View.dll
 0002:00010cc6       .idata$6                   10036cc6     U2Test:U2Test.dll
 0002:00012f4a       .idata$6                   10038f4a     U2Lang:U2Lang.dll
 0002:0001390e       .idata$6                   1003990e     U2Designer:U2Designer.dll
 0002:00019962       .idata$6                   1003f962     Qt5Widgets:Qt5Widgets.dll
 0002:00019ace       .idata$6                   1003face     Qt5Gui:Qt5Gui.dll
 0002:00019c40       .idata$6                   1003fc40     Qt5Script:Qt5Script.dll
 0002:00019c80       .idata$6                   1003fc80     Qt5Xml:Qt5Xml.dll
 0002:0001adc4       .idata$6                   10040dc4     Qt5Core:Qt5Core.dll
 0002:0001ae6a       .idata$6                   10040e6a     msvcprt:MSVCP120.dll
 0002:0001aef8       .idata$6                   10040ef8     MSVCRT:MSVCR120.dll
 0002:0001b10c       .idata$6                   1004110c     kernel32:KERNEL32.dll
 0003:0000000c       _Service_PluginViewer      1004200c     ORFDialog.obj
 0003:00000014       _Service_Project           10042014     ORFDialog.obj
 0003:0000001c       _Service_ProjectView       1004201c     ORFDialog.obj
 0003:00000024       _Service_DNAGraphPack      10042024     ORFDialog.obj
 0003:0000002c       _Service_DNAExport         1004202c     ORFDialog.obj
 0003:00000034       _Service_TestRunner        10042034     ORFDialog.obj
 0003:0000003c       _Service_ScriptRegistry    1004203c     ORFDialog.obj
 0003:00000044       _Service_ExternalToolSupport 10042044     ORFDialog.obj
 0003:0000004c       _Service_GUITesting        1004204c     ORFDialog.obj
 0003:00000054       _Service_WorkflowDesigner  10042054     ORFDialog.obj
 0003:0000005c       _Service_QueryDesigner     1004205c     ORFDialog.obj
 0003:00000064       _Service_MinCoreServiceId  10042064     ORFDialog.obj
 0003:0000006c       _Service_MaxCoreServiceId  1004206c     ORFDialog.obj
 0003:00000074       _Service_PluginViewer      10042074     ORFMarkerPlugin.obj
 0003:0000007c       _Service_Project           1004207c     ORFMarkerPlugin.obj
 0003:00000084       _Service_ProjectView       10042084     ORFMarkerPlugin.obj
 0003:0000008c       _Service_DNAGraphPack      1004208c     ORFMarkerPlugin.obj
 0003:00000094       _Service_DNAExport         10042094     ORFMarkerPlugin.obj
 0003:0000009c       _Service_TestRunner        1004209c     ORFMarkerPlugin.obj
 0003:000000a4       _Service_ScriptRegistry    100420a4     ORFMarkerPlugin.obj
 0003:000000ac       _Service_ExternalToolSupport 100420ac     ORFMarkerPlugin.obj
 0003:000000b4       _Service_GUITesting        100420b4     ORFMarkerPlugin.obj
 0003:000000bc       _Service_WorkflowDesigner  100420bc     ORFMarkerPlugin.obj
 0003:000000c4       _Service_QueryDesigner     100420c4     ORFMarkerPlugin.obj
 0003:000000cc       _Service_MinCoreServiceId  100420cc     ORFMarkerPlugin.obj
 0003:000000d4       _Service_MaxCoreServiceId  100420d4     ORFMarkerPlugin.obj
 0003:000000dc       _Service_PluginViewer      100420dc     ORFMarkerTests.obj
 0003:000000e4       _Service_Project           100420e4     ORFMarkerTests.obj
 0003:000000ec       _Service_ProjectView       100420ec     ORFMarkerTests.obj
 0003:000000f4       _Service_DNAGraphPack      100420f4     ORFMarkerTests.obj
 0003:000000fc       _Service_DNAExport         100420fc     ORFMarkerTests.obj
 0003:00000104       _Service_TestRunner        10042104     ORFMarkerTests.obj
 0003:0000010c       _Service_ScriptRegistry    1004210c     ORFMarkerTests.obj
 0003:00000114       _Service_ExternalToolSupport 10042114     ORFMarkerTests.obj
 0003:0000011c       _Service_GUITesting        1004211c     ORFMarkerTests.obj
 0003:00000124       _Service_WorkflowDesigner  10042124     ORFMarkerTests.obj
 0003:0000012c       _Service_QueryDesigner     1004212c     ORFMarkerTests.obj
 0003:00000134       _Service_MinCoreServiceId  10042134     ORFMarkerTests.obj
 0003:0000013c       _Service_MaxCoreServiceId  1004213c     ORFMarkerTests.obj
 0003:0000015c       _Service_PluginViewer      1004215c     moc_ORFMarkerPlugin.obj
 0003:00000164       _Service_Project           10042164     moc_ORFMarkerPlugin.obj
 0003:0000016c       _Service_ProjectView       1004216c     moc_ORFMarkerPlugin.obj
 0003:00000174       _Service_DNAGraphPack      10042174     moc_ORFMarkerPlugin.obj
 0003:0000017c       _Service_DNAExport         1004217c     moc_ORFMarkerPlugin.obj
 0003:00000184       _Service_TestRunner        10042184     moc_ORFMarkerPlugin.obj
 0003:0000018c       _Service_ScriptRegistry    1004218c     moc_ORFMarkerPlugin.obj
 0003:00000194       _Service_ExternalToolSupport 10042194     moc_ORFMarkerPlugin.obj
 0003:0000019c       _Service_GUITesting        1004219c     moc_ORFMarkerPlugin.obj
 0003:000001a4       _Service_WorkflowDesigner  100421a4     moc_ORFMarkerPlugin.obj
 0003:000001ac       _Service_QueryDesigner     100421ac     moc_ORFMarkerPlugin.obj
 0003:000001b4       _Service_MinCoreServiceId  100421b4     moc_ORFMarkerPlugin.obj
 0003:000001bc       _Service_MaxCoreServiceId  100421bc     moc_ORFMarkerPlugin.obj
 0003:00000224       _Service_PluginViewer      10042224     moc_ORFMarkerTests.obj
 0003:0000022c       _Service_Project           1004222c     moc_ORFMarkerTests.obj
 0003:00000234       _Service_ProjectView       10042234     moc_ORFMarkerTests.obj
 0003:0000023c       _Service_DNAGraphPack      1004223c     moc_ORFMarkerTests.obj
 0003:00000244       _Service_DNAExport         10042244     moc_ORFMarkerTests.obj
 0003:0000024c       _Service_TestRunner        1004224c     moc_ORFMarkerTests.obj
 0003:00000254       _Service_ScriptRegistry    10042254     moc_ORFMarkerTests.obj
 0003:0000025c       _Service_ExternalToolSupport 1004225c     moc_ORFMarkerTests.obj
 0003:00000264       _Service_GUITesting        10042264     moc_ORFMarkerTests.obj
 0003:0000026c       _Service_WorkflowDesigner  1004226c     moc_ORFMarkerTests.obj
 0003:00000274       _Service_QueryDesigner     10042274     moc_ORFMarkerTests.obj
 0003:0000027c       _Service_MinCoreServiceId  1004227c     moc_ORFMarkerTests.obj
 0003:00000284       _Service_MaxCoreServiceId  10042284     moc_ORFMarkerTests.obj
 0003:00001070       __Tuple_alloc              10043070     ORFDialog.obj
 0003:00001071       _ignore                    10043071     ORFDialog.obj
 0003:00001072       _allocator_arg             10043072     ORFDialog.obj
 0003:00001073       _piecewise_construct       10043073     ORFDialog.obj
 0003:00001074       _taskLog                   10043074     ORFDialog.obj
 0003:0000107c       _algoLog                   1004307c     ORFDialog.obj
 0003:00001084       _userActLog                10043084     ORFDialog.obj
 0003:0000108c       _ioLog                     1004308c     ORFDialog.obj
 0003:00001094       _coreLog                   10043094     ORFDialog.obj
 0003:0000109c       _uiLog                     1004309c     ORFDialog.obj
 0003:000010a4       _scriptLog                 100430a4     ORFDialog.obj
 0003:000010ac       _perfLog                   100430ac     ORFDialog.obj
 0003:000010b4       _cmdLog                    100430b4     ORFDialog.obj
 0003:000010c8       __Tuple_alloc              100430c8     ORFMarkerPlugin.obj
 0003:000010c9       _ignore                    100430c9     ORFMarkerPlugin.obj
 0003:000010ca       _allocator_arg             100430ca     ORFMarkerPlugin.obj
 0003:000010cb       _piecewise_construct       100430cb     ORFMarkerPlugin.obj
 0003:000010cc       _taskLog                   100430cc     ORFMarkerPlugin.obj
 0003:000010d4       _algoLog                   100430d4     ORFMarkerPlugin.obj
 0003:000010dc       _userActLog                100430dc     ORFMarkerPlugin.obj
 0003:000010e4       _ioLog                     100430e4     ORFMarkerPlugin.obj
 0003:000010ec       _coreLog                   100430ec     ORFMarkerPlugin.obj
 0003:000010f4       _uiLog                     100430f4     ORFMarkerPlugin.obj
 0003:000010fc       _scriptLog                 100430fc     ORFMarkerPlugin.obj
 0003:00001104       _perfLog                   10043104     ORFMarkerPlugin.obj
 0003:0000110c       _cmdLog                    1004310c     ORFMarkerPlugin.obj
 0003:00001114       __Tuple_alloc              10043114     ORFMarkerTask.obj
 0003:00001115       _ignore                    10043115     ORFMarkerTask.obj
 0003:00001116       _allocator_arg             10043116     ORFMarkerTask.obj
 0003:00001117       _piecewise_construct       10043117     ORFMarkerTask.obj
 0003:00001118       _taskLog                   10043118     ORFMarkerTask.obj
 0003:00001124       _algoLog                   10043124     ORFMarkerTask.obj
 0003:0000112c       _userActLog                1004312c     ORFMarkerTask.obj
 0003:00001134       _ioLog                     10043134     ORFMarkerTask.obj
 0003:0000113c       _coreLog                   1004313c     ORFMarkerTask.obj
 0003:00001148       _uiLog                     10043148     ORFMarkerTask.obj
 0003:00001150       _scriptLog                 10043150     ORFMarkerTask.obj
 0003:00001160       _perfLog                   10043160     ORFMarkerTask.obj
 0003:00001174       _cmdLog                    10043174     ORFMarkerTask.obj
 0003:00001190       __Tuple_alloc              10043190     ORFMarkerTests.obj
 0003:00001191       _ignore                    10043191     ORFMarkerTests.obj
 0003:00001192       _allocator_arg             10043192     ORFMarkerTests.obj
 0003:00001193       _piecewise_construct       10043193     ORFMarkerTests.obj
 0003:00001194       _taskLog                   10043194     ORFMarkerTests.obj
 0003:0000119c       _algoLog                   1004319c     ORFMarkerTests.obj
 0003:000011a4       _userActLog                100431a4     ORFMarkerTests.obj
 0003:000011ac       _ioLog                     100431ac     ORFMarkerTests.obj
 0003:000011b4       _coreLog                   100431b4     ORFMarkerTests.obj
 0003:000011bc       _uiLog                     100431bc     ORFMarkerTests.obj
 0003:000011c4       _scriptLog                 100431c4     ORFMarkerTests.obj
 0003:000011cc       _perfLog                   100431cc     ORFMarkerTests.obj
 0003:000011d4       _cmdLog                    100431d4     ORFMarkerTests.obj
 0003:000011dc       __Tuple_alloc              100431dc     ORFQuery.obj
 0003:000011dd       _ignore                    100431dd     ORFQuery.obj
 0003:000011de       _allocator_arg             100431de     ORFQuery.obj
 0003:000011df       _piecewise_construct       100431df     ORFQuery.obj
 0003:000011e0       _MAX_LENGTH_ATTR           100431e0     ORFQuery.obj
 0003:000011e4       _taskLog                   100431e4     ORFQuery.obj
 0003:000011ec       _algoLog                   100431ec     ORFQuery.obj
 0003:000011f4       _LIMIT_ATTR                100431f4     ORFQuery.obj
 0003:000011f8       _userActLog                100431f8     ORFQuery.obj
 0003:00001200       _ioLog                     10043200     ORFQuery.obj
 0003:00001208       _coreLog                   10043208     ORFQuery.obj
 0003:00001210       _FIT_ATTR                  10043210     ORFQuery.obj
 0003:00001214       _ID_ATTR                   10043214     ORFQuery.obj
 0003:00001218       _LEN_ATTR                  10043218     ORFQuery.obj
 0003:0000121c       _ALT_ATTR                  1004321c     ORFQuery.obj
 0003:00001220       _uiLog                     10043220     ORFQuery.obj
 0003:00001228       _scriptLog                 10043228     ORFQuery.obj
 0003:00001230       _INIT_ATTR                 10043230     ORFQuery.obj
 0003:00001234       _perfLog                   10043234     ORFQuery.obj
 0003:0000123c       _RES_ATTR                  1004323c     ORFQuery.obj
 0003:00001240       _cmdLog                    10043240     ORFQuery.obj
 0003:00001248       __Tuple_alloc              10043248     ORFWorker.obj
 0003:00001249       _ignore                    10043249     ORFWorker.obj
 0003:0000124a       _allocator_arg             1004324a     ORFWorker.obj
 0003:0000124b       _piecewise_construct       1004324b     ORFWorker.obj
 0003:0000124c       _LIMIT_ATTR                1004324c     ORFWorker.obj
 0003:00001250       _taskLog                   10043250     ORFWorker.obj
 0003:00001258       _algoLog                   10043258     ORFWorker.obj
 0003:00001260       _userActLog                10043260     ORFWorker.obj
 0003:00001268       _ioLog                     10043268     ORFWorker.obj
 0003:00001270       _coreLog                   10043270     ORFWorker.obj
 0003:00001278       _FIT_ATTR                  10043278     ORFWorker.obj
 0003:0000127c       _ID_ATTR                   1004327c     ORFWorker.obj
 0003:00001280       _LEN_ATTR                  10043280     ORFWorker.obj
 0003:00001284       _ALT_ATTR                  10043284     ORFWorker.obj
 0003:00001288       _uiLog                     10043288     ORFWorker.obj
 0003:00001290       _scriptLog                 10043290     ORFWorker.obj
 0003:00001298       _ISC_ATTR                  10043298     ORFWorker.obj
 0003:0000129c       _NAME_ATTR                 1004329c     ORFWorker.obj
 0003:000012a0       _INIT_ATTR                 100432a0     ORFWorker.obj
 0003:000012a4       _perfLog                   100432a4     ORFWorker.obj
 0003:000012ac       _RES_ATTR                  100432ac     ORFWorker.obj
 0003:000012b0       _cmdLog                    100432b0     ORFWorker.obj
 0003:000012c0       __Tuple_alloc              100432c0     moc_ORFDialog.obj
 0003:000012c1       _ignore                    100432c1     moc_ORFDialog.obj
 0003:000012c2       _allocator_arg             100432c2     moc_ORFDialog.obj
 0003:000012c3       _piecewise_construct       100432c3     moc_ORFDialog.obj
 0003:000012c4       _taskLog                   100432c4     moc_ORFDialog.obj
 0003:000012cc       _algoLog                   100432cc     moc_ORFDialog.obj
 0003:000012d4       _userActLog                100432d4     moc_ORFDialog.obj
 0003:000012dc       _ioLog                     100432dc     moc_ORFDialog.obj
 0003:000012e4       _coreLog                   100432e4     moc_ORFDialog.obj
 0003:000012ec       _uiLog                     100432ec     moc_ORFDialog.obj
 0003:000012f4       _scriptLog                 100432f4     moc_ORFDialog.obj
 0003:000012fc       _perfLog                   100432fc     moc_ORFDialog.obj
 0003:00001304       _cmdLog                    10043304     moc_ORFDialog.obj
 0003:00001310       __Tuple_alloc              10043310     moc_ORFMarkerPlugin.obj
 0003:00001311       _ignore                    10043311     moc_ORFMarkerPlugin.obj
 0003:00001312       _allocator_arg             10043312     moc_ORFMarkerPlugin.obj
 0003:00001313       _piecewise_construct       10043313     moc_ORFMarkerPlugin.obj
 0003:00001314       __Tuple_alloc              10043314     moc_ORFMarkerTask.obj
 0003:00001315       _ignore                    10043315     moc_ORFMarkerTask.obj
 0003:00001316       _allocator_arg             10043316     moc_ORFMarkerTask.obj
 0003:00001317       _piecewise_construct       10043317     moc_ORFMarkerTask.obj
 0003:00001318       _taskLog                   10043318     moc_ORFMarkerTask.obj
 0003:00001320       _algoLog                   10043320     moc_ORFMarkerTask.obj
 0003:00001328       _userActLog                10043328     moc_ORFMarkerTask.obj
 0003:00001330       _ioLog                     10043330     moc_ORFMarkerTask.obj
 0003:00001338       _coreLog                   10043338     moc_ORFMarkerTask.obj
 0003:00001340       _uiLog                     10043340     moc_ORFMarkerTask.obj
 0003:00001348       _scriptLog                 10043348     moc_ORFMarkerTask.obj
 0003:00001350       _perfLog                   10043350     moc_ORFMarkerTask.obj
 0003:00001358       _cmdLog                    10043358     moc_ORFMarkerTask.obj
 0003:00001360       __Tuple_alloc              10043360     moc_ORFMarkerTests.obj
 0003:00001361       _ignore                    10043361     moc_ORFMarkerTests.obj
 0003:00001362       _allocator_arg             10043362     moc_ORFMarkerTests.obj
 0003:00001363       _piecewise_construct       10043363     moc_ORFMarkerTests.obj
 0003:00001364       _taskLog                   10043364     moc_ORFMarkerTests.obj
 0003:0000136c       _algoLog                   1004336c     moc_ORFMarkerTests.obj
 0003:00001374       _userActLog                10043374     moc_ORFMarkerTests.obj
 0003:0000137c       _ioLog                     1004337c     moc_ORFMarkerTests.obj
 0003:00001384       _coreLog                   10043384     moc_ORFMarkerTests.obj
 0003:0000138c       _uiLog                     1004338c     moc_ORFMarkerTests.obj
 0003:00001394       _scriptLog                 10043394     moc_ORFMarkerTests.obj
 0003:0000139c       _perfLog                   1004339c     moc_ORFMarkerTests.obj
 0003:000013a4       _cmdLog                    100433a4     moc_ORFMarkerTests.obj
 0003:000013ac       __Tuple_alloc              100433ac     moc_ORFQuery.obj
 0003:000013ad       _ignore                    100433ad     moc_ORFQuery.obj
 0003:000013ae       _allocator_arg             100433ae     moc_ORFQuery.obj
 0003:000013af       _piecewise_construct       100433af     moc_ORFQuery.obj
 0003:000013b0       _taskLog                   100433b0     moc_ORFQuery.obj
 0003:000013b8       _algoLog                   100433b8     moc_ORFQuery.obj
 0003:000013c0       _userActLog                100433c0     moc_ORFQuery.obj
 0003:000013c8       _ioLog                     100433c8     moc_ORFQuery.obj
 0003:000013d0       _coreLog                   100433d0     moc_ORFQuery.obj
 0003:000013d8       _uiLog                     100433d8     moc_ORFQuery.obj
 0003:000013e0       _scriptLog                 100433e0     moc_ORFQuery.obj
 0003:000013e8       _perfLog                   100433e8     moc_ORFQuery.obj
 0003:000013f0       _cmdLog                    100433f0     moc_ORFQuery.obj
 0003:000013f8       __Tuple_alloc              100433f8     moc_ORFWorker.obj
 0003:000013f9       _ignore                    100433f9     moc_ORFWorker.obj
 0003:000013fa       _allocator_arg             100433fa     moc_ORFWorker.obj
 0003:000013fb       _piecewise_construct       100433fb     moc_ORFWorker.obj
 0003:000013fc       _taskLog                   100433fc     moc_ORFWorker.obj
 0003:00001404       _algoLog                   10043404     moc_ORFWorker.obj
 0003:0000140c       _userActLog                1004340c     moc_ORFWorker.obj
 0003:00001414       _ioLog                     10043414     moc_ORFWorker.obj
 0003:0000141c       _coreLog                   1004341c     moc_ORFWorker.obj
 0003:00001424       _uiLog                     10043424     moc_ORFWorker.obj
 0003:0000142c       _scriptLog                 1004342c     moc_ORFWorker.obj
 0003:00001434       _perfLog                   10043434     moc_ORFWorker.obj
 0003:0000143c       _cmdLog                    1004343c     moc_ORFWorker.obj
 0003:00001448       ___proc_attached           10043448     MSVCRT:crtdll.obj
 0003:00001450       _GS_ExceptionRecord        10043450     MSVCRT:gs_report.obj
 0003:000014a0       _GS_ContextRecord          100434a0     MSVCRT:gs_report.obj
 0003:0000176c       _DebuggerWasPresent        1004376c     MSVCRT:gs_report.obj
 0004:00000060       $R000000                   10044060     * linker generated manifest res *

 Exports

  ordinal    name

        1    _ugene_plugin_init
               exported name: ugene_plugin_init
